 CryAnimation

 Timestamp is 5036d291 (Fri Aug 24 03:02:09 2012)

 Preferred load address is 31500000

 Start         Length     Name                   Class
 0001:00000000 0010bf1aH .text                   CODE
 0001:0010bf20 0000058dH .text$yc                CODE
 0001:0010c4b0 00000585H .text$yd                CODE
 0002:00000000 00000164H .idata$5                DATA
 0002:00000164 00000004H .CRT$XCA                DATA
 0002:00000168 0000006cH .CRT$XCU                DATA
 0002:000001d4 00000004H .CRT$XCZ                DATA
 0002:000001d8 00000004H .CRT$XIA                DATA
 0002:000001dc 00000004H .CRT$XIAA               DATA
 0002:000001e0 00000004H .CRT$XIC                DATA
 0002:000001e4 00000004H .CRT$XIZ                DATA
 0002:000001f0 0000cbe0H .rdata                  DATA
 0002:0000cdd0 00000057H .rdata$debug            DATA
 0002:0000ce30 00000004H .rdata$sxdata           DATA
 0002:0000ce34 00000004H .rtc$IAA                DATA
 0002:0000ce38 00000004H .rtc$IZZ                DATA
 0002:0000ce3c 00000004H .rtc$TAA                DATA
 0002:0000ce40 00000004H .rtc$TZZ                DATA
 0002:0000ce48 00000064H .xdata$x                DATA
 0002:0000ceac 0000003cH .idata$2                DATA
 0002:0000cee8 00000014H .idata$3                DATA
 0002:0000cefc 00000164H .idata$4                DATA
 0002:0000d060 0000058eH .idata$6                DATA
 0002:0000d5f0 00000076H .edata                  DATA
 0003:00000000 000023e0H .data                   DATA
 0003:000023e0 0000b28cH .bss                    DATA
 0004:00000000 00000004H .tls$                   DATA
 0005:00000000 00000058H .rsrc$01                DATA
 0005:00000060 00000248H .rsrc$02                DATA

  Address         Publics by Value              Rva+Base       Lib:Object

 0000:00000000       __except_list              00000000     <absolute>
 0000:00000001       ___safe_se_handler_count   00000001     <absolute>
 0000:00009876       __fltused                  00009876     <absolute>
 0000:00009876       __ldused                   00009876     <absolute>
 0000:00000000       ___ImageBase               31500000     <linker-defined>
 0001:00000000       ??_GIMemReplay@@UAEPAXI@Z  31501000 f i AnimEventList.obj
 0001:00000000       ??_ECDummyMemReplay@@UAEPAXI@Z 31501000 f i AnimEventList.obj
 0001:00000000       ??_EIMemReplay@@UAEPAXI@Z  31501000 f i AnimEventList.obj
 0001:00000000       ??_GCDummyMemReplay@@UAEPAXI@Z 31501000 f i AnimEventList.obj
 0001:00000030       ?EnterScope@CDummyMemReplay@@UAE_NW4Class@EMemReplayAllocClass@@GH@Z 31501030 f i AnimEventList.obj
 0001:00000040       ?AddContextV@CDummyMemReplay@@UAEXHIPBDPAD@Z 31501040 f i AnimEventList.obj
 0001:00000040       ?MarkBucket@CDummyMemReplay@@UAEXHIPAXI@Z 31501040 f i AnimEventList.obj
 0001:00000040       ?SetParamVec3@CFacialEffector@@UAEXW4EFacialEffectorParam@@U?$Vec3_tpl@M@@@Z 31501040 f i FaceEffector.obj
 0001:00000040       ?ExitScope_Realloc@CDummyMemReplay@@UAEXIIII@Z 31501040 f i AnimEventList.obj
 0001:00000050       ?UnregisterContainer@CDummyMemReplay@@UAEXPBX@Z 31501050 f i AnimEventList.obj
 0001:00000050       ?StartOnCommandLine@CDummyMemReplay@@UAEXPBD@Z 31501050 f i AnimEventList.obj
 0001:00000050       ?GetMemoryUsage@CControllerOptNonVirtual@@UBEXPAVICrySizer@@@Z 31501050 f i LoaderDBA.obj
 0001:00000050       ?GetMemoryUsage@IPositionController@@UBEXPAVICrySizer@@@Z 31501050 f i LoaderTCB.obj
 0001:00000050       ?ProcessAttachment@CAttachmentSKIN@@UAEXPAUIAttachment@@@Z 31501050 f i Attachment.obj
 0001:00000050       ?CreateDecal@CCharInstance@@UAEXAAUCryEngineDecalInfo@@@Z 31501050 f i CharacterInstance.obj
 0001:00000050       ?GetMemoryUsage@IRotationController@@UBEXPAVICrySizer@@@Z 31501050 f i LoaderTCB.obj
 0001:00000050       ?ExitScope_Free@CDummyMemReplay@@UAEXI@Z 31501050 f i AnimEventList.obj
 0001:00000050       ?GetInfo@CDummyMemReplay@@UAEXAAUCryReplayInfo@@@Z 31501050 f i AnimEventList.obj
 0001:00000050       ?ProcessAttachment@CCGFAttachment@@UAEXPAUIAttachment@@@Z 31501050 f i AttachmentManager.obj
 0001:00000050       ?SetAttRelativeDefault@CAttachmentSKIN@@UAEXABU?$QuatT_tpl@M@@@Z 31501050 f i Attachment.obj
 0001:00000050       ?Free@CPool@Memory@@UAEXPAX@Z 31501050 f i Pool.obj
 0001:00000050       ?ProcessAttachment@CAttachmentFACE@@UAEXPAUIAttachment@@@Z 31501050 f i AttachmentManager.obj
 0001:00000050       ?ProcessAttachment@CAttachmentBONE@@UAEXPAUIAttachment@@@Z 31501050 f i AttachmentManager.obj
 0001:00000050       ?AddSizerTree@CDummyMemReplay@@UAEXPBD@Z 31501050 f i AnimEventList.obj
 0001:00000050       ?RemoveAllocReference@CDummyMemReplay@@UAEXPAX@Z 31501050 f i AnimEventList.obj
 0001:00000050       ?SetAttAbsoluteDefault@CAttachmentSKIN@@UAEXABU?$QuatT_tpl@M@@@Z 31501050 f i Attachment.obj
 0001:00000050       ?AddLabel@CDummyMemReplay@@UAEXPBD@Z 31501050 f i AnimEventList.obj
 0001:00000060       ?AddContext@CDummyMemReplay@@UAEXHIPBD@Z 31501060 f i AnimEventList.obj
 0001:00000060       ?AllocUsage@CDummyMemReplay@@UAEXW4Class@EMemReplayAllocClass@@II@Z 31501060 f i AnimEventList.obj
 0001:00000060       ?ExitScope_Alloc@CDummyMemReplay@@UAEXIII@Z 31501060 f i AnimEventList.obj
 0001:00000060       ?RegisterFixedAddressRange@CDummyMemReplay@@UAEXPAXIPBD@Z 31501060 f i AnimEventList.obj
 0001:00000070       ?MarkPool@CDummyMemReplay@@UAEXHIPAXIPBD@Z 31501070 f i AnimEventList.obj
 0001:00000070       ?GetRandomPos@CModelMesh@@QAEXPAUIRenderMesh@@PAU?$DualQuat_tpl@M@@AAURandomPos@@AAUGeomQuery@@W4EGeomForm@@@Z 31501070 f i ModelMesh.obj
 0001:00000080       ?AddTexturePoolContext@CDummyMemReplay@@UAEXPAXHHHPBDI@Z 31501080 f i AnimEventList.obj
 0001:00000090       ?alloc@StandardAlloc@NAlloc@@SAPAXAAI_NH@Z 31501090 f i AnimEventList.obj
 0001:00000110       ??0?$CryStringT@D@@QAE@ABV0@@Z 31501110 f i AnimEventList.obj
 0001:00000140       ?_Free@?$CryStringT@D@@IAEXXZ 31501140 f i AnimEventList.obj
 0001:00000180       ?GetByIndex@CAnimEventList@@UBEABVCAnimEventData@@I@Z 31501180 f   AnimEventList.obj
 0001:00000180       ?GetByIndex@CAnimEventList@@UAEAAVCAnimEventData@@I@Z 31501180 f   AnimEventList.obj
 0001:00000190       ?CryGetIMemReplay@@YAPAUIMemReplay@@XZ 31501190 f i AnimEventList.obj
 0001:000001f0       ??1XmlString@@QAE@XZ       315011f0 f i AnimEventLoader.obj
 0001:000001f0       ??1?$CryStringT@D@@QAE@XZ  315011f0 f i AnimEventList.obj
 0001:00000220       ??0CAnimEventData@@QAE@ABV0@@Z 31501220 f i AnimEventList.obj
 0001:000002c0       ??4CAnimEventData@@QAEAAV0@ABV0@@Z 315012c0 f i AnimEventList.obj
 0001:00000400       ?init@?$DynArray@VCAnimEventData@@HU?$SmallDynStorage@VCAnimEventData@@HUStandardAlloc@NAlloc@@@NArray@@@@KAPAVCAnimEventData@@U?$Array@VCAnimEventData@@HU?$ArrayStorage@VCAnimEventData@@H@NArray@@@@ABV2@@Z 31501400 f i AnimEventList.obj
 0001:000004e0       ??1CAnimEventData@@QAE@XZ  315014e0 f i AnimEventList.obj
 0001:00000590       ?GetAllocSize@CAnimEventList@@QBEIXZ 31501590 f   AnimEventList.obj
 0001:00000690       ??$AddObject@VCAnimEventData@@HU?$SmallDynStorage@VCAnimEventData@@HUStandardAlloc@NAlloc@@@NArray@@@ICrySizer@@QAEXABU?$DynArray@VCAnimEventData@@HU?$SmallDynStorage@VCAnimEventData@@HUStandardAlloc@NAlloc@@@NArray@@@@@Z 31501690 f i AnimEventList.obj
 0001:000007f0       ??$move_init@VCAnimEventData@@@NArray@@YAXPAVCAnimEventData@@0I@Z 315017f0 f i AnimEventList.obj
 0001:00000840       ?GetMemoryUsage@CAnimEventList@@QBEXPAVICrySizer@@@Z 31501840 f   AnimEventList.obj
 0001:00000860       ?resize_raw@?$SmallDynStorage@VCAnimEventData@@HUStandardAlloc@NAlloc@@@NArray@@QAEXHH_N@Z 31501860 f i AnimEventList.obj
 0001:000009c0       ?clear@?$DynArray@VCAnimEventData@@HU?$SmallDynStorage@VCAnimEventData@@HUStandardAlloc@NAlloc@@@NArray@@@@QAEXXZ 315019c0 f i AnimEventList.obj
 0001:00000a30       ?erase@?$DynArray@VCAnimEventData@@HU?$SmallDynStorage@VCAnimEventData@@HUStandardAlloc@NAlloc@@@NArray@@@@QAEPAVCAnimEventData@@PAV2@0@Z 31501a30 f i AnimEventList.obj
 0001:00000ad0       ??1?$DynArray@VCAnimEventData@@HU?$SmallDynStorage@VCAnimEventData@@HUStandardAlloc@NAlloc@@@NArray@@@@QAE@XZ 31501ad0 f i AnimEventList.obj
 0001:00000b30       ?expand_raw@?$DynArray@VCAnimEventData@@HU?$SmallDynStorage@VCAnimEventData@@HUStandardAlloc@NAlloc@@@NArray@@@@IAEPAVCAnimEventData@@PAV2@H@Z 31501b30 f i AnimEventList.obj
 0001:00000bc0       ??0CAnimEventList@@QAE@XZ  31501bc0 f   AnimEventList.obj
 0001:00000c10       ??1CAnimEventList@@UAE@XZ  31501c10 f   AnimEventList.obj
 0001:00000c30       ?Clear@CAnimEventList@@UAEXXZ 31501c30 f   AnimEventList.obj
 0001:00000c40       ??_GCAnimEventList@@UAEPAXI@Z 31501c40 f i AnimEventList.obj
 0001:00000c40       ??_ECAnimEventList@@UAEPAXI@Z 31501c40 f i AnimEventList.obj
 0001:00000c70       ?Remove@CAnimEventList@@UAEXI@Z 31501c70 f   AnimEventList.obj
 0001:00000c90       ?Append@CAnimEventList@@UAEXABVCAnimEventData@@@Z 31501c90 f   AnimEventList.obj
 0001:00000cd0       ?ClearBinding@CAttachmentSKIN@@UAEXXZ 31501cd0 f   Attachment.obj
 0001:00000cf0       ?ClearBinding@CAttachmentFACE@@UAEXXZ 31501cf0 f   Attachment.obj
 0001:00000cf0       ?ClearBinding@CAttachmentBONE@@UAEXXZ 31501cf0 f   Attachment.obj
 0001:00000d40       ?GetPendulumParams2@SAttachmentPendulum@@QAEXAAHAAC1AAM22AAU?$Vec3_tpl@M@@3@Z 31501d40 f   Attachment.obj
 0001:00000e20       ?CryFatalError@@YAXPBDZZ   31501e20 f i Attachment.obj
 0001:00000e90       ?CryLogAlways@@YAXPBDZZ    31501e90 f i Attachment.obj
 0001:00000ec0       ??_EIAttachment@@UAEPAXI@Z 31501ec0 f i Attachment.obj
 0001:00000ec0       ??_GIAttachment@@UAEPAXI@Z 31501ec0 f i Attachment.obj
 0001:00000ef0       ??_GIAttachmentSkin@@UAEPAXI@Z 31501ef0 f i Attachment.obj
 0001:00000ef0       ??_EIAttachmentSkin@@UAEPAXI@Z 31501ef0 f i Attachment.obj
 0001:00000f20       ?SetBoneName@CAttachmentBONE@@UAEIPBD@Z 31501f20 f   Attachment.obj
 0001:00000fb0       ??4?$OBB_tpl@M@@QAEAAU0@ABU0@@Z 31501fb0 f i Attachment.obj
 0001:00001020       ?AddBinding@CAttachmentBONE@@UAEIPAUIAttachmentObject@@V?$_smart_ptr@UISkin@@@@I@Z 31502020 f   Attachment.obj
 0001:00001020       ?AddBinding@CAttachmentFACE@@UAEIPAUIAttachmentObject@@V?$_smart_ptr@UISkin@@@@I@Z 31502020 f   Attachment.obj
 0001:000010a0       ?ToVec3@Vec3f16@@QBE?AU?$Vec3_tpl@M@@XZ 315020a0 f i Attachment.obj
 0001:000011e0       ?ToVec2@Vec2f16@@QBE?AU?$Vec2_tpl@M@@XZ 315021e0 f i Attachment.obj
 0001:000012c0       ?Draw2dLabel@IRenderer@@QAAXMMMPBM_NPBDZZ 315022c0 f i Attachment.obj
 0001:00001390       ??0?$QuatT_tpl@M@@QAE@ABU0@@Z 31502390 f i Attachment.obj
 0001:000013d0       ?GetAttWorldAbsolute@CAttachmentSKIN@@UBE?BU?$QuatTS_tpl@M@@XZ 315023d0 f   Attachment.obj
 0001:00001430       ?AlignBoneAttachment@CAttachmentBONE@@UAEXXZ 31502430 f   Attachment.obj
 0001:00001500       ?Serialize@CAttachmentFACE@@UAEXV?$CSerializeWrapper@UISerialize@@@@@Z 31502500 f   Attachment.obj
 0001:00001500       ?Serialize@CAttachmentBONE@@UAEXV?$CSerializeWrapper@UISerialize@@@@@Z 31502500 f   Attachment.obj
 0001:00001500       ?Serialize@CAttachmentSKIN@@UAEXV?$CSerializeWrapper@UISerialize@@@@@Z 31502500 f   Attachment.obj
 0001:00001590       ?GetAttWorldAbsolute@CAttachmentBONE@@UBE?BU?$QuatTS_tpl@M@@XZ 31502590 f   Attachment.obj
 0001:00001590       ?GetAttWorldAbsolute@CAttachmentFACE@@UBE?BU?$QuatTS_tpl@M@@XZ 31502590 f   Attachment.obj
 0001:00001810       ?SetPendulumParams2@SAttachmentPendulum@@QAEXHCCMMMU?$Vec3_tpl@M@@0@Z 31502810 f   Attachment.obj
 0001:00001d30       ?GetModelMesh@CSkin@@QAEPAVCModelMesh@@I@Z 31502d30 f i Attachment.obj
 0001:00001d60       ?DrawWireframeStatic@CAttachmentSKIN@@UAEXABU?$Matrix34_tpl@M@@HI@Z 31502d60 f   Attachment.obj
 0001:00001dc0       ?InitRenderMeshsSW@CAttachmentSKIN@@QAEXXZ 31502dc0 f   Attachment.obj
 0001:00002320       ?ProjectAttachment@CAttachmentBONE@@UAEIXZ 31503320 f   Attachment.obj
 0001:00002770       ?SizeOfThis@CAttachmentBONE@@UAEIXZ 31503770 f   Attachment.obj
 0001:00002780       ?GetMemoryUsage@CAttachmentBONE@@UBEXPAVICrySizer@@@Z 31503780 f   Attachment.obj
 0001:000027c0       ?SizeOfThis@CAttachmentFACE@@UAEIXZ 315037c0 f   Attachment.obj
 0001:000027d0       ?GetMemoryUsage@CAttachmentFACE@@UBEXPAVICrySizer@@@Z 315037d0 f   Attachment.obj
 0001:00002810       ?UpdatePendulumPhysics@SAttachmentPendulum@@QAEXXZ 31503810 f   Attachment.obj
 0001:00005ba0       ?set_size@?$SmallDynStorage@EHUStandardAlloc@NAlloc@@@NArray@@QAEXH@Z 31506ba0 f i Attachment.obj
 0001:00005ba0       ?set_size@?$SmallDynStorage@_NHUStandardAlloc@NAlloc@@@NArray@@QAEXH@Z 31506ba0 f i CharacterInstance.obj
 0001:00005ba0       ?set_size@?$SmallDynStorage@DHUStandardAlloc@NAlloc@@@NArray@@QAEXH@Z 31506ba0 f i LoaderCHR.obj
 0001:00005c20       ?resize_raw@?$SmallDynStorage@EHUStandardAlloc@NAlloc@@@NArray@@QAEXHH_N@Z 31506c20 f i Attachment.obj
 0001:00005d60       ?SizeOfThis@CAttachmentSKIN@@UAEIXZ 31506d60 f   Attachment.obj
 0001:00005db0       ?UpdateLocation@CAttachmentBONE@@UAEXXZ 31506db0 f   Attachment.obj
 0001:00006100       ?DrawAttachment@CAttachmentBONE@@UAEXAAUSRendParams@@ABUSRenderingPassInfo@@ABU?$Matrix34_tpl@M@@M@Z 31507100 f   Attachment.obj
 0001:000072c0       ?ProjectAttachment@CAttachmentFACE@@UAEIXZ 315082c0 f   Attachment.obj
 0001:00008810       ?UpdateLocation@CAttachmentFACE@@UAEXXZ 31509810 f   Attachment.obj
 0001:0000a560       ?DrawAttachment@CAttachmentFACE@@UAEXAAUSRendParams@@ABUSRenderingPassInfo@@ABU?$Matrix34_tpl@M@@M@Z 3150b560 f   Attachment.obj
 0001:0000b720       ?expand_raw@?$DynArray@EHU?$SmallDynStorage@EHUStandardAlloc@NAlloc@@@NArray@@@@IAEPAEPAEH@Z 3150c720 f i Attachment.obj
 0001:0000b7a0       ??$AddObject@_NHU?$SmallDynStorage@_NHUStandardAlloc@NAlloc@@@NArray@@@ICrySizer@@QAEXABU?$DynArray@_NHU?$SmallDynStorage@_NHUStandardAlloc@NAlloc@@@NArray@@@@@Z 3150c7a0 f i CharacterInstance.obj
 0001:0000b7a0       ??$AddObject@EHU?$SmallDynStorage@EHUStandardAlloc@NAlloc@@@NArray@@@ICrySizer@@QAEXABU?$DynArray@EHU?$SmallDynStorage@EHUStandardAlloc@NAlloc@@@NArray@@@@@Z 3150c7a0 f i Attachment.obj
 0001:0000b870       ?GetMemoryUsage@CAttachmentSKIN@@UBEXPAVICrySizer@@@Z 3150c870 f   Attachment.obj
 0001:0000b8b0       ??1CAttachmentSKIN@@UAE@XZ 3150c8b0 f   Attachment.obj
 0001:0000ba40       ?AddRef@CAttachmentSKIN@@UAEXXZ 3150ca40 f i Attachment.obj
 0001:0000ba50       ?Release@CAttachmentSKIN@@UAEXXZ 3150ca50 f i Attachment.obj
 0001:0000ba60       ?GetType@CAttachmentSKIN@@UBEIXZ 3150ca60 f i Attachment.obj
 0001:0000ba60       ?GetFormat@?$CKeyTimesInformation@EUByteEncoder@@@@UAEIXZ 3150ca60 f i ControllerPQ.obj
 0001:0000ba60       ?GetSplineType@CFacialAnimChannelInterpolator@@UAE?AW4ESplineType@@XZ 3150ca60 f i FaceAnimSequence.obj
 0001:0000ba60       ?GetDataRawSize@?$CKeyTimesInformationStartStop@EUByteStartStopEncoder@@@@UAEIXZ 3150ca60 f i ControllerPQ.obj
 0001:0000ba60       ?GetType@CFacialMorphTarget@@UAE?AW4EFacialEffectorType@@XZ 3150ca60 f i FaceEffectorLibrary.obj
 0001:0000ba60       ?GetFormat@?$CTrackDataStorageInt@U?$Vec3_tpl@M@@UNoCompressVec3@@VITrackPositionStorage@@@@UAEIXZ 3150ca60 f i ControllerPQ.obj
 0001:0000ba60       ?GetAttachmentType@CSKELAttachment@@UAE?AW4EType@IAttachmentObject@@XZ 3150ca60 f i AttachmentManager.obj
 0001:0000ba70       ?SetForceSkeletonUpdate@CSkeletonPose@@UAEXH@Z 3150ca70 f i SkeletonPose.obj
 0001:0000ba70       ?SetFlags@CAttachmentBONE@@UAEXI@Z 3150ca70 f i AttachmentManager.obj
 0001:0000ba70       ?SetFlags@CAttachmentSKIN@@UAEXI@Z 3150ca70 f i Attachment.obj
 0001:0000ba70       ?SetFlags@CAttachmentFACE@@UAEXI@Z 3150ca70 f i AttachmentManager.obj
 0001:0000ba80       ?HideAttachment@CAttachmentFACE@@UAEXI@Z 3150ca80 f i AttachmentManager.obj
 0001:0000ba80       ?HideAttachment@CAttachmentSKIN@@UAEXI@Z 3150ca80 f i Attachment.obj
 0001:0000ba80       ?HideAttachment@CAttachmentBONE@@UAEXI@Z 3150ca80 f i AttachmentManager.obj
 0001:0000baa0       ?IsAttachmentHidden@CAttachmentFACE@@UAEIXZ 3150caa0 f i AttachmentManager.obj
 0001:0000baa0       ?IsAttachmentHidden@CAttachmentBONE@@UAEIXZ 3150caa0 f i AttachmentManager.obj
 0001:0000baa0       ?IsAttachmentHidden@CAttachmentSKIN@@UAEIXZ 3150caa0 f i Attachment.obj
 0001:0000bab0       ?GetAttAbsoluteDefault@CAttachmentSKIN@@UBEABU?$QuatT_tpl@M@@XZ 3150cab0 f i Attachment.obj
 0001:0000bab0       ?GetAttRelativeDefault@CAttachmentSKIN@@UBEABU?$QuatT_tpl@M@@XZ 3150cab0 f i Attachment.obj
 0001:0000bab0       ?GetAttModelRelative@CAttachmentSKIN@@UBEABU?$QuatT_tpl@M@@XZ 3150cab0 f i Attachment.obj
 0001:0000bac0       ?RemoveContext@CDummyMemReplay@@UAEXXZ 3150cac0 f i AnimEventList.obj
 0001:0000bac0       ?Synchronize@CGroundAlignment@@UAEXXZ 3150cac0 f i GroundAlignment.obj
 0001:0000bac0       ?AddRef@?$CTrackDataStorage@U?$Quat_tpl@M@@UNoCompressQuat@@VITrackRotationStorage@@@@UAEXXZ 3150cac0 f i ControllerPQ.obj
 0001:0000bac0       ?Synchronize@CPoseAlignerChain@@UAEXXZ 3150cac0 f i PoseAlignerChain.obj
 0001:0000bac0       ?Stop@CDummyMemReplay@@UAEXXZ 3150cac0 f i AnimEventList.obj
 0001:0000bac0       ?AddScreenshot@CDummyMemReplay@@UAEXXZ 3150cac0 f i AnimEventList.obj
 0001:0000bac0       ?Synchronize@CFeetPoseStore@@UAEXXZ 3150cac0 f i FeetLock.obj
 0001:0000bac0       ?LockResources@CharacterManager@@UAEXXZ 3150cac0 f i CharacterManager.obj
 0001:0000bac0       ?AddRef@?$CTrackDataStorage@U?$Vec3_tpl@M@@UNoCompressVec3@@VITrackPositionStorage@@@@UAEXXZ 3150cac0 f i ControllerPQ.obj
 0001:0000bac0       ?AddLabelFmt@CDummyMemReplay@@UAAXPBDZZ 3150cac0 f i AnimEventList.obj
 0001:0000bac0       ?AddRef@?$CTrackDataStorage@U?$Quat_tpl@M@@USmallTree48BitQuat@@VITrackRotationStorage@@@@UAEXXZ 3150cac0 f i ControllerPQ.obj
 0001:0000bac0       ?Synchronize@CPoseMatching@@UAEXXZ 3150cac0 f i PoseMatching.obj
 0001:0000bac0       ?UpdateLocation@CAttachmentSKIN@@UAEXXZ 3150cac0 f i Attachment.obj
 0001:0000bac0       ?InitSpuControllerLookupTable@@YAXABU?$DynArray@IHU?$SmallDynStorage@IHUStandardAlloc@NAlloc@@@NArray@@@@@Z 3150cac0 f i SkeletonAnim.obj
 0001:0000bac0       ?AlignBoneAttachment@CAttachmentSKIN@@UAEXXZ 3150cac0 f i Attachment.obj
 0001:0000bac0       ?DumpStats@CDummyMemReplay@@UAEXXZ 3150cac0 f i AnimEventList.obj
 0001:0000bac0       ?ExitScope@CDummyMemReplay@@UAEXXZ 3150cac0 f i AnimEventList.obj
 0001:0000bac0       ?sp_enable_shared_from_this@detail@boost@@YAXZZ 3150cac0 f i OperatorQueue.obj
 0001:0000bac0       ?AddRef@CControllerOptNonVirtual@@UAEXXZ 3150cac0 f i LoaderDBA.obj
 0001:0000bac0       ?Synchronize@CRecoil@PoseModifier@@UAEXXZ 3150cac0 f i Recoil.obj
 0001:0000bac0       ?AddFrameStart@CDummyMemReplay@@UAEXXZ 3150cac0 f i AnimEventList.obj
 0001:0000bac0       ?Synchronize@CLimbIk@@UAEXXZ 3150cac0 f i LimbIk.obj
 0001:0000bac0       ?Synchronize@CFeetPoseRestore@@UAEXXZ 3150cac0 f i FeetLock.obj
 0001:0000bac0       ?DumpSymbols@CDummyMemReplay@@UAEXXZ 3150cac0 f i AnimEventList.obj
 0001:0000bac0       ?AddRef@?$CTrackDataStorage@U?$Quat_tpl@M@@USmallTree64BitQuat@@VITrackRotationStorage@@@@UAEXXZ 3150cac0 f i ControllerPQ.obj
 0001:0000bac0       ?AddRef@?$CTrackDataStorage@U?$Quat_tpl@M@@USmallTree64BitExtQuat@@VITrackRotationStorage@@@@UAEXXZ 3150cac0 f i ControllerPQ.obj
 0001:0000bac0       ?Update@CPool@Memory@@UAEXXZ 3150cac0 f i Pool.obj
 0001:0000bac0       ?Release@CControllerOptNonVirtual@@UAEXXZ 3150cac0 f i LoaderDBA.obj
 0001:0000bac0       ?Flush@CDummyMemReplay@@UAEXXZ 3150cac0 f i AnimEventList.obj
 0001:0000bac0       ?AlignBoneAttachment@CAttachmentFACE@@UAEXXZ 3150cac0 f i AttachmentManager.obj
 0001:0000bac0       ?UnlockResources@CharacterManager@@UAEXXZ 3150cac0 f i CharacterManager.obj
 0001:0000bac0       ?ReloadAllModels@CharacterManager@@UAEXXZ 3150cac0 f i CharacterManager.obj
 0001:0000bad0       ?SetPendulumParams@CAttachmentSKIN@@UAEXHCCMMMU?$Vec3_tpl@M@@0@Z 3150cad0 f i Attachment.obj
 0001:0000bae0       ?GetIVertexAnimation@CAttachmentSKIN@@UAEPAUIVertexAnimation@@XZ 3150cae0 f i Attachment.obj
 0001:0000baf0       ??_ECAttachmentSKIN@@W3AEPAXI@Z 3150caf0 f i Attachment.obj
 0001:0000bb00       ?AddRef@CAttachmentSKIN@@W3AEXXZ 3150cb00 f i Attachment.obj
 0001:0000bb10       ?Release@CAttachmentSKIN@@W3AEXXZ 3150cb10 f i Attachment.obj
 0001:0000bb20       ?GetPendulumParams@CAttachmentSKIN@@UAEXAAHAAC1AAM22AAU?$Vec3_tpl@M@@3@Z 3150cb20 f i Attachment.obj
 0001:0000bb80       ?_AllocData@?$CryStringT@D@@IAEXI@Z 3150cb80 f i Attachment.obj
 0001:0000bbd0       ?_Assign@?$CryStringT@D@@IAEXPBDI@Z 3150cbd0 f i Attachment.obj
 0001:0000bc80       ?_MakeUnique@?$CryStringT@D@@IAEXXZ 3150cc80 f i Attachment.obj
 0001:0000bd20       ??4?$CryStringT@D@@QAEAAV0@PBD@Z 3150cd20 f i Attachment.obj
 0001:0000bd60       ?append@?$CryStringT@D@@QAEAAV1@ID@Z 3150cd60 f i Attachment.obj
 0001:0000be10       ?GetMemoryUsage@CAttachmentSKIN@@W3BEXPAVICrySizer@@@Z 3150ce10 f i Attachment.obj
 0001:0000be20       ?clear@?$CryStringT@D@@QAEXXZ 3150ce20 f i Attachment.obj
 0001:0000be80       ?ReName@CAttachmentFACE@@UAEIPBDI@Z 3150ce80 f i AttachmentManager.obj
 0001:0000be80       ?ReName@CAttachmentSKIN@@UAEIPBDI@Z 3150ce80 f i Attachment.obj
 0001:0000be80       ?ReName@CAttachmentBONE@@UAEIPBDI@Z 3150ce80 f i AttachmentManager.obj
 0001:0000bed0       ??_ECAttachmentSKIN@@UAEPAXI@Z 3150ced0 f i Attachment.obj
 0001:0000bed0       ??_GCAttachmentSKIN@@UAEPAXI@Z 3150ced0 f i Attachment.obj
 0001:0000bf00       ?resize@?$DynArray@EHU?$SmallDynStorage@EHUStandardAlloc@NAlloc@@@NArray@@@@QAEXH@Z 3150cf00 f i Attachment.obj
 0001:0000bf40       ?AddBinding@CAttachmentSKIN@@UAEIPAUIAttachmentObject@@V?$_smart_ptr@UISkin@@@@I@Z 3150cf40 f   Attachment.obj
 0001:0000c1c0       ?GetStats@CControllerDefragHeap@@QAE?AUStats@1@XZ 3150d1c0 f   ControllerDefragHeap.obj
 0001:0000c200       ?SyncCopy@CControllerDefragHeap@@EAEXPAXIII@Z 3150d200 f   ControllerDefragHeap.obj
 0001:0000c210       ?__stl_throw_length_error@stlpmtx_std@@YAXPBD@Z 3150d210 f i ControllerDefragHeap.obj
 0001:0000c230       ??_GIDefragAllocatorPolicy@@MAEPAXI@Z 3150d230 f i ControllerDefragHeap.obj
 0001:0000c230       ??_EIDefragAllocatorPolicy@@MAEPAXI@Z 3150d230 f i ControllerDefragHeap.obj
 0001:0000c260       ?UsableSize@CControllerDefragHeap@@QAEIVCControllerDefragHdl@@@Z 3150d260 f   ControllerDefragHeap.obj
 0001:0000c290       ?CancelCopy@CControllerDefragHeap@@EAEXIPAX_N@Z 3150d290 f   ControllerDefragHeap.obj
 0001:0000c2d0       ??0CFrameProfiler@@QAE@PAUISystem@@PBDW4EProfiledSubsystem@@@Z 3150d2d0 f i ControllerDefragHeap.obj
 0001:0000c370       ?Relocate@CControllerDefragHeap@@EAEXIPAXIII@Z 3150d370 f   ControllerDefragHeap.obj
 0001:0000c450       ??$unique@PAI@stlpmtx_std@@YAPAIPAI0@Z 3150d450 f i ControllerDefragHeap.obj
 0001:0000c4b0       ?allocate@?$_STLP_alloc_proxy@PAV?$_smart_ptr@VCFacialEffector@@@@V1@V?$allocator@V?$_smart_ptr@VCFacialEffector@@@@@stlpmtx_std@@@priv@stlpmtx_std@@QAEPAV?$_smart_ptr@VCFacialEffector@@@@IAAI@Z 3150d4b0 f i FaceEffectorLibrary.obj
 0001:0000c4b0       ?allocate@?$_STLP_alloc_proxy@PAHHV?$allocator@H@stlpmtx_std@@@priv@stlpmtx_std@@QAEPAHIAAI@Z 3150d4b0 f i ControllerDefragHeap.obj
 0001:0000c4b0       ?allocate@?$_STLP_alloc_proxy@PAPAXPAXV?$allocator@PAX@stlpmtx_std@@@priv@stlpmtx_std@@QAEPAPAXIAAI@Z 3150d4b0 f i LoaderSKIN.obj
 0001:0000c500       ??$__unguarded_insertion_sort_aux@PAIIU?$less@I@stlpmtx_std@@@priv@stlpmtx_std@@YAXPAI00U?$less@I@1@@Z 3150d500 f i ControllerDefragHeap.obj
 0001:0000c540       ??1CControllerDefragHeap@@UAE@XZ 3150d540 f   ControllerDefragHeap.obj
 0001:0000c5b0       ?IncreaseRange@CControllerDefragHeap@@AAE_NII@Z 3150d5b0 f   ControllerDefragHeap.obj
 0001:0000c670       ?DecreaseRange@CControllerDefragHeap@@AAEXII@Z 3150d670 f   ControllerDefragHeap.obj
 0001:0000c6d0       ??$__insertion_sort@PAIIU?$less@I@stlpmtx_std@@@priv@stlpmtx_std@@YAXPAI00U?$less@I@1@@Z 3150d6d0 f i ControllerDefragHeap.obj
 0001:0000c750       ??$__make_heap@PAIU?$less@I@stlpmtx_std@@IH@stlpmtx_std@@YAXPAI0U?$less@I@0@0PAH@Z 3150d750 f i ControllerDefragHeap.obj
 0001:0000c800       ??_GCControllerDefragHeap@@UAEPAXI@Z 3150d800 f i ControllerDefragHeap.obj
 0001:0000c800       ??_ECControllerDefragHeap@@UAEPAXI@Z 3150d800 f i ControllerDefragHeap.obj
 0001:0000c830       ?AllocPinned@CControllerDefragHeap@@QAE?AVCControllerDefragHdl@@IPAVIControllerRelocatableChain@@@Z 3150d830 f   ControllerDefragHeap.obj
 0001:0000ca50       ?Free@CControllerDefragHeap@@QAEXVCControllerDefragHdl@@@Z 3150da50 f   ControllerDefragHeap.obj
 0001:0000cb50       ?BeginCopy@CControllerDefragHeap@@EAEIPAXIIIPAUIDefragAllocatorCopyNotification@@@Z 3150db50 f   ControllerDefragHeap.obj
 0001:0000cc70       ??0CControllerDefragHeap@@QAE@XZ 3150dc70 f   ControllerDefragHeap.obj
 0001:0000cd00       ??$sort_heap@PAIU?$less@I@stlpmtx_std@@@stlpmtx_std@@YAXPAI0U?$less@I@0@@Z 3150dd00 f i ControllerDefragHeap.obj
 0001:0000cda0       ??$__partial_sort@PAIIU?$less@I@stlpmtx_std@@@priv@stlpmtx_std@@YAXPAI000U?$less@I@1@@Z 3150dda0 f i ControllerDefragHeap.obj
 0001:0000ce70       ?Init@CControllerDefragHeap@@QAEXI@Z 3150de70 f   ControllerDefragHeap.obj
 0001:0000cf10       ??$__introsort_loop@PAIIHU?$less@I@stlpmtx_std@@@priv@stlpmtx_std@@YAXPAI00HU?$less@I@1@@Z 3150df10 f i ControllerDefragHeap.obj
 0001:0000cff0       ??$sort@PAI@stlpmtx_std@@YAXPAI0@Z 3150dff0 f i ControllerDefragHeap.obj
 0001:0000d070       ?UpdateInflight@CControllerDefragHeap@@AAEXH@Z 3150e070 f   ControllerDefragHeap.obj
 0001:0000d230       ?Update@CControllerDefragHeap@@QAEXXZ 3150e230 f   ControllerDefragHeap.obj
 0001:0000d310       ?Draw@DrawHelper@@YAXABUSegment@1@@Z 3150e310 f   DrawHelper.obj
 0001:0000d340       ?Draw@DrawHelper@@YAXABUSphere@1@@Z 3150e340 f   DrawHelper.obj
 0001:0000d370       ?Draw@DrawHelper@@YAXABUCylinder@1@@Z 3150e370 f   DrawHelper.obj
 0001:0000d3b0       ??$?DMM@@YA?AU?$Vec3_tpl@M@@ABU?$QuatT_tpl@M@@ABU0@@Z 3150e3b0 f i DrawHelper.obj
 0001:0000d4b0       ?DepthTest@DrawHelper@@YAX_N@Z 3150e4b0 f   DrawHelper.obj
 0001:0000d500       ?Frame@DrawHelper@@YAXABU?$Vec3_tpl@M@@000@Z 3150e500 f   DrawHelper.obj
 0001:0000d630       ?Frame@DrawHelper@@YAXABU?$Matrix34_tpl@M@@ABU?$Vec3_tpl@M@@@Z 3150e630 f   DrawHelper.obj
 0001:0000d710       ?BonePrism@DrawHelper@@YAXABU?$Vec3_tpl@M@@00U?$Color_tpl@E@@@Z 3150e710 f   DrawHelper.obj
 0001:0000ddf0       ?Frame@DrawHelper@@YAXABU?$QuatT_tpl@M@@ABU?$Vec3_tpl@M@@@Z 3150edf0 f   DrawHelper.obj
 0001:0000df80       ?Arrow@DrawHelper@@YAXABU?$QuatT_tpl@M@@ABU?$Vec3_tpl@M@@MU?$Color_tpl@E@@@Z 3150ef80 f   DrawHelper.obj
 0001:0000e780       ?CurvedArrow@DrawHelper@@YAXABU?$QuatT_tpl@M@@MMMMU?$Color_tpl@E@@@Z 3150f780 f   DrawHelper.obj
 0001:0000fa20       ?BonePrism@DrawHelper@@YAMU?$QuatT_tpl@M@@ABU?$Vec3_tpl@M@@U?$Color_tpl@E@@@Z 31510a20 f   DrawHelper.obj
 0001:000100a0       ?Pose@DrawHelper@@YAXABVCPoseData@Skeleton@@ABU?$QuatT_tpl@M@@U?$Color_tpl@E@@@Z 315110a0 f   DrawHelper.obj
 0001:00010930       ??4?$_smart_ptr@UIRenderMesh@@@@QAEAAV0@PAUIRenderMesh@@@Z 31511930 f i LoaderSKIN.obj
 0001:00010960       ??1CLoadingTimeProfiler@@QAE@XZ 31511960 f i LoaderSKIN.obj
 0001:00010980       ?CryLog@@YAXPBDZZ          31511980 f i LoaderSKIN.obj
 0001:000109b0       ?FixRanges@SMeshSubset@@QAEXPAG@Z 315119b0 f i LoaderSKIN.obj
 0001:000109f0       ?FindExtension@CryStringUtils@@YAPBDPBD@Z 315119f0 f i LoaderSKIN.obj
 0001:00010a30       ?Release@?$_i_reference_target@H@@UAEXXZ 31511a30 f i LoaderSKIN.obj
 0001:00010a60       ??1?$_smart_ptr@UIMaterial@@@@QAE@XZ 31511a60 f i LoaderSKIN.obj
 0001:00010a70       ??$move_init@UBoneWeights8@@@NArray@@YAXPAUBoneWeights8@@0I@Z 31511a70 f i LoaderSKIN.obj
 0001:00010ab0       ??$move_init@UMorphTargetVertex@@@NArray@@YAXPAUMorphTargetVertex@@0I@Z 31511ab0 f i LoaderSKIN.obj
 0001:00010af0       ??$fill@PAU?$Vec3_tpl@M@@U1@@stlpmtx_std@@YAXPAU?$Vec3_tpl@M@@0ABU1@@Z 31511af0 f i LoaderSKIN.obj
 0001:00010b30       ?IsValid@?$Vec3_tpl@M@@QBE_NXZ 31511b30 f i LoaderSKIN.obj
 0001:00010b70       ?IsOrthonormalRH@?$Matrix34_tpl@M@@QBEHM@Z 31511b70 f i LoaderSKIN.obj
 0001:00010db0       ?_AllocData@?$CryStackStringT@D$0CAA@@@QAEXI@Z 31511db0 f i LoaderSKIN.obj
 0001:00010e20       ?init@?$DynArray@U?$Vec3_tpl@M@@HU?$SmallDynStorage@U?$Vec3_tpl@M@@HUStandardAlloc@NAlloc@@@NArray@@@@KAPAU?$Vec3_tpl@M@@U?$Array@U?$Vec3_tpl@M@@HU?$ArrayStorage@U?$Vec3_tpl@M@@H@NArray@@@@PBU2@@Z 31511e20 f i LoaderSKIN.obj
 0001:00010e60       ?init@?$DynArray@U?$Quat_tpl@M@@HU?$SmallDynStorage@U?$Quat_tpl@M@@HUStandardAlloc@NAlloc@@@NArray@@@@KAPAU?$Quat_tpl@M@@U?$Array@U?$Quat_tpl@M@@HU?$ArrayStorage@U?$Quat_tpl@M@@H@NArray@@@@PBU2@@Z 31511e60 f i LoaderSKIN.obj
 0001:00010eb0       ?_Concatenate@?$CryStackStringT@D$0CAA@@@QAEXPBDI0I@Z 31511eb0 f i LoaderSKIN.obj
 0001:00010f20       ??$move_init@U?$Quat_tpl@M@@@NArray@@YAXPAU?$Quat_tpl@M@@0I@Z 31511f20 f i LoaderSKIN.obj
 0001:00011040       ??0CMemStatContextFormat@@QAA@W4Type@EMemStatContextTypes@@IPBDZZ 31512040 f i LoaderSKIN.obj
 0001:00011070       ??1CMemStatContextFormat@@QAE@XZ 31512070 f i LoaderSKIN.obj
 0001:00011080       ?assign@?$Array@U?$Vec3_tpl@M@@HU?$SmallDynStorage@U?$Vec3_tpl@M@@HUStandardAlloc@NAlloc@@@NArray@@@@QAEXU?$Array@$$CBU?$Vec3_tpl@M@@HU?$ArrayStorage@$$CBU?$Vec3_tpl@M@@H@NArray@@@@@Z 31512080 f i LoaderSKIN.obj
 0001:000110c0       ?assign@?$Array@U?$Quat_tpl@M@@HU?$SmallDynStorage@U?$Quat_tpl@M@@HUStandardAlloc@NAlloc@@@NArray@@@@QAEXU?$Array@$$CBU?$Quat_tpl@M@@HU?$ArrayStorage@$$CBU?$Quat_tpl@M@@H@NArray@@@@@Z 315120c0 f i LoaderSKIN.obj
 0001:00011120       ?init@?$DynArray@UBoneWeights8@@HU?$SmallDynStorage@UBoneWeights8@@HUStandardAlloc@NAlloc@@@NArray@@@@KAPAUBoneWeights8@@U?$Array@UBoneWeights8@@HU?$ArrayStorage@UBoneWeights8@@H@NArray@@@@PBU2@@Z 31512120 f i LoaderSKIN.obj
 0001:00011160       ?init@?$DynArray@V?$_smart_ptr@VIController@@@@HU?$SmallDynStorage@V?$_smart_ptr@VIController@@@@HUStandardAlloc@NAlloc@@@NArray@@@@KAPAV?$_smart_ptr@VIController@@@@U?$Array@V?$_smart_ptr@VIController@@@@HU?$ArrayStorage@V?$_smart_ptr@VIController@@@@H@NArray@@@@PBV2@@Z 31512160 f i CharacterManager.obj
 0001:00011160       ?init@?$DynArray@V?$_smart_ptr@UCMorphTarget@@@@HU?$SmallDynStorage@V?$_smart_ptr@UCMorphTarget@@@@HUStandardAlloc@NAlloc@@@NArray@@@@KAPAV?$_smart_ptr@UCMorphTarget@@@@U?$Array@V?$_smart_ptr@UCMorphTarget@@@@HU?$ArrayStorage@V?$_smart_ptr@UCMorphTarget@@@@H@NArray@@@@PBV2@@Z 31512160 f i LoaderSKIN.obj
 0001:000111a0       ?resize_raw@?$SmallDynStorage@UExtSkinVertex@@HUStandardAlloc@NAlloc@@@NArray@@QAEXHH_N@Z 315121a0 f i LoaderSKIN.obj
 0001:00011300       ??R?$less@V?$CryStringT@D@@@stlpmtx_std@@QBE_NABV?$CryStringT@D@@0@Z 31512300 f i LoaderSKIN.obj
 0001:00011350       ?GetCRC32Lowercase@Crc32Gen@@QBEIPBD@Z 31512350 f i LoaderSKIN.obj
 0001:000113b0       ??0?$CryStackStringT@D$0CAA@@@QAE@PBD@Z 315123b0 f i LoaderSKIN.obj
 0001:00011420       ?_ConcatenateInPlace@?$CryStackStringT@D$0CAA@@@QAEXPBDI@Z 31512420 f i LoaderSKIN.obj
 0001:00011490       ?_Assign@?$CryStackStringT@D$0CAA@@@QAEXPBDI@Z 31512490 f i LoaderSKIN.obj
 0001:00011500       ?resize_raw@?$SmallDynStorage@U?$Vec3_tpl@M@@HUStandardAlloc@NAlloc@@@NArray@@QAEXHH_N@Z 31512500 f i LoaderSKIN.obj
 0001:00011660       ?resize_raw@?$SmallDynStorage@U?$Quat_tpl@M@@HUStandardAlloc@NAlloc@@@NArray@@QAEXHH_N@Z 31512660 f i LoaderSKIN.obj
 0001:000117b0       ?_Concatenate@?$CryStringT@D@@IAEXPBDI0I@Z 315127b0 f i LoaderSKIN.obj
 0001:00011850       ?set_size@?$SmallDynStorage@UMorphTargetVertex@@HUStandardAlloc@NAlloc@@@NArray@@QAEXH@Z 31512850 f i LoaderSKIN.obj
 0001:000118e0       ?resize_raw@?$SmallDynStorage@UBoneIndices8@@HUStandardAlloc@NAlloc@@@NArray@@QAEXHH_N@Z 315128e0 f i LoaderSKIN.obj
 0001:00011a30       ?resize_raw@?$SmallDynStorage@UBoneWeights8@@HUStandardAlloc@NAlloc@@@NArray@@QAEXHH_N@Z 31512a30 f i LoaderSKIN.obj
 0001:00011b80       ?expand_raw@?$DynArray@UExtSkinVertex@@HU?$SmallDynStorage@UExtSkinVertex@@HUStandardAlloc@NAlloc@@@NArray@@@@IAEPAUExtSkinVertex@@PAU2@H@Z 31512b80 f i LoaderSKIN.obj
 0001:00011c10       ?resize_raw@?$SmallDynStorage@UMorphTargetVertex@@HUStandardAlloc@NAlloc@@@NArray@@QAEXHH_N@Z 31512c10 f i LoaderSKIN.obj
 0001:00011d70       ?expand_raw@?$DynArray@UBoneIndices8@@HU?$SmallDynStorage@UBoneIndices8@@HUStandardAlloc@NAlloc@@@NArray@@@@IAEPAUBoneIndices8@@PAU2@H@Z 31512d70 f i LoaderSKIN.obj
 0001:00011df0       ?expand_raw@?$DynArray@UBoneWeights8@@HU?$SmallDynStorage@UBoneWeights8@@HUStandardAlloc@NAlloc@@@NArray@@@@IAEPAUBoneWeights8@@PAU2@H@Z 31512df0 f i LoaderSKIN.obj
 0001:00011e70       ??$move_init@V?$_smart_ptr@VIController@@@@@NArray@@YAXPAV?$_smart_ptr@VIController@@@@0I@Z 31512e70 f i DirectionalBlender.obj
 0001:00011e70       ??$move_init@V?$_smart_ptr@UCMorphTarget@@@@@NArray@@YAXPAV?$_smart_ptr@UCMorphTarget@@@@0I@Z 31512e70 f i LoaderSKIN.obj
 0001:00011ec0       ?_M_insert_overflow@?$_Impl_vector@U?$Vec3_tpl@M@@V?$allocator@U?$Vec3_tpl@M@@@stlpmtx_std@@@priv@stlpmtx_std@@AAEXPAU?$Vec3_tpl@M@@ABU4@ABU__true_type@3@I_N@Z 31512ec0 f i LoaderSKIN.obj
 0001:00012040       ??$__uninitialized_fill_n@PAU?$Vec3_tpl@M@@IU1@@priv@stlpmtx_std@@YAPAU?$Vec3_tpl@M@@PAU2@IABU2@@Z 31513040 f i LoaderSKIN.obj
 0001:000120a0       ??$__median@U?$pair@V?$CryStringT@D@@PAUIFacialAnimChannel@@@stlpmtx_std@@VFirstLess@?$VectorMap@V?$CryStringT@D@@PAUIFacialAnimChannel@@U?$less@V?$CryStringT@D@@@stlpmtx_std@@V?$allocator@U?$pair@V?$CryStringT@D@@PAUIFacialAnimChannel@@@stlpmtx_std@@@4@@@@priv@stlpmtx_std@@YAABU?$pair@V?$CryStringT@D@@PAUIFacialAnimChannel@@@1@ABU21@00VFirstLess@?$VectorMap@V?$CryStringT@D@@PAUIFacialAnimChannel@@U?$less@V?$CryStringT@D@@@stlpmtx_std@@V?$allocator@U?$pair@V?$CryStringT@D@@PAUIFacialAnimChannel@@@stlpmtx_std@@@4@@@@Z 315130a0 f i FaceAnimation.obj
 0001:000120a0       ??$__median@U?$pair@V?$CryStringT@D@@H@stlpmtx_std@@VFirstLess@?$VectorMap@V?$CryStringT@D@@HU?$less@V?$CryStringT@D@@@stlpmtx_std@@V?$allocator@U?$pair@V?$CryStringT@D@@H@stlpmtx_std@@@3@@@@priv@stlpmtx_std@@YAABU?$pair@V?$CryStringT@D@@H@1@ABU21@00VFirstLess@?$VectorMap@V?$CryStringT@D@@HU?$less@V?$CryStringT@D@@@stlpmtx_std@@V?$allocator@U?$pair@V?$CryStringT@D@@H@stlpmtx_std@@@3@@@@Z 315130a0 f i LoaderSKIN.obj
 0001:000121c0       ??$__push_heap@PAU?$pair@V?$CryStringT@D@@H@stlpmtx_std@@HU12@VFirstLess@?$VectorMap@V?$CryStringT@D@@HU?$less@V?$CryStringT@D@@@stlpmtx_std@@V?$allocator@U?$pair@V?$CryStringT@D@@H@stlpmtx_std@@@3@@@@stlpmtx_std@@YAXPAU?$pair@V?$CryStringT@D@@H@0@HHU10@VFirstLess@?$VectorMap@V?$CryStringT@D@@HU?$less@V?$CryStringT@D@@@stlpmtx_std@@V?$allocator@U?$pair@V?$CryStringT@D@@H@stlpmtx_std@@@3@@@@Z 315131c0 f i LoaderSKIN.obj
 0001:000121c0       ??$__push_heap@PAU?$pair@V?$CryStringT@D@@PAUIFacialAnimChannel@@@stlpmtx_std@@HU12@VFirstLess@?$VectorMap@V?$CryStringT@D@@PAUIFacialAnimChannel@@U?$less@V?$CryStringT@D@@@stlpmtx_std@@V?$allocator@U?$pair@V?$CryStringT@D@@PAUIFacialAnimChannel@@@stlpmtx_std@@@4@@@@stlpmtx_std@@YAXPAU?$pair@V?$CryStringT@D@@PAUIFacialAnimChannel@@@0@HHU10@VFirstLess@?$VectorMap@V?$CryStringT@D@@PAUIFacialAnimChannel@@U?$less@V?$CryStringT@D@@@stlpmtx_std@@V?$allocator@U?$pair@V?$CryStringT@D@@PAUIFacialAnimChannel@@@stlpmtx_std@@@4@@@@Z 315131c0 f i FaceAnimation.obj
 0001:00012300       ??0?$CryStringT@D@@QAE@PBD@Z 31513300 f i LoaderSKIN.obj
 0001:00012370       ??0?$CryStringT@D@@QAE@PBDI@Z 31513370 f i LoaderSKIN.obj
 0001:000123d0       ?_ConcatenateInPlace@?$CryStringT@D@@IAEXPBDI@Z 315133d0 f i LoaderSKIN.obj
 0001:00012460       ?append@?$CryStackStringT@D$0CAA@@@QAEAAV1@PBD@Z 31513460 f i LoaderSKIN.obj
 0001:00012460       ??Y?$CryStackStringT@D$0CAA@@@QAEAAV0@PBD@Z 31513460 f i LoaderSKIN.obj
 0001:000124a0       ?expand_raw@?$DynArray@U?$Vec3_tpl@M@@HU?$SmallDynStorage@U?$Vec3_tpl@M@@HUStandardAlloc@NAlloc@@@NArray@@@@IAEPAU?$Vec3_tpl@M@@PAU2@H@Z 315134a0 f i LoaderSKIN.obj
 0001:00012530       ?expand_raw@?$DynArray@U?$Quat_tpl@M@@HU?$SmallDynStorage@U?$Quat_tpl@M@@HUStandardAlloc@NAlloc@@@NArray@@@@IAEPAU?$Quat_tpl@M@@PAU2@H@Z 31513530 f i LoaderSKIN.obj
 0001:000125b0       ?erase@?$DynArray@U?$Vec3_tpl@M@@HU?$SmallDynStorage@U?$Vec3_tpl@M@@HUStandardAlloc@NAlloc@@@NArray@@@@QAEPAU?$Vec3_tpl@M@@PAU2@0@Z 315135b0 f i LoaderSKIN.obj
 0001:00012620       ?erase@?$DynArray@U?$Quat_tpl@M@@HU?$SmallDynStorage@U?$Quat_tpl@M@@HUStandardAlloc@NAlloc@@@NArray@@@@QAEPAU?$Quat_tpl@M@@PAU2@0@Z 31513620 f i LoaderSKIN.obj
 0001:00012730       ?expand_raw@?$DynArray@UMorphTargetVertex@@HU?$SmallDynStorage@UMorphTargetVertex@@HUStandardAlloc@NAlloc@@@NArray@@@@IAEPAUMorphTargetVertex@@PAU2@H@Z 31513730 f i LoaderSKIN.obj
 0001:000127c0       ?erase@?$DynArray@UBoneIndices8@@HU?$SmallDynStorage@UBoneIndices8@@HUStandardAlloc@NAlloc@@@NArray@@@@QAEPAUBoneIndices8@@PAU2@0@Z 315137c0 f i LoaderSKIN.obj
 0001:00012820       ?erase@?$DynArray@UBoneWeights8@@HU?$SmallDynStorage@UBoneWeights8@@HUStandardAlloc@NAlloc@@@NArray@@@@QAEPAUBoneWeights8@@PAU2@0@Z 31513820 f i LoaderSKIN.obj
 0001:00012880       ?resize_raw@?$SmallDynStorage@V?$_smart_ptr@UCMorphTarget@@@@HUStandardAlloc@NAlloc@@@NArray@@QAEXHH_N@Z 31513880 f i LoaderSKIN.obj
 0001:000129d0       ?erase@?$DynArray@EHU?$SmallDynStorage@EHUStandardAlloc@NAlloc@@@NArray@@@@QAEPAEPAE0@Z 315139d0 f i LoaderSKIN.obj
 0001:00012a20       ?assign@?$CryStringT@D@@QAEAAV1@PBD0@Z 31513a20 f i LoaderSKIN.obj
 0001:00012a60       ??4?$_Impl_vector@PAXV?$allocator@PAX@stlpmtx_std@@@priv@stlpmtx_std@@QAEAAV012@ABV012@@Z 31513a60 f i LoaderSKIN.obj
 0001:00012b70       ?_M_fill_insert_aux@?$_Impl_vector@U?$Vec3_tpl@M@@V?$allocator@U?$Vec3_tpl@M@@@stlpmtx_std@@@priv@stlpmtx_std@@AAEXPAU?$Vec3_tpl@M@@IABU4@ABU__false_type@3@@Z 31513b70 f i LoaderSKIN.obj
 0001:00012c90       ??$__adjust_heap@PAU?$pair@V?$CryStringT@D@@PAUIFacialAnimChannel@@@stlpmtx_std@@HU12@VFirstLess@?$VectorMap@V?$CryStringT@D@@PAUIFacialAnimChannel@@U?$less@V?$CryStringT@D@@@stlpmtx_std@@V?$allocator@U?$pair@V?$CryStringT@D@@PAUIFacialAnimChannel@@@stlpmtx_std@@@4@@@@stlpmtx_std@@YAXPAU?$pair@V?$CryStringT@D@@PAUIFacialAnimChannel@@@0@HHU10@VFirstLess@?$VectorMap@V?$CryStringT@D@@PAUIFacialAnimChannel@@U?$less@V?$CryStringT@D@@@stlpmtx_std@@V?$allocator@U?$pair@V?$CryStringT@D@@PAUIFacialAnimChannel@@@stlpmtx_std@@@4@@@@Z 31513c90 f i FaceAnimation.obj
 0001:00012c90       ??$__adjust_heap@PAU?$pair@V?$CryStringT@D@@H@stlpmtx_std@@HU12@VFirstLess@?$VectorMap@V?$CryStringT@D@@HU?$less@V?$CryStringT@D@@@stlpmtx_std@@V?$allocator@U?$pair@V?$CryStringT@D@@H@stlpmtx_std@@@3@@@@stlpmtx_std@@YAXPAU?$pair@V?$CryStringT@D@@H@0@HHU10@VFirstLess@?$VectorMap@V?$CryStringT@D@@HU?$less@V?$CryStringT@D@@@stlpmtx_std@@V?$allocator@U?$pair@V?$CryStringT@D@@H@stlpmtx_std@@@3@@@@Z 31513c90 f i LoaderSKIN.obj
 0001:00012e00       ?substr@?$CryStringT@D@@QBE?AV1@II@Z 31513e00 f i LoaderSKIN.obj
 0001:00012e50       ??Y?$CryStringT@D@@QAEAAV0@PBD@Z 31513e50 f i LoaderSKIN.obj
 0001:00012e90       ??$?HD$0CAA@@@YA?AV?$CryStackStringT@D$0CAA@@@ABV0@PBD@Z 31513e90 f i LoaderSKIN.obj
 0001:00012f00       ??1?$DynArray@MHU?$SmallDynStorage@MHUStandardAlloc@NAlloc@@@NArray@@@@QAE@XZ 31513f00 f i CharacterInstance.obj
 0001:00012f00       ??1?$DynArray@UExtSkinVertex@@HU?$SmallDynStorage@UExtSkinVertex@@HUStandardAlloc@NAlloc@@@NArray@@@@QAE@XZ 31513f00 f i LoaderSKIN.obj
 0001:00012f30       ??4?$DynArray@U?$Vec3_tpl@M@@HU?$SmallDynStorage@U?$Vec3_tpl@M@@HUStandardAlloc@NAlloc@@@NArray@@@@QAEAAU0@U?$Array@$$CBU?$Vec3_tpl@M@@HU?$ArrayStorage@$$CBU?$Vec3_tpl@M@@H@NArray@@@@@Z 31513f30 f i LoaderSKIN.obj
 0001:00012fd0       ??4?$DynArray@U?$Quat_tpl@M@@HU?$SmallDynStorage@U?$Quat_tpl@M@@HUStandardAlloc@NAlloc@@@NArray@@@@QAEAAU0@U?$Array@$$CBU?$Quat_tpl@M@@HU?$ArrayStorage@$$CBU?$Quat_tpl@M@@H@NArray@@@@@Z 31513fd0 f i LoaderSKIN.obj
 0001:00013080       ??4?$DynArray@UBoneIndices8@@HU?$SmallDynStorage@UBoneIndices8@@HUStandardAlloc@NAlloc@@@NArray@@@@QAEAAU0@U?$Array@$$CBUBoneIndices8@@HU?$ArrayStorage@$$CBUBoneIndices8@@H@NArray@@@@@Z 31514080 f i LoaderSKIN.obj
 0001:00013160       ??4?$DynArray@UBoneWeights8@@HU?$SmallDynStorage@UBoneWeights8@@HUStandardAlloc@NAlloc@@@NArray@@@@QAEAAU0@U?$Array@$$CBUBoneWeights8@@HU?$ArrayStorage@$$CBUBoneWeights8@@H@NArray@@@@@Z 31514160 f i LoaderSKIN.obj
 0001:00013230       ??4?$DynArray@V?$_smart_ptr@UCMorphTarget@@@@HU?$SmallDynStorage@V?$_smart_ptr@UCMorphTarget@@@@HUStandardAlloc@NAlloc@@@NArray@@@@QAEAAU0@U?$Array@$$CBV?$_smart_ptr@UCMorphTarget@@@@HU?$ArrayStorage@$$CBV?$_smart_ptr@UCMorphTarget@@@@H@NArray@@@@@Z 31514230 f i LoaderSKIN.obj
 0001:000132f0       ?destroy@?$DynArray@USJointInfo@CSkin@@HU?$SmallDynStorage@USJointInfo@CSkin@@HUStandardAlloc@NAlloc@@@NArray@@@@KAXU?$Array@USJointInfo@CSkin@@HU?$ArrayStorage@USJointInfo@CSkin@@H@NArray@@@@@Z 315142f0 f i LoaderSKIN.obj
 0001:00013340       ?expand_raw@?$DynArray@V?$_smart_ptr@UCMorphTarget@@@@HU?$SmallDynStorage@V?$_smart_ptr@UCMorphTarget@@@@HUStandardAlloc@NAlloc@@@NArray@@@@IAEPAV?$_smart_ptr@UCMorphTarget@@@@PAV2@H@Z 31514340 f i LoaderSKIN.obj
 0001:000133c0       ?GetPath@PathUtil@@YA?AV?$CryStringT@D@@ABV2@@Z 315143c0 f i LoaderSKIN.obj
 0001:00013470       ??4?$DynArray@EHU?$SmallDynStorage@EHUStandardAlloc@NAlloc@@@NArray@@@@QAEAAU0@U?$Array@$$CBEHU?$ArrayStorage@$$CBEH@NArray@@@@@Z 31514470 f i LoaderSKIN.obj
 0001:00013530       ??$move_init@USJointInfo@CSkin@@@NArray@@YAXPAUSJointInfo@CSkin@@0I@Z 31514530 f i LoaderSKIN.obj
 0001:000135d0       ??$__destroy_range_aux@V?$reverse_iterator@PAU?$pair@V?$CryStringT@D@@H@stlpmtx_std@@@stlpmtx_std@@U?$pair@V?$CryStringT@D@@H@2@@stlpmtx_std@@YAXV?$reverse_iterator@PAU?$pair@V?$CryStringT@D@@H@stlpmtx_std@@@0@0PAU?$pair@V?$CryStringT@D@@H@0@ABU__false_type@0@@Z 315145d0 f i LoaderSKIN.obj
 0001:000135d0       ??$__destroy_range_aux@V?$reverse_iterator@PAU?$pair@V?$CryStringT@D@@PAUIFacialAnimChannel@@@stlpmtx_std@@@stlpmtx_std@@U?$pair@V?$CryStringT@D@@PAUIFacialAnimChannel@@@2@@stlpmtx_std@@YAXV?$reverse_iterator@PAU?$pair@V?$CryStringT@D@@PAUIFacialAnimChannel@@@stlpmtx_std@@@0@0PAU?$pair@V?$CryStringT@D@@PAUIFacialAnimChannel@@@0@ABU__false_type@0@@Z 315145d0 f i FaceAnimation.obj
 0001:00013620       ??$__ucopy@PAU?$pair@V?$CryStringT@D@@PAUIFacialAnimChannel@@@stlpmtx_std@@PAU12@H@priv@stlpmtx_std@@YAPAU?$pair@V?$CryStringT@D@@PAUIFacialAnimChannel@@@1@PAU21@00ABUrandom_access_iterator_tag@1@PAH@Z 31514620 f i FaceAnimation.obj
 0001:00013620       ??$__ucopy@PAU?$pair@V?$CryStringT@D@@H@stlpmtx_std@@PAU12@H@priv@stlpmtx_std@@YAPAU?$pair@V?$CryStringT@D@@H@1@PAU21@00ABUrandom_access_iterator_tag@1@PAH@Z 31514620 f i LoaderSKIN.obj
 0001:00013670       ??$__make_heap@PAU?$pair@V?$CryStringT@D@@PAUIFacialAnimChannel@@@stlpmtx_std@@VFirstLess@?$VectorMap@V?$CryStringT@D@@PAUIFacialAnimChannel@@U?$less@V?$CryStringT@D@@@stlpmtx_std@@V?$allocator@U?$pair@V?$CryStringT@D@@PAUIFacialAnimChannel@@@stlpmtx_std@@@4@@@U12@H@stlpmtx_std@@YAXPAU?$pair@V?$CryStringT@D@@PAUIFacialAnimChannel@@@0@0VFirstLess@?$VectorMap@V?$CryStringT@D@@PAUIFacialAnimChannel@@U?$less@V?$CryStringT@D@@@stlpmtx_std@@V?$allocator@U?$pair@V?$CryStringT@D@@PAUIFacialAnimChannel@@@stlpmtx_std@@@4@@@0PAH@Z 31514670 f i FaceAnimation.obj
 0001:00013670       ??$__make_heap@PAU?$pair@V?$CryStringT@D@@H@stlpmtx_std@@VFirstLess@?$VectorMap@V?$CryStringT@D@@HU?$less@V?$CryStringT@D@@@stlpmtx_std@@V?$allocator@U?$pair@V?$CryStringT@D@@H@stlpmtx_std@@@3@@@U12@H@stlpmtx_std@@YAXPAU?$pair@V?$CryStringT@D@@H@0@0VFirstLess@?$VectorMap@V?$CryStringT@D@@HU?$less@V?$CryStringT@D@@@stlpmtx_std@@V?$allocator@U?$pair@V?$CryStringT@D@@H@stlpmtx_std@@@3@@@0PAH@Z 31514670 f i LoaderSKIN.obj
 0001:000136d0       ??$?HD@@YA?AV?$CryStringT@D@@ABV0@PBD@Z 315146d0 f i LoaderSKIN.obj
 0001:00013b60       ??0?$DynArray@UExtSkinVertex@@HU?$SmallDynStorage@UExtSkinVertex@@HUStandardAlloc@NAlloc@@@NArray@@@@QAE@XZ 31514b60 f i LoaderSKIN.obj
 0001:00013bb0       ??0?$DynArray@UBoneIndices8@@HU?$SmallDynStorage@UBoneIndices8@@HUStandardAlloc@NAlloc@@@NArray@@@@QAE@ABU0@@Z 31514bb0 f i LoaderSKIN.obj
 0001:00013c50       ??0?$DynArray@UBoneWeights8@@HU?$SmallDynStorage@UBoneWeights8@@HUStandardAlloc@NAlloc@@@NArray@@@@QAE@ABU0@@Z 31514c50 f i LoaderSKIN.obj
 0001:00013cf0       ??0?$DynArray@EHU?$SmallDynStorage@EHUStandardAlloc@NAlloc@@@NArray@@@@QAE@ABU0@@Z 31514cf0 f i LoaderSKIN.obj
 0001:00013d80       ?push_back@?$DynArray@V?$_smart_ptr@UCMorphTarget@@@@HU?$SmallDynStorage@V?$_smart_ptr@UCMorphTarget@@@@HUStandardAlloc@NAlloc@@@NArray@@@@QAEPAV?$_smart_ptr@UCMorphTarget@@@@U?$Array@$$CBV?$_smart_ptr@UCMorphTarget@@@@HU?$ArrayStorage@$$CBV?$_smart_ptr@UCMorphTarget@@@@H@NArray@@@@@Z 31514d80 f i LoaderSKIN.obj
 0001:00013de0       ?resize_raw@?$SmallDynStorage@USJointInfo@CSkin@@HUStandardAlloc@NAlloc@@@NArray@@QAEXHH_N@Z 31514de0 f i LoaderSKIN.obj
 0001:00013f40       ??$__unguarded_partition@PAU?$pair@V?$CryStringT@D@@H@stlpmtx_std@@U12@VFirstLess@?$VectorMap@V?$CryStringT@D@@HU?$less@V?$CryStringT@D@@@stlpmtx_std@@V?$allocator@U?$pair@V?$CryStringT@D@@H@stlpmtx_std@@@3@@@@priv@stlpmtx_std@@YAPAU?$pair@V?$CryStringT@D@@H@1@PAU21@0U21@VFirstLess@?$VectorMap@V?$CryStringT@D@@HU?$less@V?$CryStringT@D@@@stlpmtx_std@@V?$allocator@U?$pair@V?$CryStringT@D@@H@stlpmtx_std@@@3@@@@Z 31514f40 f i LoaderSKIN.obj
 0001:00013f40       ??$__unguarded_partition@PAU?$pair@V?$CryStringT@D@@PAUIFacialAnimChannel@@@stlpmtx_std@@U12@VFirstLess@?$VectorMap@V?$CryStringT@D@@PAUIFacialAnimChannel@@U?$less@V?$CryStringT@D@@@stlpmtx_std@@V?$allocator@U?$pair@V?$CryStringT@D@@PAUIFacialAnimChannel@@@stlpmtx_std@@@4@@@@priv@stlpmtx_std@@YAPAU?$pair@V?$CryStringT@D@@PAUIFacialAnimChannel@@@1@PAU21@0U21@VFirstLess@?$VectorMap@V?$CryStringT@D@@PAUIFacialAnimChannel@@U?$less@V?$CryStringT@D@@@stlpmtx_std@@V?$allocator@U?$pair@V?$CryStringT@D@@PAUIFacialAnimChannel@@@stlpmtx_std@@@4@@@@Z 31514f40 f i FaceAnimation.obj
 0001:000141c0       ??0?$DynArray@U?$Vec3_tpl@M@@HU?$SmallDynStorage@U?$Vec3_tpl@M@@HUStandardAlloc@NAlloc@@@NArray@@@@QAE@XZ 315151c0 f i LoaderSKIN.obj
 0001:00014210       ??0?$DynArray@U?$Vec3_tpl@M@@HU?$SmallDynStorage@U?$Vec3_tpl@M@@HUStandardAlloc@NAlloc@@@NArray@@@@QAE@ABU0@@Z 31515210 f i LoaderSKIN.obj
 0001:000142b0       ??0?$DynArray@U?$Quat_tpl@M@@HU?$SmallDynStorage@U?$Quat_tpl@M@@HUStandardAlloc@NAlloc@@@NArray@@@@QAE@ABU0@@Z 315152b0 f i LoaderSKIN.obj
 0001:00014ea0       ??1CMorphTarget@@UAE@XZ    31515ea0 f i LoaderSKIN.obj
 0001:00014f10       ??_ECMorphTarget@@UAEPAXI@Z 31515f10 f i LoaderSKIN.obj
 0001:00014f10       ??_GCMorphTarget@@UAEPAXI@Z 31515f10 f i LoaderSKIN.obj
 0001:00014f40       ?resize@?$_Impl_vector@U?$Vec3_tpl@M@@V?$allocator@U?$Vec3_tpl@M@@@stlpmtx_std@@@priv@stlpmtx_std@@QAEXIABU?$Vec3_tpl@M@@@Z 31515f40 f i LoaderSKIN.obj
 0001:00014ff0       ?expand_raw@?$DynArray@USJointInfo@CSkin@@HU?$SmallDynStorage@USJointInfo@CSkin@@HUStandardAlloc@NAlloc@@@NArray@@@@IAEPAUSJointInfo@CSkin@@PAU23@H@Z 31515ff0 f i LoaderSKIN.obj
 0001:00015080       ??$sort_heap@PAU?$pair@V?$CryStringT@D@@PAUIFacialAnimChannel@@@stlpmtx_std@@VFirstLess@?$VectorMap@V?$CryStringT@D@@PAUIFacialAnimChannel@@U?$less@V?$CryStringT@D@@@stlpmtx_std@@V?$allocator@U?$pair@V?$CryStringT@D@@PAUIFacialAnimChannel@@@stlpmtx_std@@@4@@@@stlpmtx_std@@YAXPAU?$pair@V?$CryStringT@D@@PAUIFacialAnimChannel@@@0@0VFirstLess@?$VectorMap@V?$CryStringT@D@@PAUIFacialAnimChannel@@U?$less@V?$CryStringT@D@@@stlpmtx_std@@V?$allocator@U?$pair@V?$CryStringT@D@@PAUIFacialAnimChannel@@@stlpmtx_std@@@4@@@@Z 31516080 f i FaceAnimation.obj
 0001:00015080       ??$sort_heap@PAU?$pair@V?$CryStringT@D@@H@stlpmtx_std@@VFirstLess@?$VectorMap@V?$CryStringT@D@@HU?$less@V?$CryStringT@D@@@stlpmtx_std@@V?$allocator@U?$pair@V?$CryStringT@D@@H@stlpmtx_std@@@3@@@@stlpmtx_std@@YAXPAU?$pair@V?$CryStringT@D@@H@0@0VFirstLess@?$VectorMap@V?$CryStringT@D@@HU?$less@V?$CryStringT@D@@@stlpmtx_std@@V?$allocator@U?$pair@V?$CryStringT@D@@H@stlpmtx_std@@@3@@@@Z 31516080 f i LoaderSKIN.obj
 0001:000151e0       ?resize@?$DynArray@V?$_smart_ptr@UCMorphTarget@@@@HU?$SmallDynStorage@V?$_smart_ptr@UCMorphTarget@@@@HUStandardAlloc@NAlloc@@@NArray@@@@QAEXH@Z 315161e0 f i LoaderSKIN.obj
 0001:00015270       ?init@?$DynArray@URChunk@@HU?$SmallDynStorage@URChunk@@HUStandardAlloc@NAlloc@@@NArray@@@@KAPAURChunk@@U?$Array@URChunk@@HU?$ArrayStorage@URChunk@@H@NArray@@@@@Z 31516270 f i LoaderSKIN.obj
 0001:00015340       ?init@?$DynArray@URChunk@@HU?$SmallDynStorage@URChunk@@HUStandardAlloc@NAlloc@@@NArray@@@@KAPAURChunk@@U?$Array@URChunk@@HU?$ArrayStorage@URChunk@@H@NArray@@@@PBU2@@Z 31516340 f i LoaderSKIN.obj
 0001:00015390       ?assign@?$Array@URChunk@@HU?$SmallDynStorage@URChunk@@HUStandardAlloc@NAlloc@@@NArray@@@@QAEXU?$Array@$$CBURChunk@@HU?$ArrayStorage@$$CBURChunk@@H@NArray@@@@@Z 31516390 f i LoaderSKIN.obj
 0001:000153e0       ?_M_insert_overflow_aux@?$_Impl_vector@U?$pair@V?$CryStringT@D@@H@stlpmtx_std@@V?$allocator@U?$pair@V?$CryStringT@D@@H@stlpmtx_std@@@2@@priv@stlpmtx_std@@AAEXPAU?$pair@V?$CryStringT@D@@H@3@ABU43@ABU__false_type@3@I_N@Z 315163e0 f i LoaderSKIN.obj
 0001:000153e0       ?_M_insert_overflow_aux@?$_Impl_vector@U?$pair@V?$CryStringT@D@@PAUIFacialAnimChannel@@@stlpmtx_std@@V?$allocator@U?$pair@V?$CryStringT@D@@PAUIFacialAnimChannel@@@stlpmtx_std@@@2@@priv@stlpmtx_std@@AAEXPAU?$pair@V?$CryStringT@D@@PAUIFacialAnimChannel@@@3@ABU43@ABU__false_type@3@I_N@Z 315163e0 f i FaceAnimation.obj
 0001:00015580       ??$__partial_sort@PAU?$pair@V?$CryStringT@D@@PAUIFacialAnimChannel@@@stlpmtx_std@@U12@VFirstLess@?$VectorMap@V?$CryStringT@D@@PAUIFacialAnimChannel@@U?$less@V?$CryStringT@D@@@stlpmtx_std@@V?$allocator@U?$pair@V?$CryStringT@D@@PAUIFacialAnimChannel@@@stlpmtx_std@@@4@@@@priv@stlpmtx_std@@YAXPAU?$pair@V?$CryStringT@D@@PAUIFacialAnimChannel@@@1@000VFirstLess@?$VectorMap@V?$CryStringT@D@@PAUIFacialAnimChannel@@U?$less@V?$CryStringT@D@@@stlpmtx_std@@V?$allocator@U?$pair@V?$CryStringT@D@@PAUIFacialAnimChannel@@@stlpmtx_std@@@4@@@@Z 31516580 f i FaceAnimation.obj
 0001:00015580       ??$__partial_sort@PAU?$pair@V?$CryStringT@D@@H@stlpmtx_std@@U12@VFirstLess@?$VectorMap@V?$CryStringT@D@@HU?$less@V?$CryStringT@D@@@stlpmtx_std@@V?$allocator@U?$pair@V?$CryStringT@D@@H@stlpmtx_std@@@3@@@@priv@stlpmtx_std@@YAXPAU?$pair@V?$CryStringT@D@@H@1@000VFirstLess@?$VectorMap@V?$CryStringT@D@@HU?$less@V?$CryStringT@D@@@stlpmtx_std@@V?$allocator@U?$pair@V?$CryStringT@D@@H@stlpmtx_std@@@3@@@@Z 31516580 f i LoaderSKIN.obj
 0001:00015710       ?destroy@?$DynArray@URChunk@@HU?$SmallDynStorage@URChunk@@HUStandardAlloc@NAlloc@@@NArray@@@@KAXU?$Array@URChunk@@HU?$ArrayStorage@URChunk@@H@NArray@@@@@Z 31516710 f i LoaderSKIN.obj
 0001:000163a0       ??1?$VectorMap@V?$CryStringT@D@@HU?$less@V?$CryStringT@D@@@stlpmtx_std@@V?$allocator@U?$pair@V?$CryStringT@D@@H@stlpmtx_std@@@3@@@QAE@XZ 315173a0 f i LoaderSKIN.obj
 0001:000163f0       ?erase@?$DynArray@URChunk@@HU?$SmallDynStorage@URChunk@@HUStandardAlloc@NAlloc@@@NArray@@@@QAEPAURChunk@@PAU2@0@Z 315173f0 f i LoaderSKIN.obj
 0001:000164a0       ??$move_init@URChunk@@@NArray@@YAXPAURChunk@@0I@Z 315174a0 f i LoaderSKIN.obj
 0001:00016570       ?resize@?$DynArray@USJointInfo@CSkin@@HU?$SmallDynStorage@USJointInfo@CSkin@@HUStandardAlloc@NAlloc@@@NArray@@@@QAEXH@Z 31517570 f i LoaderSKIN.obj
 0001:000165f0       ?resize_raw@?$SmallDynStorage@URChunk@@HUStandardAlloc@NAlloc@@@NArray@@QAEXHH_N@Z 315175f0 f i LoaderSKIN.obj
 0001:00016750       ??$__introsort_loop@PAU?$pair@V?$CryStringT@D@@H@stlpmtx_std@@U12@HVFirstLess@?$VectorMap@V?$CryStringT@D@@HU?$less@V?$CryStringT@D@@@stlpmtx_std@@V?$allocator@U?$pair@V?$CryStringT@D@@H@stlpmtx_std@@@3@@@@priv@stlpmtx_std@@YAXPAU?$pair@V?$CryStringT@D@@H@1@00HVFirstLess@?$VectorMap@V?$CryStringT@D@@HU?$less@V?$CryStringT@D@@@stlpmtx_std@@V?$allocator@U?$pair@V?$CryStringT@D@@H@stlpmtx_std@@@3@@@@Z 31517750 f i LoaderSKIN.obj
 0001:00016750       ??$__introsort_loop@PAU?$pair@V?$CryStringT@D@@PAUIFacialAnimChannel@@@stlpmtx_std@@U12@HVFirstLess@?$VectorMap@V?$CryStringT@D@@PAUIFacialAnimChannel@@U?$less@V?$CryStringT@D@@@stlpmtx_std@@V?$allocator@U?$pair@V?$CryStringT@D@@PAUIFacialAnimChannel@@@stlpmtx_std@@@4@@@@priv@stlpmtx_std@@YAXPAU?$pair@V?$CryStringT@D@@PAUIFacialAnimChannel@@@1@00HVFirstLess@?$VectorMap@V?$CryStringT@D@@PAUIFacialAnimChannel@@U?$less@V?$CryStringT@D@@@stlpmtx_std@@V?$allocator@U?$pair@V?$CryStringT@D@@PAUIFacialAnimChannel@@@stlpmtx_std@@@4@@@@Z 31517750 f i FaceAnimation.obj
 0001:000169c0       ??4?$DynArray@URChunk@@HU?$SmallDynStorage@URChunk@@HUStandardAlloc@NAlloc@@@NArray@@@@QAEAAU0@U?$Array@$$CBURChunk@@HU?$ArrayStorage@$$CBURChunk@@H@NArray@@@@@Z 315179c0 f i LoaderSKIN.obj
 0001:00016a70       ?expand_raw@?$DynArray@URChunk@@HU?$SmallDynStorage@URChunk@@HUStandardAlloc@NAlloc@@@NArray@@@@IAEPAURChunk@@PAU2@H@Z 31517a70 f i LoaderSKIN.obj
 0001:00016b00       ??0CModelMesh@@QAE@XZ      31517b00 f i LoaderSKIN.obj
 0001:00016c80       ??1CModelMesh@@QAE@XZ      31517c80 f i LoaderSKIN.obj
 0001:00017220       ??4CModelMesh@@QAEAAV0@ABV0@@Z 31518220 f i LoaderSKIN.obj
 0001:000172c0       ??0?$DynArray@URChunk@@HU?$SmallDynStorage@URChunk@@HUStandardAlloc@NAlloc@@@NArray@@@@QAE@ABU0@@Z 315182c0 f i LoaderSKIN.obj
 0001:00017340       ?resize@?$DynArray@URChunk@@HU?$SmallDynStorage@URChunk@@HUStandardAlloc@NAlloc@@@NArray@@@@QAEXH@Z 31518340 f i LoaderSKIN.obj
 0001:000173b0       ??0CModelMesh@@QAE@ABV0@@Z 315183b0 f i LoaderSKIN.obj
 0001:00017460       ?erase@?$DynArray@VCModelMesh@@HU?$SmallDynStorage@VCModelMesh@@HUStandardAlloc@NAlloc@@@NArray@@@@QAEPAVCModelMesh@@PAV2@0@Z 31518460 f i LoaderSKIN.obj
 0001:00017520       ??$move_init@VCModelMesh@@@NArray@@YAXPAVCModelMesh@@0I@Z 31518520 f i LoaderSKIN.obj
 0001:00017570       ?resize_raw@?$SmallDynStorage@VCModelMesh@@HUStandardAlloc@NAlloc@@@NArray@@QAEXHH_N@Z 31518570 f i LoaderSKIN.obj
 0001:000176e0       ?expand_raw@?$DynArray@VCModelMesh@@HU?$SmallDynStorage@VCModelMesh@@HUStandardAlloc@NAlloc@@@NArray@@@@IAEPAVCModelMesh@@PAV2@H@Z 315186e0 f i LoaderSKIN.obj
 0001:00017780       ?grow@?$DynArray@VCModelMesh@@HU?$SmallDynStorage@VCModelMesh@@HUStandardAlloc@NAlloc@@@NArray@@@@QAEPAVCModelMesh@@HABV2@@Z 31518780 f i LoaderSKIN.obj
 0001:000177e0       ?resize@?$DynArray@VCModelMesh@@HU?$SmallDynStorage@VCModelMesh@@HUStandardAlloc@NAlloc@@@NArray@@@@QAEXHABVCModelMesh@@@Z 315187e0 f i LoaderSKIN.obj
 0001:00017860       ?LoadNewSKIN@CryCHRLoader@@QAEPAVCSkin@@PBDI@Z 31518860 f   LoaderSKIN.obj
 0001:00018f90       ?GetPeriodicFraction@CTimeValue@@QBEMV1@@Z 31519f90 f i ModelMesh_DebugPC.obj
 0001:00018fc0       ?DrawLabelEx@IRenderer@@QAAXU?$Vec3_tpl@M@@MPBM_N2PBDZZ 31519fc0 f i ModelMesh_DebugPC.obj
 0001:00019070       ??$__copy@PAU?$Color_tpl@E@@PAU1@H@priv@stlpmtx_std@@YAPAU?$Color_tpl@E@@PAU2@00ABUrandom_access_iterator_tag@1@PAH@Z 3151a070 f i ModelMesh_DebugPC.obj
 0001:000190c0       ??$__copy_backward@PAU?$Color_tpl@E@@PAU1@H@priv@stlpmtx_std@@YAPAU?$Color_tpl@E@@PAU2@00ABUrandom_access_iterator_tag@1@PAH@Z 3151a0c0 f i ModelMesh_DebugPC.obj
 0001:00019110       ??$fill@PAU?$Color_tpl@E@@U1@@stlpmtx_std@@YAXPAU?$Color_tpl@E@@0ABU1@@Z 3151a110 f i ModelMesh_DebugPC.obj
 0001:00019160       ??$__uninitialized_fill_n@PAU?$Color_tpl@E@@IU1@@priv@stlpmtx_std@@YAPAU?$Color_tpl@E@@PAU2@IABU2@@Z 3151a160 f i ModelMesh_DebugPC.obj
 0001:000191a0       ?_M_insert_overflow_aux@?$_Impl_vector@U?$Color_tpl@E@@V?$allocator@U?$Color_tpl@E@@@stlpmtx_std@@@priv@stlpmtx_std@@AAEXPAU?$Color_tpl@E@@ABU4@ABU__false_type@3@I_N@Z 3151a1a0 f i ModelMesh_DebugPC.obj
 0001:00019320       ?_M_fill_insert_aux@?$_Impl_vector@U?$Color_tpl@E@@V?$allocator@U?$Color_tpl@E@@@stlpmtx_std@@@priv@stlpmtx_std@@AAEXPAU?$Color_tpl@E@@IABU4@ABU__false_type@3@@Z 3151a320 f i ModelMesh_DebugPC.obj
 0001:00019420       ??0?$vector@U?$Vec3_tpl@M@@V?$allocator@U?$Vec3_tpl@M@@@stlpmtx_std@@@stlpmtx_std@@QAE@ABV?$allocator@U?$Vec3_tpl@M@@@1@@Z 3151a420 f i LoaderSKIN.obj
 0001:00019420       ??0?$vector@V?$CryStringT@D@@V?$allocator@V?$CryStringT@D@@@stlpmtx_std@@@stlpmtx_std@@QAE@ABV?$allocator@V?$CryStringT@D@@@1@@Z 3151a420 f i FaceAnimSequence.obj
 0001:00019420       ??0?$vector@U?$Color_tpl@E@@V?$allocator@U?$Color_tpl@E@@@stlpmtx_std@@@stlpmtx_std@@QAE@ABV?$allocator@U?$Color_tpl@E@@@1@@Z 3151a420 f i ModelMesh_DebugPC.obj
 0001:00019460       ?GetFile@PathUtil@@YA?AV?$CryStringT@D@@ABV2@@Z 3151a460 f i ModelMesh_DebugPC.obj
 0001:00019510       ?DrawDebugInfo@CModelMesh@@QAEXPAVCCharInstance@@HABU?$Matrix34_tpl@M@@HAAPBUIMaterial@@PAVCRenderObject@@ABUSRendParams@@@Z 3151a510 f   ModelMesh_DebugPC.obj
 0001:00019fa0       ?resize@?$DynArray@U?$Vec3_tpl@M@@HU?$SmallDynStorage@U?$Vec3_tpl@M@@HUStandardAlloc@NAlloc@@@NArray@@@@QAEXH@Z 3151afa0 f i ModelMesh_DebugPC.obj
 0001:00019fe0       ?resize@?$DynArray@UBoneIndices8@@HU?$SmallDynStorage@UBoneIndices8@@HUStandardAlloc@NAlloc@@@NArray@@@@QAEXH@Z 3151afe0 f i ModelMesh_DebugPC.obj
 0001:0001a020       ?resize@?$_Impl_vector@U?$Color_tpl@E@@V?$allocator@U?$Color_tpl@E@@@stlpmtx_std@@@priv@stlpmtx_std@@QAEXIABU?$Color_tpl@E@@@Z 3151b020 f i ModelMesh_DebugPC.obj
 0001:0001a0c0       ?DrawWireframeStatic@CModelMesh@@QAEXABU?$Matrix34_tpl@M@@PAUIRenderMesh@@I@Z 3151b0c0 f   ModelMesh_DebugPC.obj
 0001:0001a680       ?SoftwareSkinningDQ@CModelMesh@@QAEXPAUIRenderMesh@@PAVCCharInstance@@PAVCAttachmentSKIN@@U?$Matrix34_tpl@M@@EEEEPAU?$DualQuat_tpl@M@@@Z 3151b680 f   ModelMesh_DebugPC.obj
 0001:0001d750       ?GetTextureMemoryUsage@CSkin@@UBEIPAVICrySizer@@@Z 3151e750 f   ModelSkin.obj
 0001:0001d7c0       ?GetMeshMemoryUsage@CSkin@@UBEIPAVICrySizer@@@Z 3151e7c0 f   ModelSkin.obj
 0001:0001d800       ?GetIRenderMesh@CSkin@@UBEPBUIRenderMesh@@H@Z 3151e800 f   ModelSkin.obj
 0001:0001d800       ?GetIRenderMesh@CSkin@@UAEPAUIRenderMesh@@H@Z 3151e800 f   ModelSkin.obj
 0001:0001d830       ?resize_raw@?$SmallDynStorage@PAVCAttachmentSKIN@@HUStandardAlloc@NAlloc@@@NArray@@QAEXHH_N@Z 3151e830 f i ModelSkin.obj
 0001:0001d980       ?GetAttachmentTriangle@CSkin@@UAE?AUClosestTri@@ABU?$Vec3_tpl@M@@@Z 3151e980 f   ModelSkin.obj
 0001:0001d9d0       ?get_alloc_size@?$SmallDynStorage@VCModelMesh@@HUStandardAlloc@NAlloc@@@NArray@@QBEHXZ 3151e9d0 f i ModelSkin.obj
 0001:0001da30       ?expand_raw@?$DynArray@PAVCAttachmentSKIN@@HU?$SmallDynStorage@PAVCAttachmentSKIN@@HUStandardAlloc@NAlloc@@@NArray@@@@IAEPAPAVCAttachmentSKIN@@PAPAV2@H@Z 3151ea30 f i ModelSkin.obj
 0001:0001dab0       ?SizeOfModelData@CSkin@@QBEIXZ 3151eab0 f   ModelSkin.obj
 0001:0001dbf0       ??$AddObject@VCModelMesh@@HU?$SmallDynStorage@VCModelMesh@@HUStandardAlloc@NAlloc@@@NArray@@@ICrySizer@@QAEXABU?$DynArray@VCModelMesh@@HU?$SmallDynStorage@VCModelMesh@@HUStandardAlloc@NAlloc@@@NArray@@@@@Z 3151ebf0 f i ModelSkin.obj
 0001:0001dc80       ?UnregisterInstance@CSkin@@QAEXPAVCAttachmentSKIN@@@Z 3151ec80 f   ModelSkin.obj
 0001:0001dcc0       ??$push_back_unique@U?$DynArray@PAVCAttachmentSKIN@@HU?$SmallDynStorage@PAVCAttachmentSKIN@@HUStandardAlloc@NAlloc@@@NArray@@@@PAVCAttachmentSKIN@@@stl@@YA_NAAU?$DynArray@PAVCAttachmentSKIN@@HU?$SmallDynStorage@PAVCAttachmentSKIN@@HUStandardAlloc@NAlloc@@@NArray@@@@ABQAVCAttachmentSKIN@@@Z 3151ecc0 f i ModelSkin.obj
 0001:0001dd20       ?RegisterInstance@CSkin@@QAEXPAVCAttachmentSKIN@@@Z 3151ed20 f   ModelSkin.obj
 0001:0001dd80       ??1?$DynArray@VCModelMesh@@HU?$SmallDynStorage@VCModelMesh@@HUStandardAlloc@NAlloc@@@NArray@@@@QAE@XZ 3151ed80 f i ModelSkin.obj
 0001:0001dde0       ??0CSkin@@QAE@ABV?$CryStringT@D@@@Z 3151ede0 f   ModelSkin.obj
 0001:0001dfb0       ?AddRef@CSkin@@UAEXXZ      3151efb0 f i ModelSkin.obj
 0001:0001dfc0       ?DecRef@CSkin@@UAEXXZ      3151efc0 f i ModelSkin.obj
 0001:0001dfd0       ?Release@CSkin@@UAEXXZ     3151efd0 f i ModelSkin.obj
 0001:0001dff0       ?GetModelFilePath@CSkin@@UBEPBDXZ 3151eff0 f i ModelSkin.obj
 0001:0001e000       ?GetIMaterial@CSkin@@UBEPAUIMaterial@@XZ 3151f000 f i ModelSkin.obj
 0001:0001e010       ?GetNumInstances@CSkin@@UBEIXZ 3151f010 f i ModelSkin.obj
 0001:0001e020       ?GetNumLODs@CSkin@@UBEIXZ  3151f020 f i ModelSkin.obj
 0001:0001e030       ?GetNumMorphTargets@CSkin@@UBEIXZ 3151f030 f i ModelSkin.obj
 0001:0001e050       ?GetMorphTargetName@CSkin@@UBEPBDI@Z 3151f050 f i ModelSkin.obj
 0001:0001e090       ??1CSkin@@UAE@XZ           3151f090 f   ModelSkin.obj
 0001:0001e1b0       ??_ECSkin@@UAEPAXI@Z       3151f1b0 f i ModelSkin.obj
 0001:0001e1b0       ??_GCSkin@@UAEPAXI@Z       3151f1b0 f i ModelSkin.obj
 0001:0001e1e0       ?CryWarning@@YAXW4EValidatorModule@@W4EValidatorSeverity@@PBDZZ 3151f1e0 f i ParametricSampler.obj
 0001:0001e220       ?DrawLabel@IRenderer@@QAAXU?$Vec3_tpl@M@@MPBDZZ 3151f220 f i ParametricSampler.obj
 0001:0001e290       ?InitRenderingFlags@SRenderingPassInfo@@AAEXI@Z 3151f290 f i ParametricSampler.obj
 0001:0001e6e0       ?IsAssetLoaded@GlobalAnimationHeaderCAF@@QBEIXZ 3151f6e0 f i ParametricSampler.obj
 0001:0001e700       ?WeightTetrahedron@SParametricSamplerInternal@@QAE?AUBC4@@ABU?$Vec3_tpl@M@@0000@Z 3151f700 f   ParametricSampler.obj
 0001:0001eb70       ?WeightPyramid@SParametricSamplerInternal@@QAE?AUBC5@@ABU?$Vec3_tpl@M@@00000@Z 3151fb70 f   ParametricSampler.obj
 0001:0001ed30       ?CreateGeneralPassRenderingInfo@SRenderingPassInfo@@SA?AU1@ABVCCamera@@I@Z 3151fd30 f i ParametricSampler.obj
 0001:0001ef40       ??$move_init@UVirtualExample2D@@@NArray@@YAXPAUVirtualExample2D@@0I@Z 3151ff40 f i ParametricSampler.obj
 0001:0001ef40       ??$move_init@U?$SplineKey@M@spline@@@NArray@@YAXPAU?$SplineKey@M@spline@@0I@Z 3151ff40 f i FaceAnimSequence.obj
 0001:0001ef90       ??$move_init@UExtSkinVertex@@@NArray@@YAXPAUExtSkinVertex@@0I@Z 3151ff90 f i LoaderSKIN.obj
 0001:0001ef90       ??$move_init@UVirtualExample3D@@@NArray@@YAXPAUVirtualExample3D@@0I@Z 3151ff90 f i ParametricSampler.obj
 0001:0001efd0       ?UpdateWeights@@YAXMIPIAMABUGlobalAnimationHeaderLMG@@@Z 3151ffd0 f   ParametricSampler.obj
 0001:0001f0c0       ?GetWeights1D@SParametricSamplerInternal@@QAEXMABUGlobalAnimationHeaderLMG@@QAMI@Z 315200c0 f   ParametricSampler.obj
 0001:0001f280       ?GetCRC32@Crc32Gen@@QBEIPBD@Z 31520280 f i ParametricSampler.obj
 0001:0001f2d0       ?GetControllerByJointCRC32@GlobalAnimationHeaderCAF@@QBEPAVIController@@I@Z 315202d0 f i ParametricSampler.obj
 0001:0001f380       ?resize_raw@?$SmallDynStorage@UVirtualExample1D@@HUStandardAlloc@NAlloc@@@NArray@@QAEXHH_N@Z 31520380 f i ParametricSampler.obj
 0001:0001f4e0       ?resize_raw@?$SmallDynStorage@UVirtualExample2D@@HUStandardAlloc@NAlloc@@@NArray@@QAEXHH_N@Z 315204e0 f i ParametricSampler.obj
 0001:0001f640       ?set_size@?$SmallDynStorage@UCryTCBQKey@@HUStandardAlloc@NAlloc@@@NArray@@QAEXH@Z 31520640 f i LoaderTCB.obj
 0001:0001f640       ?set_size@?$SmallDynStorage@UIKLimbType@@HUStandardAlloc@NAlloc@@@NArray@@QAEXH@Z 31520640 f i ParamLoader.obj
 0001:0001f640       ?set_size@?$SmallDynStorage@UVirtualExample3D@@HUStandardAlloc@NAlloc@@@NArray@@QAEXH@Z 31520640 f i ParametricSampler.obj
 0001:0001f640       ?set_size@?$SmallDynStorage@UExtSkinVertex@@HUStandardAlloc@NAlloc@@@NArray@@QAEXH@Z 31520640 f i LoaderSKIN.obj
 0001:0001f640       ?set_size@?$SmallDynStorage@UEffectEntry@CSkeletonEffectManager@@HUStandardAlloc@NAlloc@@@NArray@@QAEXH@Z 31520640 f i SkeletonEffectManager.obj
 0001:0001f6d0       ?resize_raw@?$SmallDynStorage@UVirtualExample3D@@HUStandardAlloc@NAlloc@@@NArray@@QAEXHH_N@Z 315206d0 f i ParametricSampler.obj
 0001:0001f830       ?WeightPrism@SParametricSamplerInternal@@QAE?AUBC6@@ABU?$Vec3_tpl@M@@000000@Z 31520830 f   ParametricSampler.obj
 0001:0001fca0       ?GetConvex8@SParametricSamplerInternal@@QAE?AUBC8@@IABU?$Vec3_tpl@M@@ABUGlobalAnimationHeaderLMG@@QAMPAEPAU3@U?$Diag33_tpl@M@@U3@@Z 31520ca0 f   ParametricSampler.obj
 0001:000215f0       ?expand_raw@?$DynArray@UVirtualExample1D@@HU?$SmallDynStorage@UVirtualExample1D@@HUStandardAlloc@NAlloc@@@NArray@@@@IAEPAUVirtualExample1D@@PAU2@H@Z 315225f0 f i ParametricSampler.obj
 0001:00021680       ?expand_raw@?$DynArray@UVirtualExample2D@@HU?$SmallDynStorage@UVirtualExample2D@@HUStandardAlloc@NAlloc@@@NArray@@@@IAEPAUVirtualExample2D@@PAU2@H@Z 31522680 f i ParametricSampler.obj
 0001:00021710       ?expand_raw@?$DynArray@UVirtualExample3D@@HU?$SmallDynStorage@UVirtualExample3D@@HUStandardAlloc@NAlloc@@@NArray@@@@IAEPAUVirtualExample3D@@PAU2@H@Z 31522710 f i ParametricSampler.obj
 0001:000217a0       ?GetWeights3D@SParametricSamplerInternal@@QAEXABU?$Vec3_tpl@M@@ABUGlobalAnimationHeaderLMG@@QAMU?$Diag33_tpl@M@@U2@@Z 315227a0 f   ParametricSampler.obj
 0001:00021a50       ?ComputeWeightExtrapolate4@SParametricSamplerInternal@@QAEXAAU?$Vec4_tpl@M@@ABU?$Vec2_tpl@M@@1111@Z 31522a50 f   ParametricSampler.obj
 0001:00022260       ?GetConvex4@SParametricSamplerInternal@@QAE?AUBC4@@IABU?$Vec2_tpl@M@@ABUGlobalAnimationHeaderLMG@@QAMPAEPAU?$Vec3_tpl@M@@U?$Diag33_tpl@M@@U5@@Z 31523260 f   ParametricSampler.obj
 0001:00022c40       ?GetWeights2D@SParametricSamplerInternal@@QAEXABU?$Vec2_tpl@M@@ABUGlobalAnimationHeaderLMG@@QAMU?$Diag33_tpl@M@@U?$Vec3_tpl@M@@@Z 31523c40 f   ParametricSampler.obj
 0001:00022e50       ?VisualizeBlendSpace@SParametricSamplerInternal@@QAEXPBVCAnimationSet@@ABVCAnimation@@MIABUGlobalAnimationHeaderLMG@@U?$Vec3_tpl@M@@@Z 31523e50 f   ParametricSampler.obj
 0001:00023de0       ?resize@?$DynArray@UVirtualExample3D@@HU?$SmallDynStorage@UVirtualExample3D@@HUStandardAlloc@NAlloc@@@NArray@@@@QAEXH@Z 31524de0 f i ParametricSampler.obj
 0001:00023e20       ?BlendSpace1D@SParametricSamplerInternal@@QAEXAAUGlobalAnimationHeaderLMG@@PBVCAnimationSet@@ABVCAnimation@@MMU?$Vec3_tpl@M@@_NI@Z 31524e20 f   ParametricSampler.obj
 0001:00024b60       ?BlendSpace2D@SParametricSamplerInternal@@QAEXAAUGlobalAnimationHeaderLMG@@PBVCAnimationSet@@ABVCAnimation@@MMU?$Vec3_tpl@M@@_NI@Z 31525b60 f   ParametricSampler.obj
 0001:00026190       ?BlendSpace3D@SParametricSamplerInternal@@QAEXAAUGlobalAnimationHeaderLMG@@PBVCAnimationSet@@ABVCAnimation@@MMU?$Vec3_tpl@M@@_NI@Z 31527190 f   ParametricSampler.obj
 0001:00028140       ?CombinedBlendSpaces@SParametricSamplerInternal@@QAEXAAUGlobalAnimationHeaderLMG@@PBVCAnimationSet@@ABVCAnimation@@MM_N@Z 31529140 f   ParametricSampler.obj
 0001:00028690       ?Parameterizer@SParametricSamplerInternal@@QAEMPBVCAnimationSet@@ABVCAnimation@@MM_N@Z 31529690 f   ParametricSampler.obj
 0001:00028ce0       ?GetAllocatedObjects@CPlaceholderCharacter@@SAHXZ 31529ce0 f   PlaceholderCharacter.obj
 0001:00028cf0       ?Release@CPlaceholderCharacter@@UAEXXZ 31529cf0 f   PlaceholderCharacter.obj
 0001:00028d00       ??_EIPhonemeLibrary@@UAEPAXI@Z 31529d00 f i LipSync.obj
 0001:00028d00       ??_GIPlaceholderCharacter@@UAEPAXI@Z 31529d00 f i PlaceholderCharacter.obj
 0001:00028d00       ??_EIPlaceholderCharacter@@UAEPAXI@Z 31529d00 f i PlaceholderCharacter.obj
 0001:00028d00       ??_GIPhonemeLibrary@@UAEPAXI@Z 31529d00 f i LipSync.obj
 0001:00028d30       ?RequestHighPriorityMaterialsLoading@CPlaceholderCharacter@@UAEXXZ 31529d30 f   PlaceholderCharacter.obj
 0001:00028d70       ?GenerateIdFromName@CPlaceholderCharacter@@SAIPBD@Z 31529d70 f   PlaceholderCharacter.obj
 0001:00028da0       ??1CPlaceholderCharacter@@UAE@XZ 31529da0 f   PlaceholderCharacter.obj
 0001:00029030       ??0CPlaceholderCharacter@@QAE@XZ 3152a030 f   PlaceholderCharacter.obj
 0001:000290d0       ??_ECPlaceholderCharacter@@UAEPAXI@Z 3152a0d0 f i PlaceholderCharacter.obj
 0001:000290d0       ??_GCPlaceholderCharacter@@UAEPAXI@Z 3152a0d0 f i PlaceholderCharacter.obj
 0001:00029100       ?RegisterUsedSkin@CPlaceholderCharacter@@QAEXPAUISkin@@@Z 3152a100 f   PlaceholderCharacter.obj
 0001:00029160       ?RegisterUsedSkeleton@CPlaceholderCharacter@@QAEXPAUICharacterModel@@@Z 3152a160 f   PlaceholderCharacter.obj
 0001:000291c0       ?RegisterUsedStaticObject@CPlaceholderCharacter@@QAEXPAUIStatObj@@@Z 3152a1c0 f   PlaceholderCharacter.obj
 0001:00029220       ?RegisterUsedMaterial@CPlaceholderCharacter@@QAEXPAUIMaterial@@@Z 3152a220 f   PlaceholderCharacter.obj
 0001:00029280       ?GetISkeletonPose@CCharInstance@@UAEPAUISkeletonPose@@XZ 3152a280 f i DirectionalBlender.obj
 0001:00029290       ?cryMemcpy@@YAXPAXPBXH@Z   3152a290 f i DirectionalBlender.obj
 0001:00029490       ?AccumulateAimPoses@SDirectionalBlender@@QAEXABUSAnimationPoseModifierParams@@AAUGlobalAnimationHeaderAIM@@PAU?$QuatT_tpl@M@@MABU?$Vec3_tpl@M@@HHPAUSJointsAimIK_Rot@@IPAUSJointsAimIK_Pos@@MIABU?$Color_tpl@E@@@Z 3152a490 f   DirectionalBlender.obj
 0001:0002ad90       ?DebugVEGrid@SDirectionalBlender@@QAEXABUSAnimationPoseModifierParams@@AAUSDirInfo@@MMHPAUSJointsAimIK_Rot@@IPAUSJointsAimIK_Pos@@I@Z 3152bd90 f   DirectionalBlender.obj
 0001:0002da80       ?resize_raw@?$SmallDynStorage@V?$_smart_ptr@VIController@@@@HUStandardAlloc@NAlloc@@@NArray@@QAEXHH_N@Z 3152ea80 f i DirectionalBlender.obj
 0001:0002dbd0       ?clear@?$DynArray@V?$_smart_ptr@VIController@@@@HU?$SmallDynStorage@V?$_smart_ptr@VIController@@@@HUStandardAlloc@NAlloc@@@NArray@@@@QAEXXZ 3152ebd0 f i DirectionalBlender.obj
 0001:0002dc40       ??1?$DynArray@V?$_smart_ptr@UCMorphTarget@@@@HU?$SmallDynStorage@V?$_smart_ptr@UCMorphTarget@@@@HUStandardAlloc@NAlloc@@@NArray@@@@QAE@XZ 3152ec40 f i LoaderSKIN.obj
 0001:0002dc40       ??1?$DynArray@V?$_smart_ptr@VIController@@@@HU?$SmallDynStorage@V?$_smart_ptr@VIController@@@@HUStandardAlloc@NAlloc@@@NArray@@@@QAE@XZ 3152ec40 f i DirectionalBlender.obj
 0001:0002dca0       ?destroy@?$DynArray@UAimIKPose@@HU?$SmallDynStorage@UAimIKPose@@HUStandardAlloc@NAlloc@@@NArray@@@@KAXU?$Array@UAimIKPose@@HU?$ArrayStorage@UAimIKPose@@H@NArray@@@@@Z 3152eca0 f i DirectionalBlender.obj
 0001:0002ddc0       ??0GlobalAnimationHeaderAIM@@QAE@XZ 3152edc0 f i DirectionalBlender.obj
 0001:0002dec0       ??1GlobalAnimationHeaderAIM@@QAE@XZ 3152eec0 f i DirectionalBlender.obj
 0001:0002df80       ?ExecuteDirectionalIK@SDirectionalBlender@@QAE_NABUSAnimationPoseModifierParams@@PAUDirectionalBlends@@IPAUSJointsAimIK_Rot@@IPAUSJointsAimIK_Pos@@IABU?$Color_tpl@E@@@Z 3152ef80 f   DirectionalBlender.obj
 0001:0002f910       ?Execute@COperatorQueue@@UAE_NABUSAnimationPoseModifierParams@@@Z 31530910 f   OperatorQueue.obj
 0001:000306f0       ??1COperatorQueue@@MAE@XZ  315316f0 f   OperatorQueue.obj
 0001:00030790       ?GetFactory@COperatorQueue@@UBEPAUICryFactory@@XZ 31531790 f i OperatorQueue.obj
 0001:000307a0       ?GetMemoryUsage@COperatorQueue@@UBEXPAVICrySizer@@@Z 315317a0 f i OperatorQueue.obj
 0001:000307c0       ??$Op@$$CBVCOperatorQueue@@@?$InterfaceCast@U?$Typelist@UIAnimationPoseModifier@@U?$Typelist@UIAnimationOperatorQueue@@VNullType@TL@@@TL@@@TL@@@CW@@SAPAXPBVCOperatorQueue@@ABUCryGUID@@@Z 315317c0 f i OperatorQueue.obj
 0001:00030820       ?QueryInterface@COperatorQueue@@MBEPAXABUCryGUID@@@Z 31531820 f i OperatorQueue.obj
 0001:00030860       ?Op@?$FillIIDs@U?$Typelist@UICryUnknown@@U?$Typelist@UIAnimationPoseModifier@@U?$Typelist@UIAnimationOperatorQueue@@VNullType@TL@@@TL@@@TL@@@TL@@@CW@@SAXPAUCryGUID@@@Z 31531860 f i OperatorQueue.obj
 0001:000308e0       ?GetClassName@CFactory@COperatorQueue@@UBEPBDXZ 315318e0 f i OperatorQueue.obj
 0001:000308f0       ?GetClassID@CFactory@COperatorQueue@@UBEABUCryGUID@@XZ 315318f0 f i OperatorQueue.obj
 0001:00030900       ??_Ebad_alloc@std@@UAEPAXI@Z 31531900 f i OperatorQueue.obj
 0001:00030900       ??_Gbad_alloc@std@@UAEPAXI@Z 31531900 f i OperatorQueue.obj
 0001:00030930       ??$throw_exception@Vbad_alloc@std@@@boost@@YAXABVbad_alloc@std@@@Z 31531930 f i OperatorQueue.obj
 0001:00030960       ?dispose@?$sp_counted_impl_p@VCEngineModule_CryAnimation@@@detail@boost@@UAEXXZ 31531960 f i AnimationBase.obj
 0001:00030960       ?dispose@?$sp_counted_impl_p@VCPoseBlenderAim@@@detail@boost@@UAEXXZ 31531960 f i PoseBlenderAim.obj
 0001:00030960       ?dispose@?$sp_counted_impl_p@VCOperatorQueue@@@detail@boost@@UAEXXZ 31531960 f i OperatorQueue.obj
 0001:00030960       ?dispose@?$sp_counted_impl_p@VCPoseBlenderLook@@@detail@boost@@UAEXXZ 31531960 f i PoseBlenderLook.obj
 0001:00030960       ?dispose@?$sp_counted_impl_p@VCFeetPoseRestore@@@detail@boost@@UAEXXZ 31531960 f i FeetLock.obj
 0001:00030960       ?dispose@?$sp_counted_impl_p@VCFeetPoseStore@@@detail@boost@@UAEXXZ 31531960 f i FeetLock.obj
 0001:00030960       ?dispose@?$sp_counted_impl_p@VCRecoil@PoseModifier@@@detail@boost@@UAEXXZ 31531960 f i Recoil.obj
 0001:00030960       ?dispose@?$sp_counted_impl_p@VCLimbIk@@@detail@boost@@UAEXXZ 31531960 f i LimbIk.obj
 0001:00030960       ?dispose@?$sp_counted_impl_p@VCPoseMatching@@@detail@boost@@UAEXXZ 31531960 f i PoseMatching.obj
 0001:00030960       ?dispose@?$sp_counted_impl_p@VCGroundAlignment@@@detail@boost@@UAEXXZ 31531960 f i GroundAlignment.obj
 0001:00030960       ?dispose@?$sp_counted_impl_p@VCPoseAlignerChain@@@detail@boost@@UAEXXZ 31531960 f i PoseAlignerChain.obj
 0001:00030970       ??1?$shared_ptr@UIAnimationPoseModifier@@@boost@@QAE@XZ 31531970 f i TransitionQueue.obj
 0001:00030970       ??1?$shared_ptr@UIAnimationPoseBlenderDir@@@boost@@QAE@XZ 31531970 f i SkeletonPose.obj
 0001:00030970       ??1?$shared_ptr@UICryUnknown@@@boost@@QAE@XZ 31531970 f i OperatorQueue.obj
 0001:000309b0       ??_ECFactory@CPoseMatching@@UAEPAXI@Z 315319b0 f i PoseMatching.obj
 0001:000309b0       ??_ECFactory@COperatorQueue@@UAEPAXI@Z 315319b0 f i OperatorQueue.obj
 0001:000309b0       ??_ECFactory@CFeetPoseRestore@@UAEPAXI@Z 315319b0 f i FeetLock.obj
 0001:000309b0       ??_ECFactory@CPoseBlenderLook@@UAEPAXI@Z 315319b0 f i PoseBlenderLook.obj
 0001:000309b0       ??_GCFactory@COperatorQueue@@UAEPAXI@Z 315319b0 f i OperatorQueue.obj
 0001:000309b0       ??_ECFactory@CPoseBlenderAim@@UAEPAXI@Z 315319b0 f i PoseBlenderAim.obj
 0001:000309b0       ??_GCFactory@CPoseBlenderAim@@UAEPAXI@Z 315319b0 f i PoseBlenderAim.obj
 0001:000309b0       ??_ECFactory@CLimbIk@@UAEPAXI@Z 315319b0 f i LimbIk.obj
 0001:000309b0       ??_GCFactory@CFeetPoseStore@@UAEPAXI@Z 315319b0 f i FeetLock.obj
 0001:000309b0       ??_EICryFactory@@MAEPAXI@Z 315319b0 f i OperatorQueue.obj
 0001:000309b0       ??_ECFactory@CGroundAlignment@@UAEPAXI@Z 315319b0 f i GroundAlignment.obj
 0001:000309b0       ??_GCFactory@CPoseBlenderLook@@UAEPAXI@Z 315319b0 f i PoseBlenderLook.obj
 0001:000309b0       ??_GCFactory@CPoseMatching@@UAEPAXI@Z 315319b0 f i PoseMatching.obj
 0001:000309b0       ??_GCFactory@CLimbIk@@UAEPAXI@Z 315319b0 f i LimbIk.obj
 0001:000309b0       ??_GICryFactory@@MAEPAXI@Z 315319b0 f i OperatorQueue.obj
 0001:000309b0       ??_GCFactory@CFeetPoseRestore@@UAEPAXI@Z 315319b0 f i FeetLock.obj
 0001:000309b0       ??_GCFactory@CRecoil@PoseModifier@@UAEPAXI@Z 315319b0 f i Recoil.obj
 0001:000309b0       ??_GCFactory@CGroundAlignment@@UAEPAXI@Z 315319b0 f i GroundAlignment.obj
 0001:000309b0       ??_ECFactory@CPoseAlignerChain@@UAEPAXI@Z 315319b0 f i PoseAlignerChain.obj
 0001:000309b0       ??_GCFactory@CPoseAlignerChain@@UAEPAXI@Z 315319b0 f i PoseAlignerChain.obj
 0001:000309b0       ??_ECFactory@CFeetPoseStore@@UAEPAXI@Z 315319b0 f i FeetLock.obj
 0001:000309b0       ??_ECFactory@CRecoil@PoseModifier@@UAEPAXI@Z 315319b0 f i Recoil.obj
 0001:000309e0       ??$?0VCPoseBlenderAim@@@shared_count@detail@boost@@QAE@PAVCPoseBlenderAim@@@Z 315319e0 f i PoseBlenderAim.obj
 0001:000309e0       ??$?0VCPoseMatching@@@shared_count@detail@boost@@QAE@PAVCPoseMatching@@@Z 315319e0 f i PoseMatching.obj
 0001:000309e0       ??$?0VCRecoil@PoseModifier@@@shared_count@detail@boost@@QAE@PAVCRecoil@PoseModifier@@@Z 315319e0 f i Recoil.obj
 0001:000309e0       ??$?0VCPoseAlignerChain@@@shared_count@detail@boost@@QAE@PAVCPoseAlignerChain@@@Z 315319e0 f i PoseAlignerChain.obj
 0001:000309e0       ??$?0VCPoseBlenderLook@@@shared_count@detail@boost@@QAE@PAVCPoseBlenderLook@@@Z 315319e0 f i PoseBlenderLook.obj
 0001:000309e0       ??$?0VCGroundAlignment@@@shared_count@detail@boost@@QAE@PAVCGroundAlignment@@@Z 315319e0 f i GroundAlignment.obj
 0001:000309e0       ??$?0VCLimbIk@@@shared_count@detail@boost@@QAE@PAVCLimbIk@@@Z 315319e0 f i LimbIk.obj
 0001:000309e0       ??$?0VCFeetPoseRestore@@@shared_count@detail@boost@@QAE@PAVCFeetPoseRestore@@@Z 315319e0 f i FeetLock.obj
 0001:000309e0       ??$?0VCOperatorQueue@@@shared_count@detail@boost@@QAE@PAVCOperatorQueue@@@Z 315319e0 f i OperatorQueue.obj
 0001:000309e0       ??$?0VCFeetPoseStore@@@shared_count@detail@boost@@QAE@PAVCFeetPoseStore@@@Z 315319e0 f i FeetLock.obj
 0001:00030a60       ??_GCOperatorQueue@@MAEPAXI@Z 31531a60 f i OperatorQueue.obj
 0001:00030a60       ??_ECOperatorQueue@@MAEPAXI@Z 31531a60 f i OperatorQueue.obj
 0001:00030a90       ?reserve@?$_Impl_vector@USOp@COperatorQueue@@V?$allocator@USOp@COperatorQueue@@@stlpmtx_std@@@priv@stlpmtx_std@@QAEXI@Z 31531a90 f i OperatorQueue.obj
 0001:00030b60       ??0COperatorQueue@@IAE@XZ  31531b60 f   OperatorQueue.obj
 0001:00030c20       ?PushPosition@COperatorQueue@@UAEXIW4EOp@IAnimationOperatorQueue@@ABU?$Vec3_tpl@M@@@Z 31531c20 f   OperatorQueue.obj
 0001:00030cd0       ?PushOrientation@COperatorQueue@@UAEXIW4EOp@IAnimationOperatorQueue@@ABU?$Quat_tpl@M@@@Z 31531cd0 f   OperatorQueue.obj
 0001:00030d80       ?PushStoreRelative@COperatorQueue@@UAEXIAAU?$QuatT_tpl@M@@@Z 31531d80 f   OperatorQueue.obj
 0001:00030e00       ?PushStoreAbsolute@COperatorQueue@@UAEXIAAU?$QuatT_tpl@M@@@Z 31531e00 f   OperatorQueue.obj
 0001:00030e80       ?PushComputeAbsolute@COperatorQueue@@UAEXXZ 31531e80 f   OperatorQueue.obj
 0001:00030f00       ?Clear@COperatorQueue@@UAEXXZ 31531f00 f   OperatorQueue.obj
 0001:00030f50       ?Prepare@COperatorQueue@@UAE_NABUSAnimationPoseModifierParams@@@Z 31531f50 f   OperatorQueue.obj
 0001:00030fb0       ?Synchronize@COperatorQueue@@UAEXXZ 31531fb0 f   OperatorQueue.obj
 0001:00031000       ?CreateClassInstance@CFactory@COperatorQueue@@UBE?AV?$shared_ptr@UICryUnknown@@@boost@@XZ 31532000 f i OperatorQueue.obj
 0001:000310a0       ?Initialize@CPoseAlignerChain@@UAEXW4EType@IAnimationPoseAlignerChain@@PBDH@Z 315320a0 f   PoseAlignerChain.obj
 0001:000310d0       ?Ray_Plane@Intersect@@YA_NABURay@@ABU?$Plane_tpl@M@@AAU?$Vec3_tpl@M@@_N@Z 315320d0 f i PoseAlignerChain.obj
 0001:00031200       ?GetFactory@CPoseAlignerChain@@UBEPAUICryFactory@@XZ 31532200 f i PoseAlignerChain.obj
 0001:00031210       ?SetTarget@CPoseAlignerChain@@UAEXABU?$Plane_tpl@M@@MMMM@Z 31532210 f i PoseAlignerChain.obj
 0001:00031260       ?GetMemoryUsage@CPoseAlignerChain@@UBEXPAVICrySizer@@@Z 31532260 f i PoseAlignerChain.obj
 0001:00031280       ??$Op@$$CBVCPoseAlignerChain@@@?$InterfaceCast@U?$Typelist@UIAnimationPoseModifier@@U?$Typelist@UIAnimationPoseAlignerChain@@VNullType@TL@@@TL@@@TL@@@CW@@SAPAXPBVCPoseAlignerChain@@ABUCryGUID@@@Z 31532280 f i PoseAlignerChain.obj
 0001:000312e0       ?AlignToTarget@CPoseAlignerChain@@AAEXABUSAnimationPoseModifierParams@@@Z 315322e0 f   PoseAlignerChain.obj
 0001:00032350       ?MoveToTarget@CPoseAlignerChain@@AAE_NABUSAnimationPoseModifierParams@@AAU?$Vec3_tpl@M@@@Z 31533350 f   PoseAlignerChain.obj
 0001:000327c0       ?Execute@CPoseAlignerChain@@UAE_NABUSAnimationPoseModifierParams@@@Z 315337c0 f   PoseAlignerChain.obj
 0001:00034350       ?QueryInterface@CPoseAlignerChain@@MBEPAXABUCryGUID@@@Z 31535350 f i PoseAlignerChain.obj
 0001:00034390       ?Prepare@CPoseAlignerChain@@UAE_NABUSAnimationPoseModifierParams@@@Z 31535390 f   PoseAlignerChain.obj
 0001:00034420       ?Op@?$FillIIDs@U?$Typelist@UICryUnknown@@U?$Typelist@UIAnimationPoseModifier@@U?$Typelist@UIAnimationPoseAlignerChain@@VNullType@TL@@@TL@@@TL@@@TL@@@CW@@SAXPAUCryGUID@@@Z 31535420 f i PoseAlignerChain.obj
 0001:000344a0       ?GetClassName@CFactory@CPoseAlignerChain@@UBEPBDXZ 315354a0 f i PoseAlignerChain.obj
 0001:000344b0       ?GetClassID@CFactory@CPoseAlignerChain@@UBEABUCryGUID@@XZ 315354b0 f i PoseAlignerChain.obj
 0001:000344c0       ?CreateClassInstance@CFactory@CPoseAlignerChain@@UBE?AV?$shared_ptr@UICryUnknown@@@boost@@XZ 315354c0 f i PoseAlignerChain.obj
 0001:00034560       ?SetAnimations@CPoseMatching@@UAEXPBII@Z 31535560 f   PoseMatching.obj
 0001:00034580       ?GetMatchingAnimation@CPoseMatching@@UBE_NAAI@Z 31535580 f   PoseMatching.obj
 0001:000345a0       ?Prepare@CPoseMatching@@UAE_NABUSAnimationPoseModifierParams@@@Z 315355a0 f   PoseMatching.obj
 0001:000345b0       ??$?0M@?$Ang3_tpl@M@@QAE@ABU?$Quat_tpl@M@@@Z 315355b0 f i PoseMatching.obj
 0001:00034700       ?GetFactory@CPoseMatching@@UBEPAUICryFactory@@XZ 31535700 f i PoseMatching.obj
 0001:00034710       ?GetMemoryUsage@?$CKeyTimesInformationStartStop@MUF32StartStopEncoder@@@@UBEXPAVICrySizer@@@Z 31535710 f i ControllerPQ.obj
 0001:00034710       ?GetMemoryUsage@CPoseMatching@@UBEXPAVICrySizer@@@Z 31535710 f i PoseMatching.obj
 0001:00034730       ?get_deleter@?$sp_counted_impl_p@VCRecoil@PoseModifier@@@detail@boost@@UAEPAXABVsp_typeinfo@23@@Z 31535730 f i Recoil.obj
 0001:00034730       ?QueryComposite@CPoseBlenderLook@@MBEPAXPBD@Z 31535730 f i PoseBlenderLook.obj
 0001:00034730       ?GetParamInt@CFacialEffector@@UAEHW4EFacialEffectorParam@@@Z 31535730 f i FaceEffector.obj
 0001:00034730       ?Allocate@CPool@Memory@@UAEPAXI@Z 31535730 f i Pool.obj
 0001:00034730       ?SetBoneName@CAttachmentFACE@@UAEIPBD@Z 31535730 f i AttachmentManager.obj
 0001:00034730       ?get_deleter@?$sp_counted_impl_p@VCPoseBlenderAim@@@detail@boost@@UAEPAXABVsp_typeinfo@23@@Z 31535730 f i PoseBlenderAim.obj
 0001:00034730       ?QueryComposite@CFeetPoseRestore@@MBEPAXPBD@Z 31535730 f i FeetLock.obj
 0001:00034730       ?get_deleter@?$sp_counted_impl_p@VCEngineModule_CryAnimation@@@detail@boost@@UAEPAXABVsp_typeinfo@23@@Z 31535730 f i AnimationBase.obj
 0001:00034730       ?QueryComposite@CFeetPoseStore@@MBEPAXPBD@Z 31535730 f i FeetLock.obj
 0001:00034730       ?get_deleter@?$sp_counted_impl_p@VCFeetPoseStore@@@detail@boost@@UAEPAXABVsp_typeinfo@23@@Z 31535730 f i FeetLock.obj
 0001:00034730       ?get_deleter@?$sp_counted_impl_p@VCPoseBlenderLook@@@detail@boost@@UAEPAXABVsp_typeinfo@23@@Z 31535730 f i PoseBlenderLook.obj
 0001:00034730       ?QueryComposite@CGroundAlignment@@MBEPAXPBD@Z 31535730 f i GroundAlignment.obj
 0001:00034730       ?QueryComposite@CPoseBlenderAim@@MBEPAXPBD@Z 31535730 f i PoseBlenderAim.obj
 0001:00034730       ?QueryComposite@CPoseAlignerChain@@MBEPAXPBD@Z 31535730 f i PoseAlignerChain.obj
 0001:00034730       ?get_deleter@?$sp_counted_impl_p@VCLimbIk@@@detail@boost@@UAEPAXABVsp_typeinfo@23@@Z 31535730 f i LimbIk.obj
 0001:00034730       ?QueryComposite@CLimbIk@@MBEPAXPBD@Z 31535730 f i LimbIk.obj
 0001:00034730       ?QueryComposite@CRecoil@PoseModifier@@MBEPAXPBD@Z 31535730 f i Recoil.obj
 0001:00034730       ?SetBoneName@CAttachmentSKIN@@UAEIPBD@Z 31535730 f i Attachment.obj
 0001:00034730       ?get_deleter@?$sp_counted_impl_p@VCPoseAlignerChain@@@detail@boost@@UAEPAXABVsp_typeinfo@23@@Z 31535730 f i PoseAlignerChain.obj
 0001:00034730       ?QueryComposite@CEngineModule_CryAnimation@@MBEPAXPBD@Z 31535730 f i AnimationBase.obj
 0001:00034730       ?get_deleter@?$sp_counted_impl_p@VCPoseMatching@@@detail@boost@@UAEPAXABVsp_typeinfo@23@@Z 31535730 f i PoseMatching.obj
 0001:00034730       ?QueryComposite@COperatorQueue@@MBEPAXPBD@Z 31535730 f i OperatorQueue.obj
 0001:00034730       ?get_deleter@?$sp_counted_impl_p@VCGroundAlignment@@@detail@boost@@UAEPAXABVsp_typeinfo@23@@Z 31535730 f i GroundAlignment.obj
 0001:00034730       ?get_deleter@?$sp_counted_impl_p@VCFeetPoseRestore@@@detail@boost@@UAEPAXABVsp_typeinfo@23@@Z 31535730 f i FeetLock.obj
 0001:00034730       ?get_deleter@?$sp_counted_impl_p@VCOperatorQueue@@@detail@boost@@UAEPAXABVsp_typeinfo@23@@Z 31535730 f i OperatorQueue.obj
 0001:00034730       ?QueryComposite@CPoseMatching@@MBEPAXPBD@Z 31535730 f i PoseMatching.obj
 0001:00034740       ??$Op@$$CBVCPoseMatching@@@?$InterfaceCast@U?$Typelist@UIAnimationPoseModifier@@U?$Typelist@UIAnimationPoseMatching@@VNullType@TL@@@TL@@@TL@@@CW@@SAPAXPBVCPoseMatching@@ABUCryGUID@@@Z 31535740 f i PoseMatching.obj
 0001:000347a0       ?Execute@CPoseMatching@@UAE_NABUSAnimationPoseModifierParams@@@Z 315357a0 f   PoseMatching.obj
 0001:00035820       ?QueryInterface@CPoseMatching@@MBEPAXABUCryGUID@@@Z 31536820 f i PoseMatching.obj
 0001:00035860       ?Op@?$FillIIDs@U?$Typelist@UICryUnknown@@U?$Typelist@UIAnimationPoseModifier@@U?$Typelist@UIAnimationPoseMatching@@VNullType@TL@@@TL@@@TL@@@TL@@@CW@@SAXPAUCryGUID@@@Z 31536860 f i PoseMatching.obj
 0001:000358e0       ?GetClassName@CFactory@CPoseMatching@@UBEPBDXZ 315368e0 f i PoseMatching.obj
 0001:000358f0       ?GetClassID@CFactory@CPoseMatching@@UBEABUCryGUID@@XZ 315368f0 f i PoseMatching.obj
 0001:00035900       ?CreateClassInstance@CFactory@CPoseMatching@@UBE?AV?$shared_ptr@UICryUnknown@@@boost@@XZ 31536900 f i PoseMatching.obj
 0001:000359b0       ?NTime2KTime@GlobalAnimationHeaderCAF@@QAEMM@Z 315369b0 f i SkeletonAnim_Locator.obj
 0001:000359f0       ?ParseLayer0@CSkeletonAnim@@ABEXABVCAnimation@@PAUAnimInfo@@AAIMI@Z 315369f0 f   SkeletonAnim_Locator.obj
 0001:00035fa0       ?GetRootController@CSkeletonAnim@@ABEPAVIController@@AAUGlobalAnimationHeaderCAF@@@Z 31536fa0 f   SkeletonAnim_Locator.obj
 0001:00036090       ?Extract_DeltaMovement@CSkeletonAnim@@ABEXPAUAnimInfo@@AAIPAUSDeltaMotion@@M@Z 31537090 f   SkeletonAnim_Locator.obj
 0001:0003b390       ?CalculateRelativeMovement@CSkeletonAnim@@UBE?AU?$QuatT_tpl@M@@M_N@Z 3153c390 f   SkeletonAnim_Locator.obj
 0001:0003bd80       ?GetJointCount@CSkeletonPhysics@@ABEIXZ 3153cd80 f   SkeletonPhysics.obj
 0001:0003bd90       ?SetAuxParams@CSkeletonPhysics@@QAEXPAUpe_params@@@Z 3153cd90 f   SkeletonPhysics.obj
 0001:0003bdd0       ?GetCharacterPhysics@CSkeletonPhysics@@QAEPAUIPhysicalEntity@@PBD@Z 3153cdd0 f   SkeletonPhysics.obj
 0001:0003be30       ?GetCharacterPhysics@CSkeletonPhysics@@QAEPAUIPhysicalEntity@@H@Z 3153ce30 f   SkeletonPhysics.obj
 0001:0003be60       ??_GSBatchUpdateValidator@@UAEPAXI@Z 3153ce60 f i SkeletonPhysics.obj
 0001:0003be60       ??_ESBatchUpdateValidator@@UAEPAXI@Z 3153ce60 f i SkeletonPhysics.obj
 0001:0003bed0       ?Initialize@CSkeletonPhysics@@QAE_NAAVCSkeletonPose@@@Z 3153ced0 f   SkeletonPhysics.obj
 0001:0003bf30       ?GetPoseData@CSkeletonPhysics@@ABEABVCPoseData@Skeleton@@XZ 3153cf30 f   SkeletonPhysics.obj
 0001:0003bf40       ?SetPhysEntOnJoint@CSkeletonPhysics@@QAEXHPAUIPhysicalEntity@@@Z 3153cf40 f   SkeletonPhysics.obj
 0001:0003c020       ?DestroyPhysics@CSkeletonPhysics@@QAEXXZ 3153d020 f   SkeletonPhysics.obj
 0001:0003c110       ?getBonePhysParentOrSelfIndex@CSkeletonPhysics@@QAEHHH@Z 3153d110 f   SkeletonPhysics.obj
 0001:0003c170       ?getBonePhysChildIndex@CSkeletonPhysics@@AAEHHH@Z 3153d170 f   SkeletonPhysics.obj
 0001:0003c1e0       ?GetBoneSurfaceTypeId@CSkeletonPhysics@@QAEHHH@Z 3153d1e0 f   SkeletonPhysics.obj
 0001:0003c220       ?TranslatePartIdToDeadBody@CSkeletonPhysics@@QAEHH@Z 3153d220 f   SkeletonPhysics.obj
 0001:0003c280       ?ParsePhysInfoProps@@YAXPAVCModelJoint@@HAAUpe_params_rope@@AAUpe_simulation_params@@AAUpe_params_flags@@@Z 3153d280 f   SkeletonPhysics.obj
 0001:0003c420       ??0?$Matrix34_tpl@M@@QAE@ABU?$Vec3_tpl@M@@ABU?$Quat_tpl@M@@0@Z 3153d420 f i SkeletonPhysics.obj
 0001:0003c590       ??$?0M@?$Ang3_tpl@M@@QAE@ABU?$Matrix33_tpl@M@@@Z 3153d590 f i SkeletonPhysics.obj
 0001:0003c660       ??0pe_params_part@@QAE@XZ  3153d660 f i SkeletonPhysics.obj
 0001:0003c720       ??0pe_params_joint@@QAE@XZ 3153d720 f i SkeletonPhysics.obj
 0001:0003c830       ??0pe_params_articulated_body@@QAE@XZ 3153d830 f i SkeletonPhysics.obj
 0001:0003c930       ??0pe_params_rope@@QAE@XZ  3153d930 f i SkeletonPhysics.obj
 0001:0003cb10       ??0pe_params_softbody@@QAE@XZ 3153db10 f i SkeletonPhysics.obj
 0001:0003cc40       ??0pe_action_impulse@@QAE@XZ 3153dc40 f i SkeletonPhysics.obj
 0001:0003cca0       ??0pe_articgeomparams@@QAE@XZ 3153dca0 f i SkeletonPhysics.obj
 0001:0003cd30       ??0SBatchUpdateValidator@@QAE@XZ 3153dd30 f i SkeletonPhysics.obj
 0001:0003cdb0       ?Lock@SBatchUpdateValidator@@UAE_NXZ 3153ddb0 f i SkeletonPhysics.obj
 0001:0003ce00       ?Unlock@SBatchUpdateValidator@@UAEXXZ 3153de00 f i SkeletonPhysics.obj
 0001:0003ce40       ??$move_init@H@NArray@@YAXPAH0I@Z 3153de40 f i SkeletonPhysics.obj
 0001:0003ce40       ??$move_init@PAVCAnimationSet@@@NArray@@YAXPAPAVCAnimationSet@@0I@Z 3153de40 f i ModelAnimationSet.obj
 0001:0003ce40       ??$move_init@PAVCAttachmentSKIN@@@NArray@@YAXPAPAVCAttachmentSKIN@@0I@Z 3153de40 f i ModelSkin.obj
 0001:0003ce40       ??$move_init@UCControllerType@@@NArray@@YAXPAUCControllerType@@0I@Z 3153de40 f i LoaderCGA.obj
 0001:0003ce40       ??$move_init@PAU?$DynArray@UCryTCB3Key@@HU?$SmallDynStorage@UCryTCB3Key@@HUStandardAlloc@NAlloc@@@NArray@@@@@NArray@@YAXPAPAU?$DynArray@UCryTCB3Key@@HU?$SmallDynStorage@UCryTCB3Key@@HUStandardAlloc@NAlloc@@@NArray@@@@0I@Z 3153de40 f i LoaderTCB.obj
 0001:0003ce40       ??$move_init@I@NArray@@YAXPAI0I@Z 3153de40 f i CharacterManager.obj
 0001:0003ce40       ??$move_init@PAVCCharInstance@@@NArray@@YAXPAPAVCCharInstance@@0I@Z 3153de40 f i Model.obj
 0001:0003ce40       ??$move_init@PAU?$DynArray@UCryTCBQKey@@HU?$SmallDynStorage@UCryTCBQKey@@HUStandardAlloc@NAlloc@@@NArray@@@@@NArray@@YAXPAPAU?$DynArray@UCryTCBQKey@@HU?$SmallDynStorage@UCryTCBQKey@@HUStandardAlloc@NAlloc@@@NArray@@@@0I@Z 3153de40 f i LoaderTCB.obj
 0001:0003ce80       ?GetPhysIdOnJoint@CSkeletonPhysics@@QAEHH@Z 3153de80 f   SkeletonPhysics.obj
 0001:0003ced0       ?BuildPhysicalEntity@CSkeletonPhysics@@QAEXPAUIPhysicalEntity@@MHMHHABU?$Matrix34_tpl@M@@@Z 3153ded0 f   SkeletonPhysics.obj
 0001:0003e560       ?DestroyCharacterPhysics@CSkeletonPhysics@@QAEXH@Z 3153f560 f   SkeletonPhysics.obj
 0001:0003e7d0       ?CreateCharacterPhysics@CSkeletonPhysics@@QAEPAUIPhysicalEntity@@PAU2@MHMHABU?$Matrix34_tpl@M@@@Z 3153f7d0 f   SkeletonPhysics.obj
 0001:0003ed30       ?AddImpact@CSkeletonPhysics@@QAE_NHU?$Vec3_tpl@M@@0@Z 3153fd30 f   SkeletonPhysics.obj
 0001:0003ef10       ?Physics_SynchronizeToImpact@CSkeletonPhysics@@AAEXM@Z 3153ff10 f   SkeletonPhysics.obj
 0001:0003f1c0       ?SynchronizeWithPhysicsPost@CSkeletonPhysics@@QAEXXZ 315401c0 f   SkeletonPhysics.obj
 0001:0003f350       ?FindSpineBones@CSkeletonPhysics@@AAEXXZ 31540350 f   SkeletonPhysics.obj
 0001:0003f400       ?GoLimp@CSkeletonPhysics@@QAEXXZ 31540400 f   SkeletonPhysics.obj
 0001:0003f4c0       ?GetFallingDir@CSkeletonPhysics@@QAEHXZ 315404c0 f   SkeletonPhysics.obj
 0001:0003fc30       ??0CPhysicsJoint@@QAE@ABU0@@Z 31540c30 f i SkeletonPhysics.obj
 0001:0003fcb0       ?resize_raw@?$SmallDynStorage@HHUStandardAlloc@NAlloc@@@NArray@@QAEXHH_N@Z 31540cb0 f i SkeletonPhysics.obj
 0001:0003fe00       ?CreateAuxilaryPhysics@CSkeletonPhysics@@QAEHPAUIPhysicalEntity@@ABU?$Matrix34_tpl@M@@MU?$Vec3_tpl@M@@H@Z 31540e00 f   SkeletonPhysics.obj
 0001:000428d0       ?Physics_SynchronizeToAux@CSkeletonPhysics@@AAEXABVCPoseData@Skeleton@@@Z 315438d0 f   SkeletonPhysics.obj
 0001:00043440       ?Physics_SynchronizeToEntity@CSkeletonPhysics@@AAEXAAUIPhysicalEntity@@U?$QuatT_tpl@M@@@Z 31544440 f   SkeletonPhysics.obj
 0001:00043a50       ?Physics_SynchronizeToEntityArticulated@CSkeletonPhysics@@AAEXM@Z 31544a50 f   SkeletonPhysics.obj
 0001:00043e50       ?init@?$DynArray@UCPhysicsJoint@@HU?$SmallDynStorage@UCPhysicsJoint@@HUStandardAlloc@NAlloc@@@NArray@@@@KAPAUCPhysicsJoint@@U?$Array@UCPhysicsJoint@@HU?$ArrayStorage@UCPhysicsJoint@@H@NArray@@@@@Z 31544e50 f i SkeletonPhysics.obj
 0001:00043ef0       ?set_size@?$SmallDynStorage@U?$QuatT_tpl@M@@HUStandardAlloc@NAlloc@@@NArray@@QAEXH@Z 31544ef0 f i SkeletonPhysics.obj
 0001:00043ef0       ?set_size@?$SmallDynStorage@VCModelMesh@@HUStandardAlloc@NAlloc@@@NArray@@QAEXH@Z 31544ef0 f i LoaderSKIN.obj
 0001:00043ef0       ?set_size@?$SmallDynStorage@UVirtualExampleInit2@CHUNK_GAHAIM_INFO@@HUStandardAlloc@NAlloc@@@NArray@@QAEXH@Z 31544ef0 f i CharacterManager.obj
 0001:00043f90       ?expand_raw@?$DynArray@HHU?$SmallDynStorage@HHUStandardAlloc@NAlloc@@@NArray@@@@IAEPAHPAHH@Z 31544f90 f i SkeletonPhysics.obj
 0001:00044010       ??$move_init@U?$QuatT_tpl@M@@@NArray@@YAXPAU?$QuatT_tpl@M@@0I@Z 31545010 f i SkeletonPhysics.obj
 0001:000441a0       ?CreateAuxilaryPhysics@CSkeletonPhysics@@QAEHPAUIPhysicalEntity@@ABU?$Matrix34_tpl@M@@H@Z 315451a0 f   SkeletonPhysics.obj
 0001:00044210       ?SynchronizeWithPhysicalEntity@CSkeletonPhysics@@QAEXAAVCPoseData@Skeleton@@PAUIPhysicalEntity@@ABU?$Vec3_tpl@M@@ABU?$Quat_tpl@M@@U?$QuatT_tpl@M@@H@Z 31545210 f   SkeletonPhysics.obj
 0001:000442f0       ?SynchronizeWithPhysicalEntity@CSkeletonPhysics@@QAEXPAUIPhysicalEntity@@ABU?$Vec3_tpl@M@@ABU?$Quat_tpl@M@@@Z 315452f0 f   SkeletonPhysics.obj
 0001:000443b0       ?ProcessPhysics@CSkeletonPhysics@@AAEXAAVCPoseData@Skeleton@@MPAUSCharUpdateFeedback@@@Z 315453b0 f   SkeletonPhysics.obj
 0001:00044490       ?SynchronizeWithPhysics@CSkeletonPhysics@@QAEXAAVCPoseData@Skeleton@@@Z 31545490 f   SkeletonPhysics.obj
 0001:00044640       ?resize_raw@?$SmallDynStorage@U?$QuatT_tpl@M@@HUStandardAlloc@NAlloc@@@NArray@@QAEXHH_N@Z 31545640 f i SkeletonPhysics.obj
 0001:000447b0       ??$move_init@UCPhysicsJoint@@@NArray@@YAXPAUCPhysicsJoint@@0I@Z 315457b0 f i SkeletonPhysics.obj
 0001:000447f0       ?expand_raw@?$DynArray@U?$QuatT_tpl@M@@HU?$SmallDynStorage@U?$QuatT_tpl@M@@HUStandardAlloc@NAlloc@@@NArray@@@@IAEPAU?$QuatT_tpl@M@@PAU2@H@Z 315457f0 f i SkeletonPhysics.obj
 0001:00044890       ?resize_raw@?$SmallDynStorage@UCPhysicsJoint@@HUStandardAlloc@NAlloc@@@NArray@@QAEXHH_N@Z 31545890 f i SkeletonPhysics.obj
 0001:000449f0       ??1CSkeletonPhysics@@QAE@XZ 315459f0 f   SkeletonPhysics.obj
 0001:00044af0       ?resize@?$DynArray@HHU?$SmallDynStorage@HHUStandardAlloc@NAlloc@@@NArray@@@@QAEXH@Z 31545af0 f i SkeletonPhysics.obj
 0001:00044b30       ?expand_raw@?$DynArray@UCPhysicsJoint@@HU?$SmallDynStorage@UCPhysicsJoint@@HUStandardAlloc@NAlloc@@@NArray@@@@IAEPAUCPhysicsJoint@@PAU2@H@Z 31545b30 f i SkeletonPhysics.obj
 0001:00044bc0       ??0CSkeletonPhysics@@QAE@XZ 31545bc0 f   SkeletonPhysics.obj
 0001:00044e10       ?InitializeAnimToPhysIndexArray@CSkeletonPhysics@@QAEXXZ 31545e10 f   SkeletonPhysics.obj
 0001:00044f30       ?InitPhysicsSkeleton@CSkeletonPhysics@@QAEXXZ 31545f30 f   SkeletonPhysics.obj
 0001:00045370       ?RelinquishCharacterPhysics@CSkeletonPhysics@@QAEPAUIPhysicalEntity@@ABU?$Matrix34_tpl@M@@M_NABU?$Vec3_tpl@M@@@Z 31546370 f   SkeletonPhysics.obj
 0001:00046b30       ?BlendFromRagdoll@CSkeletonPhysics@@QAE_NAAU?$QuatTS_tpl@M@@AAPAUIPhysicalEntity@@_N@Z 31547b30 f   SkeletonPhysics.obj
 0001:00048010       ?GetParent@CModelJoint@@QAEPAV1@XZ 31549010 f i SkeletonPhysics_SPU.obj
 0001:00048030       ?getBoneParentIndex@CSkeletonPhysics@@AAEII@Z 31549030 f   SkeletonPhysics_SPU.obj
 0001:00048070       ?ResetNonphysicalBoneRotations@CSkeletonPhysics@@AAEXAAVCPoseData@Skeleton@@HM@Z 31549070 f   SkeletonPhysics_SPU.obj
 0001:00048370       ?getBonePhysParentIndex@CSkeletonPhysics@@QAEHHH@Z 31549370 f   SkeletonPhysics_SPU.obj
 0001:000483f0       ?SPU_Physics_SynchronizeFromEntityPrepare@CSkeletonPhysics@@AAEXAAVCPool@Memory@@PAUIPhysicalEntity@@@Z 315493f0 f   SkeletonPhysics_SPU.obj
 0001:000488b0       ?SPU_Physics_SynchronizeFromAuxPrepare@CSkeletonPhysics@@AAEXAAVCPool@Memory@@@Z 315498b0 f   SkeletonPhysics_SPU.obj
 0001:00048d90       ?SPU_Physics_SynchronizeFromImpactPrepare@CSkeletonPhysics@@AAEXAAVCPool@Memory@@@Z 31549d90 f   SkeletonPhysics_SPU.obj
 0001:00048ef0       ?SPU_SynchronizeWithPhysicsPrepare@CSkeletonPhysics@@QAEXAAVCPool@Memory@@@Z 31549ef0 f   SkeletonPhysics_SPU.obj
 0001:00048fb0       ?DoSetRagdollDefaultPose@CSkeletonPhysics@@AAEXAAVCPoseData@Skeleton@@@Z 31549fb0 f   SkeletonPhysics_SPU.obj
 0001:000496d0       ?UnconvertBoneGlobalFromRelativeForm@CSkeletonPhysics@@AAEXAAVCPoseData@Skeleton@@_NH1@Z 3154a6d0 f   SkeletonPhysics_SPU.obj
 0001:00049a40       ?SPU_Physics_SynchronizeFromEntity@CSkeletonPhysics@@AAEXAAVCPoseData@Skeleton@@PAUIPhysicalEntity@@ABU?$Vec3_tpl@M@@ABU?$Quat_tpl@M@@U?$QuatT_tpl@M@@@Z 3154aa40 f   SkeletonPhysics_SPU.obj
 0001:0004a2f0       ?SPU_Physics_SynchronizeFromAux@CSkeletonPhysics@@AAEXAAVCPoseData@Skeleton@@@Z 3154b2f0 f   SkeletonPhysics_SPU.obj
 0001:0004c280       ?SPU_Physics_SynchronizeFromImpact@CSkeletonPhysics@@AAEXAAVCPoseData@Skeleton@@M@Z 3154d280 f   SkeletonPhysics_SPU.obj
 0001:0004d1e0       ?SPU_Physics_BlendFromRagdoll@CSkeletonPhysics@@AAEXAAVCPoseData@Skeleton@@M@Z 3154e1e0 f   SkeletonPhysics_SPU.obj
 0001:0004d7a0       ?SPU_Physics_SynchronizeFrom@CSkeletonPhysics@@QAEXAAVCPoseData@Skeleton@@M@Z 3154e7a0 f   SkeletonPhysics_SPU.obj
 0001:0004d8e0       ?SetFirstLayer@CTransitionQueue@@QAEXXZ 3154e8e0 f   TransitionQueue.obj
 0001:0004d900       ?IsAnimationLoaded@?A0x020955a7@@YA_NABVCAnimationSet@@ABVCAnimation@@@Z 3154e900 f   TransitionQueue.obj
 0001:0004da50       ?TriggerEvents@?A0x020955a7@@YAXPBDIABUIAnimEventList@@MMAAVCCharInstance@@@Z 3154ea50 f   TransitionQueue.obj
 0001:0004db90       ?GetAnimation@CTransitionQueue@@QAEAAVCAnimation@@I@Z 3154eb90 f   TransitionQueue.obj
 0001:0004db90       ?GetAnimation@CTransitionQueue@@QBEABVCAnimation@@I@Z 3154eb90 f   TransitionQueue.obj
 0001:0004dbc0       ?ApplyManualMixingWeight@CTransitionQueue@@QAEXI@Z 3154ebc0 f   TransitionQueue.obj
 0001:0004dc20       ?TransitionsBetweenSeveralAnimations@CTransitionQueue@@QAEXI@Z 3154ec20 f   TransitionQueue.obj
 0001:0004de50       ?AdjustTransitionWeights@CTransitionQueue@@QAEXI@Z 3154ee50 f   TransitionQueue.obj
 0001:0004e1b0       ?UpdateTransitionTime@CTransitionQueue@@QAEXIMMM@Z 3154f1b0 f   TransitionQueue.obj
 0001:0004e4a0       ?AdjustAnimationTimeForTimeWarpedAnimations@CTransitionQueue@@QAEXI@Z 3154f4a0 f   TransitionQueue.obj
 0001:0004e6c0       ?Prepare@CPoseModifierQueue@@QAEXABUSAnimationPoseModifierParams@@@Z 3154f6c0 f   TransitionQueue.obj
 0001:0004e700       ?Synchronize@CPoseModifierQueue@@QAEXXZ 3154f700 f   TransitionQueue.obj
 0001:0004e740       ?init@?$DynArray@VCAnimation@@HU?$SmallDynStorage@VCAnimation@@HUStandardAlloc@NAlloc@@@NArray@@@@KAPAVCAnimation@@U?$Array@VCAnimation@@HU?$ArrayStorage@VCAnimation@@H@NArray@@@@@Z 3154f740 f i TransitionQueue.obj
 0001:0004e800       ??$move_init@VCAnimation@@@NArray@@YAXPAVCAnimation@@0I@Z 3154f800 f i TransitionQueue.obj
 0001:0004e840       ?UnloadAnimationAssets@CTransitionQueue@@QAEXH@Z 3154f840 f   TransitionQueue.obj
 0001:0004e9f0       ?ManualSeekAnimation@CTransitionQueue@@QAEXIM_NAAVCCharInstance@@@Z 3154f9f0 f   TransitionQueue.obj
 0001:0004eb50       ?get_alloc_size@?$SmallDynStorage@U?$Vec3_tpl@M@@HUStandardAlloc@NAlloc@@@NArray@@QBEHXZ 3154fb50 f i SkeletonPose_Debug.obj
 0001:0004eb50       ?get_alloc_size@?$SmallDynStorage@UModelAnimationHeader@@HUStandardAlloc@NAlloc@@@NArray@@QBEHXZ 3154fb50 f i ModelAnimationSet.obj
 0001:0004eb50       ?get_alloc_size@?$SmallDynStorage@USEntry@CPoseModifierQueue@@HUStandardAlloc@NAlloc@@@NArray@@QBEHXZ 3154fb50 f i TransitionQueue.obj
 0001:0004eb50       ?get_alloc_size@?$SmallDynStorage@URChunk@@HUStandardAlloc@NAlloc@@@NArray@@QBEHXZ 3154fb50 f i ModelMesh.obj
 0001:0004eba0       ?set_size@?$SmallDynStorage@VCAnimation@@HUStandardAlloc@NAlloc@@@NArray@@QAEXH@Z 3154fba0 f i TransitionQueue.obj
 0001:0004ec30       ?destroy@?$DynArray@USEntry@CPoseModifierQueue@@HU?$SmallDynStorage@USEntry@CPoseModifierQueue@@HUStandardAlloc@NAlloc@@@NArray@@@@KAXU?$Array@USEntry@CPoseModifierQueue@@HU?$ArrayStorage@USEntry@CPoseModifierQueue@@H@NArray@@@@@Z 3154fc30 f i TransitionQueue.obj
 0001:0004ec90       ?init@?$DynArray@USEntry@CPoseModifierQueue@@HU?$SmallDynStorage@USEntry@CPoseModifierQueue@@HUStandardAlloc@NAlloc@@@NArray@@@@KAPAUSEntry@CPoseModifierQueue@@U?$Array@USEntry@CPoseModifierQueue@@HU?$ArrayStorage@USEntry@CPoseModifierQueue@@H@NArray@@@@ABU23@@Z 3154fc90 f i TransitionQueue.obj
 0001:0004ece0       ?resize_raw@?$SmallDynStorage@VCAnimation@@HUStandardAlloc@NAlloc@@@NArray@@QAEXHH_N@Z 3154fce0 f i TransitionQueue.obj
 0001:0004ee40       ??$move_init@USEntry@CPoseModifierQueue@@@NArray@@YAXPAUSEntry@CPoseModifierQueue@@0I@Z 3154fe40 f i TransitionQueue.obj
 0001:0004eee0       ?GetSize@CPoseModifierQueue@@QAEIXZ 3154fee0 f   TransitionQueue.obj
 0001:0004ef90       ?erase@?$DynArray@VCAnimation@@HU?$SmallDynStorage@VCAnimation@@HUStandardAlloc@NAlloc@@@NArray@@@@QAEPAVCAnimation@@PAV2@0@Z 3154ff90 f i TransitionQueue.obj
 0001:0004f000       ?resize_raw@?$SmallDynStorage@USEntry@CPoseModifierQueue@@HUStandardAlloc@NAlloc@@@NArray@@QAEXHH_N@Z 31550000 f i TransitionQueue.obj
 0001:0004f160       ?expand_raw@?$DynArray@VCAnimation@@HU?$SmallDynStorage@VCAnimation@@HUStandardAlloc@NAlloc@@@NArray@@@@IAEPAVCAnimation@@PAV2@H@Z 31550160 f i TransitionQueue.obj
 0001:0004f1f0       ?expand_raw@?$DynArray@USEntry@CPoseModifierQueue@@HU?$SmallDynStorage@USEntry@CPoseModifierQueue@@HUStandardAlloc@NAlloc@@@NArray@@@@IAEPAUSEntry@CPoseModifierQueue@@PAU23@H@Z 315501f0 f i TransitionQueue.obj
 0001:0004f280       ??$AddObject@USEntry@CPoseModifierQueue@@HU?$SmallDynStorage@USEntry@CPoseModifierQueue@@HUStandardAlloc@NAlloc@@@NArray@@@ICrySizer@@QAEXABU?$DynArray@USEntry@CPoseModifierQueue@@HU?$SmallDynStorage@USEntry@CPoseModifierQueue@@HUStandardAlloc@NAlloc@@@NArray@@@@@Z 31550280 f i TransitionQueue.obj
 0001:0004f320       ?AddToSizer@CPoseModifierQueue@@QBEXPAVICrySizer@@@Z 31550320 f   TransitionQueue.obj
 0001:0004f350       ?RemoveAnimation@CTransitionQueue@@QAE_NI_N@Z 31550350 f   TransitionQueue.obj
 0001:0004f3c0       ??1CPoseModifierQueue@@QAE@XZ 315503c0 f   TransitionQueue.obj
 0001:0004f470       ?SwapBuffersAndClearActive@CPoseModifierQueue@@QAEXXZ 31550470 f   TransitionQueue.obj
 0001:0004f4e0       ?ClearAllPoseModifiers@CPoseModifierQueue@@QAEXXZ 315504e0 f   TransitionQueue.obj
 0001:0004f590       ??0CTransitionQueue@@QAE@XZ 31550590 f   TransitionQueue.obj
 0001:0004f610       ?RemoveDelayConditions@CTransitionQueue@@QAEXXZ 31550610 f   TransitionQueue.obj
 0001:0004f6e0       ??0CPoseModifierQueue@@QAE@XZ 315506e0 f   TransitionQueue.obj
 0001:0004f7a0       ?PushAnimation@CTransitionQueue@@QAEXABVCAnimation@@@Z 315507a0 f   TransitionQueue.obj
 0001:0004f920       ?Clear@CTransitionQueue@@QAEXXZ 31550920 f   TransitionQueue.obj
 0001:0004f990       ?Push@CPoseModifierQueue@@QAE_NV?$shared_ptr@UIAnimationPoseModifier@@@boost@@PBD_N@Z 31550990 f   TransitionQueue.obj
 0001:0004fad0       ?Initialize@CVertexAnimation@@QAE_NAAVCSkin@@@Z 31550ad0 f   VertexAnimation.obj
 0001:0004fb00       ??$move_init@UProcAdjust@@@NArray@@YAXPAUProcAdjust@@0I@Z 31550b00 f i ParamLoader.obj
 0001:0004fb00       ??$move_init@UBoneIndices8@@@NArray@@YAXPAUBoneIndices8@@0I@Z 31550b00 f i LoaderSKIN.obj
 0001:0004fb00       ??$move_init@UIdxAndName@@@NArray@@YAXPAUIdxAndName@@0I@Z 31550b00 f i ParamLoader.obj
 0001:0004fb00       ??$move_init@USVertexFrameState@@@NArray@@YAXPAUSVertexFrameState@@0I@Z 31550b00 f i VertexAnimation.obj
 0001:0004fb00       ??$move_init@USJointsAimIK_Pos@@@NArray@@YAXPAUSJointsAimIK_Pos@@0I@Z 31550b00 f i ParamLoader.obj
 0001:0004fb40       ?FindMorphTarget@CModelMesh@@QAEHPBD@Z 31550b40 f i VertexAnimation.obj
 0001:0004fba0       ?resize_raw@?$SmallDynStorage@USVertexFrameState@@HUStandardAlloc@NAlloc@@@NArray@@QAEXHH_N@Z 31550ba0 f i VertexAnimation.obj
 0001:0004fcf0       ?ClearAllFramesWeight@CVertexAnimation@@UAEXXZ 31550cf0 f   VertexAnimation.obj
 0001:0004fd30       ??0CVertexAnimation@@QAE@XZ 31550d30 f   VertexAnimation.obj
 0001:0004fd90       ??1CVertexAnimation@@UAE@XZ 31550d90 f   VertexAnimation.obj
 0001:0004fde0       ?SetFrameWeight@CVertexAnimation@@QAEXABUCMorphTarget@@M@Z 31550de0 f   VertexAnimation.obj
 0001:0004fec0       ?SetFrameWeightByName@CVertexAnimation@@UAEXPBDM@Z 31550ec0 f   VertexAnimation.obj
 0001:0004ff30       ??_GCVertexAnimation@@UAEPAXI@Z 31550f30 f i VertexAnimation.obj
 0001:0004ff30       ??_ECVertexAnimation@@UAEPAXI@Z 31550f30 f i VertexAnimation.obj
 0001:0004ffa0       ?Update@CVertexAnimation@@QAE_NAAVCVertexData@@@Z 31550fa0 f   VertexAnimation.obj
 0001:00050110       ?Execute@VertexCommandAdd@@SAXAAU1@PAU?$Vec3_tpl@M@@@Z 31551110 f   VertexCommand.obj
 0001:00050420       ?Process@CVertexCommandBuffer@@QAEXPAU?$Vec3_tpl@M@@@Z 31551420 f   VertexCommandBuffer.obj
 0001:00050470       ?WriteBegin@CVertexData@@QAEPAUSVF_P3F@@XZ 31551470 f   VertexData.obj
 0001:00050490       ?WriteEnd@CVertexData@@QAEXXZ 31551490 f   VertexData.obj
 0001:000504b0       ??0CVertexData@@QAE@XZ     315514b0 f   VertexData.obj
 0001:00050510       ?ReleaseMemory@CVertexData@@QAEXXZ 31551510 f   VertexData.obj
 0001:000505d0       ?Initialize@CVertexData@@QAE_NI@Z 315515d0 f   VertexData.obj
 0001:000505f0       ?AllocateMemoryFromRenderMesh@CVertexData@@QAE_NAAUIRenderMesh@@@Z 315515f0 f   VertexData.obj
 0001:00050690       ?IsGeneralPass@SRenderingPassInfo@@QBE_NXZ 31551690 f i _Render.obj
 0001:000506b0       ??0SRendParams@@QAE@ABU0@@Z 315516b0 f i _Render.obj
 0001:00050830       ?MotionBlurMotionCheck@CCharInstance@@QAE_NI@Z 31551830 f   _Render.obj
 0001:00050860       ?IsValid@?$Matrix34_tpl@M@@QBE_NXZ 31551860 f i _Render.obj
 0001:00050930       ?RenderCGA@CCharInstance@@QAEXABUSRendParams@@ABU?$Matrix34_tpl@M@@ABUSRenderingPassInfo@@@Z 31551930 f   _Render.obj
 0001:00050e50       ?GetSkinningData@CCharInstance@@QAEPAUSSkinningData@@PAVCRenderObject@@ABUSRenderingPassInfo@@@Z 31551e50 f   _Render.obj
 0001:000510f0       ?RenderCHR@CCharInstance@@QAEXABUSRendParams@@ABU?$Matrix34_tpl@M@@ABUSRenderingPassInfo@@@Z 315520f0 f   _Render.obj
 0001:00051560       ?Render@CCharInstance@@UAEXABUSRendParams@@ABU?$QuatTS_tpl@M@@ABUSRenderingPassInfo@@PA_N@Z 31552560 f   _Render.obj
 0001:00052570       ?GetSkinningData@CAttachmentSKIN@@QAEPAUSSkinningData@@PAVCRenderObject@@ABUSRenderingPassInfo@@_N@Z 31553570 f   _RenderSkins.obj
 0001:00052930       ?DrawAttachment@CAttachmentSKIN@@UAEXAAUSRendParams@@ABUSRenderingPassInfo@@ABU?$Matrix34_tpl@M@@M@Z 31553930 f   _RenderSkins.obj
 0001:00053af0       ?DephysicalizeAttachment@CAttachmentManager@@UAEXHPAUIPhysicalEntity@@@Z 31554af0 f   AttachmentManager.obj
 0001:00053b60       ?RemoveAttachmentByInterface@CAttachmentManager@@UAEHPBUIAttachment@@@Z 31554b60 f   AttachmentManager.obj
 0001:00053b80       ?GetInterfaceByName@CAttachmentManager@@UBEPAUIAttachment@@PBD@Z 31554b80 f   AttachmentManager.obj
 0001:00053bb0       ?GetIAttachmentSkinByName@CAttachmentManager@@UBEPAUIAttachmentSkin@@PBD@Z 31554bb0 f   AttachmentManager.obj
 0001:00053be0       ?GetIndexByName@CAttachmentManager@@UBEHPBD@Z 31554be0 f   AttachmentManager.obj
 0001:00053c40       ?GetInterfaceByNameCRC@CAttachmentManager@@UBEPAUIAttachment@@I@Z 31554c40 f   AttachmentManager.obj
 0001:00053c70       ?GetIndexByNameCRC@CAttachmentManager@@UBEHI@Z 31554c70 f   AttachmentManager.obj
 0001:00053cc0       ?GetExt@PathUtil@@YAPBDPBD@Z 31554cc0 f i AttachmentManager.obj
 0001:00053d50       ?PhysicalizeAttachment@IAttachmentObject@@UAE_NPAUIAttachmentManager@@HHPAUIPhysicalEntity@@ABU?$Vec3_tpl@M@@@Z 31554d50 f i AttachmentManager.obj
 0001:00053d60       ?UpdatePhysicalizedAttachment@IAttachmentObject@@UAE_NPAUIAttachmentManager@@HPAUIPhysicalEntity@@ABU?$QuatT_tpl@M@@@Z 31554d60 f i AttachmentManager.obj
 0001:00053d70       ??_GIAttachmentObject@@UAEPAXI@Z 31554d70 f i AttachmentManager.obj
 0001:00053d70       ??_EIAttachmentObject@@UAEPAXI@Z 31554d70 f i AttachmentManager.obj
 0001:00053da0       ?GetPoseData@CAttachmentManager@@QAEABVCPoseData@Skeleton@@XZ 31554da0 f   AttachmentManager.obj
 0001:00053db0       ?Serialize@CAttachmentManager@@QAEXV?$CSerializeWrapper@UISerialize@@@@@Z 31554db0 f   AttachmentManager.obj
 0001:00053e20       ??$move_init@V?$_smart_ptr@UIAttachment@@@@@NArray@@YAXPAV?$_smart_ptr@UIAttachment@@@@0I@Z 31554e20 f i AttachmentManager.obj
 0001:00053e70       ?RenderAttachment@CCGFAttachment@@UAEXAAUSRendParams@@ABUSRenderingPassInfo@@@Z 31554e70 f i AttachmentManager.obj
 0001:00053ec0       ?GetAABB@CCGFAttachment@@UAE?AUAABB@@XZ 31554ec0 f i AttachmentManager.obj
 0001:00053ee0       ?GetRadiusSqr@CCGFAttachment@@UAEMXZ 31554ee0 f i AttachmentManager.obj
 0001:00053ef0       ?GetBaseMaterial@CCGFAttachment@@UBEPAUIMaterial@@XZ 31554ef0 f i AttachmentManager.obj
 0001:00053f10       ?ProcessAttachment@CSKELAttachment@@UAEXPAUIAttachment@@@Z 31554f10 f i AttachmentManager.obj
 0001:00053f30       ?GetRadiusSqr@CSKELAttachment@@UAEMXZ 31554f30 f i AttachmentManager.obj
 0001:00053f60       ?Release@CSKELAttachment@@UAEXXZ 31554f60 f i AttachmentManager.obj
 0001:00053f80       ?GetBaseMaterial@CSKELAttachment@@UBEPAUIMaterial@@XZ 31554f80 f i AttachmentManager.obj
 0001:00053fa0       ?SetReplacementMaterial@CSKELAttachment@@UAEXPAUIMaterial@@@Z 31554fa0 f i AttachmentManager.obj
 0001:00053fa0       ?SetReplacementMaterial@CSKINAttachment@@UAEXPAUIMaterial@@@Z 31554fa0 f i AttachmentManager.obj
 0001:00053fa0       ?SetReplacementMaterial@CCGFAttachment@@UAEXPAUIMaterial@@@Z 31554fa0 f i AttachmentManager.obj
 0001:00053fd0       ?GetRadiusSqr@CSKINAttachment@@UAEMXZ 31554fd0 f i AttachmentManager.obj
 0001:00053fe0       ?ProcessAttachment@CSKINAttachment@@UAEXPAUIAttachment@@@Z 31554fe0 f i AttachmentManager.obj
 0001:00054000       ?GetBaseMaterial@CSKINAttachment@@UBEPAUIMaterial@@XZ 31555000 f i AttachmentManager.obj
 0001:00054030       ??0ClosestTri@@QAE@XZ      31555030 f i AttachmentManager.obj
 0001:00054100       ??_ECCGFAttachment@@UAEPAXI@Z 31555100 f i AttachmentManager.obj
 0001:00054100       ??_GCCGFAttachment@@UAEPAXI@Z 31555100 f i AttachmentManager.obj
 0001:00054140       ?ApplyVisibilityMask@CAttachmentManager@@UAEXH@Z 31555140 f   AttachmentManager.obj
 0001:000541e0       ?GetInterfaceByIndex@CAttachmentManager@@UBEPAUIAttachment@@I@Z 315551e0 f   AttachmentManager.obj
 0001:00054210       ?GetIAttachmentSkinByIndex@CAttachmentManager@@UBEPAUIAttachmentSkin@@I@Z 31555210 f   AttachmentManager.obj
 0001:00054250       ?UpdateAllLocations@CAttachmentManager@@QAEXXZ 31555250 f   AttachmentManager.obj
 0001:00054330       ?UpdateAllAttachedObjects@CAttachmentManager@@QAEXXZ 31555330 f   AttachmentManager.obj
 0001:00054380       ?UpdateAllLocationsFast@CAttachmentManager@@QAEXXZ 31555380 f   AttachmentManager.obj
 0001:00054420       ?ProcessAllAttachedObjectsFast@CAttachmentManager@@QAEXXZ 31555420 f   AttachmentManager.obj
 0001:000544f0       ?DrawAttachments@CAttachmentManager@@QAEXABUSRendParams@@ABU?$Matrix34_tpl@M@@ABUSRenderingPassInfo@@@Z 315554f0 f   AttachmentManager.obj
 0001:000546e0       ?resize_raw@?$SmallDynStorage@V?$_smart_ptr@UIAttachment@@@@HUStandardAlloc@NAlloc@@@NArray@@QAEXHH_N@Z 315556e0 f i AttachmentManager.obj
 0001:00054830       ?RenderAttachment@CSKELAttachment@@UAEXAAUSRendParams@@ABUSRenderingPassInfo@@@Z 31555830 f i AttachmentManager.obj
 0001:000548d0       ?GetAABB@CSKELAttachment@@UAE?AUAABB@@XZ 315558d0 f i AttachmentManager.obj
 0001:000549b0       ??_ECSKELAttachment@@UAEPAXI@Z 315559b0 f i AttachmentManager.obj
 0001:000549b0       ??_GCSKELAttachment@@UAEPAXI@Z 315559b0 f i AttachmentManager.obj
 0001:000549f0       ?GetAABB@CSKINAttachment@@UAE?AUAABB@@XZ 315559f0 f i AttachmentManager.obj
 0001:00054a50       ??_ECSKINAttachment@@UAEPAXI@Z 31555a50 f i AttachmentManager.obj
 0001:00054a50       ??_GCSKINAttachment@@UAEPAXI@Z 31555a50 f i AttachmentManager.obj
 0001:00054a90       ?set_size@?$SmallDynStorage@UCharacterAttachment@@HUStandardAlloc@NAlloc@@@NArray@@QAEXH@Z 31555a90 f i AttachmentManager.obj
 0001:00054b20       ??0CharacterAttachment@@QAE@ABU0@@Z 31555b20 f i AttachmentManager.obj
 0001:00054c10       ?InitAttachmentList@CAttachmentManager@@QAEXABU?$DynArray@UCharacterAttachment@@HU?$SmallDynStorage@UCharacterAttachment@@HUStandardAlloc@NAlloc@@@NArray@@@@V?$CryStringT@D@@I@Z 31555c10 f   AttachmentManager.obj
 0001:000553d0       ?PhysicalizeAttachment@CAttachmentManager@@QAEXHHPAUIPhysicalEntity@@ABU?$Vec3_tpl@M@@@Z 315563d0 f   AttachmentManager.obj
 0001:00055960       ?UpdatePhysicalizedAttachment@CAttachmentManager@@QAEHHPAUIPhysicalEntity@@ABU?$QuatT_tpl@M@@@Z 31556960 f   AttachmentManager.obj
 0001:00055e70       ?pop_back@?$DynArray@V?$_smart_ptr@UIAttachment@@@@HU?$SmallDynStorage@V?$_smart_ptr@UIAttachment@@@@HUStandardAlloc@NAlloc@@@NArray@@@@QAEXH@Z 31556e70 f i AttachmentManager.obj
 0001:00055ec0       ?init@?$DynArray@UCharacterAttachment@@HU?$SmallDynStorage@UCharacterAttachment@@HUStandardAlloc@NAlloc@@@NArray@@@@KAPAUCharacterAttachment@@U?$Array@UCharacterAttachment@@HU?$ArrayStorage@UCharacterAttachment@@H@NArray@@@@ABU2@@Z 31556ec0 f i AttachmentManager.obj
 0001:00055ff0       ?expand_raw@?$DynArray@V?$_smart_ptr@UIAttachment@@@@HU?$SmallDynStorage@V?$_smart_ptr@UIAttachment@@@@HUStandardAlloc@NAlloc@@@NArray@@@@IAEPAV?$_smart_ptr@UIAttachment@@@@PAV2@H@Z 31556ff0 f i AttachmentManager.obj
 0001:00056070       ??$AddObject@V?$_smart_ptr@UIAttachment@@@@HU?$SmallDynStorage@V?$_smart_ptr@UIAttachment@@@@HUStandardAlloc@NAlloc@@@NArray@@@ICrySizer@@QAEXABU?$DynArray@V?$_smart_ptr@UIAttachment@@@@HU?$SmallDynStorage@V?$_smart_ptr@UIAttachment@@@@HUStandardAlloc@NAlloc@@@NArray@@@@@Z 31557070 f i AttachmentManager.obj
 0001:00056180       ??1CharacterAttachment@@QAE@XZ 31557180 f i AttachmentManager.obj
 0001:00056220       ??0CAttachmentBONE@@QAE@XZ 31557220 f i AttachmentManager.obj
 0001:00056350       ?Release@CAttachmentFACE@@UAEXXZ 31557350 f i AttachmentManager.obj
 0001:00056350       ?Release@CAttachmentBONE@@UAEXXZ 31557350 f i AttachmentManager.obj
 0001:00056370       ?GetIAttachmentObject@CAttachmentSKIN@@UBEPAUIAttachmentObject@@XZ 31557370 f i Attachment.obj
 0001:00056370       ?GetIAttachmentObject@CAttachmentBONE@@UBEPAUIAttachmentObject@@XZ 31557370 f i AttachmentManager.obj
 0001:00056370       ?GetIAttachmentObject@CAttachmentFACE@@UBEPAUIAttachmentObject@@XZ 31557370 f i AttachmentManager.obj
 0001:00056370       ?GetName@CFacialJoystickSet@@UBEPBDXZ 31557370 f i FaceJoystick.obj
 0001:00056370       ?GetFlags@CFacialEffector@@UAEIXZ 31557370 f i FaceEffector.obj
 0001:00056380       ?HideInRecursion@CAttachmentBONE@@UAEXI@Z 31557380 f i AttachmentManager.obj
 0001:00056380       ?HideInRecursion@CAttachmentSKIN@@UAEXI@Z 31557380 f i Attachment.obj
 0001:00056380       ?HideInRecursion@CAttachmentFACE@@UAEXI@Z 31557380 f i AttachmentManager.obj
 0001:000563a0       ?GetAttModelRelative@CAttachmentBONE@@UBEABU?$QuatT_tpl@M@@XZ 315573a0 f i AttachmentManager.obj
 0001:000563a0       ?GetAttModelRelative@CAttachmentFACE@@UBEABU?$QuatT_tpl@M@@XZ 315573a0 f i AttachmentManager.obj
 0001:000563b0       ?GetBoneID@CAttachmentBONE@@UBEIXZ 315573b0 f i AttachmentManager.obj
 0001:000563c0       ?GetPendulumParams@CAttachmentBONE@@UAEXAAHAAC1AAM22AAU?$Vec3_tpl@M@@3@Z 315573c0 f i AttachmentManager.obj
 0001:000563c0       ?GetPendulumParams@CAttachmentFACE@@UAEXAAHAAC1AAM22AAU?$Vec3_tpl@M@@3@Z 315573c0 f i AttachmentManager.obj
 0001:000563d0       ?SetPendulumParams@CAttachmentFACE@@UAEXHCCMMMU?$Vec3_tpl@M@@0@Z 315573d0 f i AttachmentManager.obj
 0001:000563d0       ?SetPendulumParams@CAttachmentBONE@@UAEXHCCMMMU?$Vec3_tpl@M@@0@Z 315573d0 f i AttachmentManager.obj
 0001:00056430       ?SetAttRelativeDefault@CAttachmentFACE@@UAEXABU?$QuatT_tpl@M@@@Z 31557430 f i AttachmentManager.obj
 0001:00056430       ?SetAttRelativeDefault@CAttachmentBONE@@UAEXABU?$QuatT_tpl@M@@@Z 31557430 f i AttachmentManager.obj
 0001:00056480       ??_ECAttachmentBONE@@UAEPAXI@Z 31557480 f i AttachmentManager.obj
 0001:00056480       ??_GCAttachmentBONE@@UAEPAXI@Z 31557480 f i AttachmentManager.obj
 0001:000564e0       ??0CAttachmentFACE@@QAE@XZ 315574e0 f i AttachmentManager.obj
 0001:00056630       ?AddRef@CAttachmentFACE@@UAEXXZ 31557630 f i AttachmentManager.obj
 0001:00056630       ?AddRef@CharacterDefinition@@UAEXXZ 31557630 f i CharacterManager.obj
 0001:00056630       ?AddRef@CFacialJoystickSet@@UAEXXZ 31557630 f i FaceJoystick.obj
 0001:00056630       ?AddRef@CAttachmentBONE@@UAEXXZ 31557630 f i AttachmentManager.obj
 0001:00056640       ?IsAttachmentHiddenInRecursion@CAttachmentSKIN@@UAEIXZ 31557640 f i Attachment.obj
 0001:00056640       ?IsAttachmentHiddenInRecursion@CAttachmentFACE@@UAEIXZ 31557640 f i AttachmentManager.obj
 0001:00056640       ?IsAttachmentHiddenInRecursion@CAttachmentBONE@@UAEIXZ 31557640 f i AttachmentManager.obj
 0001:00056650       ?HideInShadow@CAttachmentSKIN@@UAEXI@Z 31557650 f i Attachment.obj
 0001:00056650       ?HideInShadow@CAttachmentBONE@@UAEXI@Z 31557650 f i AttachmentManager.obj
 0001:00056650       ?HideInShadow@CAttachmentFACE@@UAEXI@Z 31557650 f i AttachmentManager.obj
 0001:00056670       ?IsAttachmentHiddenInShadow@CAttachmentSKIN@@UAEIXZ 31557670 f i Attachment.obj
 0001:00056670       ?IsAttachmentHiddenInShadow@CAttachmentFACE@@UAEIXZ 31557670 f i AttachmentManager.obj
 0001:00056670       ?IsAttachmentHiddenInShadow@CAttachmentBONE@@UAEIXZ 31557670 f i AttachmentManager.obj
 0001:00056680       ?GetAttRelativeDefault@CAttachmentFACE@@UBEABU?$QuatT_tpl@M@@XZ 31557680 f i AttachmentManager.obj
 0001:00056680       ?GetAttRelativeDefault@CAttachmentBONE@@UBEABU?$QuatT_tpl@M@@XZ 31557680 f i AttachmentManager.obj
 0001:00056690       ?SetAttAbsoluteDefault@CAttachmentFACE@@UAEXABU?$QuatT_tpl@M@@@Z 31557690 f i AttachmentManager.obj
 0001:00056690       ?SetAttAbsoluteDefault@CAttachmentBONE@@UAEXABU?$QuatT_tpl@M@@@Z 31557690 f i AttachmentManager.obj
 0001:000566e0       ??_GCAttachmentFACE@@UAEPAXI@Z 315576e0 f i AttachmentManager.obj
 0001:000566e0       ??_ECAttachmentFACE@@UAEPAXI@Z 315576e0 f i AttachmentManager.obj
 0001:00056740       ?PhysicalizeAttachment@CAttachmentManager@@UAEXHPAUIPhysicalEntity@@H@Z 31557740 f   AttachmentManager.obj
 0001:000567a0       ?ProjectAllAttachment@CAttachmentManager@@UAEIXZ 315577a0 f   AttachmentManager.obj
 0001:000576e0       ?RemoveAttachmentByIndex@CAttachmentManager@@QAEXI@Z 315586e0 f   AttachmentManager.obj
 0001:00057780       ?RemoveAllAttachments@CAttachmentManager@@QAEIXZ 31558780 f   AttachmentManager.obj
 0001:000578a0       ?SizeOfAllAttachments@CAttachmentManager@@QAEIXZ 315588a0 f   AttachmentManager.obj
 0001:00057930       ?GetMemoryUsage@CAttachmentManager@@QBEXPAVICrySizer@@@Z 31558930 f   AttachmentManager.obj
 0001:00057950       ?UnifyFilePath@CryStringUtils@@YAXAAV?$CryStringT@D@@@Z 31558950 f i AttachmentManager.obj
 0001:000579b0       ?RemoveAttachmentByName@CAttachmentManager@@UAEHPBD@Z 315589b0 f   AttachmentManager.obj
 0001:000579f0       ?RemoveAttachmentByNameCRC@CAttachmentManager@@UAEHI@Z 315589f0 f   AttachmentManager.obj
 0001:00057a30       ?grow@?$DynArray@V?$_smart_ptr@UIAttachment@@@@HU?$SmallDynStorage@V?$_smart_ptr@UIAttachment@@@@HUStandardAlloc@NAlloc@@@NArray@@@@QAEPAV?$_smart_ptr@UIAttachment@@@@HABV2@@Z 31558a30 f i AttachmentManager.obj
 0001:00057a90       ??$move_init@UCharacterAttachment@@@NArray@@YAXPAUCharacterAttachment@@0I@Z 31558a90 f i AttachmentManager.obj
 0001:00057ae0       ?CreateXMLAttachmentList@CAttachmentManager@@QAEIVXmlNodeRef@@@Z 31558ae0 f   AttachmentManager.obj
 0001:00058280       ?resize_raw@?$SmallDynStorage@UCharacterAttachment@@HUStandardAlloc@NAlloc@@@NArray@@QAEXHH_N@Z 31559280 f i AttachmentManager.obj
 0001:000583f0       ??0CAttachmentSKIN@@QAE@XZ 315593f0 f i AttachmentManager.obj
 0001:000584b0       ?SaveAttachmentList@CAttachmentManager@@UAEIPBD@Z 315594b0 f   AttachmentManager.obj
 0001:00058520       ?CreateAttachment@CAttachmentManager@@UAEPAUIAttachment@@PBDI0_N@Z 31559520 f   AttachmentManager.obj
 0001:000587c0       ?expand_raw@?$DynArray@UCharacterAttachment@@HU?$SmallDynStorage@UCharacterAttachment@@HUStandardAlloc@NAlloc@@@NArray@@@@IAEPAUCharacterAttachment@@PAU2@H@Z 315597c0 f i AttachmentManager.obj
 0001:00058850       ??1?$DynArray@UCharacterAttachment@@HU?$SmallDynStorage@UCharacterAttachment@@HUStandardAlloc@NAlloc@@@NArray@@@@QAE@XZ 31559850 f i AttachmentManager.obj
 0001:000588b0       ?ParseXMLAttachmentList@CAttachmentManager@@SAXAAU?$DynArray@UCharacterAttachment@@HU?$SmallDynStorage@UCharacterAttachment@@HUStandardAlloc@NAlloc@@@NArray@@@@VXmlNodeRef@@@Z 315598b0 f   AttachmentManager.obj
 0001:00059140       ?LoadAttachmentList@CAttachmentManager@@UAEIPBD@Z 3155a140 f   AttachmentManager.obj
 0001:00059260       ?KillAllSkeletonEffects@CCharInstance@@UAEXXZ 3155a260 f i CharacterInstance.obj
 0001:00059270       ?Release@CharacterManager@@UAEXXZ 3155a270 f   CharacterManager.obj
 0001:00059270       ?Release@CSKINAttachment@@UAEXXZ 3155a270 f   AttachmentManager.obj
 0001:00059270       ?destroy@sp_counted_base@detail@boost@@UAEXXZ 3155a270 f   OperatorQueue.obj
 0001:00059270       ?DeleteThis@CCharInstance@@UAEXXZ 3155a270 f   CharacterInstance.obj
 0001:00059270       ?Release@CCGFAttachment@@UAEXXZ 3155a270 f   AttachmentManager.obj
 0001:00059280       ?LipSyncWithSound@CCharInstance@@UAEXI_N@Z 3155a280 f   CharacterInstance.obj
 0001:000592a0       ?EnableProceduralFacialAnimation@CCharInstance@@UAEX_N@Z 3155a2a0 f   CharacterInstance.obj
 0001:000592c0       ??_EICharacterInstance@@UAEPAXI@Z 3155a2c0 f i CharacterInstance.obj
 0001:000592c0       ??_GICharacterInstance@@UAEPAXI@Z 3155a2c0 f i CharacterInstance.obj
 0001:000592f0       ??_EIAttachmentManager@@UAEPAXI@Z 3155a2f0 f i CharacterInstance.obj
 0001:000592f0       ??_EIFacialInstance@@UAEPAXI@Z 3155a2f0 f i FacialInstance.obj
 0001:000592f0       ??_GIAttachmentManager@@UAEPAXI@Z 3155a2f0 f i CharacterInstance.obj
 0001:000592f0       ??_GIFacialInstance@@UAEPAXI@Z 3155a2f0 f i FacialInstance.obj
 0001:00059320       ??0CAnimationLightProfileSection@@QAE@XZ 3155a320 f i CharacterInstance.obj
 0001:00059340       ??1CAnimationLightProfileSection@@QAE@XZ 3155a340 f i CharacterInstance.obj
 0001:00059380       ?GetFilePath@CCharInstance@@UAEPBDXZ 3155a380 f i CharacterInstance.obj
 0001:00059390       ?CopyPoseFrom@CCharInstance@@UAEXABUICharacterInstance@@@Z 3155a390 f   CharacterInstance.obj
 0001:000593d0       ?GetAABB@CCharInstance@@UAEABUAABB@@XZ 3155a3d0 f   CharacterInstance.obj
 0001:000593e0       ??$move_init@M@NArray@@YAXPAM0I@Z 3155a3e0 f i CharacterInstance.obj
 0001:00059470       ??$move_init@E@NArray@@YAXPAE0I@Z 3155a470 f i Attachment.obj
 0001:00059470       ??$move_init@D@NArray@@YAXPAD0I@Z 3155a470 f i LoaderCHR.obj
 0001:00059470       ??$move_init@_N@NArray@@YAXPA_N0I@Z 3155a470 f i CharacterInstance.obj
 0001:000594b0       ?GetRandomPart@GeomQuery@@QBEHXZ 3155a4b0 f i CharacterInstance.obj
 0001:00059590       ?BoxRandomPos@@YAXAAURandomPos@@W4EGeomForm@@ABU?$Vec3_tpl@M@@@Z 3155a590 f i CharacterInstance.obj
 0001:00059820       ?StartAnimationProcessing@CCharInstance@@UAEXABUSAnimationProcessParams@@@Z 3155a820 f   CharacterInstance.obj
 0001:00059b90       ?GetRadiusSqr@CCharInstance@@UAEMXZ 3155ab90 f   CharacterInstance.obj
 0001:00059c10       ?OnDetach@CCharInstance@@UAEXXZ 3155ac10 f   CharacterInstance.obj
 0001:00059c50       ?Serialize@CCharInstance@@UAEXV?$CSerializeWrapper@UISerialize@@@@@Z 3155ac50 f   CharacterInstance.obj
 0001:00059d00       ?EnableFacialAnimation@CCharInstance@@UAEX_N@Z 3155ad00 f   CharacterInstance.obj
 0001:00059d60       ?ProcessAttachment@CCharInstance@@UAEXPAUIAttachment@@@Z 3155ad60 f   CharacterInstance.obj
 0001:00059f90       ?resize_raw@?$SmallDynStorage@MHUStandardAlloc@NAlloc@@@NArray@@QAEXHH_N@Z 3155af90 f i CharacterInstance.obj
 0001:0005a0e0       ?init@?$DynArray@V?$CryStringT@D@@HU?$SmallDynStorage@V?$CryStringT@D@@HUStandardAlloc@NAlloc@@@NArray@@@@KAPAV?$CryStringT@D@@U?$Array@V?$CryStringT@D@@HU?$ArrayStorage@V?$CryStringT@D@@H@NArray@@@@ABV2@@Z 3155b0e0 f i CharacterInstance.obj
 0001:0005a120       ?destroy@?$DynArray@UGeomQuery@@HU?$SmallDynStorage@UGeomQuery@@HUStandardAlloc@NAlloc@@@NArray@@@@KAXU?$Array@UGeomQuery@@HU?$ArrayStorage@UGeomQuery@@H@NArray@@@@@Z 3155b120 f i CharacterInstance.obj
 0001:0005a150       ?set_size@?$SmallDynStorage@UGeomQuery@@HUStandardAlloc@NAlloc@@@NArray@@QAEXH@Z 3155b150 f i CharacterInstance.obj
 0001:0005a150       ?set_size@?$SmallDynStorage@UADIKTarget@@HUStandardAlloc@NAlloc@@@NArray@@QAEXH@Z 3155b150 f i ParamLoader.obj
 0001:0005a150       ?set_size@?$SmallDynStorage@UPQLog@@HUStandardAlloc@NAlloc@@@NArray@@QAEXH@Z 3155b150 f i LoaderTCB.obj
 0001:0005a1e0       ?expand_raw@?$DynArray@MHU?$SmallDynStorage@MHUStandardAlloc@NAlloc@@@NArray@@@@IAEPAMPAMH@Z 3155b1e0 f i CharacterInstance.obj
 0001:0005a260       ?resize_raw@?$SmallDynStorage@_NHUStandardAlloc@NAlloc@@@NArray@@QAEXHH_N@Z 3155b260 f i CharacterInstance.obj
 0001:0005a3a0       ?get_alloc_size@?$SmallDynStorage@UEffectEntry@CSkeletonEffectManager@@HUStandardAlloc@NAlloc@@@NArray@@QBEHXZ 3155b3a0 f i CharacterInstance.obj
 0001:0005a3f0       ?ApplyJointVelocitiesToPhysics@CCharInstance@@QAEXPAUIPhysicalEntity@@ABU?$Quat_tpl@M@@ABU?$Vec3_tpl@M@@@Z 3155b3f0 f   CharacterInstance.obj
 0001:0005b0f0       ?SkinningTransformationsComputation@CCharInstance@@QAEXPAUSSkinningData@@PAVCSkel@@HPBVCPoseData@Skeleton@@PAM@Z 3155c0f0 f   CharacterInstance.obj
 0001:0005bcd0       ?destroy@?$DynArray@UGeomQuery@@HU?$SmallDynStorage@UGeomQuery@@HUStandardAlloc@NAlloc@@@NArray@@@@IAEXXZ 3155ccd0 f i CharacterInstance.obj
 0001:0005bd00       ?expand_raw@?$DynArray@_NHU?$SmallDynStorage@_NHUStandardAlloc@NAlloc@@@NArray@@@@IAEPA_NPA_NH@Z 3155cd00 f i CharacterInstance.obj
 0001:0005bd80       ?replace@?$CryStringT@D@@QAEAAV1@PBD0@Z 3155cd80 f i CharacterInstance.obj
 0001:0005bf50       ??$AddObject@V?$CryStringT@D@@HU?$SmallDynStorage@V?$CryStringT@D@@HUStandardAlloc@NAlloc@@@NArray@@@ICrySizer@@QAEXABU?$DynArray@V?$CryStringT@D@@HU?$SmallDynStorage@V?$CryStringT@D@@HUStandardAlloc@NAlloc@@@NArray@@@@@Z 3155cf50 f i CharacterInstance.obj
 0001:0005c060       ?Invoke@?$SGenInvokerTSkinningTransformationsComputation@VCCharInstance@@PAUSSkinningData@@PAVCSkel@@HPBVCPoseData@Skeleton@@PAMUSNullType@Detail@JobManager@@U678@U678@U678@U678@U678@U678@@Detail@JobManager@@SAXPAX@Z 3155d060 f i CharacterInstance.obj
 0001:0005c090       ?SizeOfThis@CFacialInstance@@QAEIXZ 3155d090 f i CharacterInstance.obj
 0001:0005c0f0       ?UpdatePhysicsCGA@CCharInstance@@QAEXAAVCPoseData@Skeleton@@MABU?$QuatTS_tpl@M@@@Z 3155d0f0 f   CharacterInstance.obj
 0001:0005c9b0       ?SizeOfCharInstance@CCharInstance@@UAEIXZ 3155d9b0 f   CharacterInstance.obj
 0001:0005cb90       ?destroy@?$DynArray@V?$CryStringT@D@@HU?$SmallDynStorage@V?$CryStringT@D@@HUStandardAlloc@NAlloc@@@NArray@@@@KAXU?$Array@V?$CryStringT@D@@HU?$ArrayStorage@V?$CryStringT@D@@H@NArray@@@@@Z 3155db90 f i CharacterInstance.obj
 0001:0005cbe0       ?GetMemoryUsage@CCharInstance@@UBEXPAVICrySizer@@@Z 3155dbe0 f   CharacterInstance.obj
 0001:0005cdb0       ??1?$DynArray@UGeomQuery@@HU?$SmallDynStorage@UGeomQuery@@HUStandardAlloc@NAlloc@@@NArray@@@@QAE@XZ 3155ddb0 f i CharacterInstance.obj
 0001:0005ce10       ??1?$DynArray@V?$_smart_ptr@UIAttachment@@@@HU?$SmallDynStorage@V?$_smart_ptr@UIAttachment@@@@HUStandardAlloc@NAlloc@@@NArray@@@@QAE@XZ 3155de10 f i CharacterInstance.obj
 0001:0005ce70       ??$?0PAUSSkinningData@@PAVCSkel@@HPBVCPoseData@Skeleton@@PAM@SGenericJobTSkinningTransformationsComputation@Detail@JobManager@@QAE@PAUSSkinningData@@PAVCSkel@@HPBVCPoseData@Skeleton@@PAM@Z 3155de70 f i CharacterInstance.obj
 0001:0005cf30       ??$move_init@V?$CryStringT@D@@@NArray@@YAXPAV?$CryStringT@D@@0I@Z 3155df30 f i CharacterInstance.obj
 0001:0005cfb0       ??0?$DynArray@MHU?$SmallDynStorage@MHUStandardAlloc@NAlloc@@@NArray@@@@QAE@ABU0@@Z 3155dfb0 f i CharacterInstance.obj
 0001:0005d040       ??1CryCHRLoader@@QAE@XZ    3155e040 f i CharacterInstance.obj
 0001:0005d0d0       ?BeginSkinningTransformationsComputation@CCharInstance@@QAEXPAUSSkinningData@@@Z 3155e0d0 f   CharacterInstance.obj
 0001:0005d190       ??_GGeomQuery@@QAEPAXI@Z   3155e190 f i CharacterInstance.obj
 0001:0005d1e0       ?resize_raw@?$SmallDynStorage@V?$CryStringT@D@@HUStandardAlloc@NAlloc@@@NArray@@QAEXHH_N@Z 3155e1e0 f i CharacterInstance.obj
 0001:0005d330       ??0GeomQuery@@QAE@XZ       3155e330 f i CharacterInstance.obj
 0001:0005d3d0       ??0CAttachmentManager@@QAE@XZ 3155e3d0 f i CharacterInstance.obj
 0001:0005d440       ?GetAttachmentCount@CAttachmentManager@@UBEHXZ 3155e440 f i CharacterInstance.obj
 0001:0005d440       ?GetCount@CAnimEventList@@UBEIXZ 3155e440 f i AnimEventList.obj
 0001:0005d450       ??_GCAttachmentManager@@UAEPAXI@Z 3155e450 f i CharacterInstance.obj
 0001:0005d450       ??_ECAttachmentManager@@UAEPAXI@Z 3155e450 f i CharacterInstance.obj
 0001:0005d480       ??0CryCHRLoader@@QAE@XZ    3155e480 f i CharacterInstance.obj
 0001:0005d510       ?ReloadCHRPARAMS@CCharInstance@@UAEXXZ 3155e510 f   CharacterInstance.obj
 0001:0005d710       ?expand_raw@?$DynArray@V?$CryStringT@D@@HU?$SmallDynStorage@V?$CryStringT@D@@HUStandardAlloc@NAlloc@@@NArray@@@@IAEPAV?$CryStringT@D@@PAV2@H@Z 3155e710 f i CharacterInstance.obj
 0001:0005d790       ??$move_init@UGeomQuery@@@NArray@@YAXPAUGeomQuery@@0I@Z 3155e790 f i CharacterInstance.obj
 0001:0005d920       ??$__destroy_range_aux@V?$reverse_iterator@PAVCAnimDecal@@@stlpmtx_std@@VCAnimDecal@@@stlpmtx_std@@YAXV?$reverse_iterator@PAVCAnimDecal@@@0@0PAVCAnimDecal@@ABU__false_type@0@@Z 3155e920 f i CharacterInstance.obj
 0001:0005da50       ?resize_raw@?$SmallDynStorage@UGeomQuery@@HUStandardAlloc@NAlloc@@@NArray@@QAEXHH_N@Z 3155ea50 f i CharacterInstance.obj
 0001:0005dbb0       ?expand_raw@?$DynArray@UGeomQuery@@HU?$SmallDynStorage@UGeomQuery@@HUStandardAlloc@NAlloc@@@NArray@@@@IAEPAUGeomQuery@@PAU2@H@Z 3155ebb0 f i CharacterInstance.obj
 0001:0005dc40       ?clear@?$DynArray@UGeomQuery@@HU?$SmallDynStorage@UGeomQuery@@HUStandardAlloc@NAlloc@@@NArray@@@@QAEXXZ 3155ec40 f i CharacterInstance.obj
 0001:0005ddc0       ?SetOwner@GeomQuery@@QAE_NPBXW4EGeomForm@@@Z 3155edc0 f i CharacterInstance.obj
 0001:0005de40       ?resize@?$DynArray@V?$CryStringT@D@@HU?$SmallDynStorage@V?$CryStringT@D@@HUStandardAlloc@NAlloc@@@NArray@@@@QAEXH@Z 3155ee40 f i CharacterInstance.obj
 0001:0005deb0       ?push_back@?$DynArray@V?$CryStringT@D@@HU?$SmallDynStorage@V?$CryStringT@D@@HUStandardAlloc@NAlloc@@@NArray@@@@QAEPAV?$CryStringT@D@@ABV2@@Z 3155eeb0 f i CharacterInstance.obj
 0001:0005dee0       ??0?$DynArray@UGeomQuery@@HU?$SmallDynStorage@UGeomQuery@@HUStandardAlloc@NAlloc@@@NArray@@@@QAE@ABU0@@Z 3155eee0 f i CharacterInstance.obj
 0001:0005df60       ?GetRandomPos@CCharInstance@@UAEXAAURandomPos@@AAUGeomQuery@@W4EGeomForm@@@Z 3155ef60 f   CharacterInstance.obj
 0001:0005e3c0       ?resize@?$DynArray@UGeomQuery@@HU?$SmallDynStorage@UGeomQuery@@HUStandardAlloc@NAlloc@@@NArray@@@@QAEXH@Z 3155f3c0 f i CharacterInstance.obj
 0001:0005e570       ??0GeomQuery@@QAE@ABU0@@Z  3155f570 f i CharacterInstance.obj
 0001:0005e5b0       ?init@?$DynArray@UGeomQuery@@HU?$SmallDynStorage@UGeomQuery@@HUStandardAlloc@NAlloc@@@NArray@@@@KAPAUGeomQuery@@U?$Array@UGeomQuery@@HU?$ArrayStorage@UGeomQuery@@H@NArray@@@@PBU2@@Z 3155f5b0 f i CharacterInstance.obj
 0001:0005e620       ??1CAnimDecalManager@@QAE@XZ 3155f620 f i CharacterInstance.obj
 0001:0005e6a0       ??0CCharInstance@@QAE@ABV?$CryStringT@D@@PAVCSkel@@@Z 3155f6a0 f   CharacterInstance.obj
 0001:0005edf0       ?GetIAttachmentManager@CCharInstance@@UAEPAUIAttachmentManager@@XZ 3155fdf0 f i CharacterInstance.obj
 0001:0005ee00       ?GetAverageFrameTime@CCharInstance@@UAEMXZ 3155fe00 f i CharacterInstance.obj
 0001:0005ee10       ?SetUniformScale@CCharInstance@@UAEXABM@Z 3155fe10 f i CharacterInstance.obj
 0001:0005ee30       ?GetUniformScale@CCharInstance@@UBEMXZ 3155fe30 f i CharacterInstance.obj
 0001:0005ee40       ?EnableDecals@CCharInstance@@UAEXI@Z 3155fe40 f i CharacterInstance.obj
 0001:0005ee60       ?GetISkeletonAnim@CCharInstance@@UAEPAUISkeletonAnim@@XZ 3155fe60 f i CharacterInstance.obj
 0001:0005ee70       ?FinishAnimationComputations@CCharInstance@@UAEXXZ 3155fe70 f i CharacterInstance.obj
 0001:0005ee80       ?EnableStartAnimation@CCharInstance@@UAEX_N@Z 3155fe80 f i CharacterInstance.obj
 0001:0005ee90       ?GetResetMode@CCharInstance@@UAEIXZ 3155fe90 f i CharacterInstance.obj
 0001:0005eea0       ?SetResetMode@CCharInstance@@UAEXI@Z 3155fea0 f i CharacterInstance.obj
 0001:0005eec0       ?SetCharEditMode@CCharInstance@@UAEXI@Z 3155fec0 f i CharacterInstance.obj
 0001:0005eee0       ?GetCharEditMode@CCharInstance@@UBE_NXZ 3155fee0 f i CharacterInstance.obj
 0001:0005eef0       ?HideMaster@CCharInstance@@UAEXI@Z 3155fef0 f i CharacterInstance.obj
 0001:0005ef20       ?IsCharacterVisible@CCharInstance@@UAEIXZ 3155ff20 f i CharacterInstance.obj
 0001:0005ef30       ?IsAnimationGraphValid@CCharInstance@@UAE_NXZ 3155ff30 f i CharacterInstance.obj
 0001:0005ef50       ?SetForceLOD@CCharInstance@@UAEX_N@Z 3155ff50 f i CharacterInstance.obj
 0001:0005ef60       ?SetForceLODNum@CCharInstance@@UAEXH@Z 3155ff60 f i CharacterInstance.obj
 0001:0005ef70       ?GetPlaybackScale@CCharInstance@@UAEMXZ 3155ff70 f i CharacterInstance.obj
 0001:0005ef80       ?SpawnSkeletonEffect@CCharInstance@@UAEXHPBD00ABU?$Vec3_tpl@M@@1ABU?$Matrix34_tpl@M@@@Z 3155ff80 f i CharacterInstance.obj
 0001:0005efc0       ?SetFlags@CCharInstance@@UAEXH@Z 3155ffc0 f i CharacterInstance.obj
 0001:0005efd0       ?GetFlags@CCharInstance@@UAEHXZ 3155ffd0 f i CharacterInstance.obj
 0001:0005efe0       ?AddRef@?$SSplineBackup@V?$CatmullRomSpline@MU?$SplineKey@M@spline@@$0A@@spline@@@spline@@UAEXXZ 3155ffe0 f i FaceEffector.obj
 0001:0005efe0       ?AddRef@CCharInstance@@UAEXXZ 3155ffe0 f i CharacterInstance.obj
 0001:0005eff0       ?GetISkin@CAttachmentSKIN@@UAEPAUISkin@@XZ 3155fff0 f i Attachment.obj
 0001:0005eff0       ?GetRefCount@CCharInstance@@UBEHXZ 3155fff0 f i CharacterInstance.obj
 0001:0005eff0       ?GetParent@CFacialAnimChannel@@UAEPAUIFacialAnimChannel@@XZ 3155fff0 f i FaceAnimSequence.obj
 0001:0005f000       ?GetIAnimationSet@CCharInstance@@UAEPAUIAnimationSet@@XZ 31560000 f i CharacterInstance.obj
 0001:0005f010       ?GetOjectType@CCharInstance@@UAEHXZ 31560010 f i CharacterInstance.obj
 0001:0005f020       ?SetIMaterial_Instance@CCharInstance@@UAEXPAUIMaterial@@@Z 31560020 f i CharacterInstance.obj
 0001:0005f050       ?GetFlags@CAttachmentSKIN@@UAEIXZ 31560050 f i Attachment.obj
 0001:0005f050       ?GetTarget@CFacialJoystickChannel@@UAEPAXXZ 31560050 f i FaceJoystick.obj
 0001:0005f050       ?GetModelFilePath@CSkel@@UBEPBDXZ 31560050 f i Model.obj
 0001:0005f050       ?GetICharacterInstance@CSKELAttachment@@UBEPAUICharacterInstance@@XZ 31560050 f i AttachmentManager.obj
 0001:0005f050       ?GetSentence@CFacialAnimSoundEntry@@UAEPAUIFacialSentence@@XZ 31560050 f i FaceAnimSequence.obj
 0001:0005f050       ?GetIAttachmentSkin@CSKINAttachment@@UBEPAUIAttachmentSkin@@XZ 31560050 f i AttachmentManager.obj
 0001:0005f050       ?GetIMaterial_Instance@CCharInstance@@UBEPAUIMaterial@@XZ 31560050 f i CharacterInstance.obj
 0001:0005f050       ?GetName@CFacialAnimSkeletalAnimationEntry@@UBEPBDXZ 31560050 f i FaceAnimSequence.obj
 0001:0005f050       ?GetFlags@CAttachmentFACE@@UAEIXZ 31560050 f i AttachmentManager.obj
 0001:0005f050       ?GetFlags@CAttachmentBONE@@UAEIXZ 31560050 f i AttachmentManager.obj
 0001:0005f050       ?GetIStatObj@CCGFAttachment@@UBEPAUIStatObj@@XZ 31560050 f i AttachmentManager.obj
 0001:0005f060       ?SetPlaybackScale@CCharInstance@@UAEXM@Z 31560060 f i CharacterInstance.obj
 0001:0005f080       ?Release@CCharInstance@@UAEXXZ 31560080 f i CharacterInstance.obj
 0001:0005f0c0       ?GetModelAnimEventDatabase@CCharInstance@@UAEPBDXZ 315600c0 f i CharacterInstance.obj
 0001:0005f0d0       ?GetIMaterial@CCharInstance@@UBEPAUIMaterial@@XZ 315600d0 f i CharacterInstance.obj
 0001:0005f100       ?SetAttachmentLocation_DEPRECATED@CCharInstance@@UAEXABU?$QuatTS_tpl@M@@@Z 31560100 f i CharacterInstance.obj
 0001:0005f160       ?GetIgnoreScaleForJoint@CCharInstance@@UBE_NI@Z 31560160 f i CharacterInstance.obj
 0001:0005f180       ?GetIsCustomScaleForJoint@CCharInstance@@UBE_NI@Z 31560180 f i CharacterInstance.obj
 0001:0005f1a0       ?GetCustomScaleForJoint@CCharInstance@@UBEMI@Z 315601a0 f i CharacterInstance.obj
 0001:0005f1c0       ?SetCustomScaleForJoint@CCharInstance@@UAEXI_NM@Z 315601c0 f i CharacterInstance.obj
 0001:0005f1f0       ?DrawWireframeStatic@CCharInstance@@UAEXABU?$Matrix34_tpl@M@@HI@Z 315601f0 f i CharacterInstance.obj
 0001:0005f250       ??1CCharInstance@@MAE@XZ   31560250 f   CharacterInstance.obj
 0001:0005f410       ?ComputeExtent@CCharInstance@@UAEMAAUGeomQuery@@W4EGeomForm@@@Z 31560410 f   CharacterInstance.obj
 0001:0005f640       ??_GCCharInstance@@MAEPAXI@Z 31560640 f i CharacterInstance.obj
 0001:0005f640       ??_ECCharInstance@@MAEPAXI@Z 31560640 f i CharacterInstance.obj
 0001:0005f670       ?GetMemoryUsage@CAnimDecal@@QBEXPAVICrySizer@@@Z 31560670 f i DecalManager.obj
 0001:0005f730       ?SizeOfThis@CAnimDecalManager@@QAEIXZ 31560730 f   DecalManager.obj
 0001:0005f7d0       ??$AddObject@VCAnimDecal@@V?$allocator@VCAnimDecal@@@stlpmtx_std@@@ICrySizer@@QAEXABV?$vector@VCAnimDecal@@V?$allocator@VCAnimDecal@@@stlpmtx_std@@@stlpmtx_std@@@Z 315607d0 f i DecalManager.obj
 0001:0005f850       ?GetMemoryUsage@CAnimDecalManager@@QBEXPAVICrySizer@@@Z 31560850 f   DecalManager.obj
 0001:0005f8c0       ?SelectRandomPathExpansion@PathExpansion@@YAXPBDPAD@Z 315608c0 f   PathExpansion.obj
 0001:0005f9c0       ??0?$_Vector_base@DV?$allocator@D@stlpmtx_std@@@priv@stlpmtx_std@@QAE@IABV?$allocator@D@2@@Z 315609c0 f i PathExpansion.obj
 0001:0005fa60       ?EnumeratePathExpansions@PathExpansion@@YAXPBDP6AXPAX0@Z1@Z 31560a60 f   PathExpansion.obj
 0001:0005fd20       ?IsPlayingAnimation@CSkeletonEffectManager@@AAE_NPAUISkeletonAnim@@H@Z 31560d20 f   SkeletonEffectManager.obj
 0001:0005fd90       ??0EffectEntry@CSkeletonEffectManager@@QAE@V?$_smart_ptr@UIParticleEffect@@@@V?$_smart_ptr@UIParticleEmitter@@@@HABU?$Vec3_tpl@M@@2H@Z 31560d90 f   SkeletonEffectManager.obj
 0001:0005fe50       ??1EffectEntry@CSkeletonEffectManager@@QAE@XZ 31560e50 f   SkeletonEffectManager.obj
 0001:0005fea0       ?IsPlayingEffect@CSkeletonEffectManager@@AAE_NPBD@Z 31560ea0 f   SkeletonEffectManager.obj
 0001:0005ff10       ??0EffectEntry@CSkeletonEffectManager@@QAE@ABU01@@Z 31560f10 f i SkeletonEffectManager.obj
 0001:0005ff80       ?Spawn@IParticleEffect@@QAEPAUIParticleEmitter@@_NABU?$Matrix34_tpl@M@@@Z 31560f80 f i SkeletonEffectManager.obj
 0001:000603a0       ?GetEffectTM@CSkeletonEffectManager@@AAEXPAUISkeletonPose@@AAU?$Matrix34_tpl@M@@HABU?$Vec3_tpl@M@@2ABU3@@Z 315613a0 f   SkeletonEffectManager.obj
 0001:00060ba0       ?destroy@?$DynArray@UEffectEntry@CSkeletonEffectManager@@HU?$SmallDynStorage@UEffectEntry@CSkeletonEffectManager@@HUStandardAlloc@NAlloc@@@NArray@@@@KAXU?$Array@UEffectEntry@CSkeletonEffectManager@@HU?$ArrayStorage@UEffectEntry@CSkeletonEffectManager@@H@NArray@@@@@Z 31561ba0 f i SkeletonEffectManager.obj
 0001:00060c10       ?init@?$DynArray@UEffectEntry@CSkeletonEffectManager@@HU?$SmallDynStorage@UEffectEntry@CSkeletonEffectManager@@HUStandardAlloc@NAlloc@@@NArray@@@@KAPAUEffectEntry@CSkeletonEffectManager@@U?$Array@UEffectEntry@CSkeletonEffectManager@@HU?$ArrayStorage@UEffectEntry@CSkeletonEffectManager@@H@NArray@@@@ABU23@@Z 31561c10 f i SkeletonEffectManager.obj
 0001:00060ca0       ??$move_init@UEffectEntry@CSkeletonEffectManager@@@NArray@@YAXPAUEffectEntry@CSkeletonEffectManager@@0I@Z 31561ca0 f i SkeletonEffectManager.obj
 0001:00060d30       ?resize_raw@?$SmallDynStorage@UEffectEntry@CSkeletonEffectManager@@HUStandardAlloc@NAlloc@@@NArray@@QAEXHH_N@Z 31561d30 f i SkeletonEffectManager.obj
 0001:00060e90       ?expand_raw@?$DynArray@UEffectEntry@CSkeletonEffectManager@@HU?$SmallDynStorage@UEffectEntry@CSkeletonEffectManager@@HUStandardAlloc@NAlloc@@@NArray@@@@IAEPAUEffectEntry@CSkeletonEffectManager@@PAU23@H@Z 31561e90 f i SkeletonEffectManager.obj
 0001:00060f20       ?erase@?$DynArray@UEffectEntry@CSkeletonEffectManager@@HU?$SmallDynStorage@UEffectEntry@CSkeletonEffectManager@@HUStandardAlloc@NAlloc@@@NArray@@@@QAEPAUEffectEntry@CSkeletonEffectManager@@PAU23@0@Z 31561f20 f i SkeletonEffectManager.obj
 0001:00061060       ?KillAllEffects@CSkeletonEffectManager@@QAEXXZ 31562060 f   SkeletonEffectManager.obj
 0001:00061140       ??0CSkeletonEffectManager@@QAE@XZ 31562140 f   SkeletonEffectManager.obj
 0001:00061190       ??1CSkeletonEffectManager@@QAE@XZ 31562190 f   SkeletonEffectManager.obj
 0001:000611e0       ?Update@CSkeletonEffectManager@@QAEXPAUISkeletonAnim@@PAUISkeletonPose@@ABU?$Matrix34_tpl@M@@@Z 315621e0 f   SkeletonEffectManager.obj
 0001:00061310       ?SpawnEffect@CSkeletonEffectManager@@QAEXPAUISkeletonPose@@HPBD11ABU?$Vec3_tpl@M@@2ABU?$Matrix34_tpl@M@@@Z 31562310 f   SkeletonEffectManager.obj
 0001:000614c0       ?GetPoseDataWriteable@CSkeletonPose@@QAEPAVCPoseData@Skeleton@@XZ 315624c0 f   SkeletonPose.obj
 0001:000614d0       ?GetPoseDataForceWriteable@CSkeletonPose@@QAEAAVCPoseData@Skeleton@@XZ 315624d0 f   SkeletonPose.obj
 0001:000614f0       ?SynchronizePoseDataAndLocatorWriteables@CSkeletonPose@@QAEXXZ 315624f0 f   SkeletonPose.obj
 0001:00061530       ?SetDefaultPose@CSkeletonPose@@UAEXXZ 31562530 f   SkeletonPose.obj
 0001:00061540       ??_GISkeletonPhysics@@UAEPAXI@Z 31562540 f i SkeletonPose.obj
 0001:00061540       ??_EISkeletonPhysics@@UAEPAXI@Z 31562540 f i SkeletonPose.obj
 0001:00061570       ?PreparePoseDataAndLocatorWriteables@CSkeletonPose@@QAE_NAAVCPool@Memory@@@Z 31562570 f   SkeletonPose.obj
 0001:000615e0       ?GetJointCRC32@CSkeletonPose@@UBEIH@Z 315625e0 f   SkeletonPose.obj
 0001:00061620       ?Init@SDirectionalBlender@@QAEXXZ 31562620 f i SkeletonPose.obj
 0001:000617d0       ??1CFeetLock@@QAE@XZ       315627d0 f i SkeletonPose.obj
 0001:00061840       ?GetStatObjOnJoint@CSkeletonPose@@UAEPAUIStatObj@@H@Z 31562840 f   SkeletonPose.obj
 0001:00061890       ?SetStatObjOnJoint@CSkeletonPose@@UAEXHPAUIStatObj@@@Z 31562890 f   SkeletonPose.obj
 0001:00061900       ??$move_init@USPostProcess@@@NArray@@YAXPAUSPostProcess@@0I@Z 31562900 f i SkeletonPose.obj
 0001:00061a90       ?destroy@?$DynArray@UCCGAJoint@@HU?$SmallDynStorage@UCCGAJoint@@HUStandardAlloc@NAlloc@@@NArray@@@@KAXU?$Array@UCCGAJoint@@HU?$ArrayStorage@UCCGAJoint@@H@NArray@@@@@Z 31562a90 f i SkeletonPose.obj
 0001:00061b00       ?set_size@?$SmallDynStorage@UCCGAJoint@@HUStandardAlloc@NAlloc@@@NArray@@QAEXH@Z 31562b00 f i SkeletonPose.obj
 0001:00061b00       ?set_size@?$SmallDynStorage@USJointsAimIK_Rot@@HUStandardAlloc@NAlloc@@@NArray@@QAEXH@Z 31562b00 f i ParamLoader.obj
 0001:00061b00       ?set_size@?$SmallDynStorage@USRecoilJoints@@HUStandardAlloc@NAlloc@@@NArray@@QAEXH@Z 31562b00 f i ParamLoader.obj
 0001:00061b00       ?set_size@?$SmallDynStorage@U?$Quat_tpl@M@@HUStandardAlloc@NAlloc@@@NArray@@QAEXH@Z 31562b00 f i LoaderSKIN.obj
 0001:00061b90       ??$move_init@UCCGAJoint@@@NArray@@YAXPAUCCGAJoint@@0I@Z 31562b90 f i SkeletonPose.obj
 0001:00061c50       ??4?$shared_ptr@UIAnimationPoseBlenderDir@@@boost@@QAEAAV01@ABV01@@Z 31562c50 f i SkeletonPose.obj
 0001:00061c50       ??4?$shared_ptr@UIAnimationPoseModifier@@@boost@@QAEAAV01@ABV01@@Z 31562c50 f i TransitionQueue.obj
 0001:00061cb0       ?Op@?$cryinterface_cast_boost_helper@UIAnimationPoseBlenderDir@@UICryUnknown@@@Internal@InterfaceCastSemantics@@SA?AV?$shared_ptr@UIAnimationPoseBlenderDir@@@boost@@ABV?$shared_ptr@UICryUnknown@@@5@@Z 31562cb0 f i SkeletonPose.obj
 0001:00061db0       ?Op@?$cryinterface_cast_boost_helper@UIAnimationPoseModifier@@UICryUnknown@@@Internal@InterfaceCastSemantics@@SA?AV?$shared_ptr@UIAnimationPoseModifier@@@boost@@ABV?$shared_ptr@UICryUnknown@@@5@@Z 31562db0 f i SkeletonPose.obj
 0001:00061eb0       ?resize_raw@?$SmallDynStorage@USPostProcess@@HUStandardAlloc@NAlloc@@@NArray@@QAEXHH_N@Z 31562eb0 f i SkeletonPose.obj
 0001:00062000       ?resize_raw@?$SmallDynStorage@UCCGAJoint@@HUStandardAlloc@NAlloc@@@NArray@@QAEXHH_N@Z 31563000 f i SkeletonPose.obj
 0001:00062150       ?expand_raw@?$DynArray@USPostProcess@@HU?$SmallDynStorage@USPostProcess@@HUStandardAlloc@NAlloc@@@NArray@@@@IAEPAUSPostProcess@@PAU2@H@Z 31563150 f i SkeletonPose.obj
 0001:000621d0       ?expand_raw@?$DynArray@UCCGAJoint@@HU?$SmallDynStorage@UCCGAJoint@@HUStandardAlloc@NAlloc@@@NArray@@@@IAEPAUCCGAJoint@@PAU2@H@Z 315631d0 f i SkeletonPose.obj
 0001:00062250       ??$CryCreateClassInstance@UIAnimationPoseBlenderDir@@@@YA_NPBDAAV?$shared_ptr@UIAnimationPoseBlenderDir@@@boost@@@Z 31563250 f i SkeletonPose.obj
 0001:00062320       ??$CryCreateClassInstance@UIAnimationPoseModifier@@@@YA_NPBDAAV?$shared_ptr@UIAnimationPoseModifier@@@boost@@@Z 31563320 f i SkeletonPose.obj
 0001:000623f0       ??1CSkeletonPose@@UAE@XZ   315633f0 f   SkeletonPose.obj
 0001:000625d0       ?GetJointCount@CSkeletonPose@@UBEIXZ 315635d0 f i SkeletonPose.obj
 0001:000625f0       ?GetJointIDByName@CSkeletonPose@@UBEFPBD@Z 315635f0 f i SkeletonPose.obj
 0001:00062610       ?GetJointIDByCRC32@CSkeletonPose@@UBEFI@Z 31563610 f i SkeletonPose.obj
 0001:00062630       ?GetParentIDByID@CSkeletonPose@@UBEFH@Z 31563630 f i SkeletonPose.obj
 0001:00062650       ?GetJointNameByID@CSkeletonPose@@UBEPBDH@Z 31563650 f i SkeletonPose.obj
 0001:00062670       ?SetPostProcessCallback@CSkeletonPose@@UAEXP6AHPAUICharacterInstance@@PAX@Z1@Z 31563670 f i SkeletonPose.obj
 0001:00062690       ?GetPhysEntOnJoint@CSkeletonPose@@UAEPAUIPhysicalEntity@@H@Z 31563690 f i SkeletonPose.obj
 0001:000626b0       ?SetPhysEntOnJoint@CSkeletonPose@@UAEXHPAUIPhysicalEntity@@@Z 315636b0 f i SkeletonPose.obj
 0001:000626c0       ?GetPhysIdOnJoint@CSkeletonPose@@UAEHH@Z 315636c0 f i SkeletonPose.obj
 0001:000626d0       ?BuildPhysicalEntity@CSkeletonPose@@UAEXPAUIPhysicalEntity@@MHMHHABU?$Matrix34_tpl@M@@@Z 315636d0 f i SkeletonPose.obj
 0001:00062710       ?CreateCharacterPhysics@CSkeletonPose@@UAEPAUIPhysicalEntity@@PAU2@MHMHABU?$Matrix34_tpl@M@@@Z 31563710 f i SkeletonPose.obj
 0001:00062740       ?CreateAuxilaryPhysics@CSkeletonPose@@UAEHPAUIPhysicalEntity@@ABU?$Matrix34_tpl@M@@H@Z 31563740 f i SkeletonPose.obj
 0001:00062750       ?GetCharacterPhysics@CSkeletonPose@@UBEPAUIPhysicalEntity@@XZ 31563750 f i SkeletonPose.obj
 0001:00062760       ?GetCharacterPhysics@CSkeletonPose@@UAEPAUIPhysicalEntity@@PBD@Z 31563760 f i SkeletonPose.obj
 0001:00062770       ?GetCharacterPhysics@CSkeletonPose@@UAEPAUIPhysicalEntity@@H@Z 31563770 f i SkeletonPose.obj
 0001:00062780       ?SetCharacterPhysics@CSkeletonPose@@UAEXPAUIPhysicalEntity@@@Z 31563780 f i SkeletonPose.obj
 0001:000627a0       ?SynchronizeWithPhysicalEntity@CSkeletonPose@@UAEXPAUIPhysicalEntity@@ABU?$Vec3_tpl@M@@ABU?$Quat_tpl@M@@@Z 315637a0 f i SkeletonPose.obj
 0001:000627b0       ?RelinquishCharacterPhysics@CSkeletonPose@@UAEPAUIPhysicalEntity@@ABU?$Matrix34_tpl@M@@M_NABU?$Vec3_tpl@M@@@Z 315637b0 f i SkeletonPose.obj
 0001:000627e0       ?DestroyCharacterPhysics@CSkeletonPose@@UAEXH@Z 315637e0 f i SkeletonPose.obj
 0001:000627f0       ?AddImpact@CSkeletonPose@@UAE_NHU?$Vec3_tpl@M@@0@Z 315637f0 f i SkeletonPose.obj
 0001:00062840       ?TranslatePartIdToDeadBody@CSkeletonPose@@UAEHH@Z 31563840 f i SkeletonPose.obj
 0001:00062850       ?GetAuxPhysicsBoneId@CSkeletonPose@@UAEHHH@Z 31563850 f i SkeletonPose.obj
 0001:00062890       ?GoLimp@CSkeletonPose@@UAEXXZ 31563890 f i SkeletonPose.obj
 0001:000628a0       ?BlendFromRagdoll@CSkeletonPose@@UAE_NAAU?$QuatTS_tpl@M@@AAPAUIPhysicalEntity@@_N@Z 315638a0 f i SkeletonPose.obj
 0001:000628b0       ?GetFallingDir@CSkeletonPose@@UAEHXZ 315638b0 f i SkeletonPose.obj
 0001:000628c0       ?getBonePhysParentOrSelfIndex@CSkeletonPose@@UAEHHH@Z 315638c0 f i SkeletonPose.obj
 0001:000628e0       ?GetBoneSurfaceTypeId@CSkeletonPose@@UAEHHH@Z 315638e0 f i SkeletonPose.obj
 0001:000628f0       ?SetRagdollDefaultPose@CSkeletonPose@@UAEXXZ 315638f0 f i SkeletonPose.obj
 0001:00062900       ?GetAbsJointByID@CSkeletonPose@@UAEABU?$QuatT_tpl@M@@H@Z 31563900 f i SkeletonPose.obj
 0001:00062940       ?GetRelJointByID@CSkeletonPose@@UAEABU?$QuatT_tpl@M@@H@Z 31563940 f i SkeletonPose.obj
 0001:00062980       ?GetDefaultAbsJointByID@CSkeletonPose@@UAEABU?$QuatT_tpl@M@@H@Z 31563980 f i SkeletonPose.obj
 0001:000629c0       ?GetDefaultRelJointByID@CSkeletonPose@@UAEABU?$QuatT_tpl@M@@H@Z 315639c0 f i SkeletonPose.obj
 0001:00062a00       ?GetIPoseBlenderLook@CSkeletonPose@@UAEPAUIAnimationPoseBlenderDir@@XZ 31563a00 f i SkeletonPose.obj
 0001:00062a10       ?GetIPoseBlenderAim@CSkeletonPose@@UAEPAUIAnimationPoseBlenderDir@@XZ 31563a10 f i SkeletonPose.obj
 0001:00062a20       ?SetMaterialOnJoint@CSkeletonPose@@UAEXHPAUIMaterial@@@Z 31563a20 f i SkeletonPose.obj
 0001:00062a70       ?GetMaterialOnJoint@CSkeletonPose@@UAEPAUIMaterial@@H@Z 31563a70 f i SkeletonPose.obj
 0001:00062aa0       ?init@?$DynArray@USPostProcess@@HU?$SmallDynStorage@USPostProcess@@HUStandardAlloc@NAlloc@@@NArray@@@@KAPAUSPostProcess@@U?$Array@USPostProcess@@HU?$ArrayStorage@USPostProcess@@H@NArray@@@@ABU2@@Z 31563aa0 f i SkeletonPose.obj
 0001:00062b10       ?SetHumanLimbIK@CSkeletonPose@@UAEIABU?$Vec3_tpl@M@@PBD@Z 31563b10 f   SkeletonPose.obj
 0001:00062db0       ?ApplyRecoilAnimation@CSkeletonPose@@UAEXMMMI@Z 31563db0 f   SkeletonPose.obj
 0001:00062e20       ??0CSkeletonPose@@QAE@XZ   31563e20 f   SkeletonPose.obj
 0001:00062f90       ??_ECSkeletonPose@@UAEPAXI@Z 31563f90 f i SkeletonPose.obj
 0001:00062f90       ??_GCSkeletonPose@@UAEPAXI@Z 31563f90 f i SkeletonPose.obj
 0001:00062fc0       ?grow@?$DynArray@UCCGAJoint@@HU?$SmallDynStorage@UCCGAJoint@@HUStandardAlloc@NAlloc@@@NArray@@@@QAEPAUCCGAJoint@@H@Z 31563fc0 f i SkeletonPose.obj
 0001:00063010       ?SetDefaultPosePerInstance@CSkeletonPose@@QAEX_N@Z 31564010 f   SkeletonPose.obj
 0001:00063930       ?SetDefaultPoseExecute@CSkeletonPose@@QAEX_N@Z 31564930 f   SkeletonPose.obj
 0001:000639f0       ?SetPostProcessQuat@CSkeletonPose@@UAEXHABU?$QuatT_tpl@M@@@Z 315649f0 f i SkeletonPose.obj
 0001:00063a80       ?InitSkeletonPose@CSkeletonPose@@QAEXPAVCCharInstance@@PAVCSkeletonAnim@@@Z 31564a80 f   SkeletonPose.obj
 0001:00063bf0       ?InitCGASkeleton@CSkeletonPose@@QAEXXZ 31564bf0 f   SkeletonPose.obj
 0001:00063d60       ?DrawBBox@CSkeletonPose@@QAEXABU?$Matrix34_tpl@M@@@Z 31564d60 f   SkeletonPose_Debug.obj
 0001:00063ed0       ??$AddObject@UCPhysicsJoint@@HU?$SmallDynStorage@UCPhysicsJoint@@HUStandardAlloc@NAlloc@@@NArray@@@ICrySizer@@QAEXABU?$DynArray@UCPhysicsJoint@@HU?$SmallDynStorage@UCPhysicsJoint@@HUStandardAlloc@NAlloc@@@NArray@@@@@Z 31564ed0 f i SkeletonPose_Debug.obj
 0001:00063fb0       ?DrawPose@CSkeletonPose@@QAEXABVCPoseData@Skeleton@@ABU?$Matrix34_tpl@M@@@Z 31564fb0 f   SkeletonPose_Debug.obj
 0001:00064d20       ?DrawSkeleton@CSkeletonPose@@UAEXABU?$Matrix34_tpl@M@@I@Z 31565d20 f   SkeletonPose_Debug.obj
 0001:00064d40       ?SizeOfThis@CSkeletonPhysics@@QAEIXZ 31565d40 f i SkeletonPose_Debug.obj
 0001:00064dc0       ?SizeOfThis@CSkeletonPose@@QAEIXZ 31565dc0 f   SkeletonPose_Debug.obj
 0001:00064f50       ?GetMemoryUsage@CSkeletonPose@@QBEXPAVICrySizer@@@Z 31565f50 f   SkeletonPose_Debug.obj
 0001:00065090       ?UpdateBBox@CSkeletonPose@@QAEXI@Z 31566090 f   SkeletonPose_Process.obj
 0001:00066370       ??$?0$0CAA@@?$CryStringT@D@@QAE@ABV?$CryStackStringT@D$0CAA@@@@Z 31567370 f i SkeletonPose_Process.obj
 0001:000663d0       ??$__ucopy@PAV?$CryStringT@D@@PAV1@H@priv@stlpmtx_std@@YAPAV?$CryStringT@D@@PAV2@00ABUrandom_access_iterator_tag@1@PAH@Z 315673d0 f i SkeletonPose_Process.obj
 0001:00066420       ?UpdateAttachments@CSkeletonPose@@QAEXAAVCPoseData@Skeleton@@@Z 31567420 f   SkeletonPose_Process.obj
 0001:00066530       ?_M_insert_overflow@?$_Impl_vector@IV?$allocator@I@stlpmtx_std@@@priv@stlpmtx_std@@AAEXPAIABIABU__true_type@3@I_N@Z 31567530 f i SkeletonPose_Process.obj
 0001:00066530       ?_M_insert_overflow@?$_Impl_vector@HV?$allocator@H@stlpmtx_std@@@priv@stlpmtx_std@@AAEXPAHABHABU__true_type@3@I_N@Z 31567530 f i ControllerDefragHeap.obj
 0001:00066530       ?_M_insert_overflow@?$_Impl_vector@PAXV?$allocator@PAX@stlpmtx_std@@@priv@stlpmtx_std@@AAEXPAPAXABQAXABU__true_type@3@I_N@Z 31567530 f i LoaderSKIN.obj
 0001:00066680       ??$__uninitialized_fill_n@PAV?$CryStringT@D@@IV1@@priv@stlpmtx_std@@YAPAV?$CryStringT@D@@PAV2@IABV2@@Z 31567680 f i SkeletonPose_Process.obj
 0001:000666d0       ??$__destroy_range_aux@V?$reverse_iterator@PAV?$CryStringT@D@@@stlpmtx_std@@V?$CryStringT@D@@@stlpmtx_std@@YAXV?$reverse_iterator@PAV?$CryStringT@D@@@0@0PAV?$CryStringT@D@@ABU__false_type@0@@Z 315676d0 f i SkeletonPose_Process.obj
 0001:00066720       ?_M_insert_overflow_aux@?$_Impl_vector@V?$CryStringT@D@@V?$allocator@V?$CryStringT@D@@@stlpmtx_std@@@priv@stlpmtx_std@@AAEXPAV?$CryStringT@D@@ABV4@ABU__false_type@3@I_N@Z 31567720 f i SkeletonPose_Process.obj
 0001:000668b0       ?push_back@?$_Impl_vector@V?$CryStringT@D@@V?$allocator@V?$CryStringT@D@@@stlpmtx_std@@@priv@stlpmtx_std@@QAEXABV?$CryStringT@D@@@Z 315678b0 f i SkeletonPose_Process.obj
 0001:00066920       ?SkeletonPostProcess@CSkeletonPose@@QAEXAAVCPoseData@Skeleton@@@Z 31567920 f   SkeletonPose_Process.obj
 0001:00067280       ?SetDebugging@CSkeletonAnim@@UAEXI@Z 31568280 f   SkeletonAnim.obj
 0001:000672a0       ?SetTrackViewExclusive@CSkeletonAnim@@UAEXI@Z 315682a0 f   SkeletonAnim.obj
 0001:000672e0       ??_EISkeletonAnim@@UAEPAXI@Z 315682e0 f i SkeletonAnim.obj
 0001:000672e0       ??_GISkeletonAnim@@UAEPAXI@Z 315682e0 f i SkeletonAnim.obj
 0001:00067310       ?Initialize@CSkeletonAnimTask@@SA_NXZ 31568310 f   SkeletonAnim.obj
 0001:00067350       ??_ECSkeletonAnimTask@@UAEPAXI@Z 31568350 f i SkeletonAnim.obj
 0001:00067350       ??_GCSkeletonAnimTask@@UAEPAXI@Z 31568350 f i SkeletonAnim.obj
 0001:00067380       ?Execute@CSkeletonAnimTask@@UAEXXZ 31568380 f   SkeletonAnim.obj
 0001:000673c0       ?InitSkeletonAnim@CSkeletonAnim@@QAEXPAVCCharInstance@@PAVCSkeletonPose@@@Z 315683c0 f   SkeletonAnim.obj
 0001:000674e0       ?PoseModifiersSynchronize@CSkeletonAnim@@QAEXXZ 315684e0 f   SkeletonAnim.obj
 0001:00067530       ?GetCurrentVelocity@CSkeletonAnim@@UAE?AU?$Vec3_tpl@M@@XZ 31568530 f   SkeletonAnim.obj
 0001:000675c0       ?SetTrackViewMixingWeight@CSkeletonAnim@@UAEXIM@Z 315685c0 f   SkeletonAnim.obj
 0001:00067610       ?AllocateRuntimeParametric@CSkeletonAnim@@QAEPAUSParametricSamplerInternal@@XZ 31568610 f   SkeletonAnim.obj
 0001:000676d0       ?Invoke@?$SGenInvokerTCommandBufferExecuteJob@VCSkeletonAnimTask@@HUSNullType@Detail@JobManager@@U234@U234@U234@U234@U234@U234@U234@U234@U234@U234@@Detail@JobManager@@SAXPAX@Z 315686d0 f i SkeletonAnim.obj
 0001:00067720       ?Serialize@SParametricSamplerInternal@@QAEXV?$CSerializeWrapper@UISerialize@@@@@Z 31568720 f i SkeletonAnim.obj
 0001:00067900       ?Wait@CSkeletonAnimTask@@QAEXXZ 31568900 f   SkeletonAnim.obj
 0001:000679d0       ?PoseModifiersExecutePost@CSkeletonAnim@@QAEXAAVCPoseData@Skeleton@@ABU?$QuatTS_tpl@M@@@Z 315689d0 f   SkeletonAnim.obj
 0001:00067a60       ?ProcessAnimationUpdate@CSkeletonAnim@@QAEXU?$QuatTS_tpl@M@@@Z 31568a60 f   SkeletonAnim.obj
 0001:00067c80       ?_M_erase@?$_Rb_tree@HU?$less@H@stlpmtx_std@@HU?$_Identity@H@priv@2@U?$_SetTraitsT@H@42@V?$allocator@H@2@@priv@stlpmtx_std@@AAEXPAU_Rb_tree_node_base@23@@Z 31568c80 f i LoaderCGA.obj
 0001:00067c80       ?_M_erase@?$_Rb_tree@IU?$less@I@stlpmtx_std@@U?$pair@$$CBIPAV?$vector@IV?$allocator@I@stlpmtx_std@@@stlpmtx_std@@@2@U?$_Select1st@U?$pair@$$CBIPAV?$vector@IV?$allocator@I@stlpmtx_std@@@stlpmtx_std@@@stlpmtx_std@@@priv@2@U?$_MapTraitsT@U?$pair@$$CBIPAV?$vector@IV?$allocator@I@stlpmtx_std@@@stlpmtx_std@@@stlpmtx_std@@@52@V?$allocator@U?$pair@$$CBIPAV?$vector@IV?$allocator@I@stlpmtx_std@@@stlpmtx_std@@@stlpmtx_std@@@2@@priv@stlpmtx_std@@AAEXPAU_Rb_tree_node_base@23@@Z 31568c80 f i CharacterManager.obj
 0001:00067c80       ?_M_erase@?$_Rb_tree@IU?$less@I@stlpmtx_std@@U?$pair@$$CBIUSFacialDisplaceInfo@CFacialModel@@@2@U?$_Select1st@U?$pair@$$CBIUSFacialDisplaceInfo@CFacialModel@@@stlpmtx_std@@@priv@2@U?$_MapTraitsT@U?$pair@$$CBIUSFacialDisplaceInfo@CFacialModel@@@stlpmtx_std@@@52@V?$allocator@U?$pair@$$CBIUSFacialDisplaceInfo@CFacialModel@@@stlpmtx_std@@@2@@priv@stlpmtx_std@@AAEXPAU_Rb_tree_node_base@23@@Z 31568c80 f i SkeletonAnim.obj
 0001:00067c80       ?_M_erase@?$_Rb_tree@IU?$less@I@stlpmtx_std@@U?$pair@$$CBIPAV?$vector@HV?$allocator@H@stlpmtx_std@@@stlpmtx_std@@@2@U?$_Select1st@U?$pair@$$CBIPAV?$vector@HV?$allocator@H@stlpmtx_std@@@stlpmtx_std@@@stlpmtx_std@@@priv@2@U?$_MapTraitsT@U?$pair@$$CBIPAV?$vector@HV?$allocator@H@stlpmtx_std@@@stlpmtx_std@@@stlpmtx_std@@@52@V?$allocator@U?$pair@$$CBIPAV?$vector@HV?$allocator@H@stlpmtx_std@@@stlpmtx_std@@@stlpmtx_std@@@2@@priv@stlpmtx_std@@AAEXPAU_Rb_tree_node_base@23@@Z 31568c80 f i CharacterManager.obj
 0001:00067c80       ?_M_erase@?$_Rb_tree@PAUIFacialEffector@@U?$less@PAUIFacialEffector@@@stlpmtx_std@@U?$pair@QAUIFacialEffector@@PAU1@@3@U?$_Select1st@U?$pair@QAUIFacialEffector@@PAU1@@stlpmtx_std@@@priv@3@U?$_MapTraitsT@U?$pair@QAUIFacialEffector@@PAU1@@stlpmtx_std@@@63@V?$allocator@U?$pair@QAUIFacialEffector@@PAU1@@stlpmtx_std@@@3@@priv@stlpmtx_std@@AAEXPAU_Rb_tree_node_base@23@@Z 31568c80 f i FaceEffectorLibrary.obj
 0001:00067c80       ?_M_erase@?$_Rb_tree@IU?$less@I@stlpmtx_std@@U?$pair@$$CBII@2@U?$_Select1st@U?$pair@$$CBII@stlpmtx_std@@@priv@2@U?$_MapTraitsT@U?$pair@$$CBII@stlpmtx_std@@@52@V?$allocator@U?$pair@$$CBII@stlpmtx_std@@@2@@priv@stlpmtx_std@@AAEXPAU_Rb_tree_node_base@23@@Z 31568c80 f i CharacterManager.obj
 0001:00067c80       ?_M_erase@?$_Rb_tree@HU?$less@H@stlpmtx_std@@U?$pair@$$CBHPAUphys_geometry@@@2@U?$_Select1st@U?$pair@$$CBHPAUphys_geometry@@@stlpmtx_std@@@priv@2@U?$_MapTraitsT@U?$pair@$$CBHPAUphys_geometry@@@stlpmtx_std@@@52@V?$allocator@U?$pair@$$CBHPAUphys_geometry@@@stlpmtx_std@@@2@@priv@stlpmtx_std@@AAEXPAU_Rb_tree_node_base@23@@Z 31568c80 f i LoaderCHR.obj
 0001:00067c80       ?_M_erase@?$_Rb_tree@IU?$less@I@stlpmtx_std@@U?$pair@$$CBIPAVCModelJoint@@@2@U?$_Select1st@U?$pair@$$CBIPAVCModelJoint@@@stlpmtx_std@@@priv@2@U?$_MapTraitsT@U?$pair@$$CBIPAVCModelJoint@@@stlpmtx_std@@@52@V?$allocator@U?$pair@$$CBIPAVCModelJoint@@@stlpmtx_std@@@2@@priv@stlpmtx_std@@AAEXPAU_Rb_tree_node_base@23@@Z 31568c80 f i Model.obj
 0001:00067cc0       ?FinishAnimationComputations@CSkeletonAnim@@AAEXW4FinishAnimationComputationCallMethod@1@@Z 31568cc0 f   SkeletonAnim.obj
 0001:00068040       ?PushPoseModifier@CSkeletonAnim@@UAE_NIV?$shared_ptr@UIAnimationPoseModifier@@@boost@@PBD@Z 31569040 f   SkeletonAnim.obj
 0001:000681b0       ?PoseModifiersPrepare@CSkeletonAnim@@QAEXABU?$QuatTS_tpl@M@@@Z 315691b0 f   SkeletonAnim.obj
 0001:00068410       ?SizeOfThis@CSkeletonAnim@@QAEIXZ 31569410 f   SkeletonAnim.obj
 0001:00068470       ??$?0I@SGenericJobTCommandBufferExecuteJob@Detail@JobManager@@QAE@I@Z 31569470 f i SkeletonAnim.obj
 0001:00068520       ??$AddObject@VCAnimation@@HU?$SmallDynStorage@VCAnimation@@HUStandardAlloc@NAlloc@@@NArray@@@ICrySizer@@QAEXABU?$DynArray@VCAnimation@@HU?$SmallDynStorage@VCAnimation@@HUStandardAlloc@NAlloc@@@NArray@@@@@Z 31569520 f i SkeletonAnim.obj
 0001:00068600       ?Prepare@CSkeletonAnimTask@@QAEXXZ 31569600 f   SkeletonAnim.obj
 0001:000686e0       ?FinishAnimationComputations@CSkeletonAnim@@QAEXXZ 315696e0 f   SkeletonAnim.obj
 0001:000686f0       ?GetMemoryUsage@CSkeletonAnim@@QBEXPAVICrySizer@@@Z 315696f0 f   SkeletonAnim.obj
 0001:00068740       ?Format@?$CryStringT@D@@QAAAAV1@PBDZZ 31569740 f i SkeletonAnim.obj
 0001:000687b0       ?Begin@CSkeletonAnimTask@@QAEXABU?$QuatTS_tpl@M@@_N@Z 315697b0 f   SkeletonAnim.obj
 0001:000688c0       ?ProcessAnimations@CSkeletonAnim@@QAEXABU?$QuatTS_tpl@M@@_N@Z 315698c0 f   SkeletonAnim.obj
 0001:00068ac0       ?Serialize@CAnimation@@QAEXV?$CSerializeWrapper@UISerialize@@@@@Z 31569ac0 f i SkeletonAnim.obj
 0001:00068cf0       ??1CSkeletonAnim@@UAE@XZ   31569cf0 f   SkeletonAnim.obj
 0001:00068e10       ?GetAnimationDrivenMotion@CSkeletonAnim@@UAEIXZ 31569e10 f i SkeletonAnim.obj
 0001:00068e20       ?GetTrackViewStatus@CSkeletonAnim@@UAEIXZ 31569e20 f i SkeletonAnim.obj
 0001:00068e30       ?GetLayerPlaybackScale@CSkeletonAnim@@UAEMI@Z 31569e30 f i SkeletonAnim.obj
 0001:00068e50       ?SetEventCallback@CSkeletonAnim@@UAEXP6AHPAUICharacterInstance@@PAX@Z1@Z 31569e50 f i SkeletonAnim.obj
 0001:00068e70       ?GetLastAnimEvent@CSkeletonAnim@@UAE?AUAnimEventInstance@@XZ 31569e70 f i SkeletonAnim.obj
 0001:00068e90       ?GetUserData@CSkeletonAnim@@UAEMH@Z 31569e90 f i SkeletonAnim.obj
 0001:00068eb0       ?GetAnimFromFIFO@CSkeletonAnim@@UBEABVCAnimation@@II@Z 31569eb0 f i SkeletonAnim.obj
 0001:00068eb0       ?GetAnimFromFIFO@CSkeletonAnim@@UAEAAVCAnimation@@II@Z 31569eb0 f i SkeletonAnim.obj
 0001:00068ed0       ?RemoveAnimFromFIFO@CSkeletonAnim@@UAE_NII_N@Z 31569ed0 f i SkeletonAnim.obj
 0001:00068ef0       ?ClearFIFOLayer@CSkeletonAnim@@UAEXI@Z 31569ef0 f i SkeletonAnim.obj
 0001:00068f10       ?RemoveTransitionDelayConditions@CSkeletonAnim@@UAEXI@Z 31569f10 f i SkeletonAnim.obj
 0001:00068f30       ?ManualSeekAnimationInFIFO@CSkeletonAnim@@UAEXIIM_N@Z 31569f30 f i SkeletonAnim.obj
 0001:00068f60       ?GetNumAnimsInFIFO@CSkeletonAnim@@UBEHI@Z 31569f60 f i SkeletonAnim.obj
 0001:00068f80       ??0CSkeletonAnim@@QAE@XZ   31569f80 f   SkeletonAnim.obj
 0001:000690f0       ??_GCSkeletonAnim@@UAEPAXI@Z 3156a0f0 f i SkeletonAnim.obj
 0001:000690f0       ??_ECSkeletonAnim@@UAEPAXI@Z 3156a0f0 f i SkeletonAnim.obj
 0001:00069120       ?Serialize@CSkeletonAnim@@QAEXV?$CSerializeWrapper@UISerialize@@@@@Z 3156a120 f   SkeletonAnim.obj
 0001:00069480       ?AnimFlags@@YAPBDI@Z       3156a480 f   SkeletonAnim_BlendMan.obj
 0001:00069500       ?GetAnimationNormalizedTime@CSkeletonAnim@@UBEMII@Z 3156a500 f   SkeletonAnim_BlendMan.obj
 0001:00069530       ?SetAnimationDrivenMotion@CSkeletonAnim@@UAEXI@Z 3156a530 f   SkeletonAnim_BlendMan.obj
 0001:00069540       ?SetMirrorAnimation@CSkeletonAnim@@UAEXI@Z 3156a540 f   SkeletonAnim_BlendMan.obj
 0001:00069560       ?SetLayerBlendWeight@CSkeletonAnim@@UAEXHM@Z 3156a560 f   SkeletonAnim_BlendMan.obj
 0001:000695a0       ?SetLayerPlaybackScale@CSkeletonAnim@@UAEXHM@Z 3156a5a0 f   SkeletonAnim_BlendMan.obj
 0001:000695f0       ?Draw2dLabel@IRenderer@@QAAXMMMABU?$Color_tpl@M@@_NPBDZZ 3156a5f0 f i SkeletonAnim_BlendMan.obj
 0001:000696a0       ?UpdateParameters@CSkeletonAnim@@AAEXPAVCAnimation@@IIM@Z 3156a6a0 f   SkeletonAnim_BlendMan.obj
 0001:000699f0       ?GetMaxSegments@CSkeletonAnim@@ABEIABVCAnimation@@@Z 3156a9f0 f   SkeletonAnim_BlendMan.obj
 0001:00069af0       ?AnimCallback@CSkeletonAnim@@QAEXPAVCAnimation@@II@Z 3156aaf0 f   SkeletonAnim_BlendMan.obj
 0001:00069e10       ?SetLayerNormalizedTimeAndSegment@CSkeletonAnim@@QAEXIMEH@Z 3156ae10 f   SkeletonAnim_BlendMan.obj
 0001:00069ea0       ?SetLayerNormalizedTime@CSkeletonAnim@@UAEXIM@Z 3156aea0 f   SkeletonAnim_BlendMan.obj
 0001:00069ee0       ?GetLayerNormalizedTime@CSkeletonAnim@@UBEMI@Z 3156aee0 f   SkeletonAnim_BlendMan.obj
 0001:00069f20       ?SetAnimationNormalizedTime@CSkeletonAnim@@UAEXPAVCAnimation@@M@Z 3156af20 f   SkeletonAnim_BlendMan.obj
 0001:0006a010       ?GetAnimationNormalizedTime@CSkeletonAnim@@UBEMPBVCAnimation@@@Z 3156b010 f   SkeletonAnim_BlendMan.obj
 0001:0006a0a0       ?LayerBlendManager@CSkeletonAnim@@QAEXMI@Z 3156b0a0 f   SkeletonAnim_BlendMan.obj
 0001:0006a160       ?GetRelMovement@CSkeletonAnim@@UBEABU?$QuatT_tpl@M@@XZ 3156b160 f   SkeletonAnim_BlendMan.obj
 0001:0006a1f0       ?CheckIsCAFLoaded@CSkeletonAnim@@AAEIPAVCAnimationSet@@H@Z 3156b1f0 f   SkeletonAnim_BlendMan.obj
 0001:0006a280       ?UpdateAnimationTime@CSkeletonAnim@@AAEXAAVCAnimation@@IIII@Z 3156b280 f   SkeletonAnim_BlendMan.obj
 0001:0006a650       ?IsAnimationInMemory@CSkeletonAnim@@AAEIPAVCAnimationSet@@PAVCAnimation@@@Z 3156b650 f   SkeletonAnim_BlendMan.obj
 0001:0006a770       ?BlendManagerDebug@CSkeletonAnim@@QAEIAAU?$DynArray@VCAnimation@@HU?$SmallDynStorage@VCAnimation@@HUStandardAlloc@NAlloc@@@NArray@@@@I@Z 3156b770 f   SkeletonAnim_BlendMan.obj
 0001:0006ae80       ?EvaluateTransitionFlags@CSkeletonAnim@@AAEIPAVCAnimation@@I@Z 3156be80 f   SkeletonAnim_BlendMan.obj
 0001:0006b1c0       ?BlendManager@CSkeletonAnim@@QAEIMAAU?$DynArray@VCAnimation@@HU?$SmallDynStorage@VCAnimation@@HUStandardAlloc@NAlloc@@@NArray@@@@I@Z 3156c1c0 f   SkeletonAnim_BlendMan.obj
 0001:0006b540       ?Commands_BasePlayback@CSkeletonAnim@@AAEXABVCAnimation@@AAVCBuffer@Command@@@Z 3156c540 f   SkeletonAnim_Commands.obj
 0001:0006b780       ?Commands_LPlayback@CSkeletonAnim@@AAEXABVCAnimation@@IIAAVCBuffer@Command@@@Z 3156c780 f   SkeletonAnim_Commands.obj
 0001:0006b950       ?Commands_BaseEvaluationLMG@CSkeletonAnim@@AAEXABVCAnimation@@IAAVCBuffer@Command@@@Z 3156c950 f   SkeletonAnim_Commands.obj
 0001:0006c160       ?Commands_Create@CSkeletonAnim@@AAEXABU?$QuatTS_tpl@M@@AAVCBuffer@Command@@@Z 3156d160 f   SkeletonAnim_Commands.obj
 0001:0006c720       ?SetDesiredMotionParam@CSkeletonAnim@@UAEXW4EMotionParamID@@MM@Z 3156d720 f   SkeletonAnim_Params.obj
 0001:0006c7c0       ?GetDesiredMotionParam@CSkeletonAnim@@UBE_NW4EMotionParamID@@AAM@Z 3156d7c0 f   SkeletonAnim_Params.obj
 0001:0006c8c0       ?StopAnimationsAllLayers@CSkeletonAnim@@UAE_NXZ 3156d8c0 f   SkeletonAnim_Queue.obj
 0001:0006c8f0       ?StartAnimation@CSkeletonAnim@@UAE_NPBDABUCryCharAnimationParams@@@Z 3156d8f0 f   SkeletonAnim_Queue.obj
 0001:0006c9d0       ?StopAnimationInLayer@CSkeletonAnim@@UAE_NHM@Z 3156d9d0 f   SkeletonAnim_Queue.obj
 0001:0006ca50       ?FindAnimInFIFO@CSkeletonAnim@@UAEPAVCAnimation@@IH@Z 3156da50 f   SkeletonAnim_Queue.obj
 0001:0006cad0       ?AnimationToQueue@CSkeletonAnim@@AAEIPBUModelAnimationHeader@@HMABUCryCharAnimationParams@@@Z 3156dad0 f   SkeletonAnim_Queue.obj
 0001:0006d210       ?StartAnimationById@CSkeletonAnim@@UAE_NHABUCryCharAnimationParams@@@Z 3156e210 f   SkeletonAnim_Queue.obj
 0001:0006d900       ?RetrieveEffectorIdentifiers@CEyeMovementFaceAnim@@ABEPBVCFaceIdentifierHandle@@XZ 3156e900 f   EyeMovementFaceAnim.obj
 0001:0006da70       ?InitialiseBoneIDs@CEyeMovementFaceAnim@@AAEXXZ 3156ea70 f   EyeMovementFaceAnim.obj
 0001:0006dac0       ??0SFacialEffectorChannel@@QAE@XZ 3156eac0 f i EyeMovementFaceAnim.obj
 0001:0006db30       ?CreateChannelForEffector@CEyeMovementFaceAnim@@AAEIW4EffectorID@1@@Z 3156eb30 f   EyeMovementFaceAnim.obj
 0001:0006dc00       ?DisplayDebugInfoForEye@CEyeMovementFaceAnim@@AAEXABU?$QuatTS_tpl@M@@W4EyeID@1@ABV?$CryStringT@D@@@Z 3156ec00 f   EyeMovementFaceAnim.obj
 0001:0006dd20       ?GetMemoryUsage@CEyeMovementFaceAnim@@QBEXPAVICrySizer@@@Z 3156ed20 f   EyeMovementFaceAnim.obj
 0001:0006dd70       ??0CEyeMovementFaceAnim@@QAE@PAVCFacialInstance@@@Z 3156ed70 f   EyeMovementFaceAnim.obj
 0001:0006ddf0       ??_GCControllerOptNonVirtual@@UAEPAXI@Z 3156edf0 f i LoaderDBA.obj
 0001:0006ddf0       ??_GCEyeMovementFaceAnim@@UAEPAXI@Z 3156edf0 f i EyeMovementFaceAnim.obj
 0001:0006ddf0       ??_GIController@@UAEPAXI@Z 3156edf0 f i LoaderCGA.obj
 0001:0006ddf0       ??_G?$_i_reference_target@H@@UAEPAXI@Z 3156edf0 f i LoaderSKIN.obj
 0001:0006ddf0       ??_ECEyeMovementFaceAnim@@UAEPAXI@Z 3156edf0 f i EyeMovementFaceAnim.obj
 0001:0006ddf0       ??_EIController@@UAEPAXI@Z 3156edf0 f i LoaderCGA.obj
 0001:0006ddf0       ??_E?$_i_reference_target@H@@UAEPAXI@Z 3156edf0 f i LoaderSKIN.obj
 0001:0006ddf0       ??_ECControllerOptNonVirtual@@UAEPAXI@Z 3156edf0 f i LoaderDBA.obj
 0001:0006de20       ?OnExpressionLibraryLoad@CEyeMovementFaceAnim@@QAEXXZ 3156ee20 f   EyeMovementFaceAnim.obj
 0001:0006de60       ?FindLookAngleAndStrength@CEyeMovementFaceAnim@@AAEXW4EyeID@1@AAM1ABU?$QuatT_tpl@M@@@Z 3156ee60 f   EyeMovementFaceAnim.obj
 0001:0006e100       ?CalculateEyeAdditionalRotation@CEyeMovementFaceAnim@@AAEXPAVCCharInstance@@PAVCFaceState@@PAVCFacialEffectorsLibrary@@QAU?$QuatT_tpl@M@@@Z 3156f100 f   EyeMovementFaceAnim.obj
 0001:0006e590       ?Format@?$CryStackStringT@D$0CAA@@@QAAAAV1@PBDZZ 3156f590 f i EyeMovementFaceAnim.obj
 0001:0006e600       ?UpdateEye@CEyeMovementFaceAnim@@AAEXABU?$QuatTS_tpl@M@@W4EyeID@1@ABU?$QuatT_tpl@M@@@Z 3156f600 f   EyeMovementFaceAnim.obj
 0001:0006e8c0       ?Update@CEyeMovementFaceAnim@@QAEXMABU?$QuatTS_tpl@M@@PAVCCharInstance@@PAVCFacialEffectorsLibrary@@PAVCFaceState@@@Z 3156f8c0 f   EyeMovementFaceAnim.obj
 0001:0006e920       ?GetPhonemeLibrary@CFacialAnimation@@UAEPAUIPhonemeLibrary@@XZ 3156f920 f   FaceAnimation.obj
 0001:0006e920       ?GetName@CFacialJoystick@@UAEPBDXZ 3156f920 f   FaceJoystick.obj
 0001:0006e930       ?CreateEffectorsLibrary@CFacialAnimation@@UAEPAUIFacialEffectorsLibrary@@XZ 3156f930 f   FaceAnimation.obj
 0001:0006e950       ?CreateSequence@CFacialAnimation@@UAEPAUIFacialAnimSequence@@XZ 3156f950 f   FaceAnimation.obj
 0001:0006e990       ?GetJoystickContext@CFacialAnimation@@UAEPAVIJoystickContext@@XZ 3156f990 f   FaceAnimation.obj
 0001:0006e9a0       ?CreateJoystick@CFacialAnimation@@UAEPAVIJoystick@@_K@Z 3156f9a0 f   FaceAnimation.obj
 0001:0006e9d0       ?CreateJoystickSet@CFacialAnimation@@UAEPAVIJoystickSet@@XZ 3156f9d0 f   FaceAnimation.obj
 0001:0006e9f0       ?CreateJoystickChannel@CFacialAnimation@@UAEPAVIJoystickChannel@@PAUIFacialAnimChannel@@@Z 3156f9f0 f   FaceAnimation.obj
 0001:0006ea10       ?TemporarilyEnableAdditionalBoneRotationSmoothing@CFacialAnimationContext@@QAEXXZ 3156fa10 f   FaceAnimation.obj
 0001:0006ea20       ?IsBoneRotationSmoothingRequired@CFacialAnimationContext@@QAE_NXZ 3156fa20 f   FaceAnimation.obj
 0001:0006ea40       ??0SFacialEffectorChannel@@QAE@ABU0@@Z 3156fa40 f i FaceAnimation.obj
 0001:0006eaf0       ??$__fill@PAMMH@priv@stlpmtx_std@@YAXPAM0ABMABUrandom_access_iterator_tag@1@PAH@Z 3156faf0 f i FaceAnimation.obj
 0001:0006eb50       ?_Rotate_left@?$_Rb_global@_N@priv@stlpmtx_std@@SAXPAU_Rb_tree_node_base@23@AAPAU423@@Z 3156fb50 f i FaceAnimation.obj
 0001:0006eba0       ?_Rotate_right@?$_Rb_global@_N@priv@stlpmtx_std@@SAXPAU_Rb_tree_node_base@23@AAPAU423@@Z 3156fba0 f i FaceAnimation.obj
 0001:0006ebf0       ?ToUnixPath@PathUtil@@YAXAAV?$CryStackStringT@D$0CAA@@@@Z 3156fbf0 f i FaceAnimation.obj
 0001:0006ec20       ?_Rebalance_for_erase@?$_Rb_global@_N@priv@stlpmtx_std@@SAPAU_Rb_tree_node_base@23@PAU423@AAPAU423@11@Z 3156fc20 f i FaceAnimation.obj
 0001:0006ef10       ??R?$less_stricmp@V?$CryStringT@D@@@stl@@QBE_NABV?$CryStringT@D@@0@Z 3156ff10 f i FaceAnimation.obj
 0001:0006ef40       ??0SPlayingSequence@CFacialAnimationContext@@QAE@ABU01@@Z 3156ff40 f i FaceAnimation.obj
 0001:0006efb0       ??$_M_lower_bound@V?$CryStringT@D@@@?$_Rb_tree@V?$CryStringT@D@@U?$less_stricmp@V?$CryStringT@D@@@stl@@U?$pair@$$CBV?$CryStringT@D@@V?$_smart_ptr@UIFacialAnimSequence@@@@@stlpmtx_std@@U?$_Select1st@U?$pair@$$CBV?$CryStringT@D@@V?$_smart_ptr@UIFacialAnimSequence@@@@@stlpmtx_std@@@priv@5@U?$_MapTraitsT@U?$pair@$$CBV?$CryStringT@D@@V?$_smart_ptr@UIFacialAnimSequence@@@@@stlpmtx_std@@@75@V?$allocator@U?$pair@$$CBV?$CryStringT@D@@V?$_smart_ptr@UIFacialAnimSequence@@@@@stlpmtx_std@@@5@@priv@stlpmtx_std@@ABEPAU_Rb_tree_node_base@12@ABV?$CryStringT@D@@@Z 3156ffb0 f i FaceAnimation.obj
 0001:0006f000       ?_Rebalance@?$_Rb_global@_N@priv@stlpmtx_std@@SAXPAU_Rb_tree_node_base@23@AAPAU423@@Z 31570000 f i FaceAnimation.obj
 0001:0006f1c0       ?GetChannel@CFacialAnimationContext@@QAEPAUSFacialEffectorChannel@@I@Z 315701c0 f   FaceAnimation.obj
 0001:0006f220       ?SetChannelWeight@CFacialAnimationContext@@QAEXIM@Z 31570220 f   FaceAnimation.obj
 0001:0006f280       ?AverageFaceState@CFacialAnimationContext@@AAEXAAVCFaceState@@@Z 31570280 f   FaceAnimation.obj
 0001:0006f320       ?AnimatePlayingSequences@CFacialAnimationContext@@AAEXABU?$QuatTS_tpl@M@@@Z 31570320 f   FaceAnimation.obj
 0001:0006f380       ?SeekSequence@CFacialAnimationContext@@QAEXPAUIFacialAnimSequence@@M@Z 31570380 f   FaceAnimation.obj
 0001:0006f3e0       ?PauseSequence@CFacialAnimationContext@@QAEXPAVCFacialAnimSequence@@_N@Z 315703e0 f   FaceAnimation.obj
 0001:0006f440       ?IsPlayingSequence@CFacialAnimationContext@@QAE_NPAVCFacialAnimSequence@@@Z 31570440 f   FaceAnimation.obj
 0001:0006f480       ??$AddObject@USFacialEffectorChannel@@V?$allocator@USFacialEffectorChannel@@@stlpmtx_std@@@ICrySizer@@QAEXABV?$vector@USFacialEffectorChannel@@V?$allocator@USFacialEffectorChannel@@@stlpmtx_std@@@stlpmtx_std@@@Z 31570480 f i FaceAnimation.obj
 0001:0006f500       ?_M_set@?$_Impl_vector@PAXV?$allocator@PAX@stlpmtx_std@@@priv@stlpmtx_std@@AAEXPAPAX00@Z 31570500 f i LoaderSKIN.obj
 0001:0006f500       ?_M_set@?$_Impl_vector@HV?$allocator@H@stlpmtx_std@@@priv@stlpmtx_std@@AAEXPAH00@Z 31570500 f i ControllerDefragHeap.obj
 0001:0006f500       ?_M_set@?$_Impl_vector@V?$_smart_ptr@VCFacialEffector@@@@V?$allocator@V?$_smart_ptr@VCFacialEffector@@@@@stlpmtx_std@@@priv@stlpmtx_std@@AAEXPAV?$_smart_ptr@VCFacialEffector@@@@00@Z 31570500 f i FaceEffectorLibrary.obj
 0001:0006f500       ?_M_set@?$_Impl_vector@USOp@COperatorQueue@@V?$allocator@USOp@COperatorQueue@@@stlpmtx_std@@@priv@stlpmtx_std@@AAEXPAUSOp@COperatorQueue@@00@Z 31570500 f i OperatorQueue.obj
 0001:0006f500       ?_M_set@?$_Impl_vector@USPhoneme@@V?$allocator@USPhoneme@@@stlpmtx_std@@@priv@stlpmtx_std@@AAEXPAUSPhoneme@@00@Z 31570500 f i LipSync.obj
 0001:0006f500       ?_M_set@?$_Impl_vector@USEffectorInfo@CFacialModel@@V?$allocator@USEffectorInfo@CFacialModel@@@stlpmtx_std@@@priv@stlpmtx_std@@AAEXPAUSEffectorInfo@CFacialModel@@00@Z 31570500 f i FacialModel.obj
 0001:0006f500       ?_M_set@?$_Impl_vector@U?$pair@V?$CryStringT@D@@PAUIFacialAnimChannel@@@stlpmtx_std@@V?$allocator@U?$pair@V?$CryStringT@D@@PAUIFacialAnimChannel@@@stlpmtx_std@@@2@@priv@stlpmtx_std@@AAEXPAU?$pair@V?$CryStringT@D@@PAUIFacialAnimChannel@@@3@00@Z 31570500 f i FaceAnimation.obj
 0001:0006f500       ?_M_set@?$_Impl_vector@USMorphTargetInfo@CFacialModel@@V?$allocator@USMorphTargetInfo@CFacialModel@@@stlpmtx_std@@@priv@stlpmtx_std@@AAEXPAUSMorphTargetInfo@CFacialModel@@00@Z 31570500 f i FacialModel.obj
 0001:0006f560       ?allocate@?$_STLP_alloc_proxy@PAU?$pair@V?$CryStringT@D@@PAUIFacialAnimChannel@@@stlpmtx_std@@U12@V?$allocator@U?$pair@V?$CryStringT@D@@PAUIFacialAnimChannel@@@stlpmtx_std@@@2@@priv@stlpmtx_std@@QAEPAU?$pair@V?$CryStringT@D@@PAUIFacialAnimChannel@@@3@IAAI@Z 31570560 f i FaceAnimation.obj
 0001:0006f5b0       ?lower_bound@?$VectorMap@V?$CryStringT@D@@HU?$less@V?$CryStringT@D@@@stlpmtx_std@@V?$allocator@U?$pair@V?$CryStringT@D@@H@stlpmtx_std@@@3@@@QBEPBU?$pair@V?$CryStringT@D@@H@stlpmtx_std@@ABV?$CryStringT@D@@@Z 315705b0 f i LoaderSKIN.obj
 0001:0006f5b0       ?lower_bound@?$VectorMap@V?$CryStringT@D@@PAUIFacialAnimChannel@@U?$less@V?$CryStringT@D@@@stlpmtx_std@@V?$allocator@U?$pair@V?$CryStringT@D@@PAUIFacialAnimChannel@@@stlpmtx_std@@@4@@@QAEPAU?$pair@V?$CryStringT@D@@PAUIFacialAnimChannel@@@stlpmtx_std@@ABV?$CryStringT@D@@@Z 315705b0 f i FaceAnimation.obj
 0001:0006f640       ??$_M_find@V?$CryStringT@D@@@?$_Rb_tree@V?$CryStringT@D@@U?$less_stricmp@V?$CryStringT@D@@@stl@@U?$pair@$$CBV?$CryStringT@D@@V?$_smart_ptr@UIFacialAnimSequence@@@@@stlpmtx_std@@U?$_Select1st@U?$pair@$$CBV?$CryStringT@D@@V?$_smart_ptr@UIFacialAnimSequence@@@@@stlpmtx_std@@@priv@5@U?$_MapTraitsT@U?$pair@$$CBV?$CryStringT@D@@V?$_smart_ptr@UIFacialAnimSequence@@@@@stlpmtx_std@@@75@V?$allocator@U?$pair@$$CBV?$CryStringT@D@@V?$_smart_ptr@UIFacialAnimSequence@@@@@stlpmtx_std@@@5@@priv@stlpmtx_std@@ABEPAU_Rb_tree_node_base@12@ABV?$CryStringT@D@@@Z 31570640 f i FaceAnimation.obj
 0001:0006f6c0       ??$__copy@PAUSFacialEffectorChannel@@PAU1@H@priv@stlpmtx_std@@YAPAUSFacialEffectorChannel@@PAU2@00ABUrandom_access_iterator_tag@1@PAH@Z 315706c0 f i FaceAnimation.obj
 0001:0006f7c0       ??$__copy@PAUSPlayingSequence@CFacialAnimationContext@@PAU12@H@priv@stlpmtx_std@@YAPAUSPlayingSequence@CFacialAnimationContext@@PAU23@00ABUrandom_access_iterator_tag@1@PAH@Z 315707c0 f i FaceAnimation.obj
 0001:0006f890       ?LoadEffectorsLibrary@CFacialAnimation@@UAEPAUIFacialEffectorsLibrary@@PBD@Z 31570890 f   FaceAnimation.obj
 0001:0006fa40       ?CreateIdentifierHandle@CFacialAnimation@@UAE?AVCFaceIdentifierHandle@@PBD@Z 31570a40 f   FaceAnimation.obj
 0001:0006fa70       ??$AddObject@V?$CryStringT@D@@V?$_smart_ptr@UIFacialAnimSequence@@@@U?$less_stricmp@V?$CryStringT@D@@@stl@@V?$allocator@U?$pair@$$CBV?$CryStringT@D@@V?$_smart_ptr@UIFacialAnimSequence@@@@@stlpmtx_std@@@stlpmtx_std@@@ICrySizer@@QAEXABV?$map@V?$CryStringT@D@@V?$_smart_ptr@UIFacialAnimSequence@@@@U?$less_stricmp@V?$CryStringT@D@@@stl@@V?$allocator@U?$pair@$$CBV?$CryStringT@D@@V?$_smart_ptr@UIFacialAnimSequence@@@@@stlpmtx_std@@@stlpmtx_std@@@stlpmtx_std@@@Z 31570a70 f i FaceAnimation.obj
 0001:0006fb00       ??$AddObject@PAVCFacialEffectorsLibrary@@V?$allocator@PAVCFacialEffectorsLibrary@@@stlpmtx_std@@@ICrySizer@@QAEXABV?$vector@PAVCFacialEffectorsLibrary@@V?$allocator@PAVCFacialEffectorsLibrary@@@stlpmtx_std@@@stlpmtx_std@@@Z 31570b00 f i FaceAnimation.obj
 0001:0006fb70       ??$__uninitialized_fill_n@PAUSFacialEffectorChannel@@IU1@@priv@stlpmtx_std@@YAPAUSFacialEffectorChannel@@PAU2@IABU2@@Z 31570b70 f i FaceAnimation.obj
 0001:0006fbc0       ??$__ufill@PAUSPlayingSequence@CFacialAnimationContext@@U12@H@priv@stlpmtx_std@@YAXPAUSPlayingSequence@CFacialAnimationContext@@0ABU23@ABUrandom_access_iterator_tag@1@PAH@Z 31570bc0 f i FaceAnimation.obj
 0001:0006fc60       ??$__destroy_range_aux@V?$reverse_iterator@PAUSPlayingSequence@CFacialAnimationContext@@@stlpmtx_std@@USPlayingSequence@CFacialAnimationContext@@@stlpmtx_std@@YAXV?$reverse_iterator@PAUSPlayingSequence@CFacialAnimationContext@@@0@0PAUSPlayingSequence@CFacialAnimationContext@@ABU__false_type@0@@Z 31570c60 f i FaceAnimation.obj
 0001:0006fca0       ??$__ucopy@PAUSPlayingSequence@CFacialAnimationContext@@PAU12@H@priv@stlpmtx_std@@YAPAUSPlayingSequence@CFacialAnimationContext@@PAU23@00ABUrandom_access_iterator_tag@1@PAH@Z 31570ca0 f i FaceAnimation.obj
 0001:0006fd40       ??$__unguarded_linear_insert@PAU?$pair@V?$CryStringT@D@@PAUIFacialAnimChannel@@@stlpmtx_std@@U12@VFirstLess@?$VectorMap@V?$CryStringT@D@@PAUIFacialAnimChannel@@U?$less@V?$CryStringT@D@@@stlpmtx_std@@V?$allocator@U?$pair@V?$CryStringT@D@@PAUIFacialAnimChannel@@@stlpmtx_std@@@4@@@@priv@stlpmtx_std@@YAXPAU?$pair@V?$CryStringT@D@@PAUIFacialAnimChannel@@@1@U21@VFirstLess@?$VectorMap@V?$CryStringT@D@@PAUIFacialAnimChannel@@U?$less@V?$CryStringT@D@@@stlpmtx_std@@V?$allocator@U?$pair@V?$CryStringT@D@@PAUIFacialAnimChannel@@@stlpmtx_std@@@4@@@@Z 31570d40 f i FaceAnimation.obj
 0001:0006fd40       ??$__unguarded_linear_insert@PAU?$pair@V?$CryStringT@D@@H@stlpmtx_std@@U12@VFirstLess@?$VectorMap@V?$CryStringT@D@@HU?$less@V?$CryStringT@D@@@stlpmtx_std@@V?$allocator@U?$pair@V?$CryStringT@D@@H@stlpmtx_std@@@3@@@@priv@stlpmtx_std@@YAXPAU?$pair@V?$CryStringT@D@@H@1@U21@VFirstLess@?$VectorMap@V?$CryStringT@D@@HU?$less@V?$CryStringT@D@@@stlpmtx_std@@V?$allocator@U?$pair@V?$CryStringT@D@@H@stlpmtx_std@@@3@@@@Z 31570d40 f i LoaderSKIN.obj
 0001:0006fe80       ??$__copy_backward@PAU?$pair@V?$CryStringT@D@@PAUIFacialAnimChannel@@@stlpmtx_std@@PAU12@H@priv@stlpmtx_std@@YAPAU?$pair@V?$CryStringT@D@@PAUIFacialAnimChannel@@@1@PAU21@00ABUrandom_access_iterator_tag@1@PAH@Z 31570e80 f i FaceAnimation.obj
 0001:0006fe80       ??$__copy_backward@PAU?$pair@V?$CryStringT@D@@H@stlpmtx_std@@PAU12@H@priv@stlpmtx_std@@YAPAU?$pair@V?$CryStringT@D@@H@1@PAU21@00ABUrandom_access_iterator_tag@1@PAH@Z 31570e80 f i LoaderSKIN.obj
 0001:00070000       ?ToUnixPath@PathUtil@@YA?AV?$CryStringT@D@@ABV2@@Z 31571000 f i FaceAnimation.obj
 0001:000700d0       ??$AddObject@USPhoneme@@V?$allocator@USPhoneme@@@stlpmtx_std@@@ICrySizer@@QAEXABV?$vector@USPhoneme@@V?$allocator@USPhoneme@@@stlpmtx_std@@@stlpmtx_std@@@Z 315710d0 f i FaceAnimation.obj
 0001:00070150       ??$find_and_erase@V?$vector@PAVCFacialEffectorsLibrary@@V?$allocator@PAVCFacialEffectorsLibrary@@@stlpmtx_std@@@stlpmtx_std@@PAVCFacialEffectorsLibrary@@@stl@@YA_NAAV?$vector@PAVCFacialEffectorsLibrary@@V?$allocator@PAVCFacialEffectorsLibrary@@@stlpmtx_std@@@stlpmtx_std@@ABQAVCFacialEffectorsLibrary@@@Z 31571150 f i FaceAnimation.obj
 0001:000701c0       ??$AddObject@USPlayingSequence@CFacialAnimationContext@@V?$allocator@USPlayingSequence@CFacialAnimationContext@@@stlpmtx_std@@@ICrySizer@@QAEXABV?$vector@USPlayingSequence@CFacialAnimationContext@@V?$allocator@USPlayingSequence@CFacialAnimationContext@@@stlpmtx_std@@@stlpmtx_std@@@Z 315711c0 f i FaceAnimation.obj
 0001:00070250       ?_M_insert_overflow@?$_Impl_vector@MV?$allocator@M@stlpmtx_std@@@priv@stlpmtx_std@@AAEXPAMABMABU__true_type@3@I_N@Z 31571250 f i FaceAnimation.obj
 0001:000703a0       ?_M_fill_insert_aux@?$_Impl_vector@MV?$allocator@M@stlpmtx_std@@@priv@stlpmtx_std@@AAEXPAMIABMABU__false_type@3@@Z 315713a0 f i FaceAnimation.obj
 0001:000704d0       ??$__unguarded_insertion_sort_aux@PAU?$pair@V?$CryStringT@D@@PAUIFacialAnimChannel@@@stlpmtx_std@@U12@VFirstLess@?$VectorMap@V?$CryStringT@D@@PAUIFacialAnimChannel@@U?$less@V?$CryStringT@D@@@stlpmtx_std@@V?$allocator@U?$pair@V?$CryStringT@D@@PAUIFacialAnimChannel@@@stlpmtx_std@@@4@@@@priv@stlpmtx_std@@YAXPAU?$pair@V?$CryStringT@D@@PAUIFacialAnimChannel@@@1@00VFirstLess@?$VectorMap@V?$CryStringT@D@@PAUIFacialAnimChannel@@U?$less@V?$CryStringT@D@@@stlpmtx_std@@V?$allocator@U?$pair@V?$CryStringT@D@@PAUIFacialAnimChannel@@@stlpmtx_std@@@4@@@@Z 315714d0 f i FaceAnimation.obj
 0001:00070520       ?ApplyEffector@CFacialAnimationContext@@QAEXAAVCFaceState@@PAVCFacialEffector@@MM_N@Z 31571520 f   FaceAnimation.obj
 0001:000706f0       ?ClearEffectorsLibraryFromCache@CFacialAnimation@@UAEXPBD@Z 315716f0 f   FaceAnimation.obj
 0001:000708a0       ?UnregisterLib@CFacialAnimation@@QAEXPAVCFacialEffectorsLibrary@@@Z 315718a0 f   FaceAnimation.obj
 0001:000708c0       ?OnSequenceStreamed@CFacialAnimation@@QAEXPAUIFacialAnimSequence@@_N@Z 315718c0 f   FaceAnimation.obj
 0001:00070970       ?GetMemoryUsage@CFacialAnimationContext@@QBEXPAVICrySizer@@@Z 31571970 f   FaceAnimation.obj
 0001:00070a30       ?_M_erase@?$_Impl_vector@USPlayingSequence@CFacialAnimationContext@@V?$allocator@USPlayingSequence@CFacialAnimationContext@@@stlpmtx_std@@@priv@stlpmtx_std@@AAEPAUSPlayingSequence@CFacialAnimationContext@@PAU45@0ABU__false_type@3@@Z 31571a30 f i FaceAnimation.obj
 0001:00070ab0       ?RemoveExtension@PathUtil@@YAXAAV?$CryStringT@D@@@Z 31571ab0 f i FaceAnimation.obj
 0001:00070bf0       ?ReplaceExtension@PathUtil@@YA?AV?$CryStringT@D@@ABV2@PBD@Z 31571bf0 f i FaceAnimation.obj
 0001:00070c60       ?ReplaceExtension@PathUtil@@YA?AV?$CryStringT@D@@PBD0@Z 31571c60 f i FaceAnimation.obj
 0001:00070d00       ??$__ufill@PAU?$pair@V?$CryStringT@D@@H@stlpmtx_std@@U12@H@priv@stlpmtx_std@@YAXPAU?$pair@V?$CryStringT@D@@H@1@0ABU21@ABUrandom_access_iterator_tag@1@PAH@Z 31571d00 f i LoaderSKIN.obj
 0001:00070d00       ??$__ufill@PAU?$pair@V?$CryStringT@D@@PAUIFacialAnimChannel@@@stlpmtx_std@@U12@H@priv@stlpmtx_std@@YAXPAU?$pair@V?$CryStringT@D@@PAUIFacialAnimChannel@@@1@0ABU21@ABUrandom_access_iterator_tag@1@PAH@Z 31571d00 f i FaceAnimation.obj
 0001:00070d40       ?LoadJoystickSet@CFacialAnimation@@UAEPAVIJoystickSet@@PBD_N@Z 31571d40 f   FaceAnimation.obj
 0001:00070ef0       ??1?$_Impl_vector@UChannelInfo@CFacialAnimSequenceInstance@@V?$allocator@UChannelInfo@CFacialAnimSequenceInstance@@@stlpmtx_std@@@priv@stlpmtx_std@@QAE@XZ 31571ef0 f i FaceAnimation.obj
 0001:00070f40       ?erase@?$vector@USFacialEffectorChannel@@V?$allocator@USFacialEffectorChannel@@@stlpmtx_std@@@stlpmtx_std@@QAEPAUSFacialEffectorChannel@@PAU3@@Z 31571f40 f i FaceAnimation.obj
 0001:00070fa0       ??1?$_Impl_vector@USFacialEffectorChannel@@V?$allocator@USFacialEffectorChannel@@@stlpmtx_std@@@priv@stlpmtx_std@@QAE@XZ 31571fa0 f i FaceAnimation.obj
 0001:00070ff0       ?erase@?$_Rb_tree@V?$CryStringT@D@@U?$less_stricmp@V?$CryStringT@D@@@stl@@U?$pair@$$CBV?$CryStringT@D@@V?$_smart_ptr@UIFacialAnimSequence@@@@@stlpmtx_std@@U?$_Select1st@U?$pair@$$CBV?$CryStringT@D@@V?$_smart_ptr@UIFacialAnimSequence@@@@@stlpmtx_std@@@priv@5@U?$_MapTraitsT@U?$pair@$$CBV?$CryStringT@D@@V?$_smart_ptr@UIFacialAnimSequence@@@@@stlpmtx_std@@@75@V?$allocator@U?$pair@$$CBV?$CryStringT@D@@V?$_smart_ptr@UIFacialAnimSequence@@@@@stlpmtx_std@@@5@@priv@stlpmtx_std@@QAEXU?$_Rb_tree_iterator@U?$pair@$$CBV?$CryStringT@D@@V?$_smart_ptr@UIFacialAnimSequence@@@@@stlpmtx_std@@U?$_MapTraitsT@U?$pair@$$CBV?$CryStringT@D@@V?$_smart_ptr@UIFacialAnimSequence@@@@@stlpmtx_std@@@priv@2@@23@@Z 31571ff0 f i FaceAnimation.obj
 0001:00071060       ?_M_insert_overflow_aux@?$_Impl_vector@USFacialEffectorChannel@@V?$allocator@USFacialEffectorChannel@@@stlpmtx_std@@@priv@stlpmtx_std@@AAEXPAUSFacialEffectorChannel@@ABU4@ABU__false_type@3@I_N@Z 31572060 f i FaceAnimation.obj
 0001:00071260       ?_M_insert_overflow_aux@?$_Impl_vector@USPlayingSequence@CFacialAnimationContext@@V?$allocator@USPlayingSequence@CFacialAnimationContext@@@stlpmtx_std@@@priv@stlpmtx_std@@AAEXPAUSPlayingSequence@CFacialAnimationContext@@ABU45@ABU__false_type@3@I_N@Z 31572260 f i FaceAnimation.obj
 0001:00071410       ?_M_erase@?$_Rb_tree@V?$CryStringT@D@@U?$less_stricmp@V?$CryStringT@D@@@stl@@U?$pair@$$CBV?$CryStringT@D@@V?$_smart_ptr@UIFacialAnimSequence@@@@@stlpmtx_std@@U?$_Select1st@U?$pair@$$CBV?$CryStringT@D@@V?$_smart_ptr@UIFacialAnimSequence@@@@@stlpmtx_std@@@priv@5@U?$_MapTraitsT@U?$pair@$$CBV?$CryStringT@D@@V?$_smart_ptr@UIFacialAnimSequence@@@@@stlpmtx_std@@@75@V?$allocator@U?$pair@$$CBV?$CryStringT@D@@V?$_smart_ptr@UIFacialAnimSequence@@@@@stlpmtx_std@@@5@@priv@stlpmtx_std@@AAEXPAU_Rb_tree_node_base@23@@Z 31572410 f i FaceAnimation.obj
 0001:00071480       ??$push_back_unique@V?$vector@PAVCFacialEffectorsLibrary@@V?$allocator@PAVCFacialEffectorsLibrary@@@stlpmtx_std@@@stlpmtx_std@@PAVCFacialEffectorsLibrary@@@stl@@YA_NAAV?$vector@PAVCFacialEffectorsLibrary@@V?$allocator@PAVCFacialEffectorsLibrary@@@stlpmtx_std@@@stlpmtx_std@@ABQAVCFacialEffectorsLibrary@@@Z 31572480 f i FaceAnimation.obj
 0001:000714f0       ?_M_create_node@?$_Rb_tree@V?$CryStringT@D@@U?$less_stricmp@V?$CryStringT@D@@@stl@@U?$pair@$$CBV?$CryStringT@D@@V?$_smart_ptr@UIFacialAnimSequence@@@@@stlpmtx_std@@U?$_Select1st@U?$pair@$$CBV?$CryStringT@D@@V?$_smart_ptr@UIFacialAnimSequence@@@@@stlpmtx_std@@@priv@5@U?$_MapTraitsT@U?$pair@$$CBV?$CryStringT@D@@V?$_smart_ptr@UIFacialAnimSequence@@@@@stlpmtx_std@@@75@V?$allocator@U?$pair@$$CBV?$CryStringT@D@@V?$_smart_ptr@UIFacialAnimSequence@@@@@stlpmtx_std@@@5@@priv@stlpmtx_std@@IAEPAU_Rb_tree_node_base@23@ABU?$pair@$$CBV?$CryStringT@D@@V?$_smart_ptr@UIFacialAnimSequence@@@@@3@@Z 315724f0 f i FaceAnimation.obj
 0001:00071560       ?StopChannel@CFacialAnimationContext@@QAEXIM@Z 31572560 f   FaceAnimation.obj
 0001:00071670       ?RemoveChannel@CFacialAnimationContext@@QAEXI@Z 31572670 f   FaceAnimation.obj
 0001:00071770       ?RemoveAllPreviewChannels@CFacialAnimationContext@@QAEXXZ 31572770 f   FaceAnimation.obj
 0001:00071820       ?StopSequence@CFacialAnimationContext@@QAEXPAVCFacialAnimSequence@@@Z 31572820 f   FaceAnimation.obj
 0001:00071960       ?RegisterLib@CFacialAnimation@@QAEXPAVCFacialEffectorsLibrary@@@Z 31572960 f   FaceAnimation.obj
 0001:00071980       ?GetMemoryUsage@CFacialAnimation@@QBEXPAVICrySizer@@@Z 31572980 f   FaceAnimation.obj
 0001:000719d0       ?resize@?$_Impl_vector@MV?$allocator@M@stlpmtx_std@@@priv@stlpmtx_std@@QAEXIABM@Z 315729d0 f i FaceAnimation.obj
 0001:00071a70       ?_M_insert@?$_Rb_tree@V?$CryStringT@D@@U?$less_stricmp@V?$CryStringT@D@@@stl@@U?$pair@$$CBV?$CryStringT@D@@V?$_smart_ptr@UIFacialAnimSequence@@@@@stlpmtx_std@@U?$_Select1st@U?$pair@$$CBV?$CryStringT@D@@V?$_smart_ptr@UIFacialAnimSequence@@@@@stlpmtx_std@@@priv@5@U?$_MapTraitsT@U?$pair@$$CBV?$CryStringT@D@@V?$_smart_ptr@UIFacialAnimSequence@@@@@stlpmtx_std@@@75@V?$allocator@U?$pair@$$CBV?$CryStringT@D@@V?$_smart_ptr@UIFacialAnimSequence@@@@@stlpmtx_std@@@5@@priv@stlpmtx_std@@AAE?AU?$_Rb_tree_iterator@U?$pair@$$CBV?$CryStringT@D@@V?$_smart_ptr@UIFacialAnimSequence@@@@@stlpmtx_std@@U?$_MapTraitsT@U?$pair@$$CBV?$CryStringT@D@@V?$_smart_ptr@UIFacialAnimSequence@@@@@stlpmtx_std@@@priv@2@@23@PAU_Rb_tree_node_base@23@ABU?$pair@$$CBV?$CryStringT@D@@V?$_smart_ptr@UIFacialAnimSequence@@@@@3@00@Z 31572a70 f i FaceAnimation.obj
 0001:00071b10       ?insert_unique@?$_Rb_tree@V?$CryStringT@D@@U?$less_stricmp@V?$CryStringT@D@@@stl@@U?$pair@$$CBV?$CryStringT@D@@V?$_smart_ptr@UIFacialAnimSequence@@@@@stlpmtx_std@@U?$_Select1st@U?$pair@$$CBV?$CryStringT@D@@V?$_smart_ptr@UIFacialAnimSequence@@@@@stlpmtx_std@@@priv@5@U?$_MapTraitsT@U?$pair@$$CBV?$CryStringT@D@@V?$_smart_ptr@UIFacialAnimSequence@@@@@stlpmtx_std@@@75@V?$allocator@U?$pair@$$CBV?$CryStringT@D@@V?$_smart_ptr@UIFacialAnimSequence@@@@@stlpmtx_std@@@5@@priv@stlpmtx_std@@QAE?AU?$pair@U?$_Rb_tree_iterator@U?$pair@$$CBV?$CryStringT@D@@V?$_smart_ptr@UIFacialAnimSequence@@@@@stlpmtx_std@@U?$_MapTraitsT@U?$pair@$$CBV?$CryStringT@D@@V?$_smart_ptr@UIFacialAnimSequence@@@@@stlpmtx_std@@@priv@2@@priv@stlpmtx_std@@_N@3@ABU?$pair@$$CBV?$CryStringT@D@@V?$_smart_ptr@UIFacialAnimSequence@@@@@3@@Z 31572b10 f i FaceAnimation.obj
 0001:00071c50       ??$__linear_insert@PAU?$pair@V?$CryStringT@D@@H@stlpmtx_std@@U12@VFirstLess@?$VectorMap@V?$CryStringT@D@@HU?$less@V?$CryStringT@D@@@stlpmtx_std@@V?$allocator@U?$pair@V?$CryStringT@D@@H@stlpmtx_std@@@3@@@@priv@stlpmtx_std@@YAXPAU?$pair@V?$CryStringT@D@@H@1@0U21@VFirstLess@?$VectorMap@V?$CryStringT@D@@HU?$less@V?$CryStringT@D@@@stlpmtx_std@@V?$allocator@U?$pair@V?$CryStringT@D@@H@stlpmtx_std@@@3@@@@Z 31572c50 f i LoaderSKIN.obj
 0001:00071c50       ??$__linear_insert@PAU?$pair@V?$CryStringT@D@@PAUIFacialAnimChannel@@@stlpmtx_std@@U12@VFirstLess@?$VectorMap@V?$CryStringT@D@@PAUIFacialAnimChannel@@U?$less@V?$CryStringT@D@@@stlpmtx_std@@V?$allocator@U?$pair@V?$CryStringT@D@@PAUIFacialAnimChannel@@@stlpmtx_std@@@4@@@@priv@stlpmtx_std@@YAXPAU?$pair@V?$CryStringT@D@@PAUIFacialAnimChannel@@@1@0U21@VFirstLess@?$VectorMap@V?$CryStringT@D@@PAUIFacialAnimChannel@@U?$less@V?$CryStringT@D@@@stlpmtx_std@@V?$allocator@U?$pair@V?$CryStringT@D@@PAUIFacialAnimChannel@@@stlpmtx_std@@@4@@@@Z 31572c50 f i FaceAnimation.obj
 0001:00071d10       ??0CFacialAnimSequenceInstance@@QAE@XZ 31572d10 f i FaceAnimation.obj
 0001:00071db0       ??1CFacialAnimSequenceInstance@@UAE@XZ 31572db0 f i FaceAnimation.obj
 0001:00071e30       ??_ECFacialAnimSequenceInstance@@UAEPAXI@Z 31572e30 f i FaceAnimation.obj
 0001:00071e30       ??_GCFacialAnimSequenceInstance@@UAEPAXI@Z 31572e30 f i FaceAnimation.obj
 0001:00071e60       ??0CFacialAnimationContext@@QAE@PAVCFacialInstance@@@Z 31572e60 f   FaceAnimation.obj
 0001:00071f20       ??1CFacialAnimationContext@@UAE@XZ 31572f20 f i FaceAnimation.obj
 0001:00072000       ??_ECFacialAnimationContext@@UAEPAXI@Z 31573000 f i FaceAnimation.obj
 0001:00072000       ??_GCFacialAnimationContext@@UAEPAXI@Z 31573000 f i FaceAnimation.obj
 0001:00072030       ?UpdatePlayingSequences@CFacialAnimationContext@@QAEXABU?$QuatTS_tpl@M@@@Z 31573030 f   FaceAnimation.obj
 0001:000722f0       ?insert_unique@?$_Rb_tree@V?$CryStringT@D@@U?$less_stricmp@V?$CryStringT@D@@@stl@@U?$pair@$$CBV?$CryStringT@D@@V?$_smart_ptr@UIFacialAnimSequence@@@@@stlpmtx_std@@U?$_Select1st@U?$pair@$$CBV?$CryStringT@D@@V?$_smart_ptr@UIFacialAnimSequence@@@@@stlpmtx_std@@@priv@5@U?$_MapTraitsT@U?$pair@$$CBV?$CryStringT@D@@V?$_smart_ptr@UIFacialAnimSequence@@@@@stlpmtx_std@@@75@V?$allocator@U?$pair@$$CBV?$CryStringT@D@@V?$_smart_ptr@UIFacialAnimSequence@@@@@stlpmtx_std@@@5@@priv@stlpmtx_std@@QAE?AU?$_Rb_tree_iterator@U?$pair@$$CBV?$CryStringT@D@@V?$_smart_ptr@UIFacialAnimSequence@@@@@stlpmtx_std@@U?$_MapTraitsT@U?$pair@$$CBV?$CryStringT@D@@V?$_smart_ptr@UIFacialAnimSequence@@@@@stlpmtx_std@@@priv@2@@23@U423@ABU?$pair@$$CBV?$CryStringT@D@@V?$_smart_ptr@UIFacialAnimSequence@@@@@3@@Z 315732f0 f i FaceAnimation.obj
 0001:00072580       ??$_M_allocate_and_copy@PAU?$pair@V?$CryStringT@D@@PAUIFacialAnimChannel@@@stlpmtx_std@@@?$_Impl_vector@U?$pair@V?$CryStringT@D@@PAUIFacialAnimChannel@@@stlpmtx_std@@V?$allocator@U?$pair@V?$CryStringT@D@@PAUIFacialAnimChannel@@@stlpmtx_std@@@2@@priv@stlpmtx_std@@AAEPAU?$pair@V?$CryStringT@D@@PAUIFacialAnimChannel@@@2@AAIPAU32@1@Z 31573580 f i FaceAnimation.obj
 0001:000725f0       ??$__insertion_sort@PAU?$pair@V?$CryStringT@D@@PAUIFacialAnimChannel@@@stlpmtx_std@@U12@VFirstLess@?$VectorMap@V?$CryStringT@D@@PAUIFacialAnimChannel@@U?$less@V?$CryStringT@D@@@stlpmtx_std@@V?$allocator@U?$pair@V?$CryStringT@D@@PAUIFacialAnimChannel@@@stlpmtx_std@@@4@@@@priv@stlpmtx_std@@YAXPAU?$pair@V?$CryStringT@D@@PAUIFacialAnimChannel@@@1@00VFirstLess@?$VectorMap@V?$CryStringT@D@@PAUIFacialAnimChannel@@U?$less@V?$CryStringT@D@@@stlpmtx_std@@V?$allocator@U?$pair@V?$CryStringT@D@@PAUIFacialAnimChannel@@@stlpmtx_std@@@4@@@@Z 315735f0 f i FaceAnimation.obj
 0001:000725f0       ??$__insertion_sort@PAU?$pair@V?$CryStringT@D@@H@stlpmtx_std@@U12@VFirstLess@?$VectorMap@V?$CryStringT@D@@HU?$less@V?$CryStringT@D@@@stlpmtx_std@@V?$allocator@U?$pair@V?$CryStringT@D@@H@stlpmtx_std@@@3@@@@priv@stlpmtx_std@@YAXPAU?$pair@V?$CryStringT@D@@H@1@00VFirstLess@?$VectorMap@V?$CryStringT@D@@HU?$less@V?$CryStringT@D@@@stlpmtx_std@@V?$allocator@U?$pair@V?$CryStringT@D@@H@stlpmtx_std@@@3@@@@Z 315735f0 f i LoaderSKIN.obj
 0001:00072650       ?ResetFaceState@CFacialAnimationContext@@AAEXAAVCFaceState@@@Z 31573650 f   FaceAnimation.obj
 0001:00072700       ?StopAllSequences@CFacialAnimationContext@@QAEXXZ 31573700 f   FaceAnimation.obj
 0001:00072780       ??1CFacialAnimation@@UAE@XZ 31573780 f   FaceAnimation.obj
 0001:00072810       ??_ECFacialAnimation@@W3AEPAXI@Z 31573810 f i FaceAnimation.obj
 0001:00072820       ?ClearAllCaches@CFacialAnimation@@UAEXXZ 31573820 f   FaceAnimation.obj
 0001:00072890       ?ClearSequenceFromCache@CFacialAnimation@@UAEXPBD@Z 31573890 f   FaceAnimation.obj
 0001:000728f0       ?reserve@?$_Impl_vector@U?$pair@V?$CryStringT@D@@PAUIFacialAnimChannel@@@stlpmtx_std@@V?$allocator@U?$pair@V?$CryStringT@D@@PAUIFacialAnimChannel@@@stlpmtx_std@@@2@@priv@stlpmtx_std@@QAEXI@Z 315738f0 f i FaceAnimation.obj
 0001:00072990       ?StartChannel@CFacialAnimationContext@@QAEIAAUSFacialEffectorChannel@@@Z 31573990 f   FaceAnimation.obj
 0001:00072a10       ?FadeInChannel@CFacialAnimationContext@@QAEIPAUIFacialEffector@@MMMH@Z 31573a10 f   FaceAnimation.obj
 0001:00072b10       ?Update@CFacialAnimationContext@@QAE_NAAVCFaceState@@ABU?$QuatTS_tpl@M@@@Z 31573b10 f   FaceAnimation.obj
 0001:000730c0       ?PlaySequence@CFacialAnimationContext@@QAEXPAVCFacialAnimSequence@@_N1@Z 315740c0 f   FaceAnimation.obj
 0001:000732c0       ??0CFacialAnimation@@QAE@XZ 315742c0 f   FaceAnimation.obj
 0001:00073350       ??_ECFacialAnimation@@UAEPAXI@Z 31574350 f i FaceAnimation.obj
 0001:00073350       ??_GCFacialAnimation@@UAEPAXI@Z 31574350 f i FaceAnimation.obj
 0001:00073380       ?push_back@?$_Impl_vector@U?$pair@V?$CryStringT@D@@PAUIFacialAnimChannel@@@stlpmtx_std@@V?$allocator@U?$pair@V?$CryStringT@D@@PAUIFacialAnimChannel@@@stlpmtx_std@@@2@@priv@stlpmtx_std@@QAEXABU?$pair@V?$CryStringT@D@@PAUIFacialAnimChannel@@@3@@Z 31574380 f i FaceAnimation.obj
 0001:000733f0       ??$?AV?$CryStringT@D@@@?$map@V?$CryStringT@D@@V?$_smart_ptr@UIFacialAnimSequence@@@@U?$less_stricmp@V?$CryStringT@D@@@stl@@V?$allocator@U?$pair@$$CBV?$CryStringT@D@@V?$_smart_ptr@UIFacialAnimSequence@@@@@stlpmtx_std@@@stlpmtx_std@@@stlpmtx_std@@QAEAAV?$_smart_ptr@UIFacialAnimSequence@@@@ABV?$CryStringT@D@@@Z 315743f0 f i FaceAnimation.obj
 0001:00073490       ?RenameAnimSequence@CFacialAnimation@@QAEXPAVCFacialAnimSequence@@PBD_N@Z 31574490 f   FaceAnimation.obj
 0001:000735b0       ?LoadSequence@CFacialAnimation@@UAEPAUIFacialAnimSequence@@PBD_N1@Z 315745b0 f   FaceAnimation.obj
 0001:00073840       ?StartStreamingSequence@CFacialAnimation@@UAEPAUIFacialAnimSequence@@PBD@Z 31574840 f   FaceAnimation.obj
 0001:000739e0       ??$sort@PAU?$pair@V?$CryStringT@D@@PAUIFacialAnimChannel@@@stlpmtx_std@@VFirstLess@?$VectorMap@V?$CryStringT@D@@PAUIFacialAnimChannel@@U?$less@V?$CryStringT@D@@@stlpmtx_std@@V?$allocator@U?$pair@V?$CryStringT@D@@PAUIFacialAnimChannel@@@stlpmtx_std@@@4@@@@stlpmtx_std@@YAXPAU?$pair@V?$CryStringT@D@@PAUIFacialAnimChannel@@@0@0VFirstLess@?$VectorMap@V?$CryStringT@D@@PAUIFacialAnimChannel@@U?$less@V?$CryStringT@D@@@stlpmtx_std@@V?$allocator@U?$pair@V?$CryStringT@D@@PAUIFacialAnimChannel@@@stlpmtx_std@@@4@@@@Z 315749e0 f i FaceAnimation.obj
 0001:00073a60       ?BindJoystickSetToSequence@CFacialAnimation@@UAEXPAVIJoystickSet@@PAUIFacialAnimSequence@@@Z 31574a60 f   FaceAnimation.obj
 0001:00073ff0       ??_GIFacialAnimSoundEntry@@UAEPAXI@Z 31574ff0 f i FaceAnimSequence.obj
 0001:00073ff0       ??_EIFacialAnimSoundEntry@@UAEPAXI@Z 31574ff0 f i FaceAnimSequence.obj
 0001:00074020       ??_GIFacialAnimSequence@@UAEPAXI@Z 31575020 f i FaceAnimSequence.obj
 0001:00074020       ??_EIFacialAnimSequence@@UAEPAXI@Z 31575020 f i FaceAnimSequence.obj
 0001:00074050       ?Release@CFacialAnimSequence@@UAEXXZ 31575050 f   FaceAnimSequence.obj
 0001:00074070       ?SetName@CFacialAnimSequence@@UAEXPBD@Z 31575070 f   FaceAnimSequence.obj
 0001:00074090       ?GetStartTime@CFacialAnimSoundEntry@@UAEMXZ 31575090 f   FaceAnimSequence.obj
 0001:000740a0       ?SetStartTime@CFacialAnimSoundEntry@@UAEXM@Z 315750a0 f   FaceAnimSequence.obj
 0001:000740c0       ?SetStartTime@CFacialAnimSkeletalAnimationEntry@@UAEXM@Z 315750c0 f   FaceAnimSequence.obj
 0001:000740e0       ?GetStartTime@CFacialAnimSkeletalAnimationEntry@@UBEMXZ 315750e0 f   FaceAnimSequence.obj
 0001:000740f0       ?SetEndTime@CFacialAnimSkeletalAnimationEntry@@UAEXM@Z 315750f0 f   FaceAnimSequence.obj
 0001:00074110       ?GetEndTime@CFacialAnimSkeletalAnimationEntry@@UBEMXZ 31575110 f   FaceAnimSequence.obj
 0001:00074120       ??$__fill@U?$_Bit_iter@U_Bit_reference@priv@stlpmtx_std@@PAU123@@priv@stlpmtx_std@@_NH@priv@stlpmtx_std@@YAXU?$_Bit_iter@U_Bit_reference@priv@stlpmtx_std@@PAU123@@01@0AB_NABUrandom_access_iterator_tag@1@PAH@Z 31575120 f i FaceAnimSequence.obj
 0001:00074180       ??$__fill_n@U?$_Bit_iter@U_Bit_reference@priv@stlpmtx_std@@PAU123@@priv@stlpmtx_std@@I_N@priv@stlpmtx_std@@YA?AU?$_Bit_iter@U_Bit_reference@priv@stlpmtx_std@@PAU123@@01@U201@IAB_N@Z 31575180 f i FaceAnimSequence.obj
 0001:000741e0       ??$__copy@U?$_Bit_iter@U_Bit_reference@priv@stlpmtx_std@@PAU123@@priv@stlpmtx_std@@U123@H@priv@stlpmtx_std@@YA?AU?$_Bit_iter@U_Bit_reference@priv@stlpmtx_std@@PAU123@@01@U201@00ABUrandom_access_iterator_tag@1@PAH@Z 315751e0 f i FaceAnimSequence.obj
 0001:00074270       ??$__copy_backward@PAUChannelInfo@CFacialAnimSequenceInstance@@PAU12@H@priv@stlpmtx_std@@YAPAUChannelInfo@CFacialAnimSequenceInstance@@PAU23@00ABUrandom_access_iterator_tag@1@PAH@Z 31575270 f i FaceAnimSequence.obj
 0001:000742f0       ??$__fill@PAUChannelInfo@CFacialAnimSequenceInstance@@U12@H@priv@stlpmtx_std@@YAXPAUChannelInfo@CFacialAnimSequenceInstance@@0ABU23@ABUrandom_access_iterator_tag@1@PAH@Z 315752f0 f i FaceAnimSequence.obj
 0001:00074360       ??_GISplineInterpolator@@UAEPAXI@Z 31575360 f i FaceAnimSequence.obj
 0001:00074360       ??_GIFacialAnimChannel@@UAEPAXI@Z 31575360 f i FaceAnimSequence.obj
 0001:00074360       ??_EIFacialAnimChannel@@UAEPAXI@Z 31575360 f i FaceAnimSequence.obj
 0001:00074360       ??_EISplineInterpolator@@UAEPAXI@Z 31575360 f i FaceAnimSequence.obj
 0001:00074390       ?StreamOnNeedStorage@IStreamCallback@@UAEPAXPAVIReadStream@@I@Z 31575390 f i FaceAnimSequence.obj
 0001:000743a0       ??_EIStreamCallback@@UAEPAXI@Z 315753a0 f i FaceAnimSequence.obj
 0001:000743a0       ??_GIStreamCallback@@UAEPAXI@Z 315753a0 f i FaceAnimSequence.obj
 0001:000743d0       ?GetFacialInstance@CCharInstance@@UAEPAUIFacialInstance@@XZ 315753d0 f   CharacterInstance.obj
 0001:000743d0       ?GetEffector@CFacialEffCtrl@@UAEPAUIFacialEffector@@XZ 315753d0 f   FaceEffector.obj
 0001:000743d0       ?GetJoystickFile@CFacialAnimSequence@@UBEPBDXZ 315753d0 f   FaceAnimSequence.obj
 0001:000743e0       ??H?$_Bit_iter@U_Bit_reference@priv@stlpmtx_std@@PAU123@@priv@stlpmtx_std@@QBE?AU012@H@Z 315753e0 f i FaceAnimSequence.obj
 0001:00074430       ??$move_init@U?$TCBSplineKey@U?$Vec3_tpl@M@@@spline@@@NArray@@YAXPAU?$TCBSplineKey@U?$Vec3_tpl@M@@@spline@@0I@Z 31575430 f i FaceAnimSequence.obj
 0001:00074470       ??$__copy_backward@U?$_Bit_iter@U_Bit_reference@priv@stlpmtx_std@@PAU123@@priv@stlpmtx_std@@U123@H@priv@stlpmtx_std@@YA?AU?$_Bit_iter@U_Bit_reference@priv@stlpmtx_std@@PAU123@@01@U201@00ABUrandom_access_iterator_tag@1@PAH@Z 31575470 f i FaceAnimSequence.obj
 0001:00074500       ?lower_bound@?$VectorMap@PAUIFacialAnimChannel@@HU?$less@PAUIFacialAnimChannel@@@stlpmtx_std@@V?$allocator@U?$pair@PAUIFacialAnimChannel@@H@stlpmtx_std@@@3@@@QAEPAU?$pair@PAUIFacialAnimChannel@@H@stlpmtx_std@@ABQAUIFacialAnimChannel@@@Z 31575500 f i FaceAnimSequence.obj
 0001:00074550       ??$__copy@PAV?$_smart_ptr@VCFacialEffector@@@@PAV1@H@priv@stlpmtx_std@@YAPAV?$_smart_ptr@VCFacialEffector@@@@PAV2@00ABUrandom_access_iterator_tag@1@PAH@Z 31575550 f i FaceEffectorLibrary.obj
 0001:00074550       ??$__copy@PAV?$_smart_ptr@VCFacialAnimChannel@@@@PAV1@H@priv@stlpmtx_std@@YAPAV?$_smart_ptr@VCFacialAnimChannel@@@@PAV2@00ABUrandom_access_iterator_tag@1@PAH@Z 31575550 f i FaceAnimSequence.obj
 0001:00074550       ??$__copy@PAV?$_smart_ptr@VCFacialEffCtrl@@@@PAV1@H@priv@stlpmtx_std@@YAPAV?$_smart_ptr@VCFacialEffCtrl@@@@PAV2@00ABUrandom_access_iterator_tag@1@PAH@Z 31575550 f i FaceEffector.obj
 0001:000745b0       ??$__copy@PAUChannelInfo@CFacialAnimSequenceInstance@@PAU12@H@priv@stlpmtx_std@@YAPAUChannelInfo@CFacialAnimSequenceInstance@@PAU23@00ABUrandom_access_iterator_tag@1@PAH@Z 315755b0 f i FaceAnimSequence.obj
 0001:00074630       ??$__lower_bound@PAVEffectorChannelPair@@V1@U?$__less_2@VEffectorChannelPair@@V1@@priv@stlpmtx_std@@U234@H@priv@stlpmtx_std@@YAPAVEffectorChannelPair@@PAV2@0ABV2@U?$__less_2@VEffectorChannelPair@@V1@@01@2PAH@Z 31575630 f i FaceAnimSequence.obj
 0001:00074670       ??$__upper_bound@PAVEffectorChannelPair@@V1@U?$__less_2@VEffectorChannelPair@@V1@@priv@stlpmtx_std@@U234@H@priv@stlpmtx_std@@YAPAVEffectorChannelPair@@PAV2@0ABV2@U?$__less_2@VEffectorChannelPair@@V1@@01@2PAH@Z 31575670 f i FaceAnimSequence.obj
 0001:000746b0       ??$__unguarded_linear_insert@PAU?$SplineKey@M@spline@@U12@U?$less@U?$SplineKey@M@spline@@@stlpmtx_std@@@priv@stlpmtx_std@@YAXPAU?$SplineKey@M@spline@@U23@U?$less@U?$SplineKey@M@spline@@@1@@Z 315756b0 f i FaceAnimSequence.obj
 0001:00074710       ??$__push_heap@PAU?$SplineKey@M@spline@@HU12@U?$less@U?$SplineKey@M@spline@@@stlpmtx_std@@@stlpmtx_std@@YAXPAU?$SplineKey@M@spline@@HHU12@U?$less@U?$SplineKey@M@spline@@@0@@Z 31575710 f i FaceAnimSequence.obj
 0001:000747a0       ??$__copy_backward_ptrs@PAU?$SplineKey@M@spline@@PAU12@@priv@stlpmtx_std@@YAPAU?$SplineKey@M@spline@@PAU23@00ABU__false_type@1@@Z 315757a0 f i FaceAnimSequence.obj
 0001:00074800       ??$__push_heap@PAVCFaceIdentifierHandle@@HV1@USFaceIdentifierHandleLess@CFacialSentence@@@stlpmtx_std@@YAXPAVCFaceIdentifierHandle@@HHV1@USFaceIdentifierHandleLess@CFacialSentence@@@Z 31575800 f i FaceAnimSequence.obj
 0001:00074850       ??1?$_smart_ptr@VIReadStream@@@@QAE@XZ 31575850 f i FaceAnimSequence.obj
 0001:00074890       ?GetMemoryUsage@CFacialSentence@@QBEXPAVICrySizer@@@Z 31575890 f i FaceAnimSequence.obj
 0001:00074900       ?GetChannel@CFacialAnimSequence@@UAEPAUIFacialAnimChannel@@H@Z 31575900 f   FaceAnimSequence.obj
 0001:00074910       ?GetSoundEntryCount@CFacialAnimSequence@@UAEHXZ 31575910 f   FaceAnimSequence.obj
 0001:00074930       ?GetSoundEntry@CFacialAnimSequence@@UAEPAUIFacialAnimSoundEntry@@H@Z 31575930 f   FaceAnimSequence.obj
 0001:00074970       ?SerializeChannelSave@CFacialAnimSequence@@AAEXPAUIFacialAnimChannel@@AAVXmlNodeRef@@@Z 31575970 f   FaceAnimSequence.obj
 0001:00074ac0       ?GetSkeletonAnimationEntryCount@CFacialAnimSequence@@UAEHXZ 31575ac0 f   FaceAnimSequence.obj
 0001:00074ad0       ?GetSkeletonAnimationEntry@CFacialAnimSequence@@UAEPAUIFacialAnimSkeletonAnimationEntry@@H@Z 31575ad0 f   FaceAnimSequence.obj
 0001:00074b10       ?GenerateProceduralChannels@CFacialAnimSequence@@AAEXAAUData@1@@Z 31575b10 f   FaceAnimSequence.obj
 0001:00074ed0       ?UpdateSoundEntriesValidateID@CFacialAnimSequence@@AAEXXZ 31575ed0 f   FaceAnimSequence.obj
 0001:00074f20       ??4?$_smart_ptr@VIReadStream@@@@QAEAAV0@ABV0@@Z 31575f20 f i FaceAnimSequence.obj
 0001:00074f90       ?resize_raw@?$SmallDynStorage@U?$SplineKey@M@spline@@HUStandardAlloc@NAlloc@@@NArray@@QAEXHH_N@Z 31575f90 f i FaceAnimSequence.obj
 0001:000750f0       ?init@?$DynArray@U?$TCBSplineKey@U?$Vec3_tpl@M@@@spline@@HU?$SmallDynStorage@U?$TCBSplineKey@U?$Vec3_tpl@M@@@spline@@HUStandardAlloc@NAlloc@@@NArray@@@@KAPAU?$TCBSplineKey@U?$Vec3_tpl@M@@@spline@@U?$Array@U?$TCBSplineKey@U?$Vec3_tpl@M@@@spline@@HU?$ArrayStorage@U?$TCBSplineKey@U?$Vec3_tpl@M@@@spline@@H@NArray@@@@@Z 315760f0 f i FaceAnimSequence.obj
 0001:00075150       ?expand_raw@?$DynArray@U?$SplineKey@M@spline@@HU?$SmallDynStorage@U?$SplineKey@M@spline@@HUStandardAlloc@NAlloc@@@NArray@@@@IAEPAU?$SplineKey@M@spline@@PAU23@H@Z 31576150 f i FaceAnimSequence.obj
 0001:000751e0       ??$AddObject@V?$_smart_ptr@VCFacialAnimChannel@@@@V?$allocator@V?$_smart_ptr@VCFacialAnimChannel@@@@@stlpmtx_std@@@ICrySizer@@QAEXABV?$vector@V?$_smart_ptr@VCFacialAnimChannel@@@@V?$allocator@V?$_smart_ptr@VCFacialAnimChannel@@@@@stlpmtx_std@@@stlpmtx_std@@@Z 315761e0 f i FaceAnimSequence.obj
 0001:00075250       ??$AddObject@UBalanceChannelEntry@CFacialAnimSequenceInstance@@V?$allocator@UBalanceChannelEntry@CFacialAnimSequenceInstance@@@stlpmtx_std@@@ICrySizer@@QAEXABV?$vector@UBalanceChannelEntry@CFacialAnimSequenceInstance@@V?$allocator@UBalanceChannelEntry@CFacialAnimSequenceInstance@@@stlpmtx_std@@@stlpmtx_std@@@Z 31576250 f i FaceAnimSequence.obj
 0001:000752c0       ??$move_init@U?$SplineKey@U?$Quat_tpl@M@@@spline@@@NArray@@YAXPAU?$SplineKey@U?$Quat_tpl@M@@@spline@@0I@Z 315762c0 f i FaceAnimSequence.obj
 0001:00075550       ??$__equal_range@PAVEffectorChannelPair@@V1@U?$__less_2@VEffectorChannelPair@@V1@@priv@stlpmtx_std@@U234@H@priv@stlpmtx_std@@YA?AU?$pair@PAVEffectorChannelPair@@PAV1@@1@PAVEffectorChannelPair@@0ABV3@U?$__less_2@VEffectorChannelPair@@V1@@01@2PAH@Z 31576550 f i FaceAnimSequence.obj
 0001:00075610       ??$__ufill@PAUChannelInfo@CFacialAnimSequenceInstance@@U12@H@priv@stlpmtx_std@@YAXPAUChannelInfo@CFacialAnimSequenceInstance@@0ABU23@ABUrandom_access_iterator_tag@1@PAH@Z 31576610 f i FaceAnimSequence.obj
 0001:00075670       ??$__ucopy@PAUChannelInfo@CFacialAnimSequenceInstance@@PAU12@H@priv@stlpmtx_std@@YAPAUChannelInfo@CFacialAnimSequenceInstance@@PAU23@00ABUrandom_access_iterator_tag@1@PAH@Z 31576670 f i FaceAnimSequence.obj
 0001:000756d0       ??$__unguarded_partition@PAVCFaceIdentifierHandle@@V1@USFaceIdentifierHandleLess@CFacialSentence@@@priv@stlpmtx_std@@YAPAVCFaceIdentifierHandle@@PAV2@0V2@USFaceIdentifierHandleLess@CFacialSentence@@@Z 315766d0 f i FaceAnimSequence.obj
 0001:00075720       ??$__unguarded_insertion_sort_aux@PAVEffectorChannelPair@@V1@U?$less@VEffectorChannelPair@@@stlpmtx_std@@@priv@stlpmtx_std@@YAXPAVEffectorChannelPair@@00U?$less@VEffectorChannelPair@@@1@@Z 31576720 f i FaceAnimSequence.obj
 0001:00075770       ??$__unguarded_insertion_sort_aux@PAU?$SplineKey@M@spline@@U12@U?$less@U?$SplineKey@M@spline@@@stlpmtx_std@@@priv@stlpmtx_std@@YAXPAU?$SplineKey@M@spline@@00U?$less@U?$SplineKey@M@spline@@@1@@Z 31576770 f i FaceAnimSequence.obj
 0001:00075800       ??$__unguarded_insertion_sort_aux@PAU?$pair@PAUIFacialAnimChannel@@H@stlpmtx_std@@U12@VFirstLess@?$VectorMap@PAUIFacialAnimChannel@@HU?$less@PAUIFacialAnimChannel@@@stlpmtx_std@@V?$allocator@U?$pair@PAUIFacialAnimChannel@@H@stlpmtx_std@@@3@@@@priv@stlpmtx_std@@YAXPAU?$pair@PAUIFacialAnimChannel@@H@1@00VFirstLess@?$VectorMap@PAUIFacialAnimChannel@@HU?$less@PAUIFacialAnimChannel@@@stlpmtx_std@@V?$allocator@U?$pair@PAUIFacialAnimChannel@@H@stlpmtx_std@@@3@@@@Z 31576800 f i FaceAnimSequence.obj
 0001:00075850       ??$__adjust_heap@PAU?$pair@PAUIFacialAnimChannel@@H@stlpmtx_std@@HU12@VFirstLess@?$VectorMap@PAUIFacialAnimChannel@@HU?$less@PAUIFacialAnimChannel@@@stlpmtx_std@@V?$allocator@U?$pair@PAUIFacialAnimChannel@@H@stlpmtx_std@@@3@@@@stlpmtx_std@@YAXPAU?$pair@PAUIFacialAnimChannel@@H@0@HHU10@VFirstLess@?$VectorMap@PAUIFacialAnimChannel@@HU?$less@PAUIFacialAnimChannel@@@stlpmtx_std@@V?$allocator@U?$pair@PAUIFacialAnimChannel@@H@stlpmtx_std@@@3@@@@Z 31576850 f i FaceAnimSequence.obj
 0001:00075850       ??$__adjust_heap@PAVEffectorChannelPair@@HV1@U?$less@VEffectorChannelPair@@@stlpmtx_std@@@stlpmtx_std@@YAXPAVEffectorChannelPair@@HHV1@U?$less@VEffectorChannelPair@@@0@@Z 31576850 f i FaceAnimSequence.obj
 0001:000758f0       ??$__adjust_heap@PAU?$SplineKey@M@spline@@HU12@U?$less@U?$SplineKey@M@spline@@@stlpmtx_std@@@stlpmtx_std@@YAXPAU?$SplineKey@M@spline@@HHU12@U?$less@U?$SplineKey@M@spline@@@0@@Z 315768f0 f i FaceAnimSequence.obj
 0001:000759d0       ??$__adjust_heap@PAVCFaceIdentifierHandle@@HV1@USFaceIdentifierHandleLess@CFacialSentence@@@stlpmtx_std@@YAXPAVCFaceIdentifierHandle@@HHV1@USFaceIdentifierHandleLess@CFacialSentence@@@Z 315769d0 f i FaceAnimSequence.obj
 0001:00075a50       ??4?$pair@V?$CryStringT@D@@H@stlpmtx_std@@QAEAAU01@ABU01@@Z 31576a50 f i LoaderSKIN.obj
 0001:00075a50       ??4?$pair@V?$CryStringT@D@@PAUIFacialAnimChannel@@@stlpmtx_std@@QAEAAU01@ABU01@@Z 31576a50 f i FaceAnimation.obj
 0001:00075a50       ??4CFaceIdentifierStorage@@QAEAAV0@ABV0@@Z 31576a50 f i FaceAnimSequence.obj
 0001:00075ac0       ?CleanupKeys@CFacialAnimChannel@@UAEXM@Z 31576ac0 f   FaceAnimSequence.obj
 0001:00075af0       ?SmoothKeys@CFacialAnimChannel@@UAEXM@Z 31576af0 f   FaceAnimSequence.obj
 0001:00075b20       ?RemoveNoise@CFacialAnimChannel@@UAEXMM@Z 31576b20 f   FaceAnimSequence.obj
 0001:00075b50       ??1CFacialAnimSoundEntry@@UAE@XZ 31576b50 f i FaceAnimSequence.obj
 0001:00075bc0       ??0CFacialAnimSoundEntry@@QAE@XZ 31576bc0 f   FaceAnimSequence.obj
 0001:00075c10       ??_ECFacialAnimSoundEntry@@UAEPAXI@Z 31576c10 f i FaceAnimSequence.obj
 0001:00075c10       ??_GCFacialAnimSoundEntry@@UAEPAXI@Z 31576c10 f i FaceAnimSequence.obj
 0001:00075c40       ??_ECFacialAnimSkeletalAnimationEntry@@UAEPAXI@Z 31576c40 f i FaceAnimSequence.obj
 0001:00075c40       ??_GCFacialAnimSkeletalAnimationEntry@@UAEPAXI@Z 31576c40 f i FaceAnimSequence.obj
 0001:00075c90       ?swap@?$TSpline@U?$SplineKey@M@spline@@VHermitBasis@2@@spline@@QAEXAAV12@@Z 31576c90 f i FaceAnimSequence.obj
 0001:00075c90       ?swap@?$TSpline@U?$TCBSplineKey@U?$Vec3_tpl@M@@@spline@@VHermitBasis@2@@spline@@QAEXAAV12@@Z 31576c90 f i FaceAnimSequence.obj
 0001:00075c90       ?swap@?$TSpline@U?$SplineKey@U?$Quat_tpl@M@@@spline@@VHermitBasis@2@@spline@@QAEXAAV12@@Z 31576c90 f i FaceAnimSequence.obj
 0001:00075d10       ?resize_raw@?$SmallDynStorage@U?$TCBSplineKey@U?$Vec3_tpl@M@@@spline@@HUStandardAlloc@NAlloc@@@NArray@@QAEXHH_N@Z 31576d10 f i FaceAnimSequence.obj
 0001:00075e60       ?resize_raw@?$SmallDynStorage@U?$SplineKey@U?$Quat_tpl@M@@@spline@@HUStandardAlloc@NAlloc@@@NArray@@QAEXHH_N@Z 31576e60 f i FaceAnimSequence.obj
 0001:00075fd0       ?set_size@?$SmallDynStorage@U?$TCBSplineKey@U?$Vec3_tpl@M@@@spline@@HUStandardAlloc@NAlloc@@@NArray@@QAEXH@Z 31576fd0 f i FaceAnimSequence.obj
 0001:00076060       ?_M_bit_alloc@?$_Bvector_base@V?$allocator@_N@stlpmtx_std@@@priv@stlpmtx_std@@IAEPAII@Z 31577060 f i FaceAnimSequence.obj
 0001:000760b0       ?expand_raw@?$DynArray@U?$TCBSplineKey@U?$Vec3_tpl@M@@@spline@@HU?$SmallDynStorage@U?$TCBSplineKey@U?$Vec3_tpl@M@@@spline@@HUStandardAlloc@NAlloc@@@NArray@@@@IAEPAU?$TCBSplineKey@U?$Vec3_tpl@M@@@spline@@PAU23@H@Z 315770b0 f i FaceAnimSequence.obj
 0001:00076130       ?expand_raw@?$DynArray@U?$SplineKey@U?$Quat_tpl@M@@@spline@@HU?$SmallDynStorage@U?$SplineKey@U?$Quat_tpl@M@@@spline@@HUStandardAlloc@NAlloc@@@NArray@@@@IAEPAU?$SplineKey@U?$Quat_tpl@M@@@spline@@PAU23@H@Z 31577130 f i FaceAnimSequence.obj
 0001:000761d0       ??$AddObject@PAVCFacialAnimChannelInterpolator@@V?$allocator@PAVCFacialAnimChannelInterpolator@@@stlpmtx_std@@@ICrySizer@@QAEXABV?$vector@PAVCFacialAnimChannelInterpolator@@V?$allocator@PAVCFacialAnimChannelInterpolator@@@stlpmtx_std@@@stlpmtx_std@@@Z 315771d0 f i FaceAnimSequence.obj
 0001:00076250       ?_M_insert_overflow@?$_Impl_vector@VCFaceIdentifierHandle@@V?$allocator@VCFaceIdentifierHandle@@@stlpmtx_std@@@priv@stlpmtx_std@@AAEXPAVCFaceIdentifierHandle@@ABV4@ABU__true_type@3@I_N@Z 31577250 f i FaceAnimSequence.obj
 0001:00076250       ?_M_insert_overflow@?$_Impl_vector@VEffectorChannelPair@@V?$allocator@VEffectorChannelPair@@@stlpmtx_std@@@priv@stlpmtx_std@@AAEXPAVEffectorChannelPair@@ABV4@ABU__true_type@3@I_N@Z 31577250 f i FaceAnimSequence.obj
 0001:00076250       ?_M_insert_overflow@?$_Impl_vector@U?$pair@PAUIFacialAnimChannel@@H@stlpmtx_std@@V?$allocator@U?$pair@PAUIFacialAnimChannel@@H@stlpmtx_std@@@2@@priv@stlpmtx_std@@AAEXPAU?$pair@PAUIFacialAnimChannel@@H@3@ABU43@ABU__true_type@3@I_N@Z 31577250 f i FaceAnimSequence.obj
 0001:000763b0       ??$_M_allocate_and_copy@PAH@?$_Impl_vector@HV?$allocator@H@stlpmtx_std@@@priv@stlpmtx_std@@AAEPAHAAIPAH1@Z 315773b0 f i FaceAnimSequence.obj
 0001:000763b0       ??$_M_allocate_and_copy@PBQAX@?$_Impl_vector@PAXV?$allocator@PAX@stlpmtx_std@@@priv@stlpmtx_std@@AAEPAPAXAAIPBQAX1@Z 315773b0 f i LoaderSKIN.obj
 0001:000763b0       ??$_M_allocate_and_copy@PAPAX@?$_Impl_vector@PAXV?$allocator@PAX@stlpmtx_std@@@priv@stlpmtx_std@@AAEPAPAXAAIPAPAX1@Z 315773b0 f i CharacterManager.obj
 0001:00076420       ??$__uninitialized_fill_n@PAV?$_smart_ptr@VCFacialAnimChannel@@@@IV1@@priv@stlpmtx_std@@YAPAV?$_smart_ptr@VCFacialAnimChannel@@@@PAV2@IABV2@@Z 31577420 f i FaceAnimSequence.obj
 0001:00076420       ??$__uninitialized_fill_n@PAV?$_smart_ptr@VCFacialEffCtrl@@@@IV1@@priv@stlpmtx_std@@YAPAV?$_smart_ptr@VCFacialEffCtrl@@@@PAV2@IABV2@@Z 31577420 f i FaceEffector.obj
 0001:00076420       ??$__uninitialized_fill_n@PAV?$_smart_ptr@VCFacialEffector@@@@IV1@@priv@stlpmtx_std@@YAPAV?$_smart_ptr@VCFacialEffector@@@@PAV2@IABV2@@Z 31577420 f i FaceEffectorLibrary.obj
 0001:00076470       ??$__copy@PAV?$CryStringT@D@@PAV1@H@priv@stlpmtx_std@@YAPAV?$CryStringT@D@@PAV2@00ABUrandom_access_iterator_tag@1@PAH@Z 31577470 f i FaceAnimSequence.obj
 0001:00076540       ??$__unguarded_partition@PAU?$SplineKey@M@spline@@U12@U?$less@U?$SplineKey@M@spline@@@stlpmtx_std@@@priv@stlpmtx_std@@YAPAU?$SplineKey@M@spline@@PAU23@0U23@U?$less@U?$SplineKey@M@spline@@@1@@Z 31577540 f i FaceAnimSequence.obj
 0001:000765c0       ??$__copy_backward@PAVCFacialAnimSkeletalAnimationEntry@@PAV1@H@priv@stlpmtx_std@@YAPAVCFacialAnimSkeletalAnimationEntry@@PAV2@00ABUrandom_access_iterator_tag@1@PAH@Z 315775c0 f i FaceAnimSequence.obj
 0001:000766a0       ??$__fill@PAVCFacialAnimSkeletalAnimationEntry@@V1@H@priv@stlpmtx_std@@YAXPAVCFacialAnimSkeletalAnimationEntry@@0ABV2@ABUrandom_access_iterator_tag@1@PAH@Z 315776a0 f i FaceAnimSequence.obj
 0001:00076770       ??$__copy_backward@PAVCFacialAnimSoundEntry@@PAV1@H@priv@stlpmtx_std@@YAPAVCFacialAnimSoundEntry@@PAV2@00ABUrandom_access_iterator_tag@1@PAH@Z 31577770 f i FaceAnimSequence.obj
 0001:000768a0       ??$__fill@PAVCFacialAnimSoundEntry@@V1@H@priv@stlpmtx_std@@YAXPAVCFacialAnimSoundEntry@@0ABV2@ABUrandom_access_iterator_tag@1@PAH@Z 315778a0 f i FaceAnimSequence.obj
 0001:000769c0       ??$__copy_backward@PAV?$CryStringT@D@@PAV1@H@priv@stlpmtx_std@@YAPAV?$CryStringT@D@@PAV2@00ABUrandom_access_iterator_tag@1@PAH@Z 315779c0 f i FaceAnimSequence.obj
 0001:00076a90       ??$__fill@PAV?$CryStringT@D@@V1@H@priv@stlpmtx_std@@YAXPAV?$CryStringT@D@@0ABV2@ABUrandom_access_iterator_tag@1@PAH@Z 31577a90 f i FaceAnimSequence.obj
 0001:00076b50       ??$__unguarded_partition@PAU?$pair@PAUIFacialAnimChannel@@H@stlpmtx_std@@U12@VFirstLess@?$VectorMap@PAUIFacialAnimChannel@@HU?$less@PAUIFacialAnimChannel@@@stlpmtx_std@@V?$allocator@U?$pair@PAUIFacialAnimChannel@@H@stlpmtx_std@@@3@@@@priv@stlpmtx_std@@YAPAU?$pair@PAUIFacialAnimChannel@@H@1@PAU21@0U21@VFirstLess@?$VectorMap@PAUIFacialAnimChannel@@HU?$less@PAUIFacialAnimChannel@@@stlpmtx_std@@V?$allocator@U?$pair@PAUIFacialAnimChannel@@H@stlpmtx_std@@@3@@@@Z 31577b50 f i FaceAnimSequence.obj
 0001:00076b50       ??$__unguarded_partition@PAVEffectorChannelPair@@V1@U?$less@VEffectorChannelPair@@@stlpmtx_std@@@priv@stlpmtx_std@@YAPAVEffectorChannelPair@@PAV2@0V2@U?$less@VEffectorChannelPair@@@1@@Z 31577b50 f i FaceAnimSequence.obj
 0001:00076ba0       ??$__make_heap@PAVEffectorChannelPair@@U?$less@VEffectorChannelPair@@@stlpmtx_std@@V1@H@stlpmtx_std@@YAXPAVEffectorChannelPair@@0U?$less@VEffectorChannelPair@@@0@0PAH@Z 31577ba0 f i FaceAnimSequence.obj
 0001:00076c80       ??$__make_heap@PAU?$SplineKey@M@spline@@U?$less@U?$SplineKey@M@spline@@@stlpmtx_std@@U12@H@stlpmtx_std@@YAXPAU?$SplineKey@M@spline@@0U?$less@U?$SplineKey@M@spline@@@0@0PAH@Z 31577c80 f i FaceAnimSequence.obj
 0001:00076dc0       ??$__make_heap@PAVCFaceIdentifierHandle@@USFaceIdentifierHandleLess@CFacialSentence@@V1@H@stlpmtx_std@@YAXPAVCFaceIdentifierHandle@@0USFaceIdentifierHandleLess@CFacialSentence@@0PAH@Z 31577dc0 f i FaceAnimSequence.obj
 0001:00076eb0       ??$__make_heap@PAU?$pair@PAUIFacialAnimChannel@@H@stlpmtx_std@@VFirstLess@?$VectorMap@PAUIFacialAnimChannel@@HU?$less@PAUIFacialAnimChannel@@@stlpmtx_std@@V?$allocator@U?$pair@PAUIFacialAnimChannel@@H@stlpmtx_std@@@3@@@U12@H@stlpmtx_std@@YAXPAU?$pair@PAUIFacialAnimChannel@@H@0@0VFirstLess@?$VectorMap@PAUIFacialAnimChannel@@HU?$less@PAUIFacialAnimChannel@@@stlpmtx_std@@V?$allocator@U?$pair@PAUIFacialAnimChannel@@H@stlpmtx_std@@@3@@@0PAH@Z 31577eb0 f i FaceAnimSequence.obj
 0001:00076f80       ?GetMemoryUsage@CFacialAnimChannel@@QBEXPAVICrySizer@@@Z 31577f80 f i FaceAnimSequence.obj
 0001:00076fe0       ?swap@CProceduralChannelSet@@QAEXAAV1@@Z 31577fe0 f i FaceAnimSequence.obj
 0001:000770f0       ??1CFacialAnimChannel@@UAE@XZ 315780f0 f   FaceAnimSequence.obj
 0001:00077200       ?SetEffectorIdentifier@CFacialAnimChannel@@UAEXVCFaceIdentifierHandle@@@Z 31578200 f i FaceAnimSequence.obj
 0001:00077220       ?GetEffectorIdentifier@CFacialAnimChannel@@UAE?BVCFaceIdentifierHandle@@XZ 31578220 f i FaceAnimSequence.obj
 0001:00077240       ?SetFlags@CFacialAnimChannel@@UAEXI@Z 31578240 f i FaceAnimSequence.obj
 0001:00077250       ??_ECFacialAnimChannel@@W3AEPAXI@Z 31578250 f i FaceAnimSequence.obj
 0001:00077260       ?SetParent@CFacialAnimChannel@@UAEXPAUIFacialAnimChannel@@@Z 31578260 f i FaceAnimSequence.obj
 0001:000772a0       ?GetInterpolatorCount@CFacialAnimChannel@@UBEHXZ 315782a0 f i FaceAnimSequence.obj
 0001:000772b0       ?GetInterpolator@CFacialAnimChannel@@UAEPAUISplineInterpolator@@H@Z 315782b0 f i FaceAnimSequence.obj
 0001:000772c0       ?GetLastInterpolator@CFacialAnimChannel@@UAEPAUISplineInterpolator@@XZ 315782c0 f i FaceAnimSequence.obj
 0001:000772e0       ?GetName@CFacialAnimChannel@@UBEPBDXZ 315782e0 f i FaceAnimSequence.obj
 0001:00077320       ?SetIdentifier@CFacialAnimChannel@@UAEXVCFaceIdentifierHandle@@@Z 31578320 f   FaceAnimSequence.obj
 0001:00077390       ?GetIdentifier@CFacialAnimChannel@@UAE?BVCFaceIdentifierHandle@@XZ 31578390 f   FaceAnimSequence.obj
 0001:00077420       ?SetEffector@CFacialAnimChannel@@UAEXPAUIFacialEffector@@@Z 31578420 f   FaceAnimSequence.obj
 0001:000774c0       ?SetName@CFacialAnimChannel@@UAEXPBD@Z 315784c0 f   FaceAnimSequence.obj
 0001:00077540       ?SetJoystickFile@CFacialAnimSequence@@UAEXPBD@Z 31578540 f   FaceAnimSequence.obj
 0001:00077580       ?SetName@CFacialAnimSkeletalAnimationEntry@@UAEXPBD@Z 31578580 f   FaceAnimSequence.obj
 0001:000775c0       ?grow@?$DynArray@U?$SplineKey@M@spline@@HU?$SmallDynStorage@U?$SplineKey@M@spline@@HUStandardAlloc@NAlloc@@@NArray@@@@QAEPAU?$SplineKey@M@spline@@H@Z 315785c0 f i FaceAnimSequence.obj
 0001:00077610       ?_M_fill_insert@?$vector@_NV?$allocator@_N@stlpmtx_std@@@stlpmtx_std@@QAEXU?$_Bit_iter@U_Bit_reference@priv@stlpmtx_std@@PAU123@@priv@2@I_N@Z 31578610 f i FaceAnimSequence.obj
 0001:00077870       ?reserve@?$_Impl_vector@HV?$allocator@H@stlpmtx_std@@@priv@stlpmtx_std@@QAEXI@Z 31578870 f i FaceAnimSequence.obj
 0001:00077900       ??$AddObject@VCFacialAnimSkeletalAnimationEntry@@V?$allocator@VCFacialAnimSkeletalAnimationEntry@@@stlpmtx_std@@@ICrySizer@@QAEXABV?$vector@VCFacialAnimSkeletalAnimationEntry@@V?$allocator@VCFacialAnimSkeletalAnimationEntry@@@stlpmtx_std@@@stlpmtx_std@@@Z 31578900 f i FaceAnimSequence.obj
 0001:00077980       ??$AddObject@UChannelInfo@CFacialAnimSequenceInstance@@V?$allocator@UChannelInfo@CFacialAnimSequenceInstance@@@stlpmtx_std@@@ICrySizer@@QAEXABV?$vector@UChannelInfo@CFacialAnimSequenceInstance@@V?$allocator@UChannelInfo@CFacialAnimSequenceInstance@@@stlpmtx_std@@@stlpmtx_std@@@Z 31578980 f i FaceAnimSequence.obj
 0001:000779f0       ?_M_fill_insert_aux@?$_Impl_vector@UChannelInfo@CFacialAnimSequenceInstance@@V?$allocator@UChannelInfo@CFacialAnimSequenceInstance@@@stlpmtx_std@@@priv@stlpmtx_std@@AAEXPAUChannelInfo@CFacialAnimSequenceInstance@@IABU45@ABU__false_type@3@@Z 315789f0 f i FaceAnimSequence.obj
 0001:00077b30       ?_M_fill_insert_aux@?$_Impl_vector@U?$TCoeffBasis@M@spline@@V?$allocator@U?$TCoeffBasis@M@spline@@@stlpmtx_std@@@priv@stlpmtx_std@@AAEXPAU?$TCoeffBasis@M@spline@@IABU45@ABU__false_type@3@@Z 31578b30 f i FaceEffector.obj
 0001:00077b30       ?_M_fill_insert_aux@?$_Impl_vector@UBalanceChannelEntry@CFacialAnimSequenceInstance@@V?$allocator@UBalanceChannelEntry@CFacialAnimSequenceInstance@@@stlpmtx_std@@@priv@stlpmtx_std@@AAEXPAUBalanceChannelEntry@CFacialAnimSequenceInstance@@IABU45@ABU__false_type@3@@Z 31578b30 f i FaceAnimSequence.obj
 0001:00077c40       ??$__uninitialized_move@PAV?$_smart_ptr@VCFacialEffCtrl@@@@PAV1@U__false_type@stlpmtx_std@@@priv@stlpmtx_std@@YAPAV?$_smart_ptr@VCFacialEffCtrl@@@@PAV2@00U__false_type@1@ABU31@@Z 31578c40 f i FaceEffector.obj
 0001:00077c40       ??$__uninitialized_move@PAV?$_smart_ptr@VCFacialAnimChannel@@@@PAV1@U__false_type@stlpmtx_std@@@priv@stlpmtx_std@@YAPAV?$_smart_ptr@VCFacialAnimChannel@@@@PAV2@00U__false_type@1@ABU31@@Z 31578c40 f i FaceAnimSequence.obj
 0001:00077c40       ??$__uninitialized_move@PAV?$_smart_ptr@VCFacialEffector@@@@PAV1@U__false_type@stlpmtx_std@@@priv@stlpmtx_std@@YAPAV?$_smart_ptr@VCFacialEffector@@@@PAV2@00U__false_type@1@ABU31@@Z 31578c40 f i FaceEffectorLibrary.obj
 0001:00077c40       ??$__ucopy_ptrs@PAV?$_smart_ptr@VCFacialEffector@@@@PAV1@@priv@stlpmtx_std@@YAPAV?$_smart_ptr@VCFacialEffector@@@@PAV2@00ABU__false_type@1@@Z 31578c40 f i FaceEffectorLibrary.obj
 0001:00077c90       ??$__copy@PAVCFacialAnimSkeletalAnimationEntry@@PAV1@H@priv@stlpmtx_std@@YAPAVCFacialAnimSkeletalAnimationEntry@@PAV2@00ABUrandom_access_iterator_tag@1@PAH@Z 31578c90 f i FaceAnimSequence.obj
 0001:00077d70       ??$__copy@PAVCFacialAnimSoundEntry@@PAV1@H@priv@stlpmtx_std@@YAPAVCFacialAnimSoundEntry@@PAV2@00ABUrandom_access_iterator_tag@1@PAH@Z 31578d70 f i FaceAnimSequence.obj
 0001:00077ea0       ??$_Copy_Construct@VCFacialAnimSoundEntry@@@stlpmtx_std@@YAXPAVCFacialAnimSoundEntry@@ABV1@@Z 31578ea0 f i FaceAnimSequence.obj
 0001:00077f00       ??$__insertion_sort@PAVEffectorChannelPair@@V1@U?$less@VEffectorChannelPair@@@stlpmtx_std@@@priv@stlpmtx_std@@YAXPAVEffectorChannelPair@@00U?$less@VEffectorChannelPair@@@1@@Z 31578f00 f i FaceAnimSequence.obj
 0001:00077f90       ??$__destroy_range_aux@PAV?$CryStringT@D@@V1@@stlpmtx_std@@YAXPAV?$CryStringT@D@@00ABU__false_type@0@@Z 31578f90 f i FaceAnimSequence.obj
 0001:00077fe0       ??$__insertion_sort@PAVCFaceIdentifierHandle@@V1@USFaceIdentifierHandleLess@CFacialSentence@@@priv@stlpmtx_std@@YAXPAVCFaceIdentifierHandle@@00USFaceIdentifierHandleLess@CFacialSentence@@@Z 31578fe0 f i FaceAnimSequence.obj
 0001:00078090       ??$__insertion_sort@PAU?$pair@PAUIFacialAnimChannel@@H@stlpmtx_std@@U12@VFirstLess@?$VectorMap@PAUIFacialAnimChannel@@HU?$less@PAUIFacialAnimChannel@@@stlpmtx_std@@V?$allocator@U?$pair@PAUIFacialAnimChannel@@H@stlpmtx_std@@@3@@@@priv@stlpmtx_std@@YAXPAU?$pair@PAUIFacialAnimChannel@@H@1@00VFirstLess@?$VectorMap@PAUIFacialAnimChannel@@HU?$less@PAUIFacialAnimChannel@@@stlpmtx_std@@V?$allocator@U?$pair@PAUIFacialAnimChannel@@H@stlpmtx_std@@@3@@@@Z 31579090 f i FaceAnimSequence.obj
 0001:00078120       ?swap@@YAXAAUData@CFacialAnimSequence@@0@Z 31579120 f i FaceAnimSequence.obj
 0001:000782b0       ??_ECFacialAnimChannel@@UAEPAXI@Z 315792b0 f i FaceAnimSequence.obj
 0001:000782b0       ??_GCFacialAnimChannel@@UAEPAXI@Z 315792b0 f i FaceAnimSequence.obj
 0001:000782e0       ?DeleteInterpolator@CFacialAnimChannel@@UAEXH@Z 315792e0 f   FaceAnimSequence.obj
 0001:00078340       ?GetMemoryUsage@CFacialAnimSequenceInstance@@QBEXPAVICrySizer@@@Z 31579340 f   FaceAnimSequence.obj
 0001:000783c0       ?grow@?$DynArray@U?$SplineKey@U?$Quat_tpl@M@@@spline@@HU?$SmallDynStorage@U?$SplineKey@U?$Quat_tpl@M@@@spline@@HUStandardAlloc@NAlloc@@@NArray@@@@QAEPAU?$SplineKey@U?$Quat_tpl@M@@@spline@@H@Z 315793c0 f i FaceAnimSequence.obj
 0001:00078430       ?Tokenize@?$CryStringT@D@@QBE?AV1@PBDAAH@Z 31579430 f i FaceAnimSequence.obj
 0001:000784f0       ?_M_fill_insert_aux@?$_Impl_vector@V?$CryStringT@D@@V?$allocator@V?$CryStringT@D@@@stlpmtx_std@@@priv@stlpmtx_std@@AAEXPAV?$CryStringT@D@@IABV4@ABU__false_type@3@@Z 315794f0 f i FaceAnimSequence.obj
 0001:00078640       ??$__insertion_sort@PAU?$SplineKey@M@spline@@U12@U?$less@U?$SplineKey@M@spline@@@stlpmtx_std@@@priv@stlpmtx_std@@YAXPAU?$SplineKey@M@spline@@00U?$less@U?$SplineKey@M@spline@@@1@@Z 31579640 f i FaceAnimSequence.obj
 0001:00078700       ??$__ufill@PAVCFacialAnimSkeletalAnimationEntry@@V1@H@priv@stlpmtx_std@@YAXPAVCFacialAnimSkeletalAnimationEntry@@0ABV2@ABUrandom_access_iterator_tag@1@PAH@Z 31579700 f i FaceAnimSequence.obj
 0001:00078760       ??$__ucopy@PAVCFacialAnimSkeletalAnimationEntry@@PAV1@H@priv@stlpmtx_std@@YAPAVCFacialAnimSkeletalAnimationEntry@@PAV2@00ABUrandom_access_iterator_tag@1@PAH@Z 31579760 f i FaceAnimSequence.obj
 0001:000787c0       ??$__ufill@PAVCFacialAnimSoundEntry@@V1@H@priv@stlpmtx_std@@YAXPAVCFacialAnimSoundEntry@@0ABV2@ABUrandom_access_iterator_tag@1@PAH@Z 315797c0 f i FaceAnimSequence.obj
 0001:00078840       ??$__ucopy@PAVCFacialAnimSoundEntry@@PAV1@H@priv@stlpmtx_std@@YAPAVCFacialAnimSoundEntry@@PAV2@00ABUrandom_access_iterator_tag@1@PAH@Z 31579840 f i FaceAnimSequence.obj
 0001:000788c0       ??$sort_heap@PAVEffectorChannelPair@@U?$less@VEffectorChannelPair@@@stlpmtx_std@@@stlpmtx_std@@YAXPAVEffectorChannelPair@@0U?$less@VEffectorChannelPair@@@0@@Z 315798c0 f i FaceAnimSequence.obj
 0001:00078920       ??$sort_heap@PAU?$SplineKey@M@spline@@U?$less@U?$SplineKey@M@spline@@@stlpmtx_std@@@stlpmtx_std@@YAXPAU?$SplineKey@M@spline@@0U?$less@U?$SplineKey@M@spline@@@0@@Z 31579920 f i FaceAnimSequence.obj
 0001:000789f0       ??$sort_heap@PAVCFaceIdentifierHandle@@USFaceIdentifierHandleLess@CFacialSentence@@@stlpmtx_std@@YAXPAVCFaceIdentifierHandle@@0USFaceIdentifierHandleLess@CFacialSentence@@@Z 315799f0 f i FaceAnimSequence.obj
 0001:00078a50       ??$sort_heap@PAU?$pair@PAUIFacialAnimChannel@@H@stlpmtx_std@@VFirstLess@?$VectorMap@PAUIFacialAnimChannel@@HU?$less@PAUIFacialAnimChannel@@@stlpmtx_std@@V?$allocator@U?$pair@PAUIFacialAnimChannel@@H@stlpmtx_std@@@3@@@@stlpmtx_std@@YAXPAU?$pair@PAUIFacialAnimChannel@@H@0@0VFirstLess@?$VectorMap@PAUIFacialAnimChannel@@HU?$less@PAUIFacialAnimChannel@@@stlpmtx_std@@V?$allocator@U?$pair@PAUIFacialAnimChannel@@H@stlpmtx_std@@@3@@@@Z 31579a50 f i FaceAnimSequence.obj
 0001:00078ac0       ??0CFacialAnimChannel@@QAE@H@Z 31579ac0 f   FaceAnimSequence.obj
 0001:00078c40       ??$AddContainer@U?$DynArray@U?$SplineKey@M@spline@@HU?$SmallDynStorage@U?$SplineKey@M@spline@@HUStandardAlloc@NAlloc@@@NArray@@@@@ICrySizer@@QAE_NABU?$DynArray@U?$SplineKey@M@spline@@HU?$SmallDynStorage@U?$SplineKey@M@spline@@HUStandardAlloc@NAlloc@@@NArray@@@@@Z 31579c40 f i FaceAnimSequence.obj
 0001:00078cc0       ??$AddContainer@U?$DynArray@U?$SplineKey@U?$Quat_tpl@M@@@spline@@HU?$SmallDynStorage@U?$SplineKey@U?$Quat_tpl@M@@@spline@@HUStandardAlloc@NAlloc@@@NArray@@@@@ICrySizer@@QAE_NABU?$DynArray@U?$SplineKey@U?$Quat_tpl@M@@@spline@@HU?$SmallDynStorage@U?$SplineKey@U?$Quat_tpl@M@@@spline@@HUStandardAlloc@NAlloc@@@NArray@@@@@Z 31579cc0 f i FaceAnimSequence.obj
 0001:00078d60       ?GetMemoryUsage@?$TSpline@U?$SplineKey@U?$Quat_tpl@M@@@spline@@VHermitBasis@2@@spline@@UBEXPAVICrySizer@@_N@Z 31579d60 f i FaceAnimSequence.obj
 0001:00078da0       ??1?$_Impl_vector@VCFacialAnimSkeletalAnimationEntry@@V?$allocator@VCFacialAnimSkeletalAnimationEntry@@@stlpmtx_std@@@priv@stlpmtx_std@@QAE@XZ 31579da0 f i FaceAnimSequence.obj
 0001:00078df0       ??1?$_Impl_vector@VCFacialAnimSoundEntry@@V?$allocator@VCFacialAnimSoundEntry@@@stlpmtx_std@@@priv@stlpmtx_std@@QAE@XZ 31579df0 f i FaceAnimSequence.obj
 0001:00078e40       ?resize@?$vector@_NV?$allocator@_N@stlpmtx_std@@@stlpmtx_std@@QAEXI_N@Z 31579e40 f i FaceAnimSequence.obj
 0001:00078f30       ??_E?$TSpline@U?$SplineKey@U?$Quat_tpl@M@@@spline@@VHermitBasis@2@@spline@@UAEPAXI@Z 31579f30 f i FaceAnimSequence.obj
 0001:00078f30       ??_G?$HermitSplineEx@U?$Quat_tpl@M@@U?$SplineKey@U?$Quat_tpl@M@@@spline@@@spline@@UAEPAXI@Z 31579f30 f i FaceAnimSequence.obj
 0001:00078f30       ??_E?$HermitSplineEx@U?$Quat_tpl@M@@U?$SplineKey@U?$Quat_tpl@M@@@spline@@@spline@@UAEPAXI@Z 31579f30 f i FaceAnimSequence.obj
 0001:00078f30       ??_G?$TSpline@U?$SplineKey@U?$Quat_tpl@M@@@spline@@VHermitBasis@2@@spline@@UAEPAXI@Z 31579f30 f i FaceAnimSequence.obj
 0001:00078f80       ?_M_erase@?$_Impl_vector@UChannelInfo@CFacialAnimSequenceInstance@@V?$allocator@UChannelInfo@CFacialAnimSequenceInstance@@@stlpmtx_std@@@priv@stlpmtx_std@@AAEPAUChannelInfo@CFacialAnimSequenceInstance@@PAU45@0ABU__false_type@3@@Z 31579f80 f i FaceAnimSequence.obj
 0001:00079000       ?_M_erase@?$_Impl_vector@VCFacialAnimSkeletalAnimationEntry@@V?$allocator@VCFacialAnimSkeletalAnimationEntry@@@stlpmtx_std@@@priv@stlpmtx_std@@AAEPAVCFacialAnimSkeletalAnimationEntry@@PAV4@0ABU__false_type@3@@Z 3157a000 f i FaceAnimSequence.obj
 0001:00079070       ?_M_erase@?$_Impl_vector@VCFacialAnimSoundEntry@@V?$allocator@VCFacialAnimSoundEntry@@@stlpmtx_std@@@priv@stlpmtx_std@@AAEPAVCFacialAnimSoundEntry@@PAV4@0ABU__false_type@3@@Z 3157a070 f i FaceAnimSequence.obj
 0001:000790e0       ?_M_insert_overflow_aux@?$_Impl_vector@V?$_smart_ptr@VCFacialEffector@@@@V?$allocator@V?$_smart_ptr@VCFacialEffector@@@@@stlpmtx_std@@@priv@stlpmtx_std@@AAEXPAV?$_smart_ptr@VCFacialEffector@@@@ABV4@ABU__false_type@3@I_N@Z 3157a0e0 f i FaceEffectorLibrary.obj
 0001:000790e0       ?_M_insert_overflow_aux@?$_Impl_vector@V?$_smart_ptr@VCFacialAnimChannel@@@@V?$allocator@V?$_smart_ptr@VCFacialAnimChannel@@@@@stlpmtx_std@@@priv@stlpmtx_std@@AAEXPAV?$_smart_ptr@VCFacialAnimChannel@@@@ABV4@ABU__false_type@3@I_N@Z 3157a0e0 f i FaceAnimSequence.obj
 0001:000790e0       ?_M_insert_overflow_aux@?$_Impl_vector@V?$_smart_ptr@VCFacialEffCtrl@@@@V?$allocator@V?$_smart_ptr@VCFacialEffCtrl@@@@@stlpmtx_std@@@priv@stlpmtx_std@@AAEXPAV?$_smart_ptr@VCFacialEffCtrl@@@@ABV4@ABU__false_type@3@I_N@Z 3157a0e0 f i FaceEffector.obj
 0001:000792b0       ??$AddObject@VCFacialAnimSoundEntry@@V?$allocator@VCFacialAnimSoundEntry@@@stlpmtx_std@@@ICrySizer@@QAEXABV?$vector@VCFacialAnimSoundEntry@@V?$allocator@VCFacialAnimSoundEntry@@@stlpmtx_std@@@stlpmtx_std@@@Z 3157a2b0 f i FaceAnimSequence.obj
 0001:00079340       ?_M_insert_overflow_aux@?$_Impl_vector@UChannelInfo@CFacialAnimSequenceInstance@@V?$allocator@UChannelInfo@CFacialAnimSequenceInstance@@@stlpmtx_std@@@priv@stlpmtx_std@@AAEXPAUChannelInfo@CFacialAnimSequenceInstance@@ABU45@ABU__false_type@3@I_N@Z 3157a340 f i FaceAnimSequence.obj
 0001:00079500       ??$__final_insertion_sort@PAU?$SplineKey@M@spline@@U?$less@U?$SplineKey@M@spline@@@stlpmtx_std@@@priv@stlpmtx_std@@YAXPAU?$SplineKey@M@spline@@0U?$less@U?$SplineKey@M@spline@@@1@@Z 3157a500 f i FaceAnimSequence.obj
 0001:00079570       ??$__partial_sort@PAVEffectorChannelPair@@V1@U?$less@VEffectorChannelPair@@@stlpmtx_std@@@priv@stlpmtx_std@@YAXPAVEffectorChannelPair@@000U?$less@VEffectorChannelPair@@@1@@Z 3157a570 f i FaceAnimSequence.obj
 0001:000795e0       ??$__partial_sort@PAU?$SplineKey@M@spline@@U12@U?$less@U?$SplineKey@M@spline@@@stlpmtx_std@@@priv@stlpmtx_std@@YAXPAU?$SplineKey@M@spline@@000U?$less@U?$SplineKey@M@spline@@@1@@Z 3157a5e0 f i FaceAnimSequence.obj
 0001:000796b0       ??$__partial_sort@PAVCFaceIdentifierHandle@@V1@USFaceIdentifierHandleLess@CFacialSentence@@@priv@stlpmtx_std@@YAXPAVCFaceIdentifierHandle@@000USFaceIdentifierHandleLess@CFacialSentence@@@Z 3157a6b0 f i FaceAnimSequence.obj
 0001:00079720       ??$__partial_sort@PAU?$pair@PAUIFacialAnimChannel@@H@stlpmtx_std@@U12@VFirstLess@?$VectorMap@PAUIFacialAnimChannel@@HU?$less@PAUIFacialAnimChannel@@@stlpmtx_std@@V?$allocator@U?$pair@PAUIFacialAnimChannel@@H@stlpmtx_std@@@3@@@@priv@stlpmtx_std@@YAXPAU?$pair@PAUIFacialAnimChannel@@H@1@000VFirstLess@?$VectorMap@PAUIFacialAnimChannel@@HU?$less@PAUIFacialAnimChannel@@@stlpmtx_std@@V?$allocator@U?$pair@PAUIFacialAnimChannel@@H@stlpmtx_std@@@3@@@@Z 3157a720 f i FaceAnimSequence.obj
 0001:000797a0       ??$AddContainer@U?$DynArray@U?$TCBSplineKey@U?$Vec3_tpl@M@@@spline@@HU?$SmallDynStorage@U?$TCBSplineKey@U?$Vec3_tpl@M@@@spline@@HUStandardAlloc@NAlloc@@@NArray@@@@@ICrySizer@@QAE_NABU?$DynArray@U?$TCBSplineKey@U?$Vec3_tpl@M@@@spline@@HU?$SmallDynStorage@U?$TCBSplineKey@U?$Vec3_tpl@M@@@spline@@HUStandardAlloc@NAlloc@@@NArray@@@@@Z 3157a7a0 f i FaceAnimSequence.obj
 0001:00079830       ?GetMemoryUsage@?$TSpline@U?$TCBSplineKey@U?$Vec3_tpl@M@@@spline@@VHermitBasis@2@@spline@@UBEXPAVICrySizer@@_N@Z 3157a830 f i FaceAnimSequence.obj
 0001:00079870       ?SerializeSpline@CFacialAnimChannelInterpolator@@UAEXAAVXmlNodeRef@@_N@Z 3157a870 f   FaceAnimSequence.obj
 0001:00079b20       ?RemoveChannel@CFacialAnimSequence@@UAEXPAUIFacialAnimChannel@@@Z 3157ab20 f   FaceAnimSequence.obj
 0001:00079d50       ?GetMemoryUsage@CFacialAnimSequence@@UBEXPAVICrySizer@@@Z 3157ad50 f   FaceAnimSequence.obj
 0001:00079e10       ??0?$TSpline@U?$SplineKey@U?$Quat_tpl@M@@@spline@@VHermitBasis@2@@spline@@QAE@XZ 3157ae10 f i FaceAnimSequence.obj
 0001:00079e70       ?resize@?$_Impl_vector@UBalanceChannelEntry@CFacialAnimSequenceInstance@@V?$allocator@UBalanceChannelEntry@CFacialAnimSequenceInstance@@@stlpmtx_std@@@priv@stlpmtx_std@@QAEXIABUBalanceChannelEntry@CFacialAnimSequenceInstance@@@Z 3157ae70 f i FaceAnimSequence.obj
 0001:00079e70       ?resize@?$_Impl_vector@U?$TCoeffBasis@M@spline@@V?$allocator@U?$TCoeffBasis@M@spline@@@stlpmtx_std@@@priv@stlpmtx_std@@QAEXIABU?$TCoeffBasis@M@spline@@@Z 3157ae70 f i FaceEffector.obj
 0001:00079f10       ?_M_fill_insert_aux@?$_Impl_vector@VCFacialAnimSkeletalAnimationEntry@@V?$allocator@VCFacialAnimSkeletalAnimationEntry@@@stlpmtx_std@@@priv@stlpmtx_std@@AAEXPAVCFacialAnimSkeletalAnimationEntry@@IABV4@ABU__false_type@3@@Z 3157af10 f i FaceAnimSequence.obj
 0001:0007a080       ?_M_fill_insert_aux@?$_Impl_vector@VCFacialAnimSoundEntry@@V?$allocator@VCFacialAnimSoundEntry@@@stlpmtx_std@@@priv@stlpmtx_std@@AAEXPAVCFacialAnimSoundEntry@@IABV4@ABU__false_type@3@@Z 3157b080 f i FaceAnimSequence.obj
 0001:0007a1e0       ??0?$TSpline@U?$TCBSplineKey@U?$Vec3_tpl@M@@@spline@@VHermitBasis@2@@spline@@QAE@XZ 3157b1e0 f i FaceAnimSequence.obj
 0001:0007a240       ?comp_deriv@?$HermitSplineEx@U?$Quat_tpl@M@@U?$SplineKey@U?$Quat_tpl@M@@@spline@@@spline@@UAEXXZ 3157b240 f i FaceAnimSequence.obj
 0001:0007a5a0       ?interp_keys@?$HermitSplineEx@U?$Quat_tpl@M@@U?$SplineKey@U?$Quat_tpl@M@@@spline@@@spline@@MAEXHHMAAU?$Quat_tpl@M@@@Z 3157b5a0 f i FaceAnimSequence.obj
 0001:0007a780       ?comp_deriv@?$HermitSplineEx@MU?$SplineKey@M@spline@@@spline@@UAEXXZ 3157b780 f i FaceAnimSequence.obj
 0001:0007a8e0       ?interp_keys@?$HermitSplineEx@MU?$SplineKey@M@spline@@@spline@@MAEXHHMAAM@Z 3157b8e0 f i FaceAnimSequence.obj
 0001:0007a9c0       ??_G?$HermitSplineEx@MU?$SplineKey@M@spline@@@spline@@UAEPAXI@Z 3157b9c0 f i FaceAnimSequence.obj
 0001:0007a9c0       ??_E?$HermitSplineEx@MU?$SplineKey@M@spline@@@spline@@UAEPAXI@Z 3157b9c0 f i FaceAnimSequence.obj
 0001:0007aa10       ?SerializeSpline@CFacialCameraPathPositionInterpolator@@UAEXAAVXmlNodeRef@@_N@Z 3157ba10 f   FaceAnimSequence.obj
 0001:0007acf0       ?SerializeSpline@CFacialCameraPathOrientationInterpolator@@UAEXAAVXmlNodeRef@@_N@Z 3157bcf0 f   FaceAnimSequence.obj
 0001:0007afd0       ?erase@?$vector@VCFacialAnimSkeletalAnimationEntry@@V?$allocator@VCFacialAnimSkeletalAnimationEntry@@@stlpmtx_std@@@stlpmtx_std@@QAEPAVCFacialAnimSkeletalAnimationEntry@@PAV3@@Z 3157bfd0 f i FaceAnimSequence.obj
 0001:0007b030       ?erase@?$vector@VCFacialAnimSoundEntry@@V?$allocator@VCFacialAnimSoundEntry@@@stlpmtx_std@@@stlpmtx_std@@QAEPAVCFacialAnimSoundEntry@@PAV3@@Z 3157c030 f i FaceAnimSequence.obj
 0001:0007b090       ?push_back@?$_Impl_vector@V?$_smart_ptr@VCFacialEffCtrl@@@@V?$allocator@V?$_smart_ptr@VCFacialEffCtrl@@@@@stlpmtx_std@@@priv@stlpmtx_std@@QAEXABV?$_smart_ptr@VCFacialEffCtrl@@@@@Z 3157c090 f i FaceEffector.obj
 0001:0007b090       ?push_back@?$_Impl_vector@V?$_smart_ptr@VCFacialAnimChannel@@@@V?$allocator@V?$_smart_ptr@VCFacialAnimChannel@@@@@stlpmtx_std@@@priv@stlpmtx_std@@QAEXABV?$_smart_ptr@VCFacialAnimChannel@@@@@Z 3157c090 f i FaceAnimSequence.obj
 0001:0007b100       ??1?$vector@V?$CryStringT@D@@V?$allocator@V?$CryStringT@D@@@stlpmtx_std@@@stlpmtx_std@@QAE@XZ 3157c100 f i FaceAnimSequence.obj
 0001:0007b150       ?_M_insert_overflow_aux@?$_Impl_vector@VCFacialAnimSkeletalAnimationEntry@@V?$allocator@VCFacialAnimSkeletalAnimationEntry@@@stlpmtx_std@@@priv@stlpmtx_std@@AAEXPAVCFacialAnimSkeletalAnimationEntry@@ABV4@ABU__false_type@3@I_N@Z 3157c150 f i FaceAnimSequence.obj
 0001:0007b330       ?_M_insert_overflow_aux@?$_Impl_vector@VCFacialAnimSoundEntry@@V?$allocator@VCFacialAnimSoundEntry@@@stlpmtx_std@@@priv@stlpmtx_std@@AAEXPAVCFacialAnimSoundEntry@@ABV4@ABU__false_type@3@I_N@Z 3157c330 f i FaceAnimSequence.obj
 0001:0007b4f0       ??$__introsort_loop@PAVEffectorChannelPair@@V1@HU?$less@VEffectorChannelPair@@@stlpmtx_std@@@priv@stlpmtx_std@@YAXPAVEffectorChannelPair@@00HU?$less@VEffectorChannelPair@@@1@@Z 3157c4f0 f i FaceAnimSequence.obj
 0001:0007b5b0       ??$__introsort_loop@PAU?$SplineKey@M@spline@@U12@HU?$less@U?$SplineKey@M@spline@@@stlpmtx_std@@@priv@stlpmtx_std@@YAXPAU?$SplineKey@M@spline@@00HU?$less@U?$SplineKey@M@spline@@@1@@Z 3157c5b0 f i FaceAnimSequence.obj
 0001:0007b6c0       ??$__introsort_loop@PAVCFaceIdentifierHandle@@V1@HUSFaceIdentifierHandleLess@CFacialSentence@@@priv@stlpmtx_std@@YAXPAVCFaceIdentifierHandle@@00HUSFaceIdentifierHandleLess@CFacialSentence@@@Z 3157c6c0 f i FaceAnimSequence.obj
 0001:0007b790       ??$__introsort_loop@PAU?$pair@PAUIFacialAnimChannel@@H@stlpmtx_std@@U12@HVFirstLess@?$VectorMap@PAUIFacialAnimChannel@@HU?$less@PAUIFacialAnimChannel@@@stlpmtx_std@@V?$allocator@U?$pair@PAUIFacialAnimChannel@@H@stlpmtx_std@@@3@@@@priv@stlpmtx_std@@YAXPAU?$pair@PAUIFacialAnimChannel@@H@1@00HVFirstLess@?$VectorMap@PAUIFacialAnimChannel@@HU?$less@PAUIFacialAnimChannel@@@stlpmtx_std@@V?$allocator@U?$pair@PAUIFacialAnimChannel@@H@stlpmtx_std@@@3@@@@Z 3157c790 f i FaceAnimSequence.obj
 0001:0007b860       ?compMiddleDeriv@?$TCBSpline@U?$Vec3_tpl@M@@U?$TCBSplineKey@U?$Vec3_tpl@M@@@spline@@@spline@@AAEXH@Z 3157c860 f i FaceAnimSequence.obj
 0001:0007bb70       ?compLastDeriv@?$TCBSpline@U?$Vec3_tpl@M@@U?$TCBSplineKey@U?$Vec3_tpl@M@@@spline@@@spline@@AAEXXZ 3157cb70 f i FaceAnimSequence.obj
 0001:0007bc50       ?comp2KeyDeriv@?$TCBSpline@U?$Vec3_tpl@M@@U?$TCBSplineKey@U?$Vec3_tpl@M@@@spline@@@spline@@AAEXXZ 3157cc50 f i FaceAnimSequence.obj
 0001:0007bd40       ?comp_deriv@?$TCBSpline@U?$Vec3_tpl@M@@U?$TCBSplineKey@U?$Vec3_tpl@M@@@spline@@@spline@@UAEXXZ 3157cd40 f i FaceAnimSequence.obj
 0001:0007bea0       ?interp_keys@?$TCBSpline@U?$Vec3_tpl@M@@U?$TCBSplineKey@U?$Vec3_tpl@M@@@spline@@@spline@@MAEXHHMAAU?$Vec3_tpl@M@@@Z 3157cea0 f i FaceAnimSequence.obj
 0001:0007c010       ??_G?$TSpline@U?$TCBSplineKey@U?$Vec3_tpl@M@@@spline@@VHermitBasis@2@@spline@@UAEPAXI@Z 3157d010 f i FaceAnimSequence.obj
 0001:0007c010       ??_G?$TCBSpline@U?$Vec3_tpl@M@@U?$TCBSplineKey@U?$Vec3_tpl@M@@@spline@@@spline@@UAEPAXI@Z 3157d010 f i FaceAnimSequence.obj
 0001:0007c010       ??_E?$TSpline@U?$TCBSplineKey@U?$Vec3_tpl@M@@@spline@@VHermitBasis@2@@spline@@UAEPAXI@Z 3157d010 f i FaceAnimSequence.obj
 0001:0007c010       ??_E?$TCBSpline@U?$Vec3_tpl@M@@U?$TCBSplineKey@U?$Vec3_tpl@M@@@spline@@@spline@@UAEPAXI@Z 3157d010 f i FaceAnimSequence.obj
 0001:0007c060       ??$__unguarded_linear_insert@PAU?$TCBSplineKey@U?$Vec3_tpl@M@@@spline@@U12@U?$less@U?$TCBSplineKey@U?$Vec3_tpl@M@@@spline@@@stlpmtx_std@@@priv@stlpmtx_std@@YAXPAU?$TCBSplineKey@U?$Vec3_tpl@M@@@spline@@U23@U?$less@U?$TCBSplineKey@U?$Vec3_tpl@M@@@spline@@@1@@Z 3157d060 f i FaceAnimSequence.obj
 0001:0007c0f0       ??$__push_heap@PAU?$TCBSplineKey@U?$Vec3_tpl@M@@@spline@@HU12@U?$less@U?$TCBSplineKey@U?$Vec3_tpl@M@@@spline@@@stlpmtx_std@@@stlpmtx_std@@YAXPAU?$TCBSplineKey@U?$Vec3_tpl@M@@@spline@@HHU12@U?$less@U?$TCBSplineKey@U?$Vec3_tpl@M@@@spline@@@0@@Z 3157d0f0 f i FaceAnimSequence.obj
 0001:0007c1b0       ??$__copy_backward@PAU?$TCBSplineKey@U?$Vec3_tpl@M@@@spline@@PAU12@H@priv@stlpmtx_std@@YAPAU?$TCBSplineKey@U?$Vec3_tpl@M@@@spline@@PAU23@00ABUrandom_access_iterator_tag@1@PAH@Z 3157d1b0 f i FaceAnimSequence.obj
 0001:0007c340       ?GetKeyTime@?$CBaseSplineInterpolator@U?$Vec3_tpl@M@@V?$TCBSpline@U?$Vec3_tpl@M@@U?$TCBSplineKey@U?$Vec3_tpl@M@@@spline@@@spline@@@spline@@UAEMH@Z 3157d340 f i FaceAnimSequence.obj
 0001:0007c370       ?GetKeyValue@?$CBaseSplineInterpolator@U?$Vec3_tpl@M@@V?$TCBSpline@U?$Vec3_tpl@M@@U?$TCBSplineKey@U?$Vec3_tpl@M@@@spline@@@spline@@@spline@@UAE_NHAAY03M@Z 3157d370 f i FaceAnimSequence.obj
 0001:0007c3c0       ?SetKeyValue@?$CBaseSplineInterpolator@U?$Vec3_tpl@M@@V?$TCBSpline@U?$Vec3_tpl@M@@U?$TCBSplineKey@U?$Vec3_tpl@M@@@spline@@@spline@@@spline@@UAEXHQAM@Z 3157d3c0 f i FaceAnimSequence.obj
 0001:0007c410       ?SetKeyTime@?$CBaseSplineInterpolator@U?$Vec3_tpl@M@@V?$TCBSpline@U?$Vec3_tpl@M@@U?$TCBSplineKey@U?$Vec3_tpl@M@@@spline@@@spline@@@spline@@UAEXHM@Z 3157d410 f i FaceAnimSequence.obj
 0001:0007c450       ?SetKeyInTangent@?$CBaseSplineInterpolator@U?$Vec3_tpl@M@@V?$TCBSpline@U?$Vec3_tpl@M@@U?$TCBSplineKey@U?$Vec3_tpl@M@@@spline@@@spline@@@spline@@UAEXHQAM@Z 3157d450 f i FaceAnimSequence.obj
 0001:0007c4a0       ?SetKeyOutTangent@?$CBaseSplineInterpolator@U?$Vec3_tpl@M@@V?$TCBSpline@U?$Vec3_tpl@M@@U?$TCBSplineKey@U?$Vec3_tpl@M@@@spline@@@spline@@@spline@@UAEXHQAM@Z 3157d4a0 f i FaceAnimSequence.obj
 0001:0007c4f0       ?SetKeyTangents@?$CBaseSplineInterpolator@U?$Vec3_tpl@M@@V?$TCBSpline@U?$Vec3_tpl@M@@U?$TCBSplineKey@U?$Vec3_tpl@M@@@spline@@@spline@@@spline@@UAEXHQAM0@Z 3157d4f0 f i FaceAnimSequence.obj
 0001:0007c550       ?GetKeyTangents@?$CBaseSplineInterpolator@U?$Vec3_tpl@M@@V?$TCBSpline@U?$Vec3_tpl@M@@U?$TCBSplineKey@U?$Vec3_tpl@M@@@spline@@@spline@@@spline@@UAE_NHAAY03M0@Z 3157d550 f i FaceAnimSequence.obj
 0001:0007c5b0       ?SetKeyFlags@?$CBaseSplineInterpolator@U?$Vec3_tpl@M@@V?$TCBSpline@U?$Vec3_tpl@M@@U?$TCBSplineKey@U?$Vec3_tpl@M@@@spline@@@spline@@@spline@@UAEXHH@Z 3157d5b0 f i FaceAnimSequence.obj
 0001:0007c5f0       ?GetKeyFlags@?$CBaseSplineInterpolator@U?$Vec3_tpl@M@@V?$TCBSpline@U?$Vec3_tpl@M@@U?$TCBSplineKey@U?$Vec3_tpl@M@@@spline@@@spline@@@spline@@UAEHH@Z 3157d5f0 f i FaceAnimSequence.obj
 0001:0007c620       ?seek_key@?$TSpline@U?$TCBSplineKey@U?$Vec3_tpl@M@@@spline@@VHermitBasis@2@@spline@@IAEHM@Z 3157d620 f i FaceAnimSequence.obj
 0001:0007c6a0       ?init@?$DynArray@U?$TCBSplineKey@U?$Vec3_tpl@M@@@spline@@HU?$SmallDynStorage@U?$TCBSplineKey@U?$Vec3_tpl@M@@@spline@@HUStandardAlloc@NAlloc@@@NArray@@@@KAPAU?$TCBSplineKey@U?$Vec3_tpl@M@@@spline@@U?$Array@U?$TCBSplineKey@U?$Vec3_tpl@M@@@spline@@HU?$ArrayStorage@U?$TCBSplineKey@U?$Vec3_tpl@M@@@spline@@H@NArray@@@@PBU23@@Z 3157d6a0 f i FaceAnimSequence.obj
 0001:0007c6e0       ?assign@?$Array@U?$TCBSplineKey@U?$Vec3_tpl@M@@@spline@@HU?$SmallDynStorage@U?$TCBSplineKey@U?$Vec3_tpl@M@@@spline@@HUStandardAlloc@NAlloc@@@NArray@@@@QAEXU?$Array@$$CBU?$TCBSplineKey@U?$Vec3_tpl@M@@@spline@@HU?$ArrayStorage@$$CBU?$TCBSplineKey@U?$Vec3_tpl@M@@@spline@@H@NArray@@@@@Z 3157d6e0 f i FaceAnimSequence.obj
 0001:0007c750       ??$__unguarded_insertion_sort_aux@PAU?$TCBSplineKey@U?$Vec3_tpl@M@@@spline@@U12@U?$less@U?$TCBSplineKey@U?$Vec3_tpl@M@@@spline@@@stlpmtx_std@@@priv@stlpmtx_std@@YAXPAU?$TCBSplineKey@U?$Vec3_tpl@M@@@spline@@00U?$less@U?$TCBSplineKey@U?$Vec3_tpl@M@@@spline@@@1@@Z 3157d750 f i FaceAnimSequence.obj
 0001:0007c810       ??$__adjust_heap@PAU?$TCBSplineKey@U?$Vec3_tpl@M@@@spline@@HU12@U?$less@U?$TCBSplineKey@U?$Vec3_tpl@M@@@spline@@@stlpmtx_std@@@stlpmtx_std@@YAXPAU?$TCBSplineKey@U?$Vec3_tpl@M@@@spline@@HHU12@U?$less@U?$TCBSplineKey@U?$Vec3_tpl@M@@@spline@@@0@@Z 3157d810 f i FaceAnimSequence.obj
 0001:0007c8f0       ?FindKeysInRange@?$CBaseSplineInterpolator@U?$Vec3_tpl@M@@V?$TCBSpline@U?$Vec3_tpl@M@@U?$TCBSplineKey@U?$Vec3_tpl@M@@@spline@@@spline@@@spline@@UAEXMMAAH0@Z 3157d8f0 f i FaceAnimSequence.obj
 0001:0007ca20       ??$__make_heap@PAU?$TCBSplineKey@U?$Vec3_tpl@M@@@spline@@U?$less@U?$TCBSplineKey@U?$Vec3_tpl@M@@@spline@@@stlpmtx_std@@U12@H@stlpmtx_std@@YAXPAU?$TCBSplineKey@U?$Vec3_tpl@M@@@spline@@0U?$less@U?$TCBSplineKey@U?$Vec3_tpl@M@@@spline@@@0@0PAH@Z 3157da20 f i FaceAnimSequence.obj
 0001:0007cb60       ?erase@?$DynArray@U?$TCBSplineKey@U?$Vec3_tpl@M@@@spline@@HU?$SmallDynStorage@U?$TCBSplineKey@U?$Vec3_tpl@M@@@spline@@HUStandardAlloc@NAlloc@@@NArray@@@@QAEPAU?$TCBSplineKey@U?$Vec3_tpl@M@@@spline@@PAU23@0@Z 3157db60 f i FaceAnimSequence.obj
 0001:0007cd10       ?insert_raw@?$DynArray@U?$TCBSplineKey@U?$Vec3_tpl@M@@@spline@@HU?$SmallDynStorage@U?$TCBSplineKey@U?$Vec3_tpl@M@@@spline@@HUStandardAlloc@NAlloc@@@NArray@@@@QAE?AU?$Array@U?$TCBSplineKey@U?$Vec3_tpl@M@@@spline@@HU?$ArrayStorage@U?$TCBSplineKey@U?$Vec3_tpl@M@@@spline@@H@NArray@@@@PAU?$TCBSplineKey@U?$Vec3_tpl@M@@@spline@@H@Z 3157dd10 f i FaceAnimSequence.obj
 0001:0007cde0       ??$__unguarded_partition@PAU?$TCBSplineKey@U?$Vec3_tpl@M@@@spline@@U12@U?$less@U?$TCBSplineKey@U?$Vec3_tpl@M@@@spline@@@stlpmtx_std@@@priv@stlpmtx_std@@YAPAU?$TCBSplineKey@U?$Vec3_tpl@M@@@spline@@PAU23@0U23@U?$less@U?$TCBSplineKey@U?$Vec3_tpl@M@@@spline@@@1@@Z 3157dde0 f i FaceAnimSequence.obj
 0001:0007ce90       ??4?$DynArray@U?$TCBSplineKey@U?$Vec3_tpl@M@@@spline@@HU?$SmallDynStorage@U?$TCBSplineKey@U?$Vec3_tpl@M@@@spline@@HUStandardAlloc@NAlloc@@@NArray@@@@QAEAAU0@U?$Array@$$CBU?$TCBSplineKey@U?$Vec3_tpl@M@@@spline@@HU?$ArrayStorage@$$CBU?$TCBSplineKey@U?$Vec3_tpl@M@@@spline@@H@NArray@@@@@Z 3157de90 f i FaceAnimSequence.obj
 0001:0007cf40       ??$sort_heap@PAU?$TCBSplineKey@U?$Vec3_tpl@M@@@spline@@U?$less@U?$TCBSplineKey@U?$Vec3_tpl@M@@@spline@@@stlpmtx_std@@@stlpmtx_std@@YAXPAU?$TCBSplineKey@U?$Vec3_tpl@M@@@spline@@0U?$less@U?$TCBSplineKey@U?$Vec3_tpl@M@@@spline@@@0@@Z 3157df40 f i FaceAnimSequence.obj
 0001:0007cff0       ?RemoveKey@?$CBaseSplineInterpolator@U?$Vec3_tpl@M@@V?$TCBSpline@U?$Vec3_tpl@M@@U?$TCBSplineKey@U?$Vec3_tpl@M@@@spline@@@spline@@@spline@@UAEXH@Z 3157dff0 f i FaceAnimSequence.obj
 0001:0007d030       ?RemoveKeysInRange@?$CBaseSplineInterpolator@U?$Vec3_tpl@M@@V?$TCBSpline@U?$Vec3_tpl@M@@U?$TCBSplineKey@U?$Vec3_tpl@M@@@spline@@@spline@@@spline@@UAEXMM@Z 3157e030 f i FaceAnimSequence.obj
 0001:0007d160       ??0?$DynArray@U?$TCBSplineKey@U?$Vec3_tpl@M@@@spline@@HU?$SmallDynStorage@U?$TCBSplineKey@U?$Vec3_tpl@M@@@spline@@HUStandardAlloc@NAlloc@@@NArray@@@@QAE@ABU0@@Z 3157e160 f i FaceAnimSequence.obj
 0001:0007d200       ??$__insertion_sort@PAU?$TCBSplineKey@U?$Vec3_tpl@M@@@spline@@U12@U?$less@U?$TCBSplineKey@U?$Vec3_tpl@M@@@spline@@@stlpmtx_std@@@priv@stlpmtx_std@@YAXPAU?$TCBSplineKey@U?$Vec3_tpl@M@@@spline@@00U?$less@U?$TCBSplineKey@U?$Vec3_tpl@M@@@spline@@@1@@Z 3157e200 f i FaceAnimSequence.obj
 0001:0007d2e0       ??$__partial_sort@PAU?$TCBSplineKey@U?$Vec3_tpl@M@@@spline@@U12@U?$less@U?$TCBSplineKey@U?$Vec3_tpl@M@@@spline@@@stlpmtx_std@@@priv@stlpmtx_std@@YAXPAU?$TCBSplineKey@U?$Vec3_tpl@M@@@spline@@000U?$less@U?$TCBSplineKey@U?$Vec3_tpl@M@@@spline@@@1@@Z 3157e2e0 f i FaceAnimSequence.obj
 0001:0007d3b0       ?InsertKey@?$CBaseSplineInterpolator@U?$Vec3_tpl@M@@V?$TCBSpline@U?$Vec3_tpl@M@@U?$TCBSplineKey@U?$Vec3_tpl@M@@@spline@@@spline@@@spline@@UAEHMQAM@Z 3157e3b0 f i FaceAnimSequence.obj
 0001:0007d580       ??$__introsort_loop@PAU?$TCBSplineKey@U?$Vec3_tpl@M@@@spline@@U12@HU?$less@U?$TCBSplineKey@U?$Vec3_tpl@M@@@spline@@@stlpmtx_std@@@priv@stlpmtx_std@@YAXPAU?$TCBSplineKey@U?$Vec3_tpl@M@@@spline@@00HU?$less@U?$TCBSplineKey@U?$Vec3_tpl@M@@@spline@@@1@@Z 3157e580 f i FaceAnimSequence.obj
 0001:0007d660       ??$__push_heap@PAU?$SplineKey@U?$Quat_tpl@M@@@spline@@HU12@U?$less@U?$SplineKey@U?$Quat_tpl@M@@@spline@@@stlpmtx_std@@@stlpmtx_std@@YAXPAU?$SplineKey@U?$Quat_tpl@M@@@spline@@HHU12@U?$less@U?$SplineKey@U?$Quat_tpl@M@@@spline@@@0@@Z 3157e660 f i FaceAnimSequence.obj
 0001:0007d6d0       ?seek_key@?$TSpline@U?$SplineKey@U?$Quat_tpl@M@@@spline@@VHermitBasis@2@@spline@@IAEHM@Z 3157e6d0 f i FaceAnimSequence.obj
 0001:0007d760       ?adjust_time@?$TSpline@U?$SplineKey@U?$Quat_tpl@M@@@spline@@VHermitBasis@2@@spline@@IAEXAAM@Z 3157e760 f i FaceAnimSequence.obj
 0001:0007d7c0       ?init@?$DynArray@U?$SplineKey@U?$Quat_tpl@M@@@spline@@HU?$SmallDynStorage@U?$SplineKey@U?$Quat_tpl@M@@@spline@@HUStandardAlloc@NAlloc@@@NArray@@@@KAPAU?$SplineKey@U?$Quat_tpl@M@@@spline@@U?$Array@U?$SplineKey@U?$Quat_tpl@M@@@spline@@HU?$ArrayStorage@U?$SplineKey@U?$Quat_tpl@M@@@spline@@H@NArray@@@@PBU23@@Z 3157e7c0 f i FaceAnimSequence.obj
 0001:0007d850       ?init@?$DynArray@U?$SplineKey@U?$Quat_tpl@M@@@spline@@HU?$SmallDynStorage@U?$SplineKey@U?$Quat_tpl@M@@@spline@@HUStandardAlloc@NAlloc@@@NArray@@@@KAPAU?$SplineKey@U?$Quat_tpl@M@@@spline@@U?$Array@U?$SplineKey@U?$Quat_tpl@M@@@spline@@HU?$ArrayStorage@U?$SplineKey@U?$Quat_tpl@M@@@spline@@H@NArray@@@@ABU23@@Z 3157e850 f i FaceAnimSequence.obj
 0001:0007d8e0       ??$__unguarded_insertion_sort_aux@PAU?$SplineKey@U?$Quat_tpl@M@@@spline@@U12@U?$less@U?$SplineKey@U?$Quat_tpl@M@@@spline@@@stlpmtx_std@@@priv@stlpmtx_std@@YAXPAU?$SplineKey@U?$Quat_tpl@M@@@spline@@00U?$less@U?$SplineKey@U?$Quat_tpl@M@@@spline@@@1@@Z 3157e8e0 f i FaceAnimSequence.obj
 0001:0007d9d0       ??$__adjust_heap@PAU?$SplineKey@U?$Quat_tpl@M@@@spline@@HU12@U?$less@U?$SplineKey@U?$Quat_tpl@M@@@spline@@@stlpmtx_std@@@stlpmtx_std@@YAXPAU?$SplineKey@U?$Quat_tpl@M@@@spline@@HHU12@U?$less@U?$SplineKey@U?$Quat_tpl@M@@@spline@@@0@@Z 3157e9d0 f i FaceAnimSequence.obj
 0001:0007db00       ?FindKeysInRange@?$CBaseSplineInterpolator@U?$Quat_tpl@M@@V?$HermitSplineEx@U?$Quat_tpl@M@@U?$SplineKey@U?$Quat_tpl@M@@@spline@@@spline@@@spline@@UAEXMMAAH0@Z 3157eb00 f i FaceAnimSequence.obj
 0001:0007dc40       ?GetKeyTime@?$CBaseSplineInterpolator@U?$Quat_tpl@M@@V?$HermitSplineEx@U?$Quat_tpl@M@@U?$SplineKey@U?$Quat_tpl@M@@@spline@@@spline@@@spline@@UAEMH@Z 3157ec40 f i FaceAnimSequence.obj
 0001:0007dc70       ?GetKeyValue@?$CBaseSplineInterpolator@U?$Quat_tpl@M@@V?$HermitSplineEx@U?$Quat_tpl@M@@U?$SplineKey@U?$Quat_tpl@M@@@spline@@@spline@@@spline@@UAE_NHAAY03M@Z 3157ec70 f i FaceAnimSequence.obj
 0001:0007dcc0       ?SetKeyValue@?$CBaseSplineInterpolator@U?$Quat_tpl@M@@V?$HermitSplineEx@U?$Quat_tpl@M@@U?$SplineKey@U?$Quat_tpl@M@@@spline@@@spline@@@spline@@UAEXHQAM@Z 3157ecc0 f i FaceAnimSequence.obj
 0001:0007dd10       ?SetKeyTime@?$CBaseSplineInterpolator@U?$Quat_tpl@M@@V?$HermitSplineEx@U?$Quat_tpl@M@@U?$SplineKey@U?$Quat_tpl@M@@@spline@@@spline@@@spline@@UAEXHM@Z 3157ed10 f i FaceAnimSequence.obj
 0001:0007dd50       ?SetKeyInTangent@?$CBaseSplineInterpolator@U?$Quat_tpl@M@@V?$HermitSplineEx@U?$Quat_tpl@M@@U?$SplineKey@U?$Quat_tpl@M@@@spline@@@spline@@@spline@@UAEXHQAM@Z 3157ed50 f i FaceAnimSequence.obj
 0001:0007dda0       ?SetKeyOutTangent@?$CBaseSplineInterpolator@U?$Quat_tpl@M@@V?$HermitSplineEx@U?$Quat_tpl@M@@U?$SplineKey@U?$Quat_tpl@M@@@spline@@@spline@@@spline@@UAEXHQAM@Z 3157eda0 f i FaceAnimSequence.obj
 0001:0007ddf0       ?SetKeyTangents@?$CBaseSplineInterpolator@U?$Quat_tpl@M@@V?$HermitSplineEx@U?$Quat_tpl@M@@U?$SplineKey@U?$Quat_tpl@M@@@spline@@@spline@@@spline@@UAEXHQAM0@Z 3157edf0 f i FaceAnimSequence.obj
 0001:0007de60       ?GetKeyTangents@?$CBaseSplineInterpolator@U?$Quat_tpl@M@@V?$HermitSplineEx@U?$Quat_tpl@M@@U?$SplineKey@U?$Quat_tpl@M@@@spline@@@spline@@@spline@@UAE_NHAAY03M0@Z 3157ee60 f i FaceAnimSequence.obj
 0001:0007ded0       ?SetKeyFlags@?$CBaseSplineInterpolator@U?$Quat_tpl@M@@V?$HermitSplineEx@U?$Quat_tpl@M@@U?$SplineKey@U?$Quat_tpl@M@@@spline@@@spline@@@spline@@UAEXHH@Z 3157eed0 f i FaceAnimSequence.obj
 0001:0007df10       ?GetKeyFlags@?$CBaseSplineInterpolator@U?$Quat_tpl@M@@V?$HermitSplineEx@U?$Quat_tpl@M@@U?$SplineKey@U?$Quat_tpl@M@@@spline@@@spline@@@spline@@UAEHH@Z 3157ef10 f i FaceAnimSequence.obj
 0001:0007df50       ?erase@?$DynArray@U?$SplineKey@U?$Quat_tpl@M@@@spline@@HU?$SmallDynStorage@U?$SplineKey@U?$Quat_tpl@M@@@spline@@HUStandardAlloc@NAlloc@@@NArray@@@@QAEPAU?$SplineKey@U?$Quat_tpl@M@@@spline@@PAU23@0@Z 3157ef50 f i FaceAnimSequence.obj
 0001:0007dfd0       ??$copy_backward@PAU?$SplineKey@U?$Quat_tpl@M@@@spline@@PAU12@@stlpmtx_std@@YAPAU?$SplineKey@U?$Quat_tpl@M@@@spline@@PAU12@00@Z 3157efd0 f i FaceAnimSequence.obj
 0001:0007e020       ??$__make_heap@PAU?$SplineKey@U?$Quat_tpl@M@@@spline@@U?$less@U?$SplineKey@U?$Quat_tpl@M@@@spline@@@stlpmtx_std@@U12@H@stlpmtx_std@@YAXPAU?$SplineKey@U?$Quat_tpl@M@@@spline@@0U?$less@U?$SplineKey@U?$Quat_tpl@M@@@spline@@@0@0PAH@Z 3157f020 f i FaceAnimSequence.obj
 0001:0007e0e0       ??4?$DynArray@U?$SplineKey@U?$Quat_tpl@M@@@spline@@HU?$SmallDynStorage@U?$SplineKey@U?$Quat_tpl@M@@@spline@@HUStandardAlloc@NAlloc@@@NArray@@@@QAEAAU0@U?$Array@$$CBU?$SplineKey@U?$Quat_tpl@M@@@spline@@HU?$ArrayStorage@$$CBU?$SplineKey@U?$Quat_tpl@M@@@spline@@H@NArray@@@@@Z 3157f0e0 f i FaceAnimSequence.obj
 0001:0007e1c0       ?insert_raw@?$DynArray@U?$SplineKey@U?$Quat_tpl@M@@@spline@@HU?$SmallDynStorage@U?$SplineKey@U?$Quat_tpl@M@@@spline@@HUStandardAlloc@NAlloc@@@NArray@@@@QAE?AU?$Array@U?$SplineKey@U?$Quat_tpl@M@@@spline@@HU?$ArrayStorage@U?$SplineKey@U?$Quat_tpl@M@@@spline@@H@NArray@@@@PAU?$SplineKey@U?$Quat_tpl@M@@@spline@@H@Z 3157f1c0 f i FaceAnimSequence.obj
 0001:0007e2d0       ??$__unguarded_partition@PAU?$SplineKey@U?$Quat_tpl@M@@@spline@@U12@U?$less@U?$SplineKey@U?$Quat_tpl@M@@@spline@@@stlpmtx_std@@@priv@stlpmtx_std@@YAPAU?$SplineKey@U?$Quat_tpl@M@@@spline@@PAU23@0U23@U?$less@U?$SplineKey@U?$Quat_tpl@M@@@spline@@@1@@Z 3157f2d0 f i FaceAnimSequence.obj
 0001:0007e3b0       ??$__linear_insert@PAU?$SplineKey@U?$Quat_tpl@M@@@spline@@U12@U?$less@U?$SplineKey@U?$Quat_tpl@M@@@spline@@@stlpmtx_std@@@priv@stlpmtx_std@@YAXPAU?$SplineKey@U?$Quat_tpl@M@@@spline@@0U23@U?$less@U?$SplineKey@U?$Quat_tpl@M@@@spline@@@1@@Z 3157f3b0 f i FaceAnimSequence.obj
 0001:0007e4a0       ?RemoveKey@?$CBaseSplineInterpolator@U?$Quat_tpl@M@@V?$HermitSplineEx@U?$Quat_tpl@M@@U?$SplineKey@U?$Quat_tpl@M@@@spline@@@spline@@@spline@@UAEXH@Z 3157f4a0 f i FaceAnimSequence.obj
 0001:0007e4f0       ?RemoveKeysInRange@?$CBaseSplineInterpolator@U?$Quat_tpl@M@@V?$HermitSplineEx@U?$Quat_tpl@M@@U?$SplineKey@U?$Quat_tpl@M@@@spline@@@spline@@@spline@@UAEXMM@Z 3157f4f0 f i FaceAnimSequence.obj
 0001:0007e640       ??0?$DynArray@U?$SplineKey@U?$Quat_tpl@M@@@spline@@HU?$SmallDynStorage@U?$SplineKey@U?$Quat_tpl@M@@@spline@@HUStandardAlloc@NAlloc@@@NArray@@@@QAE@ABU0@@Z 3157f640 f i FaceAnimSequence.obj
 0001:0007e6d0       ??$__insertion_sort@PAU?$SplineKey@U?$Quat_tpl@M@@@spline@@U12@U?$less@U?$SplineKey@U?$Quat_tpl@M@@@spline@@@stlpmtx_std@@@priv@stlpmtx_std@@YAXPAU?$SplineKey@U?$Quat_tpl@M@@@spline@@00U?$less@U?$SplineKey@U?$Quat_tpl@M@@@spline@@@1@@Z 3157f6d0 f i FaceAnimSequence.obj
 0001:0007e770       ??$sort_heap@PAU?$SplineKey@U?$Quat_tpl@M@@@spline@@U?$less@U?$SplineKey@U?$Quat_tpl@M@@@spline@@@stlpmtx_std@@@stlpmtx_std@@YAXPAU?$SplineKey@U?$Quat_tpl@M@@@spline@@0U?$less@U?$SplineKey@U?$Quat_tpl@M@@@spline@@@0@@Z 3157f770 f i FaceAnimSequence.obj
 0001:0007e8d0       ??$__final_insertion_sort@PAU?$SplineKey@U?$Quat_tpl@M@@@spline@@U?$less@U?$SplineKey@U?$Quat_tpl@M@@@spline@@@stlpmtx_std@@@priv@stlpmtx_std@@YAXPAU?$SplineKey@U?$Quat_tpl@M@@@spline@@0U?$less@U?$SplineKey@U?$Quat_tpl@M@@@spline@@@1@@Z 3157f8d0 f i FaceAnimSequence.obj
 0001:0007e940       ??$__partial_sort@PAU?$SplineKey@U?$Quat_tpl@M@@@spline@@U12@U?$less@U?$SplineKey@U?$Quat_tpl@M@@@spline@@@stlpmtx_std@@@priv@stlpmtx_std@@YAXPAU?$SplineKey@U?$Quat_tpl@M@@@spline@@000U?$less@U?$SplineKey@U?$Quat_tpl@M@@@spline@@@1@@Z 3157f940 f i FaceAnimSequence.obj
 0001:0007eac0       ?InsertKey@?$CBaseSplineInterpolator@U?$Quat_tpl@M@@V?$HermitSplineEx@U?$Quat_tpl@M@@U?$SplineKey@U?$Quat_tpl@M@@@spline@@@spline@@@spline@@UAEHMQAM@Z 3157fac0 f i FaceAnimSequence.obj
 0001:0007ec30       ?Restore@?$CBaseSplineInterpolator@U?$Quat_tpl@M@@V?$HermitSplineEx@U?$Quat_tpl@M@@U?$SplineKey@U?$Quat_tpl@M@@@spline@@@spline@@@spline@@UAEXPAUISplineBackup@@@Z 3157fc30 f i FaceAnimSequence.obj
 0001:0007ec90       ??0?$SSplineBackup@V?$HermitSplineEx@U?$Quat_tpl@M@@U?$SplineKey@U?$Quat_tpl@M@@@spline@@@spline@@@spline@@QAE@ABV?$HermitSplineEx@U?$Quat_tpl@M@@U?$SplineKey@U?$Quat_tpl@M@@@spline@@@1@@Z 3157fc90 f i FaceAnimSequence.obj
 0001:0007ed00       ?AddRef@?$SSplineBackup@V?$HermitSplineEx@MU?$SplineKey@M@spline@@@spline@@@spline@@UAEXXZ 3157fd00 f i FaceAnimSequence.obj
 0001:0007ed00       ?AddRef@?$SSplineBackup@V?$HermitSplineEx@U?$Quat_tpl@M@@U?$SplineKey@U?$Quat_tpl@M@@@spline@@@spline@@@spline@@UAEXXZ 3157fd00 f i FaceAnimSequence.obj
 0001:0007ed00       ?AddRef@?$SSplineBackup@V?$TCBSpline@U?$Vec3_tpl@M@@U?$TCBSplineKey@U?$Vec3_tpl@M@@@spline@@@spline@@@spline@@UAEXXZ 3157fd00 f i FaceAnimSequence.obj
 0001:0007ed10       ?Release@?$SSplineBackup@V?$HermitSplineEx@U?$Quat_tpl@M@@U?$SplineKey@U?$Quat_tpl@M@@@spline@@@spline@@@spline@@UAEXXZ 3157fd10 f i FaceAnimSequence.obj
 0001:0007ed10       ?Release@?$SSplineBackup@V?$HermitSplineEx@MU?$SplineKey@M@spline@@@spline@@@spline@@UAEXXZ 3157fd10 f i FaceAnimSequence.obj
 0001:0007ed10       ?Release@?$SSplineBackup@V?$TCBSpline@U?$Vec3_tpl@M@@U?$TCBSplineKey@U?$Vec3_tpl@M@@@spline@@@spline@@@spline@@UAEXXZ 3157fd10 f i FaceAnimSequence.obj
 0001:0007ed30       ??_E?$SSplineBackup@V?$HermitSplineEx@U?$Quat_tpl@M@@U?$SplineKey@U?$Quat_tpl@M@@@spline@@@spline@@@spline@@W3AEPAXI@Z 3157fd30 f i FaceAnimSequence.obj
 0001:0007ed40       ??_G?$SSplineBackup@V?$HermitSplineEx@U?$Quat_tpl@M@@U?$SplineKey@U?$Quat_tpl@M@@@spline@@@spline@@@spline@@UAEPAXI@Z 3157fd40 f i FaceAnimSequence.obj
 0001:0007ed40       ??_E?$SSplineBackup@V?$HermitSplineEx@U?$Quat_tpl@M@@U?$SplineKey@U?$Quat_tpl@M@@@spline@@@spline@@@spline@@UAEPAXI@Z 3157fd40 f i FaceAnimSequence.obj
 0001:0007eda0       ??$__introsort_loop@PAU?$SplineKey@U?$Quat_tpl@M@@@spline@@U12@HU?$less@U?$SplineKey@U?$Quat_tpl@M@@@spline@@@stlpmtx_std@@@priv@stlpmtx_std@@YAXPAU?$SplineKey@U?$Quat_tpl@M@@@spline@@00HU?$less@U?$SplineKey@U?$Quat_tpl@M@@@spline@@@1@@Z 3157fda0 f i FaceAnimSequence.obj
 0001:0007eef0       ?assign@?$Array@U?$SplineKey@M@spline@@HU?$SmallDynStorage@U?$SplineKey@M@spline@@HUStandardAlloc@NAlloc@@@NArray@@@@QAEXU?$Array@$$CBU?$SplineKey@M@spline@@HU?$ArrayStorage@$$CBU?$SplineKey@M@spline@@H@NArray@@@@@Z 3157fef0 f i FaceAnimSequence.obj
 0001:0007ef40       ?GetKeyValue@?$CBaseSplineInterpolator@MV?$HermitSplineEx@MU?$SplineKey@M@spline@@@spline@@@spline@@UAE_NHAAY03M@Z 3157ff40 f i FaceAnimSequence.obj
 0001:0007ef40       ?GetKeyValue@?$CBaseSplineInterpolator@MV?$CatmullRomSpline@MU?$SplineKey@M@spline@@$0A@@spline@@@spline@@UAE_NHAAY03M@Z 3157ff40 f i FaceEffector.obj
 0001:0007ef80       ?SetKeyValue@?$CBaseSplineInterpolator@MV?$HermitSplineEx@MU?$SplineKey@M@spline@@@spline@@@spline@@UAEXHQAM@Z 3157ff80 f i FaceAnimSequence.obj
 0001:0007ef80       ?SetKeyValue@?$CBaseSplineInterpolator@MV?$CatmullRomSpline@MU?$SplineKey@M@spline@@$0A@@spline@@@spline@@UAEXHQAM@Z 3157ff80 f i FaceEffector.obj
 0001:0007efc0       ?SetKeyOutTangent@?$CBaseSplineInterpolator@MV?$CatmullRomSpline@MU?$SplineKey@M@spline@@$0A@@spline@@@spline@@UAEXHQAM@Z 3157ffc0 f i FaceEffector.obj
 0001:0007efc0       ?SetKeyOutTangent@?$CBaseSplineInterpolator@MV?$HermitSplineEx@MU?$SplineKey@M@spline@@@spline@@@spline@@UAEXHQAM@Z 3157ffc0 f i FaceAnimSequence.obj
 0001:0007f000       ?SetKeyTangents@?$CBaseSplineInterpolator@MV?$CatmullRomSpline@MU?$SplineKey@M@spline@@$0A@@spline@@@spline@@UAEXHQAM0@Z 31580000 f i FaceEffector.obj
 0001:0007f000       ?SetKeyTangents@?$CBaseSplineInterpolator@MV?$HermitSplineEx@MU?$SplineKey@M@spline@@@spline@@@spline@@UAEXHQAM0@Z 31580000 f i FaceAnimSequence.obj
 0001:0007f050       ?init@?$DynArray@UVirtualExample2D@@HU?$SmallDynStorage@UVirtualExample2D@@HUStandardAlloc@NAlloc@@@NArray@@@@KAPAUVirtualExample2D@@U?$Array@UVirtualExample2D@@HU?$ArrayStorage@UVirtualExample2D@@H@NArray@@@@PBU2@@Z 31580050 f i CharacterManager.obj
 0001:0007f050       ?init@?$DynArray@U?$SplineKey@M@spline@@HU?$SmallDynStorage@U?$SplineKey@M@spline@@HUStandardAlloc@NAlloc@@@NArray@@@@KAPAU?$SplineKey@M@spline@@U?$Array@U?$SplineKey@M@spline@@HU?$ArrayStorage@U?$SplineKey@M@spline@@H@NArray@@@@PBU23@@Z 31580050 f i FaceAnimSequence.obj
 0001:0007f0a0       ?erase@?$DynArray@U?$SplineKey@M@spline@@HU?$SmallDynStorage@U?$SplineKey@M@spline@@HUStandardAlloc@NAlloc@@@NArray@@@@QAEPAU?$SplineKey@M@spline@@PAU23@0@Z 315800a0 f i FaceAnimSequence.obj
 0001:0007f120       ?insert_raw@?$DynArray@U?$SplineKey@M@spline@@HU?$SmallDynStorage@U?$SplineKey@M@spline@@HUStandardAlloc@NAlloc@@@NArray@@@@QAE?AU?$Array@U?$SplineKey@M@spline@@HU?$ArrayStorage@U?$SplineKey@M@spline@@H@NArray@@@@PAU?$SplineKey@M@spline@@H@Z 31580120 f i FaceAnimSequence.obj
 0001:0007f1e0       ??4?$DynArray@U?$SplineKey@M@spline@@HU?$SmallDynStorage@U?$SplineKey@M@spline@@HUStandardAlloc@NAlloc@@@NArray@@@@QAEAAU0@U?$Array@$$CBU?$SplineKey@M@spline@@HU?$ArrayStorage@$$CBU?$SplineKey@M@spline@@H@NArray@@@@@Z 315801e0 f i FaceAnimSequence.obj
 0001:0007f280       ?RemoveKey@?$CBaseSplineInterpolator@MV?$HermitSplineEx@MU?$SplineKey@M@spline@@@spline@@@spline@@UAEXH@Z 31580280 f i FaceAnimSequence.obj
 0001:0007f280       ?RemoveKey@?$CBaseSplineInterpolator@MV?$CatmullRomSpline@MU?$SplineKey@M@spline@@$0A@@spline@@@spline@@UAEXH@Z 31580280 f i FaceEffector.obj
 0001:0007f2d0       ??0?$DynArray@U?$SplineKey@M@spline@@HU?$SmallDynStorage@U?$SplineKey@M@spline@@HUStandardAlloc@NAlloc@@@NArray@@@@QAE@ABU0@@Z 315802d0 f i FaceAnimSequence.obj
 0001:0007f350       ?InsertKey@?$CBaseSplineInterpolator@MV?$HermitSplineEx@MU?$SplineKey@M@spline@@@spline@@@spline@@UAEHMQAM@Z 31580350 f i FaceAnimSequence.obj
 0001:0007f350       ?InsertKey@?$CBaseSplineInterpolator@MV?$CatmullRomSpline@MU?$SplineKey@M@spline@@$0A@@spline@@@spline@@UAEHMQAM@Z 31580350 f i FaceEffector.obj
 0001:0007f490       ?Restore@?$CBaseSplineInterpolator@MV?$HermitSplineEx@MU?$SplineKey@M@spline@@@spline@@@spline@@UAEXPAUISplineBackup@@@Z 31580490 f i FaceAnimSequence.obj
 0001:0007f4f0       ??0?$SSplineBackup@V?$HermitSplineEx@MU?$SplineKey@M@spline@@@spline@@@spline@@QAE@ABV?$HermitSplineEx@MU?$SplineKey@M@spline@@@1@@Z 315804f0 f i FaceAnimSequence.obj
 0001:0007f560       ??_E?$SSplineBackup@V?$HermitSplineEx@MU?$SplineKey@M@spline@@@spline@@@spline@@W3AEPAXI@Z 31580560 f i FaceAnimSequence.obj
 0001:0007f570       ??_E?$SSplineBackup@V?$HermitSplineEx@MU?$SplineKey@M@spline@@@spline@@@spline@@UAEPAXI@Z 31580570 f i FaceAnimSequence.obj
 0001:0007f570       ??_G?$SSplineBackup@V?$HermitSplineEx@MU?$SplineKey@M@spline@@@spline@@@spline@@UAEPAXI@Z 31580570 f i FaceAnimSequence.obj
 0001:0007f5d0       ?DeleteSoundEntry@CFacialAnimSequence@@UAEXH@Z 315805d0 f   FaceAnimSequence.obj
 0001:0007f630       ?DeleteSkeletonAnimationEntry@CFacialAnimSequence@@UAEXH@Z 31580630 f   FaceAnimSequence.obj
 0001:0007f680       ?Backup@?$CBaseSplineInterpolator@MV?$HermitSplineEx@MU?$SplineKey@M@spline@@@spline@@@spline@@UAEPAUISplineBackup@@XZ 31580680 f i FaceAnimSequence.obj
 0001:0007f6c0       ?Restore@?$CBaseSplineInterpolator@U?$Vec3_tpl@M@@V?$TCBSpline@U?$Vec3_tpl@M@@U?$TCBSplineKey@U?$Vec3_tpl@M@@@spline@@@spline@@@spline@@UAEXPAUISplineBackup@@@Z 315806c0 f i FaceAnimSequence.obj
 0001:0007f720       ?Backup@?$CBaseSplineInterpolator@U?$Quat_tpl@M@@V?$HermitSplineEx@U?$Quat_tpl@M@@U?$SplineKey@U?$Quat_tpl@M@@@spline@@@spline@@@spline@@UAEPAUISplineBackup@@XZ 31580720 f i FaceAnimSequence.obj
 0001:0007f760       ??0?$SSplineBackup@V?$TCBSpline@U?$Vec3_tpl@M@@U?$TCBSplineKey@U?$Vec3_tpl@M@@@spline@@@spline@@@spline@@QAE@ABV?$TCBSpline@U?$Vec3_tpl@M@@U?$TCBSplineKey@U?$Vec3_tpl@M@@@spline@@@1@@Z 31580760 f i FaceAnimSequence.obj
 0001:0007f7d0       ??_E?$SSplineBackup@V?$TCBSpline@U?$Vec3_tpl@M@@U?$TCBSplineKey@U?$Vec3_tpl@M@@@spline@@@spline@@@spline@@W3AEPAXI@Z 315807d0 f i FaceAnimSequence.obj
 0001:0007f7e0       ??_E?$SSplineBackup@V?$TCBSpline@U?$Vec3_tpl@M@@U?$TCBSplineKey@U?$Vec3_tpl@M@@@spline@@@spline@@@spline@@UAEPAXI@Z 315807e0 f i FaceAnimSequence.obj
 0001:0007f7e0       ??_G?$SSplineBackup@V?$TCBSpline@U?$Vec3_tpl@M@@U?$TCBSplineKey@U?$Vec3_tpl@M@@@spline@@@spline@@@spline@@UAEPAXI@Z 315807e0 f i FaceAnimSequence.obj
 0001:0007f840       ??$sort@PAVEffectorChannelPair@@@stlpmtx_std@@YAXPAVEffectorChannelPair@@0@Z 31580840 f i FaceAnimSequence.obj
 0001:0007f8c0       ??$sort@PAU?$TCBSplineKey@U?$Vec3_tpl@M@@@spline@@@stlpmtx_std@@YAXPAU?$TCBSplineKey@U?$Vec3_tpl@M@@@spline@@0@Z 315808c0 f i FaceAnimSequence.obj
 0001:0007f940       ??$sort@PAU?$SplineKey@M@spline@@@stlpmtx_std@@YAXPAU?$SplineKey@M@spline@@0@Z 31580940 f i FaceAnimSequence.obj
 0001:0007f9a0       ??$sort@PAU?$SplineKey@U?$Quat_tpl@M@@@spline@@@stlpmtx_std@@YAXPAU?$SplineKey@U?$Quat_tpl@M@@@spline@@0@Z 315809a0 f i FaceAnimSequence.obj
 0001:0007fa00       ??$sort@PAU?$pair@PAUIFacialAnimChannel@@H@stlpmtx_std@@VFirstLess@?$VectorMap@PAUIFacialAnimChannel@@HU?$less@PAUIFacialAnimChannel@@@stlpmtx_std@@V?$allocator@U?$pair@PAUIFacialAnimChannel@@H@stlpmtx_std@@@3@@@@stlpmtx_std@@YAXPAU?$pair@PAUIFacialAnimChannel@@H@0@0VFirstLess@?$VectorMap@PAUIFacialAnimChannel@@HU?$less@PAUIFacialAnimChannel@@@stlpmtx_std@@V?$allocator@U?$pair@PAUIFacialAnimChannel@@H@stlpmtx_std@@@3@@@@Z 31580a00 f i FaceAnimSequence.obj
 0001:0007fa80       ?CreateChannelGroup@Data@CFacialAnimSequence@@QAEPAUIFacialAnimChannel@@XZ 31580a80 f i FaceAnimSequence.obj
 0001:0007fb00       ??1CProceduralChannelSet@@QAE@XZ 31580b00 f i FaceAnimSequence.obj
 0001:0007fbb0       ??_ECFacialCameraPathPositionInterpolator@@W3AEPAXI@Z 31580bb0 f i FaceAnimSequence.obj
 0001:0007fbc0       ??_ECFacialCameraPathPositionInterpolator@@UAEPAXI@Z 31580bc0 f i FaceAnimSequence.obj
 0001:0007fbc0       ??_GCFacialCameraPathPositionInterpolator@@UAEPAXI@Z 31580bc0 f i FaceAnimSequence.obj
 0001:0007fc20       ??_ECFacialCameraPathOrientationInterpolator@@W3AEPAXI@Z 31580c20 f i FaceAnimSequence.obj
 0001:0007fc30       ??_ECFacialCameraPathOrientationInterpolator@@UAEPAXI@Z 31580c30 f i FaceAnimSequence.obj
 0001:0007fc30       ??_GCFacialCameraPathOrientationInterpolator@@UAEPAXI@Z 31580c30 f i FaceAnimSequence.obj
 0001:0007fc90       ??_E?$CBaseSplineInterpolator@MV?$HermitSplineEx@MU?$SplineKey@M@spline@@@spline@@@spline@@W3AEPAXI@Z 31580c90 f i FaceAnimSequence.obj
 0001:0007fc90       ??_ECFacialAnimChannelInterpolator@@W3AEPAXI@Z 31580c90 f i FaceAnimSequence.obj
 0001:0007fca0       ??_G?$CBaseSplineInterpolator@MV?$HermitSplineEx@MU?$SplineKey@M@spline@@@spline@@@spline@@UAEPAXI@Z 31580ca0 f i FaceAnimSequence.obj
 0001:0007fca0       ??_ECFacialAnimChannelInterpolator@@UAEPAXI@Z 31580ca0 f i FaceAnimSequence.obj
 0001:0007fca0       ??_GCFacialAnimChannelInterpolator@@UAEPAXI@Z 31580ca0 f i FaceAnimSequence.obj
 0001:0007fca0       ??_E?$CBaseSplineInterpolator@MV?$HermitSplineEx@MU?$SplineKey@M@spline@@@spline@@@spline@@UAEPAXI@Z 31580ca0 f i FaceAnimSequence.obj
 0001:0007fd00       ?CreateInterpolator@CFacialAnimChannel@@QAEXXZ 31580d00 f   FaceAnimSequence.obj
 0001:0007fe60       ?AddInterpolator@CFacialAnimChannel@@UAEXXZ 31580e60 f   FaceAnimSequence.obj
 0001:0007fef0       ??1Data@CFacialAnimSequence@@QAE@XZ 31580ef0 f i FaceAnimSequence.obj
 0001:00080010       ??1CFacialAnimSequence@@UAE@XZ 31581010 f   FaceAnimSequence.obj
 0001:000800b0       ?AddRef@CFacialAnimSequence@@UAEXXZ 315810b0 f i FaceAnimSequence.obj
 0001:000800c0       ?SetFlags@CFacialAnimSequence@@UAEXH@Z 315810c0 f i FaceAnimSequence.obj
 0001:000800d0       ?GetEffectorName@CFacialAnimChannel@@UAEPBDXZ 315810d0 f i FaceAnimSequence.obj
 0001:000800d0       ?GetFlags@CFacialAnimSequence@@UAEHXZ 315810d0 f i FaceAnimSequence.obj
 0001:000800d0       ?GetSpline@CFacialEffCtrl@@UAEPAUISplineInterpolator@@XZ 315810d0 f i FaceEffector.obj
 0001:000800e0       ?GetCameraPathPosition@CFacialAnimSequence@@UAEPAUISplineInterpolator@@XZ 315810e0 f i FaceAnimSequence.obj
 0001:000800f0       ?GetCameraPathOrientation@CFacialAnimSequence@@UAEPAUISplineInterpolator@@XZ 315810f0 f i FaceAnimSequence.obj
 0001:00080100       ?GetCameraPathFOV@CFacialAnimSequence@@UAEPAUISplineInterpolator@@XZ 31581100 f i FaceAnimSequence.obj
 0001:00080110       ?IsInMemory@CFacialAnimSequence@@UBE_NXZ 31581110 f i FaceAnimSequence.obj
 0001:00080120       ?SetInMemory@CFacialAnimSequence@@UAEX_N@Z 31581120 f i FaceAnimSequence.obj
 0001:00080130       ??_ECFacialAnimSequence@@W3AEPAXI@Z 31581130 f i FaceAnimSequence.obj
 0001:00080140       ?GetTimeRange@CFacialAnimSequence@@UAE?AV?$TRange@M@@XZ 31581140 f i FaceAnimSequence.obj
 0001:00080160       ?SetTimeRange@CFacialAnimSequence@@UAEXV?$TRange@M@@@Z 31581160 f i FaceAnimSequence.obj
 0001:00080180       ?GetChannelCount@CFacialAnimSequence@@UAEHXZ 31581180 f i FaceAnimSequence.obj
 0001:00080190       ?CreateChannelGroup@CFacialAnimSequence@@UAEPAUIFacialAnimChannel@@XZ 31581190 f   FaceAnimSequence.obj
 0001:000801a0       ?StreamOnComplete@CFacialAnimSequence@@UAEXPAVIReadStream@@I@Z 315811a0 f   FaceAnimSequence.obj
 0001:00080370       ?UnbindProceduralChannels@CFacialAnimSequenceInstance@@AAEXXZ 31581370 f   FaceAnimSequence.obj
 0001:000803d0       ?Backup@?$CBaseSplineInterpolator@U?$Vec3_tpl@M@@V?$TCBSpline@U?$Vec3_tpl@M@@U?$TCBSplineKey@U?$Vec3_tpl@M@@@spline@@@spline@@@spline@@UAEPAUISplineBackup@@XZ 315813d0 f i FaceAnimSequence.obj
 0001:00080410       ?resize@?$_Impl_vector@UChannelInfo@CFacialAnimSequenceInstance@@V?$allocator@UChannelInfo@CFacialAnimSequenceInstance@@@stlpmtx_std@@@priv@stlpmtx_std@@QAEXIABUChannelInfo@CFacialAnimSequenceInstance@@@Z 31581410 f i FaceAnimSequence.obj
 0001:00080490       ?SwapElementsWithVector@?$VectorMap@PAUIFacialAnimChannel@@HU?$less@PAUIFacialAnimChannel@@@stlpmtx_std@@V?$allocator@U?$pair@PAUIFacialAnimChannel@@H@stlpmtx_std@@@3@@@QAEXAAV?$vector@U?$pair@PAUIFacialAnimChannel@@H@stlpmtx_std@@V?$allocator@U?$pair@PAUIFacialAnimChannel@@H@stlpmtx_std@@@2@@stlpmtx_std@@@Z 31581490 f i FaceAnimSequence.obj
 0001:00080500       ?CreateChannel@Data@CFacialAnimSequence@@QAEPAUIFacialAnimChannel@@XZ 31581500 f i FaceAnimSequence.obj
 0001:00080570       ??_GCFacialAnimSequence@@UAEPAXI@Z 31581570 f i FaceAnimSequence.obj
 0001:00080570       ??_ECFacialAnimSequence@@UAEPAXI@Z 31581570 f i FaceAnimSequence.obj
 0001:000805a0       ?CreateChannel@CFacialAnimSequence@@UAEPAUIFacialAnimChannel@@XZ 315815a0 f   FaceAnimSequence.obj
 0001:000805b0       ?SerializeChannelLoad@CFacialAnimSequence@@AAEXAAUData@1@PAUIFacialAnimChannel@@AAVXmlNodeRef@@@Z 315815b0 f   FaceAnimSequence.obj
 0001:000807c0       ?UnbindChannels@CFacialAnimSequenceInstance@@QAEXXZ 315817c0 f   FaceAnimSequence.obj
 0001:00080890       ??0CProceduralChannelSet@@QAE@XZ 31581890 f   FaceAnimSequence.obj
 0001:000809e0       ?insert@?$_Impl_vector@VCFacialAnimSoundEntry@@V?$allocator@VCFacialAnimSoundEntry@@@stlpmtx_std@@@priv@stlpmtx_std@@QAEPAVCFacialAnimSoundEntry@@PAV4@ABV4@@Z 315819e0 f i FaceAnimSequence.obj
 0001:00080a60       ??0Data@CFacialAnimSequence@@QAE@XZ 31581a60 f i FaceAnimSequence.obj
 0001:00080ba0       ??0CFacialAnimSequence@@QAE@PAVCFacialAnimation@@@Z 31581ba0 f   FaceAnimSequence.obj
 0001:00080c00       ?StartStreaming@CFacialAnimSequence@@UAE_NPBD@Z 31581c00 f   FaceAnimSequence.obj
 0001:00080d60       ?BindProceduralChannels@CFacialAnimSequenceInstance@@AAEXPAVCFacialAnimationContext@@PAVCFacialAnimSequence@@@Z 31581d60 f   FaceAnimSequence.obj
 0001:00080ef0       ?interpolate@?$TSpline@U?$TCBSplineKey@U?$Vec3_tpl@M@@@spline@@VHermitBasis@2@@spline@@QAE_NMAAU?$Vec3_tpl@M@@@Z 31581ef0 f i FaceAnimSequence.obj
 0001:00081030       ?Interpolate@?$CBaseSplineInterpolator@MV?$HermitSplineEx@MU?$SplineKey@M@spline@@@spline@@@spline@@UAEXMAAY03M@Z 31582030 f i FaceAnimSequence.obj
 0001:00081060       ?interpolate@?$TSpline@U?$SplineKey@U?$Quat_tpl@M@@@spline@@VHermitBasis@2@@spline@@QAE_NMAAU?$Quat_tpl@M@@@Z 31582060 f i FaceAnimSequence.obj
 0001:00081180       ?insert@?$vector@VCFacialAnimSkeletalAnimationEntry@@V?$allocator@VCFacialAnimSkeletalAnimationEntry@@@stlpmtx_std@@@stlpmtx_std@@QAEPAVCFacialAnimSkeletalAnimationEntry@@PAV3@ABV3@@Z 31582180 f i FaceAnimSequence.obj
 0001:000811e0       ?resize@?$_Impl_vector@VCFacialAnimSkeletalAnimationEntry@@V?$allocator@VCFacialAnimSkeletalAnimationEntry@@@stlpmtx_std@@@priv@stlpmtx_std@@QAEXIABVCFacialAnimSkeletalAnimationEntry@@@Z 315821e0 f i FaceAnimSequence.obj
 0001:00081260       ?resize@?$_Impl_vector@VCFacialAnimSoundEntry@@V?$allocator@VCFacialAnimSoundEntry@@@stlpmtx_std@@@priv@stlpmtx_std@@QAEXIABVCFacialAnimSoundEntry@@@Z 31582260 f i FaceAnimSequence.obj
 0001:00081300       ?Interpolate@CFacialAnimChannelInterpolator@@UAEXMAAY03M@Z 31582300 f i FaceAnimSequence.obj
 0001:00081340       ?Interpolate@CFacialCameraPathPositionInterpolator@@UAEXMAAY03M@Z 31582340 f i FaceAnimSequence.obj
 0001:00081390       ?Interpolate@CFacialCameraPathOrientationInterpolator@@UAEXMAAY03M@Z 31582390 f i FaceAnimSequence.obj
 0001:00081400       ?Evaluate@CFacialAnimChannel@@QAEMM@Z 31582400 f   FaceAnimSequence.obj
 0001:000815f0       ?InsertSoundEntry@CFacialAnimSequence@@UAEXH@Z 315825f0 f   FaceAnimSequence.obj
 0001:00081670       ?InsertSkeletonAnimationEntry@CFacialAnimSequence@@UAEXH@Z 31582670 f   FaceAnimSequence.obj
 0001:00081700       ?MergeSequence@CFacialAnimSequence@@UAEXPAUIFacialAnimSequence@@ABV?$Functor1wRet@PBDW4MergeCollisionAction@@@@@Z 31582700 f   FaceAnimSequence.obj
 0001:00082bd0       ?BindChannels@CFacialAnimSequenceInstance@@QAEXPAVCFacialAnimationContext@@PAVCFacialAnimSequence@@@Z 31583bd0 f   FaceAnimSequence.obj
 0001:000833d0       ?Animate@CFacialAnimSequence@@UAEXABU?$QuatTS_tpl@M@@PAVCFacialAnimSequenceInstance@@M@Z 315843d0 f   FaceAnimSequence.obj
 0001:00083da0       ?SerializeLoad@CFacialAnimSequence@@AAEXAAUData@1@AAVXmlNodeRef@@W4ESerializationFlags@IFacialAnimSequence@@@Z 31584da0 f   FaceAnimSequence.obj
 0001:00084520       ?Serialize@CFacialAnimSequence@@UAEXAAVXmlNodeRef@@_NW4ESerializationFlags@IFacialAnimSequence@@@Z 31585520 f   FaceAnimSequence.obj
 0001:00084850       ?StreamAsyncOnComplete@CFacialAnimSequence@@UAEXPAVIReadStream@@I@Z 31585850 f   FaceAnimSequence.obj
 0001:00084920       ??$fill@PAVFaceChannelCleanupKeysKeyEntry@@V1@@stlpmtx_std@@YAXPAVFaceChannelCleanupKeysKeyEntry@@0ABV1@@Z 31585920 f i FaceChannelKeyCleanup.obj
 0001:00084960       ?_M_insert_overflow@?$_Impl_vector@VFaceChannelCleanupKeysKeyEntry@@V?$allocator@VFaceChannelCleanupKeysKeyEntry@@@stlpmtx_std@@@priv@stlpmtx_std@@AAEXPAVFaceChannelCleanupKeysKeyEntry@@ABV4@ABU__true_type@3@I_N@Z 31585960 f i FaceChannelKeyCleanup.obj
 0001:00084af0       ??$__uninitialized_fill_n@PAVFaceChannelCleanupKeysKeyEntry@@IV1@@priv@stlpmtx_std@@YAPAVFaceChannelCleanupKeysKeyEntry@@PAV2@IABV2@@Z 31585af0 f i FaceChannelKeyCleanup.obj
 0001:00084b70       ?_M_fill_insert_aux@?$_Impl_vector@VFaceChannelCleanupKeysKeyEntry@@V?$allocator@VFaceChannelCleanupKeysKeyEntry@@@stlpmtx_std@@@priv@stlpmtx_std@@AAEXPAVFaceChannelCleanupKeysKeyEntry@@IABV4@ABU__false_type@3@@Z 31585b70 f i FaceChannelKeyCleanup.obj
 0001:00084ca0       ?insert@?$_Impl_vector@VFaceChannelCleanupKeysKeyEntry@@V?$allocator@VFaceChannelCleanupKeysKeyEntry@@@stlpmtx_std@@@priv@stlpmtx_std@@QAEXPAVFaceChannelCleanupKeysKeyEntry@@IABV4@@Z 31585ca0 f i FaceChannelKeyCleanup.obj
 0001:00084d00       ?resize@?$_Impl_vector@VFaceChannelCleanupKeysKeyEntry@@V?$allocator@VFaceChannelCleanupKeysKeyEntry@@@stlpmtx_std@@@priv@stlpmtx_std@@QAEXIABVFaceChannelCleanupKeysKeyEntry@@@Z 31585d00 f i FaceChannelKeyCleanup.obj
 0001:00084d90       ??0?$CBaseSplineInterpolator@MV?$HermitSplineEx@MU?$SplineKey@M@spline@@@spline@@@spline@@QAE@ABV01@@Z 31585d90 f i FaceChannelKeyCleanup.obj
 0001:00084e00       ?CleanupKeys@FaceChannel@@YAXPAVCFacialAnimChannelInterpolator@@M@Z 31585e00 f   FaceChannelKeyCleanup.obj
 0001:00085a70       ??0GaussianKernel@FaceChannel@@QAE@M_N@Z 31586a70 f   FaceChannelSmoothing.obj
 0001:00085b30       ?ApplyKernel@FaceChannel@@YAXPAVCFacialAnimChannelInterpolator@@0HPBM@Z 31586b30 f   FaceChannelSmoothing.obj
 0001:00085c90       ?ApplyKernelNoiseFilter@FaceChannel@@YAXPAVCFacialAnimChannelInterpolator@@0HPBMM@Z 31586c90 f   FaceChannelSmoothing.obj
 0001:00085e30       ?RemoveNoise@FaceChannel@@YAXPAVCFacialAnimChannelInterpolator@@MM@Z 31586e30 f   FaceChannelSmoothing.obj
 0001:00085ed0       ?GaussianBlurKeys@FaceChannel@@YAXPAVCFacialAnimChannelInterpolator@@M@Z 31586ed0 f   FaceChannelSmoothing.obj
 0001:00085f60       ??_EIFacialEffector@@UAEPAXI@Z 31586f60 f i FaceEffector.obj
 0001:00085f60       ??_GIFacialEffector@@UAEPAXI@Z 31586f60 f i FaceEffector.obj
 0001:00085f90       ?GetParamString@CFacialEffector@@UAEPBDW4EFacialEffectorParam@@@Z 31586f90 f i FaceEffector.obj
 0001:00085fa0       ?SetVideoMarkerScale@CFacialJoystickChannel@@UAEXM@Z 31586fa0 f   FaceJoystick.obj
 0001:00085fa0       ?SetConstantBalance@CFacialEffCtrl@@UAEXM@Z 31586fa0 f   FaceEffector.obj
 0001:00085fc0       ?Interpolate@CFacialEffCtrlSplineInterpolator@@UAEXMAAY03M@Z 31586fc0 f   FaceEffector.obj
 0001:00085fe0       ?SetParamInt@CFacialEffector@@UAEXW4EFacialEffectorParam@@H@Z 31586fe0 f   FaceEffector.obj
 0001:00085fe0       ?UnMarkPool@CDummyMemReplay@@UAEXHPAX@Z 31586fe0 f   AnimEventList.obj
 0001:00085fe0       ?OnRemoveAttachment@IAttachmentObject@@UAEXPAUIAttachmentManager@@H@Z 31586fe0 f   AttachmentManager.obj
 0001:00085fe0       ?BucketEnableCleanups@CDummyMemReplay@@UAEXPAX_N@Z 31586fe0 f   AnimEventList.obj
 0001:00085fe0       ?RegisterContainer@CDummyMemReplay@@UAEXPBXH@Z 31586fe0 f   AnimEventList.obj
 0001:00085fe0       ?UnMarkBucket@CDummyMemReplay@@UAEXHPAX@Z 31586fe0 f   AnimEventList.obj
 0001:00085fe0       ?StreamAsyncOnComplete@IStreamCallback@@UAEXPAVIReadStream@@I@Z 31586fe0 f   FaceAnimSequence.obj
 0001:00085fe0       ?Start@CDummyMemReplay@@UAEX_NPBD@Z 31586fe0 f   AnimEventList.obj
 0001:00085fe0       ?RenderAttachment@IAttachmentObject@@UAEXAAUSRendParams@@ABUSRenderingPassInfo@@@Z 31586fe0 f   AttachmentManager.obj
 0001:00085fe0       ?UnMapPage@CDummyMemReplay@@UAEXPAXI@Z 31586fe0 f   AnimEventList.obj
 0001:00085fe0       ?MapPage@CDummyMemReplay@@UAEXPAXI@Z 31586fe0 f   AnimEventList.obj
 0001:00085fe0       ?SwapContainers@CDummyMemReplay@@UAEXPBX0@Z 31586fe0 f   AnimEventList.obj
 0001:00085fe0       ?AddAllocReference@CDummyMemReplay@@UAEXPAX0@Z 31586fe0 f   AnimEventList.obj
 0001:00085fe0       ?SetDefaultAbsInvJointByID@CSkeletonPose@@UAEXHABU?$QuatT_tpl@M@@@Z 31586fe0 f   SkeletonPose.obj
 0001:00085fe0       ?BindToContainer@CDummyMemReplay@@UAEXPBX0@Z 31586fe0 f   AnimEventList.obj
 0001:00085fe0       ?StreamOnComplete@IStreamCallback@@UAEXPAVIReadStream@@I@Z 31586fe0 f   FaceAnimSequence.obj
 0001:00085fe0       ?SetParamString@CFacialEffector@@UAEXW4EFacialEffectorParam@@PBD@Z 31586fe0 f   FaceEffector.obj
 0001:00085fe0       ?UnbindFromContainer@CDummyMemReplay@@UAEXPBX0@Z 31586fe0 f   AnimEventList.obj
 0001:00085fe0       ?Serialize@CFacialEffector@@UAEXAAVXmlNodeRef@@_N@Z 31586fe0 f   FaceEffector.obj
 0001:00085ff0       ?GetParamString@CFacialEffectorAttachment@@UAEPBDW4EFacialEffectorParam@@@Z 31586ff0 f   FaceEffector.obj
 0001:00086010       ?GetParamVec3@CFacialEffectorAttachment@@UAE?AU?$Vec3_tpl@M@@W4EFacialEffectorParam@@@Z 31587010 f   FaceEffector.obj
 0001:00086070       ?GetSubEffector@CFacialEffector@@UAEPAUIFacialEffector@@H@Z 31587070 f   FaceEffector.obj
 0001:000860a0       ?GetSubEffCtrl@CFacialEffector@@UAEPAUIFacialEffCtrl@@H@Z 315870a0 f   FaceEffector.obj
 0001:000860b0       ?SetParamVec3@CFacialEffectorAttachment@@UAEXW4EFacialEffectorParam@@U?$Vec3_tpl@M@@@Z 315870b0 f   FaceEffector.obj
 0001:00086210       ?GetQuatT@CFacialEffectorAttachment@@UAE?AU?$QuatT_tpl@M@@XZ 31587210 f   FaceEffector.obj
 0001:00086250       ?seek_key@?$TSpline@U?$SplineKey@M@spline@@U?$TCoeffBasis@M@2@@spline@@IAEHM@Z 31587250 f i FaceEffector.obj
 0001:00086250       ?seek_key@?$TSpline@U?$SplineKey@M@spline@@VHermitBasis@2@@spline@@IAEHM@Z 31587250 f i FaceAnimSequence.obj
 0001:000862c0       ?Set@CFacialEffectorAttachment@@UAEXQBV1@@Z 315872c0 f   FaceEffector.obj
 0001:00086370       ?SetIdentifier@CFacialEffector@@UAEXVCFaceIdentifierHandle@@@Z 31587370 f   FaceEffector.obj
 0001:000863e0       ?GetMemoryUsage@CFacialEffector@@UBEXPAVICrySizer@@@Z 315873e0 f   FaceEffector.obj
 0001:00086480       ?SetParamString@CFacialEffectorAttachment@@UAEXW4EFacialEffectorParam@@PBD@Z 31587480 f   FaceEffector.obj
 0001:000864d0       ?Serialize@CFacialEffectorAttachment@@UAEXAAVXmlNodeRef@@_N@Z 315874d0 f   FaceEffector.obj
 0001:00086730       ?_M_erase@?$_Impl_vector@V?$_smart_ptr@VCFacialEffector@@@@V?$allocator@V?$_smart_ptr@VCFacialEffector@@@@@stlpmtx_std@@@priv@stlpmtx_std@@AAEPAV?$_smart_ptr@VCFacialEffector@@@@PAV4@0ABU__false_type@3@@Z 31587730 f i FaceEffectorLibrary.obj
 0001:00086730       ?_M_erase@?$_Impl_vector@V?$_smart_ptr@VCFacialEffCtrl@@@@V?$allocator@V?$_smart_ptr@VCFacialEffCtrl@@@@@stlpmtx_std@@@priv@stlpmtx_std@@AAEPAV?$_smart_ptr@VCFacialEffCtrl@@@@PAV4@0ABU__false_type@3@@Z 31587730 f i FaceEffector.obj
 0001:00086730       ?_M_erase@?$_Impl_vector@V?$_smart_ptr@VCFacialAnimChannel@@@@V?$allocator@V?$_smart_ptr@VCFacialAnimChannel@@@@@stlpmtx_std@@@priv@stlpmtx_std@@AAEPAV?$_smart_ptr@VCFacialAnimChannel@@@@PAV4@0ABU__false_type@3@@Z 31587730 f i FaceAnimSequence.obj
 0001:000867b0       ?SerializeSpline@CFacialEffCtrlSplineInterpolator@@UAEXAAVXmlNodeRef@@_N@Z 315877b0 f   FaceEffector.obj
 0001:000869e0       ?RemoveSubEffector@CFacialEffector@@UAEXPAUIFacialEffector@@@Z 315879e0 f   FaceEffector.obj
 0001:00086ad0       ?GetMemoryUsage@?$TSpline@U?$SplineKey@M@spline@@VHermitBasis@2@@spline@@UBEXPAVICrySizer@@_N@Z 31587ad0 f i FaceAnimSequence.obj
 0001:00086ad0       ?GetMemoryUsage@?$TSpline@U?$SplineKey@M@spline@@U?$TCoeffBasis@M@2@@spline@@UBEXPAVICrySizer@@_N@Z 31587ad0 f i FaceEffector.obj
 0001:00086b10       ??_E?$TSpline@U?$SplineKey@M@spline@@U?$TCoeffBasis@M@2@@spline@@UAEPAXI@Z 31587b10 f i FaceEffector.obj
 0001:00086b10       ??_E?$TSpline@U?$SplineKey@M@spline@@VHermitBasis@2@@spline@@UAEPAXI@Z 31587b10 f i FaceAnimSequence.obj
 0001:00086b10       ??_G?$TSpline@U?$SplineKey@M@spline@@U?$TCoeffBasis@M@2@@spline@@UAEPAXI@Z 31587b10 f i FaceEffector.obj
 0001:00086b10       ??_G?$TSpline@U?$SplineKey@M@spline@@VHermitBasis@2@@spline@@UAEPAXI@Z 31587b10 f i FaceAnimSequence.obj
 0001:00086b60       ??0?$TSpline@U?$SplineKey@M@spline@@U?$TCoeffBasis@M@2@@spline@@QAE@XZ 31587b60 f i FaceEffector.obj
 0001:00086b60       ??0?$TSpline@U?$SplineKey@M@spline@@VHermitBasis@2@@spline@@QAE@XZ 31587b60 f i FaceAnimSequence.obj
 0001:00086bc0       ??0CFacialEffector@@QAE@XZ 31587bc0 f i FaceEffector.obj
 0001:00086c20       ?SetFlags@CFacialEffector@@UAEXI@Z 31587c20 f i FaceEffector.obj
 0001:00086c30       ?GetIndexInState@CFacialEffector@@UAEHXZ 31587c30 f i FaceEffector.obj
 0001:00086c30       ?GetLibrary@CFacialModel@@UAEPAUIFacialEffectorsLibrary@@XZ 31587c30 f i FacialModel.obj
 0001:00086c40       ??_ECFacialMorphTarget@@W3AEPAXI@Z 31587c40 f i FaceEffectorLibrary.obj
 0001:00086c40       ??_ECFacialEffector@@W3AEPAXI@Z 31587c40 f i FaceEffector.obj
 0001:00086c40       ??_ECFacialEffectorExpression@@W3AEPAXI@Z 31587c40 f i FaceEffectorLibrary.obj
 0001:00086c50       ?GetIdentifier@CFacialEffector@@UAE?AVCFaceIdentifierHandle@@XZ 31587c50 f i FaceEffector.obj
 0001:00086c70       ?GetParamVec3@CFacialEffector@@UAE?AU?$Vec3_tpl@M@@W4EFacialEffectorParam@@@Z 31587c70 f i FaceEffector.obj
 0001:00086c90       ?GetQuatT@CFacialEffector@@UAE?AU?$QuatT_tpl@M@@XZ 31587c90 f i FaceEffector.obj
 0001:00086cd0       ?GetSubEffectorCount@CFacialEffector@@UAEHXZ 31587cd0 f i FaceEffector.obj
 0001:00086ce0       ??0CFaceIdentifierStorage@@QAE@V?$CryStringT@D@@@Z 31587ce0 f i FaceEffector.obj
 0001:00086d80       ?SetName@CFacialEffector@@UAEXPBD@Z 31587d80 f i FaceEffector.obj
 0001:00086de0       ?GetName@CFacialEffector@@UBEPBDXZ 31587de0 f i FaceEffector.obj
 0001:00086e20       ??_GCFacialEffector@@UAEPAXI@Z 31587e20 f i FaceEffector.obj
 0001:00086e20       ??_GCFacialMorphTarget@@UAEPAXI@Z 31587e20 f i FaceEffectorLibrary.obj
 0001:00086e20       ??_ECFacialEffector@@UAEPAXI@Z 31587e20 f i FaceEffector.obj
 0001:00086e20       ??_ECFacialEffectorExpression@@UAEPAXI@Z 31587e20 f i FaceEffectorLibrary.obj
 0001:00086e20       ??_ECFacialMorphTarget@@UAEPAXI@Z 31587e20 f i FaceEffectorLibrary.obj
 0001:00086e20       ??_GCFacialEffectorExpression@@UAEPAXI@Z 31587e20 f i FaceEffectorLibrary.obj
 0001:00086e80       ??1?$CatmullRomSpline@MU?$SplineKey@M@spline@@$0A@@spline@@UAE@XZ 31587e80 f i FaceEffector.obj
 0001:00086ee0       ?comp_deriv@?$TSplineSlopes@MU?$SplineKey@M@spline@@$0A@@spline@@UAEXXZ 31587ee0 f i FaceEffector.obj
 0001:00086fd0       ?RemoveAllSubEffectors@CFacialEffector@@UAEXXZ 31587fd0 f   FaceEffector.obj
 0001:00087000       ??0CFacialEffectorAttachment@@QAE@XZ 31588000 f   FaceEffector.obj
 0001:000870a0       ?SetAttachmentCRC@CFacialEffectorAttachment@@UAEXI@Z 315880a0 f i FaceEffector.obj
 0001:000870b0       ?GetAttachmentCRC@CFacialEffectorAttachment@@UAEIXZ 315880b0 f i FaceEffector.obj
 0001:000870c0       ?SetQuatT@CFacialEffectorAttachment@@UAEXU?$QuatT_tpl@M@@@Z 315880c0 f i FaceEffector.obj
 0001:00087110       ?GetMemoryUsage@CFacialEffectorAttachment@@UBEXPAVICrySizer@@@Z 31588110 f i FaceEffector.obj
 0001:00087140       ??1CFacialEffectorAttachment@@UAE@XZ 31588140 f i FaceEffector.obj
 0001:000871b0       ??$fill@PAU?$TCoeffBasis@M@spline@@U12@@stlpmtx_std@@YAXPAU?$TCoeffBasis@M@spline@@0ABU12@@Z 315881b0 f i FaceEffector.obj
 0001:000871b0       ??$fill@PAUBalanceChannelEntry@CFacialAnimSequenceInstance@@U12@@stlpmtx_std@@YAXPAUBalanceChannelEntry@CFacialAnimSequenceInstance@@0ABU12@@Z 315881b0 f i FaceAnimSequence.obj
 0001:000871f0       ?interp_keys@?$CatmullRomSpline@MU?$SplineKey@M@spline@@$0A@@spline@@MAEXHHMAAM@Z 315881f0 f i FaceEffector.obj
 0001:00087250       ??$__uninitialized_fill_n@PAUBalanceChannelEntry@CFacialAnimSequenceInstance@@IU12@@priv@stlpmtx_std@@YAPAUBalanceChannelEntry@CFacialAnimSequenceInstance@@PAU23@IABU23@@Z 31588250 f i FaceAnimSequence.obj
 0001:00087250       ??$__uninitialized_fill_n@PAU?$TCoeffBasis@M@spline@@IU12@@priv@stlpmtx_std@@YAPAU?$TCoeffBasis@M@spline@@PAU23@IABU23@@Z 31588250 f i FaceEffector.obj
 0001:000872b0       ?GetMemoryUsage@?$CatmullRomSpline@MU?$SplineKey@M@spline@@$0A@@spline@@UBEXPAVICrySizer@@_N@Z 315882b0 f i FaceEffector.obj
 0001:00087330       ??_G?$CatmullRomSpline@MU?$SplineKey@M@spline@@$0A@@spline@@UAEPAXI@Z 31588330 f i FaceEffector.obj
 0001:00087330       ??_E?$CatmullRomSpline@MU?$SplineKey@M@spline@@$0A@@spline@@UAEPAXI@Z 31588330 f i FaceEffector.obj
 0001:00087360       ?comp_deriv@?$CatmullRomSpline@MU?$SplineKey@M@spline@@$0A@@spline@@MAEXXZ 31588360 f i FaceEffector.obj
 0001:00087570       ?FindKeysInRange@?$CBaseSplineInterpolator@MV?$CatmullRomSpline@MU?$SplineKey@M@spline@@$0A@@spline@@@spline@@UAEXMMAAH0@Z 31588570 f i FaceEffector.obj
 0001:00087570       ?FindKeysInRange@?$CBaseSplineInterpolator@MV?$HermitSplineEx@MU?$SplineKey@M@spline@@@spline@@@spline@@UAEXMMAAH0@Z 31588570 f i FaceAnimSequence.obj
 0001:000876a0       ?GetAnimationCount@CAnimationSet@@UBEIXZ 315886a0 f i ModelAnimationSet.obj
 0001:000876a0       ?GetKeyCount@?$CBaseSplineInterpolator@MV?$CatmullRomSpline@MU?$SplineKey@M@spline@@$0A@@spline@@@spline@@UAEHXZ 315886a0 f i FaceEffector.obj
 0001:000876a0       ?GetKeyCount@?$CBaseSplineInterpolator@U?$Quat_tpl@M@@V?$HermitSplineEx@U?$Quat_tpl@M@@U?$SplineKey@U?$Quat_tpl@M@@@spline@@@spline@@@spline@@UAEHXZ 315886a0 f i FaceAnimSequence.obj
 0001:000876a0       ?GetKeyCount@?$CBaseSplineInterpolator@MV?$HermitSplineEx@MU?$SplineKey@M@spline@@@spline@@@spline@@UAEHXZ 315886a0 f i FaceAnimSequence.obj
 0001:000876a0       ?GetKeyCount@?$CBaseSplineInterpolator@U?$Vec3_tpl@M@@V?$TCBSpline@U?$Vec3_tpl@M@@U?$TCBSplineKey@U?$Vec3_tpl@M@@@spline@@@spline@@@spline@@UAEHXZ 315886a0 f i FaceAnimSequence.obj
 0001:000876b0       ?GetKeyTime@?$CBaseSplineInterpolator@MV?$HermitSplineEx@MU?$SplineKey@M@spline@@@spline@@@spline@@UAEMH@Z 315886b0 f i FaceAnimSequence.obj
 0001:000876b0       ?GetKeyTime@?$CBaseSplineInterpolator@MV?$CatmullRomSpline@MU?$SplineKey@M@spline@@$0A@@spline@@@spline@@UAEMH@Z 315886b0 f i FaceEffector.obj
 0001:000876e0       ?SetKeyTime@?$CBaseSplineInterpolator@MV?$CatmullRomSpline@MU?$SplineKey@M@spline@@$0A@@spline@@@spline@@UAEXHM@Z 315886e0 f i FaceEffector.obj
 0001:000876e0       ?SetKeyTime@?$CBaseSplineInterpolator@MV?$HermitSplineEx@MU?$SplineKey@M@spline@@@spline@@@spline@@UAEXHM@Z 315886e0 f i FaceAnimSequence.obj
 0001:00087720       ?SetKeyInTangent@?$CBaseSplineInterpolator@MV?$CatmullRomSpline@MU?$SplineKey@M@spline@@$0A@@spline@@@spline@@UAEXHQAM@Z 31588720 f i FaceEffector.obj
 0001:00087720       ?SetKeyInTangent@?$CBaseSplineInterpolator@MV?$HermitSplineEx@MU?$SplineKey@M@spline@@@spline@@@spline@@UAEXHQAM@Z 31588720 f i FaceAnimSequence.obj
 0001:00087760       ?GetKeyTangents@?$CBaseSplineInterpolator@MV?$CatmullRomSpline@MU?$SplineKey@M@spline@@$0A@@spline@@@spline@@UAE_NHAAY03M0@Z 31588760 f i FaceEffector.obj
 0001:00087760       ?GetKeyTangents@?$CBaseSplineInterpolator@MV?$HermitSplineEx@MU?$SplineKey@M@spline@@@spline@@@spline@@UAE_NHAAY03M0@Z 31588760 f i FaceAnimSequence.obj
 0001:000877a0       ?SetKeyFlags@?$CBaseSplineInterpolator@MV?$CatmullRomSpline@MU?$SplineKey@M@spline@@$0A@@spline@@@spline@@UAEXHH@Z 315887a0 f i FaceEffector.obj
 0001:000877a0       ?SetKeyFlags@?$CBaseSplineInterpolator@MV?$HermitSplineEx@MU?$SplineKey@M@spline@@@spline@@@spline@@UAEXHH@Z 315887a0 f i FaceAnimSequence.obj
 0001:000877e0       ?GetKeyFlags@?$CBaseSplineInterpolator@MV?$HermitSplineEx@MU?$SplineKey@M@spline@@@spline@@@spline@@UAEHH@Z 315887e0 f i FaceAnimSequence.obj
 0001:000877e0       ?GetKeyFlags@?$CBaseSplineInterpolator@MV?$CatmullRomSpline@MU?$SplineKey@M@spline@@$0A@@spline@@@spline@@UAEHH@Z 315887e0 f i FaceEffector.obj
 0001:00087810       ??$_M_allocate_and_copy@PBUPhoneme@IFacialSentence@@@?$_Impl_vector@UPhoneme@IFacialSentence@@V?$allocator@UPhoneme@IFacialSentence@@@stlpmtx_std@@@priv@stlpmtx_std@@AAEPAUPhoneme@IFacialSentence@@AAIPBU34@1@Z 31588810 f i LipSync.obj
 0001:00087810       ??$_M_allocate_and_copy@PBU?$TCoeffBasis@M@spline@@@?$_Impl_vector@U?$TCoeffBasis@M@spline@@V?$allocator@U?$TCoeffBasis@M@spline@@@stlpmtx_std@@@priv@stlpmtx_std@@AAEPAU?$TCoeffBasis@M@spline@@AAIPBU34@1@Z 31588810 f i FaceEffector.obj
 0001:00087880       ?RemoveKeysInRange@?$CBaseSplineInterpolator@MV?$HermitSplineEx@MU?$SplineKey@M@spline@@@spline@@@spline@@UAEXMM@Z 31588880 f i FaceAnimSequence.obj
 0001:00087880       ?RemoveKeysInRange@?$CBaseSplineInterpolator@MV?$CatmullRomSpline@MU?$SplineKey@M@spline@@$0A@@spline@@@spline@@UAEXMM@Z 31588880 f i FaceEffector.obj
 0001:000879b0       ??0?$CatmullRomSpline@MU?$SplineKey@M@spline@@$0A@@spline@@QAE@ABV01@@Z 315889b0 f i FaceEffector.obj
 0001:00087a50       ?Release@?$SSplineBackup@V?$CatmullRomSpline@MU?$SplineKey@M@spline@@$0A@@spline@@@spline@@UAEXXZ 31588a50 f i FaceEffector.obj
 0001:00087a70       ??_E?$SSplineBackup@V?$CatmullRomSpline@MU?$SplineKey@M@spline@@$0A@@spline@@@spline@@W3AEPAXI@Z 31588a70 f i FaceEffector.obj
 0001:00087a80       ??_G?$SSplineBackup@V?$CatmullRomSpline@MU?$SplineKey@M@spline@@$0A@@spline@@@spline@@UAEPAXI@Z 31588a80 f i FaceEffector.obj
 0001:00087a80       ??_E?$SSplineBackup@V?$CatmullRomSpline@MU?$SplineKey@M@spline@@$0A@@spline@@@spline@@UAEPAXI@Z 31588a80 f i FaceEffector.obj
 0001:00087ab0       ?Backup@?$CBaseSplineInterpolator@MV?$CatmullRomSpline@MU?$SplineKey@M@spline@@$0A@@spline@@@spline@@UAEPAUISplineBackup@@XZ 31588ab0 f i FaceEffector.obj
 0001:00087b00       ?Restore@?$CBaseSplineInterpolator@MV?$CatmullRomSpline@MU?$SplineKey@M@spline@@$0A@@spline@@@spline@@UAEXPAUISplineBackup@@@Z 31588b00 f i FaceEffector.obj
 0001:00087b70       ??0CFacialEffCtrlSplineInterpolator@@QAE@PAVCFacialEffCtrl@@@Z 31588b70 f i FaceEffector.obj
 0001:00087bd0       ??_ECFacialEffCtrlSplineInterpolator@@W3AEPAXI@Z 31588bd0 f i FaceEffector.obj
 0001:00087be0       ??_ECFacialEffCtrlSplineInterpolator@@UAEPAXI@Z 31588be0 f i FaceEffector.obj
 0001:00087be0       ??_GCFacialEffCtrlSplineInterpolator@@UAEPAXI@Z 31588be0 f i FaceEffector.obj
 0001:00087c10       ?SetType@CFacialEffCtrl@@UAEXW4ControlType@IFacialEffCtrl@@@Z 31588c10 f   FaceEffector.obj
 0001:00087d90       ?SetConstantWeight@CFacialEffCtrl@@UAEXM@Z 31588d90 f   FaceEffector.obj
 0001:00087e50       ??0CFacialEffCtrl@@QAE@XZ  31588e50 f   FaceEffector.obj
 0001:00087ed0       ?GetType@CFacialEffCtrl@@UAE?AW4ControlType@IFacialEffCtrl@@XZ 31588ed0 f i FaceEffector.obj
 0001:00087ed0       ?GetText@CFacialSentence@@UAEPBDXZ 31588ed0 f i LipSync.obj
 0001:00087ed0       ?GetFlags@CFacialAnimChannel@@UAEIXZ 31588ed0 f i FaceAnimSequence.obj
 0001:00087ed0       ?GetNameCRC@CAttachmentFACE@@UBEIXZ 31588ed0 f i AttachmentManager.obj
 0001:00087ed0       ?GetNameCRC@CAttachmentSKIN@@UBEIXZ 31588ed0 f i Attachment.obj
 0001:00087ed0       ?GetName@CFacialAnimSequence@@UAEPBDXZ 31588ed0 f i FaceAnimSequence.obj
 0001:00087ed0       ?GetNameCRC@CAttachmentBONE@@UBEIXZ 31588ed0 f i AttachmentManager.obj
 0001:00087ee0       ?GetConstantWeight@CFacialEffCtrl@@UAEMXZ 31588ee0 f i FaceEffector.obj
 0001:00087ee0       ?GetVideoMarkerOffset@CFacialJoystickChannel@@UBEMXZ 31588ee0 f i FaceJoystick.obj
 0001:00087ef0       ?SetFlags@CFacialEffCtrl@@UAEXH@Z 31588ef0 f i FaceEffector.obj
 0001:00087f00       ?GetAttachmentType@CCGFAttachment@@UAE?AW4EType@IAttachmentObject@@XZ 31588f00 f i AttachmentManager.obj
 0001:00087f00       ?GetNumDimensions@?$CBaseSplineInterpolator@MV?$HermitSplineEx@MU?$SplineKey@M@spline@@@spline@@@spline@@UAEHXZ 31588f00 f i FaceAnimSequence.obj
 0001:00087f00       ?GetType@CAttachmentFACE@@UBEIXZ 31588f00 f i AttachmentManager.obj
 0001:00087f00       ?GetSplineType@?$CBaseSplineInterpolator@MV?$HermitSplineEx@MU?$SplineKey@M@spline@@@spline@@@spline@@UAE?AW4ESplineType@@XZ 31588f00 f i FaceAnimSequence.obj
 0001:00087f00       ?GetType@CFacialEffectorExpression@@UAE?AW4EFacialEffectorType@@XZ 31588f00 f i FaceEffectorLibrary.obj
 0001:00087f00       ?GetNumDimensions@CFacialEffCtrlSplineInterpolator@@UAEHXZ 31588f00 f i FaceEffector.obj
 0001:00087f00       ?GetSplineType@?$CBaseSplineInterpolator@MV?$CatmullRomSpline@MU?$SplineKey@M@spline@@$0A@@spline@@@spline@@UAE?AW4ESplineType@@XZ 31588f00 f i FaceEffector.obj
 0001:00087f00       ?GetFormat@?$CKeyTimesInformation@GUUINT16Encoder@@@@UAEIXZ 31588f00 f i ControllerPQ.obj
 0001:00087f00       ?GetSplineType@CFacialEffCtrl@@UAE?AW4ESplineType@@XZ 31588f00 f i FaceEffector.obj
 0001:00087f00       ?GetNumDimensions@CFacialAnimChannelInterpolator@@UAEHXZ 31588f00 f i FaceAnimSequence.obj
 0001:00087f00       ?GetFormat@?$CTrackDataStorageInt@U?$Quat_tpl@M@@UNoCompressQuat@@VITrackRotationStorage@@@@UAEIXZ 31588f00 f i ControllerPQ.obj
 0001:00087f10       ?SerializeSpline@CFacialEffCtrl@@UAEXAAVXmlNodeRef@@_N@Z 31588f10 f i FaceEffector.obj
 0001:00087f30       ??_ECFacialEffCtrl@@W3AEPAXI@Z 31588f30 f i FaceEffector.obj
 0001:00087f40       ??_ECFacialEffCtrl@@UAEPAXI@Z 31588f40 f i FaceEffector.obj
 0001:00087f40       ??_GCFacialEffCtrl@@UAEPAXI@Z 31588f40 f i FaceEffector.obj
 0001:00087fa0       ?AddSubEffector@CFacialEffector@@UAEPAUIFacialEffCtrl@@PAUIFacialEffector@@@Z 31588fa0 f   FaceEffector.obj
 0001:00088020       ?interpolate@?$TSpline@U?$SplineKey@M@spline@@VHermitBasis@2@@spline@@QAE_NMAAM@Z 31589020 f i FaceAnimSequence.obj
 0001:00088020       ?interpolate@?$TSpline@U?$SplineKey@M@spline@@U?$TCoeffBasis@M@2@@spline@@QAE_NMAAM@Z 31589020 f i FaceEffector.obj
 0001:00088140       ?Evaluate@CFacialEffCtrl@@UAEMM@Z 31589140 f   FaceEffector.obj
 0001:00088190       ??_EIFacialEffectorsLibrary@@UAEPAXI@Z 31589190 f i FaceEffectorLibrary.obj
 0001:00088190       ??_EIFacialAnimation@@UAEPAXI@Z 31589190 f i FaceAnimation.obj
 0001:00088190       ??_GIFacialAnimation@@UAEPAXI@Z 31589190 f i FaceAnimation.obj
 0001:00088190       ??_EIJoystick@@UAEPAXI@Z   31589190 f i FaceJoystick.obj
 0001:00088190       ??_EIJoystickChannel@@UAEPAXI@Z 31589190 f i FaceJoystick.obj
 0001:00088190       ??_GIFacialEffectorsLibrary@@UAEPAXI@Z 31589190 f i FaceEffectorLibrary.obj
 0001:00088190       ??_GIJoystick@@UAEPAXI@Z   31589190 f i FaceJoystick.obj
 0001:00088190       ??_GIJoystickChannel@@UAEPAXI@Z 31589190 f i FaceJoystick.obj
 0001:000881c0       ?NameToEffectorType@@YA?AW4EFacialEffectorType@@PBD@Z 315891c0 f i FaceEffectorLibrary.obj
 0001:000884f0       ??$__copy_backward@PAV?$_smart_ptr@VCFacialEffector@@@@PAV1@H@priv@stlpmtx_std@@YAPAV?$_smart_ptr@VCFacialEffector@@@@PAV2@00ABUrandom_access_iterator_tag@1@PAH@Z 315894f0 f i FaceEffectorLibrary.obj
 0001:00088550       ??$__fill@PAV?$_smart_ptr@VCFacialEffector@@@@V1@H@priv@stlpmtx_std@@YAXPAV?$_smart_ptr@VCFacialEffector@@@@0ABV2@ABUrandom_access_iterator_tag@1@PAH@Z 31589550 f i FaceEffectorLibrary.obj
 0001:000885a0       ?Find@CFacialEffectorsLibrary@@UAEPAUIFacialEffector@@PBD@Z 315895a0 f   FaceEffectorLibrary.obj
 0001:000885e0       ?GetEffector@CFacialAnimChannel@@UAEPAUIFacialEffector@@XZ 315895e0 f   FaceAnimSequence.obj
 0001:000885e0       ?GetRoot@CFacialEffectorsLibrary@@UAEPAUIFacialEffector@@XZ 315895e0 f   FaceEffectorLibrary.obj
 0001:000885f0       ?CreateEffector@CFacialEffectorsLibrary@@UAEPAUIFacialEffector@@W4EFacialEffectorType@@PBD@Z 315895f0 f   FaceEffectorLibrary.obj
 0001:000886e0       ??F?$_Rb_tree_iterator@U?$pair@$$CBV?$CryStringT@D@@V?$_smart_ptr@UIFacialAnimSequence@@@@@stlpmtx_std@@U?$_MapTraitsT@U?$pair@$$CBV?$CryStringT@D@@V?$_smart_ptr@UIFacialAnimSequence@@@@@stlpmtx_std@@@priv@2@@priv@stlpmtx_std@@QAEAAU012@XZ 315896e0 f i FaceAnimation.obj
 0001:000886e0       ??F?$_Rb_tree_iterator@U?$pair@$$CBIUSFacialDisplaceInfo@CFacialModel@@@stlpmtx_std@@U?$_MapTraitsT@U?$pair@$$CBIUSFacialDisplaceInfo@CFacialModel@@@stlpmtx_std@@@priv@2@@priv@stlpmtx_std@@QAEAAU012@XZ 315896e0 f i FacialModel.obj
 0001:000886e0       ??F?$_Rb_tree_iterator@U?$pair@$$CBIPAV?$vector@IV?$allocator@I@stlpmtx_std@@@stlpmtx_std@@@stlpmtx_std@@U?$_MapTraitsT@U?$pair@$$CBIPAV?$vector@IV?$allocator@I@stlpmtx_std@@@stlpmtx_std@@@stlpmtx_std@@@priv@2@@priv@stlpmtx_std@@QAEAAU012@XZ 315896e0 f i AnimationManager.obj
 0001:000886e0       ??F?$_Rb_tree_iterator@U?$pair@QAUIFacialEffector@@PAU1@@stlpmtx_std@@U?$_MapTraitsT@U?$pair@QAUIFacialEffector@@PAU1@@stlpmtx_std@@@priv@2@@priv@stlpmtx_std@@QAEAAU012@XZ 315896e0 f i FaceEffectorLibrary.obj
 0001:000886e0       ??F?$_Rb_tree_iterator@U?$pair@$$CBIV?$_smart_ptr@VCFacialEffector@@@@@stlpmtx_std@@U?$_MapTraitsT@U?$pair@$$CBIV?$_smart_ptr@VCFacialEffector@@@@@stlpmtx_std@@@priv@2@@priv@stlpmtx_std@@QAEAAU012@XZ 315896e0 f i FaceEffectorLibrary.obj
 0001:000886e0       ??F?$_Rb_tree_iterator@U?$pair@$$CBIV?$CryStringT@D@@@stlpmtx_std@@U?$_MapTraitsT@U?$pair@$$CBIV?$CryStringT@D@@@stlpmtx_std@@@priv@2@@priv@stlpmtx_std@@QAEAAU012@XZ 315896e0 f i ModelAnimationSet.obj
 0001:000886e0       ??F?$_Rb_tree_iterator@U?$pair@$$CBIV?$_smart_ptr@UIPlaceholderCharacter@@@@@stlpmtx_std@@U?$_MapTraitsT@U?$pair@$$CBIV?$_smart_ptr@UIPlaceholderCharacter@@@@@stlpmtx_std@@@priv@2@@priv@stlpmtx_std@@QAEAAU012@XZ 315896e0 f i CharacterManager.obj
 0001:000886e0       ??F?$_Rb_tree_iterator@HU?$_SetTraitsT@H@priv@stlpmtx_std@@@priv@stlpmtx_std@@QAEAAU012@XZ 315896e0 f i LoaderCGA.obj
 0001:000886e0       ??F?$_Rb_tree_iterator@U?$pair@$$CBIPAV?$vector@HV?$allocator@H@stlpmtx_std@@@stlpmtx_std@@@stlpmtx_std@@U?$_MapTraitsT@U?$pair@$$CBIPAV?$vector@HV?$allocator@H@stlpmtx_std@@@stlpmtx_std@@@stlpmtx_std@@@priv@2@@priv@stlpmtx_std@@QAEAAU012@XZ 315896e0 f i AnimationManager.obj
 0001:000886e0       ??F?$_Rb_tree_iterator@V?$CryStringT@D@@U?$_SetTraitsT@V?$CryStringT@D@@@priv@stlpmtx_std@@@priv@stlpmtx_std@@QAEAAU012@XZ 315896e0 f i CharacterManager.obj
 0001:000886e0       ??F?$_Rb_tree_iterator@U?$pair@$$CBHPAUphys_geometry@@@stlpmtx_std@@U?$_MapTraitsT@U?$pair@$$CBHPAUphys_geometry@@@stlpmtx_std@@@priv@2@@priv@stlpmtx_std@@QAEAAU012@XZ 315896e0 f i LoaderCHR.obj
 0001:000886e0       ??F?$_Rb_tree_iterator@U?$pair@$$CBII@stlpmtx_std@@U?$_MapTraitsT@U?$pair@$$CBII@stlpmtx_std@@@priv@2@@priv@stlpmtx_std@@QAEAAU012@XZ 315896e0 f i CharacterManager.obj
 0001:000886e0       ??F?$_Rb_tree_iterator@U?$pair@$$CBIPAVCModelJoint@@@stlpmtx_std@@U?$_MapTraitsT@U?$pair@$$CBIPAVCModelJoint@@@stlpmtx_std@@@priv@2@@priv@stlpmtx_std@@QAEAAU012@XZ 315896e0 f i ModelSkeleton.obj
 0001:00088730       ??$AddObject@V?$_smart_ptr@VCFacialEffector@@@@V?$allocator@V?$_smart_ptr@VCFacialEffector@@@@@stlpmtx_std@@@ICrySizer@@QAEXABV?$vector@V?$_smart_ptr@VCFacialEffector@@@@V?$allocator@V?$_smart_ptr@VCFacialEffector@@@@@stlpmtx_std@@@stlpmtx_std@@@Z 31589730 f i FaceEffectorLibrary.obj
 0001:000887a0       ?VisitEffectors@CFacialEffectorsLibrary@@UAEXPAUIFacialEffectorsLibraryEffectorVisitor@@@Z 315897a0 f   FaceEffectorLibrary.obj
 0001:00088820       ?GetEffectorFromIndex@CFacialEffectorsLibrary@@QAEPAVCFacialEffector@@H@Z 31589820 f   FaceEffectorLibrary.obj
 0001:00088850       ?SerializeEffectorSubCtrls@CFacialEffectorsLibrary@@AAEXPAVCFacialEffector@@AAVXmlNodeRef@@_N@Z 31589850 f   FaceEffectorLibrary.obj
 0001:00088a70       ?_M_erase@?$_Rb_tree@IU?$less@I@stlpmtx_std@@U?$pair@$$CBIV?$_smart_ptr@VCFacialEffector@@@@@2@U?$_Select1st@U?$pair@$$CBIV?$_smart_ptr@VCFacialEffector@@@@@stlpmtx_std@@@priv@2@U?$_MapTraitsT@U?$pair@$$CBIV?$_smart_ptr@VCFacialEffector@@@@@stlpmtx_std@@@52@V?$allocator@U?$pair@$$CBIV?$_smart_ptr@VCFacialEffector@@@@@stlpmtx_std@@@2@@priv@stlpmtx_std@@AAEXPAU_Rb_tree_node_base@23@@Z 31589a70 f i FaceEffectorLibrary.obj
 0001:00088ac0       ??$AddObject@IV?$_smart_ptr@VCFacialEffector@@@@U?$less@I@stlpmtx_std@@V?$allocator@U?$pair@$$CBIV?$_smart_ptr@VCFacialEffector@@@@@stlpmtx_std@@@3@@ICrySizer@@QAEXABV?$map@IV?$_smart_ptr@VCFacialEffector@@@@U?$less@I@stlpmtx_std@@V?$allocator@U?$pair@$$CBIV?$_smart_ptr@VCFacialEffector@@@@@stlpmtx_std@@@3@@stlpmtx_std@@@Z 31589ac0 f i FaceEffectorLibrary.obj
 0001:00088b40       ??$find@I@?$_Rb_tree@IU?$less@I@stlpmtx_std@@U?$pair@$$CBIV?$_smart_ptr@VCFacialEffector@@@@@2@U?$_Select1st@U?$pair@$$CBIV?$_smart_ptr@VCFacialEffector@@@@@stlpmtx_std@@@priv@2@U?$_MapTraitsT@U?$pair@$$CBIV?$_smart_ptr@VCFacialEffector@@@@@stlpmtx_std@@@52@V?$allocator@U?$pair@$$CBIV?$_smart_ptr@VCFacialEffector@@@@@stlpmtx_std@@@2@@priv@stlpmtx_std@@QAE?AU?$_Rb_tree_iterator@U?$pair@$$CBIV?$_smart_ptr@VCFacialEffector@@@@@stlpmtx_std@@U?$_MapTraitsT@U?$pair@$$CBIV?$_smart_ptr@VCFacialEffector@@@@@stlpmtx_std@@@priv@2@@12@ABI@Z 31589b40 f i FaceEffectorLibrary.obj
 0001:00088b90       ?_M_create_node@?$_Rb_tree@IU?$less@I@stlpmtx_std@@U?$pair@$$CBIV?$_smart_ptr@VCFacialEffector@@@@@2@U?$_Select1st@U?$pair@$$CBIV?$_smart_ptr@VCFacialEffector@@@@@stlpmtx_std@@@priv@2@U?$_MapTraitsT@U?$pair@$$CBIV?$_smart_ptr@VCFacialEffector@@@@@stlpmtx_std@@@52@V?$allocator@U?$pair@$$CBIV?$_smart_ptr@VCFacialEffector@@@@@stlpmtx_std@@@2@@priv@stlpmtx_std@@IAEPAU_Rb_tree_node_base@23@ABU?$pair@$$CBIV?$_smart_ptr@VCFacialEffector@@@@@3@@Z 31589b90 f i FaceEffectorLibrary.obj
 0001:00088bf0       ?GetMemoryUsage@CFacialEffectorsLibrary@@QBEXPAVICrySizer@@@Z 31589bf0 f   FaceEffectorLibrary.obj
 0001:00088c60       ?erase@?$map@IV?$_smart_ptr@VCFacialEffector@@@@U?$less@I@stlpmtx_std@@V?$allocator@U?$pair@$$CBIV?$_smart_ptr@VCFacialEffector@@@@@stlpmtx_std@@@3@@stlpmtx_std@@QAEXU?$_Rb_tree_iterator@U?$pair@$$CBIV?$_smart_ptr@VCFacialEffector@@@@@stlpmtx_std@@U?$_MapTraitsT@U?$pair@$$CBIV?$_smart_ptr@VCFacialEffector@@@@@stlpmtx_std@@@priv@2@@priv@2@@Z 31589c60 f i FaceEffectorLibrary.obj
 0001:00088cb0       ?erase_unique@?$_Rb_tree@IU?$less@I@stlpmtx_std@@U?$pair@$$CBIV?$_smart_ptr@VCFacialEffector@@@@@2@U?$_Select1st@U?$pair@$$CBIV?$_smart_ptr@VCFacialEffector@@@@@stlpmtx_std@@@priv@2@U?$_MapTraitsT@U?$pair@$$CBIV?$_smart_ptr@VCFacialEffector@@@@@stlpmtx_std@@@52@V?$allocator@U?$pair@$$CBIV?$_smart_ptr@VCFacialEffector@@@@@stlpmtx_std@@@2@@priv@stlpmtx_std@@QAEIABI@Z 31589cb0 f i FaceEffectorLibrary.obj
 0001:00088d20       ?_M_fill_insert_aux@?$_Impl_vector@V?$_smart_ptr@VCFacialEffector@@@@V?$allocator@V?$_smart_ptr@VCFacialEffector@@@@@stlpmtx_std@@@priv@stlpmtx_std@@AAEXPAV?$_smart_ptr@VCFacialEffector@@@@IABV4@ABU__false_type@3@@Z 31589d20 f i FaceEffectorLibrary.obj
 0001:00088e50       ?_M_insert@?$_Rb_tree@PAUIFacialEffector@@U?$less@PAUIFacialEffector@@@stlpmtx_std@@U?$pair@QAUIFacialEffector@@PAU1@@3@U?$_Select1st@U?$pair@QAUIFacialEffector@@PAU1@@stlpmtx_std@@@priv@3@U?$_MapTraitsT@U?$pair@QAUIFacialEffector@@PAU1@@stlpmtx_std@@@63@V?$allocator@U?$pair@QAUIFacialEffector@@PAU1@@stlpmtx_std@@@3@@priv@stlpmtx_std@@AAE?AU?$_Rb_tree_iterator@U?$pair@QAUIFacialEffector@@PAU1@@stlpmtx_std@@U?$_MapTraitsT@U?$pair@QAUIFacialEffector@@PAU1@@stlpmtx_std@@@priv@2@@23@PAU_Rb_tree_node_base@23@ABU?$pair@QAUIFacialEffector@@PAU1@@3@00@Z 31589e50 f i FaceEffectorLibrary.obj
 0001:00088e50       ?_M_insert@?$_Rb_tree@IU?$less@I@stlpmtx_std@@U?$pair@$$CBII@2@U?$_Select1st@U?$pair@$$CBII@stlpmtx_std@@@priv@2@U?$_MapTraitsT@U?$pair@$$CBII@stlpmtx_std@@@52@V?$allocator@U?$pair@$$CBII@stlpmtx_std@@@2@@priv@stlpmtx_std@@AAE?AU?$_Rb_tree_iterator@U?$pair@$$CBII@stlpmtx_std@@U?$_MapTraitsT@U?$pair@$$CBII@stlpmtx_std@@@priv@2@@23@PAU_Rb_tree_node_base@23@ABU?$pair@$$CBII@3@00@Z 31589e50 f i CharacterManager.obj
 0001:00088e50       ?_M_insert@?$_Rb_tree@IU?$less@I@stlpmtx_std@@U?$pair@$$CBIPAV?$vector@IV?$allocator@I@stlpmtx_std@@@stlpmtx_std@@@2@U?$_Select1st@U?$pair@$$CBIPAV?$vector@IV?$allocator@I@stlpmtx_std@@@stlpmtx_std@@@stlpmtx_std@@@priv@2@U?$_MapTraitsT@U?$pair@$$CBIPAV?$vector@IV?$allocator@I@stlpmtx_std@@@stlpmtx_std@@@stlpmtx_std@@@52@V?$allocator@U?$pair@$$CBIPAV?$vector@IV?$allocator@I@stlpmtx_std@@@stlpmtx_std@@@stlpmtx_std@@@2@@priv@stlpmtx_std@@AAE?AU?$_Rb_tree_iterator@U?$pair@$$CBIPAV?$vector@IV?$allocator@I@stlpmtx_std@@@stlpmtx_std@@@stlpmtx_std@@U?$_MapTraitsT@U?$pair@$$CBIPAV?$vector@IV?$allocator@I@stlpmtx_std@@@stlpmtx_std@@@stlpmtx_std@@@priv@2@@23@PAU_Rb_tree_node_base@23@ABU?$pair@$$CBIPAV?$vector@IV?$allocator@I@stlpmtx_std@@@stlpmtx_std@@@3@00@Z 31589e50 f i AnimationManager.obj
 0001:00088e50       ?_M_insert@?$_Rb_tree@IU?$less@I@stlpmtx_std@@U?$pair@$$CBIPAV?$vector@HV?$allocator@H@stlpmtx_std@@@stlpmtx_std@@@2@U?$_Select1st@U?$pair@$$CBIPAV?$vector@HV?$allocator@H@stlpmtx_std@@@stlpmtx_std@@@stlpmtx_std@@@priv@2@U?$_MapTraitsT@U?$pair@$$CBIPAV?$vector@HV?$allocator@H@stlpmtx_std@@@stlpmtx_std@@@stlpmtx_std@@@52@V?$allocator@U?$pair@$$CBIPAV?$vector@HV?$allocator@H@stlpmtx_std@@@stlpmtx_std@@@stlpmtx_std@@@2@@priv@stlpmtx_std@@AAE?AU?$_Rb_tree_iterator@U?$pair@$$CBIPAV?$vector@HV?$allocator@H@stlpmtx_std@@@stlpmtx_std@@@stlpmtx_std@@U?$_MapTraitsT@U?$pair@$$CBIPAV?$vector@HV?$allocator@H@stlpmtx_std@@@stlpmtx_std@@@stlpmtx_std@@@priv@2@@23@PAU_Rb_tree_node_base@23@ABU?$pair@$$CBIPAV?$vector@HV?$allocator@H@stlpmtx_std@@@stlpmtx_std@@@3@00@Z 31589e50 f i AnimationManager.obj
 0001:00088e50       ?_M_insert@?$_Rb_tree@IU?$less@I@stlpmtx_std@@U?$pair@$$CBIPAVCModelJoint@@@2@U?$_Select1st@U?$pair@$$CBIPAVCModelJoint@@@stlpmtx_std@@@priv@2@U?$_MapTraitsT@U?$pair@$$CBIPAVCModelJoint@@@stlpmtx_std@@@52@V?$allocator@U?$pair@$$CBIPAVCModelJoint@@@stlpmtx_std@@@2@@priv@stlpmtx_std@@AAE?AU?$_Rb_tree_iterator@U?$pair@$$CBIPAVCModelJoint@@@stlpmtx_std@@U?$_MapTraitsT@U?$pair@$$CBIPAVCModelJoint@@@stlpmtx_std@@@priv@2@@23@PAU_Rb_tree_node_base@23@ABU?$pair@$$CBIPAVCModelJoint@@@3@00@Z 31589e50 f i ModelSkeleton.obj
 0001:00088f10       ?_M_insert@?$_Rb_tree@IU?$less@I@stlpmtx_std@@U?$pair@$$CBIV?$_smart_ptr@VCFacialEffector@@@@@2@U?$_Select1st@U?$pair@$$CBIV?$_smart_ptr@VCFacialEffector@@@@@stlpmtx_std@@@priv@2@U?$_MapTraitsT@U?$pair@$$CBIV?$_smart_ptr@VCFacialEffector@@@@@stlpmtx_std@@@52@V?$allocator@U?$pair@$$CBIV?$_smart_ptr@VCFacialEffector@@@@@stlpmtx_std@@@2@@priv@stlpmtx_std@@AAE?AU?$_Rb_tree_iterator@U?$pair@$$CBIV?$_smart_ptr@VCFacialEffector@@@@@stlpmtx_std@@U?$_MapTraitsT@U?$pair@$$CBIV?$_smart_ptr@VCFacialEffector@@@@@stlpmtx_std@@@priv@2@@23@PAU_Rb_tree_node_base@23@ABU?$pair@$$CBIV?$_smart_ptr@VCFacialEffector@@@@@3@00@Z 31589f10 f i FaceEffectorLibrary.obj
 0001:00088fa0       ?insert_unique@?$_Rb_tree@IU?$less@I@stlpmtx_std@@U?$pair@$$CBIV?$_smart_ptr@VCFacialEffector@@@@@2@U?$_Select1st@U?$pair@$$CBIV?$_smart_ptr@VCFacialEffector@@@@@stlpmtx_std@@@priv@2@U?$_MapTraitsT@U?$pair@$$CBIV?$_smart_ptr@VCFacialEffector@@@@@stlpmtx_std@@@52@V?$allocator@U?$pair@$$CBIV?$_smart_ptr@VCFacialEffector@@@@@stlpmtx_std@@@2@@priv@stlpmtx_std@@QAE?AU?$pair@U?$_Rb_tree_iterator@U?$pair@$$CBIV?$_smart_ptr@VCFacialEffector@@@@@stlpmtx_std@@U?$_MapTraitsT@U?$pair@$$CBIV?$_smart_ptr@VCFacialEffector@@@@@stlpmtx_std@@@priv@2@@priv@stlpmtx_std@@_N@3@ABU?$pair@$$CBIV?$_smart_ptr@VCFacialEffector@@@@@3@@Z 31589fa0 f i FaceEffectorLibrary.obj
 0001:000890b0       ?Find@CFacialEffectorsLibrary@@UAEPAUIFacialEffector@@VCFaceIdentifierHandle@@@Z 3158a0b0 f   FaceEffectorLibrary.obj
 0001:00089110       ?RemoveEffector@CFacialEffectorsLibrary@@UAEXPAUIFacialEffector@@@Z 3158a110 f   FaceEffectorLibrary.obj
 0001:00089220       ?ReplaceEffector@CFacialEffectorsLibrary@@AAEXPAVCFacialEffector@@0@Z 3158a220 f   FaceEffectorLibrary.obj
 0001:00089340       ?insert_unique@?$_Rb_tree@IU?$less@I@stlpmtx_std@@U?$pair@$$CBIPAV?$vector@HV?$allocator@H@stlpmtx_std@@@stlpmtx_std@@@2@U?$_Select1st@U?$pair@$$CBIPAV?$vector@HV?$allocator@H@stlpmtx_std@@@stlpmtx_std@@@stlpmtx_std@@@priv@2@U?$_MapTraitsT@U?$pair@$$CBIPAV?$vector@HV?$allocator@H@stlpmtx_std@@@stlpmtx_std@@@stlpmtx_std@@@52@V?$allocator@U?$pair@$$CBIPAV?$vector@HV?$allocator@H@stlpmtx_std@@@stlpmtx_std@@@stlpmtx_std@@@2@@priv@stlpmtx_std@@QAE?AU?$pair@U?$_Rb_tree_iterator@U?$pair@$$CBIPAV?$vector@HV?$allocator@H@stlpmtx_std@@@stlpmtx_std@@@stlpmtx_std@@U?$_MapTraitsT@U?$pair@$$CBIPAV?$vector@HV?$allocator@H@stlpmtx_std@@@stlpmtx_std@@@stlpmtx_std@@@priv@2@@priv@stlpmtx_std@@_N@3@ABU?$pair@$$CBIPAV?$vector@HV?$allocator@H@stlpmtx_std@@@stlpmtx_std@@@3@@Z 3158a340 f i AnimationManager.obj
 0001:00089340       ?insert_unique@?$_Rb_tree@IU?$less@I@stlpmtx_std@@U?$pair@$$CBIPAVCModelJoint@@@2@U?$_Select1st@U?$pair@$$CBIPAVCModelJoint@@@stlpmtx_std@@@priv@2@U?$_MapTraitsT@U?$pair@$$CBIPAVCModelJoint@@@stlpmtx_std@@@52@V?$allocator@U?$pair@$$CBIPAVCModelJoint@@@stlpmtx_std@@@2@@priv@stlpmtx_std@@QAE?AU?$pair@U?$_Rb_tree_iterator@U?$pair@$$CBIPAVCModelJoint@@@stlpmtx_std@@U?$_MapTraitsT@U?$pair@$$CBIPAVCModelJoint@@@stlpmtx_std@@@priv@2@@priv@stlpmtx_std@@_N@3@ABU?$pair@$$CBIPAVCModelJoint@@@3@@Z 3158a340 f i ModelSkeleton.obj
 0001:00089340       ?insert_unique@?$_Rb_tree@IU?$less@I@stlpmtx_std@@U?$pair@$$CBIPAV?$vector@IV?$allocator@I@stlpmtx_std@@@stlpmtx_std@@@2@U?$_Select1st@U?$pair@$$CBIPAV?$vector@IV?$allocator@I@stlpmtx_std@@@stlpmtx_std@@@stlpmtx_std@@@priv@2@U?$_MapTraitsT@U?$pair@$$CBIPAV?$vector@IV?$allocator@I@stlpmtx_std@@@stlpmtx_std@@@stlpmtx_std@@@52@V?$allocator@U?$pair@$$CBIPAV?$vector@IV?$allocator@I@stlpmtx_std@@@stlpmtx_std@@@stlpmtx_std@@@2@@priv@stlpmtx_std@@QAE?AU?$pair@U?$_Rb_tree_iterator@U?$pair@$$CBIPAV?$vector@IV?$allocator@I@stlpmtx_std@@@stlpmtx_std@@@stlpmtx_std@@U?$_MapTraitsT@U?$pair@$$CBIPAV?$vector@IV?$allocator@I@stlpmtx_std@@@stlpmtx_std@@@stlpmtx_std@@@priv@2@@priv@stlpmtx_std@@_N@3@ABU?$pair@$$CBIPAV?$vector@IV?$allocator@I@stlpmtx_std@@@stlpmtx_std@@@3@@Z 3158a340 f i AnimationManager.obj
 0001:00089340       ?insert_unique@?$_Rb_tree@IU?$less@I@stlpmtx_std@@U?$pair@$$CBII@2@U?$_Select1st@U?$pair@$$CBII@stlpmtx_std@@@priv@2@U?$_MapTraitsT@U?$pair@$$CBII@stlpmtx_std@@@52@V?$allocator@U?$pair@$$CBII@stlpmtx_std@@@2@@priv@stlpmtx_std@@QAE?AU?$pair@U?$_Rb_tree_iterator@U?$pair@$$CBII@stlpmtx_std@@U?$_MapTraitsT@U?$pair@$$CBII@stlpmtx_std@@@priv@2@@priv@stlpmtx_std@@_N@3@ABU?$pair@$$CBII@3@@Z 3158a340 f i CharacterManager.obj
 0001:00089340       ?insert_unique@?$_Rb_tree@PAUIFacialEffector@@U?$less@PAUIFacialEffector@@@stlpmtx_std@@U?$pair@QAUIFacialEffector@@PAU1@@3@U?$_Select1st@U?$pair@QAUIFacialEffector@@PAU1@@stlpmtx_std@@@priv@3@U?$_MapTraitsT@U?$pair@QAUIFacialEffector@@PAU1@@stlpmtx_std@@@63@V?$allocator@U?$pair@QAUIFacialEffector@@PAU1@@stlpmtx_std@@@3@@priv@stlpmtx_std@@QAE?AU?$pair@U?$_Rb_tree_iterator@U?$pair@QAUIFacialEffector@@PAU1@@stlpmtx_std@@U?$_MapTraitsT@U?$pair@QAUIFacialEffector@@PAU1@@stlpmtx_std@@@priv@2@@priv@stlpmtx_std@@_N@3@ABU?$pair@QAUIFacialEffector@@PAU1@@3@@Z 3158a340 f i FaceEffectorLibrary.obj
 0001:00089400       ?_M_clear@?$_Impl_vector@V?$_smart_ptr@VCFacialEffector@@@@V?$allocator@V?$_smart_ptr@VCFacialEffector@@@@@stlpmtx_std@@@priv@stlpmtx_std@@AAEXXZ 3158a400 f i FaceEffectorLibrary.obj
 0001:00089440       ?insert_unique@?$_Rb_tree@IU?$less@I@stlpmtx_std@@U?$pair@$$CBIV?$_smart_ptr@VCFacialEffector@@@@@2@U?$_Select1st@U?$pair@$$CBIV?$_smart_ptr@VCFacialEffector@@@@@stlpmtx_std@@@priv@2@U?$_MapTraitsT@U?$pair@$$CBIV?$_smart_ptr@VCFacialEffector@@@@@stlpmtx_std@@@52@V?$allocator@U?$pair@$$CBIV?$_smart_ptr@VCFacialEffector@@@@@stlpmtx_std@@@2@@priv@stlpmtx_std@@QAE?AU?$_Rb_tree_iterator@U?$pair@$$CBIV?$_smart_ptr@VCFacialEffector@@@@@stlpmtx_std@@U?$_MapTraitsT@U?$pair@$$CBIV?$_smart_ptr@VCFacialEffector@@@@@stlpmtx_std@@@priv@2@@23@U423@ABU?$pair@$$CBIV?$_smart_ptr@VCFacialEffector@@@@@3@@Z 3158a440 f i FaceEffectorLibrary.obj
 0001:00089630       ??$_M_allocate_and_copy@PAV?$_smart_ptr@VCFacialEffector@@@@@?$_Impl_vector@V?$_smart_ptr@VCFacialEffector@@@@V?$allocator@V?$_smart_ptr@VCFacialEffector@@@@@stlpmtx_std@@@priv@stlpmtx_std@@AAEPAV?$_smart_ptr@VCFacialEffector@@@@AAIPAV3@1@Z 3158a630 f i FaceEffectorLibrary.obj
 0001:000896c0       ??1?$_Impl_vector@V?$_smart_ptr@VCFacialEffCtrl@@@@V?$allocator@V?$_smart_ptr@VCFacialEffCtrl@@@@@stlpmtx_std@@@priv@stlpmtx_std@@QAE@XZ 3158a6c0 f i FaceEffector.obj
 0001:000896c0       ??1?$_Impl_vector@V?$_smart_ptr@VCFacialAnimChannel@@@@V?$allocator@V?$_smart_ptr@VCFacialAnimChannel@@@@@stlpmtx_std@@@priv@stlpmtx_std@@QAE@XZ 3158a6c0 f i FaceAnimSequence.obj
 0001:000896c0       ??1?$_Impl_vector@V?$_smart_ptr@VCFacialEffector@@@@V?$allocator@V?$_smart_ptr@VCFacialEffector@@@@@stlpmtx_std@@@priv@stlpmtx_std@@QAE@XZ 3158a6c0 f i FaceEffectorLibrary.obj
 0001:00089710       ??1CFacialEffectorsLibrary@@UAE@XZ 3158a710 f   FaceEffectorLibrary.obj
 0001:000897b0       ?AddRef@CFacialEffectorsLibrary@@UAEXXZ 3158a7b0 f i FaceEffectorLibrary.obj
 0001:000897b0       ?AddRef@CPlaceholderCharacter@@UAEXXZ 3158a7b0 f i PlaceholderCharacter.obj
 0001:000897b0       ?AddRef@?$_i_reference_target@H@@UAEXXZ 3158a7b0 f i LoaderSKIN.obj
 0001:000897c0       ?Release@CFacialEffectorsLibrary@@UAEXXZ 3158a7c0 f i FaceEffectorLibrary.obj
 0001:000897e0       ?SetSoundFile@CFacialAnimSoundEntry@@UAEXPBD@Z 3158a7e0 f i FaceAnimSequence.obj
 0001:000897e0       ?SetName@CFacialEffectorsLibrary@@UAEXPBD@Z 3158a7e0 f i FaceEffectorLibrary.obj
 0001:00089b30       ??$?AI@?$map@IV?$_smart_ptr@VCFacialEffector@@@@U?$less@I@stlpmtx_std@@V?$allocator@U?$pair@$$CBIV?$_smart_ptr@VCFacialEffector@@@@@stlpmtx_std@@@3@@stlpmtx_std@@QAEAAV?$_smart_ptr@VCFacialEffector@@@@ABI@Z 3158ab30 f i FaceEffectorLibrary.obj
 0001:00089bb0       ??0CFacialMorphTarget@@QAE@I@Z 3158abb0 f i FaceEffectorLibrary.obj
 0001:00089c30       ??_ECFacialEffectorsLibrary@@UAEPAXI@Z 3158ac30 f i FaceEffectorLibrary.obj
 0001:00089c30       ??_GCFacialEffectorsLibrary@@UAEPAXI@Z 3158ac30 f i FaceEffectorLibrary.obj
 0001:00089c60       ?NewRoot@CFacialEffectorsLibrary@@AAEXXZ 3158ac60 f   FaceEffectorLibrary.obj
 0001:00089d40       ??0CFacialEffectorExpression@@QAE@XZ 3158ad40 f i FaceEffectorLibrary.obj
 0001:00089db0       ??0CFacialEffectorBone@@QAE@XZ 3158adb0 f i FaceEffectorLibrary.obj
 0001:00089dd0       ??_ECFacialEffectorBone@@W3AEPAXI@Z 3158add0 f i FaceEffectorLibrary.obj
 0001:00089dd0       ??_ECFacialEffectorAttachment@@W3AEPAXI@Z 3158add0 f i FaceEffector.obj
 0001:00089de0       ??_ECFacialEffectorAttachment@@UAEPAXI@Z 3158ade0 f i FaceEffector.obj
 0001:00089de0       ??_GCFacialEffectorBone@@UAEPAXI@Z 3158ade0 f i FaceEffectorLibrary.obj
 0001:00089de0       ??_GCFacialEffectorAttachment@@UAEPAXI@Z 3158ade0 f i FaceEffector.obj
 0001:00089de0       ??_ECFacialEffectorBone@@UAEPAXI@Z 3158ade0 f i FaceEffectorLibrary.obj
 0001:00089e10       ?RenameEffector@CFacialEffectorsLibrary@@QAEXPAVCFacialEffector@@VCFaceIdentifierHandle@@@Z 3158ae10 f   FaceEffectorLibrary.obj
 0001:00089ed0       ?SerializeEffectorSelf@CFacialEffectorsLibrary@@AAEXPAVCFacialEffector@@AAVXmlNodeRef@@_N@Z 3158aed0 f   FaceEffectorLibrary.obj
 0001:0008a040       ?SerializeEffector@CFacialEffectorsLibrary@@UAEXPAUIFacialEffector@@AAVXmlNodeRef@@_N@Z 3158b040 f   FaceEffectorLibrary.obj
 0001:0008a070       ??0CFacialEffectorsLibrary@@QAE@PAVCFacialAnimation@@@Z 3158b070 f   FaceEffectorLibrary.obj
 0001:0008a170       ?MergeLibrary@CFacialEffectorsLibrary@@UAEXPAUIFacialEffectorsLibrary@@ABV?$Functor1wRet@PBDW4MergeCollisionAction@@@@@Z 3158b170 f   FaceEffectorLibrary.obj
 0001:0008a220       ?Serialize@CFacialEffectorsLibrary@@UAEXAAVXmlNodeRef@@_N@Z 3158b220 f   FaceEffectorLibrary.obj
 0001:0008a660       ?resize@?$_Impl_vector@V?$_smart_ptr@VCFacialEffector@@@@V?$allocator@V?$_smart_ptr@VCFacialEffector@@@@@stlpmtx_std@@@priv@stlpmtx_std@@QAEXIABV?$_smart_ptr@VCFacialEffector@@@@@Z 3158b660 f i FaceEffectorLibrary.obj
 0001:0008a6e0       ?SetEffectorIndex@CFacialEffectorsLibrary@@AAEXPAVCFacialEffector@@@Z 3158b6e0 f   FaceEffectorLibrary.obj
 0001:0008a740       ?CreateEffector@CFacialEffectorsLibrary@@UAEPAUIFacialEffector@@W4EFacialEffectorType@@VCFaceIdentifierHandle@@@Z 3158b740 f   FaceEffectorLibrary.obj
 0001:0008a890       ??_EIFacialEffCtrl@@UAEPAXI@Z 3158b890 f i FaceEffector.obj
 0001:0008a890       ??_GIJoystickSet@@UAEPAXI@Z 3158b890 f i FaceJoystick.obj
 0001:0008a890       ??_EIJoystickSet@@UAEPAXI@Z 3158b890 f i FaceJoystick.obj
 0001:0008a890       ??_GIFacialEffCtrl@@UAEPAXI@Z 3158b890 f i FaceEffector.obj
 0001:0008a8c0       ?AddRef@CFacialJoystickChannel@@UAEXXZ 3158b8c0 f   FaceJoystick.obj
 0001:0008a8d0       ?Release@CFacialJoystickChannel@@UAEXXZ 3158b8d0 f   FaceJoystick.obj
 0001:0008a8f0       ?GetName@CFacialJoystickChannel@@UBEPBDXZ 3158b8f0 f   FaceJoystick.obj
 0001:0008a920       ?GetSplineCount@CFacialJoystickChannel@@UAEHXZ 3158b920 f   FaceJoystick.obj
 0001:0008a940       ?GetSpline@CFacialJoystickChannel@@UAEPAUISplineInterpolator@@H@Z 3158b940 f   FaceJoystick.obj
 0001:0008a980       ?SetFlipped@CFacialJoystickChannel@@UAEX_N@Z 3158b980 f   FaceJoystick.obj
 0001:0008a990       ?GetFlipped@CFacialJoystickChannel@@UBE_NXZ 3158b990 f   FaceJoystick.obj
 0001:0008a9a0       ?GetVideoMarkerScale@CFacialJoystickChannel@@UBEMXZ 3158b9a0 f   FaceJoystick.obj
 0001:0008a9a0       ?GetConstantBalance@CFacialEffCtrl@@UAEMXZ 3158b9a0 f   FaceEffector.obj
 0001:0008a9b0       ?CleanupKeys@CFacialJoystickChannel@@UAEXM@Z 3158b9b0 f   FaceJoystick.obj
 0001:0008a9d0       ?AddRef@CFacialJoystick@@UAEXXZ 3158b9d0 f   FaceJoystick.obj
 0001:0008a9e0       ?Release@CFacialJoystick@@UAEXXZ 3158b9e0 f   FaceJoystick.obj
 0001:0008aa00       ?GetID@CFacialJoystick@@UBE_KXZ 3158ba00 f   FaceJoystick.obj
 0001:0008aa10       ?GetCentre@CFacialJoystick@@UBEABU?$Vec2_tpl@M@@XZ 3158ba10 f   FaceJoystick.obj
 0001:0008aa20       ?GetDimensions@CFacialJoystick@@UBEABU?$Vec2_tpl@M@@XZ 3158ba20 f   FaceJoystick.obj
 0001:0008aa30       ?SetColor@CFacialJoystick@@UAEXABU?$Vec3_tpl@E@@@Z 3158ba30 f   FaceJoystick.obj
 0001:0008aa50       ?GetColor@CFacialJoystick@@UBE?AU?$Vec3_tpl@E@@XZ 3158ba50 f   FaceJoystick.obj
 0001:0008aa70       ?Release@CFacialJoystickSet@@UAEXXZ 3158ba70 f   FaceJoystick.obj
 0001:0008aa90       ??_9CFacialJoystick@@$BCA@AE 3158ba90 f i FaceJoystick.obj
 0001:0008aaa0       ??_9CFacialJoystick@@$BCE@AE 3158baa0 f i FaceJoystick.obj
 0001:0008aab0       ??_9CFacialJoystick@@$BCI@AE 3158bab0 f i FaceJoystick.obj
 0001:0008aac0       ??_9CFacialJoystick@@$BCM@AE 3158bac0 f i FaceJoystick.obj
 0001:0008aad0       ?GetChannel@CFacialJoystick@@UAEPAVIJoystickChannel@@W4ChannelType@IJoystick@@@Z 3158bad0 f   FaceJoystick.obj
 0001:0008aaf0       ?SetChannel@CFacialJoystick@@UAEXW4ChannelType@IJoystick@@PAVIJoystickChannel@@@Z 3158baf0 f   FaceJoystick.obj
 0001:0008ab30       ?SetCentre@CFacialJoystick@@UAEXABU?$Vec2_tpl@M@@@Z 3158bb30 f   FaceJoystick.obj
 0001:0008ab50       ?SetDimensions@CFacialJoystick@@UAEXABU?$Vec2_tpl@M@@@Z 3158bb50 f   FaceJoystick.obj
 0001:0008ab70       ??$remove_copy@PAV?$_smart_ptr@VCFacialJoystick@@@@PAV1@PAVIJoystick@@@stlpmtx_std@@YAPAV?$_smart_ptr@VCFacialJoystick@@@@PAV1@00ABQAVIJoystick@@@Z 3158bb70 f i FaceJoystick.obj
 0001:0008abc0       ??$__copy@PAV?$_smart_ptr@VCFacialJoystick@@@@PAV1@H@priv@stlpmtx_std@@YAPAV?$_smart_ptr@VCFacialJoystick@@@@PAV2@00ABUrandom_access_iterator_tag@1@PAH@Z 3158bbc0 f i FaceJoystick.obj
 0001:0008ac20       ?GetJoystickCount@CFacialJoystickSet@@UBEHXZ 3158bc20 f   FaceJoystick.obj
 0001:0008ac30       ?GetJoystick@CFacialJoystickSet@@UAEPAVIJoystick@@H@Z 3158bc30 f   FaceJoystick.obj
 0001:0008ac40       ?GetJoystickAtPoint@CFacialJoystickSet@@UAEPAVIJoystick@@ABU?$Vec2_tpl@M@@@Z 3158bc40 f   FaceJoystick.obj
 0001:0008acd0       ?GetJoystickByID@CFacialJoystickSet@@UAEPAVIJoystick@@_K@Z 3158bcd0 f   FaceJoystick.obj
 0001:0008ad20       ?Bind@CFacialJoystickSet@@QAEXPAVIFacialJoystickSerializeContext@@@Z 3158bd20 f   FaceJoystick.obj
 0001:0008ada0       ??0CFacialJoystickChannel@@QAE@ABV?$CryStringT@D@@@Z 3158bda0 f   FaceJoystick.obj
 0001:0008adf0       ??0CFacialJoystick@@QAE@_K@Z 3158bdf0 f   FaceJoystick.obj
 0001:0008ae30       ??1CFacialJoystick@@UAE@XZ 3158be30 f i FaceJoystick.obj
 0001:0008ae90       ??$__uninitialized_fill_n@PAV?$_smart_ptr@VCFacialJoystick@@@@IV1@@priv@stlpmtx_std@@YAPAV?$_smart_ptr@VCFacialJoystick@@@@PAV2@IABV2@@Z 3158be90 f i FaceJoystick.obj
 0001:0008aee0       ??_ECFacialJoystickChannel@@UAEPAXI@Z 3158bee0 f i FaceJoystick.obj
 0001:0008aee0       ??_GCFacialJoystickChannel@@UAEPAXI@Z 3158bee0 f i FaceJoystick.obj
 0001:0008af30       ??_ECFacialJoystick@@UAEPAXI@Z 3158bf30 f i FaceJoystick.obj
 0001:0008af30       ??_GCFacialJoystick@@UAEPAXI@Z 3158bf30 f i FaceJoystick.obj
 0001:0008af60       ?SetName@CFacialJoystick@@UAEXPBD@Z 3158bf60 f   FaceJoystick.obj
 0001:0008afa0       ?SetName@CFacialJoystickSet@@UAEXPBD@Z 3158bfa0 f   FaceJoystick.obj
 0001:0008afe0       ?_M_erase@?$_Impl_vector@V?$_smart_ptr@VCFacialJoystick@@@@V?$allocator@V?$_smart_ptr@VCFacialJoystick@@@@@stlpmtx_std@@@priv@stlpmtx_std@@AAEPAV?$_smart_ptr@VCFacialJoystick@@@@PAV4@0ABU__false_type@3@@Z 3158bfe0 f i FaceJoystick.obj
 0001:0008b050       ??0CFacialJoystickChannel@@QAE@PAUIFacialAnimChannel@@@Z 3158c050 f   FaceJoystick.obj
 0001:0008b330       ?RemoveJoystick@CFacialJoystickSet@@UAEXPAVIJoystick@@@Z 3158c330 f   FaceJoystick.obj
 0001:0008b3c0       ??1?$_Impl_vector@V?$_smart_ptr@VCFacialJoystick@@@@V?$allocator@V?$_smart_ptr@VCFacialJoystick@@@@@stlpmtx_std@@@priv@stlpmtx_std@@QAE@XZ 3158c3c0 f i FaceJoystick.obj
 0001:0008b410       ?_M_insert_overflow_aux@?$_Impl_vector@V?$_smart_ptr@VCFacialJoystick@@@@V?$allocator@V?$_smart_ptr@VCFacialJoystick@@@@@stlpmtx_std@@@priv@stlpmtx_std@@AAEXPAV?$_smart_ptr@VCFacialJoystick@@@@ABV4@ABU__false_type@3@I_N@Z 3158c410 f i FaceJoystick.obj
 0001:0008b5f0       ??0CFacialJoystickSet@@QAE@XZ 3158c5f0 f   FaceJoystick.obj
 0001:0008b640       ??_GCFacialJoystickSet@@UAEPAXI@Z 3158c640 f i FaceJoystick.obj
 0001:0008b640       ??_ECFacialJoystickSet@@UAEPAXI@Z 3158c640 f i FaceJoystick.obj
 0001:0008b6a0       ?AddJoystick@CFacialJoystickSet@@UAEXPAVIJoystick@@@Z 3158c6a0 f   FaceJoystick.obj
 0001:0008b720       ?Serialize@CFacialJoystickSet@@UAEXAAVXmlNodeRef@@_N@Z 3158c720 f   FaceJoystick.obj
 0001:0008c0c0       ?Reset@CFaceState@@QAEXXZ  3158d0c0 f   FaceState.obj
 0001:0008c110       ?SetNumWeights@CFaceState@@QAEXH@Z 3158d110 f   FaceState.obj
 0001:0008c190       ?LoadSequence@CFacialInstance@@UAEPAUIFacialAnimSequence@@PBD_N@Z 3158d190 f   FacialInstance.obj
 0001:0008c280       ?PrecacheFacialExpressionCallback@@YAXPAXPBD@Z 3158d280 f   FacialInstance.obj
 0001:0008c2b0       ?PrecacheFacialExpression@CFacialInstance@@UAEXPBD@Z 3158d2b0 f   FacialInstance.obj
 0001:0008c350       ?EnableProceduralFacialAnimation@CFacialInstance@@UAEX_N@Z 3158d350 f   FacialInstance.obj
 0001:0008c360       ?SetMasterCharacter@CFacialInstance@@UAEXPAUICharacterInstance@@@Z 3158d360 f   FacialInstance.obj
 0001:0008c370       ?GetFacialModel@CFacialInstance@@UAEPAUIFacialModel@@XZ 3158d370 f   FacialInstance.obj
 0001:0008c380       ?GetFaceState@CFacialInstance@@UAEPAUIFaceState@@XZ 3158d380 f   FacialInstance.obj
 0001:0008c390       ?StartEffectorChannel@CFacialInstance@@UAEIPAUIFacialEffector@@MMMH@Z 3158d390 f   FacialInstance.obj
 0001:0008c3d0       ?StopEffectorChannel@CFacialInstance@@UAEXIM@Z 3158d3d0 f   FacialInstance.obj
 0001:0008c3f0       ?FindEffector@CFacialInstance@@QAEPAUIFacialEffector@@VCFaceIdentifierHandle@@@Z 3158d3f0 f   FacialInstance.obj
 0001:0008c420       ?SeekSequence@CFacialInstance@@UAEXW4EFacialSequenceLayer@@M@Z 3158d420 f   FacialInstance.obj
 0001:0008c450       ?IsPlaySequence@CFacialInstance@@UAE_NPAUIFacialAnimSequence@@W4EFacialSequenceLayer@@@Z 3158d450 f   FacialInstance.obj
 0001:0008c490       ?PauseSequence@CFacialInstance@@UAEXW4EFacialSequenceLayer@@_N@Z 3158d490 f   FacialInstance.obj
 0001:0008c4b0       ?ProcessWaitingLipSync@CFacialInstance@@QAEXXZ 3158d4b0 f   FacialInstance.obj
 0001:0008c560       ?OnExpressionLibraryLoad@CFacialInstance@@UAEXXZ 3158d560 f   FacialInstance.obj
 0001:0008c570       ?ApplyProceduralFaceBehaviour@CFacialInstance@@QAEXAAU?$Vec3_tpl@M@@@Z 3158d570 f   FacialInstance.obj
 0001:0008c6d0       ?TemporarilyEnableBoneRotationSmoothing@CFacialInstance@@UAEXXZ 3158d6d0 f   FacialInstance.obj
 0001:0008c700       ?UpdateCurrentSequence@CFacialInstance@@AAEXPAUIFacialAnimSequence@@@Z 3158d700 f   FacialInstance.obj
 0001:0008c850       ?find@?$CryStackStringT@D$0CAA@@@QBEIDI@Z 3158d850 f i FacialInstance.obj
 0001:0008c890       ?replace@?$CryStackStringT@D$0CAA@@@QAEAAV1@DD@Z 3158d890 f i FacialInstance.obj
 0001:0008c8d0       ?UpdateDue@CConstantFrameRateSkipper@@QAE_NXZ 3158d8d0 f i FacialInstance.obj
 0001:0008c980       ?UpdatePlayingSequences@CFacialInstance@@QAEXMABU?$QuatTS_tpl@M@@@Z 3158d980 f   FacialInstance.obj
 0001:0008cae0       ?PreviewEffector@CFacialInstance@@UAEXPAUIFacialEffector@@MM@Z 3158dae0 f   FacialInstance.obj
 0001:0008cbb0       ?PreviewEffectors@CFacialInstance@@UAEXPAPAUIFacialEffector@@PAM1H@Z 3158dbb0 f   FacialInstance.obj
 0001:0008ccc0       ?PlaySequence@CFacialInstance@@UAEXPAUIFacialAnimSequence@@W4EFacialSequenceLayer@@_N2@Z 3158dcc0 f   FacialInstance.obj
 0001:0008cdf0       ?StopSequence@CFacialInstance@@UAEXW4EFacialSequenceLayer@@@Z 3158ddf0 f   FacialInstance.obj
 0001:0008cee0       ?UpdateProceduralFaceBehaviour@CFacialInstance@@QAEXXZ 3158dee0 f   FacialInstance.obj
 0001:0008d030       ?Reset@CFacialInstance@@AAEXXZ 3158e030 f   FacialInstance.obj
 0001:0008d100       ?replace@?$CryStackStringT@D$0CAA@@@QAEAAV1@PBD0@Z 3158e100 f i FacialInstance.obj
 0001:0008d2a0       ??$move_init@VCFacialAnimForcedRotationEntry@@@NArray@@YAXPAVCFacialAnimForcedRotationEntry@@0I@Z 3158e2a0 f i FacialInstance.obj
 0001:0008d3e0       ?substr@?$CryStackStringT@D$0CAA@@@QBE?AV1@II@Z 3158e3e0 f i FacialInstance.obj
 0001:0008d470       ?GetMemoryUsage@CFacialInstance@@QBEXPAVICrySizer@@@Z 3158e470 f   FacialInstance.obj
 0001:0008d530       ?resize_raw@?$SmallDynStorage@VCFacialAnimForcedRotationEntry@@HUStandardAlloc@NAlloc@@@NArray@@QAEXHH_N@Z 3158e530 f i FacialInstance.obj
 0001:0008d690       ?GetPath@PathUtil@@YA?AV?$CryStackStringT@D$0CAA@@@ABV2@@Z 3158e690 f i FacialInstance.obj
 0001:0008d6f0       ?Update@CFacialInstance@@QAEXAAV?$map@IUSFacialDisplaceInfo@CFacialModel@@U?$less@I@stlpmtx_std@@V?$allocator@U?$pair@$$CBIUSFacialDisplaceInfo@CFacialModel@@@stlpmtx_std@@@4@@stlpmtx_std@@MABU?$QuatTS_tpl@M@@@Z 3158e6f0 f   FacialInstance.obj
 0001:0008d7e0       ?expand_raw@?$DynArray@VCFacialAnimForcedRotationEntry@@HU?$SmallDynStorage@VCFacialAnimForcedRotationEntry@@HUStandardAlloc@NAlloc@@@NArray@@@@IAEPAVCFacialAnimForcedRotationEntry@@PAV2@H@Z 3158e7e0 f i FacialInstance.obj
 0001:0008d870       ?GetFileName@PathUtil@@YA?AV?$CryStringT@D@@ABV2@@Z 3158e870 f i FacialInstance.obj
 0001:0008d8e0       ?AddSlash@PathUtil@@YA?AV?$CryStackStringT@D$0CAA@@@ABV2@@Z 3158e8e0 f i FacialInstance.obj
 0001:0008d9a0       ?Make@PathUtil@@YA?AV?$CryStackStringT@D$0CAA@@@ABV2@0@Z 3158e9a0 f i FacialInstance.obj
 0001:0008da30       ?LipSyncWithSound@CFacialInstance@@UAEXI_N@Z 3158ea30 f   FacialInstance.obj
 0001:0008e1d0       ??0CFacialInstance@@QAE@PAVCFacialModel@@PAVCCharInstance@@@Z 3158f1d0 f   FacialInstance.obj
 0001:0008e4b0       ??_ECFacialInstance@@W3AEPAXI@Z 3158f4b0 f i FacialInstance.obj
 0001:0008e4c0       ??1CFacialInstance@@UAE@XZ 3158f4c0 f i FacialInstance.obj
 0001:0008e590       ??_GCFacialInstance@@UAEPAXI@Z 3158f590 f i FacialInstance.obj
 0001:0008e590       ??_ECFacialInstance@@UAEPAXI@Z 3158f590 f i FacialInstance.obj
 0001:0008e5c0       ?SetForcedRotations@CFacialInstance@@UAEXHPAVCFacialAnimForcedRotationEntry@@@Z 3158f5c0 f   FacialInstance.obj
 0001:0008e630       ??_EValidator@pe_action_batch_parts_update@@UAEPAXI@Z 3158f630 f i SkeletonPhysics.obj
 0001:0008e630       ??_EISplineBackup@@UAEPAXI@Z 3158f630 f i FaceAnimSequence.obj
 0001:0008e630       ??_GIVertexAnimation@@UAEPAXI@Z 3158f630 f i VertexAnimation.obj
 0001:0008e630       ??_GValidator@pe_action_batch_parts_update@@UAEPAXI@Z 3158f630 f i SkeletonPhysics.obj
 0001:0008e630       ??_GISplineBackup@@UAEPAXI@Z 3158f630 f i FaceAnimSequence.obj
 0001:0008e630       ??_GIFaceState@@UAEPAXI@Z  3158f630 f i FacialModel.obj
 0001:0008e630       ??_EIFaceState@@UAEPAXI@Z  3158f630 f i FacialModel.obj
 0001:0008e630       ??_EIVertexAnimation@@UAEPAXI@Z 3158f630 f i VertexAnimation.obj
 0001:0008e660       ?GetMorphTargetCount@CFacialModel@@UBEHXZ 3158f660 f   FacialModel.obj
 0001:0008e680       ?ApplyBoneEffector@CFacialModel@@AAEHPAVCSkeletonPose@@PAVCFacialEffector@@MAAU?$QuatT_tpl@M@@@Z 3158f680 f   FacialModel.obj
 0001:0008e7d0       ?TransformTranslations@CFacialModel@@AAEXAAV?$map@IUSFacialDisplaceInfo@CFacialModel@@U?$less@I@stlpmtx_std@@V?$allocator@U?$pair@$$CBIUSFacialDisplaceInfo@CFacialModel@@@stlpmtx_std@@@4@@stlpmtx_std@@QBVCSkeletonPose@@@Z 3158f7d0 f   FacialModel.obj
 0001:0008e970       ?SetAffectedJointsToDefaultPose@CFacialModel@@SAXABV?$map@IUSFacialDisplaceInfo@CFacialModel@@U?$less@I@stlpmtx_std@@V?$allocator@U?$pair@$$CBIUSFacialDisplaceInfo@CFacialModel@@@stlpmtx_std@@@4@@stlpmtx_std@@QAU?$QuatT_tpl@M@@QBU4@@Z 3158f970 f   FacialModel.obj
 0001:0008ea20       ?ApplyDisplaceInfoToJoints@CFacialModel@@SAXABV?$map@IUSFacialDisplaceInfo@CFacialModel@@U?$less@I@stlpmtx_std@@V?$allocator@U?$pair@$$CBIUSFacialDisplaceInfo@CFacialModel@@@stlpmtx_std@@@4@@stlpmtx_std@@QBVCModelSkeleton@@QAVCPoseData@Skeleton@@@Z 3158fa20 f   FacialModel.obj
 0001:0008efd0       ?SizeOfThis@CFacialModel@@QAEIXZ 3158ffd0 f   FacialModel.obj
 0001:0008f020       ??$__unguarded_linear_insert@PAUSMorphTargetInfo@CFacialModel@@U12@U?$less@USMorphTargetInfo@CFacialModel@@@stlpmtx_std@@@priv@stlpmtx_std@@YAXPAUSMorphTargetInfo@CFacialModel@@U23@U?$less@USMorphTargetInfo@CFacialModel@@@1@@Z 31590020 f i FacialModel.obj
 0001:0008f120       ??$__push_heap@PAUSMorphTargetInfo@CFacialModel@@HU12@U?$less@USMorphTargetInfo@CFacialModel@@@stlpmtx_std@@@stlpmtx_std@@YAXPAUSMorphTargetInfo@CFacialModel@@HHU12@U?$less@USMorphTargetInfo@CFacialModel@@@0@@Z 31590120 f i FacialModel.obj
 0001:0008f250       ??$__copy_backward@PAUSMorphTargetInfo@CFacialModel@@PAU12@H@priv@stlpmtx_std@@YAPAUSMorphTargetInfo@CFacialModel@@PAU23@00ABUrandom_access_iterator_tag@1@PAH@Z 31590250 f i FacialModel.obj
 0001:0008f340       ?GetMorphTargetName@CFacialModel@@UBEPBDH@Z 31590340 f   FacialModel.obj
 0001:0008f3d0       ??$AddObject@USEffectorInfo@CFacialModel@@V?$allocator@USEffectorInfo@CFacialModel@@@stlpmtx_std@@@ICrySizer@@QAEXABV?$vector@USEffectorInfo@CFacialModel@@V?$allocator@USEffectorInfo@CFacialModel@@@stlpmtx_std@@@stlpmtx_std@@@Z 315903d0 f i FacialModel.obj
 0001:0008f450       ??$__unguarded_insertion_sort_aux@PAUSMorphTargetInfo@CFacialModel@@U12@U?$less@USMorphTargetInfo@CFacialModel@@@stlpmtx_std@@@priv@stlpmtx_std@@YAXPAUSMorphTargetInfo@CFacialModel@@00U?$less@USMorphTargetInfo@CFacialModel@@@1@@Z 31590450 f i FacialModel.obj
 0001:0008f4a0       ??$__adjust_heap@PAUSMorphTargetInfo@CFacialModel@@HU12@U?$less@USMorphTargetInfo@CFacialModel@@@stlpmtx_std@@@stlpmtx_std@@YAXPAUSMorphTargetInfo@CFacialModel@@HHU12@U?$less@USMorphTargetInfo@CFacialModel@@@0@@Z 315904a0 f i FacialModel.obj
 0001:0008f620       ??$AddObject@USMorphTargetInfo@CFacialModel@@V?$allocator@USMorphTargetInfo@CFacialModel@@@stlpmtx_std@@@ICrySizer@@QAEXABV?$vector@USMorphTargetInfo@CFacialModel@@V?$allocator@USMorphTargetInfo@CFacialModel@@@stlpmtx_std@@@stlpmtx_std@@@Z 31590620 f i FacialModel.obj
 0001:0008f6a0       ??$__ufill@PAUSEffectorInfo@CFacialModel@@U12@H@priv@stlpmtx_std@@YAXPAUSEffectorInfo@CFacialModel@@0ABU23@ABUrandom_access_iterator_tag@1@PAH@Z 315906a0 f i FacialModel.obj
 0001:0008f710       ??$__destroy_range_aux@V?$reverse_iterator@PAUSEffectorInfo@CFacialModel@@@stlpmtx_std@@USEffectorInfo@CFacialModel@@@stlpmtx_std@@YAXV?$reverse_iterator@PAUSEffectorInfo@CFacialModel@@@0@0PAUSEffectorInfo@CFacialModel@@ABU__false_type@0@@Z 31590710 f i FacialModel.obj
 0001:0008f770       ??$__destroy_range_aux@V?$reverse_iterator@PAUSMorphTargetInfo@CFacialModel@@@stlpmtx_std@@USMorphTargetInfo@CFacialModel@@@stlpmtx_std@@YAXV?$reverse_iterator@PAUSMorphTargetInfo@CFacialModel@@@0@0PAUSMorphTargetInfo@CFacialModel@@ABU__false_type@0@@Z 31590770 f i FacialModel.obj
 0001:0008f7c0       ?_M_create_node@?$_Rb_tree@IU?$less@I@stlpmtx_std@@U?$pair@$$CBIUSFacialDisplaceInfo@CFacialModel@@@2@U?$_Select1st@U?$pair@$$CBIUSFacialDisplaceInfo@CFacialModel@@@stlpmtx_std@@@priv@2@U?$_MapTraitsT@U?$pair@$$CBIUSFacialDisplaceInfo@CFacialModel@@@stlpmtx_std@@@52@V?$allocator@U?$pair@$$CBIUSFacialDisplaceInfo@CFacialModel@@@stlpmtx_std@@@2@@priv@stlpmtx_std@@IAEPAU_Rb_tree_node_base@23@ABU?$pair@$$CBIUSFacialDisplaceInfo@CFacialModel@@@3@@Z 315907c0 f i FacialModel.obj
 0001:0008f840       ??$__ucopy@PAUSEffectorInfo@CFacialModel@@PAU12@H@priv@stlpmtx_std@@YAPAUSEffectorInfo@CFacialModel@@PAU23@00ABUrandom_access_iterator_tag@1@PAH@Z 31590840 f i FacialModel.obj
 0001:0008f8b0       ??$__pop_heap@PAUSMorphTargetInfo@CFacialModel@@U12@U?$less@USMorphTargetInfo@CFacialModel@@@stlpmtx_std@@H@stlpmtx_std@@YAXPAUSMorphTargetInfo@CFacialModel@@00U12@U?$less@USMorphTargetInfo@CFacialModel@@@0@PAH@Z 315908b0 f i FacialModel.obj
 0001:0008f950       ??$__make_heap@PAUSMorphTargetInfo@CFacialModel@@U?$less@USMorphTargetInfo@CFacialModel@@@stlpmtx_std@@U12@H@stlpmtx_std@@YAXPAUSMorphTargetInfo@CFacialModel@@0U?$less@USMorphTargetInfo@CFacialModel@@@0@0PAH@Z 31590950 f i FacialModel.obj
 0001:0008f9d0       ??0CFaceState@@QAE@PAVCFacialModel@@@Z 315909d0 f i FacialModel.obj
 0001:0008fa40       ??_ECFaceState@@W3AEPAXI@Z 31590a40 f i FacialModel.obj
 0001:0008fa50       ?SetEffectorWeight@CFaceState@@UAEXHM@Z 31590a50 f i FacialModel.obj
 0001:0008fa80       ?GetEffectorWeight@CFaceState@@UAEMH@Z 31590a80 f i FacialModel.obj
 0001:0008fab0       ??_ECFaceState@@UAEPAXI@Z  31590ab0 f i FacialModel.obj
 0001:0008fab0       ??_GCFaceState@@UAEPAXI@Z  31590ab0 f i FacialModel.obj
 0001:0008fb30       ?CreateState@CFacialModel@@QAEPAVCFaceState@@XZ 31590b30 f   FacialModel.obj
 0001:0008fb70       ?GetMemoryUsage@CFacialModel@@QBEXPAVICrySizer@@@Z 31590b70 f   FacialModel.obj
 0001:0008fc00       ??$__ufill@PAUSMorphTargetInfo@CFacialModel@@U12@H@priv@stlpmtx_std@@YAXPAUSMorphTargetInfo@CFacialModel@@0ABU23@ABUrandom_access_iterator_tag@1@PAH@Z 31590c00 f i FacialModel.obj
 0001:0008fc60       ?_M_insert@?$_Rb_tree@IU?$less@I@stlpmtx_std@@U?$pair@$$CBIUSFacialDisplaceInfo@CFacialModel@@@2@U?$_Select1st@U?$pair@$$CBIUSFacialDisplaceInfo@CFacialModel@@@stlpmtx_std@@@priv@2@U?$_MapTraitsT@U?$pair@$$CBIUSFacialDisplaceInfo@CFacialModel@@@stlpmtx_std@@@52@V?$allocator@U?$pair@$$CBIUSFacialDisplaceInfo@CFacialModel@@@stlpmtx_std@@@2@@priv@stlpmtx_std@@AAE?AU?$_Rb_tree_iterator@U?$pair@$$CBIUSFacialDisplaceInfo@CFacialModel@@@stlpmtx_std@@U?$_MapTraitsT@U?$pair@$$CBIUSFacialDisplaceInfo@CFacialModel@@@stlpmtx_std@@@priv@2@@23@PAU_Rb_tree_node_base@23@ABU?$pair@$$CBIUSFacialDisplaceInfo@CFacialModel@@@3@00@Z 31590c60 f i FacialModel.obj
 0001:0008fcf0       ?insert_unique@?$_Rb_tree@IU?$less@I@stlpmtx_std@@U?$pair@$$CBIUSFacialDisplaceInfo@CFacialModel@@@2@U?$_Select1st@U?$pair@$$CBIUSFacialDisplaceInfo@CFacialModel@@@stlpmtx_std@@@priv@2@U?$_MapTraitsT@U?$pair@$$CBIUSFacialDisplaceInfo@CFacialModel@@@stlpmtx_std@@@52@V?$allocator@U?$pair@$$CBIUSFacialDisplaceInfo@CFacialModel@@@stlpmtx_std@@@2@@priv@stlpmtx_std@@QAE?AU?$pair@U?$_Rb_tree_iterator@U?$pair@$$CBIUSFacialDisplaceInfo@CFacialModel@@@stlpmtx_std@@U?$_MapTraitsT@U?$pair@$$CBIUSFacialDisplaceInfo@CFacialModel@@@stlpmtx_std@@@priv@2@@priv@stlpmtx_std@@_N@3@ABU?$pair@$$CBIUSFacialDisplaceInfo@CFacialModel@@@3@@Z 31590cf0 f i FacialModel.obj
 0001:0008fe00       ??$__ucopy@PAUSMorphTargetInfo@CFacialModel@@PAU12@H@priv@stlpmtx_std@@YAPAUSMorphTargetInfo@CFacialModel@@PAU23@00ABUrandom_access_iterator_tag@1@PAH@Z 31590e00 f i FacialModel.obj
 0001:0008fe60       ?insert_unique@?$_Rb_tree@IU?$less@I@stlpmtx_std@@U?$pair@$$CBIUSFacialDisplaceInfo@CFacialModel@@@2@U?$_Select1st@U?$pair@$$CBIUSFacialDisplaceInfo@CFacialModel@@@stlpmtx_std@@@priv@2@U?$_MapTraitsT@U?$pair@$$CBIUSFacialDisplaceInfo@CFacialModel@@@stlpmtx_std@@@52@V?$allocator@U?$pair@$$CBIUSFacialDisplaceInfo@CFacialModel@@@stlpmtx_std@@@2@@priv@stlpmtx_std@@QAE?AU?$_Rb_tree_iterator@U?$pair@$$CBIUSFacialDisplaceInfo@CFacialModel@@@stlpmtx_std@@U?$_MapTraitsT@U?$pair@$$CBIUSFacialDisplaceInfo@CFacialModel@@@stlpmtx_std@@@priv@2@@23@U423@ABU?$pair@$$CBIUSFacialDisplaceInfo@CFacialModel@@@3@@Z 31590e60 f i FacialModel.obj
 0001:00090050       ??$__unguarded_partition@PAUSMorphTargetInfo@CFacialModel@@U12@U?$less@USMorphTargetInfo@CFacialModel@@@stlpmtx_std@@@priv@stlpmtx_std@@YAPAUSMorphTargetInfo@CFacialModel@@PAU23@0U23@U?$less@USMorphTargetInfo@CFacialModel@@@1@@Z 31591050 f i FacialModel.obj
 0001:00090210       ??$__linear_insert@PAUSMorphTargetInfo@CFacialModel@@U12@U?$less@USMorphTargetInfo@CFacialModel@@@stlpmtx_std@@@priv@stlpmtx_std@@YAXPAUSMorphTargetInfo@CFacialModel@@0U23@U?$less@USMorphTargetInfo@CFacialModel@@@1@@Z 31591210 f i FacialModel.obj
 0001:000902c0       ??$sort_heap@PAUSMorphTargetInfo@CFacialModel@@U?$less@USMorphTargetInfo@CFacialModel@@@stlpmtx_std@@@stlpmtx_std@@YAXPAUSMorphTargetInfo@CFacialModel@@0U?$less@USMorphTargetInfo@CFacialModel@@@0@@Z 315912c0 f i FacialModel.obj
 0001:00090350       ?_M_insert_overflow_aux@?$_Impl_vector@USEffectorInfo@CFacialModel@@V?$allocator@USEffectorInfo@CFacialModel@@@stlpmtx_std@@@priv@stlpmtx_std@@AAEXPAUSEffectorInfo@CFacialModel@@ABU45@ABU__false_type@3@I_N@Z 31591350 f i FacialModel.obj
 0001:00090530       ??$_M_allocate_and_copy@PAUSEffectorInfo@CFacialModel@@@?$_Impl_vector@USEffectorInfo@CFacialModel@@V?$allocator@USEffectorInfo@CFacialModel@@@stlpmtx_std@@@priv@stlpmtx_std@@AAEPAUSEffectorInfo@CFacialModel@@AAIPAU34@1@Z 31591530 f i FacialModel.obj
 0001:000905a0       ??$__insertion_sort@PAUSMorphTargetInfo@CFacialModel@@U12@U?$less@USMorphTargetInfo@CFacialModel@@@stlpmtx_std@@@priv@stlpmtx_std@@YAXPAUSMorphTargetInfo@CFacialModel@@00U?$less@USMorphTargetInfo@CFacialModel@@@1@@Z 315915a0 f i FacialModel.obj
 0001:00090600       ??$__partial_sort@PAUSMorphTargetInfo@CFacialModel@@U12@U?$less@USMorphTargetInfo@CFacialModel@@@stlpmtx_std@@@priv@stlpmtx_std@@YAXPAUSMorphTargetInfo@CFacialModel@@000U?$less@USMorphTargetInfo@CFacialModel@@@1@@Z 31591600 f i FacialModel.obj
 0001:00090680       ?AssignLibrary@CFacialModel@@UAEXPAUIFacialEffectorsLibrary@@@Z 31591680 f   FacialModel.obj
 0001:000909f0       ?reserve@?$_Impl_vector@USEffectorInfo@CFacialModel@@V?$allocator@USEffectorInfo@CFacialModel@@@stlpmtx_std@@@priv@stlpmtx_std@@QAEXI@Z 315919f0 f i FacialModel.obj
 0001:00090ac0       ?_M_insert_overflow_aux@?$_Impl_vector@USMorphTargetInfo@CFacialModel@@V?$allocator@USMorphTargetInfo@CFacialModel@@@stlpmtx_std@@@priv@stlpmtx_std@@AAEXPAUSMorphTargetInfo@CFacialModel@@ABU45@ABU__false_type@3@I_N@Z 31591ac0 f i FacialModel.obj
 0001:00090c90       ??$?AH@?$map@IUSFacialDisplaceInfo@CFacialModel@@U?$less@I@stlpmtx_std@@V?$allocator@U?$pair@$$CBIUSFacialDisplaceInfo@CFacialModel@@@stlpmtx_std@@@4@@stlpmtx_std@@QAEAAUSFacialDisplaceInfo@CFacialModel@@ABH@Z 31591c90 f i FacialModel.obj
 0001:00090d50       ??$_M_allocate_and_copy@PAUSMorphTargetInfo@CFacialModel@@@?$_Impl_vector@USMorphTargetInfo@CFacialModel@@V?$allocator@USMorphTargetInfo@CFacialModel@@@stlpmtx_std@@@priv@stlpmtx_std@@AAEPAUSMorphTargetInfo@CFacialModel@@AAIPAU34@1@Z 31591d50 f i FacialModel.obj
 0001:00090dc0       ?FillInfoMapFromFaceState@CFacialModel@@QAEXAAV?$map@IUSFacialDisplaceInfo@CFacialModel@@U?$less@I@stlpmtx_std@@V?$allocator@U?$pair@$$CBIUSFacialDisplaceInfo@CFacialModel@@@stlpmtx_std@@@4@@stlpmtx_std@@QAVCFaceState@@QAVCSkeletonPose@@HQBVCFacialAnimForcedRotationEntry@@_N@Z 31591dc0 f   FacialModel.obj
 0001:00091390       ?push_back@?$_Impl_vector@USEffectorInfo@CFacialModel@@V?$allocator@USEffectorInfo@CFacialModel@@@stlpmtx_std@@@priv@stlpmtx_std@@QAEXABUSEffectorInfo@CFacialModel@@@Z 31592390 f i FacialModel.obj
 0001:00091420       ?reserve@?$_Impl_vector@USMorphTargetInfo@CFacialModel@@V?$allocator@USMorphTargetInfo@CFacialModel@@@stlpmtx_std@@@priv@stlpmtx_std@@QAEXI@Z 31592420 f i FacialModel.obj
 0001:000914f0       ??$__introsort_loop@PAUSMorphTargetInfo@CFacialModel@@U12@HU?$less@USMorphTargetInfo@CFacialModel@@@stlpmtx_std@@@priv@stlpmtx_std@@YAXPAUSMorphTargetInfo@CFacialModel@@00HU?$less@USMorphTargetInfo@CFacialModel@@@1@@Z 315924f0 f i FacialModel.obj
 0001:000915f0       ?push_back@?$_Impl_vector@USMorphTargetInfo@CFacialModel@@V?$allocator@USMorphTargetInfo@CFacialModel@@@stlpmtx_std@@@priv@stlpmtx_std@@QAEXABUSMorphTargetInfo@CFacialModel@@@Z 315925f0 f i FacialModel.obj
 0001:00091670       ?InitMorphTargets@CFacialModel@@AAEXXZ 31592670 f   FacialModel.obj
 0001:00091ac0       ??0CFacialModel@@QAE@PAVCSkel@@@Z 31592ac0 f   FacialModel.obj
 0001:00091b60       ??_ECFacialModel@@W3AEPAXI@Z 31592b60 f i FacialModel.obj
 0001:00091b70       ?GetNumFacialAnimations@CAnimationSet@@UAEHXZ 31592b70 f i ModelAnimationSet.obj
 0001:00091b70       ?GetEffectorCount@CFacialModel@@UBEHXZ 31592b70 f i FacialModel.obj
 0001:00091b90       ?GetEffector@CFacialModel@@UBEPAVCFacialEffector@@H@Z 31592b90 f i FacialModel.obj
 0001:00091bb0       ??1CFacialModel@@UAE@XZ    31592bb0 f i FacialModel.obj
 0001:00091c90       ??_GCFacialModel@@UAEPAXI@Z 31592c90 f i FacialModel.obj
 0001:00091c90       ??_ECFacialModel@@UAEPAXI@Z 31592c90 f i FacialModel.obj
 0001:00091cc0       ??_EISkin@@UAEPAXI@Z       31592cc0 f i ModelSkin.obj
 0001:00091cc0       ??_GIFacialSentence@@UAEPAXI@Z 31592cc0 f i LipSync.obj
 0001:00091cc0       ??_EIFacialSentence@@UAEPAXI@Z 31592cc0 f i LipSync.obj
 0001:00091cc0       ??_GISkin@@UAEPAXI@Z       31592cc0 f i ModelSkin.obj
 0001:00091cf0       ?phoneme_less@@YA_NABUSPhoneme@@0@Z 31592cf0 f i LipSync.obj
 0001:00091d20       ?GetPhonemeLib@CFacialSentence@@UAEPAUIPhonemeLibrary@@XZ 31592d20 f   LipSync.obj
 0001:00091d40       ??_G?$_reference_target@H@@UAEPAXI@Z 31592d40 f i LipSync.obj
 0001:00091d40       ??_E?$_reference_target@H@@UAEPAXI@Z 31592d40 f i LipSync.obj
 0001:00091d70       ?GetPhonemeCount@CPhonemesLibrary@@UBEHXZ 31592d70 f   LipSync.obj
 0001:00091d90       ?GetPhonemeInfo@CPhonemesLibrary@@UAE_NHAAUSPhonemeInfo@@@Z 31592d90 f   LipSync.obj
 0001:00091df0       ?allocate@?$_STLP_alloc_proxy@PAUSPhoneme@@U1@V?$allocator@USPhoneme@@@stlpmtx_std@@@priv@stlpmtx_std@@QAEPAUSPhoneme@@IAAI@Z 31592df0 f i LipSync.obj
 0001:00091df0       ?allocate@?$_STLP_alloc_proxy@PAUSEffectorInfo@CFacialModel@@U12@V?$allocator@USEffectorInfo@CFacialModel@@@stlpmtx_std@@@priv@stlpmtx_std@@QAEPAUSEffectorInfo@CFacialModel@@IAAI@Z 31592df0 f i FacialModel.obj
 0001:00091df0       ?allocate@?$_STLP_alloc_proxy@PAUSMorphTargetInfo@CFacialModel@@U12@V?$allocator@USMorphTargetInfo@CFacialModel@@@stlpmtx_std@@@priv@stlpmtx_std@@QAEPAUSMorphTargetInfo@CFacialModel@@IAAI@Z 31592df0 f i FacialModel.obj
 0001:00091e50       ??$__lower_bound@PAUSPhoneme@@U1@P6A_NABU1@0@ZP6A_N00@ZH@priv@stlpmtx_std@@YAPAUSPhoneme@@PAU2@0ABU2@P6A_N11@Z2PAH@Z 31592e50 f i LipSync.obj
 0001:00091ec0       ??0?$_Vector_base@UPhoneme@IFacialSentence@@V?$allocator@UPhoneme@IFacialSentence@@@stlpmtx_std@@@priv@stlpmtx_std@@QAE@IABV?$allocator@UPhoneme@IFacialSentence@@@2@@Z 31592ec0 f i LipSync.obj
 0001:00091ec0       ??0?$_Vector_base@U?$TCoeffBasis@M@spline@@V?$allocator@U?$TCoeffBasis@M@spline@@@stlpmtx_std@@@priv@stlpmtx_std@@QAE@IABV?$allocator@U?$TCoeffBasis@M@spline@@@2@@Z 31592ec0 f i FaceEffector.obj
 0001:00091f70       ?GetPhoneme@CFacialSentence@@UAE_NHAAUPhoneme@IFacialSentence@@@Z 31592f70 f   LipSync.obj
 0001:00091fc0       ?GetWord@CFacialSentence@@UAE_NHAAUWord@IFacialSentence@@@Z 31592fc0 f   LipSync.obj
 0001:00092020       ?Evaluate@CFacialSentence@@UAEHMMHPAUChannelSample@IFacialSentence@@@Z 31593020 f   LipSync.obj
 0001:000921f0       ?_M_insert_overflow@?$_Impl_vector@UBalanceChannelEntry@CFacialAnimSequenceInstance@@V?$allocator@UBalanceChannelEntry@CFacialAnimSequenceInstance@@@stlpmtx_std@@@priv@stlpmtx_std@@AAEXPAUBalanceChannelEntry@CFacialAnimSequenceInstance@@ABU45@ABU__true_type@3@I_N@Z 315931f0 f i FaceAnimSequence.obj
 0001:000921f0       ?_M_insert_overflow@?$_Impl_vector@U?$TCoeffBasis@M@spline@@V?$allocator@U?$TCoeffBasis@M@spline@@@stlpmtx_std@@@priv@stlpmtx_std@@AAEXPAU?$TCoeffBasis@M@spline@@ABU45@ABU__true_type@3@I_N@Z 315931f0 f i FaceEffector.obj
 0001:000921f0       ?_M_insert_overflow@?$_Impl_vector@UPhoneme@IFacialSentence@@V?$allocator@UPhoneme@IFacialSentence@@@stlpmtx_std@@@priv@stlpmtx_std@@AAEXPAUPhoneme@IFacialSentence@@ABU45@ABU__true_type@3@I_N@Z 315931f0 f i LipSync.obj
 0001:00092360       ??4SPhoneme@@QAEAAU0@ABU0@@Z 31593360 f i LipSync.obj
 0001:00092430       ??$__unguarded_linear_insert@PAUSPhoneme@@U1@P6A_NABU1@0@Z@priv@stlpmtx_std@@YAXPAUSPhoneme@@U2@P6A_NABU2@2@Z@Z 31593430 f i LipSync.obj
 0001:000924b0       ??$__push_heap@PAUSPhoneme@@HU1@P6A_NABU1@0@Z@stlpmtx_std@@YAXPAUSPhoneme@@HHU1@P6A_NABU1@2@Z@Z 315934b0 f i LipSync.obj
 0001:00092550       ??$__copy_backward@PAUSPhoneme@@PAU1@H@priv@stlpmtx_std@@YAPAUSPhoneme@@PAU2@00ABUrandom_access_iterator_tag@1@PAH@Z 31593550 f i LipSync.obj
 0001:00092650       ?FindPhonemeByName@CPhonemesLibrary@@UAEHPBD@Z 31593650 f   LipSync.obj
 0001:00092720       ?push_back@?$_Impl_vector@UPhoneme@IFacialSentence@@V?$allocator@UPhoneme@IFacialSentence@@@stlpmtx_std@@@priv@stlpmtx_std@@QAEXABUPhoneme@IFacialSentence@@@Z 31593720 f i LipSync.obj
 0001:00092790       ??4?$_Impl_vector@U?$TCoeffBasis@M@spline@@V?$allocator@U?$TCoeffBasis@M@spline@@@stlpmtx_std@@@priv@stlpmtx_std@@QAEAAV012@ABV012@@Z 31593790 f i FaceEffector.obj
 0001:00092790       ??4?$_Impl_vector@UPhoneme@IFacialSentence@@V?$allocator@UPhoneme@IFacialSentence@@@stlpmtx_std@@@priv@stlpmtx_std@@QAEAAV012@ABV012@@Z 31593790 f i LipSync.obj
 0001:000928a0       ??$__unguarded_insertion_sort_aux@PAUSPhoneme@@U1@P6A_NABU1@0@Z@priv@stlpmtx_std@@YAXPAUSPhoneme@@00P6A_NABU2@1@Z@Z 315938a0 f i LipSync.obj
 0001:00092900       ??$__adjust_heap@PAUSPhoneme@@HU1@P6A_NABU1@0@Z@stlpmtx_std@@YAXPAUSPhoneme@@HHU1@P6A_NABU1@2@Z@Z 31593900 f i LipSync.obj
 0001:000929e0       ??0WordRec@CFacialSentence@@QAE@ABU01@@Z 315939e0 f i LipSync.obj
 0001:00092a70       ??$__ufill@PAUSPhoneme@@U1@H@priv@stlpmtx_std@@YAXPAUSPhoneme@@0ABU2@ABUrandom_access_iterator_tag@1@PAH@Z 31593a70 f i LipSync.obj
 0001:00092ae0       ??$__destroy_range_aux@V?$reverse_iterator@PAUSPhoneme@@@stlpmtx_std@@USPhoneme@@@stlpmtx_std@@YAXV?$reverse_iterator@PAUSPhoneme@@@0@0PAUSPhoneme@@ABU__false_type@0@@Z 31593ae0 f i LipSync.obj
 0001:00092b30       ??$__ucopy@PAUSPhoneme@@PAU1@H@priv@stlpmtx_std@@YAPAUSPhoneme@@PAU2@00ABUrandom_access_iterator_tag@1@PAH@Z 31593b30 f i LipSync.obj
 0001:00092b90       ??$__pop_heap@PAUSPhoneme@@U1@P6A_NABU1@0@ZH@stlpmtx_std@@YAXPAUSPhoneme@@00U1@P6A_NABU1@2@ZPAH@Z 31593b90 f i LipSync.obj
 0001:00092c20       ??$__make_heap@PAUSPhoneme@@P6A_NABU1@0@ZU1@H@stlpmtx_std@@YAXPAUSPhoneme@@0P6A_NABU1@1@Z0PAH@Z 31593c20 f i LipSync.obj
 0001:00092ca0       ?AddPhoneme@CFacialSentence@@UAEHABUPhoneme@IFacialSentence@@@Z 31593ca0 f   LipSync.obj
 0001:00092cd0       ?Animate@CFacialSentence@@QAEXABU?$QuatTS_tpl@M@@PAVCFacialAnimationContext@@MMABV?$VectorSet@VCFaceIdentifierHandle@@USFaceIdentifierHandleLess@CFacialSentence@@V?$allocator@VCFaceIdentifierHandle@@@stlpmtx_std@@@@@Z 31593cd0 f   LipSync.obj
 0001:00093000       ??$__unguarded_partition@PAUSPhoneme@@U1@P6A_NABU1@0@Z@priv@stlpmtx_std@@YAPAUSPhoneme@@PAU2@0U2@P6A_NABU2@2@Z@Z 31594000 f i LipSync.obj
 0001:00093100       ??$__destroy_range_aux@V?$reverse_iterator@PAUWordRec@CFacialSentence@@@stlpmtx_std@@UWordRec@CFacialSentence@@@stlpmtx_std@@YAXV?$reverse_iterator@PAUWordRec@CFacialSentence@@@0@0PAUWordRec@CFacialSentence@@ABU__false_type@0@@Z 31594100 f i LipSync.obj
 0001:000931d0       ??$__destroy_range_aux@PAUWordRec@CFacialSentence@@U12@@stlpmtx_std@@YAXPAUWordRec@CFacialSentence@@00ABU__false_type@0@@Z 315941d0 f i LipSync.obj
 0001:000932a0       ??$__copy@PAUWordRec@CFacialSentence@@PAU12@H@priv@stlpmtx_std@@YAPAUWordRec@CFacialSentence@@PAU23@00ABUrandom_access_iterator_tag@1@PAH@Z 315942a0 f i LipSync.obj
 0001:00093390       ??$__linear_insert@PAUSPhoneme@@U1@P6A_NABU1@0@Z@priv@stlpmtx_std@@YAXPAUSPhoneme@@0U2@P6A_NABU2@2@Z@Z 31594390 f i LipSync.obj
 0001:00093440       ??$sort_heap@PAUSPhoneme@@P6A_NABU1@0@Z@stlpmtx_std@@YAXPAUSPhoneme@@0P6A_NABU1@1@Z@Z 31594440 f i LipSync.obj
 0001:000934d0       ?_M_insert_overflow_aux@?$_Impl_vector@USPhoneme@@V?$allocator@USPhoneme@@@stlpmtx_std@@@priv@stlpmtx_std@@AAEXPAUSPhoneme@@ABU4@ABU__false_type@3@I_N@Z 315944d0 f i LipSync.obj
 0001:00093690       ??$_M_allocate_and_copy@PAUSPhoneme@@@?$_Impl_vector@USPhoneme@@V?$allocator@USPhoneme@@@stlpmtx_std@@@priv@stlpmtx_std@@AAEPAUSPhoneme@@AAIPAU3@1@Z 31594690 f i LipSync.obj
 0001:00093700       ??$__uninitialized_fill_n@PAUWordRec@CFacialSentence@@IU12@@priv@stlpmtx_std@@YAPAUWordRec@CFacialSentence@@PAU23@IABU23@@Z 31594700 f i LipSync.obj
 0001:00093750       ??$__insertion_sort@PAUSPhoneme@@U1@P6A_NABU1@0@Z@priv@stlpmtx_std@@YAXPAUSPhoneme@@00P6A_NABU2@1@Z@Z 31594750 f i LipSync.obj
 0001:000937c0       ??$__partial_sort@PAUSPhoneme@@U1@P6A_NABU1@0@Z@priv@stlpmtx_std@@YAXPAUSPhoneme@@000P6A_NABU2@1@Z@Z 315947c0 f i LipSync.obj
 0001:00093850       ?reserve@?$_Impl_vector@USPhoneme@@V?$allocator@USPhoneme@@@stlpmtx_std@@@priv@stlpmtx_std@@QAEXI@Z 31594850 f i LipSync.obj
 0001:00093920       ?_M_insert_overflow_aux@?$_Impl_vector@UWordRec@CFacialSentence@@V?$allocator@UWordRec@CFacialSentence@@@stlpmtx_std@@@priv@stlpmtx_std@@AAEXPAUWordRec@CFacialSentence@@ABU45@ABU__false_type@3@I_N@Z 31594920 f i LipSync.obj
 0001:00093b10       ??$__introsort_loop@PAUSPhoneme@@U1@HP6A_NABU1@0@Z@priv@stlpmtx_std@@YAXPAUSPhoneme@@00HP6A_NABU2@1@Z@Z 31594b10 f i LipSync.obj
 0001:00093c40       ??0CFacialSentence@@QAE@XZ 31594c40 f   LipSync.obj
 0001:00093cb0       ??_ECFacialSentence@@W3AEPAXI@Z 31594cb0 f i LipSync.obj
 0001:00093cc0       ?GetPhonemeCount@CFacialSentence@@UAEHXZ 31594cc0 f i LipSync.obj
 0001:00093cd0       ?GetWordCount@CFacialSentence@@UAEHXZ 31594cd0 f i LipSync.obj
 0001:00093cf0       ?SetText@CFacialSentence@@UAEXPBD@Z 31594cf0 f i LipSync.obj
 0001:00093d30       ??1CFacialSentence@@UAE@XZ 31594d30 f i LipSync.obj
 0001:00093de0       ??_GCFacialSentence@@UAEPAXI@Z 31594de0 f i LipSync.obj
 0001:00093de0       ??_ECFacialSentence@@UAEPAXI@Z 31594de0 f i LipSync.obj
 0001:00093e10       ??0CPhonemesLibrary@@QAE@XZ 31594e10 f   LipSync.obj
 0001:00094020       ??_ECPhonemesLibrary@@UAEPAXI@Z 31595020 f i LipSync.obj
 0001:00094020       ??_GCPhonemesLibrary@@UAEPAXI@Z 31595020 f i LipSync.obj
 0001:00094090       ?clear@?$vector@UWordRec@CFacialSentence@@V?$allocator@UWordRec@CFacialSentence@@@stlpmtx_std@@@stlpmtx_std@@QAEXXZ 31595090 f i LipSync.obj
 0001:000940f0       ?ClearAllPhonemes@CFacialSentence@@UAEXXZ 315950f0 f i LipSync.obj
 0001:00094190       ?ClearAllWords@CFacialSentence@@UAEXXZ 31595190 f i LipSync.obj
 0001:000941f0       ?AddWord@CFacialSentence@@UAEXABUWord@IFacialSentence@@@Z 315951f0 f   LipSync.obj
 0001:00094310       ?Serialize@CFacialSentence@@QAEXAAVXmlNodeRef@@_N@Z 31595310 f   LipSync.obj
 0001:000949f0       ?GetFactory@CFeetPoseRestore@@UBEPAUICryFactory@@XZ 315959f0 f i FeetLock.obj
 0001:00094a00       ?Prepare@CFeetPoseRestore@@UAE_NABUSAnimationPoseModifierParams@@@Z 31595a00 f i FeetLock.obj
 0001:00094a00       ?Prepare@CFeetPoseStore@@UAE_NABUSAnimationPoseModifierParams@@@Z 31595a00 f i FeetLock.obj
 0001:00094a10       ?GetFactory@CFeetPoseStore@@UBEPAUICryFactory@@XZ 31595a10 f i FeetLock.obj
 0001:00094a20       ?GetMemoryUsage@CFeetPoseStore@@UBEXPAVICrySizer@@@Z 31595a20 f i FeetLock.obj
 0001:00094a20       ?GetMemoryUsage@CFeetPoseRestore@@UBEXPAVICrySizer@@@Z 31595a20 f i FeetLock.obj
 0001:00094a60       ?Execute@CFeetPoseStore@@UAE_NABUSAnimationPoseModifierParams@@@Z 31595a60 f   FeetLock.obj
 0001:00094e20       ?Execute@CFeetPoseRestore@@UAE_NABUSAnimationPoseModifierParams@@@Z 31595e20 f   FeetLock.obj
 0001:000952d0       ??0CFactory@CFeetPoseStore@@AAE@XZ 315962d0 f i FeetLock.obj
 0001:00095370       ?GetClassName@CFactory@CFeetPoseStore@@UBEPBDXZ 31596370 f i FeetLock.obj
 0001:00095380       ?GetClassID@CFactory@CFeetPoseStore@@UBEABUCryGUID@@XZ 31596380 f i FeetLock.obj
 0001:00095390       ?ClassSupports@CFactory@CLimbIk@@UBEXAAPBUCryGUID@@AAI@Z 31596390 f i LimbIk.obj
 0001:00095390       ?ClassSupports@CFactory@CFeetPoseStore@@UBEXAAPBUCryGUID@@AAI@Z 31596390 f i FeetLock.obj
 0001:00095390       ?ClassSupports@CFactory@CPoseBlenderAim@@UBEXAAPBUCryGUID@@AAI@Z 31596390 f i PoseBlenderAim.obj
 0001:00095390       ?ClassSupports@CFactory@CPoseAlignerChain@@UBEXAAPBUCryGUID@@AAI@Z 31596390 f i PoseAlignerChain.obj
 0001:00095390       ?ClassSupports@CFactory@CGroundAlignment@@UBEXAAPBUCryGUID@@AAI@Z 31596390 f i GroundAlignment.obj
 0001:00095390       ?ClassSupports@CFactory@CFeetPoseRestore@@UBEXAAPBUCryGUID@@AAI@Z 31596390 f i FeetLock.obj
 0001:00095390       ?ClassSupports@CFactory@CEngineModule_CryAnimation@@UBEXAAPBUCryGUID@@AAI@Z 31596390 f i AnimationBase.obj
 0001:00095390       ?ClassSupports@CFactory@CPoseMatching@@UBEXAAPBUCryGUID@@AAI@Z 31596390 f i PoseMatching.obj
 0001:00095390       ?ClassSupports@CFactory@CPoseBlenderLook@@UBEXAAPBUCryGUID@@AAI@Z 31596390 f i PoseBlenderLook.obj
 0001:00095390       ?ClassSupports@CFactory@CRecoil@PoseModifier@@UBEXAAPBUCryGUID@@AAI@Z 31596390 f i Recoil.obj
 0001:00095390       ?ClassSupports@CFactory@COperatorQueue@@UBEXAAPBUCryGUID@@AAI@Z 31596390 f i OperatorQueue.obj
 0001:000953b0       ?CreateClassInstance@CFactory@CFeetPoseStore@@UBE?AV?$shared_ptr@UICryUnknown@@@boost@@XZ 315963b0 f i FeetLock.obj
 0001:00095450       ??0CFactory@CFeetPoseRestore@@AAE@XZ 31596450 f i FeetLock.obj
 0001:000954f0       ?GetClassName@CFactory@CFeetPoseRestore@@UBEPBDXZ 315964f0 f i FeetLock.obj
 0001:00095500       ?GetClassID@CFactory@CFeetPoseRestore@@UBEABUCryGUID@@XZ 31596500 f i FeetLock.obj
 0001:00095510       ?CreateClassInstance@CFactory@CFeetPoseRestore@@UBE?AV?$shared_ptr@UICryUnknown@@@boost@@XZ 31596510 f i FeetLock.obj
 0001:000955b0       ?QueryInterface@CFeetPoseStore@@MBEPAXABUCryGUID@@@Z 315965b0 f i FeetLock.obj
 0001:000955b0       ?QueryInterface@CRecoil@PoseModifier@@MBEPAXABUCryGUID@@@Z 315965b0 f i Recoil.obj
 0001:000955b0       ?QueryInterface@CLimbIk@@MBEPAXABUCryGUID@@@Z 315965b0 f i LimbIk.obj
 0001:000955b0       ?QueryInterface@CFeetPoseRestore@@MBEPAXABUCryGUID@@@Z 315965b0 f i FeetLock.obj
 0001:00095610       ??0CFeetLock@@QAE@XZ       31596610 f   FeetLock.obj
 0001:00095650       ?Prepare@CGroundAlignment@@UAE_NABUSAnimationPoseModifierParams@@@Z 31596650 f   GroundAlignment.obj
 0001:000956c0       ??0CGroundAlignment@@IAE@XZ 315966c0 f   GroundAlignment.obj
 0001:00095780       ?GetFactory@CGroundAlignment@@UBEPAUICryFactory@@XZ 31596780 f i GroundAlignment.obj
 0001:00095790       ?SetData@CGroundAlignment@@UAEX_NMABU?$Plane_tpl@M@@1@Z 31596790 f i GroundAlignment.obj
 0001:000957e0       ?GetMemoryUsage@CGroundAlignment@@UBEXPAVICrySizer@@@Z 315967e0 f i GroundAlignment.obj
 0001:00095800       ??$Op@$$CBVCGroundAlignment@@@?$InterfaceCast@U?$Typelist@UIAnimationPoseModifier@@U?$Typelist@UIAnimationGroundAlignment@@VNullType@TL@@@TL@@@TL@@@CW@@SAPAXPBVCGroundAlignment@@ABUCryGUID@@@Z 31596800 f i GroundAlignment.obj
 0001:00095860       ?SetFootGroundAlignment@CGroundAlignment@@AAEIABUSAnimationPoseModifierParams@@ABU?$Vec3_tpl@M@@HHHH@Z 31596860 f   GroundAlignment.obj
 0001:000967e0       ?PerformGroundAlignmentCCD@CGroundAlignment@@AAEIABUSAnimationPoseModifierParams@@PBDABU?$Plane_tpl@M@@@Z 315977e0 f   GroundAlignment.obj
 0001:00097980       ?MoveSkeletonVertical@CGroundAlignment@@AAEXABUSAnimationPoseModifierParams@@M@Z 31598980 f   GroundAlignment.obj
 0001:00097db0       ?AlignJointToPlane@@YA_NABUSAnimationPoseModifierParams@@IABU?$Vec3_tpl@M@@1@Z 31598db0 f   GroundAlignment.obj
 0001:000985d0       ?QueryInterface@CGroundAlignment@@MBEPAXABUCryGUID@@@Z 315995d0 f i GroundAlignment.obj
 0001:00098610       ?LimbAlign@CGroundAlignment@@AAE_NABUSAnimationPoseModifierParams@@IPBDABU?$Plane_tpl@M@@@Z 31599610 f   GroundAlignment.obj
 0001:000988a0       ?Execute@CGroundAlignment@@UAE_NABUSAnimationPoseModifierParams@@@Z 315998a0 f   GroundAlignment.obj
 0001:00098930       ?Op@?$FillIIDs@U?$Typelist@UICryUnknown@@U?$Typelist@UIAnimationPoseModifier@@U?$Typelist@UIAnimationGroundAlignment@@VNullType@TL@@@TL@@@TL@@@TL@@@CW@@SAXPAUCryGUID@@@Z 31599930 f i GroundAlignment.obj
 0001:000989b0       ?GetClassName@CFactory@CGroundAlignment@@UBEPBDXZ 315999b0 f i GroundAlignment.obj
 0001:000989c0       ?GetClassID@CFactory@CGroundAlignment@@UBEABUCryGUID@@XZ 315999c0 f i GroundAlignment.obj
 0001:000989d0       ?CreateClassInstance@CFactory@CGroundAlignment@@UBE?AV?$shared_ptr@UICryUnknown@@@boost@@XZ 315999d0 f i GroundAlignment.obj
 0001:00098a70       ?AddSetup@CLimbIk@@QAEX_KABU?$Vec3_tpl@M@@@Z 31599a70 f   LimbIk.obj
 0001:00098b20       ?Prepare@CLimbIk@@UAE_NABUSAnimationPoseModifierParams@@@Z 31599b20 f   LimbIk.obj
 0001:00098b60       ?Execute@CLimbIk@@UAE_NABUSAnimationPoseModifierParams@@@Z 31599b60 f   LimbIk.obj
 0001:00098be0       ?GetFactory@CLimbIk@@UBEPAUICryFactory@@XZ 31599be0 f i LimbIk.obj
 0001:00098bf0       ?GetMemoryUsage@CLimbIk@@UBEXPAVICrySizer@@@Z 31599bf0 f i LimbIk.obj
 0001:00098c10       ??0CFactory@CLimbIk@@AAE@XZ 31599c10 f i LimbIk.obj
 0001:00098cb0       ?GetClassName@CFactory@CLimbIk@@UBEPBDXZ 31599cb0 f i LimbIk.obj
 0001:00098cc0       ?GetClassID@CFactory@CLimbIk@@UBEABUCryGUID@@XZ 31599cc0 f i LimbIk.obj
 0001:00098cd0       ?ClassSupports@CFactory@CEngineModule_CryAnimation@@UBE_NABUCryGUID@@@Z 31599cd0 f i AnimationBase.obj
 0001:00098cd0       ?ClassSupports@CFactory@CPoseBlenderLook@@UBE_NABUCryGUID@@@Z 31599cd0 f i PoseBlenderLook.obj
 0001:00098cd0       ?ClassSupports@CFactory@CPoseMatching@@UBE_NABUCryGUID@@@Z 31599cd0 f i PoseMatching.obj
 0001:00098cd0       ?ClassSupports@CFactory@CLimbIk@@UBE_NABUCryGUID@@@Z 31599cd0 f i LimbIk.obj
 0001:00098cd0       ?ClassSupports@CFactory@CPoseBlenderAim@@UBE_NABUCryGUID@@@Z 31599cd0 f i PoseBlenderAim.obj
 0001:00098cd0       ?ClassSupports@CFactory@CGroundAlignment@@UBE_NABUCryGUID@@@Z 31599cd0 f i GroundAlignment.obj
 0001:00098cd0       ?ClassSupports@CFactory@CFeetPoseStore@@UBE_NABUCryGUID@@@Z 31599cd0 f i FeetLock.obj
 0001:00098cd0       ?ClassSupports@CFactory@CPoseAlignerChain@@UBE_NABUCryGUID@@@Z 31599cd0 f i PoseAlignerChain.obj
 0001:00098cd0       ?ClassSupports@CFactory@COperatorQueue@@UBE_NABUCryGUID@@@Z 31599cd0 f i OperatorQueue.obj
 0001:00098cd0       ?ClassSupports@CFactory@CRecoil@PoseModifier@@UBE_NABUCryGUID@@@Z 31599cd0 f i Recoil.obj
 0001:00098cd0       ?ClassSupports@CFactory@CFeetPoseRestore@@UBE_NABUCryGUID@@@Z 31599cd0 f i FeetLock.obj
 0001:00098d20       ?CreateClassInstance@CFactory@CLimbIk@@UBE?AV?$shared_ptr@UICryUnknown@@@boost@@XZ 31599d20 f i LimbIk.obj
 0001:00098df0       ??0SDirectionalBlender@@QAE@XZ 31599df0 f i PoseBlenderAim.obj
 0001:00098e70       ?GetFactory@CPoseBlenderAim@@UBEPAUICryFactory@@XZ 31599e70 f i PoseBlenderAim.obj
 0001:00098e80       ?SetState@CPoseBlenderAim@@UAEX_N@Z 31599e80 f i PoseBlenderAim.obj
 0001:00098e90       ?SetLayer@CPoseBlenderAim@@UAEXI@Z 31599e90 f i PoseBlenderAim.obj
 0001:00098eb0       ?SetFadeoutAngle@CPoseBlenderAim@@UAEXM@Z 31599eb0 f i PoseBlenderAim.obj
 0001:00098ed0       ?SetFadeOutSpeed@CPoseBlenderAim@@UAEXM@Z 31599ed0 f i PoseBlenderAim.obj
 0001:00098f10       ?SetFadeInSpeed@CPoseBlenderAim@@UAEXM@Z 31599f10 f i PoseBlenderAim.obj
 0001:00098f50       ?SetVideoMarkerOffset@CFacialJoystickChannel@@UAEXM@Z 31599f50 f i FaceJoystick.obj
 0001:00098f50       ?SetTargetSmoothTime@CPoseBlenderAim@@UAEXM@Z 31599f50 f i PoseBlenderAim.obj
 0001:00098f70       ?GetBlend@CPoseBlenderAim@@UAEMXZ 31599f70 f i PoseBlenderAim.obj
 0001:00098f80       ?Synchronize@CPoseBlenderAim@@UAEXXZ 31599f80 f i PoseBlenderAim.obj
 0001:00098f90       ?GetMemoryUsage@CPoseBlenderAim@@UBEXPAVICrySizer@@@Z 31599f90 f i PoseBlenderAim.obj
 0001:00098fb0       ?SetPolarCoordinates@CPoseBlenderAim@@UAEXABU?$Vec2_tpl@M@@@Z 31599fb0 f i PoseBlenderAim.obj
 0001:00098fd0       ??_EIJoystickContext@@UAEPAXI@Z 31599fd0 f i FaceAnimation.obj
 0001:00098fd0       ??_EICryUnknown@@MAEPAXI@Z 31599fd0 f i OperatorQueue.obj
 0001:00098fd0       ??_GCRecoil@PoseModifier@@MAEPAXI@Z 31599fd0 f i Recoil.obj
 0001:00098fd0       ??_GCPoseBlenderAim@@MAEPAXI@Z 31599fd0 f i PoseBlenderAim.obj
 0001:00098fd0       ??_GCPoseAlignerChain@@MAEPAXI@Z 31599fd0 f i PoseAlignerChain.obj
 0001:00098fd0       ??_GCFeetPoseRestore@@MAEPAXI@Z 31599fd0 f i FeetLock.obj
 0001:00098fd0       ??_ECFeetPoseRestore@@MAEPAXI@Z 31599fd0 f i FeetLock.obj
 0001:00098fd0       ??_ECPoseBlenderLook@@MAEPAXI@Z 31599fd0 f i PoseBlenderLook.obj
 0001:00098fd0       ??_GCPoseMatching@@MAEPAXI@Z 31599fd0 f i PoseMatching.obj
 0001:00098fd0       ??_ECPoseBlenderAim@@MAEPAXI@Z 31599fd0 f i PoseBlenderAim.obj
 0001:00098fd0       ??_ECFeetPoseStore@@MAEPAXI@Z 31599fd0 f i FeetLock.obj
 0001:00098fd0       ??_GCLimbIk@@MAEPAXI@Z     31599fd0 f i LimbIk.obj
 0001:00098fd0       ??_GCEngineModule_CryAnimation@@MAEPAXI@Z 31599fd0 f i AnimationBase.obj
 0001:00098fd0       ??_GIJoystickContext@@UAEPAXI@Z 31599fd0 f i FaceAnimation.obj
 0001:00098fd0       ??_ECPoseAlignerChain@@MAEPAXI@Z 31599fd0 f i PoseAlignerChain.obj
 0001:00098fd0       ??_GICryUnknown@@MAEPAXI@Z 31599fd0 f i OperatorQueue.obj
 0001:00098fd0       ??_ECPoseMatching@@MAEPAXI@Z 31599fd0 f i PoseMatching.obj
 0001:00098fd0       ??_ECLimbIk@@MAEPAXI@Z     31599fd0 f i LimbIk.obj
 0001:00098fd0       ??_GCPoseBlenderLook@@MAEPAXI@Z 31599fd0 f i PoseBlenderLook.obj
 0001:00098fd0       ??_ECGroundAlignment@@MAEPAXI@Z 31599fd0 f i GroundAlignment.obj
 0001:00098fd0       ??_ECEngineModule_CryAnimation@@MAEPAXI@Z 31599fd0 f i AnimationBase.obj
 0001:00098fd0       ??_ECRecoil@PoseModifier@@MAEPAXI@Z 31599fd0 f i Recoil.obj
 0001:00098fd0       ??_GCFeetPoseStore@@MAEPAXI@Z 31599fd0 f i FeetLock.obj
 0001:00098fd0       ??_GCGroundAlignment@@MAEPAXI@Z 31599fd0 f i GroundAlignment.obj
 0001:00099000       ?SetTarget@CPoseBlenderAim@@UAEXABU?$Vec3_tpl@M@@@Z 3159a000 f i PoseBlenderAim.obj
 0001:00099050       ??$Op@$$CBVCPoseBlenderAim@@@?$InterfaceCast@U?$Typelist@UIAnimationPoseModifier@@U?$Typelist@UIAnimationPoseBlenderDir@@VNullType@TL@@@TL@@@TL@@@CW@@SAPAXPBVCPoseBlenderAim@@ABUCryGUID@@@Z 3159a050 f i PoseBlenderAim.obj
 0001:00099050       ??$Op@$$CBVCPoseBlenderLook@@@?$InterfaceCast@U?$Typelist@UIAnimationPoseModifier@@U?$Typelist@UIAnimationPoseBlenderDir@@VNullType@TL@@@TL@@@TL@@@CW@@SAPAXPBVCPoseBlenderLook@@ABUCryGUID@@@Z 3159a050 f i PoseBlenderLook.obj
 0001:000990b0       ?Prepare@CPoseBlenderAim@@UAE_NABUSAnimationPoseModifierParams@@@Z 3159a0b0 f   PoseBlenderAim.obj
 0001:000999a0       ?Execute@CPoseBlenderAim@@UAE_NABUSAnimationPoseModifierParams@@@Z 3159a9a0 f   PoseBlenderAim.obj
 0001:0009a8f0       ?Op@?$FillIIDs@U?$Typelist@UICryUnknown@@U?$Typelist@UIAnimationPoseModifier@@U?$Typelist@UIAnimationPoseBlenderDir@@VNullType@TL@@@TL@@@TL@@@TL@@@CW@@SAXPAUCryGUID@@@Z 3159b8f0 f i PoseBlenderAim.obj
 0001:0009a970       ?GetClassName@CFactory@CPoseBlenderAim@@UBEPBDXZ 3159b970 f i PoseBlenderAim.obj
 0001:0009a980       ?GetClassID@CFactory@CPoseBlenderAim@@UBEABUCryGUID@@XZ 3159b980 f i PoseBlenderAim.obj
 0001:0009a990       ?CreateClassInstance@CFactory@CPoseBlenderAim@@UBE?AV?$shared_ptr@UICryUnknown@@@boost@@XZ 3159b990 f i PoseBlenderAim.obj
 0001:0009aa30       ?Synchronize@CPoseBlenderLook@@UAEXXZ 3159ba30 f   PoseBlenderLook.obj
 0001:0009ad90       ?GetFactory@CPoseBlenderLook@@UBEPAUICryFactory@@XZ 3159bd90 f i PoseBlenderLook.obj
 0001:0009ada0       ?SetState@CPoseBlenderLook@@UAEX_N@Z 3159bda0 f i PoseBlenderLook.obj
 0001:0009adb0       ?SetLayer@CPoseBlenderLook@@UAEXI@Z 3159bdb0 f i PoseBlenderLook.obj
 0001:0009add0       ?SetFadeoutAngle@CPoseBlenderLook@@UAEXM@Z 3159bdd0 f i PoseBlenderLook.obj
 0001:0009adf0       ?SetFadeOutSpeed@CPoseBlenderLook@@UAEXM@Z 3159bdf0 f i PoseBlenderLook.obj
 0001:0009ae30       ?SetFadeInSpeed@CPoseBlenderLook@@UAEXM@Z 3159be30 f i PoseBlenderLook.obj
 0001:0009ae70       ?SetTargetSmoothTime@CPoseBlenderLook@@UAEXM@Z 3159be70 f i PoseBlenderLook.obj
 0001:0009ae90       ?GetBlend@CPoseBlenderLook@@UAEMXZ 3159be90 f i PoseBlenderLook.obj
 0001:0009aea0       ?GetMemoryUsage@CPoseBlenderLook@@UBEXPAVICrySizer@@@Z 3159bea0 f i PoseBlenderLook.obj
 0001:0009aec0       ?SetPolarCoordinates@CPoseBlenderLook@@UAEXABU?$Vec2_tpl@M@@@Z 3159bec0 f i PoseBlenderLook.obj
 0001:0009aee0       ?SetTarget@CPoseBlenderLook@@UAEXABU?$Vec3_tpl@M@@@Z 3159bee0 f i PoseBlenderLook.obj
 0001:0009af30       ?Prepare@CPoseBlenderLook@@UAE_NABUSAnimationPoseModifierParams@@@Z 3159bf30 f   PoseBlenderLook.obj
 0001:0009ba60       ?Execute@CPoseBlenderLook@@UAE_NABUSAnimationPoseModifierParams@@@Z 3159ca60 f   PoseBlenderLook.obj
 0001:0009d890       ?GetClassName@CFactory@CPoseBlenderLook@@UBEPBDXZ 3159e890 f i PoseBlenderLook.obj
 0001:0009d8a0       ?GetClassID@CFactory@CPoseBlenderLook@@UBEABUCryGUID@@XZ 3159e8a0 f i PoseBlenderLook.obj
 0001:0009d8b0       ?CreateClassInstance@CFactory@CPoseBlenderLook@@UBE?AV?$shared_ptr@UICryUnknown@@@boost@@XZ 3159e8b0 f i PoseBlenderLook.obj
 0001:0009d9a0       ?QueryInterface@CPoseBlenderLook@@MBEPAXABUCryGUID@@@Z 3159e9a0 f i PoseBlenderLook.obj
 0001:0009d9a0       ?QueryInterface@CPoseBlenderAim@@MBEPAXABUCryGUID@@@Z 3159e9a0 f i PoseBlenderAim.obj
 0001:0009d9e0       ?IK_Solver2Bones@PoseModifierHelper@@YAXABU?$Vec3_tpl@M@@ABUIKLimbType@@AAVCPoseData@Skeleton@@@Z 3159e9e0 f   PoseModifierHelper.obj
 0001:0009ead0       ?IK_Solver3Bones@PoseModifierHelper@@YAXABU?$Vec3_tpl@M@@ABUIKLimbType@@AAVCPoseData@Skeleton@@@Z 3159fad0 f   PoseModifierHelper.obj
 0001:000a1940       ?IK_SolverCCD@PoseModifierHelper@@YAXABU?$Vec3_tpl@M@@ABUIKLimbType@@AAVCPoseData@Skeleton@@@Z 315a2940 f   PoseModifierHelper.obj
 0001:000a2b30       ?IK_Solver@PoseModifierHelper@@YA_NPIBVCModelSkeleton@@PBDABU?$Vec3_tpl@M@@AAVCPoseData@Skeleton@@@Z 315a3b30 f   PoseModifierHelper.obj
 0001:000a3120       ?Prepare@CRecoil@PoseModifier@@UAE_NABUSAnimationPoseModifierParams@@@Z 315a4120 f   Recoil.obj
 0001:000a3150       ?RecoilEffect@CRecoil@PoseModifier@@AAEMM@Z 315a4150 f   Recoil.obj
 0001:000a31d0       ?GetFactory@CRecoil@PoseModifier@@UBEPAUICryFactory@@XZ 315a41d0 f i Recoil.obj
 0001:000a31e0       ?GetMemoryUsage@CRecoil@PoseModifier@@UBEXPAVICrySizer@@@Z 315a41e0 f i Recoil.obj
 0001:000a3200       ??0CFactory@CRecoil@PoseModifier@@AAE@XZ 315a4200 f i Recoil.obj
 0001:000a32a0       ?GetClassName@CFactory@CRecoil@PoseModifier@@UBEPBDXZ 315a42a0 f i Recoil.obj
 0001:000a32b0       ?GetClassID@CFactory@CRecoil@PoseModifier@@UBEABUCryGUID@@XZ 315a42b0 f i Recoil.obj
 0001:000a32c0       ?Execute@CRecoil@PoseModifier@@UAE_NABUSAnimationPoseModifierParams@@@Z 315a42c0 f   Recoil.obj
 0001:000a44e0       ?CreateClassInstance@CFactory@CRecoil@PoseModifier@@UBE?AV?$shared_ptr@UICryUnknown@@@boost@@XZ 315a54e0 f i Recoil.obj
 0001:000a45c0       ?Initialize@CState@Command@@QAE_NPAVCCharInstance@@ABU?$QuatTS_tpl@M@@@Z 315a55c0 f   Command_Buffer.obj
 0001:000a4650       ?Initialize@CBuffer@Command@@QAE_NPAVCCharInstance@@ABU?$QuatTS_tpl@M@@@Z 315a5650 f   Command_Buffer.obj
 0001:000a4690       ?DebugDraw@CBuffer@Command@@AAEXXZ 315a5690 f   Command_Buffer.obj
 0001:000a4a80       ?ProcessAnimationDrivenIk@@YAXAAVCCharInstance@@ABUSAnimationPoseModifierParams@@@Z 315a5a80 f   Command_Buffer.obj
 0001:000a5d10       ?Execute@CBuffer@Command@@QAEXXZ 315a6d10 f   Command_Buffer.obj
 0001:000a60e0       ?Execute@ClearFull@Command@@QBEXABVCState@2@QAPAX@Z 315a70e0 f   Command_Commands.obj
 0001:000a6150       ?Execute@ClearSingle@Command@@QBEXABVCState@2@QAPAX@Z 315a7150 f   Command_Commands.obj
 0001:000a6190       ?Execute@NormalizeFull@Command@@QBEXABVCState@2@QAPAX@Z 315a7190 f   Command_Commands.obj
 0001:000a6340       ?Execute@ScaleUniformFull@Command@@QBEXABVCState@2@QAPAX@Z 315a7340 f   Command_Commands.obj
 0001:000a64b0       ?Execute@CopyAddAnimFull@Command@@QBEXABVCState@2@QAPAX@Z 315a74b0 f   Command_Commands.obj
 0001:000a69c0       ?Execute@SampleAddPoseFull@Command@@QBEXABVCState@2@QAPAX@Z 315a79c0 f   Command_Commands.obj
 0001:000a6d00       ?Execute@SamplePosePart@Command@@QBEXABVCState@2@QAPAX@Z 315a7d00 f   Command_Commands.obj
 0001:000a7070       ?Execute@PoseModifier@Command@@QBEXABVCState@2@QAPAX@Z 315a8070 f   Command_Commands.obj
 0001:000a70f0       ?LoadControllers@Command@@YAXAAUGlobalAnimationHeaderCAF@@ABVCState@1@PAPAVIController@@@Z 315a80f0 f   Command_Commands.obj
 0001:000a7310       ?Execute@SampleAddAnimFull@Command@@QBEXABVCState@2@QAPAX@Z 315a8310 f   Command_Commands.obj
 0001:000a7aa0       ?Execute@SampleAnimPart@Command@@QBEXABVCState@2@QAPAX@Z 315a8aa0 f   Command_Commands.obj
 0001:000a8080       ?AllocationRelease@CPoseData@Skeleton@@QAEXXZ 315a9080 f   Skeleton.obj
 0001:000a80d0       ?GetAllocationLength@CPoseData@Skeleton@@QBEIXZ 315a90d0 f   Skeleton.obj
 0001:000a80e0       ?SetJointRelativeP@CPoseData@Skeleton@@UAEXIABU?$Vec3_tpl@M@@@Z 315a90e0 f   Skeleton.obj
 0001:000a8110       ?GetJointRelative@CPoseData@Skeleton@@UBEABU?$QuatT_tpl@M@@I@Z 315a9110 f   Skeleton.obj
 0001:000a8130       ?SetJointAbsoluteP@CPoseData@Skeleton@@UAEXIABU?$Vec3_tpl@M@@@Z 315a9130 f   Skeleton.obj
 0001:000a8160       ?GetJointAbsolute@CPoseData@Skeleton@@UBEABU?$QuatT_tpl@M@@I@Z 315a9160 f   Skeleton.obj
 0001:000a8180       ?GetParentIndex@CPoseData@Skeleton@@QBEHI@Z 315a9180 f   Skeleton.obj
 0001:000a8190       ??_GIAnimationPoseData@@UAEPAXI@Z 315a9190 f i Skeleton.obj
 0001:000a8190       ??_EIAnimationPoseData@@UAEPAXI@Z 315a9190 f i Skeleton.obj
 0001:000a81c0       ??0CPoseData@Skeleton@@QAE@XZ 315a91c0 f   Skeleton.obj
 0001:000a81e0       ??1CPoseData@Skeleton@@UAE@XZ 315a91e0 f   Skeleton.obj
 0001:000a8230       ?AllocateData@CPoseData@Skeleton@@QAE_NI@Z 315a9230 f   Skeleton.obj
 0001:000a82e0       ?Initialize@CPoseData@Skeleton@@QAE_NABVCModelSkeleton@@I@Z 315a92e0 f   Skeleton.obj
 0001:000a8300       ?SetJointRelativeO@CPoseData@Skeleton@@UAEXIABU?$Quat_tpl@M@@@Z 315a9300 f   Skeleton.obj
 0001:000a8340       ?SetJointAbsoluteO@CPoseData@Skeleton@@UAEXIABU?$Quat_tpl@M@@@Z 315a9340 f   Skeleton.obj
 0001:000a8380       ??_ECPoseData@Skeleton@@UAEPAXI@Z 315a9380 f i Skeleton.obj
 0001:000a8380       ??_GCPoseData@Skeleton@@UAEPAXI@Z 315a9380 f i Skeleton.obj
 0001:000a83e0       ?SetJointRelative@CPoseData@Skeleton@@UAEXIABU?$QuatT_tpl@M@@@Z 315a93e0 f   Skeleton.obj
 0001:000a8430       ?SetJointAbsolute@CPoseData@Skeleton@@UAEXIABU?$QuatT_tpl@M@@@Z 315a9430 f   Skeleton.obj
 0001:000a8480       ?Initialize@CPoseData@Skeleton@@QAE_NABVCModelSkeleton@@@Z 315a9480 f   Skeleton.obj
 0001:000a8530       ?Initialize@CPoseData@Skeleton@@QAE_NABV12@@Z 315a9530 f   Skeleton.obj
 0001:000a85d0       ?ComputeAbsolutePose@CPoseData@Skeleton@@QAEX_N@Z 315a95d0 f   Skeleton.obj
 0001:000a8c50       ?ComputeRelativePose@CPoseData@Skeleton@@QAEX_N@Z 315a9c50 f   Skeleton.obj
 0001:000a93d0       ?ValidateRelative@CPoseData@Skeleton@@QBEXXZ 315aa3d0 f   Skeleton.obj
 0001:000a9900       ?ValidateAbsolute@CPoseData@Skeleton@@QBEXXZ 315aa900 f   Skeleton.obj
 0001:000aa170       ?Validate@CPoseData@Skeleton@@QBEXXZ 315ab170 f   Skeleton.obj
 0001:000aa180       ?SetPreLoadParticleEffects@AnimEventLoader@@YAX_N@Z 315ab180 f   AnimEventLoader.obj
 0001:000aa190       ?DoAdditionalAnimEventInitialization@AnimEventLoader@@YAXPBDAAVCAnimEventData@@@Z 315ab190 f   AnimEventLoader.obj
 0001:000aa1f0       ?LoadAnimationEventDatabase@AnimEventLoader@@YA_NPAVCSkel@@PBD@Z 315ab1f0 f   AnimEventLoader.obj
 0001:000aa500       ?GetIFacialAnimation@CharacterManager@@UAEPAUIFacialAnimation@@XZ 315ab500 f   CharacterManager.obj
 0001:000aa510       ?GetRendererMainThreadId@CharacterManager@@SAIXZ 315ab510 f   CharacterManager.obj
 0001:000aa560       ?UpdateRendererFrame@CharacterManager@@UAEXXZ 315ab560 f   CharacterManager.obj
 0001:000aa570       ?DummyUpdate@CharacterManager@@UAEXXZ 315ab570 f   CharacterManager.obj
 0001:000aa580       ??4?$_smart_ptr@VCSkel@@@@QAEAAV0@ABV0@@Z 315ab580 f i CharacterManager.obj
 0001:000aa580       ??4?$_smart_ptr@VCSkin@@@@QAEAAV0@ABV0@@Z 315ab580 f i CharacterManager.obj
 0001:000aa580       ??4?$_smart_ptr@UIPlaceholderCharacter@@@@QAEAAV0@ABV0@@Z 315ab580 f i CharacterManager.obj
 0001:000aa5b0       ?fxopen@@YAPAU_iobuf@@PBD0_N@Z 315ab5b0 f i CharacterManager.obj
 0001:000aa680       ??_EICharacterManager@@UAEPAXI@Z 315ab680 f i CharacterManager.obj
 0001:000aa680       ??_GICharacterManager@@UAEPAXI@Z 315ab680 f i CharacterManager.obj
 0001:000aa6b0       ?SaveCharacterDefinition@CharacterManager@@UAEIPAUICharacterInstance@@PBD@Z 315ab6b0 f   CharacterManager.obj
 0001:000aa810       ?DBA_PreLoad@CharacterManager@@UAE_NPBDW4EStreamingDBAPriority@ICharacterManager@@@Z 315ab810 f   CharacterManager.obj
 0001:000aa840       ?DBA_LockStatus@CharacterManager@@UAE_NPBDIW4EStreamingDBAPriority@ICharacterManager@@@Z 315ab840 f   CharacterManager.obj
 0001:000aa870       ?DBA_Unload@CharacterManager@@UAE_NPBD@Z 315ab870 f   CharacterManager.obj
 0001:000aa8a0       ?MakeLower@?$CryStackStringT@D$0CAA@@@QAEAAV1@XZ 315ab8a0 f i CharacterManager.obj
 0001:000aa8d0       ??$move_init@UVirtualExampleInit2@CHUNK_GAHAIM_INFO@@@NArray@@YAXPAUVirtualExampleInit2@CHUNK_GAHAIM_INFO@@0I@Z 315ab8d0 f i CharacterManager.obj
 0001:000aa920       ?DeleteDebugInstances@CharacterManager@@UAEXXZ 315ab920 f   CharacterManager.obj
 0001:000aa970       ?GetAverageFrameTime@CharacterManager@@AAEMMMMM@Z 315ab970 f   CharacterManager.obj
 0001:000aaaf0       ?GetDBAFilePathByGlobalID@CharacterManager@@UAEPBDH@Z 315abaf0 f   CharacterManager.obj
 0001:000aab50       ??$_M_find@V?$CryStringT@D@@@?$_Rb_tree@V?$CryStringT@D@@U?$less@V?$CryStringT@D@@@stlpmtx_std@@V1@U?$_Identity@V?$CryStringT@D@@@priv@3@U?$_SetTraitsT@V?$CryStringT@D@@@53@V?$allocator@V?$CryStringT@D@@@3@@priv@stlpmtx_std@@ABEPAU_Rb_tree_node_base@12@ABV?$CryStringT@D@@@Z 315abb50 f i CharacterManager.obj
 0001:000aabf0       ?FindAimposeByGlobalID@CAnimationSet@@QAEHI@Z 315abbf0 f i CharacterManager.obj
 0001:000aac40       ?resize_raw@?$SmallDynStorage@IHUStandardAlloc@NAlloc@@@NArray@@QAEXHH_N@Z 315abc40 f i CharacterManager.obj
 0001:000aad90       ??$UnifyFilePath@$0CAA@@CryStringUtils@@YAXAAV?$CryStackStringT@D$0CAA@@@@Z 315abd90 f i CharacterManager.obj
 0001:000aadd0       ??4CharacterAttachment@@QAEAAU0@ABU0@@Z 315abdd0 f i CharacterManager.obj
 0001:000aaf60       ?set_size@?$SmallDynStorage@UBSParameter@@HUStandardAlloc@NAlloc@@@NArray@@QAEXH@Z 315abf60 f i CharacterManager.obj
 0001:000aaf60       ?set_size@?$SmallDynStorage@VCAnimEventData@@HUStandardAlloc@NAlloc@@@NArray@@QAEXH@Z 315abf60 f i AnimEventList.obj
 0001:000aaff0       ?resize_raw@?$SmallDynStorage@UBSBlendable@@HUStandardAlloc@NAlloc@@@NArray@@QAEXHH_N@Z 315abff0 f i CharacterManager.obj
 0001:000ab150       ?set_size@?$SmallDynStorage@USVertexFrameState@@HUStandardAlloc@NAlloc@@@NArray@@QAEXH@Z 315ac150 f i VertexAnimation.obj
 0001:000ab150       ?set_size@?$SmallDynStorage@UIdxAndName@@HUStandardAlloc@NAlloc@@@NArray@@QAEXH@Z 315ac150 f i ParamLoader.obj
 0001:000ab150       ?set_size@?$SmallDynStorage@USCRCName@@HUStandardAlloc@NAlloc@@@NArray@@QAEXH@Z 315ac150 f i CharacterManager.obj
 0001:000ab150       ?set_size@?$SmallDynStorage@UBoneIndices8@@HUStandardAlloc@NAlloc@@@NArray@@QAEXH@Z 315ac150 f i LoaderSKIN.obj
 0001:000ab150       ?set_size@?$SmallDynStorage@UAimIKPose@@HUStandardAlloc@NAlloc@@@NArray@@QAEXH@Z 315ac150 f i CharacterManager.obj
 0001:000ab1d0       ?resize_raw@?$SmallDynStorage@UVirtualExampleInit2@CHUNK_GAHAIM_INFO@@HUStandardAlloc@NAlloc@@@NArray@@QAEXHH_N@Z 315ac1d0 f i CharacterManager.obj
 0001:000ab340       ?SetFilePath@CCharInstance@@QAEXABV?$CryStringT@D@@@Z 315ac340 f i CharacterManager.obj
 0001:000ab3a0       ?CheckIfModelSKELLoaded@CharacterManager@@QAEPAVCSkel@@ABV?$CryStringT@D@@I@Z 315ac3a0 f   CharacterManager.obj
 0001:000ab450       ?CheckIfModelSKINLoaded@CharacterManager@@QAEPAVCSkin@@ABV?$CryStringT@D@@I@Z 315ac450 f   CharacterManager.obj
 0001:000ab510       ?GetStatistics@CharacterManager@@UAEXAAUStatistics@ICharacterManager@@@Z 315ac510 f   CharacterManager.obj
 0001:000ab560       ?GetCharacterInstancesSize@CharacterManager@@QBEXPAVICrySizer@@@Z 315ac560 f   CharacterManager.obj
 0001:000ab600       ?GetModelByAimPoseID@CharacterManager@@QAEPAVCSkel@@I@Z 315ac600 f   CharacterManager.obj
 0001:000ab830       ?TrackSkinTransMemory@CharacterManager@@AAEIAAV?$vector@PAVCSkel@@V?$allocator@PAVCSkel@@@stlpmtx_std@@@stlpmtx_std@@AAV?$vector@PAVCSkin@@V?$allocator@PAVCSkin@@@stlpmtx_std@@@3@@Z 315ac830 f   CharacterManager.obj
 0001:000ab940       ?DebugModelCache@CharacterManager@@AAEXIAAV?$vector@PAVCSkel@@V?$allocator@PAVCSkel@@@stlpmtx_std@@@stlpmtx_std@@AAV?$vector@PAVCSkin@@V?$allocator@PAVCSkin@@@stlpmtx_std@@@3@@Z 315ac940 f   CharacterManager.obj
 0001:000ac360       ?GetAnimationSetUsedInCharEdit@CharacterManager@@QAEPAVCAnimationSet@@XZ 315ad360 f   CharacterManager.obj
 0001:000ac4b0       ?DatabaseUnloading@CharacterManager@@QAEXXZ 315ad4b0 f   CharacterManager.obj
 0001:000ac880       ?SaveCAF@CAnimationStatsResourceList@@QAEXXZ 315ad880 f i CharacterManager.obj
 0001:000ac9c0       ?SaveLMG@CAnimationStatsResourceList@@QAEXXZ 315ad9c0 f i CharacterManager.obj
 0001:000acad0       ?GetLoadedModels@CharacterManager@@UAEXPAPAUICharacterModel@@AAH@Z 315adad0 f   CharacterManager.obj
 0001:000acb20       ?set_size@?$SmallDynStorage@UGlobalAnimationHeaderCAF@@HUStandardAlloc@NAlloc@@@NArray@@QAEXH@Z 315adb20 f i CharacterManager.obj
 0001:000acbb0       ?set_size@?$SmallDynStorage@UGlobalAnimationHeaderAIM@@HUStandardAlloc@NAlloc@@@NArray@@QAEXH@Z 315adbb0 f i CharacterManager.obj
 0001:000acc40       ?set_size@?$SmallDynStorage@UDebugInstances@@HUStandardAlloc@NAlloc@@@NArray@@QAEXH@Z 315adc40 f i CharacterManager.obj
 0001:000acc40       ?set_size@?$SmallDynStorage@UCryTCB3Key@@HUStandardAlloc@NAlloc@@@NArray@@QAEXH@Z 315adc40 f i LoaderTCB.obj
 0001:000accd0       ??$AddObject@PAVCSkel@@V?$allocator@PAVCSkel@@@stlpmtx_std@@@ICrySizer@@QAEXABV?$vector@PAVCSkel@@V?$allocator@PAVCSkel@@@stlpmtx_std@@@stlpmtx_std@@@Z 315adcd0 f i CharacterManager.obj
 0001:000acd40       ?_M_create_node@?$_Rb_tree@IU?$less@I@stlpmtx_std@@U?$pair@$$CBIV?$_smart_ptr@UIPlaceholderCharacter@@@@@2@U?$_Select1st@U?$pair@$$CBIV?$_smart_ptr@UIPlaceholderCharacter@@@@@stlpmtx_std@@@priv@2@U?$_MapTraitsT@U?$pair@$$CBIV?$_smart_ptr@UIPlaceholderCharacter@@@@@stlpmtx_std@@@52@V?$allocator@U?$pair@$$CBIV?$_smart_ptr@UIPlaceholderCharacter@@@@@stlpmtx_std@@@2@@priv@stlpmtx_std@@IAEPAU_Rb_tree_node_base@23@ABU?$pair@$$CBIV?$_smart_ptr@UIPlaceholderCharacter@@@@@3@@Z 315add40 f i CharacterManager.obj
 0001:000acda0       ?_M_create_node@?$_Rb_tree@V?$CryStringT@D@@U?$less@V?$CryStringT@D@@@stlpmtx_std@@V1@U?$_Identity@V?$CryStringT@D@@@priv@3@U?$_SetTraitsT@V?$CryStringT@D@@@53@V?$allocator@V?$CryStringT@D@@@3@@priv@stlpmtx_std@@IAEPAU_Rb_tree_node_base@23@ABV?$CryStringT@D@@@Z 315adda0 f i CharacterManager.obj
 0001:000ace00       ?SetFilePathCAF@GlobalAnimationHeaderCAF@@QAEXABV?$CryStringT@D@@@Z 315ade00 f i CharacterManager.obj
 0001:000ace00       ?SetFilePath@GlobalAnimationHeaderAIM@@QAEXABV?$CryStringT@D@@@Z 315ade00 f i AnimationManager.obj
 0001:000acef0       ?clear@?$_Rb_tree@IU?$less@I@stlpmtx_std@@U?$pair@$$CBIUSFacialDisplaceInfo@CFacialModel@@@2@U?$_Select1st@U?$pair@$$CBIUSFacialDisplaceInfo@CFacialModel@@@stlpmtx_std@@@priv@2@U?$_MapTraitsT@U?$pair@$$CBIUSFacialDisplaceInfo@CFacialModel@@@stlpmtx_std@@@52@V?$allocator@U?$pair@$$CBIUSFacialDisplaceInfo@CFacialModel@@@stlpmtx_std@@@2@@priv@stlpmtx_std@@QAEXXZ 315adef0 f i SkeletonAnim.obj
 0001:000acef0       ?clear@?$_Rb_tree@HU?$less@H@stlpmtx_std@@U?$pair@$$CBHPAUphys_geometry@@@2@U?$_Select1st@U?$pair@$$CBHPAUphys_geometry@@@stlpmtx_std@@@priv@2@U?$_MapTraitsT@U?$pair@$$CBHPAUphys_geometry@@@stlpmtx_std@@@52@V?$allocator@U?$pair@$$CBHPAUphys_geometry@@@stlpmtx_std@@@2@@priv@stlpmtx_std@@QAEXXZ 315adef0 f i LoaderCHR.obj
 0001:000acef0       ?clear@?$_Rb_tree@PAUIFacialEffector@@U?$less@PAUIFacialEffector@@@stlpmtx_std@@U?$pair@QAUIFacialEffector@@PAU1@@3@U?$_Select1st@U?$pair@QAUIFacialEffector@@PAU1@@stlpmtx_std@@@priv@3@U?$_MapTraitsT@U?$pair@QAUIFacialEffector@@PAU1@@stlpmtx_std@@@63@V?$allocator@U?$pair@QAUIFacialEffector@@PAU1@@stlpmtx_std@@@3@@priv@stlpmtx_std@@QAEXXZ 315adef0 f i FaceEffectorLibrary.obj
 0001:000acef0       ?clear@?$_Rb_tree@IU?$less@I@stlpmtx_std@@U?$pair@$$CBIPAV?$vector@IV?$allocator@I@stlpmtx_std@@@stlpmtx_std@@@2@U?$_Select1st@U?$pair@$$CBIPAV?$vector@IV?$allocator@I@stlpmtx_std@@@stlpmtx_std@@@stlpmtx_std@@@priv@2@U?$_MapTraitsT@U?$pair@$$CBIPAV?$vector@IV?$allocator@I@stlpmtx_std@@@stlpmtx_std@@@stlpmtx_std@@@52@V?$allocator@U?$pair@$$CBIPAV?$vector@IV?$allocator@I@stlpmtx_std@@@stlpmtx_std@@@stlpmtx_std@@@2@@priv@stlpmtx_std@@QAEXXZ 315adef0 f i CharacterManager.obj
 0001:000acef0       ?clear@?$_Rb_tree@IU?$less@I@stlpmtx_std@@U?$pair@$$CBIPAV?$vector@HV?$allocator@H@stlpmtx_std@@@stlpmtx_std@@@2@U?$_Select1st@U?$pair@$$CBIPAV?$vector@HV?$allocator@H@stlpmtx_std@@@stlpmtx_std@@@stlpmtx_std@@@priv@2@U?$_MapTraitsT@U?$pair@$$CBIPAV?$vector@HV?$allocator@H@stlpmtx_std@@@stlpmtx_std@@@stlpmtx_std@@@52@V?$allocator@U?$pair@$$CBIPAV?$vector@HV?$allocator@H@stlpmtx_std@@@stlpmtx_std@@@stlpmtx_std@@@2@@priv@stlpmtx_std@@QAEXXZ 315adef0 f i CharacterManager.obj
 0001:000acef0       ?clear@?$_Rb_tree@IU?$less@I@stlpmtx_std@@U?$pair@$$CBII@2@U?$_Select1st@U?$pair@$$CBII@stlpmtx_std@@@priv@2@U?$_MapTraitsT@U?$pair@$$CBII@stlpmtx_std@@@52@V?$allocator@U?$pair@$$CBII@stlpmtx_std@@@2@@priv@stlpmtx_std@@QAEXXZ 315adef0 f i CharacterManager.obj
 0001:000acef0       ?clear@?$_Rb_tree@HU?$less@H@stlpmtx_std@@HU?$_Identity@H@priv@2@U?$_SetTraitsT@H@42@V?$allocator@H@2@@priv@stlpmtx_std@@QAEXXZ 315adef0 f i LoaderCGA.obj
 0001:000acf40       ?expand_raw@?$DynArray@IHU?$SmallDynStorage@IHUStandardAlloc@NAlloc@@@NArray@@@@IAEPAIPAIH@Z 315adf40 f i CharacterManager.obj
 0001:000acfc0       ?get_alloc_size@?$SmallDynStorage@UCharacterAttachment@@HUStandardAlloc@NAlloc@@@NArray@@QBEHXZ 315adfc0 f i CharacterManager.obj
 0001:000ad010       ?init@?$DynArray@VCAnimEventData@@HU?$SmallDynStorage@VCAnimEventData@@HUStandardAlloc@NAlloc@@@NArray@@@@KAPAVCAnimEventData@@U?$Array@VCAnimEventData@@HU?$ArrayStorage@VCAnimEventData@@H@NArray@@@@PBV2@@Z 315ae010 f i CharacterManager.obj
 0001:000ad0f0       ?init@?$DynArray@UBlendSpaceInfo@@HU?$SmallDynStorage@UBlendSpaceInfo@@HUStandardAlloc@NAlloc@@@NArray@@@@KAPAUBlendSpaceInfo@@U?$Array@UBlendSpaceInfo@@HU?$ArrayStorage@UBlendSpaceInfo@@H@NArray@@@@PBU2@@Z 315ae0f0 f i CharacterManager.obj
 0001:000ad140       ?init@?$DynArray@USCRCName@@HU?$SmallDynStorage@USCRCName@@HUStandardAlloc@NAlloc@@@NArray@@@@KAPAUSCRCName@@U?$Array@USCRCName@@HU?$ArrayStorage@USCRCName@@H@NArray@@@@PBU2@@Z 315ae140 f i CharacterManager.obj
 0001:000ad190       ?init@?$DynArray@UCharacterAttachment@@HU?$SmallDynStorage@UCharacterAttachment@@HUStandardAlloc@NAlloc@@@NArray@@@@KAPAUCharacterAttachment@@U?$Array@UCharacterAttachment@@HU?$ArrayStorage@UCharacterAttachment@@H@NArray@@@@PBU2@@Z 315ae190 f i CharacterManager.obj
 0001:000ad2d0       ??0BSParameter@@QAE@ABU0@@Z 315ae2d0 f i CharacterManager.obj
 0001:000ad340       ?expand_raw@?$DynArray@UBSBlendable@@HU?$SmallDynStorage@UBSBlendable@@HUStandardAlloc@NAlloc@@@NArray@@@@IAEPAUBSBlendable@@PAU2@H@Z 315ae340 f i CharacterManager.obj
 0001:000ad3d0       ?expand_raw@?$DynArray@V?$_smart_ptr@VIController@@@@HU?$SmallDynStorage@V?$_smart_ptr@VIController@@@@HUStandardAlloc@NAlloc@@@NArray@@@@IAEPAV?$_smart_ptr@VIController@@@@PAV2@H@Z 315ae3d0 f i CharacterManager.obj
 0001:000ad450       ?expand_raw@?$DynArray@UVirtualExampleInit2@CHUNK_GAHAIM_INFO@@HU?$SmallDynStorage@UVirtualExampleInit2@CHUNK_GAHAIM_INFO@@HUStandardAlloc@NAlloc@@@NArray@@@@IAEPAUVirtualExampleInit2@CHUNK_GAHAIM_INFO@@PAU23@H@Z 315ae450 f i CharacterManager.obj
 0001:000ad4f0       ?CheckIfPlaceholderCharacterLoaded@CharacterManager@@QBE?AV?$_smart_ptr@UIPlaceholderCharacter@@@@PBD@Z 315ae4f0 f   CharacterManager.obj
 0001:000ad5b0       ?UnregisterModelSKEL@CharacterManager@@QAEXPAVCSkel@@@Z 315ae5b0 f   CharacterManager.obj
 0001:000ad750       ?UnregisterModelSKIN@CharacterManager@@QAEXPAVCSkin@@@Z 315ae750 f   CharacterManager.obj
 0001:000ad8f0       ?TrackMemoryOfModels@CharacterManager@@QAEXXZ 315ae8f0 f   CharacterManager.obj
 0001:000ad920       ?UnifyFilename@CAnimationStatsResourceList@@QAE?AV?$CryStackStringT@D$0CAA@@@PBD@Z 315ae920 f i CharacterManager.obj
 0001:000ad980       ?ClearPoseModifiersFromSynchQueue@CharacterManager@@AAEXXZ 315ae980 f   CharacterManager.obj
 0001:000ada60       ?PreloadModelsCHR@CharacterManager@@AAEXXZ 315aea60 f   CharacterManager.obj
 0001:000adfa0       ?Enable@CLogIndenter@@QAAX_NPBDZZ 315aefa0 f i CharacterManager.obj
 0001:000ae040       ?_M_erase@?$_Rb_tree@IU?$less@I@stlpmtx_std@@U?$pair@$$CBIV?$_smart_ptr@UIPlaceholderCharacter@@@@@2@U?$_Select1st@U?$pair@$$CBIV?$_smart_ptr@UIPlaceholderCharacter@@@@@stlpmtx_std@@@priv@2@U?$_MapTraitsT@U?$pair@$$CBIV?$_smart_ptr@UIPlaceholderCharacter@@@@@stlpmtx_std@@@52@V?$allocator@U?$pair@$$CBIV?$_smart_ptr@UIPlaceholderCharacter@@@@@stlpmtx_std@@@2@@priv@stlpmtx_std@@AAEXPAU_Rb_tree_node_base@23@@Z 315af040 f i CharacterManager.obj
 0001:000ae090       ??$move_init@UDebugInstances@@@NArray@@YAXPAUDebugInstances@@0I@Z 315af090 f i CharacterManager.obj
 0001:000ae130       ?_M_fill_insert_aux@?$_Impl_vector@HV?$allocator@H@stlpmtx_std@@@priv@stlpmtx_std@@AAEXPAHIABHABU__false_type@3@@Z 315af130 f i ControllerDefragHeap.obj
 0001:000ae130       ?_M_fill_insert_aux@?$_Impl_vector@IV?$allocator@I@stlpmtx_std@@@priv@stlpmtx_std@@AAEXPAIIABIABU__false_type@3@@Z 315af130 f i CharacterManager.obj
 0001:000ae130       ?_M_fill_insert_aux@?$_Impl_vector@PAXV?$allocator@PAX@stlpmtx_std@@@priv@stlpmtx_std@@AAEXPAPAXIABQAXABU__false_type@3@@Z 315af130 f i LoaderSKIN.obj
 0001:000ae270       ?_M_insert@?$_Rb_tree@V?$CryStringT@D@@U?$less@V?$CryStringT@D@@@stlpmtx_std@@V1@U?$_Identity@V?$CryStringT@D@@@priv@3@U?$_SetTraitsT@V?$CryStringT@D@@@53@V?$allocator@V?$CryStringT@D@@@3@@priv@stlpmtx_std@@AAE?AU?$_Rb_tree_iterator@V?$CryStringT@D@@U?$_SetTraitsT@V?$CryStringT@D@@@priv@stlpmtx_std@@@23@PAU_Rb_tree_node_base@23@ABV?$CryStringT@D@@00@Z 315af270 f i CharacterManager.obj
 0001:000ae310       ??$_M_find@V?$CryStackStringT@D$0CAA@@@@?$_Rb_tree@V?$CryStringT@D@@U?$less@V?$CryStringT@D@@@stlpmtx_std@@V1@U?$_Identity@V?$CryStringT@D@@@priv@3@U?$_SetTraitsT@V?$CryStringT@D@@@53@V?$allocator@V?$CryStringT@D@@@3@@priv@stlpmtx_std@@ABEPAU_Rb_tree_node_base@12@ABV?$CryStackStringT@D$0CAA@@@@Z 315af310 f i CharacterManager.obj
 0001:000ae480       ?destroy@?$DynArray@USCRCName@@HU?$SmallDynStorage@USCRCName@@HUStandardAlloc@NAlloc@@@NArray@@@@KAXU?$Array@USCRCName@@HU?$ArrayStorage@USCRCName@@H@NArray@@@@@Z 315af480 f i CharacterManager.obj
 0001:000ae4d0       ??$AddObject@UCharacterAttachment@@HU?$SmallDynStorage@UCharacterAttachment@@HUStandardAlloc@NAlloc@@@NArray@@@ICrySizer@@QAEXABU?$DynArray@UCharacterAttachment@@HU?$SmallDynStorage@UCharacterAttachment@@HUStandardAlloc@NAlloc@@@NArray@@@@@Z 315af4d0 f i CharacterManager.obj
 0001:000ae5a0       ?init@?$DynArray@UBSParameter@@HU?$SmallDynStorage@UBSParameter@@HUStandardAlloc@NAlloc@@@NArray@@@@KAPAUBSParameter@@U?$Array@UBSParameter@@HU?$ArrayStorage@UBSParameter@@H@NArray@@@@PBU2@@Z 315af5a0 f i CharacterManager.obj
 0001:000ae640       ??$move_init@USCRCName@@@NArray@@YAXPAUSCRCName@@0I@Z 315af640 f i CharacterManager.obj
 0001:000ae6d0       ?StopAnimationsOnAllInstances@CharacterManager@@QAEXXZ 315af6d0 f   CharacterManager.obj
 0001:000ae990       ?RemoveAnimationToSyncQueue@CharacterManager@@UAEXPAUICharacterInstance@@@Z 315af990 f   CharacterManager.obj
 0001:000aea90       ?DBA_Unload_All@CharacterManager@@UAE_NXZ 315afa90 f   CharacterManager.obj
 0001:000aeac0       ?CAF_AddRef@CharacterManager@@UAE_NI@Z 315afac0 f   CharacterManager.obj
 0001:000aeb60       ?CAF_IsLoaded@CharacterManager@@UBE_NI@Z 315afb60 f   CharacterManager.obj
 0001:000aebf0       ?CAF_Release@CharacterManager@@UAE_NI@Z 315afbf0 f   CharacterManager.obj
 0001:000aec70       ?CAF_LoadSynchronously@CharacterManager@@UAE_NI@Z 315afc70 f   CharacterManager.obj
 0001:000aed30       ??1?$DynArray@UDebugInstances@@HU?$SmallDynStorage@UDebugInstances@@HUStandardAlloc@NAlloc@@@NArray@@@@QAE@XZ 315afd30 f i CharacterManager.obj
 0001:000aed90       ??1?$DynArray@VTCBAngleAxisSpline@spline@@HU?$SmallDynStorage@VTCBAngleAxisSpline@spline@@HUStandardAlloc@NAlloc@@@NArray@@@@QAE@XZ 315afd90 f i CharacterManager.obj
 0001:000aed90       ??1?$DynArray@V?$TCBSpline@U?$Vec3_tpl@M@@U?$TCBSplineKey@U?$Vec3_tpl@M@@@spline@@@spline@@HU?$SmallDynStorage@V?$TCBSpline@U?$Vec3_tpl@M@@U?$TCBSplineKey@U?$Vec3_tpl@M@@@spline@@@spline@@HUStandardAlloc@NAlloc@@@NArray@@@@QAE@XZ 315afd90 f i CharacterManager.obj
 0001:000aedf0       ??1?$DynArray@UCControllerTCB@@HU?$SmallDynStorage@UCControllerTCB@@HUStandardAlloc@NAlloc@@@NArray@@@@QAE@XZ 315afdf0 f i CharacterManager.obj
 0001:000aee50       ?erase@?$_Rb_tree@V?$CryStringT@D@@U?$less@V?$CryStringT@D@@@stlpmtx_std@@V1@U?$_Identity@V?$CryStringT@D@@@priv@3@U?$_SetTraitsT@V?$CryStringT@D@@@53@V?$allocator@V?$CryStringT@D@@@3@@priv@stlpmtx_std@@QAEXU?$_Rb_tree_iterator@V?$CryStringT@D@@U?$_SetTraitsT@V?$CryStringT@D@@@priv@stlpmtx_std@@@23@@Z 315afe50 f i CharacterManager.obj
 0001:000aeec0       ?resize_raw@?$SmallDynStorage@UDebugInstances@@HUStandardAlloc@NAlloc@@@NArray@@QAEXHH_N@Z 315afec0 f i CharacterManager.obj
 0001:000af020       ?_M_erase@?$_Rb_tree@V?$CryStringT@D@@U?$less@V?$CryStringT@D@@@stlpmtx_std@@V1@U?$_Identity@V?$CryStringT@D@@@priv@3@U?$_SetTraitsT@V?$CryStringT@D@@@53@V?$allocator@V?$CryStringT@D@@@3@@priv@stlpmtx_std@@AAEXPAU_Rb_tree_node_base@23@@Z 315b0020 f i CharacterManager.obj
 0001:000af080       ?insert_unique@?$_Rb_tree@V?$CryStringT@D@@U?$less@V?$CryStringT@D@@@stlpmtx_std@@V1@U?$_Identity@V?$CryStringT@D@@@priv@3@U?$_SetTraitsT@V?$CryStringT@D@@@53@V?$allocator@V?$CryStringT@D@@@3@@priv@stlpmtx_std@@QAE?AU?$pair@U?$_Rb_tree_iterator@V?$CryStringT@D@@U?$_SetTraitsT@V?$CryStringT@D@@@priv@stlpmtx_std@@@priv@stlpmtx_std@@_N@3@ABV?$CryStringT@D@@@Z 315b0080 f i CharacterManager.obj
 0001:000af200       ?insert_unique@?$_Rb_tree@IU?$less@I@stlpmtx_std@@U?$pair@$$CBIV?$_smart_ptr@UIPlaceholderCharacter@@@@@2@U?$_Select1st@U?$pair@$$CBIV?$_smart_ptr@UIPlaceholderCharacter@@@@@stlpmtx_std@@@priv@2@U?$_MapTraitsT@U?$pair@$$CBIV?$_smart_ptr@UIPlaceholderCharacter@@@@@stlpmtx_std@@@52@V?$allocator@U?$pair@$$CBIV?$_smart_ptr@UIPlaceholderCharacter@@@@@stlpmtx_std@@@2@@priv@stlpmtx_std@@QAE?AU?$pair@U?$_Rb_tree_iterator@U?$pair@$$CBIV?$_smart_ptr@UIPlaceholderCharacter@@@@@stlpmtx_std@@U?$_MapTraitsT@U?$pair@$$CBIV?$_smart_ptr@UIPlaceholderCharacter@@@@@stlpmtx_std@@@priv@2@@priv@stlpmtx_std@@_N@3@ABU?$pair@$$CBIV?$_smart_ptr@UIPlaceholderCharacter@@@@@3@@Z 315b0200 f i CharacterManager.obj
 0001:000af310       ??1?$DynArray@UCGlobalHeaderDBA@@HU?$SmallDynStorage@UCGlobalHeaderDBA@@HUStandardAlloc@NAlloc@@@NArray@@@@QAE@XZ 315b0310 f i CharacterManager.obj
 0001:000af370       ?resize_raw@?$SmallDynStorage@UCGlobalHeaderDBA@@HUStandardAlloc@NAlloc@@@NArray@@QAEXHH_N@Z 315b0370 f i CharacterManager.obj
 0001:000af4d0       ?destroy@?$DynArray@UBSParameter@@HU?$SmallDynStorage@UBSParameter@@HUStandardAlloc@NAlloc@@@NArray@@@@KAXU?$Array@UBSParameter@@HU?$ArrayStorage@UBSParameter@@H@NArray@@@@@Z 315b04d0 f i CharacterManager.obj
 0001:000af520       ??0?$DynArray@IHU?$SmallDynStorage@IHUStandardAlloc@NAlloc@@@NArray@@@@QAE@ABU0@@Z 315b0520 f i CharacterManager.obj
 0001:000af5b0       ?push_back@?$DynArray@V?$_smart_ptr@VIController@@@@HU?$SmallDynStorage@V?$_smart_ptr@VIController@@@@HUStandardAlloc@NAlloc@@@NArray@@@@QAEPAV?$_smart_ptr@VIController@@@@U?$Array@$$CBV?$_smart_ptr@VIController@@@@HU?$ArrayStorage@$$CBV?$_smart_ptr@VIController@@@@H@NArray@@@@@Z 315b05b0 f i CharacterManager.obj
 0001:000af610       ?push_back@?$DynArray@UVirtualExampleInit2@CHUNK_GAHAIM_INFO@@HU?$SmallDynStorage@UVirtualExampleInit2@CHUNK_GAHAIM_INFO@@HUStandardAlloc@NAlloc@@@NArray@@@@QAEPAUVirtualExampleInit2@CHUNK_GAHAIM_INFO@@U?$Array@$$CBUVirtualExampleInit2@CHUNK_GAHAIM_INFO@@HU?$ArrayStorage@$$CBUVirtualExampleInit2@CHUNK_GAHAIM_INFO@@H@NArray@@@@@Z 315b0610 f i CharacterManager.obj
 0001:000af680       ?resize_raw@?$SmallDynStorage@USCRCName@@HUStandardAlloc@NAlloc@@@NArray@@QAEXHH_N@Z 315b0680 f i CharacterManager.obj
 0001:000af7d0       ??$move_init@UBSParameter@@@NArray@@YAXPAUBSParameter@@0I@Z 315b07d0 f i CharacterManager.obj
 0001:000af840       ??$move_init@UBlendSpaceInfo@@@NArray@@YAXPAUBlendSpaceInfo@@0I@Z 315b0840 f i CharacterManager.obj
 0001:000af8c0       ??1CryCGALoader@@QAE@XZ    315b08c0 f i CharacterManager.obj
 0001:000af960       ??1?$_Impl_vector@UCharacterDefinition@@V?$allocator@UCharacterDefinition@@@stlpmtx_std@@@priv@stlpmtx_std@@QAE@XZ 315b0960 f i CharacterManager.obj
 0001:000af9b0       ?expand_raw@?$DynArray@UDebugInstances@@HU?$SmallDynStorage@UDebugInstances@@HUStandardAlloc@NAlloc@@@NArray@@@@IAEPAUDebugInstances@@PAU2@H@Z 315b09b0 f i CharacterManager.obj
 0001:000afa40       ??1GlobalAnimationHeaderCAF@@QAE@XZ 315b0a40 f i CharacterManager.obj
 0001:000afaf0       ??0AnimSearchHelper@@QAE@XZ 315b0af0 f i CharacterManager.obj
 0001:000afb60       ??0?$DynArray@UBSBlendable@@HU?$SmallDynStorage@UBSBlendable@@HUStandardAlloc@NAlloc@@@NArray@@@@QAE@ABU0@@Z 315b0b60 f i CharacterManager.obj
 0001:000afc00       ??0?$DynArray@UVirtualExample1D@@HU?$SmallDynStorage@UVirtualExample1D@@HUStandardAlloc@NAlloc@@@NArray@@@@QAE@ABU0@@Z 315b0c00 f i CharacterManager.obj
 0001:000afca0       ??0?$DynArray@UVirtualExample2D@@HU?$SmallDynStorage@UVirtualExample2D@@HUStandardAlloc@NAlloc@@@NArray@@@@QAE@ABU0@@Z 315b0ca0 f i CharacterManager.obj
 0001:000afd20       ??0?$DynArray@UVirtualExample3D@@HU?$SmallDynStorage@UVirtualExample3D@@HUStandardAlloc@NAlloc@@@NArray@@@@QAE@ABU0@@Z 315b0d20 f i CharacterManager.obj
 0001:000afdd0       ?erase@?$DynArray@UCharacterAttachment@@HU?$SmallDynStorage@UCharacterAttachment@@HUStandardAlloc@NAlloc@@@NArray@@@@QAEPAUCharacterAttachment@@PAU2@0@Z 315b0dd0 f i CharacterManager.obj
 0001:000afe80       ?expand_raw@?$DynArray@USCRCName@@HU?$SmallDynStorage@USCRCName@@HUStandardAlloc@NAlloc@@@NArray@@@@IAEPAUSCRCName@@PAU2@H@Z 315b0e80 f i CharacterManager.obj
 0001:000aff00       ?resize_raw@?$SmallDynStorage@UBSParameter@@HUStandardAlloc@NAlloc@@@NArray@@QAEXHH_N@Z 315b0f00 f i CharacterManager.obj
 0001:000b0060       ?resize_raw@?$SmallDynStorage@UBlendSpaceInfo@@HUStandardAlloc@NAlloc@@@NArray@@QAEXHH_N@Z 315b1060 f i CharacterManager.obj
 0001:000b01c0       ??0CryCGALoader@@QAE@XZ    315b11c0 f i CharacterManager.obj
 0001:000b0310       ?RegisterModelSKEL@CharacterManager@@QAEXPAVCSkel@@I@Z 315b1310 f   CharacterManager.obj
 0001:000b0410       ?RegisterModelSKIN@CharacterManager@@QAEXPAVCSkin@@I@Z 315b1410 f   CharacterManager.obj
 0001:000b0510       ?ReloadAllCHRPARAMS@CharacterManager@@AAEXXZ 315b1510 f   CharacterManager.obj
 0001:000b0880       ?Add@CAnimationStatsResourceList@@QAEXPBD@Z 315b1880 f i CharacterManager.obj
 0001:000b0960       ?IsExist@CAnimationStatsResourceList@@QAE_NPBD@Z 315b1960 f i CharacterManager.obj
 0001:000b09f0       ?LoadCAF@CAnimationStatsResourceList@@QAEXPBD@Z 315b19f0 f i CharacterManager.obj
 0001:000b0ad0       ?LoadLMG@CAnimationStatsResourceList@@QAEXPBD@Z 315b1ad0 f i CharacterManager.obj
 0001:000b0bb0       ?SyncAllAnimations@CharacterManager@@UAEXXZ 315b1bb0 f   CharacterManager.obj
 0001:000b0d00       ?AddAnimationToSyncQueue@CharacterManager@@UAEXPAUICharacterInstance@@@Z 315b1d00 f   CharacterManager.obj
 0001:000b0d60       ?PreloadModelsCGA@CharacterManager@@AAEXXZ 315b1d60 f   CharacterManager.obj
 0001:000b1110       ?resize@?$_Impl_vector@IV?$allocator@I@stlpmtx_std@@@priv@stlpmtx_std@@QAEXIABI@Z 315b2110 f i CharacterManager.obj
 0001:000b1110       ?resize@?$_Impl_vector@PAXV?$allocator@PAX@stlpmtx_std@@@priv@stlpmtx_std@@QAEXIABQAX@Z 315b2110 f i LoaderSKIN.obj
 0001:000b1110       ?resize@?$_Impl_vector@HV?$allocator@H@stlpmtx_std@@@priv@stlpmtx_std@@QAEXIABH@Z 315b2110 f i ControllerDefragHeap.obj
 0001:000b11b0       ??$AddObject@UCharacterDefinition@@V?$allocator@UCharacterDefinition@@@stlpmtx_std@@@ICrySizer@@QAEXABV?$vector@UCharacterDefinition@@V?$allocator@UCharacterDefinition@@@stlpmtx_std@@@stlpmtx_std@@@Z 315b21b0 f i CharacterManager.obj
 0001:000b1260       ??0GlobalAnimationHeaderCAF@@QAE@XZ 315b2260 f i CharacterManager.obj
 0001:000b1380       ??4?$DynArray@UCharacterAttachment@@HU?$SmallDynStorage@UCharacterAttachment@@HUStandardAlloc@NAlloc@@@NArray@@@@QAEAAU0@U?$Array@$$CBUCharacterAttachment@@HU?$ArrayStorage@$$CBUCharacterAttachment@@H@NArray@@@@@Z 315b2380 f i CharacterManager.obj
 0001:000b1470       ?expand_raw@?$DynArray@UBSParameter@@HU?$SmallDynStorage@UBSParameter@@HUStandardAlloc@NAlloc@@@NArray@@@@IAEPAUBSParameter@@PAU2@H@Z 315b2470 f i CharacterManager.obj
 0001:000b1500       ?expand_raw@?$DynArray@UBlendSpaceInfo@@HU?$SmallDynStorage@UBlendSpaceInfo@@HUStandardAlloc@NAlloc@@@NArray@@@@IAEPAUBlendSpaceInfo@@PAU2@H@Z 315b2500 f i CharacterManager.obj
 0001:000b1590       ?FetchModelSKIN@CharacterManager@@QAE?AV?$_smart_ptr@VCSkin@@@@PBDI@Z 315b2590 f   CharacterManager.obj
 0001:000b1600       ?GetMemoryUsage@CharacterManager@@UBEXPAVICrySizer@@@Z 315b2600 f   CharacterManager.obj
 0001:000b1730       ?Remove@CAnimationStatsResourceList@@QAEXPBD@Z 315b2730 f i CharacterManager.obj
 0001:000b1820       ?init@?$DynArray@UAimIKPose@@HU?$SmallDynStorage@UAimIKPose@@HUStandardAlloc@NAlloc@@@NArray@@@@KAPAUAimIKPose@@U?$Array@UAimIKPose@@HU?$ArrayStorage@UAimIKPose@@H@NArray@@@@@Z 315b2820 f i CharacterManager.obj
 0001:000b1980       ?init@?$DynArray@UGlobalAnimationHeaderCAF@@HU?$SmallDynStorage@UGlobalAnimationHeaderCAF@@HUStandardAlloc@NAlloc@@@NArray@@@@KAPAUGlobalAnimationHeaderCAF@@U?$Array@UGlobalAnimationHeaderCAF@@HU?$ArrayStorage@UGlobalAnimationHeaderCAF@@H@NArray@@@@@Z 315b2980 f i CharacterManager.obj
 0001:000b1b80       ??$reconstruct@V?$map@IV?$_smart_ptr@UIPlaceholderCharacter@@@@U?$less@I@stlpmtx_std@@V?$allocator@U?$pair@$$CBIV?$_smart_ptr@UIPlaceholderCharacter@@@@@stlpmtx_std@@@3@@stlpmtx_std@@@stl@@YAXAAV?$map@IV?$_smart_ptr@UIPlaceholderCharacter@@@@U?$less@I@stlpmtx_std@@V?$allocator@U?$pair@$$CBIV?$_smart_ptr@UIPlaceholderCharacter@@@@@stlpmtx_std@@@3@@stlpmtx_std@@@Z 315b2b80 f i CharacterManager.obj
 0001:000b1bf0       ?InsertValue@CNameCRCMap@@QAE_NII@Z 315b2bf0 f i CharacterManager.obj
 0001:000b1c40       ??1GlobalAnimationHeaderLMG@@QAE@XZ 315b2c40 f i CharacterManager.obj
 0001:000b1f10       ??1CharacterDefinition@@UAE@XZ 315b2f10 f i CharacterManager.obj
 0001:000b1f90       ??0CharacterDefinition@@QAE@XZ 315b2f90 f i CharacterManager.obj
 0001:000b2000       ??_ECharacterDefinition@@UAEPAXI@Z 315b3000 f i CharacterManager.obj
 0001:000b2000       ??_GCharacterDefinition@@UAEPAXI@Z 315b3000 f i CharacterManager.obj
 0001:000b2030       ?init@?$DynArray@UAimIKPose@@HU?$SmallDynStorage@UAimIKPose@@HUStandardAlloc@NAlloc@@@NArray@@@@KAPAUAimIKPose@@U?$Array@UAimIKPose@@HU?$ArrayStorage@UAimIKPose@@H@NArray@@@@PBU2@@Z 315b3030 f i CharacterManager.obj
 0001:000b2080       ??$move_init@UAimIKPose@@@NArray@@YAXPAUAimIKPose@@0I@Z 315b3080 f i CharacterManager.obj
 0001:000b21d0       ?LoadModelSKIN@CharacterManager@@UAE?AV?$_smart_ptr@UISkin@@@@PBDI@Z 315b31d0 f   CharacterManager.obj
 0001:000b2450       ?resize@?$DynArray@UDebugInstances@@HU?$SmallDynStorage@UDebugInstances@@HUStandardAlloc@NAlloc@@@NArray@@@@QAEXH@Z 315b3450 f i CharacterManager.obj
 0001:000b24f0       ??1?$DynArray@UGlobalAnimationHeaderCAF@@HU?$SmallDynStorage@UGlobalAnimationHeaderCAF@@HUStandardAlloc@NAlloc@@@NArray@@@@QAE@XZ 315b34f0 f i CharacterManager.obj
 0001:000b2550       ??4CharacterDefinition@@QAEAAU0@ABU0@@Z 315b3550 f i CharacterManager.obj
 0001:000b2620       ??0?$DynArray@VCAnimEventData@@HU?$SmallDynStorage@VCAnimEventData@@HUStandardAlloc@NAlloc@@@NArray@@@@QAE@ABU0@@Z 315b3620 f i CharacterManager.obj
 0001:000b26a0       ??0?$DynArray@USCRCName@@HU?$SmallDynStorage@USCRCName@@HUStandardAlloc@NAlloc@@@NArray@@@@QAE@ABU0@@Z 315b36a0 f i CharacterManager.obj
 0001:000b2720       ?resize_raw@?$SmallDynStorage@UAimIKPose@@HUStandardAlloc@NAlloc@@@NArray@@QAEXHH_N@Z 315b3720 f i CharacterManager.obj
 0001:000b2870       ?CreateDebugInstances@CharacterManager@@UAEXPBD@Z 315b3870 f   CharacterManager.obj
 0001:000b2980       ?DumpAssetStatistics@CharacterManager@@AAEXXZ 315b3980 f   CharacterManager.obj
 0001:000b32d0       ?ReleaseCDF@CharacterManager@@QAEXPBD@Z 315b42d0 f   CharacterManager.obj
 0001:000b3430       ??0?$DynArray@UCharacterAttachment@@HU?$SmallDynStorage@UCharacterAttachment@@HUStandardAlloc@NAlloc@@@NArray@@@@QAE@ABU0@@Z 315b4430 f i CharacterManager.obj
 0001:000b34c0       ??$__copy@PAUCharacterDefinition@@PAU1@H@priv@stlpmtx_std@@YAPAUCharacterDefinition@@PAU2@00ABUrandom_access_iterator_tag@1@PAH@Z 315b44c0 f i CharacterManager.obj
 0001:000b3670       ??0?$DynArray@UBSParameter@@HU?$SmallDynStorage@UBSParameter@@HUStandardAlloc@NAlloc@@@NArray@@@@QAE@ABU0@@Z 315b4670 f i CharacterManager.obj
 0001:000b36f0       ??0?$DynArray@UBlendSpaceInfo@@HU?$SmallDynStorage@UBlendSpaceInfo@@HUStandardAlloc@NAlloc@@@NArray@@@@QAE@ABU0@@Z 315b46f0 f i CharacterManager.obj
 0001:000b3770       ?expand_raw@?$DynArray@UAimIKPose@@HU?$SmallDynStorage@UAimIKPose@@HUStandardAlloc@NAlloc@@@NArray@@@@IAEPAUAimIKPose@@PAU2@H@Z 315b4770 f i CharacterManager.obj
 0001:000b37f0       ?init@?$DynArray@UGlobalAnimationHeaderAIM@@HU?$SmallDynStorage@UGlobalAnimationHeaderAIM@@HUStandardAlloc@NAlloc@@@NArray@@@@KAPAUGlobalAnimationHeaderAIM@@U?$Array@UGlobalAnimationHeaderAIM@@HU?$ArrayStorage@UGlobalAnimationHeaderAIM@@H@NArray@@@@@Z 315b47f0 f i CharacterManager.obj
 0001:000b3a30       ??0CharacterDefinition@@QAE@ABU0@@Z 315b4a30 f i CharacterManager.obj
 0001:000b3aa0       ??1?$DynArray@UGlobalAnimationHeaderLMG@@HU?$SmallDynStorage@UGlobalAnimationHeaderLMG@@HUStandardAlloc@NAlloc@@@NArray@@@@QAE@XZ 315b4aa0 f i CharacterManager.obj
 0001:000b3b00       ??0GlobalAnimationHeaderLMG@@QAE@ABU0@@Z 315b4b00 f i CharacterManager.obj
 0001:000b3f30       ?_M_erase@?$_Impl_vector@UCharacterDefinition@@V?$allocator@UCharacterDefinition@@@stlpmtx_std@@@priv@stlpmtx_std@@AAEPAUCharacterDefinition@@PAU4@0ABU__false_type@3@@Z 315b4f30 f i CharacterManager.obj
 0001:000b3fa0       ?Update@CharacterManager@@UAEX_N@Z 315b4fa0 f   CharacterManager.obj
 0001:000b46d0       ??$__ufill@PAUCharacterDefinition@@U1@H@priv@stlpmtx_std@@YAXPAUCharacterDefinition@@0ABU2@ABUrandom_access_iterator_tag@1@PAH@Z 315b56d0 f i CharacterManager.obj
 0001:000b4770       ??$__ucopy@PAUCharacterDefinition@@PAU1@H@priv@stlpmtx_std@@YAPAUCharacterDefinition@@PAU2@00ABUrandom_access_iterator_tag@1@PAH@Z 315b5770 f i CharacterManager.obj
 0001:000b4810       ??1?$DynArray@UGlobalAnimationHeaderAIM@@HU?$SmallDynStorage@UGlobalAnimationHeaderAIM@@HUStandardAlloc@NAlloc@@@NArray@@@@QAE@XZ 315b5810 f i CharacterManager.obj
 0001:000b4870       ??$move_init@UGlobalAnimationHeaderLMG@@@NArray@@YAXPAUGlobalAnimationHeaderLMG@@0I@Z 315b5870 f i CharacterManager.obj
 0001:000b48c0       ??0?$DynArray@UAimIKPose@@HU?$SmallDynStorage@UAimIKPose@@HUStandardAlloc@NAlloc@@@NArray@@@@QAE@ABU0@@Z 315b58c0 f i CharacterManager.obj
 0001:000b4940       ??1CAnimationManager@@UAE@XZ 315b5940 f i CharacterManager.obj
 0001:000b4a10       ?GetGlobalAnimCount@CAnimationManager@@UAEIXZ 315b5a10 f i CharacterManager.obj
 0001:000b4a20       ??_ECAnimationManager@@UAEPAXI@Z 315b5a20 f i CharacterManager.obj
 0001:000b4a20       ??_GCAnimationManager@@UAEPAXI@Z 315b5a20 f i CharacterManager.obj
 0001:000b4a50       ?resize_raw@?$SmallDynStorage@UGlobalAnimationHeaderCAF@@HUStandardAlloc@NAlloc@@@NArray@@QAEXHH_N@Z 315b5a50 f i CharacterManager.obj
 0001:000b4bc0       ?resize_raw@?$SmallDynStorage@UGlobalAnimationHeaderLMG@@HUStandardAlloc@NAlloc@@@NArray@@QAEXHH_N@Z 315b5bc0 f i CharacterManager.obj
 0001:000b4d30       ??0GlobalAnimationHeaderAIM@@QAE@ABU0@@Z 315b5d30 f i CharacterManager.obj
 0001:000b4ea0       ?clear@?$DynArray@UGlobalAnimationHeaderCAF@@HU?$SmallDynStorage@UGlobalAnimationHeaderCAF@@HUStandardAlloc@NAlloc@@@NArray@@@@QAEXXZ 315b5ea0 f i CharacterManager.obj
 0001:000b4f10       ?expand_raw@?$DynArray@UGlobalAnimationHeaderCAF@@HU?$SmallDynStorage@UGlobalAnimationHeaderCAF@@HUStandardAlloc@NAlloc@@@NArray@@@@IAEPAUGlobalAnimationHeaderCAF@@PAU2@H@Z 315b5f10 f i CharacterManager.obj
 0001:000b4fa0       ?reserve@?$DynArray@UGlobalAnimationHeaderCAF@@HU?$SmallDynStorage@UGlobalAnimationHeaderCAF@@HUStandardAlloc@NAlloc@@@NArray@@@@QAEXH@Z 315b5fa0 f i CharacterManager.obj
 0001:000b4ff0       ?CleanupModelCache@CharacterManager@@QAEX_N@Z 315b5ff0 f   CharacterManager.obj
 0001:000b5180       ?ClearResources@CharacterManager@@UAEX_N@Z 315b6180 f   CharacterManager.obj
 0001:000b51e0       ??1CharacterManager@@UAE@XZ 315b61e0 f   CharacterManager.obj
 0001:000b5440       ?SetAnimMemoryTracker@CharacterManager@@UAEXABUSAnimMemoryTracker@@@Z 315b6440 f i CharacterManager.obj
 0001:000b54b0       ?GetAnimMemoryTracker@CharacterManager@@UAE?AUSAnimMemoryTracker@@XZ 315b64b0 f i CharacterManager.obj
 0001:000b54e0       ?ReloadCAF@CharacterManager@@UAEHPBD@Z 315b64e0 f i CharacterManager.obj
 0001:000b5500       ?ReloadLMG@CharacterManager@@UAEHPBD@Z 315b6500 f i CharacterManager.obj
 0001:000b5520       ?SetStreamingListener@CharacterManager@@UAEXPAUIAnimationStreamingListener@@@Z 315b6520 f i CharacterManager.obj
 0001:000b5530       ?AddFrameTicks@CharacterManager@@UAEX_K@Z 315b6530 f i CharacterManager.obj
 0001:000b5550       ?AddFrameSyncTicks@CharacterManager@@UAEX_K@Z 315b6550 f i CharacterManager.obj
 0001:000b5570       ?ResetFrameTicks@CharacterManager@@UAEXXZ 315b6570 f i CharacterManager.obj
 0001:000b5590       ?NumFrameTicks@CharacterManager@@UBE_KXZ 315b6590 f i CharacterManager.obj
 0001:000b55a0       ?NumFrameSyncTicks@CharacterManager@@UBE_KXZ 315b65a0 f i CharacterManager.obj
 0001:000b55b0       ?GetIAnimEvents@CharacterManager@@UAEPAUIAnimEvents@@XZ 315b65b0 f i CharacterManager.obj
 0001:000b55c0       ?_M_insert_overflow_aux@?$_Impl_vector@UCharacterDefinition@@V?$allocator@UCharacterDefinition@@@stlpmtx_std@@@priv@stlpmtx_std@@AAEXPAUCharacterDefinition@@ABU4@ABU__false_type@3@I_N@Z 315b65c0 f i CharacterManager.obj
 0001:000b5780       ??$_M_allocate_and_copy@PAUCharacterDefinition@@@?$_Impl_vector@UCharacterDefinition@@V?$allocator@UCharacterDefinition@@@stlpmtx_std@@@priv@stlpmtx_std@@AAEPAUCharacterDefinition@@AAIPAU3@1@Z 315b6780 f i CharacterManager.obj
 0001:000b57f0       ?ClearCDFCache@CharacterManager@@EAEXXZ 315b67f0 f i CharacterManager.obj
 0001:000b5820       ??$move_init@UGlobalAnimationHeaderAIM@@@NArray@@YAXPAUGlobalAnimationHeaderAIM@@0I@Z 315b6820 f i CharacterManager.obj
 0001:000b5870       ??_ECharacterManager@@UAEPAXI@Z 315b6870 f i CharacterManager.obj
 0001:000b5870       ??_GCharacterManager@@UAEPAXI@Z 315b6870 f i CharacterManager.obj
 0001:000b58a0       ?resize_raw@?$SmallDynStorage@UGlobalAnimationHeaderAIM@@HUStandardAlloc@NAlloc@@@NArray@@QAEXHH_N@Z 315b68a0 f i CharacterManager.obj
 0001:000b59f0       ?resize@?$DynArray@UGlobalAnimationHeaderCAF@@HU?$SmallDynStorage@UGlobalAnimationHeaderCAF@@HUStandardAlloc@NAlloc@@@NArray@@@@QAEXH@Z 315b69f0 f i CharacterManager.obj
 0001:000b5a70       ?clear@?$DynArray@UGlobalAnimationHeaderAIM@@HU?$SmallDynStorage@UGlobalAnimationHeaderAIM@@HUStandardAlloc@NAlloc@@@NArray@@@@QAEXXZ 315b6a70 f i CharacterManager.obj
 0001:000b5af0       ?expand_raw@?$DynArray@UGlobalAnimationHeaderAIM@@HU?$SmallDynStorage@UGlobalAnimationHeaderAIM@@HUStandardAlloc@NAlloc@@@NArray@@@@IAEPAUGlobalAnimationHeaderAIM@@PAU2@H@Z 315b6af0 f i CharacterManager.obj
 0001:000b5b80       ?LoadAnimationImageFileCAF@CharacterManager@@AAE_NPBDPAUIChunkFile@@@Z 315b6b80 f   CharacterManager.obj
 0001:000b6020       ??0CAnimationManager@@QAE@XZ 315b7020 f i CharacterManager.obj
 0001:000b6370       ?LoadCDF@CharacterManager@@QAEHPBD@Z 315b7370 f   CharacterManager.obj
 0001:000b6700       ?GetOrLoadCDFId@CharacterManager@@QAEIABV?$CryStringT@D@@@Z 315b7700 f   CharacterManager.obj
 0001:000b67a0       ??0CharacterManager@@QAE@XZ 315b77a0 f   CharacterManager.obj
 0001:000b6d30       ?PreloadModelsCDF@CharacterManager@@AAEXXZ 315b7d30 f   CharacterManager.obj
 0001:000b7010       ?LoadCharacterDefinition@CharacterManager@@QAEPAUICharacterInstance@@V?$CryStringT@D@@I@Z 315b8010 f   CharacterManager.obj
 0001:000b7300       ?PreloadLevelModels@CharacterManager@@UAEXXZ 315b8300 f   CharacterManager.obj
 0001:000b73a0       ?resize@?$DynArray@UGlobalAnimationHeaderAIM@@HU?$SmallDynStorage@UGlobalAnimationHeaderAIM@@HUStandardAlloc@NAlloc@@@NArray@@@@QAEXH@Z 315b83a0 f i CharacterManager.obj
 0001:000b7430       ?LoadAnimationImageFileAIM@CharacterManager@@AAE_NPBDPAUIChunkFile@@@Z 315b8430 f   CharacterManager.obj
 0001:000b7a60       ?LoadAnimationImageFile@CharacterManager@@AAEXPBD0@Z 315b8a60 f   CharacterManager.obj
 0001:000b7b40       ?FetchModelSKEL@CharacterManager@@QAE?AV?$_smart_ptr@VCSkel@@@@PBDI@Z 315b8b40 f   CharacterManager.obj
 0001:000b7bc0       ?FetchModelSKELForGCA@CharacterManager@@QAE?AV?$_smart_ptr@VCSkel@@@@PBDI@Z 315b8bc0 f   CharacterManager.obj
 0001:000b7c30       ?FetchPlaceHolderCharacterFromCDFInternal@CharacterManager@@QAE_NAAVCPlaceholderCharacter@@PBDI@Z 315b8c30 f   CharacterManager.obj
 0001:000b8300       ?CreateCGAInstance@CharacterManager@@QAEPAUICharacterInstance@@PBDI@Z 315b9300 f   CharacterManager.obj
 0001:000b8620       ?CreateSKELInstance@CharacterManager@@QAEPAUICharacterInstance@@PBDI@Z 315b9620 f   CharacterManager.obj
 0001:000b88c0       ?LoadModelSKEL@CharacterManager@@UAE?AV?$_smart_ptr@UICharacterModel@@@@PBDI@Z 315b98c0 f   CharacterManager.obj
 0001:000b8b40       ?FetchPlaceHolderCharacterFromCDF@CharacterManager@@QAE?AV?$_smart_ptr@UIPlaceholderCharacter@@@@PBDI@Z 315b9b40 f   CharacterManager.obj
 0001:000b8c20       ?CreateCPFInstance@CharacterManager@@QAEPAUICharacterInstance@@PBD0@Z 315b9c20 f   CharacterManager.obj
 0001:000b8ea0       ?CreateInstance@CharacterManager@@UAEPAUICharacterInstance@@PBDI@Z 315b9ea0 f   CharacterManager.obj
 0001:000b90c0       ?PrefetchCharacterResources@CharacterManager@@UAE?AV?$_smart_ptr@UIPlaceholderCharacter@@@@PBDI@Z 315ba0c0 f   CharacterManager.obj
 0001:000b95b0       ?LoadANM@CryCGALoader@@QAEIPAVCSkel@@PBD1AAU?$DynArray@UCControllerTCB@@HU?$SmallDynStorage@UCControllerTCB@@HUStandardAlloc@NAlloc@@@NArray@@@@@Z 315ba5b0 f   LoaderCGA.obj
 0001:000b9630       ?GetStreamInfo@CMesh@@QBEXHAAPAXAAH@Z 315ba630 f i LoaderCGA.obj
 0001:000b97b0       ?StripFileExtension@CryStringUtils@@YAPADPAD@Z 315ba7b0 f i LoaderCGA.obj
 0001:000b9840       ?stristr@CryStringUtils@@YAPBDPBD0@Z 315ba840 f i LoaderCGA.obj
 0001:000b98b0       ??$__find@PAPAVCAttachmentSKIN@@PAV1@@priv@stlpmtx_std@@YAPAPAVCAttachmentSKIN@@PAPAV2@0ABQAV2@ABUrandom_access_iterator_tag@1@@Z 315ba8b0 f i ModelSkin.obj
 0001:000b98b0       ??$__find@PAHH@priv@stlpmtx_std@@YAPAHPAH0ABHABUrandom_access_iterator_tag@1@@Z 315ba8b0 f i LoaderCGA.obj
 0001:000b98b0       ??$__find@PAPAVCFacialEffectorsLibrary@@PAV1@@priv@stlpmtx_std@@YAPAPAVCFacialEffectorsLibrary@@PAPAV2@0ABQAV2@ABUrandom_access_iterator_tag@1@@Z 315ba8b0 f i FaceAnimation.obj
 0001:000b98b0       ??$__find@PAV?$_smart_ptr@VCFacialJoystick@@@@PAVIJoystick@@@priv@stlpmtx_std@@YAPAV?$_smart_ptr@VCFacialJoystick@@@@PAV2@0ABQAVIJoystick@@ABUrandom_access_iterator_tag@1@@Z 315ba8b0 f i FaceJoystick.obj
 0001:000b98b0       ??$__find@PAPAVCCharInstance@@PAV1@@priv@stlpmtx_std@@YAPAPAVCCharInstance@@PAPAV2@0ABQAV2@ABUrandom_access_iterator_tag@1@@Z 315ba8b0 f i Model.obj
 0001:000b9920       ?GetBoneID@CAttachmentFACE@@UBEIXZ 315ba920 f i AttachmentManager.obj
 0001:000b9920       ?GetBoneID@CAttachmentSKIN@@UBEIXZ 315ba920 f i Attachment.obj
 0001:000b9920       ?GetO_numKey@IController@@UBEHXZ 315ba920 f i LoaderCGA.obj
 0001:000b9920       ?GetP_numKey@IController@@UBEHXZ 315ba920 f i LoaderCGA.obj
 0001:000b9930       ?SetStreamData@CMesh@@AAEXHPAXH@Z 315ba930 f i LoaderCGA.obj
 0001:000b9aa0       ??0?$CInt32HashMap@E$0CAA@@@QAE@F@Z 315baaa0 f i LoaderCGA.obj
 0001:000b9b20       ?Insert@?$CInt32HashMap@E$0CAA@@@QAEXIE@Z 315bab20 f i LoaderCGA.obj
 0001:000b9c00       ??$ComputeTexMappingAreas@U?$Vec3_tpl@M@@USMeshTexCoord@@@CMeshHelpers@@SA_NIPBGIPBU?$Vec3_tpl@M@@IPBUSMeshTexCoord@@IAAM3AAPBD@Z 315bac00 f i LoaderCGA.obj
 0001:000b9ef0       ?CryModuleCRTRealloc@@YAPAXPAXI@Z 315baef0 f i LoaderCGA.obj
 0001:000b9f40       ?init@?$DynArray@U?$QuatT_tpl@M@@HU?$SmallDynStorage@U?$QuatT_tpl@M@@HUStandardAlloc@NAlloc@@@NArray@@@@KAPAU?$QuatT_tpl@M@@U?$Array@U?$QuatT_tpl@M@@HU?$ArrayStorage@U?$QuatT_tpl@M@@H@NArray@@@@ABU2@@Z 315baf40 f i LoaderCGA.obj
 0001:000b9fa0       ?set_size@?$SmallDynStorage@V?$TCBSpline@U?$Vec3_tpl@M@@U?$TCBSplineKey@U?$Vec3_tpl@M@@@spline@@@spline@@HUStandardAlloc@NAlloc@@@NArray@@QAEXH@Z 315bafa0 f i LoaderCGA.obj
 0001:000b9fa0       ?set_size@?$SmallDynStorage@VCFacialAnimForcedRotationEntry@@HUStandardAlloc@NAlloc@@@NArray@@QAEXH@Z 315bafa0 f i FacialInstance.obj
 0001:000b9fa0       ?set_size@?$SmallDynStorage@UVirtualExample2D@@HUStandardAlloc@NAlloc@@@NArray@@QAEXH@Z 315bafa0 f i ParametricSampler.obj
 0001:000b9fa0       ?set_size@?$SmallDynStorage@U?$SplineKey@M@spline@@HUStandardAlloc@NAlloc@@@NArray@@QAEXH@Z 315bafa0 f i FaceAnimSequence.obj
 0001:000b9fa0       ?set_size@?$SmallDynStorage@VTCBAngleAxisSpline@spline@@HUStandardAlloc@NAlloc@@@NArray@@QAEXH@Z 315bafa0 f i LoaderCGA.obj
 0001:000ba030       ?init@?$DynArray@UNodeDesc@@HU?$SmallDynStorage@UNodeDesc@@HUStandardAlloc@NAlloc@@@NArray@@@@KAPAUNodeDesc@@U?$Array@UNodeDesc@@HU?$ArrayStorage@UNodeDesc@@H@NArray@@@@@Z 315bb030 f i LoaderCGA.obj
 0001:000ba080       ?set_size@?$SmallDynStorage@UCPhysicsJoint@@HUStandardAlloc@NAlloc@@@NArray@@QAEXH@Z 315bb080 f i SkeletonPhysics.obj
 0001:000ba080       ?set_size@?$SmallDynStorage@UCControllerTCB@@HUStandardAlloc@NAlloc@@@NArray@@QAEXH@Z 315bb080 f i LoaderCGA.obj
 0001:000ba110       ??0?$TCBSplineKey@U?$Quat_tpl@M@@@spline@@QAE@ABU01@@Z 315bb110 f i LoaderCGA.obj
 0001:000ba190       ?set_size@?$SmallDynStorage@VCModelJoint@@HUStandardAlloc@NAlloc@@@NArray@@QAEXH@Z 315bb190 f i LoaderCGA.obj
 0001:000ba220       ?resize_raw@?$SmallDynStorage@UNodeDesc@@HUStandardAlloc@NAlloc@@@NArray@@QAEXHH_N@Z 315bb220 f i LoaderCGA.obj
 0001:000ba380       ?ReallocStream@CMesh@@QAEXHH@Z 315bb380 f i LoaderCGA.obj
 0001:000ba450       ?Append@CMesh@@QAEXAAV1@HHHHPAV?$vector@HV?$allocator@H@stlpmtx_std@@@stlpmtx_std@@@Z 315bb450 f i LoaderCGA.obj
 0001:000ba800       ?PrepareJointIDHash@CModelSkeleton@@QAEXXZ 315bb800 f i LoaderCGA.obj
 0001:000ba890       ??$ComputeTexMappingAreas@UVec3f16@@USMeshTexCoord@@@CMeshHelpers@@SA_NIPBGIPBUVec3f16@@IPBUSMeshTexCoord@@IAAM3AAPBD@Z 315bb890 f i LoaderCGA.obj
 0001:000bab70       ?assign@?$Array@UTCBAngAxisKey@spline@@HU?$SmallDynStorage@UTCBAngAxisKey@spline@@HUStandardAlloc@NAlloc@@@NArray@@@@QAEXU?$Array@$$CBUTCBAngAxisKey@spline@@HU?$ArrayStorage@$$CBUTCBAngAxisKey@spline@@H@NArray@@@@@Z 315bbb70 f i LoaderCGA.obj
 0001:000bac00       ?set_size@?$SmallDynStorage@UTCBAngAxisKey@spline@@HUStandardAlloc@NAlloc@@@NArray@@QAEXH@Z 315bbc00 f i LoaderCGA.obj
 0001:000bac90       ?resize_raw@?$SmallDynStorage@UCControllerType@@HUStandardAlloc@NAlloc@@@NArray@@QAEXHH_N@Z 315bbc90 f i LoaderCGA.obj
 0001:000bade0       ??0CModelJoint@@QAE@ABV0@@Z 315bbde0 f i LoaderCGA.obj
 0001:000baef0       ?expand_raw@?$DynArray@UCControllerType@@HU?$SmallDynStorage@UCControllerType@@HUStandardAlloc@NAlloc@@@NArray@@@@IAEPAUCControllerType@@PAU2@H@Z 315bbef0 f i LoaderCGA.obj
 0001:000baf70       ?expand_raw@?$DynArray@UNodeDesc@@HU?$SmallDynStorage@UNodeDesc@@HUStandardAlloc@NAlloc@@@NArray@@@@IAEPAUNodeDesc@@PAU2@H@Z 315bbf70 f i LoaderCGA.obj
 0001:000bb000       ?SetVertexCount@CMesh@@QAEXH@Z 315bc000 f i LoaderCGA.obj
 0001:000bb070       ?ComputeSubsetTexMappingAreas@CMesh@@QAE_NIAAM0AAPBD@Z 315bc070 f i LoaderCGA.obj
 0001:000bb190       ?RecomputeTexMappingDensity@CMesh@@QAE_NXZ 315bc190 f i LoaderCGA.obj
 0001:000bb270       ?comp_deriv@TCBAngleAxisSpline@spline@@UAEXXZ 315bc270 f i LoaderCGA.obj
 0001:000bb4f0       ??0CModelJoint@@QAE@XZ     315bc4f0 f i LoaderCGA.obj
 0001:000bb5a0       ?SetModelAnimEventDatabase@CSkel@@QAEXABV?$CryStringT@D@@@Z 315bc5a0 f i LoaderCGA.obj
 0001:000bb600       ?set_size@?$SmallDynStorage@USMeshSubset@@HUStandardAlloc@NAlloc@@@NArray@@QAEXH@Z 315bc600 f i LoaderCGA.obj
 0001:000bb690       ?AddList@?$PodArray@G$0A@@@QAEXABV1@@Z 315bc690 f i LoaderCGA.obj
 0001:000bb740       ?erase@?$DynArray@UTCBAngAxisKey@spline@@HU?$SmallDynStorage@UTCBAngAxisKey@spline@@HUStandardAlloc@NAlloc@@@NArray@@@@QAEPAUTCBAngAxisKey@spline@@PAU23@0@Z 315bc740 f i LoaderCGA.obj
 0001:000bb9a0       ?init@?$DynArray@UTCBAngAxisKey@spline@@HU?$SmallDynStorage@UTCBAngAxisKey@spline@@HUStandardAlloc@NAlloc@@@NArray@@@@KAPAUTCBAngAxisKey@spline@@U?$Array@UTCBAngAxisKey@spline@@HU?$ArrayStorage@UTCBAngAxisKey@spline@@H@NArray@@@@PBU23@@Z 315bc9a0 f i LoaderCGA.obj
 0001:000bba00       ??$move_init@UTCBAngAxisKey@spline@@@NArray@@YAXPAUTCBAngAxisKey@spline@@0I@Z 315bca00 f i LoaderCGA.obj
 0001:000bba60       ??$move_init@VCModelJoint@@@NArray@@YAXPAVCModelJoint@@0I@Z 315bca60 f i LoaderCGA.obj
 0001:000bbab0       ?_M_insert@?$_Rb_tree@HU?$less@H@stlpmtx_std@@HU?$_Identity@H@priv@2@U?$_SetTraitsT@H@42@V?$allocator@H@2@@priv@stlpmtx_std@@AAE?AU?$_Rb_tree_iterator@HU?$_SetTraitsT@H@priv@stlpmtx_std@@@23@PAU_Rb_tree_node_base@23@ABH00@Z 315bcab0 f i LoaderCGA.obj
 0001:000bbbb0       ?ToLower@PathUtil@@YA?AV?$CryStringT@D@@ABV2@@Z 315bcbb0 f i LoaderCGA.obj
 0001:000bbc10       ?SetNameChar@CModelJoint@@QAEXPBD@Z 315bcc10 f i LoaderCGA.obj
 0001:000bbcb0       ?SetJointName@CModelJoint@@QAEXPBD@Z 315bccb0 f i LoaderCGA.obj
 0001:000bbd00       ?SetAnimName@ModelAnimationHeader@@QAEXPBD@Z 315bcd00 f i LoaderCGA.obj
 0001:000bbdd0       ?destroy@?$DynArray@USMeshSubset@@HU?$SmallDynStorage@USMeshSubset@@HUStandardAlloc@NAlloc@@@NArray@@@@KAXU?$Array@USMeshSubset@@HU?$ArrayStorage@USMeshSubset@@H@NArray@@@@@Z 315bcdd0 f i LoaderCGA.obj
 0001:000bbe90       ??4?$DynArray@UCControllerType@@HU?$SmallDynStorage@UCControllerType@@HUStandardAlloc@NAlloc@@@NArray@@@@QAEAAU0@U?$Array@$$CBUCControllerType@@HU?$ArrayStorage@$$CBUCControllerType@@H@NArray@@@@@Z 315bce90 f i LoaderCGA.obj
 0001:000bbf50       ?init@?$DynArray@USMeshSubset@@HU?$SmallDynStorage@USMeshSubset@@HUStandardAlloc@NAlloc@@@NArray@@@@KAPAUSMeshSubset@@U?$Array@USMeshSubset@@HU?$ArrayStorage@USMeshSubset@@H@NArray@@@@@Z 315bcf50 f i LoaderCGA.obj
 0001:000bc050       ?resize_raw@?$SmallDynStorage@UTCBAngAxisKey@spline@@HUStandardAlloc@NAlloc@@@NArray@@QAEXHH_N@Z 315bd050 f i LoaderCGA.obj
 0001:000bc1b0       ?expand_raw@?$DynArray@UTCBAngAxisKey@spline@@HU?$SmallDynStorage@UTCBAngAxisKey@spline@@HUStandardAlloc@NAlloc@@@NArray@@@@IAEPAUTCBAngAxisKey@spline@@PAU23@H@Z 315bd1b0 f i LoaderCGA.obj
 0001:000bc240       ?resize_raw@?$SmallDynStorage@VCModelJoint@@HUStandardAlloc@NAlloc@@@NArray@@QAEXHH_N@Z 315bd240 f i LoaderCGA.obj
 0001:000bc3a0       ?insert_unique@?$_Rb_tree@HU?$less@H@stlpmtx_std@@HU?$_Identity@H@priv@2@U?$_SetTraitsT@H@42@V?$allocator@H@2@@priv@stlpmtx_std@@QAE?AU?$pair@U?$_Rb_tree_iterator@HU?$_SetTraitsT@H@priv@stlpmtx_std@@@priv@stlpmtx_std@@_N@3@ABH@Z 315bd3a0 f i LoaderCGA.obj
 0001:000bc460       ??0SMeshSubset@@QAE@ABU0@@Z 315bd460 f i LoaderCGA.obj
 0001:000bc4f0       ?resize@?$DynArray@UCControllerType@@HU?$SmallDynStorage@UCControllerType@@HUStandardAlloc@NAlloc@@@NArray@@@@QAEXH@Z 315bd4f0 f i LoaderCGA.obj
 0001:000bc550       ??4?$DynArray@UTCBAngAxisKey@spline@@HU?$SmallDynStorage@UTCBAngAxisKey@spline@@HUStandardAlloc@NAlloc@@@NArray@@@@QAEAAU0@U?$Array@$$CBUTCBAngAxisKey@spline@@HU?$ArrayStorage@$$CBUTCBAngAxisKey@spline@@H@NArray@@@@@Z 315bd550 f i LoaderCGA.obj
 0001:000bc600       ?expand_raw@?$DynArray@VCModelJoint@@HU?$SmallDynStorage@VCModelJoint@@HUStandardAlloc@NAlloc@@@NArray@@@@IAEPAVCModelJoint@@PAV2@H@Z 315bd600 f i LoaderCGA.obj
 0001:000bc690       ??$AddContainer@U?$DynArray@UTCBAngAxisKey@spline@@HU?$SmallDynStorage@UTCBAngAxisKey@spline@@HUStandardAlloc@NAlloc@@@NArray@@@@@ICrySizer@@QAE_NABU?$DynArray@UTCBAngAxisKey@spline@@HU?$SmallDynStorage@UTCBAngAxisKey@spline@@HUStandardAlloc@NAlloc@@@NArray@@@@@Z 315bd690 f i LoaderCGA.obj
 0001:000bc720       ?GetMemoryUsage@?$TSpline@UTCBAngAxisKey@spline@@VHermitBasis@2@@spline@@UBEXPAVICrySizer@@_N@Z 315bd720 f i LoaderCGA.obj
 0001:000bc760       ??$move_init@USMeshSubset@@@NArray@@YAXPAUSMeshSubset@@0I@Z 315bd760 f i LoaderCGA.obj
 0001:000bc840       ??0?$DynArray@UTCBAngAxisKey@spline@@HU?$SmallDynStorage@UTCBAngAxisKey@spline@@HUStandardAlloc@NAlloc@@@NArray@@@@QAE@ABU0@@Z 315bd840 f i LoaderCGA.obj
 0001:000bc8c0       ??0CMesh@@QAE@XZ           315bd8c0 f i LoaderCGA.obj
 0001:000bc9e0       ?resize_raw@?$SmallDynStorage@USMeshSubset@@HUStandardAlloc@NAlloc@@@NArray@@QAEXHH_N@Z 315bd9e0 f i LoaderCGA.obj
 0001:000bcb50       ?expand_raw@?$DynArray@USMeshSubset@@HU?$SmallDynStorage@USMeshSubset@@HUStandardAlloc@NAlloc@@@NArray@@@@IAEPAUSMeshSubset@@PAU2@H@Z 315bdb50 f i LoaderCGA.obj
 0001:000bcbf0       ?calc_ease@?$TCBSpline@U?$Quat_tpl@M@@UTCBAngAxisKey@spline@@@spline@@IAEMMMM@Z 315bdbf0 f i LoaderCGA.obj
 0001:000bcbf0       ?calc_ease@?$TCBSpline@U?$Vec3_tpl@M@@U?$TCBSplineKey@U?$Vec3_tpl@M@@@spline@@@spline@@IAEMMMM@Z 315bdbf0 f i FaceAnimSequence.obj
 0001:000bccd0       ?init@?$DynArray@V?$TCBSpline@U?$Vec3_tpl@M@@U?$TCBSplineKey@U?$Vec3_tpl@M@@@spline@@@spline@@HU?$SmallDynStorage@V?$TCBSpline@U?$Vec3_tpl@M@@U?$TCBSplineKey@U?$Vec3_tpl@M@@@spline@@@spline@@HUStandardAlloc@NAlloc@@@NArray@@@@KAPAV?$TCBSpline@U?$Vec3_tpl@M@@U?$TCBSplineKey@U?$Vec3_tpl@M@@@spline@@@spline@@U?$Array@V?$TCBSpline@U?$Vec3_tpl@M@@U?$TCBSplineKey@U?$Vec3_tpl@M@@@spline@@@spline@@HU?$ArrayStorage@V?$TCBSpline@U?$Vec3_tpl@M@@U?$TCBSplineKey@U?$Vec3_tpl@M@@@spline@@@spline@@H@NArray@@@@@Z 315bdcd0 f i LoaderCGA.obj
 0001:000bcdc0       ?init@?$DynArray@V?$TCBSpline@U?$Vec3_tpl@M@@U?$TCBSplineKey@U?$Vec3_tpl@M@@@spline@@@spline@@HU?$SmallDynStorage@V?$TCBSpline@U?$Vec3_tpl@M@@U?$TCBSplineKey@U?$Vec3_tpl@M@@@spline@@@spline@@HUStandardAlloc@NAlloc@@@NArray@@@@KAPAV?$TCBSpline@U?$Vec3_tpl@M@@U?$TCBSplineKey@U?$Vec3_tpl@M@@@spline@@@spline@@U?$Array@V?$TCBSpline@U?$Vec3_tpl@M@@U?$TCBSplineKey@U?$Vec3_tpl@M@@@spline@@@spline@@HU?$ArrayStorage@V?$TCBSpline@U?$Vec3_tpl@M@@U?$TCBSplineKey@U?$Vec3_tpl@M@@@spline@@@spline@@H@NArray@@@@ABV23@@Z 315bddc0 f i LoaderCGA.obj
 0001:000bce40       ??$move_init@V?$TCBSpline@U?$Vec3_tpl@M@@U?$TCBSplineKey@U?$Vec3_tpl@M@@@spline@@@spline@@@NArray@@YAXPAV?$TCBSpline@U?$Vec3_tpl@M@@U?$TCBSplineKey@U?$Vec3_tpl@M@@@spline@@@spline@@0I@Z 315bde40 f i LoaderCGA.obj
 0001:000bced0       ?compKeyDeriv@TCBAngleAxisSpline@spline@@EAEXH@Z 315bded0 f i LoaderCGA.obj
 0001:000bda40       ?interp_keys@TCBAngleAxisSpline@spline@@MAEXHHMAAU?$Quat_tpl@M@@@Z 315bea40 f i LoaderCGA.obj
 0001:000c01c0       ??_ETCBAngleAxisSpline@spline@@UAEPAXI@Z 315c11c0 f i LoaderCGA.obj
 0001:000c01c0       ??_E?$TSpline@UTCBAngAxisKey@spline@@VHermitBasis@2@@spline@@UAEPAXI@Z 315c11c0 f i LoaderCGA.obj
 0001:000c01c0       ??_G?$TSpline@UTCBAngAxisKey@spline@@VHermitBasis@2@@spline@@UAEPAXI@Z 315c11c0 f i LoaderCGA.obj
 0001:000c01c0       ??_GTCBAngleAxisSpline@spline@@UAEPAXI@Z 315c11c0 f i LoaderCGA.obj
 0001:000c0210       ?resize_raw@?$SmallDynStorage@V?$TCBSpline@U?$Vec3_tpl@M@@U?$TCBSplineKey@U?$Vec3_tpl@M@@@spline@@@spline@@HUStandardAlloc@NAlloc@@@NArray@@QAEXHH_N@Z 315c1210 f i LoaderCGA.obj
 0001:000c0370       ?init@?$DynArray@VTCBAngleAxisSpline@spline@@HU?$SmallDynStorage@VTCBAngleAxisSpline@spline@@HUStandardAlloc@NAlloc@@@NArray@@@@KAPAVTCBAngleAxisSpline@spline@@U?$Array@VTCBAngleAxisSpline@spline@@HU?$ArrayStorage@VTCBAngleAxisSpline@spline@@H@NArray@@@@@Z 315c1370 f i LoaderCGA.obj
 0001:000c0460       ?expand_raw@?$DynArray@V?$TCBSpline@U?$Vec3_tpl@M@@U?$TCBSplineKey@U?$Vec3_tpl@M@@@spline@@@spline@@HU?$SmallDynStorage@V?$TCBSpline@U?$Vec3_tpl@M@@U?$TCBSplineKey@U?$Vec3_tpl@M@@@spline@@@spline@@HUStandardAlloc@NAlloc@@@NArray@@@@IAEPAV?$TCBSpline@U?$Vec3_tpl@M@@U?$TCBSplineKey@U?$Vec3_tpl@M@@@spline@@@spline@@PAV23@H@Z 315c1460 f i LoaderCGA.obj
 0001:000c04f0       ??0CControllerTCB@@QAE@ABU0@@Z 315c14f0 f i LoaderCGA.obj
 0001:000c05e0       ?GetMemoryUsage@CControllerTCB@@UBEXPAVICrySizer@@@Z 315c15e0 f i LoaderCGA.obj
 0001:000c0630       ?SizeOfController@CControllerTCB@@UBEIXZ 315c1630 f i LoaderCGA.obj
 0001:000c06e0       ??1CControllerTCB@@UAE@XZ  315c16e0 f i LoaderCGA.obj
 0001:000c0780       ??_ECControllerTCB@@UAEPAXI@Z 315c1780 f i LoaderCGA.obj
 0001:000c0780       ??_GCControllerTCB@@UAEPAXI@Z 315c1780 f i LoaderCGA.obj
 0001:000c07b0       ?resize@?$DynArray@USMeshSubset@@HU?$SmallDynStorage@USMeshSubset@@HUStandardAlloc@NAlloc@@@NArray@@@@QAEXH@Z 315c17b0 f i LoaderCGA.obj
 0001:000c0820       ?clear@?$DynArray@V?$TCBSpline@U?$Vec3_tpl@M@@U?$TCBSplineKey@U?$Vec3_tpl@M@@@spline@@@spline@@HU?$SmallDynStorage@V?$TCBSpline@U?$Vec3_tpl@M@@U?$TCBSplineKey@U?$Vec3_tpl@M@@@spline@@@spline@@HUStandardAlloc@NAlloc@@@NArray@@@@QAEXXZ 315c1820 f i LoaderCGA.obj
 0001:000c0890       ?init@?$DynArray@VTCBAngleAxisSpline@spline@@HU?$SmallDynStorage@VTCBAngleAxisSpline@spline@@HUStandardAlloc@NAlloc@@@NArray@@@@KAPAVTCBAngleAxisSpline@spline@@U?$Array@VTCBAngleAxisSpline@spline@@HU?$ArrayStorage@VTCBAngleAxisSpline@spline@@H@NArray@@@@ABV23@@Z 315c1890 f i LoaderCGA.obj
 0001:000c0910       ?init@?$DynArray@UCControllerTCB@@HU?$SmallDynStorage@UCControllerTCB@@HUStandardAlloc@NAlloc@@@NArray@@@@KAPAUCControllerTCB@@U?$Array@UCControllerTCB@@HU?$ArrayStorage@UCControllerTCB@@H@NArray@@@@@Z 315c1910 f i LoaderCGA.obj
 0001:000c0b70       ??$move_init@VTCBAngleAxisSpline@spline@@@NArray@@YAXPAVTCBAngleAxisSpline@spline@@0I@Z 315c1b70 f i LoaderCGA.obj
 0001:000c0c00       ?resize_raw@?$SmallDynStorage@VTCBAngleAxisSpline@spline@@HUStandardAlloc@NAlloc@@@NArray@@QAEXHH_N@Z 315c1c00 f i LoaderCGA.obj
 0001:000c0d60       ?expand_raw@?$DynArray@VTCBAngleAxisSpline@spline@@HU?$SmallDynStorage@VTCBAngleAxisSpline@spline@@HUStandardAlloc@NAlloc@@@NArray@@@@IAEPAVTCBAngleAxisSpline@spline@@PAV23@H@Z 315c1d60 f i LoaderCGA.obj
 0001:000c0df0       ??$move_init@UCControllerTCB@@@NArray@@YAXPAUCControllerTCB@@0I@Z 315c1df0 f i LoaderCGA.obj
 0001:000c0e40       ?resize@?$DynArray@V?$TCBSpline@U?$Vec3_tpl@M@@U?$TCBSplineKey@U?$Vec3_tpl@M@@@spline@@@spline@@HU?$SmallDynStorage@V?$TCBSpline@U?$Vec3_tpl@M@@U?$TCBSplineKey@U?$Vec3_tpl@M@@@spline@@@spline@@HUStandardAlloc@NAlloc@@@NArray@@@@QAEXH@Z 315c1e40 f i LoaderCGA.obj
 0001:000c0ed0       ?clear@?$DynArray@VTCBAngleAxisSpline@spline@@HU?$SmallDynStorage@VTCBAngleAxisSpline@spline@@HUStandardAlloc@NAlloc@@@NArray@@@@QAEXXZ 315c1ed0 f i LoaderCGA.obj
 0001:000c0f40       ?resize_raw@?$SmallDynStorage@UCControllerTCB@@HUStandardAlloc@NAlloc@@@NArray@@QAEXHH_N@Z 315c1f40 f i LoaderCGA.obj
 0001:000c10a0       ?expand_raw@?$DynArray@UCControllerTCB@@HU?$SmallDynStorage@UCControllerTCB@@HUStandardAlloc@NAlloc@@@NArray@@@@IAEPAUCControllerTCB@@PAU2@H@Z 315c20a0 f i LoaderCGA.obj
 0001:000c1130       ?clear@?$DynArray@UCControllerTCB@@HU?$SmallDynStorage@UCControllerTCB@@HUStandardAlloc@NAlloc@@@NArray@@@@QAEXXZ 315c2130 f i LoaderCGA.obj
 0001:000c11a0       ?resize@?$DynArray@VTCBAngleAxisSpline@spline@@HU?$SmallDynStorage@VTCBAngleAxisSpline@spline@@HUStandardAlloc@NAlloc@@@NArray@@@@QAEXH@Z 315c21a0 f i LoaderCGA.obj
 0001:000c1230       ?resize@?$DynArray@UCControllerTCB@@HU?$SmallDynStorage@UCControllerTCB@@HUStandardAlloc@NAlloc@@@NArray@@@@QAEXH@Z 315c2230 f i LoaderCGA.obj
 0001:000c12b0       ?Reset@CryCGALoader@@QAEXXZ 315c22b0 f   LoaderCGA.obj
 0001:000c1320       ?resize@?$DynArray@VCModelMesh@@HU?$SmallDynStorage@VCModelMesh@@HUStandardAlloc@NAlloc@@@NArray@@@@QAEXH@Z 315c2320 f i LoaderCGA.obj
 0001:000c13d0       ?InitNodes@CryCGALoader@@QAEXPAUCHeaderTCB@@PAVCSkel@@PBDABV?$CryStringT@D@@_NII@Z 315c23d0 f   LoaderCGA.obj
 0001:000c4480       ?LoadAnimationANM@CryCGALoader@@QAE_NPBDPAVCSkel@@II@Z 315c5480 f   LoaderCGA.obj
 0001:000c45d0       ?LoadAnimations@CryCGALoader@@QAEXPBDPAVCSkel@@II@Z 315c55d0 f   LoaderCGA.obj
 0001:000c4c20       ?LoadNewCGA@CryCGALoader@@QAEPAVCSkel@@PBDPAVCharacterManager@@I@Z 315c5c20 f   LoaderCGA.obj
 0001:000c5240       ??$move_init@USAnimFile@@@NArray@@YAXPAUSAnimFile@@0I@Z 315c6240 f i LoaderCHR.obj
 0001:000c54d0       ?init@?$DynArray@V?$CryStringT@D@@HU?$SmallDynStorage@V?$CryStringT@D@@HUStandardAlloc@NAlloc@@@NArray@@@@KAPAV?$CryStringT@D@@U?$Array@V?$CryStringT@D@@HU?$ArrayStorage@V?$CryStringT@D@@H@NArray@@@@PBV2@@Z 315c64d0 f i LoaderCHR.obj
 0001:000c5510       ?resize_raw@?$SmallDynStorage@DHUStandardAlloc@NAlloc@@@NArray@@QAEXHH_N@Z 315c6510 f i LoaderCHR.obj
 0001:000c5650       ?PostInitBonePhysGeom@CSkel@@QAE_NAAV?$map@HPAUphys_geometry@@U?$less@H@stlpmtx_std@@V?$allocator@U?$pair@$$CBHPAUphys_geometry@@@stlpmtx_std@@@3@@stlpmtx_std@@H@Z 315c6650 f i LoaderCHR.obj
 0001:000c56c0       ?resize_raw@?$SmallDynStorage@USAnimFile@@HUStandardAlloc@NAlloc@@@NArray@@QAEXHH_N@Z 315c66c0 f i LoaderCHR.obj
 0001:000c5830       ?resize_raw@?$SmallDynStorage@GHUStandardAlloc@NAlloc@@@NArray@@QAEXHH_N@Z 315c6830 f i LoaderCHR.obj
 0001:000c5970       ??1FacialAnimationEntry@CAnimationSet@@QAE@XZ 315c6970 f i LoaderCHR.obj
 0001:000c59d0       ?ReuseAnimationFiles@CryCHRLoader@@AAEIAAVCParamLoader@@IPAVCSkel@@@Z 315c69d0 f   LoaderCHR.obj
 0001:000c5a90       ?expand_raw@?$DynArray@DHU?$SmallDynStorage@DHUStandardAlloc@NAlloc@@@NArray@@@@IAEPADPADH@Z 315c6a90 f i LoaderCHR.obj
 0001:000c5b10       ??4FacialAnimationEntry@CAnimationSet@@QAEAAU01@ABU01@@Z 315c6b10 f i LoaderCHR.obj
 0001:000c5bb0       ??$__unguarded_linear_insert@PAUFacialAnimationEntry@CAnimationSet@@U12@U?$less_stricmp@UFacialAnimationEntry@CAnimationSet@@@stl@@@priv@stlpmtx_std@@YAXPAUFacialAnimationEntry@CAnimationSet@@U23@U?$less_stricmp@UFacialAnimationEntry@CAnimationSet@@@stl@@@Z 315c6bb0 f i LoaderCHR.obj
 0001:000c5c60       ??$__copy_backward@PAUFacialAnimationEntry@CAnimationSet@@PAU12@H@priv@stlpmtx_std@@YAPAUFacialAnimationEntry@CAnimationSet@@PAU23@00ABUrandom_access_iterator_tag@1@PAH@Z 315c6c60 f i LoaderCHR.obj
 0001:000c5dd0       ??$swap@UFacialAnimationEntry@CAnimationSet@@@stlpmtx_std@@YAXAAUFacialAnimationEntry@CAnimationSet@@0@Z 315c6dd0 f i LoaderCHR.obj
 0001:000c5e80       ??$__push_heap@PAUFacialAnimationEntry@CAnimationSet@@HU12@U?$less_stricmp@UFacialAnimationEntry@CAnimationSet@@@stl@@@stlpmtx_std@@YAXPAUFacialAnimationEntry@CAnimationSet@@HHU12@U?$less_stricmp@UFacialAnimationEntry@CAnimationSet@@@stl@@@Z 315c6e80 f i LoaderCHR.obj
 0001:000c5f50       ??$__copy@PBUFacialAnimationEntry@CAnimationSet@@PAU12@H@priv@stlpmtx_std@@YAPAUFacialAnimationEntry@CAnimationSet@@PBU23@0PAU23@ABUrandom_access_iterator_tag@1@PAH@Z 315c6f50 f i LoaderCHR.obj
 0001:000c60b0       ?expand_raw@?$DynArray@GHU?$SmallDynStorage@GHUStandardAlloc@NAlloc@@@NArray@@@@IAEPAGPAGH@Z 315c70b0 f i LoaderCHR.obj
 0001:000c6130       ?GetParentDirectory@PathUtil@@YA?AV?$CryStringT@D@@ABV2@H@Z 315c7130 f i LoaderCHR.obj
 0001:000c6210       ?_M_insert@?$_Rb_tree@HU?$less@H@stlpmtx_std@@U?$pair@$$CBHPAUphys_geometry@@@2@U?$_Select1st@U?$pair@$$CBHPAUphys_geometry@@@stlpmtx_std@@@priv@2@U?$_MapTraitsT@U?$pair@$$CBHPAUphys_geometry@@@stlpmtx_std@@@52@V?$allocator@U?$pair@$$CBHPAUphys_geometry@@@stlpmtx_std@@@2@@priv@stlpmtx_std@@AAE?AU?$_Rb_tree_iterator@U?$pair@$$CBHPAUphys_geometry@@@stlpmtx_std@@U?$_MapTraitsT@U?$pair@$$CBHPAUphys_geometry@@@stlpmtx_std@@@priv@2@@23@PAU_Rb_tree_node_base@23@ABU?$pair@$$CBHPAUphys_geometry@@@3@00@Z 315c7210 f i LoaderCHR.obj
 0001:000c62d0       ?insert_unique@?$_Rb_tree@HU?$less@H@stlpmtx_std@@U?$pair@$$CBHPAUphys_geometry@@@2@U?$_Select1st@U?$pair@$$CBHPAUphys_geometry@@@stlpmtx_std@@@priv@2@U?$_MapTraitsT@U?$pair@$$CBHPAUphys_geometry@@@stlpmtx_std@@@52@V?$allocator@U?$pair@$$CBHPAUphys_geometry@@@stlpmtx_std@@@2@@priv@stlpmtx_std@@QAE?AU?$pair@U?$_Rb_tree_iterator@U?$pair@$$CBHPAUphys_geometry@@@stlpmtx_std@@U?$_MapTraitsT@U?$pair@$$CBHPAUphys_geometry@@@stlpmtx_std@@@priv@2@@priv@stlpmtx_std@@_N@3@ABU?$pair@$$CBHPAUphys_geometry@@@3@@Z 315c72d0 f i LoaderCHR.obj
 0001:000c6390       ??$__unguarded_insertion_sort_aux@PAUFacialAnimationEntry@CAnimationSet@@U12@U?$less_stricmp@UFacialAnimationEntry@CAnimationSet@@@stl@@@priv@stlpmtx_std@@YAXPAUFacialAnimationEntry@CAnimationSet@@00U?$less_stricmp@UFacialAnimationEntry@CAnimationSet@@@stl@@@Z 315c7390 f i LoaderCHR.obj
 0001:000c6400       ??$__adjust_heap@PAUFacialAnimationEntry@CAnimationSet@@HU12@U?$less_stricmp@UFacialAnimationEntry@CAnimationSet@@@stl@@@stlpmtx_std@@YAXPAUFacialAnimationEntry@CAnimationSet@@HHU12@U?$less_stricmp@UFacialAnimationEntry@CAnimationSet@@@stl@@@Z 315c7400 f i LoaderCHR.obj
 0001:000c6520       ??$__ucopy@PBUFacialAnimationEntry@CAnimationSet@@PAU12@H@priv@stlpmtx_std@@YAPAUFacialAnimationEntry@CAnimationSet@@PBU23@0PAU23@ABUrandom_access_iterator_tag@1@PAH@Z 315c7520 f i LoaderCHR.obj
 0001:000c6520       ??$__ucopy@PAUFacialAnimationEntry@CAnimationSet@@PAU12@H@priv@stlpmtx_std@@YAPAUFacialAnimationEntry@CAnimationSet@@PAU23@00ABUrandom_access_iterator_tag@1@PAH@Z 315c7520 f i LoaderCHR.obj
 0001:000c65a0       ?init@?$DynArray@UModelAnimationHeader@@HU?$SmallDynStorage@UModelAnimationHeader@@HUStandardAlloc@NAlloc@@@NArray@@@@KAPAUModelAnimationHeader@@U?$Array@UModelAnimationHeader@@HU?$ArrayStorage@UModelAnimationHeader@@H@NArray@@@@ABU2@@Z 315c75a0 f i LoaderCHR.obj
 0001:000c6600       ??$move_init@UModelAnimationHeader@@@NArray@@YAXPAUModelAnimationHeader@@0I@Z 315c7600 f i LoaderCHR.obj
 0001:000c6690       ?ClearModel@CryCHRLoader@@AAEXXZ 315c7690 f   LoaderCHR.obj
 0001:000c66f0       ?GetDefaultAnimDir@CryCHRLoader@@AAE?BV?$CryStringT@D@@XZ 315c76f0 f   LoaderCHR.obj
 0001:000c6810       ?insert_unique@?$_Rb_tree@HU?$less@H@stlpmtx_std@@U?$pair@$$CBHPAUphys_geometry@@@2@U?$_Select1st@U?$pair@$$CBHPAUphys_geometry@@@stlpmtx_std@@@priv@2@U?$_MapTraitsT@U?$pair@$$CBHPAUphys_geometry@@@stlpmtx_std@@@52@V?$allocator@U?$pair@$$CBHPAUphys_geometry@@@stlpmtx_std@@@2@@priv@stlpmtx_std@@QAE?AU?$_Rb_tree_iterator@U?$pair@$$CBHPAUphys_geometry@@@stlpmtx_std@@U?$_MapTraitsT@U?$pair@$$CBHPAUphys_geometry@@@stlpmtx_std@@@priv@2@@23@U423@ABU?$pair@$$CBHPAUphys_geometry@@@3@@Z 315c7810 f i LoaderCHR.obj
 0001:000c6a00       ??$__pop_heap@PAUFacialAnimationEntry@CAnimationSet@@U12@U?$less_stricmp@UFacialAnimationEntry@CAnimationSet@@@stl@@H@stlpmtx_std@@YAXPAUFacialAnimationEntry@CAnimationSet@@00U12@U?$less_stricmp@UFacialAnimationEntry@CAnimationSet@@@stl@@PAH@Z 315c7a00 f i LoaderCHR.obj
 0001:000c6ae0       ??$__make_heap@PAUFacialAnimationEntry@CAnimationSet@@U?$less_stricmp@UFacialAnimationEntry@CAnimationSet@@@stl@@U12@H@stlpmtx_std@@YAXPAUFacialAnimationEntry@CAnimationSet@@0U?$less_stricmp@UFacialAnimationEntry@CAnimationSet@@@stl@@0PAH@Z 315c7ae0 f i LoaderCHR.obj
 0001:000c6b70       ?resize_raw@?$SmallDynStorage@UModelAnimationHeader@@HUStandardAlloc@NAlloc@@@NArray@@QAEXHH_N@Z 315c7b70 f i LoaderCHR.obj
 0001:000c6cd0       ??1PhysicalProxy@@QAE@XZ   315c7cd0 f i LoaderCHR.obj
 0001:000c6d60       ?expand_raw@?$DynArray@UModelAnimationHeader@@HU?$SmallDynStorage@UModelAnimationHeader@@HUStandardAlloc@NAlloc@@@NArray@@@@IAEPAUModelAnimationHeader@@PAU2@H@Z 315c7d60 f i LoaderCHR.obj
 0001:000c6df0       ??$__destroy_range_aux@V?$reverse_iterator@PAUFacialAnimationEntry@CAnimationSet@@@stlpmtx_std@@UFacialAnimationEntry@CAnimationSet@@@stlpmtx_std@@YAXV?$reverse_iterator@PAUFacialAnimationEntry@CAnimationSet@@@0@0PAUFacialAnimationEntry@CAnimationSet@@ABU__false_type@0@@Z 315c7df0 f i LoaderCHR.obj
 0001:000c7300       ??0?$DynArray@DHU?$SmallDynStorage@DHUStandardAlloc@NAlloc@@@NArray@@@@QAE@ABU0@@Z 315c8300 f i LoaderCHR.obj
 0001:000c7390       ??0?$DynArray@GHU?$SmallDynStorage@GHUStandardAlloc@NAlloc@@@NArray@@@@QAE@ABU0@@Z 315c8390 f i LoaderCHR.obj
 0001:000c7420       ?AddSlash@PathUtil@@YA?AV?$CryStringT@D@@ABV2@@Z 315c8420 f i LoaderCHR.obj
 0001:000c74c0       ?Make@PathUtil@@YA?AV?$CryStringT@D@@ABV2@0@Z 315c84c0 f i LoaderCHR.obj
 0001:000c7530       ?Make@PathUtil@@YA?AV?$CryStringT@D@@QBD0@Z 315c8530 f i LoaderCHR.obj
 0001:000c75c0       ??$__unguarded_partition@PAUFacialAnimationEntry@CAnimationSet@@U12@U?$less_stricmp@UFacialAnimationEntry@CAnimationSet@@@stl@@@priv@stlpmtx_std@@YAPAUFacialAnimationEntry@CAnimationSet@@PAU23@0U23@U?$less_stricmp@UFacialAnimationEntry@CAnimationSet@@@stl@@@Z 315c85c0 f i LoaderCHR.obj
 0001:000c76a0       ??$__linear_insert@PAUFacialAnimationEntry@CAnimationSet@@U12@U?$less_stricmp@UFacialAnimationEntry@CAnimationSet@@@stl@@@priv@stlpmtx_std@@YAXPAUFacialAnimationEntry@CAnimationSet@@0U23@U?$less_stricmp@UFacialAnimationEntry@CAnimationSet@@@stl@@@Z 315c86a0 f i LoaderCHR.obj
 0001:000c7990       ?LoadFaceLib@CryCHRLoader@@AAEXPBD0PAVCSkel@@@Z 315c8990 f   LoaderCHR.obj
 0001:000c7bc0       ??$?AI@?$map@HPAUphys_geometry@@U?$less@H@stlpmtx_std@@V?$allocator@U?$pair@$$CBHPAUphys_geometry@@@stlpmtx_std@@@3@@stlpmtx_std@@QAEAAPAUphys_geometry@@ABI@Z 315c8bc0 f i LoaderCHR.obj
 0001:000c7c40       ??$__insertion_sort@PAUFacialAnimationEntry@CAnimationSet@@U12@U?$less_stricmp@UFacialAnimationEntry@CAnimationSet@@@stl@@@priv@stlpmtx_std@@YAXPAUFacialAnimationEntry@CAnimationSet@@00U?$less_stricmp@UFacialAnimationEntry@CAnimationSet@@@stl@@@Z 315c8c40 f i LoaderCHR.obj
 0001:000c7cb0       ??$sort_heap@PAUFacialAnimationEntry@CAnimationSet@@U?$less_stricmp@UFacialAnimationEntry@CAnimationSet@@@stl@@@stlpmtx_std@@YAXPAUFacialAnimationEntry@CAnimationSet@@0U?$less_stricmp@UFacialAnimationEntry@CAnimationSet@@@stl@@@Z 315c8cb0 f i LoaderCHR.obj
 0001:000c7d60       ?HeadersLoaded@SAnimListInfo@@QAEXXZ 315c8d60 f i LoaderCHR.obj
 0001:000c82b0       ??$_M_range_insert_aux@PBUFacialAnimationEntry@CAnimationSet@@@?$_Impl_vector@UFacialAnimationEntry@CAnimationSet@@V?$allocator@UFacialAnimationEntry@CAnimationSet@@@stlpmtx_std@@@priv@stlpmtx_std@@AAEXPAUFacialAnimationEntry@CAnimationSet@@PBU34@1IABU__false_type@2@@Z 315c92b0 f i LoaderCHR.obj
 0001:000c83a0       ??$__partial_sort@PAUFacialAnimationEntry@CAnimationSet@@U12@U?$less_stricmp@UFacialAnimationEntry@CAnimationSet@@@stl@@@priv@stlpmtx_std@@YAXPAUFacialAnimationEntry@CAnimationSet@@000U?$less_stricmp@UFacialAnimationEntry@CAnimationSet@@@stl@@@Z 315c93a0 f i LoaderCHR.obj
 0001:000c8440       ??$_M_range_insert_realloc@PBUFacialAnimationEntry@CAnimationSet@@@?$_Impl_vector@UFacialAnimationEntry@CAnimationSet@@V?$allocator@UFacialAnimationEntry@CAnimationSet@@@stlpmtx_std@@@priv@stlpmtx_std@@AAEXPAUFacialAnimationEntry@CAnimationSet@@PBU34@1I@Z 315c9440 f i LoaderCHR.obj
 0001:000c85b0       ?AddLoadedHeader@CParamLoader@@QAEXIABUModelAnimationHeader@@@Z 315c95b0 f i LoaderCHR.obj
 0001:000c8600       ?LoadAnimationFiles@CryCHRLoader@@AAEIAAVCParamLoader@@IPAVCSkel@@@Z 315c9600 f   LoaderCHR.obj
 0001:000c8a70       ?resize@?$DynArray@VCModelJoint@@HU?$SmallDynStorage@VCModelJoint@@HUStandardAlloc@NAlloc@@@NArray@@@@QAEXH@Z 315c9a70 f i LoaderCHR.obj
 0001:000c8b20       ??$__introsort_loop@PAUFacialAnimationEntry@CAnimationSet@@U12@HU?$less_stricmp@UFacialAnimationEntry@CAnimationSet@@@stl@@@priv@stlpmtx_std@@YAXPAUFacialAnimationEntry@CAnimationSet@@00HU?$less_stricmp@UFacialAnimationEntry@CAnimationSet@@@stl@@@Z 315c9b20 f i LoaderCHR.obj
 0001:000c95f0       ?LoadAnimations@CryCHRLoader@@AAE_NAAVCParamLoader@@PAVCSkel@@@Z 315ca5f0 f   LoaderCHR.obj
 0001:000ca200       ?LoadCHRPARAMS@CryCHRLoader@@QAEXPAVCSkel@@PBD@Z 315cb200 f   LoaderCHR.obj
 0001:000ca260       ?LoadNewCHR@CryCHRLoader@@QAEPAVCSkel@@PBDI@Z 315cb260 f   LoaderCHR.obj
 0001:000cbf80       ?InMemory@CGlobalHeaderDBA@@QAE_NXZ 315ccf80 f   LoaderDBA.obj
 0001:000cbf90       ??$__copy_backward@PAV?$_smart_ptr@VIController@@@@PAV1@H@priv@stlpmtx_std@@YAPAV?$_smart_ptr@VIController@@@@PAV2@00ABUrandom_access_iterator_tag@1@PAH@Z 315ccf90 f i LoaderDBA.obj
 0001:000cbff0       ??_GIControllerRelocatableChain@@MAEPAXI@Z 315ccff0 f i LoaderDBA.obj
 0001:000cbff0       ??_EIControllerRelocatableChain@@MAEPAXI@Z 315ccff0 f i LoaderDBA.obj
 0001:000cc020       ?Relocate@CInternalDatabaseInfo@@UAEXPAD0@Z 315cd020 f   LoaderDBA.obj
 0001:000cc0d0       ?SizeOf_DBA@CGlobalHeaderDBA@@QBE?BIXZ 315cd0d0 f   LoaderDBA.obj
 0001:000cc100       ??$__unguarded_linear_insert@PAV?$_smart_ptr@VIController@@@@V1@VAnimCtrlSortPred@@@priv@stlpmtx_std@@YAXPAV?$_smart_ptr@VIController@@@@V2@VAnimCtrlSortPred@@@Z 315cd100 f i LoaderDBA.obj
 0001:000cc180       ??$__push_heap@PAV?$_smart_ptr@VIController@@@@HV1@VAnimCtrlSortPred@@@stlpmtx_std@@YAXPAV?$_smart_ptr@VIController@@@@HHV1@VAnimCtrlSortPred@@@Z 315cd180 f i LoaderDBA.obj
 0001:000cc220       ?GetOPS@CControllerOptNonVirtual@@UBEEMAAU?$Quat_tpl@M@@AAU?$Vec3_tpl@M@@AAU?$Diag33_tpl@M@@@Z 315cd220 f i LoaderDBA.obj
 0001:000cc220       ?GetOPS@CController@@UBEEMAAU?$Quat_tpl@M@@AAU?$Vec3_tpl@M@@AAU?$Diag33_tpl@M@@@Z 315cd220 f i LoaderTCB.obj
 0001:000cc280       ?GetS@CControllerOptNonVirtual@@UBEEMAAU?$Diag33_tpl@M@@@Z 315cd280 f i LoaderDBA.obj
 0001:000cc280       ?GetS@CController@@UBEEMAAU?$Diag33_tpl@M@@@Z 315cd280 f i LoaderTCB.obj
 0001:000cc280       ?GetS@CControllerPQLog@@UBEEMAAU?$Diag33_tpl@M@@@Z 315cd280 f i ControllerPQLog.obj
 0001:000cc290       ?SetRotationKeyTimes@CControllerOptNonVirtual@@UAEXIPAD@Z 315cd290 f i LoaderDBA.obj
 0001:000cc2b0       ?SetPositionKeyTimes@CControllerOptNonVirtual@@UAEXIPAD@Z 315cd2b0 f i LoaderDBA.obj
 0001:000cc2d0       ?SetRotationKeys@CControllerOptNonVirtual@@UAEXIPAD@Z 315cd2d0 f i LoaderDBA.obj
 0001:000cc2f0       ?SetPositionKeys@CControllerOptNonVirtual@@UAEXIPAD@Z 315cd2f0 f i LoaderDBA.obj
 0001:000cc310       ?GetRotationFormat@CControllerOptNonVirtual@@UBEIXZ 315cd310 f i LoaderDBA.obj
 0001:000cc320       ?GetRotationKeyTimesFormat@CControllerOptNonVirtual@@UBEIXZ 315cd320 f i LoaderDBA.obj
 0001:000cc330       ?GetPositionFormat@CControllerOptNonVirtual@@UBEIXZ 315cd330 f i LoaderDBA.obj
 0001:000cc340       ?GetPositionKeyTimesFormat@CControllerOptNonVirtual@@UBEIXZ 315cd340 f i LoaderDBA.obj
 0001:000cc350       ?GetRotationKeyData@CControllerOptNonVirtual@@UBEPBDXZ 315cd350 f i LoaderDBA.obj
 0001:000cc360       ?GetRotationKeyTimesData@CControllerOptNonVirtual@@UBEPBDXZ 315cd360 f i LoaderDBA.obj
 0001:000cc370       ?GetPositionKeyData@CControllerOptNonVirtual@@UBEPBDXZ 315cd370 f i LoaderDBA.obj
 0001:000cc380       ?GetPositionKeyTimesData@CControllerOptNonVirtual@@UBEPBDXZ 315cd380 f i LoaderDBA.obj
 0001:000cc390       ?SizeOfController@CControllerOptNonVirtual@@UBEIXZ 315cd390 f i LoaderDBA.obj
 0001:000cc3a0       ?GetPosValueFromKey@CControllerOptNonVirtual@@QBEXIAAU?$Vec3_tpl@M@@@Z 315cd3a0 f i LoaderDBA.obj
 0001:000cc410       ?ApproximateSizeOfThis@CControllerOptNonVirtual@@UBEIXZ 315cd410 f i LoaderDBA.obj
 0001:000cc480       ?GetRotationKeysNum@CControllerOptNonVirtual@@UBEIXZ 315cd480 f i LoaderDBA.obj
 0001:000cc4a0       ?GetPositionKeysNum@CControllerOptNonVirtual@@UBEIXZ 315cd4a0 f i LoaderDBA.obj
 0001:000cc4c0       ??$GetKeyByteData@E@ControllerData@@QBEIMAAMPBX@Z 315cd4c0 f i LoaderDBA.obj
 0001:000cc580       ??$GetKeyByteData@G@ControllerData@@QBEIMAAMPBX@Z 315cd580 f i LoaderDBA.obj
 0001:000cc650       ??$GetKeyByteData@M@ControllerData@@QBEIMAAMPBX@Z 315cd650 f i LoaderDBA.obj
 0001:000cc720       ?GetKeyBitData@ControllerData@@QBEIMAAM@Z 315cd720 f i LoaderDBA.obj
 0001:000cc920       ??0CInternalDatabaseInfo@@QAE@IABV?$CryStringT@D@@@Z 315cd920 f   LoaderDBA.obj
 0001:000cc980       ??_ECInternalDatabaseInfo@@W3AEPAXI@Z 315cd980 f i LoaderDBA.obj
 0001:000cc990       ??1CInternalDatabaseInfo@@UAE@XZ 315cd990 f   LoaderDBA.obj
 0001:000cca30       ?GetMemoryUsage@CGlobalHeaderDBA@@QBEXPAVICrySizer@@@Z 315cda30 f   LoaderDBA.obj
 0001:000cca80       ??0CGlobalHeaderDBA@@QAE@XZ 315cda80 f   LoaderDBA.obj
 0001:000ccaf0       ??1CGlobalHeaderDBA@@QAE@XZ 315cdaf0 f   LoaderDBA.obj
 0001:000ccbe0       ??$__adjust_heap@PAV?$_smart_ptr@VIController@@@@HV1@VAnimCtrlSortPred@@@stlpmtx_std@@YAXPAV?$_smart_ptr@VIController@@@@HHV1@VAnimCtrlSortPred@@@Z 315cdbe0 f i LoaderDBA.obj
 0001:000cccb0       ?GetKey@ControllerData@@QBEIMAAM@Z 315cdcb0 f i LoaderDBA.obj
 0001:000ccd20       ?GetPosValue@CControllerOptNonVirtual@@QBE?AU?$Vec3_tpl@M@@M@Z 315cdd20 f i LoaderDBA.obj
 0001:000ccec0       ?CreateDatabaseDBA@CGlobalHeaderDBA@@QAEXPBD@Z 315cdec0 f   LoaderDBA.obj
 0001:000cd010       ?StartStreamingDBA@CGlobalHeaderDBA@@QAE_N_N@Z 315ce010 f   LoaderDBA.obj
 0001:000cd120       ??_GCInternalDatabaseInfo@@UAEPAXI@Z 315ce120 f i LoaderDBA.obj
 0001:000cd120       ??_ECInternalDatabaseInfo@@UAEPAXI@Z 315ce120 f i LoaderDBA.obj
 0001:000cd150       ?ReportLoadError@CGlobalHeaderDBA@@QAEXPBD0@Z 315ce150 f   LoaderDBA.obj
 0001:000cd1b0       ??0?$_Vector_base@PAXV?$allocator@PAX@stlpmtx_std@@@priv@stlpmtx_std@@QAE@IABV?$allocator@PAX@2@@Z 315ce1b0 f i LoaderDBA.obj
 0001:000cd1b0       ??0?$_Vector_base@IV?$allocator@I@stlpmtx_std@@@priv@stlpmtx_std@@QAE@IABV?$allocator@I@2@@Z 315ce1b0 f i LoaderDBA.obj
 0001:000cd260       ??$__unguarded_insertion_sort@PAV?$_smart_ptr@VIController@@@@VAnimCtrlSortPred@@@priv@stlpmtx_std@@YAXPAV?$_smart_ptr@VIController@@@@0VAnimCtrlSortPred@@@Z 315ce260 f i LoaderDBA.obj
 0001:000cd2a0       ??$__linear_insert@PAV?$_smart_ptr@VIController@@@@V1@VAnimCtrlSortPred@@@priv@stlpmtx_std@@YAXPAV?$_smart_ptr@VIController@@@@0V2@VAnimCtrlSortPred@@@Z 315ce2a0 f i LoaderDBA.obj
 0001:000cd330       ??$__make_heap@PAV?$_smart_ptr@VIController@@@@VAnimCtrlSortPred@@V1@H@stlpmtx_std@@YAXPAV?$_smart_ptr@VIController@@@@0VAnimCtrlSortPred@@0PAH@Z 315ce330 f i LoaderDBA.obj
 0001:000cd380       ?GetP@CControllerOptNonVirtual@@UBEEMAAU?$Vec3_tpl@M@@@Z 315ce380 f i LoaderDBA.obj
 0001:000cd3c0       ?CompleteStreamingDBA@CGlobalHeaderDBA@@QAEXPAUCInternalDatabaseInfo@@@Z 315ce3c0 f   LoaderDBA.obj
 0001:000cd4a0       ?StreamOnComplete@CInternalDatabaseInfo@@UAEXPAVIReadStream@@I@Z 315ce4a0 f   LoaderDBA.obj
 0001:000cd4e0       ?DeleteDatabaseDBA@CGlobalHeaderDBA@@QAEXXZ 315ce4e0 f   LoaderDBA.obj
 0001:000cd6e0       ??$__unguarded_partition@PAV?$_smart_ptr@VIController@@@@V1@VAnimCtrlSortPred@@@priv@stlpmtx_std@@YAPAV?$_smart_ptr@VIController@@@@PAV2@0V2@VAnimCtrlSortPred@@@Z 315ce6e0 f i LoaderDBA.obj
 0001:000cd740       ??$__insertion_sort@PAV?$_smart_ptr@VIController@@@@V1@VAnimCtrlSortPred@@@priv@stlpmtx_std@@YAXPAV?$_smart_ptr@VIController@@@@00VAnimCtrlSortPred@@@Z 315ce740 f i LoaderDBA.obj
 0001:000cd790       ?resize@?$DynArray@V?$_smart_ptr@VIController@@@@HU?$SmallDynStorage@V?$_smart_ptr@VIController@@@@HUStandardAlloc@NAlloc@@@NArray@@@@QAEXH@Z 315ce790 f i LoaderDBA.obj
 0001:000cd820       ??$sort_heap@PAV?$_smart_ptr@VIController@@@@VAnimCtrlSortPred@@@stlpmtx_std@@YAXPAV?$_smart_ptr@VIController@@@@0VAnimCtrlSortPred@@@Z 315ce820 f i LoaderDBA.obj
 0001:000cd8d0       ?resize@?$DynArray@IHU?$SmallDynStorage@IHUStandardAlloc@NAlloc@@@NArray@@@@QAEXH@Z 315ce8d0 f i LoaderDBA.obj
 0001:000cd910       ??$__partial_sort@PAV?$_smart_ptr@VIController@@@@V1@VAnimCtrlSortPred@@@priv@stlpmtx_std@@YAXPAV?$_smart_ptr@VIController@@@@000VAnimCtrlSortPred@@@Z 315ce910 f i LoaderDBA.obj
 0001:000cd9d0       ?InitControllerLookup@GlobalAnimationHeaderCAF@@QAEXI@Z 315ce9d0 f i LoaderDBA.obj
 0001:000cda50       ??$__introsort_loop@PAV?$_smart_ptr@VIController@@@@V1@HVAnimCtrlSortPred@@@priv@stlpmtx_std@@YAXPAV?$_smart_ptr@VIController@@@@00HVAnimCtrlSortPred@@@Z 315cea50 f i LoaderDBA.obj
 0001:000cdb30       ??$sort@PAV?$_smart_ptr@VIController@@@@VAnimCtrlSortPred@@@stlpmtx_std@@YAXPAV?$_smart_ptr@VIController@@@@0VAnimCtrlSortPred@@@Z 315ceb30 f i LoaderDBA.obj
 0001:000cdbb0       ?ReadController905@CInternalDatabaseInfo@@QAE_NPAUChunkDesc@IChunkFile@@_N@Z 315cebb0 f   LoaderDBA.obj
 0001:000cef50       ?LoadChunks@CInternalDatabaseInfo@@QAE_NPAUIChunkFile@@_N@Z 315cff50 f   LoaderDBA.obj
 0001:000cf040       ?LoadDatabaseDBA@CGlobalHeaderDBA@@QAEXPBD@Z 315d0040 f   LoaderDBA.obj
 0001:000cf190       ?StreamAsyncOnComplete@CInternalDatabaseInfo@@UAEXPAVIReadStream@@I@Z 315d0190 f   LoaderDBA.obj
 0001:000cf3b0       ??4?$_smart_ptr@VIKeyTimesInformation@@@@QAEAAV0@PAVIKeyTimesInformation@@@Z 315d03b0 f i LoaderTCB.obj
 0001:000cf400       ??$move_init@UCryTCB3Key@@@NArray@@YAXPAUCryTCB3Key@@0I@Z 315d0400 f i LoaderTCB.obj
 0001:000cf440       ?SizeOfController@CController@@UBEIXZ 315d0440 f i LoaderTCB.obj
 0001:000cf480       ?ApproximateSizeOfThis@CController@@UBEIXZ 315d0480 f i LoaderTCB.obj
 0001:000cf480       ?ApproximateSizeOfThis@CControllerPQLog@@UBEIXZ 315d0480 f i ControllerPQLog.obj
 0001:000cf480       ?ApproximateSizeOfThis@CControllerTCB@@UBEIXZ 315d0480 f i LoaderCGA.obj
 0001:000cf490       ?GetO_numKey@CController@@UBEHXZ 315d0490 f i LoaderTCB.obj
 0001:000cf4b0       ?GetP_numKey@CController@@UBEHXZ 315d04b0 f i LoaderTCB.obj
 0001:000cf4d0       ?GetRotationKeysNum@CController@@UBEIXZ 315d04d0 f i LoaderTCB.obj
 0001:000cf4f0       ?GetPositionKeysNum@CController@@UBEIXZ 315d04f0 f i LoaderTCB.obj
 0001:000cf510       ??_ECController@@UAEPAXI@Z 315d0510 f i LoaderTCB.obj
 0001:000cf510       ??_GCController@@UAEPAXI@Z 315d0510 f i LoaderTCB.obj
 0001:000cf560       ??1?$_smart_ptr@VIKeyTimesInformation@@@@QAE@XZ 315d0560 f i LoaderTCB.obj
 0001:000cf590       ??$move_init@UPQLog@@@NArray@@YAXPAUPQLog@@0I@Z 315d0590 f i LoaderTCB.obj
 0001:000cf590       ??$move_init@UADIKTarget@@@NArray@@YAXPAUADIKTarget@@0I@Z 315d0590 f i ParamLoader.obj
 0001:000cf5f0       ?resize_raw@?$SmallDynStorage@PAU?$DynArray@UCryTCB3Key@@HU?$SmallDynStorage@UCryTCB3Key@@HUStandardAlloc@NAlloc@@@NArray@@@@HUStandardAlloc@NAlloc@@@NArray@@QAEXHH_N@Z 315d05f0 f i LoaderTCB.obj
 0001:000cf740       ?resize_raw@?$SmallDynStorage@PAU?$DynArray@UCryTCBQKey@@HU?$SmallDynStorage@UCryTCBQKey@@HUStandardAlloc@NAlloc@@@NArray@@@@HUStandardAlloc@NAlloc@@@NArray@@QAEXHH_N@Z 315d0740 f i LoaderTCB.obj
 0001:000cf890       ?resize_raw@?$SmallDynStorage@UTCBFlags@@HUStandardAlloc@NAlloc@@@NArray@@QAEXHH_N@Z 315d0890 f i LoaderTCB.obj
 0001:000cf9d0       ?set_size@?$SmallDynStorage@UCControllerType@@HUStandardAlloc@NAlloc@@@NArray@@QAEXH@Z 315d09d0 f i LoaderCGA.obj
 0001:000cf9d0       ?set_size@?$SmallDynStorage@U?$DynArray@IHU?$SmallDynStorage@IHUStandardAlloc@NAlloc@@@NArray@@@@HUStandardAlloc@NAlloc@@@NArray@@QAEXH@Z 315d09d0 f i ParamLoader.obj
 0001:000cf9d0       ?set_size@?$SmallDynStorage@PAU?$DynArray@UCryTCB3Key@@HU?$SmallDynStorage@UCryTCB3Key@@HUStandardAlloc@NAlloc@@@NArray@@@@HUStandardAlloc@NAlloc@@@NArray@@QAEXH@Z 315d09d0 f i LoaderTCB.obj
 0001:000cf9d0       ?set_size@?$SmallDynStorage@IHUStandardAlloc@NAlloc@@@NArray@@QAEXH@Z 315d09d0 f i CharacterManager.obj
 0001:000cf9d0       ?set_size@?$SmallDynStorage@V?$CryStringT@D@@HUStandardAlloc@NAlloc@@@NArray@@QAEXH@Z 315d09d0 f i CharacterInstance.obj
 0001:000cf9d0       ?set_size@?$SmallDynStorage@V?$_smart_ptr@VIController@@@@HUStandardAlloc@NAlloc@@@NArray@@QAEXH@Z 315d09d0 f i CharacterManager.obj
 0001:000cf9d0       ?set_size@?$SmallDynStorage@PAVCAttachmentSKIN@@HUStandardAlloc@NAlloc@@@NArray@@QAEXH@Z 315d09d0 f i ModelSkin.obj
 0001:000cf9d0       ?set_size@?$SmallDynStorage@PAVCAnimationSet@@HUStandardAlloc@NAlloc@@@NArray@@QAEXH@Z 315d09d0 f i ModelAnimationSet.obj
 0001:000cf9d0       ?set_size@?$SmallDynStorage@HHUStandardAlloc@NAlloc@@@NArray@@QAEXH@Z 315d09d0 f i SkeletonPhysics.obj
 0001:000cf9d0       ?set_size@?$SmallDynStorage@V?$_smart_ptr@UCMorphTarget@@@@HUStandardAlloc@NAlloc@@@NArray@@QAEXH@Z 315d09d0 f i LoaderSKIN.obj
 0001:000cf9d0       ?set_size@?$SmallDynStorage@V?$_smart_ptr@UIAttachment@@@@HUStandardAlloc@NAlloc@@@NArray@@QAEXH@Z 315d09d0 f i AttachmentManager.obj
 0001:000cf9d0       ?set_size@?$SmallDynStorage@MHUStandardAlloc@NAlloc@@@NArray@@QAEXH@Z 315d09d0 f i CharacterInstance.obj
 0001:000cf9d0       ?set_size@?$SmallDynStorage@PAVCCharInstance@@HUStandardAlloc@NAlloc@@@NArray@@QAEXH@Z 315d09d0 f i Model.obj
 0001:000cf9d0       ?set_size@?$SmallDynStorage@PAU?$DynArray@UCryTCBQKey@@HU?$SmallDynStorage@UCryTCBQKey@@HUStandardAlloc@NAlloc@@@NArray@@@@HUStandardAlloc@NAlloc@@@NArray@@QAEXH@Z 315d09d0 f i LoaderTCB.obj
 0001:000cfa50       ?resize_raw@?$SmallDynStorage@UCryTCB3Key@@HUStandardAlloc@NAlloc@@@NArray@@QAEXHH_N@Z 315d0a50 f i LoaderTCB.obj
 0001:000cfbb0       ?SetKeyTimesInformation@ITrackInformation@@QAEXAAV?$_smart_ptr@VIKeyTimesInformation@@@@@Z 315d0bb0 f i LoaderTCB.obj
 0001:000cfc10       ??_EITrackInformation@@UAEPAXI@Z 315d0c10 f i LoaderTCB.obj
 0001:000cfc10       ??_GITrackInformation@@UAEPAXI@Z 315d0c10 f i LoaderTCB.obj
 0001:000cfc60       ?GetRotationStorage@IRotationController@@UAEAAPAVITrackRotationStorage@@XZ 315d0c60 f i LoaderTCB.obj
 0001:000cfc60       ?GetData@?$CKeyTimesInformationStartStop@GUUINT16StartStopEncoder@@@@UAEPADXZ 315d0c60 f i ControllerPQ.obj
 0001:000cfc60       ?GetPositionStorage@IPositionController@@UAEAAPAVITrackPositionStorage@@XZ 315d0c60 f i LoaderTCB.obj
 0001:000cfc60       ?GetData@?$CKeyTimesInformationStartStop@MUF32StartStopEncoder@@@@UAEPADXZ 315d0c60 f i ControllerPQ.obj
 0001:000cfc60       ?GetData@?$CKeyTimesInformationStartStop@EUByteStartStopEncoder@@@@UAEPADXZ 315d0c60 f i ControllerPQ.obj
 0001:000cfc70       ?GetFormat@IRotationController@@UAEIXZ 315d0c70 f i LoaderTCB.obj
 0001:000cfc70       ?GetFormat@IPositionController@@UAEIXZ 315d0c70 f i LoaderTCB.obj
 0001:000cfc80       ?GetData@IPositionController@@UAEPADXZ 315d0c80 f i LoaderTCB.obj
 0001:000cfc80       ?GetData@IRotationController@@UAEPADXZ 315d0c80 f i LoaderTCB.obj
 0001:000cfc90       ?SizeOfPosController@IPositionController@@UAEIXZ 315d0c90 f i LoaderTCB.obj
 0001:000cfcd0       ?SetPositionStorage@IPositionController@@UAEXAAPAVITrackPositionStorage@@@Z 315d0cd0 f i LoaderTCB.obj
 0001:000cfcd0       ?SetRotationStorage@IRotationController@@UAEXAAPAVITrackRotationStorage@@@Z 315d0cd0 f i LoaderTCB.obj
 0001:000cfce0       ?SizeOfRotController@IRotationController@@UAEIXZ 315d0ce0 f i LoaderTCB.obj
 0001:000cfd10       ?GetMemoryUsage@CController@@UBEXPAVICrySizer@@@Z 315d0d10 f i LoaderTCB.obj
 0001:000cfd40       ?resize_raw@?$SmallDynStorage@UPQLog@@HUStandardAlloc@NAlloc@@@NArray@@QAEXHH_N@Z 315d0d40 f i LoaderTCB.obj
 0001:000cfea0       ??0CLoaderTCB@@QAE@XZ      315d0ea0 f   LoaderTCB.obj
 0001:000cfec0       ??1CLoaderTCB@@QAE@XZ      315d0ec0 f   LoaderTCB.obj
 0001:000cff30       ?ReadMotionParameters@CLoaderTCB@@AAE_NPAUChunkDesc@IChunkFile@@@Z 315d0f30 f   LoaderTCB.obj
 0001:000cffd0       ?Blend@QuatLerp@@SAXAAU?$Quat_tpl@M@@ABU2@1M@Z 315d0fd0 f i LoaderTCB.obj
 0001:000d0130       ?GetValue@?$CAdvancedTrackInformation@U?$Quat_tpl@M@@UQuatLerp@@VIRotationController@@@@UAEXMAAU?$Quat_tpl@M@@@Z 315d1130 f i LoaderTCB.obj
 0001:000d0210       ?GetValue@?$CAdvancedTrackInformation@U?$Vec3_tpl@M@@UVec3Lerp@@VIPositionController@@@@UAEXMAAU?$Vec3_tpl@M@@@Z 315d1210 f i LoaderTCB.obj
 0001:000d0300       ??_E?$CAdvancedTrackInformation@U?$Quat_tpl@M@@UQuatLerp@@VIRotationController@@@@UAEPAXI@Z 315d1300 f i LoaderTCB.obj
 0001:000d0300       ??_EIRotationController@@UAEPAXI@Z 315d1300 f i LoaderTCB.obj
 0001:000d0300       ??_G?$CAdvancedTrackInformation@U?$Quat_tpl@M@@UQuatLerp@@VIRotationController@@@@UAEPAXI@Z 315d1300 f i LoaderTCB.obj
 0001:000d0300       ??_GIRotationController@@UAEPAXI@Z 315d1300 f i LoaderTCB.obj
 0001:000d0370       ??_EIPositionController@@UAEPAXI@Z 315d1370 f i LoaderTCB.obj
 0001:000d0370       ??_GIPositionController@@UAEPAXI@Z 315d1370 f i LoaderTCB.obj
 0001:000d0370       ??_E?$CAdvancedTrackInformation@U?$Vec3_tpl@M@@UVec3Lerp@@VIPositionController@@@@UAEPAXI@Z 315d1370 f i LoaderTCB.obj
 0001:000d0370       ??_G?$CAdvancedTrackInformation@U?$Vec3_tpl@M@@UVec3Lerp@@VIPositionController@@@@UAEPAXI@Z 315d1370 f i LoaderTCB.obj
 0001:000d03e0       ?expand_raw@?$DynArray@UPQLog@@HU?$SmallDynStorage@UPQLog@@HUStandardAlloc@NAlloc@@@NArray@@@@IAEPAUPQLog@@PAU2@H@Z 315d13e0 f i LoaderTCB.obj
 0001:000d0470       ?expand_raw@?$DynArray@UTCBFlags@@HU?$SmallDynStorage@UTCBFlags@@HUStandardAlloc@NAlloc@@@NArray@@@@IAEPAUTCBFlags@@PAU2@H@Z 315d1470 f i LoaderTCB.obj
 0001:000d04f0       ?expand_raw@?$DynArray@PAU?$DynArray@UCryTCB3Key@@HU?$SmallDynStorage@UCryTCB3Key@@HUStandardAlloc@NAlloc@@@NArray@@@@HU?$SmallDynStorage@PAU?$DynArray@UCryTCB3Key@@HU?$SmallDynStorage@UCryTCB3Key@@HUStandardAlloc@NAlloc@@@NArray@@@@HUStandardAlloc@NAlloc@@@NArray@@@@IAEPAPAU?$DynArray@UCryTCB3Key@@HU?$SmallDynStorage@UCryTCB3Key@@HUStandardAlloc@NAlloc@@@NArray@@@@PAPAU2@H@Z 315d14f0 f i LoaderTCB.obj
 0001:000d0570       ?expand_raw@?$DynArray@PAU?$DynArray@UCryTCBQKey@@HU?$SmallDynStorage@UCryTCBQKey@@HUStandardAlloc@NAlloc@@@NArray@@@@HU?$SmallDynStorage@PAU?$DynArray@UCryTCBQKey@@HU?$SmallDynStorage@UCryTCBQKey@@HUStandardAlloc@NAlloc@@@NArray@@@@HUStandardAlloc@NAlloc@@@NArray@@@@IAEPAPAU?$DynArray@UCryTCBQKey@@HU?$SmallDynStorage@UCryTCBQKey@@HUStandardAlloc@NAlloc@@@NArray@@@@PAPAU2@H@Z 315d1570 f i LoaderTCB.obj
 0001:000d05f0       ?expand_raw@?$DynArray@UCryTCB3Key@@HU?$SmallDynStorage@UCryTCB3Key@@HUStandardAlloc@NAlloc@@@NArray@@@@IAEPAUCryTCB3Key@@PAU2@H@Z 315d15f0 f i LoaderTCB.obj
 0001:000d0680       ??$move_init@UCryTCBQKey@@@NArray@@YAXPAUCryTCBQKey@@0I@Z 315d1680 f i LoaderTCB.obj
 0001:000d0860       ?grow@?$DynArray@V?$_smart_ptr@VIController@@@@HU?$SmallDynStorage@V?$_smart_ptr@VIController@@@@HUStandardAlloc@NAlloc@@@NArray@@@@QAEPAV?$_smart_ptr@VIController@@@@HABV2@@Z 315d1860 f i LoaderTCB.obj
 0001:000d08c0       ?resize_raw@?$SmallDynStorage@UCryTCBQKey@@HUStandardAlloc@NAlloc@@@NArray@@QAEXHH_N@Z 315d18c0 f i LoaderTCB.obj
 0001:000d0a20       ?push_back@?$DynArray@IHU?$SmallDynStorage@IHUStandardAlloc@NAlloc@@@NArray@@@@QAEPAIABI@Z 315d1a20 f i LoaderTCB.obj
 0001:000d0a60       ?resize@?$DynArray@UPQLog@@HU?$SmallDynStorage@UPQLog@@HUStandardAlloc@NAlloc@@@NArray@@@@QAEXH@Z 315d1a60 f i LoaderTCB.obj
 0001:000d0aa0       ?push_back@?$DynArray@UTCBFlags@@HU?$SmallDynStorage@UTCBFlags@@HUStandardAlloc@NAlloc@@@NArray@@@@QAEPAUTCBFlags@@ABU2@@Z 315d1aa0 f i LoaderTCB.obj
 0001:000d0ae0       ??0?$DynArray@UCryTCB3Key@@HU?$SmallDynStorage@UCryTCB3Key@@HUStandardAlloc@NAlloc@@@NArray@@@@QAE@XZ 315d1ae0 f i LoaderTCB.obj
 0001:000d0b30       ?resize@?$DynArray@UCryTCB3Key@@HU?$SmallDynStorage@UCryTCB3Key@@HUStandardAlloc@NAlloc@@@NArray@@@@QAEXH@Z 315d1b30 f i LoaderTCB.obj
 0001:000d0b70       ??0?$DynArray@UCryTCBQKey@@HU?$SmallDynStorage@UCryTCBQKey@@HUStandardAlloc@NAlloc@@@NArray@@@@QAE@XZ 315d1b70 f i LoaderTCB.obj
 0001:000d0bc0       ?expand_raw@?$DynArray@UCryTCBQKey@@HU?$SmallDynStorage@UCryTCBQKey@@HUStandardAlloc@NAlloc@@@NArray@@@@IAEPAUCryTCBQKey@@PAU2@H@Z 315d1bc0 f i LoaderTCB.obj
 0001:000d0c50       ??0CHeaderTCB@@QAE@XZ      315d1c50 f i LoaderTCB.obj
 0001:000d0e20       ??1CHeaderTCB@@UAE@XZ      315d1e20 f i LoaderTCB.obj
 0001:000d1330       ??_GCHeaderTCB@@UAEPAXI@Z  315d2330 f i LoaderTCB.obj
 0001:000d1330       ??_ECHeaderTCB@@UAEPAXI@Z  315d2330 f i LoaderTCB.obj
 0001:000d1360       ?resize@?$DynArray@UCryTCBQKey@@HU?$SmallDynStorage@UCryTCBQKey@@HUStandardAlloc@NAlloc@@@NArray@@@@QAEXH@Z 315d2360 f i LoaderTCB.obj
 0001:000d13a0       ?ReadController@CLoaderTCB@@AAE_NPAUChunkDesc@IChunkFile@@@Z 315d23a0 f   LoaderTCB.obj
 0001:000d2120       ?LoadChunksTCB@CLoaderTCB@@AAE_NPAUIChunkFile@@@Z 315d3120 f   LoaderTCB.obj
 0001:000d2420       ?LoadTCB@CLoaderTCB@@QAEPAUCHeaderTCB@@PBDPAUIChunkFile@@PAVILoaderCAFListener@@@Z 315d3420 f   LoaderTCB.obj
 0001:000d2690       ?LoadTCB@CLoaderTCB@@QAEPAUCHeaderTCB@@PBDPAVILoaderCAFListener@@@Z 315d3690 f   LoaderTCB.obj
 0001:000d26d0       ?Warning@@YAXPBDW4EValidatorSeverity@@0ZZ 315d36d0 f   ParamLoader.obj
 0001:000d2700       ??$__find_if@PAUSAnimFile@@UFindByAliasName@?A0x32a97809@@@priv@stlpmtx_std@@YAPAUSAnimFile@@PAU2@0UFindByAliasName@?A0x32a97809@@ABUrandom_access_iterator_tag@1@@Z 315d3700 f i ParamLoader.obj
 0001:000d27d0       ?getAttr@IXmlNode@@QBE_NPBDAAE@Z 315d37d0 f i ParamLoader.obj
 0001:000d2800       ?GetFile@PathUtil@@YAPBDPBD@Z 315d3800 f i ParamLoader.obj
 0001:000d2840       ?MatchWildcard@PathUtil@@YA_NPBD0@Z 315d3840 f i ParamLoader.obj
 0001:000d2900       ??$move_init@USRecoilJoints@@@NArray@@YAXPAUSRecoilJoints@@0I@Z 315d3900 f i ParamLoader.obj
 0001:000d2900       ??$move_init@USJointsAimIK_Rot@@@NArray@@YAXPAUSJointsAimIK_Rot@@0I@Z 315d3900 f i ParamLoader.obj
 0001:000d2950       ??$move_init@F@NArray@@YAXPAF0I@Z 315d3950 f i ParamLoader.obj
 0001:000d2950       ??$move_init@UTCBFlags@@@NArray@@YAXPAUTCBFlags@@0I@Z 315d3950 f i LoaderTCB.obj
 0001:000d2950       ??$move_init@G@NArray@@YAXPAG0I@Z 315d3950 f i LoaderCHR.obj
 0001:000d2990       ?TrimLeft@?$CryStackStringT@D$0CAA@@@QAEAAV1@PBD@Z 315d3990 f i ParamLoader.obj
 0001:000d2a00       ?GetNameCStr@CSkel@@QBEPBDXZ 315d3a00 f i ParamLoader.obj
 0001:000d2a40       ?ListProcessed@CParamLoader@@AAEHPBD@Z 315d3a40 f   ParamLoader.obj
 0001:000d2aa0       ?resize_raw@?$SmallDynStorage@USJointsAimIK_Rot@@HUStandardAlloc@NAlloc@@@NArray@@QAEXHH_N@Z 315d3aa0 f i ParamLoader.obj
 0001:000d2bf0       ?resize_raw@?$SmallDynStorage@USJointsAimIK_Pos@@HUStandardAlloc@NAlloc@@@NArray@@QAEXHH_N@Z 315d3bf0 f i ParamLoader.obj
 0001:000d2d40       ?resize_raw@?$SmallDynStorage@USRecoilJoints@@HUStandardAlloc@NAlloc@@@NArray@@QAEXHH_N@Z 315d3d40 f i ParamLoader.obj
 0001:000d2e90       ?resize_raw@?$SmallDynStorage@UProcAdjust@@HUStandardAlloc@NAlloc@@@NArray@@QAEXHH_N@Z 315d3e90 f i ParamLoader.obj
 0001:000d2fe0       ?resize_raw@?$SmallDynStorage@UADIKTarget@@HUStandardAlloc@NAlloc@@@NArray@@QAEXHH_N@Z 315d3fe0 f i ParamLoader.obj
 0001:000d3130       ?init@?$DynArray@UADIKTarget@@HU?$SmallDynStorage@UADIKTarget@@HUStandardAlloc@NAlloc@@@NArray@@@@KAPAUADIKTarget@@U?$Array@UADIKTarget@@HU?$ArrayStorage@UADIKTarget@@H@NArray@@@@ABU2@@Z 315d4130 f i ParamLoader.obj
 0001:000d3180       ?init@?$DynArray@USAnimFile@@HU?$SmallDynStorage@USAnimFile@@HUStandardAlloc@NAlloc@@@NArray@@@@KAPAUSAnimFile@@U?$Array@USAnimFile@@HU?$ArrayStorage@USAnimFile@@H@NArray@@@@ABU2@@Z 315d4180 f i ParamLoader.obj
 0001:000d31c0       ?set_size@?$SmallDynStorage@UCGlobalHeaderDBA@@HUStandardAlloc@NAlloc@@@NArray@@QAEXH@Z 315d41c0 f i AnimationManager.obj
 0001:000d31c0       ?set_size@?$SmallDynStorage@UBoneWeights8@@HUStandardAlloc@NAlloc@@@NArray@@QAEXH@Z 315d41c0 f i LoaderSKIN.obj
 0001:000d31c0       ?set_size@?$SmallDynStorage@UDirectionalBlends@@HUStandardAlloc@NAlloc@@@NArray@@QAEXH@Z 315d41c0 f i ParamLoader.obj
 0001:000d31c0       ?set_size@?$SmallDynStorage@USPostProcess@@HUStandardAlloc@NAlloc@@@NArray@@QAEXH@Z 315d41c0 f i SkeletonPose.obj
 0001:000d3250       ?set_size@?$SmallDynStorage@USAnimListInfo@@HUStandardAlloc@NAlloc@@@NArray@@QAEXH@Z 315d4250 f i ParamLoader.obj
 0001:000d3250       ?set_size@?$SmallDynStorage@U?$SplineKey@U?$Quat_tpl@M@@@spline@@HUStandardAlloc@NAlloc@@@NArray@@QAEXH@Z 315d4250 f i FaceAnimSequence.obj
 0001:000d32f0       ?init@?$DynArray@USAnimFile@@HU?$SmallDynStorage@USAnimFile@@HUStandardAlloc@NAlloc@@@NArray@@@@KAPAUSAnimFile@@U?$Array@USAnimFile@@HU?$ArrayStorage@USAnimFile@@H@NArray@@@@PBU2@@Z 315d42f0 f i ParamLoader.obj
 0001:000d3340       ??$__find@PAV?$CryStringT@D@@PBD@priv@stlpmtx_std@@YAPAV?$CryStringT@D@@PAV2@0ABQBDABUrandom_access_iterator_tag@1@@Z 315d4340 f i ParamLoader.obj
 0001:000d3510       ??1?$CryStackStringT@D$0CAA@@@QAE@XZ 315d4510 f i LoaderSKIN.obj
 0001:000d3510       ??1?$CryFixedStringT@$0CAA@@@QAE@XZ 315d4510 f i ParamLoader.obj
 0001:000d3530       ?NoAnimationAliasInDependencies@CParamLoader@@AAE_NAAUSAnimListInfo@@PBD@Z 315d4530 f   ParamLoader.obj
 0001:000d35f0       ?NoFacialAnimationAliasInDependencies@CParamLoader@@AAE_NAAUSAnimListInfo@@PBD@Z 315d45f0 f   ParamLoader.obj
 0001:000d36b0       ?set_size@?$SmallDynStorage@GHUStandardAlloc@NAlloc@@@NArray@@QAEXH@Z 315d46b0 f i LoaderCHR.obj
 0001:000d36b0       ?set_size@?$SmallDynStorage@FHUStandardAlloc@NAlloc@@@NArray@@QAEXH@Z 315d46b0 f i ParamLoader.obj
 0001:000d36b0       ?set_size@?$SmallDynStorage@UTCBFlags@@HUStandardAlloc@NAlloc@@@NArray@@QAEXH@Z 315d46b0 f i LoaderTCB.obj
 0001:000d3730       ?expand_raw@?$DynArray@UADIKTarget@@HU?$SmallDynStorage@UADIKTarget@@HUStandardAlloc@NAlloc@@@NArray@@@@IAEPAUADIKTarget@@PAU2@H@Z 315d4730 f i ParamLoader.obj
 0001:000d37c0       ?resize_raw@?$SmallDynStorage@FHUStandardAlloc@NAlloc@@@NArray@@QAEXHH_N@Z 315d47c0 f i ParamLoader.obj
 0001:000d3900       ?resize_raw@?$SmallDynStorage@UIdxAndName@@HUStandardAlloc@NAlloc@@@NArray@@QAEXHH_N@Z 315d4900 f i ParamLoader.obj
 0001:000d3a50       ?set_size@?$SmallDynStorage@USAnimFile@@HUStandardAlloc@NAlloc@@@NArray@@QAEXH@Z 315d4a50 f i ParamLoader.obj
 0001:000d3ae0       ?Left@?$CryStackStringT@D$0CAA@@@QBE?AV1@I@Z 315d4ae0 f i ParamLoader.obj
 0001:000d3b60       ??$GetParentDirectoryStackString@D$0CAA@@PathUtil@@YA?AV?$CryStackStringT@D$0CAA@@@ABV1@H@Z 315d4b60 f i ParamLoader.obj
 0001:000d3c30       ?TrimRight@?$CryStringT@D@@QAEAAV1@PBD@Z 315d4c30 f i ParamLoader.obj
 0001:000d3ca0       ?NoModelTracksDatabaseInDependencies@CParamLoader@@AAE_NAAUSAnimListInfo@@PBD@Z 315d4ca0 f   ParamLoader.obj
 0001:000d3d40       ?LoadIKDefFeetLock@CParamLoader@@AAE_NVXmlNodeRef@@@Z 315d4d40 f   ParamLoader.obj
 0001:000d3e40       ?init@?$DynArray@UDirectionalBlends@@HU?$SmallDynStorage@UDirectionalBlends@@HUStandardAlloc@NAlloc@@@NArray@@@@KAPAUDirectionalBlends@@U?$Array@UDirectionalBlends@@HU?$ArrayStorage@UDirectionalBlends@@H@NArray@@@@ABU2@@Z 315d4e40 f i ParamLoader.obj
 0001:000d3ec0       ?expand_raw@?$DynArray@FHU?$SmallDynStorage@FHUStandardAlloc@NAlloc@@@NArray@@@@IAEPAFPAFH@Z 315d4ec0 f i ParamLoader.obj
 0001:000d3f40       ?expand_raw@?$DynArray@UIdxAndName@@HU?$SmallDynStorage@UIdxAndName@@HUStandardAlloc@NAlloc@@@NArray@@@@IAEPAUIdxAndName@@PAU2@H@Z 315d4f40 f i ParamLoader.obj
 0001:000d3fc0       ?expand_raw@?$DynArray@USAnimFile@@HU?$SmallDynStorage@USAnimFile@@HUStandardAlloc@NAlloc@@@NArray@@@@IAEPAUSAnimFile@@PAU2@H@Z 315d4fc0 f i ParamLoader.obj
 0001:000d4050       ?init@?$DynArray@UModelAnimationHeader@@HU?$SmallDynStorage@UModelAnimationHeader@@HUStandardAlloc@NAlloc@@@NArray@@@@KAPAUModelAnimationHeader@@U?$Array@UModelAnimationHeader@@HU?$ArrayStorage@UModelAnimationHeader@@H@NArray@@@@PBU2@@Z 315d5050 f i ParamLoader.obj
 0001:000d40b0       ??0?$_Vector_base@UFacialAnimationEntry@CAnimationSet@@V?$allocator@UFacialAnimationEntry@CAnimationSet@@@stlpmtx_std@@@priv@stlpmtx_std@@QAE@IABV?$allocator@UFacialAnimationEntry@CAnimationSet@@@2@@Z 315d50b0 f i ParamLoader.obj
 0001:000d4170       ?Tokenize@?$CryStackStringT@D$0CAA@@@QBE?AV1@PBDAAH@Z 315d5170 f i ParamLoader.obj
 0001:000d4270       ??0SAnimFile@@QAE@ABV?$CryStackStringT@D$0CAA@@@0@Z 315d5270 f i ParamLoader.obj
 0001:000d43b0       ?destroy@?$DynArray@UModelAnimationHeader@@HU?$SmallDynStorage@UModelAnimationHeader@@HUStandardAlloc@NAlloc@@@NArray@@@@KAXU?$Array@UModelAnimationHeader@@HU?$ArrayStorage@UModelAnimationHeader@@H@NArray@@@@@Z 315d53b0 f i ParamLoader.obj
 0001:000d43b0       ?destroy@?$DynArray@UBlendSpaceInfo@@HU?$SmallDynStorage@UBlendSpaceInfo@@HUStandardAlloc@NAlloc@@@NArray@@@@KAXU?$Array@UBlendSpaceInfo@@HU?$ArrayStorage@UBlendSpaceInfo@@H@NArray@@@@@Z 315d53b0 f i CharacterManager.obj
 0001:000d4400       ??$__ufill@PAUFacialAnimationEntry@CAnimationSet@@U12@H@priv@stlpmtx_std@@YAXPAUFacialAnimationEntry@CAnimationSet@@0ABU23@ABUrandom_access_iterator_tag@1@PAH@Z 315d5400 f i ParamLoader.obj
 0001:000d4480       ?destroy@?$DynArray@UDirectionalBlends@@HU?$SmallDynStorage@UDirectionalBlends@@HUStandardAlloc@NAlloc@@@NArray@@@@KAXU?$Array@UDirectionalBlends@@HU?$ArrayStorage@UDirectionalBlends@@H@NArray@@@@@Z 315d5480 f i ParamLoader.obj
 0001:000d44d0       ??1IKLimbType@@QAE@XZ      315d54d0 f i ParamLoader.obj
 0001:000d4560       ?MemFindFirst@CParamLoader@@AAE?AUCAF_ID@@PAPBDPBDIU2@@Z 315d5560 f   ParamLoader.obj
 0001:000d4770       ?push_back@?$DynArray@HHU?$SmallDynStorage@HHUStandardAlloc@NAlloc@@@NArray@@@@QAEPAHABH@Z 315d5770 f i ParamLoader.obj
 0001:000d47b0       ??0?$DynArray@FHU?$SmallDynStorage@FHUStandardAlloc@NAlloc@@@NArray@@@@QAE@ABU0@@Z 315d57b0 f i ParamLoader.obj
 0001:000d4840       ??0?$DynArray@HHU?$SmallDynStorage@HHUStandardAlloc@NAlloc@@@NArray@@@@QAE@ABU0@@Z 315d5840 f i ParamLoader.obj
 0001:000d48d0       ??0?$DynArray@UIdxAndName@@HU?$SmallDynStorage@UIdxAndName@@HUStandardAlloc@NAlloc@@@NArray@@@@QAE@ABU0@@Z 315d58d0 f i ParamLoader.obj
 0001:000d4970       ??0?$DynArray@USAnimFile@@HU?$SmallDynStorage@USAnimFile@@HUStandardAlloc@NAlloc@@@NArray@@@@QAE@ABU0@@Z 315d5970 f i ParamLoader.obj
 0001:000d4a00       ??$move_init@UDirectionalBlends@@@NArray@@YAXPAUDirectionalBlends@@0I@Z 315d5a00 f i ParamLoader.obj
 0001:000d4ac0       ?BuildDependencyList@CParamLoader@@AAE_NHAAU?$DynArray@IHU?$SmallDynStorage@IHUStandardAlloc@NAlloc@@@NArray@@@@@Z 315d5ac0 f   ParamLoader.obj
 0001:000d4ba0       ?LoadIKDefAnimDrivenIKTargets@CParamLoader@@AAE_NVXmlNodeRef@@@Z 315d5ba0 f   ParamLoader.obj
 0001:000d4d90       ?LoadIKDefRecoil@CParamLoader@@AAE_NVXmlNodeRef@@@Z 315d5d90 f   ParamLoader.obj
 0001:000d5110       ?resize@?$DynArray@FHU?$SmallDynStorage@FHUStandardAlloc@NAlloc@@@NArray@@@@QAEXH@Z 315d6110 f i ParamLoader.obj
 0001:000d5150       ?resize@?$DynArray@UIdxAndName@@HU?$SmallDynStorage@UIdxAndName@@HUStandardAlloc@NAlloc@@@NArray@@@@QAEXH@Z 315d6150 f i ParamLoader.obj
 0001:000d51b0       ?push_back@?$DynArray@USAnimFile@@HU?$SmallDynStorage@USAnimFile@@HUStandardAlloc@NAlloc@@@NArray@@@@QAEPAUSAnimFile@@ABU2@@Z 315d61b0 f i ParamLoader.obj
 0001:000d51f0       ?resize_raw@?$SmallDynStorage@UDirectionalBlends@@HUStandardAlloc@NAlloc@@@NArray@@QAEXHH_N@Z 315d61f0 f i ParamLoader.obj
 0001:000d5340       ?init@?$DynArray@U?$DynArray@IHU?$SmallDynStorage@IHUStandardAlloc@NAlloc@@@NArray@@@@HU?$SmallDynStorage@U?$DynArray@IHU?$SmallDynStorage@IHUStandardAlloc@NAlloc@@@NArray@@@@HUStandardAlloc@NAlloc@@@NArray@@@@KAPAU?$DynArray@IHU?$SmallDynStorage@IHUStandardAlloc@NAlloc@@@NArray@@@@U?$Array@U?$DynArray@IHU?$SmallDynStorage@IHUStandardAlloc@NAlloc@@@NArray@@@@HU?$ArrayStorage@U?$DynArray@IHU?$SmallDynStorage@IHUStandardAlloc@NAlloc@@@NArray@@@@H@NArray@@@@@Z 315d6340 f i ParamLoader.obj
 0001:000d5400       ??0?$_Impl_vector@UFacialAnimationEntry@CAnimationSet@@V?$allocator@UFacialAnimationEntry@CAnimationSet@@@stlpmtx_std@@@priv@stlpmtx_std@@QAE@ABV012@@Z 315d6400 f i ParamLoader.obj
 0001:000d5470       ??0IKLimbType@@QAE@XZ      315d6470 f i ParamLoader.obj
 0001:000d5550       ?PrepareHeaderList@SAnimListInfo@@QAEXXZ 315d6550 f i ParamLoader.obj
 0001:000d55f0       ?AddIfNewAnimationAlias@CParamLoader@@AAE_NAAUSAnimListInfo@@PBD1@Z 315d65f0 f   ParamLoader.obj
 0001:000d56e0       ?init@?$DynArray@UIKLimbType@@HU?$SmallDynStorage@UIKLimbType@@HUStandardAlloc@NAlloc@@@NArray@@@@KAPAUIKLimbType@@U?$Array@UIKLimbType@@HU?$ArrayStorage@UIKLimbType@@H@NArray@@@@ABU2@@Z 315d66e0 f i ParamLoader.obj
 0001:000d5760       ??0?$DynArray@UModelAnimationHeader@@HU?$SmallDynStorage@UModelAnimationHeader@@HUStandardAlloc@NAlloc@@@NArray@@@@QAE@ABU0@@Z 315d6760 f i ParamLoader.obj
 0001:000d57e0       ??$move_init@UIKLimbType@@@NArray@@YAXPAUIKLimbType@@0I@Z 315d67e0 f i ParamLoader.obj
 0001:000d5880       ??$move_init@U?$DynArray@IHU?$SmallDynStorage@IHUStandardAlloc@NAlloc@@@NArray@@@@@NArray@@YAXPAU?$DynArray@IHU?$SmallDynStorage@IHUStandardAlloc@NAlloc@@@NArray@@@@0I@Z 315d6880 f i ParamLoader.obj
 0001:000d5940       ??$reconstruct@U?$DynArray@V?$CryStringT@D@@HU?$SmallDynStorage@V?$CryStringT@D@@HUStandardAlloc@NAlloc@@@NArray@@@@@stl@@YAXAAU?$DynArray@V?$CryStringT@D@@HU?$SmallDynStorage@V?$CryStringT@D@@HUStandardAlloc@NAlloc@@@NArray@@@@@Z 315d6940 f i ParamLoader.obj
 0001:000d59c0       ?ExpandWildcardsForPath@CParamLoader@@AAEXAAUSAnimListInfo@@PBDI11@Z 315d69c0 f   ParamLoader.obj
 0001:000d5de0       ?resize_raw@?$SmallDynStorage@UIKLimbType@@HUStandardAlloc@NAlloc@@@NArray@@QAEXHH_N@Z 315d6de0 f i ParamLoader.obj
 0001:000d5f30       ??0?$DynArray@V?$CryStringT@D@@HU?$SmallDynStorage@V?$CryStringT@D@@HUStandardAlloc@NAlloc@@@NArray@@@@QAE@ABU0@@Z 315d6f30 f i ParamLoader.obj
 0001:000d5fb0       ?expand_raw@?$DynArray@UIKLimbType@@HU?$SmallDynStorage@UIKLimbType@@HUStandardAlloc@NAlloc@@@NArray@@@@IAEPAUIKLimbType@@PAU2@H@Z 315d6fb0 f i ParamLoader.obj
 0001:000d6040       ?resize_raw@?$SmallDynStorage@U?$DynArray@IHU?$SmallDynStorage@IHUStandardAlloc@NAlloc@@@NArray@@@@HUStandardAlloc@NAlloc@@@NArray@@QAEXHH_N@Z 315d7040 f i ParamLoader.obj
 0001:000d6190       ?_M_insert_overflow_aux@?$_Impl_vector@UFacialAnimationEntry@CAnimationSet@@V?$allocator@UFacialAnimationEntry@CAnimationSet@@@stlpmtx_std@@@priv@stlpmtx_std@@AAEXPAUFacialAnimationEntry@CAnimationSet@@ABU45@ABU__false_type@3@I_N@Z 315d7190 f i ParamLoader.obj
 0001:000d6370       ??1SAnimListInfo@@QAE@XZ   315d7370 f i ParamLoader.obj
 0001:000d65a0       ?clear@?$DynArray@UIKLimbType@@HU?$SmallDynStorage@UIKLimbType@@HUStandardAlloc@NAlloc@@@NArray@@@@QAEXXZ 315d75a0 f i ParamLoader.obj
 0001:000d6610       ??0SAnimListInfo@@QAE@ABU0@@Z 315d7610 f i ParamLoader.obj
 0001:000d66e0       ?expand_raw@?$DynArray@U?$DynArray@IHU?$SmallDynStorage@IHUStandardAlloc@NAlloc@@@NArray@@@@HU?$SmallDynStorage@U?$DynArray@IHU?$SmallDynStorage@IHUStandardAlloc@NAlloc@@@NArray@@@@HUStandardAlloc@NAlloc@@@NArray@@@@IAEPAU?$DynArray@IHU?$SmallDynStorage@IHUStandardAlloc@NAlloc@@@NArray@@@@PAU2@H@Z 315d76e0 f i ParamLoader.obj
 0001:000d6760       ??0SAnimListInfo@@QAE@PBD@Z 315d7760 f i ParamLoader.obj
 0001:000d6a20       ?AddIfNewModelTracksDatabase@CParamLoader@@AAE_NAAUSAnimListInfo@@PBD@Z 315d7a20 f   ParamLoader.obj
 0001:000d6b80       ?LoadIKDefLookIK@CParamLoader@@AAE_NVXmlNodeRef@@@Z 315d7b80 f   ParamLoader.obj
 0001:000d7660       ?LoadIKDefAimIK@CParamLoader@@AAE_NVXmlNodeRef@@@Z 315d8660 f   ParamLoader.obj
 0001:000d8280       ?push_back@?$_Impl_vector@UFacialAnimationEntry@CAnimationSet@@V?$allocator@UFacialAnimationEntry@CAnimationSet@@@stlpmtx_std@@@priv@stlpmtx_std@@QAEXABUFacialAnimationEntry@CAnimationSet@@@Z 315d9280 f i ParamLoader.obj
 0001:000d8310       ??$move_init@USAnimListInfo@@@NArray@@YAXPAUSAnimListInfo@@0I@Z 315d9310 f i ParamLoader.obj
 0001:000d8360       ?ScanDirectoryFiles@SDirectoryEnumeratorHelper@@AAEXABV?$CryStringT@D@@00AAV?$vector@V?$CryStringT@D@@V?$allocator@V?$CryStringT@D@@@stlpmtx_std@@@stlpmtx_std@@@Z 315d9360 f i ParamLoader.obj
 0001:000d8590       ?resize_raw@?$SmallDynStorage@USAnimListInfo@@HUStandardAlloc@NAlloc@@@NArray@@QAEXHH_N@Z 315d9590 f i ParamLoader.obj
 0001:000d8700       ?expand_raw@?$DynArray@USAnimListInfo@@HU?$SmallDynStorage@USAnimListInfo@@HUStandardAlloc@NAlloc@@@NArray@@@@IAEPAUSAnimListInfo@@PAU2@H@Z 315d9700 f i ParamLoader.obj
 0001:000d87a0       ?ScanDirectoryRecursive@SDirectoryEnumeratorHelper@@QAEXABV?$CryStringT@D@@00AAV?$vector@V?$CryStringT@D@@V?$allocator@V?$CryStringT@D@@@stlpmtx_std@@@stlpmtx_std@@@Z 315d97a0 f i ParamLoader.obj
 0001:000d8ad0       ?AddIfNewFacialAnimationAlias@CParamLoader@@AAE_NAAUSAnimListInfo@@PBD1@Z 315d9ad0 f   ParamLoader.obj
 0001:000d8bb0       ?LoadIKDefLimbIK@CParamLoader@@AAE_NVXmlNodeRef@@@Z 315d9bb0 f   ParamLoader.obj
 0001:000d9730       ??1?$DynArray@USAnimListInfo@@HU?$SmallDynStorage@USAnimListInfo@@HUStandardAlloc@NAlloc@@@NArray@@@@QAE@XZ 315da730 f i ParamLoader.obj
 0001:000d9790       ??0CParamLoader@@QAE@XZ    315da790 f   ParamLoader.obj
 0001:000d9830       ?ExpandWildcards@CParamLoader@@QAE_NI_N@Z 315da830 f   ParamLoader.obj
 0001:000dbde0       ?LoadLod@CParamLoader@@AAE_NVXmlNodeRef@@@Z 315dcde0 f   ParamLoader.obj
 0001:000dc100       ?ParseIKDef@CParamLoader@@AAE_NVXmlNodeRef@@@Z 315dd100 f   ParamLoader.obj
 0001:000dc460       ?LoadAnimList@CParamLoader@@AAEHVXmlNodeRef@@PBDV?$CryStringT@D@@AA_N@Z 315dd460 f   ParamLoader.obj
 0001:000dd1c0       ?LoadXML@CParamLoader@@QAE_NPAVCSkel@@V?$CryStringT@D@@QBDAAU?$DynArray@IHU?$SmallDynStorage@IHUStandardAlloc@NAlloc@@@NArray@@@@@Z 315de1c0 f   ParamLoader.obj
 0001:000dd6e0       ?ClearLists@CParamLoader@@QAEXXZ 315de6e0 f   ParamLoader.obj
 0001:000ddb80       ??1CParamLoader@@QAE@XZ    315deb80 f   ParamLoader.obj
 0001:000ddbc0       ?Release@CSkel@@UAEXXZ     315debc0 f   Model.obj
 0001:000ddbe0       ??_EICharacterModelSkeleton@@UAEPAXI@Z 315debe0 f i Model.obj
 0001:000ddbe0       ??_GIFacialAnimSkeletonAnimationEntry@@UAEPAXI@Z 315debe0 f i FaceAnimSequence.obj
 0001:000ddbe0       ??_EIFacialModel@@UAEPAXI@Z 315debe0 f i FacialModel.obj
 0001:000ddbe0       ??_GICharacterModelSkeleton@@UAEPAXI@Z 315debe0 f i Model.obj
 0001:000ddbe0       ??_EIAnimEvents@@UAEPAXI@Z 315debe0 f i CharacterManager.obj
 0001:000ddbe0       ??_EIAnimEventList@@UAEPAXI@Z 315debe0 f i AnimEventList.obj
 0001:000ddbe0       ??_EIFacialAnimSkeletonAnimationEntry@@UAEPAXI@Z 315debe0 f i FaceAnimSequence.obj
 0001:000ddbe0       ??_GIFacialModel@@UAEPAXI@Z 315debe0 f i FacialModel.obj
 0001:000ddbe0       ??_GIAnimEvents@@UAEPAXI@Z 315debe0 f i CharacterManager.obj
 0001:000ddbe0       ??_GIAnimEventList@@UAEPAXI@Z 315debe0 f i AnimEventList.obj
 0001:000ddc10       ??_GICharacterModel@@UAEPAXI@Z 315dec10 f i Model.obj
 0001:000ddc10       ??_EICharacterModel@@UAEPAXI@Z 315dec10 f i Model.obj
 0001:000ddc40       ?strnstr@CryStringUtils@@YAPBDPBD0H@Z 315dec40 f i Model.obj
 0001:000ddcc0       ?GetMeshApproxFlags@@YAHPBDH@Z 315decc0 f   Model.obj
 0001:000ddd50       ?GetTextureMemoryUsage@CSkel@@UBEIPAVICrySizer@@@Z 315ded50 f   Model.obj
 0001:000dddd0       ?GetMeshMemoryUsage@CSkel@@UBEIPAVICrySizer@@@Z 315dedd0 f   Model.obj
 0001:000dde10       ?GetIRenderMesh@CSkel@@UBEPBUIRenderMesh@@H@Z 315dee10 f   Model.obj
 0001:000dde10       ?GetIRenderMesh@CSkel@@UAEPAUIRenderMesh@@H@Z 315dee10 f   Model.obj
 0001:000dde40       ?GetNumLods@CSkel@@UBEIXZ  315dee40 f   Model.obj
 0001:000dde70       ??$move_init@UVirtualExample1D@@@NArray@@YAXPAUVirtualExample1D@@0I@Z 315dee70 f i ParametricSampler.obj
 0001:000dde70       ??$move_init@USJointProperty@@@NArray@@YAXPAUSJointProperty@@0I@Z 315dee70 f i Model.obj
 0001:000dde70       ??$move_init@UNodeDesc@@@NArray@@YAXPAUNodeDesc@@0I@Z 315dee70 f i LoaderCGA.obj
 0001:000dde70       ??$move_init@U?$Vec3_tpl@M@@@NArray@@YAXPAU?$Vec3_tpl@M@@0I@Z 315dee70 f i LoaderSKIN.obj
 0001:000dde70       ??$move_init@UBSBlendable@@@NArray@@YAXPAUBSBlendable@@0I@Z 315dee70 f i CharacterManager.obj
 0001:000ddec0       ?GetJointPhysGeom@CSkel@@UBEPBUphys_geometry@@IH@Z 315deec0 f   Model.obj
 0001:000ddec0       ?GetJointPhysGeom@CSkel@@UAEPAUphys_geometry@@IH@Z 315deec0 f   Model.obj
 0001:000ddee0       ?ParsePhysInfoProperties_ROPE@CSkel@@SA_NAAUCryBonePhysics@@ABU?$DynArray@USJointProperty@@HU?$SmallDynStorage@USJointProperty@@HUStandardAlloc@NAlloc@@@NArray@@@@@Z 315deee0 f   Model.obj
 0001:000de750       ?resize_raw@?$SmallDynStorage@PAVCCharInstance@@HUStandardAlloc@NAlloc@@@NArray@@QAEXHH_N@Z 315df750 f i Model.obj
 0001:000de8a0       ?set_size@?$SmallDynStorage@UModelAnimationHeader@@HUStandardAlloc@NAlloc@@@NArray@@QAEXH@Z 315df8a0 f i LoaderCHR.obj
 0001:000de8a0       ?set_size@?$SmallDynStorage@UVirtualExample1D@@HUStandardAlloc@NAlloc@@@NArray@@QAEXH@Z 315df8a0 f i ParametricSampler.obj
 0001:000de8a0       ?set_size@?$SmallDynStorage@UBSBlendable@@HUStandardAlloc@NAlloc@@@NArray@@QAEXH@Z 315df8a0 f i CharacterManager.obj
 0001:000de8a0       ?set_size@?$SmallDynStorage@USJointInfo@CSkin@@HUStandardAlloc@NAlloc@@@NArray@@QAEXH@Z 315df8a0 f i LoaderSKIN.obj
 0001:000de8a0       ?set_size@?$SmallDynStorage@USEntry@CPoseModifierQueue@@HUStandardAlloc@NAlloc@@@NArray@@QAEXH@Z 315df8a0 f i TransitionQueue.obj
 0001:000de8a0       ?set_size@?$SmallDynStorage@U?$Vec3_tpl@M@@HUStandardAlloc@NAlloc@@@NArray@@QAEXH@Z 315df8a0 f i LoaderSKIN.obj
 0001:000de8a0       ?set_size@?$SmallDynStorage@UNodeDesc@@HUStandardAlloc@NAlloc@@@NArray@@QAEXH@Z 315df8a0 f i LoaderCGA.obj
 0001:000de8a0       ?set_size@?$SmallDynStorage@URChunk@@HUStandardAlloc@NAlloc@@@NArray@@QAEXH@Z 315df8a0 f i LoaderSKIN.obj
 0001:000de8a0       ?set_size@?$SmallDynStorage@UBlendSpaceInfo@@HUStandardAlloc@NAlloc@@@NArray@@QAEXH@Z 315df8a0 f i CharacterManager.obj
 0001:000de8a0       ?set_size@?$SmallDynStorage@USJointProperty@@HUStandardAlloc@NAlloc@@@NArray@@QAEXH@Z 315df8a0 f i Model.obj
 0001:000de930       ?resize_raw@?$SmallDynStorage@USJointProperty@@HUStandardAlloc@NAlloc@@@NArray@@QAEXHH_N@Z 315df930 f i Model.obj
 0001:000dea90       ?CreateFacialInstance@CSkel@@QAEXXZ 315dfa90 f   Model.obj
 0001:000deae0       ?SetJointPhysProperties_ROPE@CSkel@@UAE_NIHABU?$DynArray@USJointProperty@@HU?$SmallDynStorage@USJointProperty@@HUStandardAlloc@NAlloc@@@NArray@@@@@Z 315dfae0 f   Model.obj
 0001:000deb10       ?GetAttachmentTriangle@CSkel@@UAE?AUClosestTri@@ABU?$Vec3_tpl@M@@@Z 315dfb10 f   Model.obj
 0001:000deb60       ?expand_raw@?$DynArray@USJointProperty@@HU?$SmallDynStorage@USJointProperty@@HUStandardAlloc@NAlloc@@@NArray@@@@IAEPAUSJointProperty@@PAU2@H@Z 315dfb60 f i Model.obj
 0001:000debf0       ?expand_raw@?$DynArray@PAVCCharInstance@@HU?$SmallDynStorage@PAVCCharInstance@@HUStandardAlloc@NAlloc@@@NArray@@@@IAEPAPAVCCharInstance@@PAPAV2@H@Z 315dfbf0 f i Model.obj
 0001:000dec70       ??$AddObject@IHU?$SmallDynStorage@IHUStandardAlloc@NAlloc@@@NArray@@@ICrySizer@@QAEXABU?$DynArray@IHU?$SmallDynStorage@IHUStandardAlloc@NAlloc@@@NArray@@@@@Z 315dfc70 f i Model.obj
 0001:000dec70       ??$AddObject@MHU?$SmallDynStorage@MHUStandardAlloc@NAlloc@@@NArray@@@ICrySizer@@QAEXABU?$DynArray@MHU?$SmallDynStorage@MHUStandardAlloc@NAlloc@@@NArray@@@@@Z 315dfc70 f i CharacterInstance.obj
 0001:000dec70       ??$AddObject@HHU?$SmallDynStorage@HHUStandardAlloc@NAlloc@@@NArray@@@ICrySizer@@QAEXABU?$DynArray@HHU?$SmallDynStorage@HHUStandardAlloc@NAlloc@@@NArray@@@@@Z 315dfc70 f i ControllerPQLog.obj
 0001:000ded40       ?SizeOfModelData@CSkel@@QBEIXZ 315dfd40 f   Model.obj
 0001:000defa0       ??$AddObject@U?$DynArray@IHU?$SmallDynStorage@IHUStandardAlloc@NAlloc@@@NArray@@@@HU?$SmallDynStorage@U?$DynArray@IHU?$SmallDynStorage@IHUStandardAlloc@NAlloc@@@NArray@@@@HUStandardAlloc@NAlloc@@@NArray@@@ICrySizer@@QAEXABU?$DynArray@U?$DynArray@IHU?$SmallDynStorage@IHUStandardAlloc@NAlloc@@@NArray@@@@HU?$SmallDynStorage@U?$DynArray@IHU?$SmallDynStorage@IHUStandardAlloc@NAlloc@@@NArray@@@@HUStandardAlloc@NAlloc@@@NArray@@@@@Z 315dffa0 f i Model.obj
 0001:000df0b0       ??$AddObject@GHU?$SmallDynStorage@GHUStandardAlloc@NAlloc@@@NArray@@@ICrySizer@@QAEXABU?$DynArray@GHU?$SmallDynStorage@GHUStandardAlloc@NAlloc@@@NArray@@@@@Z 315e00b0 f i ModelAnimationSet.obj
 0001:000df0b0       ??$AddObject@FHU?$SmallDynStorage@FHUStandardAlloc@NAlloc@@@NArray@@@ICrySizer@@QAEXABU?$DynArray@FHU?$SmallDynStorage@FHUStandardAlloc@NAlloc@@@NArray@@@@@Z 315e00b0 f i Model.obj
 0001:000df180       ?erase@?$DynArray@PAVCAttachmentSKIN@@HU?$SmallDynStorage@PAVCAttachmentSKIN@@HUStandardAlloc@NAlloc@@@NArray@@@@QAEPAPAVCAttachmentSKIN@@PAPAV2@@Z 315e0180 f i ModelSkin.obj
 0001:000df180       ?erase@?$DynArray@PAVCCharInstance@@HU?$SmallDynStorage@PAVCCharInstance@@HUStandardAlloc@NAlloc@@@NArray@@@@QAEPAPAVCCharInstance@@PAPAV2@@Z 315e0180 f i Model.obj
 0001:000df180       ?erase@?$DynArray@PAVCAnimationSet@@HU?$SmallDynStorage@PAVCAnimationSet@@HUStandardAlloc@NAlloc@@@NArray@@@@QAEPAPAVCAnimationSet@@PAPAV2@@Z 315e0180 f i ModelAnimationSet.obj
 0001:000df1d0       ??1?$DynArray@VCModelJoint@@HU?$SmallDynStorage@VCModelJoint@@HUStandardAlloc@NAlloc@@@NArray@@@@QAE@XZ 315e01d0 f i Model.obj
 0001:000df230       ??0?$DynArray@USJointProperty@@HU?$SmallDynStorage@USJointProperty@@HUStandardAlloc@NAlloc@@@NArray@@@@QAE@XZ 315e0230 f i Model.obj
 0001:000df280       ?push_back@?$DynArray@USJointProperty@@HU?$SmallDynStorage@USJointProperty@@HUStandardAlloc@NAlloc@@@NArray@@@@QAEPAUSJointProperty@@ABU2@@Z 315e0280 f i Model.obj
 0001:000df2e0       ??1RecoilDesc@@QAE@XZ      315e02e0 f i Model.obj
 0001:000df360       ?UnregisterInstance@CSkel@@QAEXPAVCCharInstance@@@Z 315e0360 f   Model.obj
 0001:000df3b0       ?UpdatePhysBonePrimitives@CSkel@@QAEXABU?$DynArray@UBONE_ENTITY@@HU?$SmallDynStorage@UBONE_ENTITY@@HUStandardAlloc@NAlloc@@@NArray@@@@H@Z 315e03b0 f   Model.obj
 0001:000df890       ?GetPhysInfoProperties_ROPE@CSkel@@SA?AU?$DynArray@USJointProperty@@HU?$SmallDynStorage@USJointProperty@@HUStandardAlloc@NAlloc@@@NArray@@@@ABUCryBonePhysics@@H@Z 315e0890 f   Model.obj
 0001:000dfd50       ?destroy@?$DynArray@U?$DynArray@IHU?$SmallDynStorage@IHUStandardAlloc@NAlloc@@@NArray@@@@HU?$SmallDynStorage@U?$DynArray@IHU?$SmallDynStorage@IHUStandardAlloc@NAlloc@@@NArray@@@@HUStandardAlloc@NAlloc@@@NArray@@@@KAXU?$Array@U?$DynArray@IHU?$SmallDynStorage@IHUStandardAlloc@NAlloc@@@NArray@@@@HU?$ArrayStorage@U?$DynArray@IHU?$SmallDynStorage@IHUStandardAlloc@NAlloc@@@NArray@@@@H@NArray@@@@@Z 315e0d50 f i Model.obj
 0001:000dfe00       ??$push_back_unique@U?$DynArray@PAVCCharInstance@@HU?$SmallDynStorage@PAVCCharInstance@@HUStandardAlloc@NAlloc@@@NArray@@@@PAVCCharInstance@@@stl@@YA_NAAU?$DynArray@PAVCCharInstance@@HU?$SmallDynStorage@PAVCCharInstance@@HUStandardAlloc@NAlloc@@@NArray@@@@ABQAVCCharInstance@@@Z 315e0e00 f i Model.obj
 0001:000dfe60       ??$AddObject@UMeshCollisionInfo@@HU?$SmallDynStorage@UMeshCollisionInfo@@HUStandardAlloc@NAlloc@@@NArray@@@ICrySizer@@QAEXABU?$DynArray@UMeshCollisionInfo@@HU?$SmallDynStorage@UMeshCollisionInfo@@HUStandardAlloc@NAlloc@@@NArray@@@@@Z 315e0e60 f i Model.obj
 0001:000dff70       ?destroy@?$DynArray@UMeshCollisionInfo@@HU?$SmallDynStorage@UMeshCollisionInfo@@HUStandardAlloc@NAlloc@@@NArray@@@@KAXU?$Array@UMeshCollisionInfo@@HU?$ArrayStorage@UMeshCollisionInfo@@H@NArray@@@@@Z 315e0f70 f i Model.obj
 0001:000e0020       ?RegisterInstance@CSkel@@QAEXPAVCCharInstance@@@Z 315e1020 f   Model.obj
 0001:000e0080       ?GetJointPhysProperties_ROPE@CSkel@@UBE?AU?$DynArray@USJointProperty@@HU?$SmallDynStorage@USJointProperty@@HUStandardAlloc@NAlloc@@@NArray@@@@IH@Z 315e1080 f   Model.obj
 0001:000e0260       ?GetMemoryUsage@CSkel@@QBEXPAVICrySizer@@@Z 315e1260 f   Model.obj
 0001:000e0360       ??0PoseBlenderLookDesc@@QAE@XZ 315e1360 f i Model.obj
 0001:000e0430       ??1PoseBlenderLookDesc@@QAE@XZ 315e1430 f i Model.obj
 0001:000e0520       ??0PoseBlenderAimDesc@@QAE@XZ 315e1520 f i Model.obj
 0001:000e0620       ??1PoseBlenderAimDesc@@QAE@XZ 315e1620 f i Model.obj
 0001:000e06e0       ??1?$DynArray@UIKLimbType@@HU?$SmallDynStorage@UIKLimbType@@HUStandardAlloc@NAlloc@@@NArray@@@@QAE@XZ 315e16e0 f i Model.obj
 0001:000e0740       ??0CModelSkeleton@@QAE@XZ  315e1740 f i Model.obj
 0001:000e08c0       ??_ECModelSkeleton@@W3AEPAXI@Z 315e18c0 f i Model.obj
 0001:000e08d0       ?GetJointParentIDByID@CModelSkeleton@@UBEHH@Z 315e18d0 f i Model.obj
 0001:000e0900       ?GetLimbDefinitionIdx@CModelSkeleton@@UBEH_K@Z 315e1900 f i Model.obj
 0001:000e0940       ??1CModelSkeleton@@UAE@XZ  315e1940 f i Model.obj
 0001:000e0a20       ??_GCModelSkeleton@@UAEPAXI@Z 315e1a20 f i Model.obj
 0001:000e0a20       ??_ECModelSkeleton@@UAEPAXI@Z 315e1a20 f i Model.obj
 0001:000e0a50       ??0CSkel@@QAE@ABV?$CryStringT@D@@IPBD@Z 315e1a50 f   Model.obj
 0001:000e0d20       ?AddRef@CSkel@@UAEXXZ      315e1d20 f i Model.obj
 0001:000e0d30       ?DecRef@CSkel@@UAEXXZ      315e1d30 f i Model.obj
 0001:000e0d40       ?GetAttAbsoluteDefault@CAttachmentFACE@@UBEABU?$QuatT_tpl@M@@XZ 315e1d40 f i AttachmentManager.obj
 0001:000e0d40       ?GetAttAbsoluteDefault@CAttachmentBONE@@UBEABU?$QuatT_tpl@M@@XZ 315e1d40 f i AttachmentManager.obj
 0001:000e0d40       ?GetICharacterModelSkeleton@CSkel@@UAEPAUICharacterModelSkeleton@@XZ 315e1d40 f i Model.obj
 0001:000e0d40       ?GetICharacterModelSkeleton@CSkel@@UBEPBUICharacterModelSkeleton@@XZ 315e1d40 f i Model.obj
 0001:000e0d50       ?GetNamePART@CSkel@@UBEPBDXZ 315e1d50 f i Model.obj
 0001:000e0d50       ?NumCharacters@CharacterManager@@UBEIXZ 315e1d50 f i CharacterManager.obj
 0001:000e0d60       ?GetNumJoints@CSkel@@UBEIXZ 315e1d60 f i Model.obj
 0001:000e0d70       ?GetICharInstanceFromModel@CSkel@@UBEPBUICharacterInstance@@I@Z 315e1d70 f i Model.obj
 0001:000e0d70       ?GetICharInstanceFromModel@CSkel@@UAEPAUICharacterInstance@@I@Z 315e1d70 f i Model.obj
 0001:000e0da0       ?GetNumInstances@CSkel@@UBEIXZ 315e1da0 f i Model.obj
 0001:000e0db0       ??1CSkel@@UAE@XZ           315e1db0 f   Model.obj
 0001:000e0fd0       ??_GCSkel@@UAEPAXI@Z       315e1fd0 f i Model.obj
 0001:000e0fd0       ??_ECSkel@@UAEPAXI@Z       315e1fd0 f i Model.obj
 0001:000e1000       ?GetAnimationDCCWorldSpaceLocation@CAnimationSet@@UBE_NPBDAAU?$QuatT_tpl@M@@@Z 315e2000 f   ModelAnimationSet.obj
 0001:000e1030       ?GetAnimationEndLocation@CAnimationSet@@UBE_NPBDAAU?$QuatT_tpl@M@@@Z 315e2030 f   ModelAnimationSet.obj
 0001:000e1060       ?FindMorphTarget@IAnimationSet@@UAEHPBD@Z 315e2060 f i ModelAnimationSet.obj
 0001:000e1070       ?GetStart@IAnimationSet@@UAEMH@Z 315e2070 f i ModelAnimationSet.obj
 0001:000e1080       ??_EIAnimationSet@@UAEPAXI@Z 315e2080 f i ModelAnimationSet.obj
 0001:000e1080       ??_GIAnimationSet@@UAEPAXI@Z 315e2080 f i ModelAnimationSet.obj
 0001:000e10b0       ?GetModelAnimationHeader@CAnimationSet@@QBEPBUModelAnimationHeader@@H@Z 315e20b0 f   ModelAnimationSet.obj
 0001:000e11b0       ?GetNameByAnimID@CAnimationSet@@UBEPBDH@Z 315e21b0 f   ModelAnimationSet.obj
 0001:000e1240       ?GetCRCByAnimID@CAnimationSet@@UBEIH@Z 315e2240 f   ModelAnimationSet.obj
 0001:000e1270       ?GetFilePathCRCByAnimID@CAnimationSet@@UBEIH@Z 315e2270 f   ModelAnimationSet.obj
 0001:000e12f0       ?IsAnimLoaded@CAnimationSet@@UBE_NH@Z 315e22f0 f   ModelAnimationSet.obj
 0001:000e1400       ?GetGAH_CAF@CAnimationSet@@QBEPAUGlobalAnimationHeaderCAF@@H@Z 315e2400 f   ModelAnimationSet.obj
 0001:000e1480       ?GetGAH_LMG@CAnimationSet@@QAEPAUGlobalAnimationHeaderLMG@@H@Z 315e2480 f   ModelAnimationSet.obj
 0001:000e1500       ?GetDuration_sec@CAnimationSet@@UBEMH@Z 315e2500 f   ModelAnimationSet.obj
 0001:000e1680       ?GetAnimationFlags@CAnimationSet@@UBEIH@Z 315e2680 f   ModelAnimationSet.obj
 0001:000e1780       ?GetAnimationStatus@CAnimationSet@@UBEPBDH@Z 315e2780 f   ModelAnimationSet.obj
 0001:000e1820       ?GetStart@CAnimationSet@@UAEMH@Z 315e2820 f   ModelAnimationSet.obj
 0001:000e18a0       ?GetAnimationDCCWorldSpaceLocation@CAnimationSet@@UBE_NHAAU?$QuatT_tpl@M@@@Z 315e28a0 f   ModelAnimationSet.obj
 0001:000e1980       ?GetFilePathByName@CAnimationSet@@UBEPBDPBD@Z 315e2980 f   ModelAnimationSet.obj
 0001:000e1a50       ?GetFilePathByID@CAnimationSet@@UBEPBDH@Z 315e2a50 f   ModelAnimationSet.obj
 0001:000e1ad0       ?GetGlobalIDByName@CAnimationSet@@UAEHPBD@Z 315e2ad0 f   ModelAnimationSet.obj
 0001:000e1b40       ?GetGlobalIDByAnimID@CAnimationSet@@UAEHH@Z 315e2b40 f   ModelAnimationSet.obj
 0001:000e1b60       ?GetTotalPosKeys@CAnimationSet@@UBEII@Z 315e2b60 f   ModelAnimationSet.obj
 0001:000e1ba0       ?GetTotalRotKeys@CAnimationSet@@UBEII@Z 315e2ba0 f   ModelAnimationSet.obj
 0001:000e1be0       ?GetDBAFilePath@CAnimationSet@@UBEPBDI@Z 315e2be0 f   ModelAnimationSet.obj
 0001:000e1c20       ?VerifyLMGs@CAnimationSet@@QAEXXZ 315e2c20 f   ModelAnimationSet.obj
 0001:000e1d50       ??$__lower_bound@PAUFacialAnimationEntry@CAnimationSet@@PBDU?$less_stricmp@PBD@stl@@U34@H@priv@stlpmtx_std@@YAPAUFacialAnimationEntry@CAnimationSet@@PAU23@0ABQBDU?$less_stricmp@PBD@stl@@2PAH@Z 315e2d50 f i ModelAnimationSet.obj
 0001:000e1dc0       ?resize_raw@?$SmallDynStorage@PAVCAnimationSet@@HUStandardAlloc@NAlloc@@@NArray@@QAEXHH_N@Z 315e2dc0 f i ModelAnimationSet.obj
 0001:000e1f10       ??$__lower_bound@PBIIU?$__less_2@II@priv@stlpmtx_std@@U123@H@priv@stlpmtx_std@@YAPBIPBI0ABIU?$__less_2@II@01@2PAH@Z 315e2f10 f i ModelAnimationSet.obj
 0001:000e1f10       ??$__lower_bound@PAPAVCAnimationSet@@PAV1@U?$__less_2@PAVCAnimationSet@@PAV1@@priv@stlpmtx_std@@U234@H@priv@stlpmtx_std@@YAPAPAVCAnimationSet@@PAPAV2@0ABQAV2@U?$__less_2@PAVCAnimationSet@@PAV1@@01@2PAH@Z 315e2f10 f i ModelAnimationSet.obj
 0001:000e1f10       ??$__lower_bound@PAIIU?$__less_2@II@priv@stlpmtx_std@@U123@H@priv@stlpmtx_std@@YAPAIPAI0ABIU?$__less_2@II@01@2PAH@Z 315e2f10 f i ControllerDefragHeap.obj
 0001:000e1f50       ?numMorphTargets@CAnimationSet@@UBEIXZ 315e2f50 f   ModelAnimationSet.obj
 0001:000e1f80       ?GetNameMorphTarget@CAnimationSet@@UAEPBDH@Z 315e2f80 f   ModelAnimationSet.obj
 0001:000e1ff0       ?GetJointStartLocation@CAnimationSet@@UAE_NPBDHAAU?$QuatT_tpl@M@@@Z 315e2ff0 f   ModelAnimationSet.obj
 0001:000e20f0       ?GetAnimationDCCWorldSpaceLocation@CAnimationSet@@UBE_NPBVCAnimation@@AAU?$QuatT_tpl@M@@@Z 315e30f0 f   ModelAnimationSet.obj
 0001:000e2820       ?GetClosestQuatInChannel@CAnimationSet@@UAEMPBDHABU?$Quat_tpl@M@@@Z 315e3820 f   ModelAnimationSet.obj
 0001:000e2a30       ?ExportCAF2HTR@CAnimationSet@@UAE_NPBD0PBUISkeletonAnim@@@Z 315e3a30 f   ModelAnimationSet.obj
 0001:000e2af0       ?ExportVGrid@CAnimationSet@@UAE_NPBD0PBUISkeletonAnim@@@Z 315e3af0 f   ModelAnimationSet.obj
 0001:000e2b80       ?GetAnimationEndLocation@CAnimationSet@@UBE_NHAAU?$QuatT_tpl@M@@@Z 315e3b80 f   ModelAnimationSet.obj
 0001:000e2fe0       ??$AddObject@IV?$CryStringT@D@@U?$less@I@stlpmtx_std@@V?$allocator@U?$pair@$$CBIV?$CryStringT@D@@@stlpmtx_std@@@3@@ICrySizer@@QAEXABV?$map@IV?$CryStringT@D@@U?$less@I@stlpmtx_std@@V?$allocator@U?$pair@$$CBIV?$CryStringT@D@@@stlpmtx_std@@@3@@stlpmtx_std@@@Z 315e3fe0 f i ModelAnimationSet.obj
 0001:000e3060       ?expand_raw@?$DynArray@PAVCAnimationSet@@HU?$SmallDynStorage@PAVCAnimationSet@@HUStandardAlloc@NAlloc@@@NArray@@@@IAEPAPAVCAnimationSet@@PAPAV2@H@Z 315e4060 f i ModelAnimationSet.obj
 0001:000e30e0       ?GetFacialAnimationPathByName@CAnimationSet@@UAEPBDPBD@Z 315e40e0 f   ModelAnimationSet.obj
 0001:000e3150       ?GetFacialAnimationName@CAnimationSet@@UAEPBDH@Z 315e4150 f   ModelAnimationSet.obj
 0001:000e3190       ?GetFacialAnimationPath@CAnimationSet@@UAEPBDH@Z 315e4190 f   ModelAnimationSet.obj
 0001:000e31d0       ?PrepareToReuseAnimations@CAnimationSet@@QAEXI@Z 315e41d0 f   ModelAnimationSet.obj
 0001:000e3270       ?SizeOfAnimationSet@CAnimationSet@@QBEIXZ 315e4270 f   ModelAnimationSet.obj
 0001:000e3450       ??$AddObject@UModelAnimationHeader@@HU?$SmallDynStorage@UModelAnimationHeader@@HUStandardAlloc@NAlloc@@@NArray@@@ICrySizer@@QAEXABU?$DynArray@UModelAnimationHeader@@HU?$SmallDynStorage@UModelAnimationHeader@@HUStandardAlloc@NAlloc@@@NArray@@@@@Z 315e4450 f i ModelAnimationSet.obj
 0001:000e34e0       ??$AddObject@UFacialAnimationEntry@CAnimationSet@@V?$allocator@UFacialAnimationEntry@CAnimationSet@@@stlpmtx_std@@@ICrySizer@@QAEXABV?$vector@UFacialAnimationEntry@CAnimationSet@@V?$allocator@UFacialAnimationEntry@CAnimationSet@@@stlpmtx_std@@@stlpmtx_std@@@Z 315e44e0 f i ModelAnimationSet.obj
 0001:000e3570       ?SizeOfLMG@GlobalAnimationHeaderLMG@@QBEIXZ 315e4570 f i ModelAnimationSet.obj
 0001:000e37c0       ?GetValue@CAnimationSet@@ABEIPBD@Z 315e47c0 f i ModelAnimationSet.obj
 0001:000e38c0       ?insert_raw@?$DynArray@IHU?$SmallDynStorage@IHUStandardAlloc@NAlloc@@@NArray@@@@QAE?AU?$Array@IHU?$ArrayStorage@IH@NArray@@@@PAIH@Z 315e48c0 f i ModelAnimationSet.obj
 0001:000e3950       ?insert_raw@?$DynArray@GHU?$SmallDynStorage@GHUStandardAlloc@NAlloc@@@NArray@@@@QAE?AU?$Array@GHU?$ArrayStorage@GH@NArray@@@@PAGH@Z 315e4950 f i ModelAnimationSet.obj
 0001:000e39e0       ?insert_raw@?$DynArray@PAVCAnimationSet@@HU?$SmallDynStorage@PAVCAnimationSet@@HUStandardAlloc@NAlloc@@@NArray@@@@QAE?AU?$Array@PAVCAnimationSet@@HU?$ArrayStorage@PAVCAnimationSet@@H@NArray@@@@PAPAVCAnimationSet@@H@Z 315e49e0 f i ModelAnimationSet.obj
 0001:000e3a70       ?GetAnimIDByName@CAnimationSet@@UBEHPBD@Z 315e4a70 f   ModelAnimationSet.obj
 0001:000e3ac0       ?GetAnimIDByCRC@CAnimationSet@@UBEHI@Z 315e4ac0 f   ModelAnimationSet.obj
 0001:000e3b30       ?GetAnimationSize@CAnimationSet@@UBEII@Z 315e4b30 f   ModelAnimationSet.obj
 0001:000e3ba0       ?_M_create_node@?$_Rb_tree@IU?$less@I@stlpmtx_std@@U?$pair@$$CBIV?$CryStringT@D@@@2@U?$_Select1st@U?$pair@$$CBIV?$CryStringT@D@@@stlpmtx_std@@@priv@2@U?$_MapTraitsT@U?$pair@$$CBIV?$CryStringT@D@@@stlpmtx_std@@@52@V?$allocator@U?$pair@$$CBIV?$CryStringT@D@@@stlpmtx_std@@@2@@priv@stlpmtx_std@@IAEPAU_Rb_tree_node_base@23@ABU?$pair@$$CBIV?$CryStringT@D@@@3@@Z 315e4ba0 f i ModelAnimationSet.obj
 0001:000e3c10       ?_M_erase@?$_Rb_tree@IU?$less@I@stlpmtx_std@@U?$pair@$$CBIV?$CryStringT@D@@@2@U?$_Select1st@U?$pair@$$CBIV?$CryStringT@D@@@stlpmtx_std@@@priv@2@U?$_MapTraitsT@U?$pair@$$CBIV?$CryStringT@D@@@stlpmtx_std@@@52@V?$allocator@U?$pair@$$CBIV?$CryStringT@D@@@stlpmtx_std@@@2@@priv@stlpmtx_std@@AAEXPAU_Rb_tree_node_base@23@@Z 315e4c10 f i ModelAnimationSet.obj
 0001:000e3c70       ?Register@CAnimationManager@@QAEXPAVCAnimationSet@@@Z 315e4c70 f i ModelAnimationSet.obj
 0001:000e3ce0       ?InsertHash@CAnimationSet@@AAEXII@Z 315e4ce0 f i ModelAnimationSet.obj
 0001:000e3d90       ?_M_insert@?$_Rb_tree@IU?$less@I@stlpmtx_std@@U?$pair@$$CBIV?$CryStringT@D@@@2@U?$_Select1st@U?$pair@$$CBIV?$CryStringT@D@@@stlpmtx_std@@@priv@2@U?$_MapTraitsT@U?$pair@$$CBIV?$CryStringT@D@@@stlpmtx_std@@@52@V?$allocator@U?$pair@$$CBIV?$CryStringT@D@@@stlpmtx_std@@@2@@priv@stlpmtx_std@@AAE?AU?$_Rb_tree_iterator@U?$pair@$$CBIV?$CryStringT@D@@@stlpmtx_std@@U?$_MapTraitsT@U?$pair@$$CBIV?$CryStringT@D@@@stlpmtx_std@@@priv@2@@23@PAU_Rb_tree_node_base@23@ABU?$pair@$$CBIV?$CryStringT@D@@@3@00@Z 315e4d90 f i ModelAnimationSet.obj
 0001:000e3e20       ?insert_unique@?$_Rb_tree@IU?$less@I@stlpmtx_std@@U?$pair@$$CBIV?$CryStringT@D@@@2@U?$_Select1st@U?$pair@$$CBIV?$CryStringT@D@@@stlpmtx_std@@@priv@2@U?$_MapTraitsT@U?$pair@$$CBIV?$CryStringT@D@@@stlpmtx_std@@@52@V?$allocator@U?$pair@$$CBIV?$CryStringT@D@@@stlpmtx_std@@@2@@priv@stlpmtx_std@@QAE?AU?$pair@U?$_Rb_tree_iterator@U?$pair@$$CBIV?$CryStringT@D@@@stlpmtx_std@@U?$_MapTraitsT@U?$pair@$$CBIV?$CryStringT@D@@@stlpmtx_std@@@priv@2@@priv@stlpmtx_std@@_N@3@ABU?$pair@$$CBIV?$CryStringT@D@@@3@@Z 315e4e20 f i ModelAnimationSet.obj
 0001:000e3f30       ?Init@CAnimationSet@@QAEXXZ 315e4f30 f   ModelAnimationSet.obj
 0001:000e3f50       ?prepareLoadCAFs@CAnimationSet@@QAEXI@Z 315e4f50 f   ModelAnimationSet.obj
 0001:000e3fc0       ?prepareLoadANMs@CAnimationSet@@QAEXI@Z 315e4fc0 f   ModelAnimationSet.obj
 0001:000e4020       ?GetMemoryUsage@CAnimationSet@@QBEXPAVICrySizer@@@Z 315e5020 f   ModelAnimationSet.obj
 0001:000e4070       ?insert_unique@?$_Rb_tree@IU?$less@I@stlpmtx_std@@U?$pair@$$CBIV?$CryStringT@D@@@2@U?$_Select1st@U?$pair@$$CBIV?$CryStringT@D@@@stlpmtx_std@@@priv@2@U?$_MapTraitsT@U?$pair@$$CBIV?$CryStringT@D@@@stlpmtx_std@@@52@V?$allocator@U?$pair@$$CBIV?$CryStringT@D@@@stlpmtx_std@@@2@@priv@stlpmtx_std@@QAE?AU?$_Rb_tree_iterator@U?$pair@$$CBIV?$CryStringT@D@@@stlpmtx_std@@U?$_MapTraitsT@U?$pair@$$CBIV?$CryStringT@D@@@stlpmtx_std@@@priv@2@@23@U423@ABU?$pair@$$CBIV?$CryStringT@D@@@3@@Z 315e5070 f i ModelAnimationSet.obj
 0001:000e4260       ?ReuseAnimation@CAnimationSet@@QAEXABUModelAnimationHeader@@@Z 315e5260 f   ModelAnimationSet.obj
 0001:000e42c0       ?ReleaseAnimationData@CAnimationSet@@QAEXXZ 315e52c0 f   ModelAnimationSet.obj
 0001:000e4630       ??$?AI@?$map@IV?$CryStringT@D@@U?$less@I@stlpmtx_std@@V?$allocator@U?$pair@$$CBIV?$CryStringT@D@@@stlpmtx_std@@@3@@stlpmtx_std@@QAEAAV?$CryStringT@D@@ABI@Z 315e5630 f i ModelAnimationSet.obj
 0001:000e4720       ??1CAnimationSet@@UAE@XZ   315e5720 f   ModelAnimationSet.obj
 0001:000e48a0       ??0CAnimationSet@@QAE@XZ   315e58a0 f   ModelAnimationSet.obj
 0001:000e49c0       ??_ECAnimationSet@@UAEPAXI@Z 315e59c0 f i ModelAnimationSet.obj
 0001:000e49c0       ??_GCAnimationSet@@UAEPAXI@Z 315e59c0 f i ModelAnimationSet.obj
 0001:000e49f0       ?LoadFileCAF@CAnimationSet@@QAEHPBD0@Z 315e59f0 f   ModelAnimationSet.obj
 0001:000e4c20       ?LoadFileAIM@CAnimationSet@@QAEHPBD0@Z 315e5c20 f   ModelAnimationSet.obj
 0001:000e4f50       ?LoadFileANM@CAnimationSet@@QAEHPBD0AAU?$DynArray@UCControllerTCB@@HU?$SmallDynStorage@UCControllerTCB@@HUStandardAlloc@NAlloc@@@NArray@@@@PAVCryCGALoader@@@Z 315e5f50 f   ModelAnimationSet.obj
 0001:000e5150       ?LoadFileLMG@CAnimationSet@@QAEHPBD0@Z 315e6150 f   ModelAnimationSet.obj
 0001:000e53b0       ?AddAnimationByPath@CAnimationSet@@UAEHPBD0@Z 315e63b0 f   ModelAnimationSet.obj
 0001:000e5470       ?TriExtent@@YAMW4EGeomForm@@ABU?$Vec3_tpl@M@@11@Z 315e6470 f i ModelMesh.obj
 0001:000e5670       ?GetAttachmentTriangle@CModelMesh@@QAE?AUClosestTri@@PAUIRenderMesh@@ABU?$Vec3_tpl@M@@@Z 315e6670 f   ModelMesh.obj
 0001:000e5a70       ??$AddObject@UDirectionalBlends@@HU?$SmallDynStorage@UDirectionalBlends@@HUStandardAlloc@NAlloc@@@NArray@@@ICrySizer@@QAEXABU?$DynArray@UDirectionalBlends@@HU?$SmallDynStorage@UDirectionalBlends@@HUStandardAlloc@NAlloc@@@NArray@@@@@Z 315e6a70 f i ModelSkeleton.obj
 0001:000e5a70       ??$AddObject@USPostProcess@@HU?$SmallDynStorage@USPostProcess@@HUStandardAlloc@NAlloc@@@NArray@@@ICrySizer@@QAEXABU?$DynArray@USPostProcess@@HU?$SmallDynStorage@USPostProcess@@HUStandardAlloc@NAlloc@@@NArray@@@@@Z 315e6a70 f i SkeletonPose_Debug.obj
 0001:000e5a70       ??$AddObject@UBoneWeights8@@HU?$SmallDynStorage@UBoneWeights8@@HUStandardAlloc@NAlloc@@@NArray@@@ICrySizer@@QAEXABU?$DynArray@UBoneWeights8@@HU?$SmallDynStorage@UBoneWeights8@@HUStandardAlloc@NAlloc@@@NArray@@@@@Z 315e6a70 f i ModelMesh.obj
 0001:000e5b50       ?SizeOfModelMesh@CModelMesh@@QBEIXZ 315e6b50 f   ModelMesh.obj
 0001:000e5e30       ??$AddObject@UMorphTargetVertex@@HU?$SmallDynStorage@UMorphTargetVertex@@HUStandardAlloc@NAlloc@@@NArray@@@ICrySizer@@QAEXABU?$DynArray@UMorphTargetVertex@@HU?$SmallDynStorage@UMorphTargetVertex@@HUStandardAlloc@NAlloc@@@NArray@@@@@Z 315e6e30 f i ModelMesh.obj
 0001:000e5f10       ?ComputeExtent@CModelMesh@@QAEMAAUGeomQuery@@W4EGeomForm@@PAUIRenderMesh@@@Z 315e6f10 f   ModelMesh.obj
 0001:000e6110       ?InitSWSkinBuffer@CModelMesh@@QAEIPAUIRenderMesh@@@Z 315e7110 f   ModelMesh.obj
 0001:000e69b0       ??$AddObject@URChunk@@HU?$SmallDynStorage@URChunk@@HUStandardAlloc@NAlloc@@@NArray@@@ICrySizer@@QAEXABU?$DynArray@URChunk@@HU?$SmallDynStorage@URChunk@@HUStandardAlloc@NAlloc@@@NArray@@@@@Z 315e79b0 f i ModelMesh.obj
 0001:000e6a40       ??$AddObject@V?$_smart_ptr@UCMorphTarget@@@@HU?$SmallDynStorage@V?$_smart_ptr@UCMorphTarget@@@@HUStandardAlloc@NAlloc@@@NArray@@@ICrySizer@@QAEXABU?$DynArray@V?$_smart_ptr@UCMorphTarget@@@@HU?$SmallDynStorage@V?$_smart_ptr@UCMorphTarget@@@@HUStandardAlloc@NAlloc@@@NArray@@@@@Z 315e7a40 f i ModelMesh.obj
 0001:000e6b50       ?GetMemoryUsage@CModelMesh@@QBEXPAVICrySizer@@@Z 315e7b50 f   ModelMesh.obj
 0001:000e6bc0       ?CopyPhysInfo@@YAXAAUCryBonePhysics@@ABUCryBonePhysics_Comp@@@Z 315e7bc0 f i ModelSkeleton.obj
 0001:000e6c70       ?PostInitialize@CModelJoint@@QAEXABVCPoseData@Skeleton@@@Z 315e7c70 f   ModelSkeleton.obj
 0001:000e6eb0       ?Retrieve@?$CInt32HashMap@E$0CAA@@@QBEHI@Z 315e7eb0 f i ModelSkeleton.obj
 0001:000e6f00       ?SetIKJointID@CModelSkeleton@@QAEXXZ 315e7f00 f   ModelSkeleton.obj
 0001:000e7040       ?GetJointIDByCRC32@CModelSkeleton@@UBEHI@Z 315e8040 f   ModelSkeleton.obj
 0001:000e7060       ?GetJointNameByID@CModelSkeleton@@UBEPBDH@Z 315e8060 f   ModelSkeleton.obj
 0001:000e70a0       ?SizeOfEmptyPhysics@CModelSkeleton@@QBEIXZ 315e80a0 f   ModelSkeleton.obj
 0001:000e70e0       ??1CModelJoint@@QAE@XZ     315e80e0 f   ModelSkeleton.obj
 0001:000e71a0       ?GetJointIDByName@CModelSkeleton@@UBEHPBD@Z 315e81a0 f   ModelSkeleton.obj
 0001:000e71d0       ?get_alloc_size@?$SmallDynStorage@VCModelJoint@@HUStandardAlloc@NAlloc@@@NArray@@QBEHXZ 315e81d0 f i ModelSkeleton.obj
 0001:000e7220       ?get_alloc_size@?$SmallDynStorage@UIKLimbType@@HUStandardAlloc@NAlloc@@@NArray@@QBEHXZ 315e8220 f i ModelSkeleton.obj
 0001:000e7270       ??$AddObject@UCCGAJoint@@HU?$SmallDynStorage@UCCGAJoint@@HUStandardAlloc@NAlloc@@@NArray@@@ICrySizer@@QAEXABU?$DynArray@UCCGAJoint@@HU?$SmallDynStorage@UCCGAJoint@@HUStandardAlloc@NAlloc@@@NArray@@@@@Z 315e8270 f i SkeletonPose_Debug.obj
 0001:000e7270       ??$AddObject@USRecoilJoints@@HU?$SmallDynStorage@USRecoilJoints@@HUStandardAlloc@NAlloc@@@NArray@@@ICrySizer@@QAEXABU?$DynArray@USRecoilJoints@@HU?$SmallDynStorage@USRecoilJoints@@HUStandardAlloc@NAlloc@@@NArray@@@@@Z 315e8270 f i ModelSkeleton.obj
 0001:000e7270       ??$AddObject@USJointsAimIK_Rot@@HU?$SmallDynStorage@USJointsAimIK_Rot@@HUStandardAlloc@NAlloc@@@NArray@@@ICrySizer@@QAEXABU?$DynArray@USJointsAimIK_Rot@@HU?$SmallDynStorage@USJointsAimIK_Rot@@HUStandardAlloc@NAlloc@@@NArray@@@@@Z 315e8270 f i ModelSkeleton.obj
 0001:000e7270       ??$AddObject@U?$Quat_tpl@M@@HU?$SmallDynStorage@U?$Quat_tpl@M@@HUStandardAlloc@NAlloc@@@NArray@@@ICrySizer@@QAEXABU?$DynArray@U?$Quat_tpl@M@@HU?$SmallDynStorage@U?$Quat_tpl@M@@HUStandardAlloc@NAlloc@@@NArray@@@@@Z 315e8270 f i ModelMesh.obj
 0001:000e7350       ?_M_create_node@?$_Rb_tree@IU?$less@I@stlpmtx_std@@U?$pair@$$CBIPAVCModelJoint@@@2@U?$_Select1st@U?$pair@$$CBIPAVCModelJoint@@@stlpmtx_std@@@priv@2@U?$_MapTraitsT@U?$pair@$$CBIPAVCModelJoint@@@stlpmtx_std@@@52@V?$allocator@U?$pair@$$CBIPAVCModelJoint@@@stlpmtx_std@@@2@@priv@stlpmtx_std@@IAEPAU_Rb_tree_node_base@23@ABU?$pair@$$CBIPAVCModelJoint@@@3@@Z 315e8350 f i ModelSkeleton.obj
 0001:000e7350       ?_M_create_node@?$_Rb_tree@HU?$less@H@stlpmtx_std@@U?$pair@$$CBHPAUphys_geometry@@@2@U?$_Select1st@U?$pair@$$CBHPAUphys_geometry@@@stlpmtx_std@@@priv@2@U?$_MapTraitsT@U?$pair@$$CBHPAUphys_geometry@@@stlpmtx_std@@@52@V?$allocator@U?$pair@$$CBHPAUphys_geometry@@@stlpmtx_std@@@2@@priv@stlpmtx_std@@IAEPAU_Rb_tree_node_base@23@ABU?$pair@$$CBHPAUphys_geometry@@@3@@Z 315e8350 f i LoaderCHR.obj
 0001:000e7350       ?_M_create_node@?$_Rb_tree@IU?$less@I@stlpmtx_std@@U?$pair@$$CBIPAV?$vector@HV?$allocator@H@stlpmtx_std@@@stlpmtx_std@@@2@U?$_Select1st@U?$pair@$$CBIPAV?$vector@HV?$allocator@H@stlpmtx_std@@@stlpmtx_std@@@stlpmtx_std@@@priv@2@U?$_MapTraitsT@U?$pair@$$CBIPAV?$vector@HV?$allocator@H@stlpmtx_std@@@stlpmtx_std@@@stlpmtx_std@@@52@V?$allocator@U?$pair@$$CBIPAV?$vector@HV?$allocator@H@stlpmtx_std@@@stlpmtx_std@@@stlpmtx_std@@@2@@priv@stlpmtx_std@@IAEPAU_Rb_tree_node_base@23@ABU?$pair@$$CBIPAV?$vector@HV?$allocator@H@stlpmtx_std@@@stlpmtx_std@@@3@@Z 315e8350 f i AnimationManager.obj
 0001:000e7350       ?_M_create_node@?$_Rb_tree@PAUIFacialEffector@@U?$less@PAUIFacialEffector@@@stlpmtx_std@@U?$pair@QAUIFacialEffector@@PAU1@@3@U?$_Select1st@U?$pair@QAUIFacialEffector@@PAU1@@stlpmtx_std@@@priv@3@U?$_MapTraitsT@U?$pair@QAUIFacialEffector@@PAU1@@stlpmtx_std@@@63@V?$allocator@U?$pair@QAUIFacialEffector@@PAU1@@stlpmtx_std@@@3@@priv@stlpmtx_std@@IAEPAU_Rb_tree_node_base@23@ABU?$pair@QAUIFacialEffector@@PAU1@@3@@Z 315e8350 f i FaceEffectorLibrary.obj
 0001:000e7350       ?_M_create_node@?$_Rb_tree@IU?$less@I@stlpmtx_std@@U?$pair@$$CBIPAV?$vector@IV?$allocator@I@stlpmtx_std@@@stlpmtx_std@@@2@U?$_Select1st@U?$pair@$$CBIPAV?$vector@IV?$allocator@I@stlpmtx_std@@@stlpmtx_std@@@stlpmtx_std@@@priv@2@U?$_MapTraitsT@U?$pair@$$CBIPAV?$vector@IV?$allocator@I@stlpmtx_std@@@stlpmtx_std@@@stlpmtx_std@@@52@V?$allocator@U?$pair@$$CBIPAV?$vector@IV?$allocator@I@stlpmtx_std@@@stlpmtx_std@@@stlpmtx_std@@@2@@priv@stlpmtx_std@@IAEPAU_Rb_tree_node_base@23@ABU?$pair@$$CBIPAV?$vector@IV?$allocator@I@stlpmtx_std@@@stlpmtx_std@@@3@@Z 315e8350 f i AnimationManager.obj
 0001:000e7350       ?_M_create_node@?$_Rb_tree@IU?$less@I@stlpmtx_std@@U?$pair@$$CBII@2@U?$_Select1st@U?$pair@$$CBII@stlpmtx_std@@@priv@2@U?$_MapTraitsT@U?$pair@$$CBII@stlpmtx_std@@@52@V?$allocator@U?$pair@$$CBII@stlpmtx_std@@@2@@priv@stlpmtx_std@@IAEPAU_Rb_tree_node_base@23@ABU?$pair@$$CBII@3@@Z 315e8350 f i CharacterManager.obj
 0001:000e73a0       ?SizeOfSkeleton@CModelSkeleton@@QBEIXZ 315e83a0 f   ModelSkeleton.obj
 0001:000e7880       ??$AddObject@VCModelJoint@@HU?$SmallDynStorage@VCModelJoint@@HUStandardAlloc@NAlloc@@@NArray@@@ICrySizer@@QAEXABU?$DynArray@VCModelJoint@@HU?$SmallDynStorage@VCModelJoint@@HUStandardAlloc@NAlloc@@@NArray@@@@@Z 315e8880 f i ModelSkeleton.obj
 0001:000e7930       ?PostInitPhysGeom@CModelJoint@@QAE_NAAV?$map@HPAUphys_geometry@@U?$less@H@stlpmtx_std@@V?$allocator@U?$pair@$$CBHPAUphys_geometry@@@stlpmtx_std@@@3@@stlpmtx_std@@H_N@Z 315e8930 f   ModelSkeleton.obj
 0001:000e7a10       ?AddHierarchyToControllerIdMap@CModelJoint@@QAEXAAV?$map@IPAVCModelJoint@@U?$less@I@stlpmtx_std@@V?$allocator@U?$pair@$$CBIPAVCModelJoint@@@stlpmtx_std@@@3@@stlpmtx_std@@@Z 315e8a10 f   ModelSkeleton.obj
 0001:000e7a70       ??$AddObject@UIKLimbType@@HU?$SmallDynStorage@UIKLimbType@@HUStandardAlloc@NAlloc@@@NArray@@@ICrySizer@@QAEXABU?$DynArray@UIKLimbType@@HU?$SmallDynStorage@UIKLimbType@@HUStandardAlloc@NAlloc@@@NArray@@@@@Z 315e8a70 f i ModelSkeleton.obj
 0001:000e7b10       ?UpdateHierarchyPhysics@CModelJoint@@QAEXABU?$DynArray@UBONE_ENTITY@@HU?$SmallDynStorage@UBONE_ENTITY@@HUStandardAlloc@NAlloc@@@NArray@@@@H@Z 315e8b10 f   ModelSkeleton.obj
 0001:000e7da0       ?GetMemoryUsage@CModelSkeleton@@QBEXPAVICrySizer@@@Z 315e8da0 f   ModelSkeleton.obj
 0001:000e7f80       ?GetAnimEventList@CAnimationManager@@UAEPAUIAnimEventList@@PBD@Z 315e8f80 f   AnimationManager.obj
 0001:000e7f90       ?DestroyRunTimePools@CAnimationManager@@QAEXXZ 315e8f90 f   AnimationManager.obj
 0001:000e7fc0       ?AnimationReleaseCAF@CAnimationManager@@QAEXAAUGlobalAnimationHeaderCAF@@@Z 315e8fc0 f   AnimationManager.obj
 0001:000e7fe0       ?AnimationReleaseLMG@CAnimationManager@@QAEXAAUGlobalAnimationHeaderLMG@@@Z 315e8fe0 f   AnimationManager.obj
 0001:000e8000       ?InitialiseRunTimePools@CAnimationManager@@QAEXXZ 315e9000 f   AnimationManager.obj
 0001:000e8140       ??E?$_Rb_tree_iterator@U?$pair@$$CBHPAUphys_geometry@@@stlpmtx_std@@U?$_MapTraitsT@U?$pair@$$CBHPAUphys_geometry@@@stlpmtx_std@@@priv@2@@priv@stlpmtx_std@@QAEAAU012@XZ 315e9140 f i LoaderCHR.obj
 0001:000e8140       ??E?$_Rb_tree_iterator@U?$pair@$$CBII@stlpmtx_std@@U?$_MapTraitsT@U?$pair@$$CBII@stlpmtx_std@@@priv@2@@priv@stlpmtx_std@@QAEAAU012@XZ 315e9140 f i CharacterManager.obj
 0001:000e8140       ??E?$_Rb_tree_iterator@U?$pair@$$CBIV?$_smart_ptr@VCFacialEffector@@@@@stlpmtx_std@@U?$_MapTraitsT@U?$pair@$$CBIV?$_smart_ptr@VCFacialEffector@@@@@stlpmtx_std@@@priv@2@@priv@stlpmtx_std@@QAEAAU012@XZ 315e9140 f i FaceEffectorLibrary.obj
 0001:000e8140       ??E?$_Rb_tree_iterator@U?$pair@$$CBV?$CryStringT@D@@V?$_smart_ptr@UIFacialAnimSequence@@@@@stlpmtx_std@@U?$_MapTraitsT@U?$pair@$$CBV?$CryStringT@D@@V?$_smart_ptr@UIFacialAnimSequence@@@@@stlpmtx_std@@@priv@2@@priv@stlpmtx_std@@QAEAAU012@XZ 315e9140 f i FaceAnimation.obj
 0001:000e8140       ??E?$_Rb_tree_iterator@U?$pair@$$CBIV?$CryStringT@D@@@stlpmtx_std@@U?$_MapTraitsT@U?$pair@$$CBIV?$CryStringT@D@@@stlpmtx_std@@@priv@2@@priv@stlpmtx_std@@QAEAAU012@XZ 315e9140 f i ModelAnimationSet.obj
 0001:000e8140       ??E?$_Rb_tree_iterator@U?$pair@$$CBIPAV?$vector@IV?$allocator@I@stlpmtx_std@@@stlpmtx_std@@@stlpmtx_std@@U?$_MapTraitsT@U?$pair@$$CBIPAV?$vector@IV?$allocator@I@stlpmtx_std@@@stlpmtx_std@@@stlpmtx_std@@@priv@2@@priv@stlpmtx_std@@QAEAAU012@XZ 315e9140 f i AnimationManager.obj
 0001:000e8140       ??E?$_Rb_tree_iterator@U?$pair@$$CBIUSFacialDisplaceInfo@CFacialModel@@@stlpmtx_std@@U?$_MapTraitsT@U?$pair@$$CBIUSFacialDisplaceInfo@CFacialModel@@@stlpmtx_std@@@priv@2@@priv@stlpmtx_std@@QAEAAU012@XZ 315e9140 f i FacialModel.obj
 0001:000e8140       ??E?$_Rb_tree_iterator@U?$pair@$$CBIPAV?$vector@HV?$allocator@H@stlpmtx_std@@@stlpmtx_std@@@stlpmtx_std@@U?$_MapTraitsT@U?$pair@$$CBIPAV?$vector@HV?$allocator@H@stlpmtx_std@@@stlpmtx_std@@@stlpmtx_std@@@priv@2@@priv@stlpmtx_std@@QAEAAU012@XZ 315e9140 f i AnimationManager.obj
 0001:000e8180       ?FindGlobalHeaderByCRC_DBA@CAnimationManager@@QAEPAUCGlobalHeaderDBA@@I@Z 315e9180 f   AnimationManager.obj
 0001:000e81c0       ?SaveAnimEventToXml@CAnimationManager@@UAE_NABVCAnimEventData@@AAVXmlNodeRef@@@Z 315e91c0 f   AnimationManager.obj
 0001:000e82a0       ?Unload_All_Animation@CAnimationManager@@QAE_NXZ 315e92a0 f   AnimationManager.obj
 0001:000e8320       ?DBA_Unload_All@CAnimationManager@@QAE_NXZ 315e9320 f   AnimationManager.obj
 0001:000e8400       ?IsDatabaseInMemory@CAnimationManager@@QAE_NI@Z 315e9400 f   AnimationManager.obj
 0001:000e8450       ?assign@?$Array@V?$_smart_ptr@VIController@@@@HU?$SmallDynStorage@V?$_smart_ptr@VIController@@@@HUStandardAlloc@NAlloc@@@NArray@@@@QAEXU?$Array@$$CBV?$_smart_ptr@VIController@@@@HU?$ArrayStorage@$$CBV?$_smart_ptr@VIController@@@@H@NArray@@@@@Z 315e9450 f i AnimationManager.obj
 0001:000e8450       ?assign@?$Array@V?$_smart_ptr@UCMorphTarget@@@@HU?$SmallDynStorage@V?$_smart_ptr@UCMorphTarget@@@@HUStandardAlloc@NAlloc@@@NArray@@@@QAEXU?$Array@$$CBV?$_smart_ptr@UCMorphTarget@@@@HU?$ArrayStorage@$$CBV?$_smart_ptr@UCMorphTarget@@@@H@NArray@@@@@Z 315e9450 f i LoaderSKIN.obj
 0001:000e84a0       ?GetGlobalIDbyFilePath_AIM@CAnimationManager@@QBEHPBD@Z 315e94a0 f   AnimationManager.obj
 0001:000e8500       ?GetGlobalIDbyFilePath_LMG@CAnimationManager@@QBEHPBD@Z 315e9500 f   AnimationManager.obj
 0001:000e8560       ??4?$CryStringT@D@@QAEAAV0@ABV0@@Z 315e9560 f i AnimEventList.obj
 0001:000e8560       ??4XmlString@@QAEAAV0@ABV0@@Z 315e9560 f i AnimationManager.obj
 0001:000e85c0       ?DBA_LockStatus@CAnimationManager@@QAE_NPBDI_N@Z 315e95c0 f   AnimationManager.obj
 0001:000e8720       ?DBA_Unload@CAnimationManager@@QAE_NPBD@Z 315e9720 f   AnimationManager.obj
 0001:000e8920       ?ReloadCAF@CAnimationManager@@QAEHPBD@Z 315e9920 f   AnimationManager.obj
 0001:000e8bd0       ?ReloadLMG@CAnimationManager@@QAEHPBD@Z 315e9bd0 f   AnimationManager.obj
 0001:000e8cc0       ?GetDBACRC32fromFilePath@CAnimationManager@@QAEIPBD@Z 315e9cc0 f   AnimationManager.obj
 0001:000e8d10       ?get_alloc_size@?$SmallDynStorage@UGlobalAnimationHeaderAIM@@HUStandardAlloc@NAlloc@@@NArray@@QBEHXZ 315e9d10 f i AnimationManager.obj
 0001:000e8d60       ?get_alloc_size@?$SmallDynStorage@UGlobalAnimationHeaderLMG@@HUStandardAlloc@NAlloc@@@NArray@@QBEHXZ 315e9d60 f i AnimationManager.obj
 0001:000e8db0       ?erase@?$DynArray@V?$_smart_ptr@UCMorphTarget@@@@HU?$SmallDynStorage@V?$_smart_ptr@UCMorphTarget@@@@HUStandardAlloc@NAlloc@@@NArray@@@@QAEPAV?$_smart_ptr@UCMorphTarget@@@@PAV2@0@Z 315e9db0 f i LoaderSKIN.obj
 0001:000e8db0       ?erase@?$DynArray@V?$_smart_ptr@VIController@@@@HU?$SmallDynStorage@V?$_smart_ptr@VIController@@@@HUStandardAlloc@NAlloc@@@NArray@@@@QAEPAV?$_smart_ptr@VIController@@@@PAV2@0@Z 315e9db0 f i AnimationManager.obj
 0001:000e8e60       ?init@?$DynArray@UCGlobalHeaderDBA@@HU?$SmallDynStorage@UCGlobalHeaderDBA@@HUStandardAlloc@NAlloc@@@NArray@@@@KAPAUCGlobalHeaderDBA@@U?$Array@UCGlobalHeaderDBA@@HU?$ArrayStorage@UCGlobalHeaderDBA@@H@NArray@@@@ABU2@@Z 315e9e60 f i AnimationManager.obj
 0001:000e8f10       ?set_size@?$SmallDynStorage@UGlobalAnimationHeaderLMG@@HUStandardAlloc@NAlloc@@@NArray@@QAEXH@Z 315e9f10 f i AnimationManager.obj
 0001:000e8fa0       ??$AddObject@UGlobalAnimationHeaderCAF@@HU?$SmallDynStorage@UGlobalAnimationHeaderCAF@@HUStandardAlloc@NAlloc@@@NArray@@@ICrySizer@@QAEXABU?$DynArray@UGlobalAnimationHeaderCAF@@HU?$SmallDynStorage@UGlobalAnimationHeaderCAF@@HUStandardAlloc@NAlloc@@@NArray@@@@@Z 315e9fa0 f i AnimationManager.obj
 0001:000e90b0       ?SetFilePath@GlobalAnimationHeaderLMG@@QAEXABV?$CryStringT@D@@@Z 315ea0b0 f i AnimationManager.obj
 0001:000e9120       ??$AddObject@IIU?$less@I@stlpmtx_std@@V?$allocator@U?$pair@$$CBII@stlpmtx_std@@@2@@ICrySizer@@QAEXABV?$map@IIU?$less@I@stlpmtx_std@@V?$allocator@U?$pair@$$CBII@stlpmtx_std@@@2@@stlpmtx_std@@@Z 315ea120 f i AnimationManager.obj
 0001:000e9190       ??$AddObject@UBSParameter@@HU?$SmallDynStorage@UBSParameter@@HUStandardAlloc@NAlloc@@@NArray@@@ICrySizer@@QAEXABU?$DynArray@UBSParameter@@HU?$SmallDynStorage@UBSParameter@@HUStandardAlloc@NAlloc@@@NArray@@@@@Z 315ea190 f i AnimationManager.obj
 0001:000e92c0       ??$AddObject@UBoneIndices8@@HU?$SmallDynStorage@UBoneIndices8@@HUStandardAlloc@NAlloc@@@NArray@@@ICrySizer@@QAEXABU?$DynArray@UBoneIndices8@@HU?$SmallDynStorage@UBoneIndices8@@HUStandardAlloc@NAlloc@@@NArray@@@@@Z 315ea2c0 f i ModelMesh.obj
 0001:000e92c0       ??$AddObject@UIdxAndName@@HU?$SmallDynStorage@UIdxAndName@@HUStandardAlloc@NAlloc@@@NArray@@@ICrySizer@@QAEXABU?$DynArray@UIdxAndName@@HU?$SmallDynStorage@UIdxAndName@@HUStandardAlloc@NAlloc@@@NArray@@@@@Z 315ea2c0 f i ModelSkeleton.obj
 0001:000e92c0       ??$AddObject@USJointsAimIK_Pos@@HU?$SmallDynStorage@USJointsAimIK_Pos@@HUStandardAlloc@NAlloc@@@NArray@@@ICrySizer@@QAEXABU?$DynArray@USJointsAimIK_Pos@@HU?$SmallDynStorage@USJointsAimIK_Pos@@HUStandardAlloc@NAlloc@@@NArray@@@@@Z 315ea2c0 f i ModelSkeleton.obj
 0001:000e92c0       ??$AddObject@USCRCName@@HU?$SmallDynStorage@USCRCName@@HUStandardAlloc@NAlloc@@@NArray@@@ICrySizer@@QAEXABU?$DynArray@USCRCName@@HU?$SmallDynStorage@USCRCName@@HUStandardAlloc@NAlloc@@@NArray@@@@@Z 315ea2c0 f i AnimationManager.obj
 0001:000e9390       ??$AddObject@V?$_smart_ptr@VIController@@@@HU?$SmallDynStorage@V?$_smart_ptr@VIController@@@@HUStandardAlloc@NAlloc@@@NArray@@@ICrySizer@@QAEXABU?$DynArray@V?$_smart_ptr@VIController@@@@HU?$SmallDynStorage@V?$_smart_ptr@VIController@@@@HUStandardAlloc@NAlloc@@@NArray@@@@@Z 315ea390 f i AnimationManager.obj
 0001:000e94a0       ?GetSubFoldersVector@AnimSearchHelper@@QAEPAV?$vector@IV?$allocator@I@stlpmtx_std@@@stlpmtx_std@@I@Z 315ea4a0 f   AnimationManager.obj
 0001:000e94f0       ?GetAnimationsVector@AnimSearchHelper@@QAEPAV?$vector@HV?$allocator@H@stlpmtx_std@@@stlpmtx_std@@I@Z 315ea4f0 f   AnimationManager.obj
 0001:000e9530       ??4?$DynArray@V?$_smart_ptr@VIController@@@@HU?$SmallDynStorage@V?$_smart_ptr@VIController@@@@HUStandardAlloc@NAlloc@@@NArray@@@@QAEAAU0@U?$Array@$$CBV?$_smart_ptr@VIController@@@@HU?$ArrayStorage@$$CBV?$_smart_ptr@VIController@@@@H@NArray@@@@@Z 315ea530 f i AnimationManager.obj
 0001:000e95f0       ?erase@?$DynArray@UCControllerType@@HU?$SmallDynStorage@UCControllerType@@HUStandardAlloc@NAlloc@@@NArray@@@@QAEPAUCControllerType@@PAU2@0@Z 315ea5f0 f i LoaderCGA.obj
 0001:000e95f0       ?erase@?$DynArray@IHU?$SmallDynStorage@IHUStandardAlloc@NAlloc@@@NArray@@@@QAEPAIPAI0@Z 315ea5f0 f i AnimationManager.obj
 0001:000e9640       ??$AddObject@UCGlobalHeaderDBA@@HU?$SmallDynStorage@UCGlobalHeaderDBA@@HUStandardAlloc@NAlloc@@@NArray@@@ICrySizer@@QAEXABU?$DynArray@UCGlobalHeaderDBA@@HU?$SmallDynStorage@UCGlobalHeaderDBA@@HUStandardAlloc@NAlloc@@@NArray@@@@@Z 315ea640 f i AnimationManager.obj
 0001:000e9750       ?SetName@CAnimEventData@@QAEXPBD@Z 315ea750 f i AnimationManager.obj
 0001:000e97b0       ?GetValue@CNameCRCMap@@QBEIPBD@Z 315ea7b0 f i AnimationManager.obj
 0001:000e9890       ?SizeOfAIM@GlobalAnimationHeaderAIM@@QBEIXZ 315ea890 f i AnimationManager.obj
 0001:000e9a40       ?GetGlobalIDbyFilePath_CAF@CAnimationManager@@QBEHPBD@Z 315eaa40 f   AnimationManager.obj
 0001:000e9a70       ?GetAnimEventList@CAnimationManager@@UBEPBUIAnimEventList@@PBD@Z 315eaa70 f   AnimationManager.obj
 0001:000e9ad0       ?LoadAnimEventFromXml@CAnimationManager@@UAE_NABVXmlNodeRef@@AAVCAnimEventData@@@Z 315eaad0 f   AnimationManager.obj
 0001:000e9f40       ?InitializeSegmentationDataFromAnimEvents@CAnimationManager@@UAEXPBD@Z 315eaf40 f   AnimationManager.obj
 0001:000ea090       ?UnloadAnimationCAF@CAnimationManager@@QAEXAAUGlobalAnimationHeaderCAF@@@Z 315eb090 f   AnimationManager.obj
 0001:000ea100       ?DebugAnimUsage@CAnimationManager@@QAEXI@Z 315eb100 f   AnimationManager.obj
 0001:000eae50       ??4?$DynArray@IHU?$SmallDynStorage@IHUStandardAlloc@NAlloc@@@NArray@@@@QAEAAU0@U?$Array@$$CBIHU?$ArrayStorage@$$CBIH@NArray@@@@@Z 315ebe50 f i AnimationManager.obj
 0001:000eaf10       ?insert_unique@?$_Rb_tree@IU?$less@I@stlpmtx_std@@U?$pair@$$CBII@2@U?$_Select1st@U?$pair@$$CBII@stlpmtx_std@@@priv@2@U?$_MapTraitsT@U?$pair@$$CBII@stlpmtx_std@@@52@V?$allocator@U?$pair@$$CBII@stlpmtx_std@@@2@@priv@stlpmtx_std@@QAE?AU?$_Rb_tree_iterator@U?$pair@$$CBII@stlpmtx_std@@U?$_MapTraitsT@U?$pair@$$CBII@stlpmtx_std@@@priv@2@@23@U423@ABU?$pair@$$CBII@3@@Z 315ebf10 f i CharacterManager.obj
 0001:000eaf10       ?insert_unique@?$_Rb_tree@IU?$less@I@stlpmtx_std@@U?$pair@$$CBIPAV?$vector@HV?$allocator@H@stlpmtx_std@@@stlpmtx_std@@@2@U?$_Select1st@U?$pair@$$CBIPAV?$vector@HV?$allocator@H@stlpmtx_std@@@stlpmtx_std@@@stlpmtx_std@@@priv@2@U?$_MapTraitsT@U?$pair@$$CBIPAV?$vector@HV?$allocator@H@stlpmtx_std@@@stlpmtx_std@@@stlpmtx_std@@@52@V?$allocator@U?$pair@$$CBIPAV?$vector@HV?$allocator@H@stlpmtx_std@@@stlpmtx_std@@@stlpmtx_std@@@2@@priv@stlpmtx_std@@QAE?AU?$_Rb_tree_iterator@U?$pair@$$CBIPAV?$vector@HV?$allocator@H@stlpmtx_std@@@stlpmtx_std@@@stlpmtx_std@@U?$_MapTraitsT@U?$pair@$$CBIPAV?$vector@HV?$allocator@H@stlpmtx_std@@@stlpmtx_std@@@stlpmtx_std@@@priv@2@@23@U423@ABU?$pair@$$CBIPAV?$vector@HV?$allocator@H@stlpmtx_std@@@stlpmtx_std@@@3@@Z 315ebf10 f i AnimationManager.obj
 0001:000eaf10       ?insert_unique@?$_Rb_tree@IU?$less@I@stlpmtx_std@@U?$pair@$$CBIPAV?$vector@IV?$allocator@I@stlpmtx_std@@@stlpmtx_std@@@2@U?$_Select1st@U?$pair@$$CBIPAV?$vector@IV?$allocator@I@stlpmtx_std@@@stlpmtx_std@@@stlpmtx_std@@@priv@2@U?$_MapTraitsT@U?$pair@$$CBIPAV?$vector@IV?$allocator@I@stlpmtx_std@@@stlpmtx_std@@@stlpmtx_std@@@52@V?$allocator@U?$pair@$$CBIPAV?$vector@IV?$allocator@I@stlpmtx_std@@@stlpmtx_std@@@stlpmtx_std@@@2@@priv@stlpmtx_std@@QAE?AU?$_Rb_tree_iterator@U?$pair@$$CBIPAV?$vector@IV?$allocator@I@stlpmtx_std@@@stlpmtx_std@@@stlpmtx_std@@U?$_MapTraitsT@U?$pair@$$CBIPAV?$vector@IV?$allocator@I@stlpmtx_std@@@stlpmtx_std@@@stlpmtx_std@@@priv@2@@23@U423@ABU?$pair@$$CBIPAV?$vector@IV?$allocator@I@stlpmtx_std@@@stlpmtx_std@@@3@@Z 315ebf10 f i AnimationManager.obj
 0001:000eb100       ??$AddObject@UAimIKPose@@HU?$SmallDynStorage@UAimIKPose@@HUStandardAlloc@NAlloc@@@NArray@@@ICrySizer@@QAEXABU?$DynArray@UAimIKPose@@HU?$SmallDynStorage@UAimIKPose@@HUStandardAlloc@NAlloc@@@NArray@@@@@Z 315ec100 f i AnimationManager.obj
 0001:000eb270       ?AnimationReleaseAIM@CAnimationManager@@QAEXAAUGlobalAnimationHeaderAIM@@@Z 315ec270 f   AnimationManager.obj
 0001:000eb290       ?Clear@AnimSearchHelper@@QAEXXZ 315ec290 f   AnimationManager.obj
 0001:000eb4f0       ??$AddObject@UGlobalAnimationHeaderLMG@@HU?$SmallDynStorage@UGlobalAnimationHeaderLMG@@HUStandardAlloc@NAlloc@@@NArray@@@ICrySizer@@QAEXABU?$DynArray@UGlobalAnimationHeaderLMG@@HU?$SmallDynStorage@UGlobalAnimationHeaderLMG@@HUStandardAlloc@NAlloc@@@NArray@@@@@Z 315ec4f0 f i AnimationManager.obj
 0001:000eb5c0       ?GetMemoryUsage@GlobalAnimationHeaderAIM@@QBEXPAVICrySizer@@@Z 315ec5c0 f i AnimationManager.obj
 0001:000eb630       ??4?$DynArray@VCAnimEventData@@HU?$SmallDynStorage@VCAnimEventData@@HUStandardAlloc@NAlloc@@@NArray@@@@QAEAAU0@U?$Array@$$CBVCAnimEventData@@HU?$ArrayStorage@$$CBVCAnimEventData@@H@NArray@@@@@Z 315ec630 f i AnimationManager.obj
 0001:000eb710       ??$?AI@?$map@IIU?$less@I@stlpmtx_std@@V?$allocator@U?$pair@$$CBII@stlpmtx_std@@@2@@stlpmtx_std@@QAEAAIABI@Z 315ec710 f i CharacterManager.obj
 0001:000eb710       ??$?AI@?$map@IPAV?$vector@IV?$allocator@I@stlpmtx_std@@@stlpmtx_std@@U?$less@I@2@V?$allocator@U?$pair@$$CBIPAV?$vector@IV?$allocator@I@stlpmtx_std@@@stlpmtx_std@@@stlpmtx_std@@@2@@stlpmtx_std@@QAEAAPAV?$vector@IV?$allocator@I@stlpmtx_std@@@1@ABI@Z 315ec710 f i AnimationManager.obj
 0001:000eb710       ??$?AI@?$map@IPAV?$vector@HV?$allocator@H@stlpmtx_std@@@stlpmtx_std@@U?$less@I@2@V?$allocator@U?$pair@$$CBIPAV?$vector@HV?$allocator@H@stlpmtx_std@@@stlpmtx_std@@@stlpmtx_std@@@2@@stlpmtx_std@@QAEAAPAV?$vector@HV?$allocator@H@stlpmtx_std@@@1@ABI@Z 315ec710 f i AnimationManager.obj
 0001:000eb790       ?AddAnimation@AnimSearchHelper@@QAE_NII@Z 315ec790 f   AnimationManager.obj
 0001:000eb870       ?AddAnimation@AnimSearchHelper@@QAEXABV?$CryStringT@D@@I@Z 315ec870 f   AnimationManager.obj
 0001:000ebb70       ??$AddObject@UGlobalAnimationHeaderAIM@@HU?$SmallDynStorage@UGlobalAnimationHeaderAIM@@HUStandardAlloc@NAlloc@@@NArray@@@ICrySizer@@QAEXABU?$DynArray@UGlobalAnimationHeaderAIM@@HU?$SmallDynStorage@UGlobalAnimationHeaderAIM@@HUStandardAlloc@NAlloc@@@NArray@@@@@Z 315ecb70 f i AnimationManager.obj
 0001:000ebc00       ??0GlobalAnimationHeaderLMG@@QAE@XZ 315ecc00 f i AnimationManager.obj
 0001:000ebf80       ?GetMemoryUsage@CAnimationManager@@QBEXPAVICrySizer@@@Z 315ecf80 f   AnimationManager.obj
 0001:000ebfe0       ??4GlobalAnimationHeaderCAF@@QAEAAU0@ABU0@@Z 315ecfe0 f i AnimationManager.obj
 0001:000ec120       ?CreateGlobalHeaderDBA@CAnimationManager@@QAE_NAAU?$DynArray@V?$CryStringT@D@@HU?$SmallDynStorage@V?$CryStringT@D@@HUStandardAlloc@NAlloc@@@NArray@@@@@Z 315ed120 f   AnimationManager.obj
 0001:000ec250       ?DBA_PreLoad@CAnimationManager@@QAE_NPBD_N@Z 315ed250 f   AnimationManager.obj
 0001:000ec470       ??4CControllerTCB@@QAEAAU0@ABU0@@Z 315ed470 f i AnimationManager.obj
 0001:000ec540       ?LoadAnimationTCB@CAnimationManager@@QAE_NHAAU?$DynArray@UCControllerTCB@@HU?$SmallDynStorage@UCControllerTCB@@HUStandardAlloc@NAlloc@@@NArray@@@@PAVCryCGALoader@@PBVCSkel@@@Z 315ed540 f   AnimationManager.obj
 0001:000eca80       ?init@?$DynArray@UGlobalAnimationHeaderAIM@@HU?$SmallDynStorage@UGlobalAnimationHeaderAIM@@HUStandardAlloc@NAlloc@@@NArray@@@@KAPAUGlobalAnimationHeaderAIM@@U?$Array@UGlobalAnimationHeaderAIM@@HU?$ArrayStorage@UGlobalAnimationHeaderAIM@@H@NArray@@@@ABU2@@Z 315eda80 f i AnimationManager.obj
 0001:000ecdd0       ?expand_raw@?$DynArray@UGlobalAnimationHeaderLMG@@HU?$SmallDynStorage@UGlobalAnimationHeaderLMG@@HUStandardAlloc@NAlloc@@@NArray@@@@IAEPAUGlobalAnimationHeaderLMG@@PAU2@H@Z 315eddd0 f i AnimationManager.obj
 0001:000ece60       ?CreateGAH_CAF@CAnimationManager@@QAEHABV?$CryStringT@D@@@Z 315ede60 f   AnimationManager.obj
 0001:000ecf30       ?CreateGAH_LMG@CAnimationManager@@QAEHABV?$CryStringT@D@@@Z 315edf30 f   AnimationManager.obj
 0001:000ecfe0       ?CreateGAH_AIM@CAnimationManager@@QAEHABV?$CryStringT@D@@@Z 315edfe0 f   AnimationManager.obj
 0001:000ed070       ?GetPositionsFormatSizeOf@ControllerHelper@@YAII@Z 315ee070 f   ControllerPQ.obj
 0001:000ed090       ?GetRotationFormatSizeOf@ControllerHelper@@YAII@Z 315ee090 f   ControllerPQ.obj
 0001:000ed0e0       ?GetKeyTimesFormatSizeOf@ControllerHelper@@YAII@Z 315ee0e0 f   ControllerPQ.obj
 0001:000ed130       ?GetOP@CController@@UBEEMAAU?$Quat_tpl@M@@AAU?$Vec3_tpl@M@@@Z 315ee130 f   ControllerPQ.obj
 0001:000ed170       ?GetO@CController@@UBEEMAAU?$Quat_tpl@M@@@Z 315ee170 f   ControllerPQ.obj
 0001:000ed1a0       ?GetP@CController@@UBEEMAAU?$Vec3_tpl@M@@@Z 315ee1a0 f   ControllerPQ.obj
 0001:000ed1d0       ?ToExternalType@SmallTree48BitQuat@@QBEXAAU?$Quat_tpl@M@@@Z 315ee1d0 f i ControllerPQ.obj
 0001:000ed4b0       ?ToExternalType@SmallTree64BitQuat@@QBEXAAU?$Quat_tpl@M@@@Z 315ee4b0 f i ControllerPQ.obj
 0001:000ed5e0       ?ToExternalType@SmallTree64BitExtQuat@@QBEXAAU?$Quat_tpl@M@@@Z 315ee5e0 f i ControllerPQ.obj
 0001:000ed790       ?AssignData@?$CTrackDataStorageInt@U?$Vec3_tpl@M@@UNoCompressVec3@@VITrackPositionStorage@@@@UAEIPBDI@Z 315ee790 f i ControllerPQ.obj
 0001:000ed850       ?GetDataRawSize@?$CTrackDataStorageInt@U?$Vec3_tpl@M@@UNoCompressVec3@@VITrackPositionStorage@@@@UAEIXZ 315ee850 f i ControllerPQ.obj
 0001:000ed860       ?GetValue@?$CTrackDataStorageInt@U?$Vec3_tpl@M@@UNoCompressVec3@@VITrackPositionStorage@@@@UAEXIAAU?$Vec3_tpl@M@@@Z 315ee860 f i ControllerPQ.obj
 0001:000ed8b0       ?SizeOfPosController@?$CTrackDataStorageInt@U?$Vec3_tpl@M@@UNoCompressVec3@@VITrackPositionStorage@@@@UAEIXZ 315ee8b0 f i ControllerPQ.obj
 0001:000ed8b0       ?SizeOfRotController@?$CTrackDataStorageInt@U?$Vec3_tpl@M@@UNoCompressVec3@@VITrackPositionStorage@@@@UAEIXZ 315ee8b0 f i ControllerPQ.obj
 0001:000ed8d0       ?AssignData@?$CTrackDataStorageInt@U?$Quat_tpl@M@@UNoCompressQuat@@VITrackRotationStorage@@@@UAEIPBDI@Z 315ee8d0 f i ControllerPQ.obj
 0001:000ed980       ?GetDataRawSize@?$CTrackDataStorageInt@U?$Quat_tpl@M@@UNoCompressQuat@@VITrackRotationStorage@@@@UAEIXZ 315ee980 f i ControllerPQ.obj
 0001:000ed990       ?GetValue@?$CTrackDataStorageInt@U?$Quat_tpl@M@@UNoCompressQuat@@VITrackRotationStorage@@@@UAEXIAAU?$Quat_tpl@M@@@Z 315ee990 f i ControllerPQ.obj
 0001:000ed9f0       ?SizeOfRotController@?$CTrackDataStorageInt@U?$Quat_tpl@M@@UNoCompressQuat@@VITrackRotationStorage@@@@UAEIXZ 315ee9f0 f i ControllerPQ.obj
 0001:000ed9f0       ?SizeOfPosController@?$CTrackDataStorageInt@U?$Quat_tpl@M@@UNoCompressQuat@@VITrackRotationStorage@@@@UAEIXZ 315ee9f0 f i ControllerPQ.obj
 0001:000eda00       ?AssignData@?$CTrackDataStorageInt@U?$Quat_tpl@M@@USmallTree48BitQuat@@VITrackRotationStorage@@@@UAEIPBDI@Z 315eea00 f i ControllerPQ.obj
 0001:000edab0       ?GetDataRawSize@?$CTrackDataStorageInt@U?$Quat_tpl@M@@USmallTree48BitQuat@@VITrackRotationStorage@@@@UAEIXZ 315eeab0 f i ControllerPQ.obj
 0001:000edac0       ?GetValue@?$CTrackDataStorageInt@U?$Quat_tpl@M@@USmallTree48BitQuat@@VITrackRotationStorage@@@@UAEXIAAU?$Quat_tpl@M@@@Z 315eeac0 f i ControllerPQ.obj
 0001:000edb00       ?GetFormat@?$CKeyTimesInformationStartStop@EUByteStartStopEncoder@@@@UAEIXZ 315eeb00 f i ControllerPQ.obj
 0001:000edb00       ?GetType@CFacialEffectorAttachment@@UAE?AW4EFacialEffectorType@@XZ 315eeb00 f i FaceEffector.obj
 0001:000edb00       ?GetFormat@?$CTrackDataStorageInt@U?$Quat_tpl@M@@USmallTree48BitQuat@@VITrackRotationStorage@@@@UAEIXZ 315eeb00 f i ControllerPQ.obj
 0001:000edb10       ?SizeOfRotController@?$CTrackDataStorageInt@U?$Quat_tpl@M@@USmallTree48BitQuat@@VITrackRotationStorage@@@@UAEIXZ 315eeb10 f i ControllerPQ.obj
 0001:000edb10       ?SizeOfPosController@?$CTrackDataStorageInt@U?$Quat_tpl@M@@USmallTree48BitQuat@@VITrackRotationStorage@@@@UAEIXZ 315eeb10 f i ControllerPQ.obj
 0001:000edb20       ?AssignData@?$CTrackDataStorageInt@U?$Quat_tpl@M@@USmallTree64BitExtQuat@@VITrackRotationStorage@@@@UAEIPBDI@Z 315eeb20 f i ControllerPQ.obj
 0001:000edb20       ?AssignData@?$CTrackDataStorageInt@U?$Quat_tpl@M@@USmallTree64BitQuat@@VITrackRotationStorage@@@@UAEIPBDI@Z 315eeb20 f i ControllerPQ.obj
 0001:000edbe0       ?GetValue@?$CTrackDataStorageInt@U?$Quat_tpl@M@@USmallTree64BitQuat@@VITrackRotationStorage@@@@UAEXIAAU?$Quat_tpl@M@@@Z 315eebe0 f i ControllerPQ.obj
 0001:000edc10       ?GetData@CKeyTimesInformationBitSet@@UAEPADXZ 315eec10 f i ControllerPQ.obj
 0001:000edc10       ?GetReplacementMaterial@CSKELAttachment@@UBEPAUIMaterial@@XZ 315eec10 f i AttachmentManager.obj
 0001:000edc10       ?GetReplacementMaterial@CCGFAttachment@@UBEPAUIMaterial@@XZ 315eec10 f i AttachmentManager.obj
 0001:000edc10       ?GetData@?$CTrackDataStorageInt@U?$Quat_tpl@M@@USmallTree64BitQuat@@VITrackRotationStorage@@@@UAEPADXZ 315eec10 f i ControllerPQ.obj
 0001:000edc10       ?GetSkelInstance@CAttachmentManager@@UBEPAUICharacterInstance@@XZ 315eec10 f i AttachmentManager.obj
 0001:000edc10       ?GetName@CAttachmentFACE@@UBEPBDXZ 315eec10 f i AttachmentManager.obj
 0001:000edc10       ?GetReplacementMaterial@CSKINAttachment@@UBEPAUIMaterial@@XZ 315eec10 f i AttachmentManager.obj
 0001:000edc10       ?GetICharacterModel@CCharInstance@@UAEPAUICharacterModel@@XZ 315eec10 f i CharacterInstance.obj
 0001:000edc10       ?GetName@CAttachmentBONE@@UBEPBDXZ 315eec10 f i AttachmentManager.obj
 0001:000edc10       ?GetName@CAttachmentSKIN@@UBEPBDXZ 315eec10 f i Attachment.obj
 0001:000edc10       ?GetName@CFacialEffectorsLibrary@@UAEPBDXZ 315eec10 f i FaceEffectorLibrary.obj
 0001:000edc10       ?GetData@?$CTrackDataStorageInt@U?$Quat_tpl@M@@USmallTree64BitExtQuat@@VITrackRotationStorage@@@@UAEPADXZ 315eec10 f i ControllerPQ.obj
 0001:000edc10       ?GetData@?$CTrackDataStorageInt@U?$Vec3_tpl@M@@UNoCompressVec3@@VITrackPositionStorage@@@@UAEPADXZ 315eec10 f i ControllerPQ.obj
 0001:000edc10       ?GetData@?$CTrackDataStorageInt@U?$Quat_tpl@M@@USmallTree48BitQuat@@VITrackRotationStorage@@@@UAEPADXZ 315eec10 f i ControllerPQ.obj
 0001:000edc10       ?GetData@?$CTrackDataStorageInt@U?$Quat_tpl@M@@UNoCompressQuat@@VITrackRotationStorage@@@@UAEPADXZ 315eec10 f i ControllerPQ.obj
 0001:000edc10       ?GetSoundFile@CFacialAnimSoundEntry@@UAEPBDXZ 315eec10 f i FaceAnimSequence.obj
 0001:000edc10       ?GetJointCount@CPoseData@Skeleton@@UBEIXZ 315eec10 f i Skeleton.obj
 0001:000edc20       ?GetDataRawSize@?$CTrackDataStorageInt@U?$Quat_tpl@M@@USmallTree64BitQuat@@VITrackRotationStorage@@@@UAEIXZ 315eec20 f i ControllerPQ.obj
 0001:000edc20       ?GetDataRawSize@?$CTrackDataStorageInt@U?$Quat_tpl@M@@USmallTree64BitExtQuat@@VITrackRotationStorage@@@@UAEIXZ 315eec20 f i ControllerPQ.obj
 0001:000edc30       ?GetValue@?$CTrackDataStorageInt@U?$Quat_tpl@M@@USmallTree64BitExtQuat@@VITrackRotationStorage@@@@UAEXIAAU?$Quat_tpl@M@@@Z 315eec30 f i ControllerPQ.obj
 0001:000edc60       ?GetDataRawSize@?$CKeyTimesInformationStartStop@MUF32StartStopEncoder@@@@UAEIXZ 315eec60 f i ControllerPQ.obj
 0001:000edc60       ?GetFormat@?$CTrackDataStorageInt@U?$Quat_tpl@M@@USmallTree64BitExtQuat@@VITrackRotationStorage@@@@UAEIXZ 315eec60 f i ControllerPQ.obj
 0001:000edc70       ?SizeOfPosController@?$CTrackDataStorageInt@U?$Quat_tpl@M@@USmallTree64BitExtQuat@@VITrackRotationStorage@@@@UAEIXZ 315eec70 f i ControllerPQ.obj
 0001:000edc70       ?SizeOfPosController@?$CTrackDataStorageInt@U?$Quat_tpl@M@@USmallTree64BitQuat@@VITrackRotationStorage@@@@UAEIXZ 315eec70 f i ControllerPQ.obj
 0001:000edc70       ?SizeOfRotController@?$CTrackDataStorageInt@U?$Quat_tpl@M@@USmallTree64BitExtQuat@@VITrackRotationStorage@@@@UAEIXZ 315eec70 f i ControllerPQ.obj
 0001:000edc70       ?SizeOfRotController@?$CTrackDataStorageInt@U?$Quat_tpl@M@@USmallTree64BitQuat@@VITrackRotationStorage@@@@UAEIXZ 315eec70 f i ControllerPQ.obj
 0001:000edc80       ?GetKey@?$CKeyTimesInformation@MUF32Encoder@@@@UAEIMAAM@Z 315eec80 f i ControllerPQ.obj
 0001:000edd40       ?GetKey@?$CKeyTimesInformation@GUUINT16Encoder@@@@UAEIMAAM@Z 315eed40 f i ControllerPQ.obj
 0001:000ede50       ?GetNumKeys@?$CKeyTimesInformation@MUF32Encoder@@@@UBEIXZ 315eee50 f i ControllerPQ.obj
 0001:000ede50       ?GetNumKeys@?$CKeyTimesInformation@GUUINT16Encoder@@@@UBEIXZ 315eee50 f i ControllerPQ.obj
 0001:000ede50       ?GetNumKeys@?$CKeyTimesInformation@EUByteEncoder@@@@UBEIXZ 315eee50 f i ControllerPQ.obj
 0001:000ede50       ?GetDataRawSize@?$CKeyTimesInformation@EUByteEncoder@@@@UAEIXZ 315eee50 f i ControllerPQ.obj
 0001:000ede60       ?GetKey@?$CKeyTimesInformation@EUByteEncoder@@@@UAEIMAAM@Z 315eee60 f i ControllerPQ.obj
 0001:000edf60       ??_E?$CTrackDataStorageInt@U?$Vec3_tpl@M@@UNoCompressVec3@@VITrackPositionStorage@@@@UAEPAXI@Z 315eef60 f i ControllerPQ.obj
 0001:000edf60       ??_E?$CTrackDataStorage@U?$Vec3_tpl@M@@UNoCompressVec3@@VITrackPositionStorage@@@@UAEPAXI@Z 315eef60 f i ControllerPQ.obj
 0001:000edf60       ??_G?$CTrackDataStorageInt@U?$Vec3_tpl@M@@UNoCompressVec3@@VITrackPositionStorage@@@@UAEPAXI@Z 315eef60 f i ControllerPQ.obj
 0001:000edf60       ??_G?$CTrackDataStorage@U?$Vec3_tpl@M@@UNoCompressVec3@@VITrackPositionStorage@@@@UAEPAXI@Z 315eef60 f i ControllerPQ.obj
 0001:000edfb0       ??_E?$CTrackDataStorageInt@U?$Quat_tpl@M@@UNoCompressQuat@@VITrackRotationStorage@@@@UAEPAXI@Z 315eefb0 f i ControllerPQ.obj
 0001:000edfb0       ??_E?$CTrackDataStorage@U?$Quat_tpl@M@@UNoCompressQuat@@VITrackRotationStorage@@@@UAEPAXI@Z 315eefb0 f i ControllerPQ.obj
 0001:000edfb0       ??_G?$CTrackDataStorage@U?$Quat_tpl@M@@UNoCompressQuat@@VITrackRotationStorage@@@@UAEPAXI@Z 315eefb0 f i ControllerPQ.obj
 0001:000edfb0       ??_G?$CTrackDataStorageInt@U?$Quat_tpl@M@@UNoCompressQuat@@VITrackRotationStorage@@@@UAEPAXI@Z 315eefb0 f i ControllerPQ.obj
 0001:000ee000       ??_G?$CTrackDataStorageInt@U?$Quat_tpl@M@@USmallTree48BitQuat@@VITrackRotationStorage@@@@UAEPAXI@Z 315ef000 f i ControllerPQ.obj
 0001:000ee000       ??_G?$CTrackDataStorage@U?$Quat_tpl@M@@USmallTree48BitQuat@@VITrackRotationStorage@@@@UAEPAXI@Z 315ef000 f i ControllerPQ.obj
 0001:000ee000       ??_E?$CTrackDataStorage@U?$Quat_tpl@M@@USmallTree48BitQuat@@VITrackRotationStorage@@@@UAEPAXI@Z 315ef000 f i ControllerPQ.obj
 0001:000ee000       ??_E?$CTrackDataStorageInt@U?$Quat_tpl@M@@USmallTree48BitQuat@@VITrackRotationStorage@@@@UAEPAXI@Z 315ef000 f i ControllerPQ.obj
 0001:000ee050       ??_E?$CTrackDataStorageInt@U?$Quat_tpl@M@@USmallTree64BitQuat@@VITrackRotationStorage@@@@UAEPAXI@Z 315ef050 f i ControllerPQ.obj
 0001:000ee050       ??_G?$CTrackDataStorageInt@U?$Quat_tpl@M@@USmallTree64BitQuat@@VITrackRotationStorage@@@@UAEPAXI@Z 315ef050 f i ControllerPQ.obj
 0001:000ee050       ??_G?$CTrackDataStorage@U?$Quat_tpl@M@@USmallTree64BitQuat@@VITrackRotationStorage@@@@UAEPAXI@Z 315ef050 f i ControllerPQ.obj
 0001:000ee050       ??_E?$CTrackDataStorage@U?$Quat_tpl@M@@USmallTree64BitQuat@@VITrackRotationStorage@@@@UAEPAXI@Z 315ef050 f i ControllerPQ.obj
 0001:000ee0a0       ??_E?$CTrackDataStorage@U?$Quat_tpl@M@@USmallTree64BitExtQuat@@VITrackRotationStorage@@@@UAEPAXI@Z 315ef0a0 f i ControllerPQ.obj
 0001:000ee0a0       ??_E?$CTrackDataStorageInt@U?$Quat_tpl@M@@USmallTree64BitExtQuat@@VITrackRotationStorage@@@@UAEPAXI@Z 315ef0a0 f i ControllerPQ.obj
 0001:000ee0a0       ??_G?$CTrackDataStorage@U?$Quat_tpl@M@@USmallTree64BitExtQuat@@VITrackRotationStorage@@@@UAEPAXI@Z 315ef0a0 f i ControllerPQ.obj
 0001:000ee0a0       ??_G?$CTrackDataStorageInt@U?$Quat_tpl@M@@USmallTree64BitExtQuat@@VITrackRotationStorage@@@@UAEPAXI@Z 315ef0a0 f i ControllerPQ.obj
 0001:000ee0f0       ?GetFormat@CKeyTimesInformationBitSet@@UAEIXZ 315ef0f0 f i ControllerPQ.obj
 0001:000ee0f0       ?GetFormat@?$CTrackDataStorageInt@U?$Quat_tpl@M@@USmallTree64BitQuat@@VITrackRotationStorage@@@@UAEIXZ 315ef0f0 f i ControllerPQ.obj
 0001:000ee100       ?GetDataRawSize@CKeyTimesInformationBitSet@@UAEIXZ 315ef100 f i ControllerPQ.obj
 0001:000ee110       ?GetKeyValueFloat@CKeyTimesInformationBitSet@@UBEMI@Z 315ef110 f i ControllerPQ.obj
 0001:000ee1c0       ?GetKey@CKeyTimesInformationBitSet@@UAEIMAAM@Z 315ef1c0 f i ControllerPQ.obj
 0001:000ee3e0       ?GetNumKeys@CKeyTimesInformationBitSet@@UBEIXZ 315ef3e0 f i ControllerPQ.obj
 0001:000ee3f0       ?AssignKeyTime@CKeyTimesInformationBitSet@@UAEIPBDI@Z 315ef3f0 f i ControllerPQ.obj
 0001:000ee450       ?GetMemoryUsage@CKeyTimesInformationBitSet@@UBEXPAVICrySizer@@@Z 315ef450 f i ControllerPQ.obj
 0001:000ee490       ?GetRotValueFromKey@CControllerOptNonVirtual@@QBEXIAAU?$Quat_tpl@M@@@Z 315ef490 f i ControllerPQ.obj
 0001:000ee530       ??_ECKeyTimesInformationBitSet@@UAEPAXI@Z 315ef530 f i ControllerPQ.obj
 0001:000ee5f0       ?GetValueFromKey@IRotationController@@UAEXIAAU?$Quat_tpl@M@@@Z 315ef5f0 f   ControllerPQ.obj
 0001:000ee5f0       ?GetValueFromKey@IPositionController@@UAEXIAAU?$Vec3_tpl@M@@@Z 315ef5f0 f   ControllerPQ.obj
 0001:000ee620       ?GetMemoryUsage@?$CTrackDataStorage@U?$Vec3_tpl@M@@UNoCompressVec3@@VITrackPositionStorage@@@@UBEXPAVICrySizer@@@Z 315ef620 f i ControllerPQ.obj
 0001:000ee620       ?GetMemoryUsage@?$CTrackDataStorage@U?$Quat_tpl@M@@USmallTree64BitExtQuat@@VITrackRotationStorage@@@@UBEXPAVICrySizer@@@Z 315ef620 f i ControllerPQ.obj
 0001:000ee620       ?GetMemoryUsage@?$CTrackDataStorage@U?$Quat_tpl@M@@USmallTree48BitQuat@@VITrackRotationStorage@@@@UBEXPAVICrySizer@@@Z 315ef620 f i ControllerPQ.obj
 0001:000ee620       ?GetMemoryUsage@?$CTrackDataStorage@U?$Quat_tpl@M@@USmallTree64BitQuat@@VITrackRotationStorage@@@@UBEXPAVICrySizer@@@Z 315ef620 f i ControllerPQ.obj
 0001:000ee620       ?GetMemoryUsage@?$CTrackDataStorage@U?$Quat_tpl@M@@UNoCompressQuat@@VITrackRotationStorage@@@@UBEXPAVICrySizer@@@Z 315ef620 f i ControllerPQ.obj
 0001:000ee640       ??0?$CTrackDataStorage@U?$Quat_tpl@M@@UNoCompressQuat@@VITrackRotationStorage@@@@QAE@PAUNoCompressQuat@@I@Z 315ef640 f i ControllerPQ.obj
 0001:000ee680       ?Release@?$CTrackDataStorage@U?$Quat_tpl@M@@USmallTree64BitExtQuat@@VITrackRotationStorage@@@@UAEXXZ 315ef680 f i ControllerPQ.obj
 0001:000ee680       ?Release@?$CTrackDataStorage@U?$Quat_tpl@M@@USmallTree64BitQuat@@VITrackRotationStorage@@@@UAEXXZ 315ef680 f i ControllerPQ.obj
 0001:000ee680       ?Release@?$CTrackDataStorage@U?$Vec3_tpl@M@@UNoCompressVec3@@VITrackPositionStorage@@@@UAEXXZ 315ef680 f i ControllerPQ.obj
 0001:000ee680       ?Release@?$CTrackDataStorage@U?$Quat_tpl@M@@USmallTree48BitQuat@@VITrackRotationStorage@@@@UAEXXZ 315ef680 f i ControllerPQ.obj
 0001:000ee680       ?Release@?$CTrackDataStorage@U?$Quat_tpl@M@@UNoCompressQuat@@VITrackRotationStorage@@@@UAEXXZ 315ef680 f i ControllerPQ.obj
 0001:000ee690       ??0?$CTrackDataStorage@U?$Quat_tpl@M@@USmallTree48BitQuat@@VITrackRotationStorage@@@@QAE@PAUSmallTree48BitQuat@@I@Z 315ef690 f i ControllerPQ.obj
 0001:000ee6d0       ??0?$CTrackDataStorage@U?$Quat_tpl@M@@USmallTree64BitQuat@@VITrackRotationStorage@@@@QAE@PAUSmallTree64BitQuat@@I@Z 315ef6d0 f i ControllerPQ.obj
 0001:000ee710       ??0?$CTrackDataStorage@U?$Quat_tpl@M@@USmallTree64BitExtQuat@@VITrackRotationStorage@@@@QAE@PAUSmallTree64BitExtQuat@@I@Z 315ef710 f i ControllerPQ.obj
 0001:000ee750       ?GetKeyValueFloat@?$CKeyTimesInformation@MUF32Encoder@@@@UBEMI@Z 315ef750 f i ControllerPQ.obj
 0001:000ee760       ?GetMemoryUsage@?$CKeyTimesInformation@EUByteEncoder@@@@UBEXPAVICrySizer@@@Z 315ef760 f i ControllerPQ.obj
 0001:000ee760       ?GetMemoryUsage@?$CKeyTimesInformation@GUUINT16Encoder@@@@UBEXPAVICrySizer@@@Z 315ef760 f i ControllerPQ.obj
 0001:000ee760       ?GetMemoryUsage@?$CKeyTimesInformation@MUF32Encoder@@@@UBEXPAVICrySizer@@@Z 315ef760 f i ControllerPQ.obj
 0001:000ee780       ?AssignKeyTime@?$CKeyTimesInformation@MUF32Encoder@@@@UAEIPBDI@Z 315ef780 f i ControllerPQ.obj
 0001:000ee840       ?GetDataRawSize@?$CKeyTimesInformation@MUF32Encoder@@@@UAEIXZ 315ef840 f i ControllerPQ.obj
 0001:000ee850       ??0?$CKeyTimesInformation@MUF32Encoder@@@@QAE@PAMI@Z 315ef850 f i ControllerPQ.obj
 0001:000ee8a0       ?GetKeyValueFloat@?$CKeyTimesInformation@GUUINT16Encoder@@@@UBEMI@Z 315ef8a0 f i ControllerPQ.obj
 0001:000ee8c0       ?GetRelocateChain@?$CKeyTimesInformation@GUUINT16Encoder@@@@UAEPAVIControllerRelocatableChain@@XZ 315ef8c0 f i ControllerPQ.obj
 0001:000ee8c0       ?GetRelocateChain@?$CKeyTimesInformation@EUByteEncoder@@@@UAEPAVIControllerRelocatableChain@@XZ 315ef8c0 f i ControllerPQ.obj
 0001:000ee8c0       ?GetRelocateChain@?$CKeyTimesInformation@MUF32Encoder@@@@UAEPAVIControllerRelocatableChain@@XZ 315ef8c0 f i ControllerPQ.obj
 0001:000ee8d0       ?AssignKeyTime@?$CKeyTimesInformation@GUUINT16Encoder@@@@UAEIPBDI@Z 315ef8d0 f i ControllerPQ.obj
 0001:000ee990       ?GetDataRawSize@?$CKeyTimesInformation@GUUINT16Encoder@@@@UAEIXZ 315ef990 f i ControllerPQ.obj
 0001:000ee9a0       ??0?$CKeyTimesInformation@GUUINT16Encoder@@@@QAE@PAGI@Z 315ef9a0 f i ControllerPQ.obj
 0001:000ee9f0       ?GetKeyValueFloat@?$CKeyTimesInformation@EUByteEncoder@@@@UBEMI@Z 315ef9f0 f i ControllerPQ.obj
 0001:000eea10       ?GetData@?$CKeyTimesInformation@MUF32Encoder@@@@UAEPADXZ 315efa10 f i ControllerPQ.obj
 0001:000eea10       ?GetData@?$CKeyTimesInformation@GUUINT16Encoder@@@@UAEPADXZ 315efa10 f i ControllerPQ.obj
 0001:000eea10       ?GetFlags@CFacialEffCtrl@@UAEHXZ 315efa10 f i FaceEffector.obj
 0001:000eea10       ?GetData@?$CKeyTimesInformation@EUByteEncoder@@@@UAEPADXZ 315efa10 f i ControllerPQ.obj
 0001:000eea20       ?Relocate@?$CKeyTimesInformation@EUByteEncoder@@@@UAEXPAD0@Z 315efa20 f i ControllerPQ.obj
 0001:000eea20       ?Relocate@?$CKeyTimesInformation@MUF32Encoder@@@@UAEXPAD0@Z 315efa20 f i ControllerPQ.obj
 0001:000eea20       ?Relocate@?$CTrackDataStorageInt@U?$Quat_tpl@M@@UNoCompressQuat@@VITrackRotationStorage@@@@UAEXPAD0@Z 315efa20 f i ControllerPQ.obj
 0001:000eea20       ?Relocate@?$CKeyTimesInformation@GUUINT16Encoder@@@@UAEXPAD0@Z 315efa20 f i ControllerPQ.obj
 0001:000eea20       ?Relocate@?$CTrackDataStorageInt@U?$Quat_tpl@M@@USmallTree64BitQuat@@VITrackRotationStorage@@@@UAEXPAD0@Z 315efa20 f i ControllerPQ.obj
 0001:000eea20       ?Relocate@?$CTrackDataStorageInt@U?$Vec3_tpl@M@@UNoCompressVec3@@VITrackPositionStorage@@@@UAEXPAD0@Z 315efa20 f i ControllerPQ.obj
 0001:000eea20       ?Relocate@?$CTrackDataStorageInt@U?$Quat_tpl@M@@USmallTree64BitExtQuat@@VITrackRotationStorage@@@@UAEXPAD0@Z 315efa20 f i ControllerPQ.obj
 0001:000eea20       ?Relocate@?$CTrackDataStorageInt@U?$Quat_tpl@M@@USmallTree48BitQuat@@VITrackRotationStorage@@@@UAEXPAD0@Z 315efa20 f i ControllerPQ.obj
 0001:000eea30       ?AssignKeyTime@?$CKeyTimesInformation@EUByteEncoder@@@@UAEIPBDI@Z 315efa30 f i ControllerPQ.obj
 0001:000eeaf0       ??0?$CKeyTimesInformation@EUByteEncoder@@@@QAE@PAEI@Z 315efaf0 f i ControllerPQ.obj
 0001:000eeb40       ?GetKeyValueFloat@?$CKeyTimesInformationStartStop@MUF32StartStopEncoder@@@@UBEMI@Z 315efb40 f i ControllerPQ.obj
 0001:000eeb60       ?GetKey@?$CKeyTimesInformationStartStop@MUF32StartStopEncoder@@@@UAEIMAAM@Z 315efb60 f i ControllerPQ.obj
 0001:000eec00       ?GetNumKeys@?$CKeyTimesInformationStartStop@MUF32StartStopEncoder@@@@UBEIXZ 315efc00 f i ControllerPQ.obj
 0001:000eec30       ?AssignKeyTime@?$CKeyTimesInformationStartStop@MUF32StartStopEncoder@@@@UAEIPBDI@Z 315efc30 f i ControllerPQ.obj
 0001:000eec50       ?GetNumDimensions@CFacialCameraPathPositionInterpolator@@UAEHXZ 315efc50 f i FaceAnimSequence.obj
 0001:000eec50       ?GetType@CFacialEffectorBone@@UAE?AW4EFacialEffectorType@@XZ 315efc50 f i FaceEffectorLibrary.obj
 0001:000eec50       ?GetAttachmentType@CSKINAttachment@@UAE?AW4EType@IAttachmentObject@@XZ 315efc50 f i AttachmentManager.obj
 0001:000eec50       ?GetSplineType@CFacialCameraPathPositionInterpolator@@UAE?AW4ESplineType@@XZ 315efc50 f i FaceAnimSequence.obj
 0001:000eec50       ?GetSplineType@CFacialCameraPathOrientationInterpolator@@UAE?AW4ESplineType@@XZ 315efc50 f i FaceAnimSequence.obj
 0001:000eec50       ?GetFormat@?$CKeyTimesInformationStartStop@MUF32StartStopEncoder@@@@UAEIXZ 315efc50 f i ControllerPQ.obj
 0001:000eec60       ?GetKeyValueFloat@?$CKeyTimesInformationStartStop@GUUINT16StartStopEncoder@@@@UBEMI@Z 315efc60 f i ControllerPQ.obj
 0001:000eec80       ?GetKey@?$CKeyTimesInformationStartStop@GUUINT16StartStopEncoder@@@@UAEIMAAM@Z 315efc80 f i ControllerPQ.obj
 0001:000eed00       ?GetNumKeys@?$CKeyTimesInformationStartStop@GUUINT16StartStopEncoder@@@@UBEIXZ 315efd00 f i ControllerPQ.obj
 0001:000eed10       ?AssignKeyTime@?$CKeyTimesInformationStartStop@GUUINT16StartStopEncoder@@@@UAEIPBDI@Z 315efd10 f i ControllerPQ.obj
 0001:000eed30       ?GetRotationKeysNum@CControllerTCB@@UBEIXZ 315efd30 f i LoaderCGA.obj
 0001:000eed30       ?GetFormat@?$CKeyTimesInformation@MUF32Encoder@@@@UAEIXZ 315efd30 f i ControllerPQ.obj
 0001:000eed30       ?GetAttachmentCRC@CFacialEffector@@UAEIXZ 315efd30 f i FaceEffector.obj
 0001:000eed30       ?GetPositionKeysNum@CControllerPQLog@@UBEIXZ 315efd30 f i ControllerPQLog.obj
 0001:000eed30       ?GetRelocateChain@CKeyTimesInformationBitSet@@UAEPAVIControllerRelocatableChain@@XZ 315efd30 f i ControllerPQ.obj
 0001:000eed30       ?GetRelocateChain@?$CKeyTimesInformationStartStop@GUUINT16StartStopEncoder@@@@UAEPAVIControllerRelocatableChain@@XZ 315efd30 f i ControllerPQ.obj
 0001:000eed30       ?GetRotationKeysNum@CControllerPQLog@@UBEIXZ 315efd30 f i ControllerPQLog.obj
 0001:000eed30       ?GetType@CFacialEffector@@UAE?AW4EFacialEffectorType@@XZ 315efd30 f i FaceEffector.obj
 0001:000eed30       ?GetRelocateChain@?$CKeyTimesInformationStartStop@MUF32StartStopEncoder@@@@UAEPAVIControllerRelocatableChain@@XZ 315efd30 f i ControllerPQ.obj
 0001:000eed30       ?GetRelocateChain@?$CKeyTimesInformationStartStop@EUByteStartStopEncoder@@@@UAEPAVIControllerRelocatableChain@@XZ 315efd30 f i ControllerPQ.obj
 0001:000eed30       ?GetType@CAttachmentBONE@@UBEIXZ 315efd30 f i AttachmentManager.obj
 0001:000eed30       ?GetIStatObj@IAttachmentObject@@UBEPAUIStatObj@@XZ 315efd30 f i AttachmentManager.obj
 0001:000eed30       ?GetIAttachmentSkin@IAttachmentObject@@UBEPAUIAttachmentSkin@@XZ 315efd30 f i AttachmentManager.obj
 0001:000eed30       ?GetICharacterInstance@IAttachmentObject@@UBEPAUICharacterInstance@@XZ 315efd30 f i AttachmentManager.obj
 0001:000eed30       ?ProjectAttachment@CAttachmentSKIN@@UAEIXZ 315efd30 f i Attachment.obj
 0001:000eed30       ?GetPositionKeysNum@CControllerTCB@@UBEIXZ 315efd30 f i LoaderCGA.obj
 0001:000eed40       ?GetMemoryUsage@?$CKeyTimesInformationStartStop@GUUINT16StartStopEncoder@@@@UBEXPAVICrySizer@@@Z 315efd40 f i ControllerPQ.obj
 0001:000eed40       ?GetMemoryUsage@?$CKeyTimesInformationStartStop@EUByteStartStopEncoder@@@@UBEXPAVICrySizer@@@Z 315efd40 f i ControllerPQ.obj
 0001:000eed60       ?GetFormat@?$CKeyTimesInformationStartStop@GUUINT16StartStopEncoder@@@@UAEIXZ 315efd60 f i ControllerPQ.obj
 0001:000eed60       ?GetDataRawSize@?$CKeyTimesInformationStartStop@GUUINT16StartStopEncoder@@@@UAEIXZ 315efd60 f i ControllerPQ.obj
 0001:000eed60       ?GetNumDimensions@CFacialCameraPathOrientationInterpolator@@UAEHXZ 315efd60 f i FaceAnimSequence.obj
 0001:000eed70       ?GetKeyValueFloat@?$CKeyTimesInformationStartStop@EUByteStartStopEncoder@@@@UBEMI@Z 315efd70 f i ControllerPQ.obj
 0001:000eed90       ?GetKey@?$CKeyTimesInformationStartStop@EUByteStartStopEncoder@@@@UAEIMAAM@Z 315efd90 f i ControllerPQ.obj
 0001:000eee10       ?GetNumKeys@?$CKeyTimesInformationStartStop@EUByteStartStopEncoder@@@@UBEIXZ 315efe10 f i ControllerPQ.obj
 0001:000eee20       ?AssignKeyTime@?$CKeyTimesInformationStartStop@EUByteStartStopEncoder@@@@UAEIPBDI@Z 315efe20 f i ControllerPQ.obj
 0001:000eee40       ??0CKeyTimesInformationBitSet@@QAE@PAGI@Z 315efe40 f i ControllerPQ.obj
 0001:000eee90       ?GetPositionControllerPtr@ControllerHelper@@YAPAVITrackPositionStorage@@IPAXI@Z 315efe90 f   ControllerPQ.obj
 0001:000eeef0       ?GetRotationControllerPtr@ControllerHelper@@YAPAVITrackRotationStorage@@IPAXI@Z 315efef0 f   ControllerPQ.obj
 0001:000eefb0       ?GetKeyTimesControllerPtr@ControllerHelper@@YAPAVIKeyTimesInformation@@IPAXI@Z 315effb0 f   ControllerPQ.obj
 0001:000ef100       ??_E?$CKeyTimesInformation@MUF32Encoder@@@@UAEPAXI@Z 315f0100 f i ControllerPQ.obj
 0001:000ef1e0       ??_E?$CKeyTimesInformation@GUUINT16Encoder@@@@UAEPAXI@Z 315f01e0 f i ControllerPQ.obj
 0001:000ef2c0       ??_E?$CKeyTimesInformation@EUByteEncoder@@@@UAEPAXI@Z 315f02c0 f i ControllerPQ.obj
 0001:000ef3a0       ??_E?$CKeyTimesInformationStartStop@MUF32StartStopEncoder@@@@UAEPAXI@Z 315f03a0 f i ControllerPQ.obj
 0001:000ef400       ??_E?$CKeyTimesInformationStartStop@EUByteStartStopEncoder@@@@UAEPAXI@Z 315f0400 f i ControllerPQ.obj
 0001:000ef400       ??_E?$CKeyTimesInformationStartStop@GUUINT16StartStopEncoder@@@@UAEPAXI@Z 315f0400 f i ControllerPQ.obj
 0001:000ef460       ??_E?$CKeyTimesInformation@GUUINT16Encoder@@@@W7AEPAXI@Z 315f0460 f i ControllerPQ.obj
 0001:000ef470       ??_E?$CKeyTimesInformation@EUByteEncoder@@@@W7AEPAXI@Z 315f0470 f i ControllerPQ.obj
 0001:000ef480       ??_E?$CKeyTimesInformation@MUF32Encoder@@@@W7AEPAXI@Z 315f0480 f i ControllerPQ.obj
 0001:000ef490       ?GetRotValue@CControllerOptNonVirtual@@QBE?AU?$Quat_tpl@M@@M@Z 315f0490 f i ControllerPQ.obj
 0001:000ef6e0       ?GetO@CControllerOptNonVirtual@@UBEEMAAU?$Quat_tpl@M@@@Z 315f06e0 f   ControllerPQ.obj
 0001:000ef730       ?GetOP@CControllerOptNonVirtual@@UBEEMAAU?$Quat_tpl@M@@AAU?$Vec3_tpl@M@@@Z 315f0730 f   ControllerPQ.obj
 0001:000ef7c0       ?AdjustLogRotations@@YAXAAU?$Vec3_tpl@M@@0@Z 315f07c0 f   ControllerPQLog.obj
 0001:000ef8b0       ?blendPQ@PQLog@@QAEXABU1@0M@Z 315f08b0 f   ControllerPQLog.obj
 0001:000efc40       ?GetOPS@CControllerPQLog@@UBEEMAAU?$Quat_tpl@M@@AAU?$Vec3_tpl@M@@AAU?$Diag33_tpl@M@@@Z 315f0c40 f   ControllerPQLog.obj
 0001:000f0160       ?GetOP@CControllerPQLog@@UBEEMAAU?$Quat_tpl@M@@AAU?$Vec3_tpl@M@@@Z 315f1160 f   ControllerPQLog.obj
 0001:000f0680       ?GetO@CControllerPQLog@@UBEEMAAU?$Quat_tpl@M@@@Z 315f1680 f   ControllerPQLog.obj
 0001:000f0b90       ?GetP@CControllerPQLog@@UBEEMAAU?$Vec3_tpl@M@@@Z 315f1b90 f   ControllerPQLog.obj
 0001:000f1060       ??1CControllerPQLog@@UAE@XZ 315f2060 f   ControllerPQLog.obj
 0001:000f10d0       ?GetJointCount@CModelSkeleton@@UBEIXZ 315f20d0 f i Model.obj
 0001:000f10d0       ?GetP_numKey@CControllerPQLog@@UBEHXZ 315f20d0 f i ControllerPQLog.obj
 0001:000f10d0       ?GetO_numKey@CControllerPQLog@@UBEHXZ 315f20d0 f i ControllerPQLog.obj
 0001:000f10e0       ?get_alloc_size@?$SmallDynStorage@UPQLog@@HUStandardAlloc@NAlloc@@@NArray@@QBEHXZ 315f20e0 f i ControllerPQLog.obj
 0001:000f1130       ?SizeOfController@CControllerPQLog@@UBEIXZ 315f2130 f i ControllerPQLog.obj
 0001:000f11e0       ?GetMemoryUsage@CControllerPQLog@@UBEXPAVICrySizer@@@Z 315f21e0 f i ControllerPQLog.obj
 0001:000f1230       ??0CControllerPQLog@@QAE@XZ 315f2230 f   ControllerPQLog.obj
 0001:000f12e0       ??_ECControllerPQLog@@UAEPAXI@Z 315f22e0 f i ControllerPQLog.obj
 0001:000f12e0       ??_GCControllerPQLog@@UAEPAXI@Z 315f22e0 f i ControllerPQLog.obj
 0001:000f1310       ??$__unguarded_linear_insert@PAUTCBAngAxisKey@spline@@U12@U?$less@UTCBAngAxisKey@spline@@@stlpmtx_std@@@priv@stlpmtx_std@@YAXPAUTCBAngAxisKey@spline@@U23@U?$less@UTCBAngAxisKey@spline@@@1@@Z 315f2310 f i ControllerTCB.obj
 0001:000f13d0       ??$__push_heap@PAUTCBAngAxisKey@spline@@HU12@U?$less@UTCBAngAxisKey@spline@@@stlpmtx_std@@@stlpmtx_std@@YAXPAUTCBAngAxisKey@spline@@HHU12@U?$less@UTCBAngAxisKey@spline@@@0@@Z 315f23d0 f i ControllerTCB.obj
 0001:000f14c0       ??$__copy_backward@PAUTCBAngAxisKey@spline@@PAU12@H@priv@stlpmtx_std@@YAPAUTCBAngAxisKey@spline@@PAU23@00ABUrandom_access_iterator_tag@1@PAH@Z 315f24c0 f i ControllerTCB.obj
 0001:000f1700       ?seek_key@?$TSpline@UTCBAngAxisKey@spline@@VHermitBasis@2@@spline@@IAEHM@Z 315f2700 f i ControllerTCB.obj
 0001:000f1780       ??$__unguarded_insertion_sort_aux@PAUTCBAngAxisKey@spline@@U12@U?$less@UTCBAngAxisKey@spline@@@stlpmtx_std@@@priv@stlpmtx_std@@YAXPAUTCBAngAxisKey@spline@@00U?$less@UTCBAngAxisKey@spline@@@1@@Z 315f2780 f i ControllerTCB.obj
 0001:000f1850       ??$__adjust_heap@PAUTCBAngAxisKey@spline@@HU12@U?$less@UTCBAngAxisKey@spline@@@stlpmtx_std@@@stlpmtx_std@@YAXPAUTCBAngAxisKey@spline@@HHU12@U?$less@UTCBAngAxisKey@spline@@@0@@Z 315f2850 f i ControllerTCB.obj
 0001:000f1980       ??$swap@UTCBAngAxisKey@spline@@@stlpmtx_std@@YAXAAUTCBAngAxisKey@spline@@0@Z 315f2980 f i ControllerTCB.obj
 0001:000f1a50       ??$__pop_heap@PAUTCBAngAxisKey@spline@@U12@U?$less@UTCBAngAxisKey@spline@@@stlpmtx_std@@H@stlpmtx_std@@YAXPAUTCBAngAxisKey@spline@@00U12@U?$less@UTCBAngAxisKey@spline@@@0@PAH@Z 315f2a50 f i ControllerTCB.obj
 0001:000f1b00       ??$__make_heap@PAUTCBAngAxisKey@spline@@U?$less@UTCBAngAxisKey@spline@@@stlpmtx_std@@U12@H@stlpmtx_std@@YAXPAUTCBAngAxisKey@spline@@0U?$less@UTCBAngAxisKey@spline@@@0@0PAH@Z 315f2b00 f i ControllerTCB.obj
 0001:000f1c00       ??$__linear_insert@PAUTCBAngAxisKey@spline@@U12@U?$less@UTCBAngAxisKey@spline@@@stlpmtx_std@@@priv@stlpmtx_std@@YAXPAUTCBAngAxisKey@spline@@0U23@U?$less@UTCBAngAxisKey@spline@@@1@@Z 315f2c00 f i ControllerTCB.obj
 0001:000f1cd0       ??$sort_heap@PAUTCBAngAxisKey@spline@@U?$less@UTCBAngAxisKey@spline@@@stlpmtx_std@@@stlpmtx_std@@YAXPAUTCBAngAxisKey@spline@@0U?$less@UTCBAngAxisKey@spline@@@0@@Z 315f2cd0 f i ControllerTCB.obj
 0001:000f1dd0       ??$__insertion_sort@PAUTCBAngAxisKey@spline@@U12@U?$less@UTCBAngAxisKey@spline@@@stlpmtx_std@@@priv@stlpmtx_std@@YAXPAUTCBAngAxisKey@spline@@00U?$less@UTCBAngAxisKey@spline@@@1@@Z 315f2dd0 f i ControllerTCB.obj
 0001:000f1e40       ??$__partial_sort@PAUTCBAngAxisKey@spline@@U12@U?$less@UTCBAngAxisKey@spline@@@stlpmtx_std@@@priv@stlpmtx_std@@YAXPAUTCBAngAxisKey@spline@@000U?$less@UTCBAngAxisKey@spline@@@1@@Z 315f2e40 f i ControllerTCB.obj
 0001:000f1ed0       ??$__final_insertion_sort@PAUTCBAngAxisKey@spline@@U?$less@UTCBAngAxisKey@spline@@@stlpmtx_std@@@priv@stlpmtx_std@@YAXPAUTCBAngAxisKey@spline@@0U?$less@UTCBAngAxisKey@spline@@@1@@Z 315f2ed0 f i ControllerTCB.obj
 0001:000f1f40       ??$__introsort_loop@PAUTCBAngAxisKey@spline@@U12@HU?$less@UTCBAngAxisKey@spline@@@stlpmtx_std@@@priv@stlpmtx_std@@YAXPAUTCBAngAxisKey@spline@@00HU?$less@UTCBAngAxisKey@spline@@@1@@Z 315f2f40 f i ControllerTCB.obj
 0001:000f2070       ??$sort@PAUTCBAngAxisKey@spline@@@stlpmtx_std@@YAXPAUTCBAngAxisKey@spline@@0@Z 315f3070 f i ControllerTCB.obj
 0001:000f20d0       ?GetP@CControllerTCB@@UBEEMAAU?$Vec3_tpl@M@@@Z 315f30d0 f   ControllerTCB.obj
 0001:000f21c0       ?GetS@CControllerTCB@@UBEEMAAU?$Diag33_tpl@M@@@Z 315f31c0 f   ControllerTCB.obj
 0001:000f2290       ?interpolate@?$TSpline@UTCBAngAxisKey@spline@@VHermitBasis@2@@spline@@QAE_NMAAU?$Quat_tpl@M@@@Z 315f3290 f i ControllerTCB.obj
 0001:000f23e0       ?GetOPS@CControllerTCB@@UBEEMAAU?$Quat_tpl@M@@AAU?$Vec3_tpl@M@@AAU?$Diag33_tpl@M@@@Z 315f33e0 f   ControllerTCB.obj
 0001:000f2640       ?GetOP@CControllerTCB@@UBEEMAAU?$Quat_tpl@M@@AAU?$Vec3_tpl@M@@@Z 315f3640 f   ControllerTCB.obj
 0001:000f2800       ?GetO@CControllerTCB@@UBEEMAAU?$Quat_tpl@M@@@Z 315f3800 f   ControllerTCB.obj
 0001:000f28f0       ?AnnotateExamples@VExampleInit@@QAEIIPAUQuadIndices@@@Z 315f38f0 f   GlobalAnimationHeaderAIM.obj
 0001:000f28f0       ?Debug_AnnotateExamples2@GlobalAnimationHeaderAIM@@QAEIIPAUQuadIndices@@@Z 315f38f0 f   GlobalAnimationHeaderAIM.obj
 0001:000f35e0       ?Debug_PolarCoordinate@GlobalAnimationHeaderAIM@@QAE?AU?$Vec3_tpl@M@@ABU?$Quat_tpl@M@@@Z 315f45e0 f   GlobalAnimationHeaderAIM.obj
 0001:000f3720       ?ReadMotionParameters@GlobalAnimationHeaderAIM@@QAE_NPAUChunkDesc@IChunkFile@@@Z 315f4720 f   GlobalAnimationHeaderAIM.obj
 0001:000f3810       ?Debug_NLerp2AimPose@GlobalAnimationHeaderAIM@@QAEXPAVCModelSkeleton@@PAUSJointsAimIK_Rot@@IPAUSJointsAimIK_Pos@@IPAU?$QuatT_tpl@M@@3M3@Z 315f4810 f   GlobalAnimationHeaderAIM.obj
 0001:000f3cc0       ?Debug_Blend4AimPose@GlobalAnimationHeaderAIM@@QAEXPAVCModelSkeleton@@PAUSJointsAimIK_Rot@@IPAUSJointsAimIK_Pos@@ICCCCABU?$Vec4_tpl@M@@PAU?$QuatT_tpl@M@@4@Z 315f4cc0 f   GlobalAnimationHeaderAIM.obj
 0001:000f48c0       ?CopyPoses2@VExampleInit@@QAEXAAU?$DynArray@USJointsAimIK_Rot@@HU?$SmallDynStorage@USJointsAimIK_Rot@@HUStandardAlloc@NAlloc@@@NArray@@@@AAU?$DynArray@USJointsAimIK_Pos@@HU?$SmallDynStorage@USJointsAimIK_Pos@@HUStandardAlloc@NAlloc@@@NArray@@@@AAUGlobalAnimationHeaderAIM@@II@Z 315f58c0 f   GlobalAnimationHeaderAIM.obj
 0001:000f4c10       ?ComputeAimPose@VExampleInit@@QAEXAAUGlobalAnimationHeaderAIM@@PAVCModelSkeleton@@AAU?$DynArray@USJointsAimIK_Rot@@HU?$SmallDynStorage@USJointsAimIK_Rot@@HUStandardAlloc@NAlloc@@@NArray@@@@AAU?$DynArray@USJointsAimIK_Pos@@HU?$SmallDynStorage@USJointsAimIK_Pos@@HUStandardAlloc@NAlloc@@@NArray@@@@PAU?$QuatT_tpl@N@@I@Z 315f5c10 f   GlobalAnimationHeaderAIM.obj
 0001:000f4e10       ?NLerp2AimPose@VExampleInit@@QAEXAAU?$DynArray@USJointsAimIK_Rot@@HU?$SmallDynStorage@USJointsAimIK_Rot@@HUStandardAlloc@NAlloc@@@NArray@@@@AAU?$DynArray@USJointsAimIK_Pos@@HU?$SmallDynStorage@USJointsAimIK_Pos@@HUStandardAlloc@NAlloc@@@NArray@@@@PAU?$QuatT_tpl@N@@2N2@Z 315f5e10 f   GlobalAnimationHeaderAIM.obj
 0001:000f5130       ?LinesegOverlap2D@VExampleInit@@QAEIABU?$Plane_tpl@N@@ABU?$Vec2_tpl@N@@111@Z 315f6130 f   GlobalAnimationHeaderAIM.obj
 0001:000f5240       ?PolarCoordinate@VExampleInit@@QAE?AU?$Vec3_tpl@N@@ABU?$Quat_tpl@N@@@Z 315f6240 f   GlobalAnimationHeaderAIM.obj
 0001:000f5320       ?Blend4AimPose@VExampleInit@@QAEXAAUGlobalAnimationHeaderAIM@@AAU?$DynArray@USJointsAimIK_Rot@@HU?$SmallDynStorage@USJointsAimIK_Rot@@HUStandardAlloc@NAlloc@@@NArray@@@@AAU?$DynArray@USJointsAimIK_Pos@@HU?$SmallDynStorage@USJointsAimIK_Pos@@HUStandardAlloc@NAlloc@@@NArray@@@@CCCCABU?$Vec4_tpl@N@@PAU?$QuatT_tpl@N@@4@Z 315f6320 f   GlobalAnimationHeaderAIM.obj
 0001:000f5ab0       ?PointInQuat@VExampleInit@@QAEIABU?$Vec2_tpl@N@@AAUGlobalAnimationHeaderAIM@@AAU?$DynArray@USJointsAimIK_Rot@@HU?$SmallDynStorage@USJointsAimIK_Rot@@HUStandardAlloc@NAlloc@@@NArray@@@@AAU?$DynArray@USJointsAimIK_Pos@@HU?$SmallDynStorage@USJointsAimIK_Pos@@HUStandardAlloc@NAlloc@@@NArray@@@@HHHHHABU?$Vec4_tpl@N@@444@Z 315f6ab0 f   GlobalAnimationHeaderAIM.obj
 0001:000f6b50       ?grow@?$DynArray@UVirtualExampleInit2@CHUNK_GAHAIM_INFO@@HU?$SmallDynStorage@UVirtualExampleInit2@CHUNK_GAHAIM_INFO@@HUStandardAlloc@NAlloc@@@NArray@@@@QAEPAUVirtualExampleInit2@CHUNK_GAHAIM_INFO@@HABU23@@Z 315f7b50 f i GlobalAnimationHeaderAIM.obj
 0001:000f6bb0       ?RecursiveTest@VExampleInit@@QAEXABU?$Vec2_tpl@N@@AAUGlobalAnimationHeaderAIM@@AAU?$DynArray@USJointsAimIK_Rot@@HU?$SmallDynStorage@USJointsAimIK_Rot@@HUStandardAlloc@NAlloc@@@NArray@@@@AAU?$DynArray@USJointsAimIK_Pos@@HU?$SmallDynStorage@USJointsAimIK_Pos@@HUStandardAlloc@NAlloc@@@NArray@@@@HHHHHABU?$Vec4_tpl@N@@444@Z 315f7bb0 f   GlobalAnimationHeaderAIM.obj
 0001:000f8050       ?ReadController@GlobalAnimationHeaderAIM@@QAE_NPAUChunkDesc@IChunkFile@@I@Z 315f9050 f   GlobalAnimationHeaderAIM.obj
 0001:000f8a00       ?LoadChunks@GlobalAnimationHeaderAIM@@QAE_NPAUIChunkFile@@@Z 315f9a00 f   GlobalAnimationHeaderAIM.obj
 0001:000f8c60       ?LoadAIM@GlobalAnimationHeaderAIM@@QAEIXZ 315f9c60 f   GlobalAnimationHeaderAIM.obj
 0001:000f8e80       ?Init@VExampleInit@@QAEXPAVCModelSkeleton@@AAU?$DynArray@USJointsAimIK_Rot@@HU?$SmallDynStorage@USJointsAimIK_Rot@@HUStandardAlloc@NAlloc@@@NArray@@@@AAU?$DynArray@USJointsAimIK_Pos@@HU?$SmallDynStorage@USJointsAimIK_Pos@@HUStandardAlloc@NAlloc@@@NArray@@@@AAUGlobalAnimationHeaderAIM@@HI@Z 315f9e80 f   GlobalAnimationHeaderAIM.obj
 0001:000fc780       ?ProcessAimPoses@GlobalAnimationHeaderAIM@@QAEXPAVCSkel@@AAU?$DynArray@UDirectionalBlends@@HU?$SmallDynStorage@UDirectionalBlends@@HUStandardAlloc@NAlloc@@@NArray@@@@AAU?$DynArray@USJointsAimIK_Rot@@HU?$SmallDynStorage@USJointsAimIK_Rot@@HUStandardAlloc@NAlloc@@@NArray@@@@AAU?$DynArray@USJointsAimIK_Pos@@HU?$SmallDynStorage@USJointsAimIK_Pos@@HUStandardAlloc@NAlloc@@@NArray@@@@@Z 315fd780 f   GlobalAnimationHeaderAIM.obj
 0001:000fc9e0       ?ChangeBoneName@@YAXPBDQAD@Z 315fd9e0 f   GlobalAnimationHeaderCAF.obj
 0001:000fca30       ?_M_allocate@?$allocator@UCryKeyPQLog@@@stlpmtx_std@@QAEPAUCryKeyPQLog@@IAAI@Z 315fda30 f i GlobalAnimationHeaderCAF.obj
 0001:000fca30       ?_M_allocate@?$allocator@USOp@COperatorQueue@@@stlpmtx_std@@QAEPAUSOp@COperatorQueue@@IAAI@Z 315fda30 f i OperatorQueue.obj
 0001:000fcaa0       ?ClearControllerData@GlobalAnimationHeaderCAF@@QAEXXZ 315fdaa0 f   GlobalAnimationHeaderCAF.obj
 0001:000fcac0       ?FlagsSanityFilter@GlobalAnimationHeaderCAFStreamContent@@QAEII@Z 315fdac0 f   GlobalAnimationHeaderCAF.obj
 0001:000fcb00       ??$fill@PAUCryKeyPQLog@@U1@@stlpmtx_std@@YAXPAUCryKeyPQLog@@0ABU1@@Z 315fdb00 f i GlobalAnimationHeaderCAF.obj
 0001:000fcb40       ?DoesExistCAF@GlobalAnimationHeaderCAF@@QAEIXZ 315fdb40 f   GlobalAnimationHeaderCAF.obj
 0001:000fcc00       ?GetTotalPosKeys@GlobalAnimationHeaderCAF@@QBEIXZ 315fdc00 f   GlobalAnimationHeaderCAF.obj
 0001:000fcc40       ?GetTotalRotKeys@GlobalAnimationHeaderCAF@@QBEIXZ 315fdc40 f   GlobalAnimationHeaderCAF.obj
 0001:000fcc80       ?ConnectCAFandDBA@GlobalAnimationHeaderCAF@@QAEXXZ 315fdc80 f   GlobalAnimationHeaderCAF.obj
 0001:000fccd0       ?init@?$DynArray@U?$QuatT_tpl@M@@HU?$SmallDynStorage@U?$QuatT_tpl@M@@HUStandardAlloc@NAlloc@@@NArray@@@@KAPAU?$QuatT_tpl@M@@U?$Array@U?$QuatT_tpl@M@@HU?$ArrayStorage@U?$QuatT_tpl@M@@H@NArray@@@@PBU2@@Z 315fdcd0 f i GlobalAnimationHeaderCAF.obj
 0001:000fcd40       ?assign@?$Array@U?$QuatT_tpl@M@@HU?$SmallDynStorage@U?$QuatT_tpl@M@@HUStandardAlloc@NAlloc@@@NArray@@@@QAEXU?$Array@$$CBU?$QuatT_tpl@M@@HU?$ArrayStorage@$$CBU?$QuatT_tpl@M@@H@NArray@@@@@Z 315fdd40 f i GlobalAnimationHeaderCAF.obj
 0001:000fcdb0       ?LoadDBA@GlobalAnimationHeaderCAF@@QAEXXZ 315fddb0 f   GlobalAnimationHeaderCAF.obj
 0001:000fcea0       ?StreamOnNeedStorage@GlobalAnimationHeaderCAFStreamContent@@UAEPAXPAVIReadStream@@I@Z 315fdea0 f   GlobalAnimationHeaderCAF.obj
 0001:000fcf30       ?ReadMotionParameters@GlobalAnimationHeaderCAFStreamContent@@QAE_NPAUChunkDesc@IChunkFile@@@Z 315fdf30 f   GlobalAnimationHeaderCAF.obj
 0001:000fd0c0       ?CommitContent@GlobalAnimationHeaderCAF@@AAEXAAUGlobalAnimationHeaderCAFStreamContent@@@Z 315fe0c0 f   GlobalAnimationHeaderCAF.obj
 0001:000fd170       ?_M_insert_overflow@?$_Impl_vector@UCryKeyPQLog@@V?$allocator@UCryKeyPQLog@@@stlpmtx_std@@@priv@stlpmtx_std@@AAEXPAUCryKeyPQLog@@ABU4@ABU__true_type@3@I_N@Z 315fe170 f i GlobalAnimationHeaderCAF.obj
 0001:000fd170       ?_M_insert_overflow@?$_Impl_vector@USOp@COperatorQueue@@V?$allocator@USOp@COperatorQueue@@@stlpmtx_std@@@priv@stlpmtx_std@@AAEXPAUSOp@COperatorQueue@@ABU45@ABU__true_type@3@I_N@Z 315fe170 f i OperatorQueue.obj
 0001:000fd2c0       ??$__uninitialized_fill_n@PAUCryKeyPQLog@@IU1@@priv@stlpmtx_std@@YAPAUCryKeyPQLog@@PAU2@IABU2@@Z 315fe2c0 f i GlobalAnimationHeaderCAF.obj
 0001:000fd340       ?SizeOfCAF@GlobalAnimationHeaderCAF@@QBEI_N@Z 315fe340 f   GlobalAnimationHeaderCAF.obj
 0001:000fd480       ?GetMemoryUsage@GlobalAnimationHeaderCAF@@QBEXPAVICrySizer@@@Z 315fe480 f   GlobalAnimationHeaderCAF.obj
 0001:000fd500       ?_M_fill_insert_aux@?$_Impl_vector@UCryKeyPQLog@@V?$allocator@UCryKeyPQLog@@@stlpmtx_std@@@priv@stlpmtx_std@@AAEXPAUCryKeyPQLog@@IABU4@ABU__false_type@3@@Z 315fe500 f i GlobalAnimationHeaderCAF.obj
 0001:000fd630       ?erase@?$DynArray@U?$QuatT_tpl@M@@HU?$SmallDynStorage@U?$QuatT_tpl@M@@HUStandardAlloc@NAlloc@@@NArray@@@@QAEPAU?$QuatT_tpl@M@@PAU2@0@Z 315fe630 f i GlobalAnimationHeaderCAF.obj
 0001:000fd7e0       ?ClearControllers@GlobalAnimationHeaderCAF@@QAEXXZ 315fe7e0 f   GlobalAnimationHeaderCAF.obj
 0001:000fd8c0       ??4?$DynArray@U?$QuatT_tpl@M@@HU?$SmallDynStorage@U?$QuatT_tpl@M@@HUStandardAlloc@NAlloc@@@NArray@@@@QAEAAU0@U?$Array@$$CBU?$QuatT_tpl@M@@HU?$ArrayStorage@$$CBU?$QuatT_tpl@M@@H@NArray@@@@@Z 315fe8c0 f i GlobalAnimationHeaderCAF.obj
 0001:000fd970       ??1GlobalAnimationHeaderCAFStreamContent@@UAE@XZ 315fe970 f   GlobalAnimationHeaderCAF.obj
 0001:000fd9b0       ?SaveHTR@GlobalAnimationHeaderCAF@@SA_NPBD0ABV?$vector@V?$CryStringT@D@@V?$allocator@V?$CryStringT@D@@@stlpmtx_std@@@stlpmtx_std@@1ABV?$vector@U?$DynArray@U?$QuatT_tpl@M@@HU?$SmallDynStorage@U?$QuatT_tpl@M@@HUStandardAlloc@NAlloc@@@NArray@@@@V?$allocator@U?$DynArray@U?$QuatT_tpl@M@@HU?$SmallDynStorage@U?$QuatT_tpl@M@@HUStandardAlloc@NAlloc@@@NArray@@@@@stlpmtx_std@@@3@PBU?$QuatT_tpl@M@@@Z 315fe9b0 f   GlobalAnimationHeaderCAF.obj
 0001:000fe300       ??$__copy_backward@PAU?$DynArray@U?$QuatT_tpl@M@@HU?$SmallDynStorage@U?$QuatT_tpl@M@@HUStandardAlloc@NAlloc@@@NArray@@@@PAU1@H@priv@stlpmtx_std@@YAPAU?$DynArray@U?$QuatT_tpl@M@@HU?$SmallDynStorage@U?$QuatT_tpl@M@@HUStandardAlloc@NAlloc@@@NArray@@@@PAU2@00ABUrandom_access_iterator_tag@1@PAH@Z 315ff300 f i GlobalAnimationHeaderCAF.obj
 0001:000fe350       ??0GlobalAnimationHeaderCAFStreamContent@@QAE@XZ 315ff350 f   GlobalAnimationHeaderCAF.obj
 0001:000fe3b0       ??_GGlobalAnimationHeaderCAFStreamContent@@UAEPAXI@Z 315ff3b0 f i GlobalAnimationHeaderCAF.obj
 0001:000fe3b0       ??_EGlobalAnimationHeaderCAFStreamContent@@UAEPAXI@Z 315ff3b0 f i GlobalAnimationHeaderCAF.obj
 0001:000fe400       ?ParseChunkHeaders@GlobalAnimationHeaderCAFStreamContent@@QAEIPAUIChunkFile@@AA_N1AAI@Z 315ff400 f   GlobalAnimationHeaderCAF.obj
 0001:000fe720       ?ReadController@GlobalAnimationHeaderCAFStreamContent@@QAE_NPAUChunkDesc@IChunkFile@@_NAAPADAAPAVIControllerRelocatableChain@@@Z 315ff720 f   GlobalAnimationHeaderCAF.obj
 0001:000ff240       ??$__copy@PAU?$DynArray@U?$QuatT_tpl@M@@HU?$SmallDynStorage@U?$QuatT_tpl@M@@HUStandardAlloc@NAlloc@@@NArray@@@@PAU1@H@priv@stlpmtx_std@@YAPAU?$DynArray@U?$QuatT_tpl@M@@HU?$SmallDynStorage@U?$QuatT_tpl@M@@HUStandardAlloc@NAlloc@@@NArray@@@@PAU2@00ABUrandom_access_iterator_tag@1@PAH@Z 31600240 f i GlobalAnimationHeaderCAF.obj
 0001:000ff290       ??0?$DynArray@U?$QuatT_tpl@M@@HU?$SmallDynStorage@U?$QuatT_tpl@M@@HUStandardAlloc@NAlloc@@@NArray@@@@QAE@ABU0@@Z 31600290 f i GlobalAnimationHeaderCAF.obj
 0001:000ff320       ??$fill@PAU?$DynArray@U?$QuatT_tpl@M@@HU?$SmallDynStorage@U?$QuatT_tpl@M@@HUStandardAlloc@NAlloc@@@NArray@@@@U1@@stlpmtx_std@@YAXPAU?$DynArray@U?$QuatT_tpl@M@@HU?$SmallDynStorage@U?$QuatT_tpl@M@@HUStandardAlloc@NAlloc@@@NArray@@@@0ABU1@@Z 31600320 f i GlobalAnimationHeaderCAF.obj
 0001:000ff360       ??$__destroy_range_aux@V?$reverse_iterator@PAU?$DynArray@U?$QuatT_tpl@M@@HU?$SmallDynStorage@U?$QuatT_tpl@M@@HUStandardAlloc@NAlloc@@@NArray@@@@@stlpmtx_std@@U?$DynArray@U?$QuatT_tpl@M@@HU?$SmallDynStorage@U?$QuatT_tpl@M@@HUStandardAlloc@NAlloc@@@NArray@@@@@stlpmtx_std@@YAXV?$reverse_iterator@PAU?$DynArray@U?$QuatT_tpl@M@@HU?$SmallDynStorage@U?$QuatT_tpl@M@@HUStandardAlloc@NAlloc@@@NArray@@@@@0@0PAU?$DynArray@U?$QuatT_tpl@M@@HU?$SmallDynStorage@U?$QuatT_tpl@M@@HUStandardAlloc@NAlloc@@@NArray@@@@ABU__false_type@0@@Z 31600360 f i GlobalAnimationHeaderCAF.obj
 0001:000ff410       ??$__destroy_range_aux@PAU?$DynArray@U?$QuatT_tpl@M@@HU?$SmallDynStorage@U?$QuatT_tpl@M@@HUStandardAlloc@NAlloc@@@NArray@@@@U1@@stlpmtx_std@@YAXPAU?$DynArray@U?$QuatT_tpl@M@@HU?$SmallDynStorage@U?$QuatT_tpl@M@@HUStandardAlloc@NAlloc@@@NArray@@@@00ABU__false_type@0@@Z 31600410 f i GlobalAnimationHeaderCAF.obj
 0001:000ff4b0       ?ParseChunkRange@GlobalAnimationHeaderCAFStreamContent@@QAE_NPAUIChunkFile@@II_NAAPADAAPAVIControllerRelocatableChain@@@Z 316004b0 f   GlobalAnimationHeaderCAF.obj
 0001:000ff580       ?StreamAsyncOnComplete@GlobalAnimationHeaderCAFStreamContent@@UAEXPAVIReadStream@@I@Z 31600580 f   GlobalAnimationHeaderCAF.obj
 0001:000ff720       ?SaveCAF@GlobalAnimationHeaderCAF@@SA_NPBD0ABV?$vector@V?$CryStringT@D@@V?$allocator@V?$CryStringT@D@@@stlpmtx_std@@@stlpmtx_std@@ABV?$vector@U?$DynArray@U?$QuatT_tpl@M@@HU?$SmallDynStorage@U?$QuatT_tpl@M@@HUStandardAlloc@NAlloc@@@NArray@@@@V?$allocator@U?$DynArray@U?$QuatT_tpl@M@@HU?$SmallDynStorage@U?$QuatT_tpl@M@@HUStandardAlloc@NAlloc@@@NArray@@@@@stlpmtx_std@@@3@@Z 31600720 f   GlobalAnimationHeaderCAF.obj
 0001:000ffdf0       ??$__uninitialized_fill_n@PAU?$DynArray@U?$QuatT_tpl@M@@HU?$SmallDynStorage@U?$QuatT_tpl@M@@HUStandardAlloc@NAlloc@@@NArray@@@@IU1@@priv@stlpmtx_std@@YAPAU?$DynArray@U?$QuatT_tpl@M@@HU?$SmallDynStorage@U?$QuatT_tpl@M@@HUStandardAlloc@NAlloc@@@NArray@@@@PAU2@IABU2@@Z 31600df0 f i GlobalAnimationHeaderCAF.obj
 0001:000ffe30       ??$__ucopy_ptrs@PAU?$DynArray@U?$QuatT_tpl@M@@HU?$SmallDynStorage@U?$QuatT_tpl@M@@HUStandardAlloc@NAlloc@@@NArray@@@@PAU1@@priv@stlpmtx_std@@YAPAU?$DynArray@U?$QuatT_tpl@M@@HU?$SmallDynStorage@U?$QuatT_tpl@M@@HUStandardAlloc@NAlloc@@@NArray@@@@PAU2@00ABU__false_type@1@@Z 31600e30 f i GlobalAnimationHeaderCAF.obj
 0001:000ffe70       ?StartStreamingCAF@GlobalAnimationHeaderCAF@@QAEXXZ 31600e70 f   GlobalAnimationHeaderCAF.obj
 0001:00100170       ?ControllerInit@GlobalAnimationHeaderCAF@@QAEXXZ 31601170 f   GlobalAnimationHeaderCAF.obj
 0001:001001f0       ?_M_fill_insert_aux@?$_Impl_vector@U?$DynArray@U?$QuatT_tpl@M@@HU?$SmallDynStorage@U?$QuatT_tpl@M@@HUStandardAlloc@NAlloc@@@NArray@@@@V?$allocator@U?$DynArray@U?$QuatT_tpl@M@@HU?$SmallDynStorage@U?$QuatT_tpl@M@@HUStandardAlloc@NAlloc@@@NArray@@@@@stlpmtx_std@@@priv@stlpmtx_std@@AAEXPAU?$DynArray@U?$QuatT_tpl@M@@HU?$SmallDynStorage@U?$QuatT_tpl@M@@HUStandardAlloc@NAlloc@@@NArray@@@@IABU4@ABU__false_type@3@@Z 316011f0 f i GlobalAnimationHeaderCAF.obj
 0001:00100310       ?LoadCAF@GlobalAnimationHeaderCAF@@QAEIXZ 31601310 f   GlobalAnimationHeaderCAF.obj
 0001:001005b0       ?LoadControllersCAF@GlobalAnimationHeaderCAF@@QAEXXZ 316015b0 f   GlobalAnimationHeaderCAF.obj
 0001:001005d0       ?FinishLoading@GlobalAnimationHeaderCAF@@AAEXI@Z 316015d0 f   GlobalAnimationHeaderCAF.obj
 0001:001006a0       ?_M_insert_overflow_aux@?$_Impl_vector@U?$DynArray@U?$QuatT_tpl@M@@HU?$SmallDynStorage@U?$QuatT_tpl@M@@HUStandardAlloc@NAlloc@@@NArray@@@@V?$allocator@U?$DynArray@U?$QuatT_tpl@M@@HU?$SmallDynStorage@U?$QuatT_tpl@M@@HUStandardAlloc@NAlloc@@@NArray@@@@@stlpmtx_std@@@priv@stlpmtx_std@@AAEXPAU?$DynArray@U?$QuatT_tpl@M@@HU?$SmallDynStorage@U?$QuatT_tpl@M@@HUStandardAlloc@NAlloc@@@NArray@@@@ABU4@ABU__false_type@3@I_N@Z 316016a0 f i GlobalAnimationHeaderCAF.obj
 0001:00100880       ?StreamOnComplete@GlobalAnimationHeaderCAFStreamContent@@UAEXPAVIReadStream@@I@Z 31601880 f   GlobalAnimationHeaderCAF.obj
 0001:00100990       ?Export2HTR@GlobalAnimationHeaderCAF@@QAE_NPBD0PBVCSkel@@@Z 31601990 f   GlobalAnimationHeaderCAF.obj
 0001:00101330       ?ExportVGrid@GlobalAnimationHeaderLMG@@QAE_NPBD0PBVCSkel@@PAVCSkeletonAnim@@@Z 31602330 f   GlobalAnimationHeaderLMG.obj
 0001:00101440       ?Init_TravelDist@GlobalAnimationHeaderLMG@@QAEXPBVCAnimationSet@@I@Z 31602440 f   GlobalAnimationHeaderLMG.obj
 0001:00101620       ?reserve@?$DynArray@UBSBlendable@@HU?$SmallDynStorage@UBSBlendable@@HUStandardAlloc@NAlloc@@@NArray@@@@QAEXH@Z 31602620 f i GlobalAnimationHeaderLMG.obj
 0001:00101680       ?init@?$DynArray@UBSParameter@@HU?$SmallDynStorage@UBSParameter@@HUStandardAlloc@NAlloc@@@NArray@@@@KAPAUBSParameter@@U?$Array@UBSParameter@@HU?$ArrayStorage@UBSParameter@@H@NArray@@@@@Z 31602680 f i GlobalAnimationHeaderLMG.obj
 0001:001016f0       ?push_back@?$DynArray@UBSBlendable@@HU?$SmallDynStorage@UBSBlendable@@HUStandardAlloc@NAlloc@@@NArray@@@@QAEPAUBSBlendable@@ABU2@@Z 316026f0 f i GlobalAnimationHeaderLMG.obj
 0001:00101750       ?Init_MoveSpeed@GlobalAnimationHeaderLMG@@QAEXPBVCAnimationSet@@I@Z 31602750 f   GlobalAnimationHeaderLMG.obj
 0001:00101ae0       ?Init_TurnSpeed@GlobalAnimationHeaderLMG@@QAEXPBVCAnimationSet@@I@Z 31602ae0 f   GlobalAnimationHeaderLMG.obj
 0001:00101fb0       ?Init_TurnAngle@GlobalAnimationHeaderLMG@@QAEXPBVCAnimationSet@@I@Z 31602fb0 f   GlobalAnimationHeaderLMG.obj
 0001:00102360       ?Init_TravelAngle@GlobalAnimationHeaderLMG@@QAEXPBVCAnimationSet@@I@Z 31603360 f   GlobalAnimationHeaderLMG.obj
 0001:001028e0       ?Init_SlopeAngle@GlobalAnimationHeaderLMG@@QAEXPBVCAnimationSet@@I@Z 316038e0 f   GlobalAnimationHeaderLMG.obj
 0001:00102e20       ?clear@?$DynArray@UBSParameter@@HU?$SmallDynStorage@UBSParameter@@HUStandardAlloc@NAlloc@@@NArray@@@@QAEXXZ 31603e20 f i GlobalAnimationHeaderLMG.obj
 0001:00102e80       ?init@?$DynArray@UBlendSpaceInfo@@HU?$SmallDynStorage@UBlendSpaceInfo@@HUStandardAlloc@NAlloc@@@NArray@@@@KAPAUBlendSpaceInfo@@U?$Array@UBlendSpaceInfo@@HU?$ArrayStorage@UBlendSpaceInfo@@H@NArray@@@@@Z 31603e80 f i GlobalAnimationHeaderLMG.obj
 0001:00102f20       ?ParameterExtraction@GlobalAnimationHeaderLMG@@QAEXPBVCAnimationSet@@II@Z 31603f20 f   GlobalAnimationHeaderLMG.obj
 0001:00102fb0       ?resize@?$DynArray@USCRCName@@HU?$SmallDynStorage@USCRCName@@HUStandardAlloc@NAlloc@@@NArray@@@@QAEXH@Z 31603fb0 f i GlobalAnimationHeaderLMG.obj
 0001:00103020       ?resize@?$DynArray@UBSParameter@@HU?$SmallDynStorage@UBSParameter@@HUStandardAlloc@NAlloc@@@NArray@@@@QAEXH@Z 31604020 f i GlobalAnimationHeaderLMG.obj
 0001:00103090       ?resize@?$DynArray@UBlendSpaceInfo@@HU?$SmallDynStorage@UBlendSpaceInfo@@HUStandardAlloc@NAlloc@@@NArray@@@@QAEXH@Z 31604090 f i GlobalAnimationHeaderLMG.obj
 0001:00103100       ?LoadAndParseXML@GlobalAnimationHeaderLMG@@QAE_NPAVCAnimationSet@@_N@Z 31604100 f   GlobalAnimationHeaderLMG.obj
 0001:001062b0       ?CreateInternalType_Para1D@GlobalAnimationHeaderLMG@@QAEXXZ 316072b0 f   GlobalAnimationHeaderLMG.obj
 0001:001064f0       ?Export2HTR@GlobalAnimationHeaderLMG@@QAE_NPBD0PBVCSkel@@PAVCSkeletonAnim@@@Z 316074f0 f   GlobalAnimationHeaderLMG.obj
 0001:00107b50       ??0CryLock_CritSection@@QAE@XZ 31608b50 f   AnimationBase.obj
 0001:00107b60       ??1CryLock_CritSection@@QAE@XZ 31608b60 f   AnimationBase.obj
 0001:00107b70       ?Lock@CryLock_CritSection@@QAEXXZ 31608b70 f   AnimationBase.obj
 0001:00107b80       ?Unlock@CryLock_CritSection@@QAEXXZ 31608b80 f   AnimationBase.obj
 0001:00107b90       ?cry_rand32@@YAIXZ         31608b90 f   AnimationBase.obj
 0001:00107bd0       ?cry_rand@@YAIXZ           31608bd0 f   AnimationBase.obj
 0001:00107c10       ?cry_frand@@YAMXZ          31608c10 f   AnimationBase.obj
 0001:00107c70       ?Init@_CryMemoryManagerPoolHelper@@SAXXZ 31608c70 f i AnimationBase.obj
 0001:00107df0       ?CryGetIMemoryManager@@YAPAUIMemoryManager@@XZ 31608df0 f   AnimationBase.obj
 0001:00107e30       ?CrySleep@@YAXI@Z          31608e30 f   AnimationBase.obj
 0001:00107e40       ?CryInterlockedIncrement@@YAJPCH@Z 31608e40 f   AnimationBase.obj
 0001:00107e50       ?CryInterlockedDecrement@@YAJPCH@Z 31608e50 f   AnimationBase.obj
 0001:00107e60       ?CryInterlockedCompareExchangePointer@@YAPAXPCRAXPAX1@Z 31608e60 f   AnimationBase.obj
 0001:00107e80       ?CryCreateCriticalSectionInplace@@YAXPAX@Z 31608e80 f   AnimationBase.obj
 0001:00107e90       ?CryGetCurrentThreadId@@YAIXZ 31608e90 f   AnimationBase.obj
 0001:00107ea0       ?CryPureCallHandler@@YAXXZ 31608ea0 f   AnimationBase.obj
 0001:00107eb0       ?CryInvalidParameterHandler@@YAXPB_W00II@Z 31608eb0 f   AnimationBase.obj
 0001:00107ec0       _ModuleInitISystem         31608ec0 f   AnimationBase.obj
 0001:00107f70       _CryModuleGetMemoryInfo    31608f70 f   AnimationBase.obj
 0001:00107f70       _CryGetMemoryInfoForModule 31608f70 f   AnimationBase.obj
 0001:00107fc0       ?CryDeleteCriticalSectionInplace@@YAXPAX@Z 31608fc0 f   AnimationBase.obj
 0001:00107ff0       _CryModuleMalloc           31608ff0 f   AnimationBase.obj
 0001:00108080       _CryModuleRealloc          31609080 f   AnimationBase.obj
 0001:00108120       _CryModuleFree             31609120 f   AnimationBase.obj
 0001:00108180       _CryModuleMemalign         31609180 f   AnimationBase.obj
 0001:00108210       _CryModuleMemalignFree     31609210 f   AnimationBase.obj
 0001:00108270       ??2@YAPAXI@Z               31609270 f   AnimationBase.obj
 0001:001082c0       ??_U@YAPAXI@Z              316092c0 f   AnimationBase.obj
 0001:00108310       ??3@YAXPAX@Z               31609310 f   AnimationBase.obj
 0001:00108390       ??_V@YAXPAX@Z              31609390 f   AnimationBase.obj
 0001:00108410       ?OnSystemEvent@CSystemEventListner_Animation@@UAEXW4ESystemEvent@@II@Z 31609410 f i AnimationBase.obj
 0001:001085d0       ??_EJoystickSerializeContext@?4??BindJoystickSetToSequence@CFacialAnimation@@UAEXPAVIJoystickSet@@PAUIFacialAnimSequence@@@Z@UAEPAXI@Z 316095d0 f i FaceAnimation.obj
 0001:001085d0       ??_ECSystemEventListner_Animation@@UAEPAXI@Z 316095d0 f i AnimationBase.obj
 0001:001085d0       ??_GJoystickSerializeContext@?4??BindJoystickSetToSequence@CFacialAnimation@@UAEXPAVIJoystickSet@@PAUIFacialAnimSequence@@@Z@UAEPAXI@Z 316095d0 f i FaceAnimation.obj
 0001:001085d0       ??_GIFacialJoystickSerializeContext@@UAEPAXI@Z 316095d0 f i FaceAnimation.obj
 0001:001085d0       ??_EISystemEventListener@@UAEPAXI@Z 316095d0 f i AnimationBase.obj
 0001:001085d0       ??_EIFacialJoystickSerializeContext@@UAEPAXI@Z 316095d0 f i FaceAnimation.obj
 0001:001085d0       ??_GISystemEventListener@@UAEPAXI@Z 316095d0 f i AnimationBase.obj
 0001:001085d0       ??_GCSystemEventListner_Animation@@UAEPAXI@Z 316095d0 f i AnimationBase.obj
 0001:00108600       ?GetFactory@CEngineModule_CryAnimation@@UBEPAUICryFactory@@XZ 31609600 f i AnimationBase.obj
 0001:00108610       ?GetName@CEngineModule_CryAnimation@@MAEPBDXZ 31609610 f i AnimationBase.obj
 0001:00108620       ?GetCategory@CEngineModule_CryAnimation@@MAEPBDXZ 31609620 f i AnimationBase.obj
 0001:00108630       ?Initialize@CEngineModule_CryAnimation@@MAE_NAAUSSystemGlobalEnvironment@@ABUSSystemInitParams@@@Z 31609630 f i AnimationBase.obj
 0001:00108780       ??0CFactory@CEngineModule_CryAnimation@@AAE@XZ 31609780 f i AnimationBase.obj
 0001:00108830       ?GetClassName@CFactory@CEngineModule_CryAnimation@@UBEPBDXZ 31609830 f i AnimationBase.obj
 0001:00108840       ?GetClassID@CFactory@CEngineModule_CryAnimation@@UBEABUCryGUID@@XZ 31609840 f i AnimationBase.obj
 0001:00108850       ??_ECFactory@CEngineModule_CryAnimation@@UAEPAXI@Z 31609850 f i AnimationBase.obj
 0001:00108850       ??_GCFactory@CEngineModule_CryAnimation@@UAEPAXI@Z 31609850 f i AnimationBase.obj
 0001:00108880       ??$?0VCEngineModule_CryAnimation@@@shared_count@detail@boost@@QAE@PAVCEngineModule_CryAnimation@@@Z 31609880 f i AnimationBase.obj
 0001:00108930       ??_G?$sp_counted_impl_p@VCPoseBlenderLook@@@detail@boost@@UAEPAXI@Z 31609930 f i PoseBlenderLook.obj
 0001:00108930       ??_Esp_counted_base@detail@boost@@UAEPAXI@Z 31609930 f i OperatorQueue.obj
 0001:00108930       ??_G?$sp_counted_impl_p@VCFeetPoseStore@@@detail@boost@@UAEPAXI@Z 31609930 f i FeetLock.obj
 0001:00108930       ??_G?$sp_counted_impl_p@VCFeetPoseRestore@@@detail@boost@@UAEPAXI@Z 31609930 f i FeetLock.obj
 0001:00108930       ??_E?$sp_counted_impl_p@VCPoseMatching@@@detail@boost@@UAEPAXI@Z 31609930 f i PoseMatching.obj
 0001:00108930       ??_G?$sp_counted_impl_p@VCGroundAlignment@@@detail@boost@@UAEPAXI@Z 31609930 f i GroundAlignment.obj
 0001:00108930       ??_G?$sp_counted_impl_p@VCPoseBlenderAim@@@detail@boost@@UAEPAXI@Z 31609930 f i PoseBlenderAim.obj
 0001:00108930       ??_E?$sp_counted_impl_p@VCPoseAlignerChain@@@detail@boost@@UAEPAXI@Z 31609930 f i PoseAlignerChain.obj
 0001:00108930       ??_E?$sp_counted_impl_p@VCFeetPoseRestore@@@detail@boost@@UAEPAXI@Z 31609930 f i FeetLock.obj
 0001:00108930       ??_G?$sp_counted_impl_p@VCRecoil@PoseModifier@@@detail@boost@@UAEPAXI@Z 31609930 f i Recoil.obj
 0001:00108930       ??_G?$sp_counted_impl_p@VCOperatorQueue@@@detail@boost@@UAEPAXI@Z 31609930 f i OperatorQueue.obj
 0001:00108930       ??_Gsp_counted_base@detail@boost@@UAEPAXI@Z 31609930 f i OperatorQueue.obj
 0001:00108930       ??_E?$sp_counted_impl_p@VCGroundAlignment@@@detail@boost@@UAEPAXI@Z 31609930 f i GroundAlignment.obj
 0001:00108930       ??_E?$sp_counted_impl_p@VCOperatorQueue@@@detail@boost@@UAEPAXI@Z 31609930 f i OperatorQueue.obj
 0001:00108930       ??_E?$sp_counted_impl_p@VCLimbIk@@@detail@boost@@UAEPAXI@Z 31609930 f i LimbIk.obj
 0001:00108930       ??_E?$sp_counted_impl_p@VCFeetPoseStore@@@detail@boost@@UAEPAXI@Z 31609930 f i FeetLock.obj
 0001:00108930       ??_E?$sp_counted_impl_p@VCEngineModule_CryAnimation@@@detail@boost@@UAEPAXI@Z 31609930 f i AnimationBase.obj
 0001:00108930       ??_E?$sp_counted_impl_p@VCPoseBlenderLook@@@detail@boost@@UAEPAXI@Z 31609930 f i PoseBlenderLook.obj
 0001:00108930       ??_G?$sp_counted_impl_p@VCEngineModule_CryAnimation@@@detail@boost@@UAEPAXI@Z 31609930 f i AnimationBase.obj
 0001:00108930       ??_E?$sp_counted_impl_p@VCRecoil@PoseModifier@@@detail@boost@@UAEPAXI@Z 31609930 f i Recoil.obj
 0001:00108930       ??_G?$sp_counted_impl_p@VCPoseAlignerChain@@@detail@boost@@UAEPAXI@Z 31609930 f i PoseAlignerChain.obj
 0001:00108930       ??_G?$sp_counted_impl_p@VCPoseMatching@@@detail@boost@@UAEPAXI@Z 31609930 f i PoseMatching.obj
 0001:00108930       ??_G?$sp_counted_impl_p@VCLimbIk@@@detail@boost@@UAEPAXI@Z 31609930 f i LimbIk.obj
 0001:00108930       ??_E?$sp_counted_impl_p@VCPoseBlenderAim@@@detail@boost@@UAEPAXI@Z 31609930 f i PoseBlenderAim.obj
 0001:00108960       ?QueryInterface@CEngineModule_CryAnimation@@MBEPAXABUCryGUID@@@Z 31609960 f i AnimationBase.obj
 0001:001089c0       ?CreateClassInstance@CFactory@CEngineModule_CryAnimation@@UBE?AV?$shared_ptr@UICryUnknown@@@boost@@XZ 316099c0 f i AnimationBase.obj
 0001:00108a90       ??0CAnimationThreadTask@@QAE@XZ 31609a90 f   AnimationThreadTask.obj
 0001:00108ab0       ??1CAnimationThreadTask@@UAE@XZ 31609ab0 f   AnimationThreadTask.obj
 0001:00108ac0       ??_ECAnimationThreadTask@@UAEPAXI@Z 31609ac0 f i AnimationThreadTask.obj
 0001:00108ac0       ??_GCAnimationThreadTask@@UAEPAXI@Z 31609ac0 f i AnimationThreadTask.obj
 0001:00108af0       ?Begin@CAnimationThreadTask@@QAEXXZ 31609af0 f   AnimationThreadTask.obj
 0001:00108b10       ?DrawPose@Console@@QAE_ND@Z 31609b10 f   cvars.obj
 0001:00108c90       ?Init@Console@@QAEXXZ      31609c90 f   cvars.obj
 0001:00109eb0       ?DeInitialize@?$Node_Alloc_Lock@$00$00@@SAXXZ 3160aeb0 f i stdafx.obj
 0001:00109f00       ??0CContext@Memory@@QAE@XZ 3160af00 f   Memory.obj
 0001:00109f10       ?RemovePool@CContext@Memory@@QAEXAAVCPool@2@@Z 3160af10 f   Memory.obj
 0001:00109f50       ?Update@CAnimationContext@@QAEXXZ 3160af50 f   Memory.obj
 0001:00109f70       ?AddPool@CContext@Memory@@QAEXAAVCPool@2@@Z 3160af70 f   Memory.obj
 0001:00109f90       ?GetMemoryUsage@CAnimationContext@@QBEXPAVICrySizer@@@Z 3160af90 f   Memory.obj
 0001:00109fd0       ??_ECPool@Memory@@MAEPAXI@Z 3160afd0 f i Pool.obj
 0001:00109fd0       ??_GCPool@Memory@@MAEPAXI@Z 3160afd0 f i Pool.obj
 0001:0010a000       ?Create@CBucket@CPoolFrameLocal@Memory@@SAPAV123@I@Z 3160b000 f   Pool.obj
 0001:0010a060       ?Update@CPoolFrameLocal@Memory@@UAEXXZ 3160b060 f   Pool.obj
 0001:0010a090       ??$AddObject@PAVCBucket@CPoolFrameLocal@Memory@@V?$allocator@PAVCBucket@CPoolFrameLocal@Memory@@@stlpmtx_std@@@ICrySizer@@QAEXABV?$vector@PAVCBucket@CPoolFrameLocal@Memory@@V?$allocator@PAVCBucket@CPoolFrameLocal@Memory@@@stlpmtx_std@@@stlpmtx_std@@@Z 3160b090 f i Pool.obj
 0001:0010a110       ?GetMemoryUsage@CPoolFrameLocal@Memory@@UBEXPAVICrySizer@@@Z 3160b110 f   Pool.obj
 0001:0010a140       ??0CPoolFrameLocal@Memory@@AAE@AAVCContext@1@I@Z 3160b140 f   Pool.obj
 0001:0010a210       ?push_back@?$vector@PAVCBucket@CPoolFrameLocal@Memory@@V?$allocator@PAVCBucket@CPoolFrameLocal@Memory@@@stlpmtx_std@@@stlpmtx_std@@QAEXABQAVCBucket@CPoolFrameLocal@Memory@@@Z 3160b210 f i Pool.obj
 0001:0010a260       ?Create@CPoolFrameLocal@Memory@@SAPAV12@AAVCContext@2@I@Z 3160b260 f   Pool.obj
 0001:0010a290       ?CreateBucket@CPoolFrameLocal@Memory@@AAEPAVCBucket@12@XZ 3160b290 f   Pool.obj
 0001:0010a300       ?ReleaseBuckets@CPoolFrameLocal@Memory@@QAEXXZ 3160b300 f   Pool.obj
 0001:0010a3e0       ?Allocate@CPoolFrameLocal@Memory@@UAEPAXI@Z 3160b3e0 f   Pool.obj
 0001:0010a490       ??_ECPoolFrameLocal@Memory@@EAEPAXI@Z 3160b490 f i Pool.obj
 0001:0010a490       ??_GCPoolFrameLocal@Memory@@EAEPAXI@Z 3160b490 f i Pool.obj
 0001:0010a4f0       ?SwSkinTangents@CAttachmentSKIN@@QAEXPAUSSkinningData@@PAUSSoftwareSkinningData@@@Z 3160b4f0 f   _RenderSkinsSW.obj
 0001:0010b2a0       ?Invoke@?$SGenInvokerTSkinAttachmentTangents@VCAttachmentSKIN@@PAUSSkinningData@@PAUSSoftwareSkinningData@@USNullType@Detail@JobManager@@U456@U456@U456@U456@U456@U456@U456@U456@U456@@Detail@JobManager@@SAXPAX@Z 3160c2a0 f i _RenderSkinsSW.obj
 0001:0010b2c0       ?RegisterSoftwareSkinningJobs@CAttachmentSKIN@@SAXXZ 3160c2c0 f   _RenderSkinsSW.obj
 0001:0010b2f0       ??$?0PAUSSkinningData@@PAUSSoftwareSkinningData@@@SGenericJobTSkinAttachmentTangents@Detail@JobManager@@QAE@PAUSSkinningData@@PAUSSoftwareSkinningData@@@Z 3160c2f0 f i _RenderSkinsSW.obj
 0001:0010b3a0       ?InvokeSoftwareSkinning@CAttachmentSKIN@@SAXPAUSSkinningData@@PAUSSoftwareSkinningData@@@Z 3160c3a0 f   _RenderSkinsSW.obj
 0001:0010b428       __purecall                 3160c428 f   MSVCRT:MSVCR100.dll
 0001:0010b42e       __onexit                   3160c42e f   MSVCRT:atonexit.obj
 0001:0010b4cf       _atexit                    3160c4cf f   MSVCRT:atonexit.obj
 0001:0010b4f0       __CIacos                   3160c4f0 f   MSVCRT:MSVCR100.dll
 0001:0010b500       __chkstk                   3160c500 f   MSVCRT:chkstk.obj
 0001:0010b500       __alloca_probe             3160c500     MSVCRT:chkstk.obj
 0001:0010b52c       _memcpy                    3160c52c f   MSVCRT:MSVCR100.dll
 0001:0010b532       _memset                    3160c532 f   MSVCRT:MSVCR100.dll
 0001:0010b540       __ftol2_sse                3160c540 f   MSVCRT:ftol2.obj
 0001:0010b549       __ftol2_pentium4           3160c549 f   MSVCRT:ftol2.obj
 0001:0010b55c       __ftol2_sse_excpt          3160c55c f   MSVCRT:ftol2.obj
 0001:0010b576       __ftol2                    3160c576 f   MSVCRT:ftol2.obj
 0001:0010b5f0       __allshl                   3160c5f0 f   MSVCRT:llshl.obj
 0001:0010b610       ?what@exception@std@@UBEPBDXZ 3160c610 f   MSVCRT:MSVCR100.dll
 0001:0010b616       __CIasin                   3160c616 f   MSVCRT:MSVCR100.dll
 0001:0010b620       __alloca_probe_16          3160c620 f   MSVCRT:alloca16.obj
 0001:0010b636       __alloca_probe_8           3160c636     MSVCRT:alloca16.obj
 0001:0010b64c       _floor                     3160c64c f   MSVCRT:MSVCR100.dll
 0001:0010b652       __CIpow                    3160c652 f   MSVCRT:MSVCR100.dll
 0001:0010b658       __CIfmod                   3160c658 f   MSVCRT:MSVCR100.dll
 0001:0010b660       __aulldiv                  3160c660 f   MSVCRT:ulldiv.obj
 0001:0010b6d0       __allmul                   3160c6d0 f   MSVCRT:llmul.obj
 0001:0010b710       __aullshr                  3160c710 f   MSVCRT:ullshr.obj
 0001:0010b77d       __CRT_INIT@12              3160c77d f   MSVCRT:crtdll.obj
 0001:0010ba9d       __DllMainCRTStartup@12     3160ca9d f   MSVCRT:crtdll.obj
 0001:0010bac0       __unlock                   3160cac0 f   MSVCRT:MSVCR100.dll
 0001:0010bac6       ___dllonexit               3160cac6 f   MSVCRT:MSVCR100.dll
 0001:0010bacc       __lock                     3160cacc f   MSVCRT:MSVCR100.dll
 0001:0010bae0       __SEH_prolog4              3160cae0 f   MSVCRT:sehprolg4.obj
 0001:0010bb25       __SEH_epilog4              3160cb25 f   MSVCRT:sehprolg4.obj
 0001:0010bb39       __except_handler4          3160cb39 f   MSVCRT:chandler4gs.obj
 0001:0010bb5e       ___sse2_available_init     3160cb5e f   MSVCRT:cpu_disp.obj
 0001:0010bb6e       ___clean_type_info_names   3160cb6e f   MSVCRT:tncleanup.obj
 0001:0010bb7a       __RTC_Initialize           3160cb7a f   MSVCRT:_initsect_.obj
 0001:0010bba0       __RTC_Terminate            3160cba0 f   MSVCRT:_initsect_.obj
 0001:0010bbd0       __ValidateImageBase        3160cbd0 f   MSVCRT:pesect.obj
 0001:0010bc10       __FindPESection            3160cc10 f   MSVCRT:pesect.obj
 0001:0010bc60       __IsNonwritableInCurrentImage 3160cc60 f   MSVCRT:pesect.obj
 0001:0010bd1c       __initterm                 3160cd1c f   MSVCRT:MSVCR100.dll
 0001:0010bd22       __initterm_e               3160cd22 f   MSVCRT:MSVCR100.dll
 0001:0010bd28       __amsg_exit                3160cd28 f   MSVCRT:MSVCR100.dll
 0001:0010bd2e       ___CppXcptFilter           3160cd2e f   MSVCRT:MSVCR100.dll
 0001:0010bd34       _DllMain@12                3160cd34 f   MSVCRT:dllmain.obj
 0001:0010bd58       ___security_init_cookie    3160cd58 f   MSVCRT:gs_support.obj
 0001:0010bdf3       @__security_check_cookie@4 3160cdf3 f   MSVCRT:secchk.obj
 0001:0010be02       __except_handler4_common   3160ce02 f   MSVCRT:MSVCR100.dll
 0001:0010be08       ___clean_type_info_names_internal 3160ce08 f   MSVCRT:MSVCR100.dll
 0001:0010be0e       ___report_gsfailure        3160ce0e f   MSVCRT:gs_report.obj
 0001:0010bf14       __crt_debugger_hook        3160cf14 f   MSVCRT:MSVCR100.dll
 0001:0010c4b0       ??__Fs_dummyMemReplay@?1??CryGetIMemReplay@@YAPAUIMemReplay@@XZ@YAXXZ 3160d4b0 f i AnimEventList.obj
 0001:0010c970       ??__Fp@?1??CreateClassInstance@CFactory@CEngineModule_CryAnimation@@UBE?AV?$shared_ptr@UICryUnknown@@@boost@@XZ@YAXXZ 3160d970 f i AnimationBase.obj
 0002:00000000       __imp__InterlockedCompareExchange@12 3160e000     kernel32:KERNEL32.dll
 0002:00000004       __imp__InitializeCriticalSection@4 3160e004     kernel32:KERNEL32.dll
 0002:00000008       __imp__DeleteCriticalSection@4 3160e008     kernel32:KERNEL32.dll
 0002:0000000c       __imp__EnterCriticalSection@4 3160e00c     kernel32:KERNEL32.dll
 0002:00000010       __imp__LeaveCriticalSection@4 3160e010     kernel32:KERNEL32.dll
 0002:00000014       __imp__GetCurrentThreadId@0 3160e014     kernel32:KERNEL32.dll
 0002:00000018       __imp__LoadLibraryA@4      3160e018     kernel32:KERNEL32.dll
 0002:0000001c       __imp__GetProcAddress@8    3160e01c     kernel32:KERNEL32.dll
 0002:00000020       __imp__GetModuleHandleA@4  3160e020     kernel32:KERNEL32.dll
 0002:00000024       __imp__IsDebuggerPresent@0 3160e024     kernel32:KERNEL32.dll
 0002:00000028       __imp__Sleep@4             3160e028     kernel32:KERNEL32.dll
 0002:0000002c       __imp__InterlockedIncrement@4 3160e02c     kernel32:KERNEL32.dll
 0002:00000030       __imp__InterlockedDecrement@4 3160e030     kernel32:KERNEL32.dll
 0002:00000034       __imp__InterlockedExchangeAdd@8 3160e034     kernel32:KERNEL32.dll
 0002:00000038       __imp__UnhandledExceptionFilter@4 3160e038     kernel32:KERNEL32.dll
 0002:0000003c       __imp__GetCurrentProcess@0 3160e03c     kernel32:KERNEL32.dll
 0002:00000040       __imp__TerminateProcess@8  3160e040     kernel32:KERNEL32.dll
 0002:00000044       __imp__GetSystemTimeAsFileTime@4 3160e044     kernel32:KERNEL32.dll
 0002:00000048       __imp__GetCurrentProcessId@0 3160e048     kernel32:KERNEL32.dll
 0002:0000004c       __imp__GetTickCount@0      3160e04c     kernel32:KERNEL32.dll
 0002:00000050       __imp__QueryPerformanceCounter@4 3160e050     kernel32:KERNEL32.dll
 0002:00000054       __imp__DisableThreadLibraryCalls@4 3160e054     kernel32:KERNEL32.dll
 0002:00000058       __imp__IsProcessorFeaturePresent@4 3160e058     kernel32:KERNEL32.dll
 0002:0000005c       __imp__InterlockedExchange@8 3160e05c     kernel32:KERNEL32.dll
 0002:00000060       __imp__DecodePointer@4     3160e060     kernel32:KERNEL32.dll
 0002:00000064       __imp__EncodePointer@4     3160e064     kernel32:KERNEL32.dll
 0002:00000068       __imp__SetUnhandledExceptionFilter@4 3160e068     kernel32:KERNEL32.dll
 0002:0000006c       \177KERNEL32_NULL_THUNK_DATA 3160e06c     kernel32:KERNEL32.dll
 0002:00000070       __imp__fclose              3160e070     MSVCRT:MSVCR100.dll
 0002:00000074       __imp__fprintf             3160e074     MSVCRT:MSVCR100.dll
 0002:00000078       __imp__fopen               3160e078     MSVCRT:MSVCR100.dll
 0002:0000007c       __imp_??0exception@std@@QAE@ABQBDH@Z 3160e07c     MSVCRT:MSVCR100.dll
 0002:00000080       __imp_?what@exception@std@@UBEPBDXZ 3160e080     MSVCRT:MSVCR100.dll
 0002:00000084       __imp_??1exception@std@@UAE@XZ 3160e084     MSVCRT:MSVCR100.dll
 0002:00000088       __imp___CIasin             3160e088     MSVCRT:MSVCR100.dll
 0002:0000008c       __imp__floor               3160e08c     MSVCRT:MSVCR100.dll
 0002:00000090       __imp__atof                3160e090     MSVCRT:MSVCR100.dll
 0002:00000094       __imp__strstr              3160e094     MSVCRT:MSVCR100.dll
 0002:00000098       __imp__strncmp             3160e098     MSVCRT:MSVCR100.dll
 0002:0000009c       __imp__strchr              3160e09c     MSVCRT:MSVCR100.dll
 0002:000000a0       __imp___CIpow              3160e0a0     MSVCRT:MSVCR100.dll
 0002:000000a4       __imp__tolower             3160e0a4     MSVCRT:MSVCR100.dll
 0002:000000a8       __imp___vscprintf          3160e0a8     MSVCRT:MSVCR100.dll
 0002:000000ac       __imp__vsnprintf           3160e0ac     MSVCRT:MSVCR100.dll
 0002:000000ac       __imp___vsnprintf          3160e0ac     MSVCRT:MSVCR100.dll
 0002:000000b0       __imp__ceil                3160e0b0     MSVCRT:MSVCR100.dll
 0002:000000b4       __imp___CIfmod             3160e0b4     MSVCRT:MSVCR100.dll
 0002:000000b8       __imp__strcspn             3160e0b8     MSVCRT:MSVCR100.dll
 0002:000000bc       __imp__strspn              3160e0bc     MSVCRT:MSVCR100.dll
 0002:000000c0       __imp__sscanf              3160e0c0     MSVCRT:MSVCR100.dll
 0002:000000c4       __imp__strtod              3160e0c4     MSVCRT:MSVCR100.dll
 0002:000000c8       __imp__strncpy             3160e0c8     MSVCRT:MSVCR100.dll
 0002:000000cc       __imp__strtok              3160e0cc     MSVCRT:MSVCR100.dll
 0002:000000d0       __imp__fread               3160e0d0     MSVCRT:MSVCR100.dll
 0002:000000d4       __imp__ftell               3160e0d4     MSVCRT:MSVCR100.dll
 0002:000000d8       __imp__fseek               3160e0d8     MSVCRT:MSVCR100.dll
 0002:000000dc       __imp__strrchr             3160e0dc     MSVCRT:MSVCR100.dll
 0002:000000e0       __imp___set_invalid_parameter_handler 3160e0e0     MSVCRT:MSVCR100.dll
 0002:000000e4       __imp___set_purecall_handler 3160e0e4     MSVCRT:MSVCR100.dll
 0002:000000e8       __imp__atoi                3160e0e8     MSVCRT:MSVCR100.dll
 0002:000000ec       __imp___unlock             3160e0ec     MSVCRT:MSVCR100.dll
 0002:000000f0       __imp____dllonexit         3160e0f0     MSVCRT:MSVCR100.dll
 0002:000000f4       __imp___lock               3160e0f4     MSVCRT:MSVCR100.dll
 0002:000000f8       __imp___onexit             3160e0f8     MSVCRT:MSVCR100.dll
 0002:000000fc       __imp__vsnprintf_s         3160e0fc     MSVCRT:MSVCR100.dll
 0002:000000fc       __imp___vsnprintf_s        3160e0fc     MSVCRT:MSVCR100.dll
 0002:00000100       __imp___malloc_crt         3160e100     MSVCRT:MSVCR100.dll
 0002:00000104       __imp__free                3160e104     MSVCRT:MSVCR100.dll
 0002:00000108       __imp___encoded_null       3160e108     MSVCRT:MSVCR100.dll
 0002:0000010c       __imp___initterm           3160e10c     MSVCRT:MSVCR100.dll
 0002:00000110       __imp___initterm_e         3160e110     MSVCRT:MSVCR100.dll
 0002:00000114       __imp___amsg_exit          3160e114     MSVCRT:MSVCR100.dll
 0002:00000118       __imp____CppXcptFilter     3160e118     MSVCRT:MSVCR100.dll
 0002:0000011c       __imp___except_handler4_common 3160e11c     MSVCRT:MSVCR100.dll
 0002:00000120       __imp____clean_type_info_names_internal 3160e120     MSVCRT:MSVCR100.dll
 0002:00000124       __imp___crt_debugger_hook  3160e124     MSVCRT:MSVCR100.dll
 0002:00000128       __imp__sprintf             3160e128     MSVCRT:MSVCR100.dll
 0002:0000012c       __imp__exit                3160e12c     MSVCRT:MSVCR100.dll
 0002:00000130       __imp__puts                3160e130     MSVCRT:MSVCR100.dll
 0002:00000134       __imp__abort               3160e134     MSVCRT:MSVCR100.dll
 0002:00000138       __imp__memmove             3160e138     MSVCRT:MSVCR100.dll
 0002:0000013c       __imp__memset              3160e13c     MSVCRT:MSVCR100.dll
 0002:00000140       __imp__memcpy              3160e140     MSVCRT:MSVCR100.dll
 0002:00000144       __imp___CIacos             3160e144     MSVCRT:MSVCR100.dll
 0002:00000148       __imp___purecall           3160e148     MSVCRT:MSVCR100.dll
 0002:0000014c       __imp__strcmpi             3160e14c     MSVCRT:MSVCR100.dll
 0002:0000014c       __imp__stricmp             3160e14c     MSVCRT:MSVCR100.dll
 0002:0000014c       __imp___stricmp            3160e14c     MSVCRT:MSVCR100.dll
 0002:00000150       __imp__strnicmp            3160e150     MSVCRT:MSVCR100.dll
 0002:00000150       __imp___strnicmp           3160e150     MSVCRT:MSVCR100.dll
 0002:00000154       __imp__isdigit             3160e154     MSVCRT:MSVCR100.dll
 0002:00000158       \177MSVCR100_NULL_THUNK_DATA 3160e158     MSVCRT:MSVCR100.dll
 0002:0000015c       __imp__MessageBoxA@16      3160e15c     user32:USER32.dll
 0002:00000160       \177USER32_NULL_THUNK_DATA 3160e160     user32:USER32.dll
 0002:00000164       ___xc_a                    3160e164     MSVCRT:cinitexe.obj
 0002:000001d4       ___xc_z                    3160e1d4     MSVCRT:cinitexe.obj
 0002:000001d8       ___xi_a                    3160e1d8     MSVCRT:cinitexe.obj
 0002:000001e4       ___xi_z                    3160e1e4     MSVCRT:cinitexe.obj
 0002:00000210       ??_7IMemReplay@@6B@        3160e210     AnimEventList.obj
 0002:000002a8       ??_7CDummyMemReplay@@6B@   3160e2a8     AnimEventList.obj
 0002:00000340       ??_7CAnimEventList@@6B@    3160e340     AnimEventList.obj
 0002:00000360       __real@3f000000            3160e360     Attachment.obj
 0002:00000364       __real@3fc00000            3160e364     Attachment.obj
 0002:00000368       __real@bf800000            3160e368     Attachment.obj
 0002:0000036c       __real@00800000            3160e36c     Attachment.obj
 0002:00000370       __real@42652ee1            3160e370     Attachment.obj
 0002:00000374       ??_C@_02DKCKIIND@?$CFs?$AA@ 3160e374     Attachment.obj
 0002:00000378       __real@46fffe00            3160e378     Attachment.obj
 0002:0000037c       __real@38000100            3160e37c     Attachment.obj
 0002:00000380       ??_7IAttachment@@6B@       3160e380     Attachment.obj
 0002:0000040c       ??_7IAttachmentSkin@@6B@   3160e40c     Attachment.obj
 0002:00000430       __mask@@NegFloat@          3160e430     Attachment.obj
 0002:00000440       ??_C@_0LJ@MJDPKDNI@AttachObjectToBone?5is?5called?5for@ 3160e440     Attachment.obj
 0002:000004fc       __real@1e3ce508            3160e4fc     Attachment.obj
 0002:00000500       __real@40000000            3160e500     Attachment.obj
 0002:00000504       __real@bf000000            3160e504     Attachment.obj
 0002:00000508       __real@3f4f5c28            3160e508     Attachment.obj
 0002:0000050c       __real@38d1b717            3160e50c     Attachment.obj
 0002:00000510       ??_C@_0P@OFCFADAK@HideInMainPass?$AA@ 3160e510     Attachment.obj
 0002:00000520       ??_C@_0BA@KIHOGAB@CAttachmentSKIN?$AA@ 3160e520     Attachment.obj
 0002:00000530       __real@3e4ccccd            3160e530     Attachment.obj
 0002:00000538       __real@3f1a36e2eb1c432d    3160e538     Attachment.obj
 0002:00000540       __real@3c8efa35            3160e540     Attachment.obj
 0002:00000544       ??_C@_0CI@POBBGDGM@vertex?5stream?5declarations?5have?5@ 3160e544     Attachment.obj
 0002:0000056c       ??_C@_09EDIHJNKH@Character?$AA@ 3160e56c     Attachment.obj
 0002:00000578       ??_C@_0BG@KLDDMFMG@cloned?5for?5swskinning?$AA@ 3160e578     Attachment.obj
 0002:00000590       __real@41800000            3160e590     Attachment.obj
 0002:00000594       ??_C@_0BA@HAKOGMIL@SW?9Skinning?3?5?$CFs?$AA@ 3160e594     Attachment.obj
 0002:000005a4       __real@3fa66666            3160e5a4     Attachment.obj
 0002:000005a8       __real@3cf5c28f            3160e5a8     Attachment.obj
 0002:000005ac       __real@3d23d70a            3160e5ac     Attachment.obj
 0002:000005b0       __real@3d4ccccd            3160e5b0     Attachment.obj
 0002:000005b4       __real@40490fdb            3160e5b4     Attachment.obj
 0002:000005b8       __real@3c23d70a            3160e5b8     Attachment.obj
 0002:000005bc       __real@c0490fdb            3160e5bc     Attachment.obj
 0002:000005c0       __real@c11cf5c3            3160e5c0     Attachment.obj
 0002:000005c4       __real@00000000            3160e5c4     Attachment.obj
 0002:000005c8       __real@3ba3d70a            3160e5c8     Attachment.obj
 0002:000005cc       __real@3ca3d70a            3160e5cc     Attachment.obj
 0002:000005d0       __real@bcf5c28f            3160e5d0     Attachment.obj
 0002:000005d4       __real@bca3d70a            3160e5d4     Attachment.obj
 0002:000005d8       __real@3eaaaaab            3160e5d8     Attachment.obj
 0002:000005e0       ??_7CAttachmentSKIN@@6BIAttachment@@@ 3160e5e0     Attachment.obj
 0002:0000066c       ??_7CAttachmentSKIN@@6BIAttachmentSkin@@@ 3160e66c     Attachment.obj
 0002:0000068c       ??_C@_0BD@HKEJKAJE@?$CF03d?5JointName?3?5?$CFs?$AA@ 3160e68c     Attachment.obj
 0002:000006a0       ??_C@_0BK@BIGEPFME@SLAVE?5?5SKELETON?3?5path?3?5?$CFs?$AA@ 3160e6a0     Attachment.obj
 0002:000006bc       ??_C@_0BK@CNDDAMJA@MASTER?5SKELETON?3?5path?3?5?$CFs?$AA@ 3160e6bc     Attachment.obj
 0002:000006d8       ??_C@_0FB@JGGJBAML@Bone?9names?5of?5SLAVE?9skeleton?5don@ 3160e6d8     Attachment.obj
 0002:00000730       ??_C@_0FB@OCMIBIFK@SLAVE?9skeleton?5needs?5to?5have?5les@ 3160e730     Attachment.obj
 0002:00000788       ??_C@_0HF@NPAHMHBP@CryAnimation?3?5if?5you?5create?5the?5@ 3160e788     Attachment.obj
 0002:00000800       ??_7IDefragAllocatorPolicy@@6B@ 3160e800     ControllerDefragHeap.obj
 0002:00000814       ??_C@_0P@PCJPAHLM@out?5of?5memory?6?$AA@ 3160e814     ControllerDefragHeap.obj
 0002:00000824       ??_C@_06NBFPPGEG@vector?$AA@ 3160e824     ControllerDefragHeap.obj
 0002:0000082c       ??_7CControllerDefragHeap@@6B@ 3160e82c     ControllerDefragHeap.obj
 0002:00000840       ??_C@_00CNPNBAHC@?$AA@     3160e840     ControllerDefragHeap.obj
 0002:00000844       ??_C@_0BB@OMBAPGD@Anim?5Defrag?5Heap?$AA@ 3160e844     ControllerDefragHeap.obj
 0002:00000858       ??_C@_0BO@ECPGPOHM@CControllerDefragHeap?3?3Update?$AA@ 3160e858     ControllerDefragHeap.obj
 0002:00000878       __real@0000000000000000    3160e878     DrawHelper.obj
 0002:00000880       __real@3ff0000000000000    3160e880     DrawHelper.obj
 0002:00000888       __real@3f666666            3160e888     DrawHelper.obj
 0002:0000088c       __real@3f400000            3160e88c     DrawHelper.obj
 0002:00000890       __real@4000000000000000    3160e890     DrawHelper.obj
 0002:00000898       __real@3f7d70a4            3160e898     DrawHelper.obj
 0002:0000089c       __real@3e19999a            3160e89c     DrawHelper.obj
 0002:000008a0       __real@3c1374bc            3160e8a0     DrawHelper.obj
 0002:000008a8       __real@3f8eb851eb851eb8    3160e8a8     DrawHelper.obj
 0002:000008b0       __real@3fe0000000000000    3160e8b0     DrawHelper.obj
 0002:000008b8       __real@3f947ae147ae147b    3160e8b8     DrawHelper.obj
 0002:000008c0       __real@3d99999a            3160e8c0     DrawHelper.obj
 0002:000008c4       __real@3e800000            3160e8c4     DrawHelper.obj
 0002:000008cc       ??_C@_0CI@IOKCCNHB@Deleting?5Reference?5Counted?5Objec@ 3160e8cc     LoaderSKIN.obj
 0002:000008f4       __real@d8635fa9            3160e8f4     LoaderSKIN.obj
 0002:000008f8       __real@58635fa9            3160e8f8     LoaderSKIN.obj
 0002:00000900       __real@3fefffffff7ffe00    3160e900     LoaderSKIN.obj
 0002:00000908       ??_C@_0EL@JEKIGBJA@Character?5LOD?5mismatch?4?5The?5bone@ 3160e908     LoaderSKIN.obj
 0002:00000954       ??_C@_0BD@GAJPFAIO@Hierarchy?5of?5LOD?$CFi?$AA@ 3160e954     LoaderSKIN.obj
 0002:00000968       ??_C@_0ED@EMLDLHGL@?9?9?9?9?9?9?9?9?9?9?9?9?9?9?9?9?9?9?9?9?9?9?9?9?9?9?9?9?9?9?9?9@ 3160e968     LoaderSKIN.obj
 0002:000009ac       ??_C@_0BD@JKBIHFBO@Joint?5ID?5?3?5?$CF02d?5?$CFs?$AA@ 3160e9ac     LoaderSKIN.obj
 0002:000009c0       ??_C@_0BC@CMAFGEHH@Hierarchy?5of?5LOD0?$AA@ 3160e9c0     LoaderSKIN.obj
 0002:000009d8       ??_C@_0EC@CDOMHHGC@Failed?5to?5Load?5Character?0?5Differ@ 3160e9d8     LoaderSKIN.obj
 0002:00000a1c       __real@3dcccccd            3160ea1c     LoaderSKIN.obj
 0002:00000a20       ??_C@_02GMHACPFF@?$CFu?$AA@ 3160ea20     LoaderSKIN.obj
 0002:00000a24       ??_C@_04NHPAFEHJ@skin?$AA@ 3160ea24     LoaderSKIN.obj
 0002:00000a2c       ??_C@_01LFCBOECM@?4?$AA@   3160ea2c     LoaderSKIN.obj
 0002:00000a30       ??_C@_04LAHEDKPN@_lod?$AA@ 3160ea30     LoaderSKIN.obj
 0002:00000a38       ??_C@_0EG@EBKKPPLH@Failed?5to?5Load?5Character?5file?4?5S@ 3160ea38     LoaderSKIN.obj
 0002:00000a80       ??_C@_0DB@FJJGDDBE@Failed?5to?5Load?5Character?5file?4?5G@ 3160ea80     LoaderSKIN.obj
 0002:00000ab4       ??_C@_0BM@PPPNKEGO@Invalid?5vertex?5?$CFd?5in?5lod?5?$CFd?$AA@ 3160eab4     LoaderSKIN.obj
 0002:00000ad0       ??_7CMorphTarget@@6B@      3160ead0     LoaderSKIN.obj
 0002:00000adc       ??_C@_0CB@NMCAMOME@Bound?5box?5is?5too?5small?5in?5lod?5?$CFd@ 3160eadc     LoaderSKIN.obj
 0002:00000b00       ??_C@_0CF@IBDHFABJ@Vertex?5extension?5z?5is?5zero?5in?5lo@ 3160eb00     LoaderSKIN.obj
 0002:00000b28       ??_C@_0CF@COJOBNND@Vertex?5extension?5y?5is?5zero?5in?5lo@ 3160eb28     LoaderSKIN.obj
 0002:00000b50       ??_C@_0CF@ELPJCGJF@Vertex?5extension?5x?5is?5zero?5in?5lo@ 3160eb50     LoaderSKIN.obj
 0002:00000b78       ??_C@_0CE@KGCDEIAK@Vertex?5id?50x?$CFx?5is?5too?5big?5in?5lod@ 3160eb78     LoaderSKIN.obj
 0002:00000b9c       ??_C@_0CB@EIMOFNGE@arrExtMorph?$FL?$FN?5is?5empty?5in?5lod?5?$CFd@ 3160eb9c     LoaderSKIN.obj
 0002:00000bc0       __real@3a83126f            3160ebc0     LoaderSKIN.obj
 0002:00000bc4       __real@41700000            3160ebc4     LoaderSKIN.obj
 0002:00000bc8       __real@437f0000            3160ebc8     LoaderSKIN.obj
 0002:00000bcc       __real@c7c34f80            3160ebcc     LoaderSKIN.obj
 0002:00000bd0       __real@47c34f80            3160ebd0     LoaderSKIN.obj
 0002:00000bd4       ??_C@_0CN@IPOFNMHK@Bone?5?$CFd?3?5B2W?5is?5not?5orthonormal?5@ 3160ebd4     LoaderSKIN.obj
 0002:00000c04       ??_C@_0BF@JHCFNCDB@Model?5has?5no?5Joints?4?$AA@ 3160ec04     LoaderSKIN.obj
 0002:00000c1c       ??_C@_0CP@JEJKDKLN@Too?5many?5Joints?5in?5model?4?5Curren@ 3160ec1c     LoaderSKIN.obj
 0002:00000c4c       ??_C@_0BP@OOOCOAFP@Duplicated?5morph?5mask?5found?5?$CFs?$AA@ 3160ec4c     LoaderSKIN.obj
 0002:00000c6c       ??_C@_0BO@KMGPEDAO@Base?5skinned?5model?5is?5missing?$AA@ 3160ec6c     LoaderSKIN.obj
 0002:00000c8c       ??_C@_0CK@FPIIFKJK@The?5Chunk?9Loader?5failed?5to?5load?5@ 3160ec8c     LoaderSKIN.obj
 0002:00000cb8       ??_C@_0CI@LFMLLEBF@Failed?5to?5create?5render?5mesh?5for@ 3160ecb8     LoaderSKIN.obj
 0002:00000ce0       ??_C@_0BM@JOPKNICB@No?5internal?5faces?5in?5lod?5?$CFd?$AA@ 3160ece0     LoaderSKIN.obj
 0002:00000cfc       ??_C@_0BG@JBIGAFMF@No?5material?5in?5lod?5?$CFd?$AA@ 3160ecfc     LoaderSKIN.obj
 0002:00000d14       ??_C@_0BP@CMMDHOGJ@Ext2Int?5map?5is?5empty?5in?5lod?5?$CFd?$AA@ 3160ed14     LoaderSKIN.obj
 0002:00000d34       ??_C@_0CD@BBJOEHHB@Skinning?5info?5is?5missing?5in?5lod?5@ 3160ed34     LoaderSKIN.obj
 0002:00000d58       ??_C@_0FF@BMNHAGLP@external?5and?5internal?5face?9amoun@ 3160ed58     LoaderSKIN.obj
 0002:00000db0       ??_C@_0N@EGPCGIEE@e_CharLodMin?$AA@ 3160edb0     LoaderSKIN.obj
 0002:00000dc0       ??_C@_0N@MAGOOHJD@e_charLodMin?$AA@ 3160edc0     LoaderSKIN.obj
 0002:00000dd0       ??_C@_0O@NMCPHDFF@consoles_lod0?$AA@ 3160edd0     LoaderSKIN.obj
 0002:00000de0       ??_C@_0BG@EFLJKDCI@ca_UseAssetDefinedLod?$AA@ 3160ede0     LoaderSKIN.obj
 0002:00000df8       ??_C@_0BJ@BIICHPJO@Wrong?5character?5filename?$AA@ 3160edf8     LoaderSKIN.obj
 0002:00000e14       ??_C@_03KMOFPJOC@chr?$AA@  3160ee14     LoaderSKIN.obj
 0002:00000e18       ??_C@_0BB@CGHIGGGM@LoadCharacter?5?$CFs?$AA@ 3160ee18     LoaderSKIN.obj
 0002:00000e2c       ??_C@_0BK@HNKMOAFK@CryCHRLoader?3?3LoadNewSKIN?$AA@ 3160ee2c     LoaderSKIN.obj
 0002:00000e4c       __real@3727c5ac            3160ee4c     ModelMesh_DebugPC.obj
 0002:00000e4c       ?minPosArea@?1???$ComputeTexMappingAreas@U?$Vec3_tpl@M@@USMeshTexCoord@@@CMeshHelpers@@SA_NIPBGIPBU?$Vec3_tpl@M@@IPBUSMeshTexCoord@@IAAM3AAPBD@Z@4MB 3160ee4c     LoaderCGA.obj
 0002:00000e50       __real@47c35000            3160ee50     ModelMesh_DebugPC.obj
 0002:00000e54       ??_C@_04GEFJINEE@?$CF?42f?$AA@ 3160ee54     ModelMesh_DebugPC.obj
 0002:00000e5c       ??_C@_08GDAMKODC@?$CFd?0?$CFd?0?$CFd?$AA@ 3160ee5c     ModelMesh_DebugPC.obj
 0002:00000e68       ??_C@_0M@MLCONGPP@?$CFd?0?$CFd?0?$CFd?0?$CFd?$AA@ 3160ee68     ModelMesh_DebugPC.obj
 0002:00000e74       ??_C@_05LCKIIOJE@?$CFd?1?$CFd?$AA@ 3160ee74     ModelMesh_DebugPC.obj
 0002:00000e7c       __real@42f00000            3160ee7c     ModelMesh_DebugPC.obj
 0002:00000e80       __real@40c90fdb            3160ee80     ModelMesh_DebugPC.obj
 0002:00000e84       ??_C@_02DPKJAMEF@?$CFd?$AA@ 3160ee84     ModelMesh_DebugPC.obj
 0002:00000e88       ??_C@_0BB@CDDPHBIK@?$CFs?6?$CFd?5LOD?$CI?$CFi?2?$CFi?$CJ?$AA@ 3160ee88     ModelMesh_DebugPC.obj
 0002:00000e9c       ??_C@_02PCIJFNDE@?$AN?6?$AA@ 3160ee9c     ModelMesh_DebugPC.obj
 0002:00000ea0       ??_C@_03ELIABIOC@w?$CLb?$AA@ 3160eea0     ModelMesh_DebugPC.obj
 0002:00000ea4       __real@3b808081            3160eea4     ModelMesh_DebugPC.obj
 0002:00000ea8       ??_C@_0BD@KNEHJKOE@SoftwareSkinningDQ?$AA@ 3160eea8     ModelMesh_DebugPC.obj
 0002:00000ebc       ??_C@_0BP@KJMNBCEI@CModelMesh?3?3SoftwareSkinningDQ?$AA@ 3160eebc     ModelMesh_DebugPC.obj
 0002:00000ee0       ??_C@_0L@JGFNFNNF@CModelMesh?$AA@ 3160eee0     ModelSkin.obj
 0002:00000eec       ??_7CSkin@@6B@             3160eeec     ModelSkin.obj
 0002:00000f28       ??_C@_0BP@NOKONOFF@?$CBMORPH?5TARGET?5ID?5OUT?5OF?5RANGE?$CB?$AA@ 3160ef28     ModelSkin.obj
 0002:00000f48       ??_C@_0BC@LGKPNEPG@CSkin?5Release?3?5?$CFs?$AA@ 3160ef48     ModelSkin.obj
 0002:00000f60       ??_C@_0FJ@LKDGMGOG@The?5model?5?8?$CFs?8?5still?5has?5?$CFd?5skin@ 3160ef60     ModelSkin.obj
 0002:00000fc8       ??_C@_08IFJOJHOO@e_Clouds?$AA@ 3160efc8     ParametricSampler.obj
 0002:00000fd4       ??_C@_07EFDJIHNI@e_Roads?$AA@ 3160efd4     ParametricSampler.obj
 0002:00000fdc       ??_C@_0P@GLJFAGLA@e_WaterVolumes?$AA@ 3160efdc     ParametricSampler.obj
 0002:00000fec       ??_C@_0N@DNCIPFKM@e_WaterWaves?$AA@ 3160efec     ParametricSampler.obj
 0002:00000ffc       ??_C@_08HDKOIENJ@e_Decals?$AA@ 3160effc     ParametricSampler.obj
 0002:00001008       ??_C@_0M@BBFEECFK@e_Particles?$AA@ 3160f008     ParametricSampler.obj
 0002:00001014       ??_C@_0N@BCKEBKIL@e_WaterOcean?$AA@ 3160f014     ParametricSampler.obj
 0002:00001024       ??_C@_09HEKIHBOB@e_Terrain?$AA@ 3160f024     ParametricSampler.obj
 0002:00001030       ??_C@_0L@JLCOCKLP@e_Entities?$AA@ 3160f030     ParametricSampler.obj
 0002:0000103c       ??_C@_0N@IDHCJDNJ@e_Vegetation?$AA@ 3160f03c     ParametricSampler.obj
 0002:0000104c       ??_C@_09MHBOCIPH@e_Brushes?$AA@ 3160f04c     ParametricSampler.obj
 0002:00001058       ??_C@_09HMFDJOHK@e_Shadows?$AA@ 3160f058     ParametricSampler.obj
 0002:00001064       ??_C@_08OEHLIOJG@e_VoxTer?$AA@ 3160f064     ParametricSampler.obj
 0002:00001070       ??_C@_07DPCBLJHC@e_Voxel?$AA@ 3160f070     ParametricSampler.obj
 0002:00001078       ??_C@_0BC@BEKKKHMP@e_DefaultMaterial?$AA@ 3160f078     ParametricSampler.obj
 0002:0000108c       __real@3f333333            3160f08c     ParametricSampler.obj
 0002:00001090       __real@3f4ccccd            3160f090     ParametricSampler.obj
 0002:00001094       __real@3c888889            3160f094     ParametricSampler.obj
 0002:00001098       ??_C@_0P@IINHJLIF@e_CameraFreeze?$AA@ 3160f098     ParametricSampler.obj
 0002:000010a8       __real@461c3c00            3160f0a8     ParametricSampler.obj
 0002:000010ac       __real@42200000            3160f0ac     ParametricSampler.obj
 0002:000010b0       ??_C@_0BC@BOLHFEBM@Inside?5Block1?3?5?$CFd?$AA@ 3160f0b0     ParametricSampler.obj
 0002:000010c4       __real@40800000            3160f0c4     ParametricSampler.obj
 0002:000010c8       __real@40166666            3160f0c8     ParametricSampler.obj
 0002:000010cc       __real@40600000            3160f0cc     ParametricSampler.obj
 0002:000010d0       ??_C@_0P@ONCKKLGM@InternalPara1D?$AA@ 3160f0d0     ParametricSampler.obj
 0002:000010e0       ??_C@_0BE@PBKONPHH@Not?5an?5Internal?5LMG?$AA@ 3160f0e0     ParametricSampler.obj
 0002:000010f4       ??_C@_0DH@CPEAIGHN@CryAnimation?3?5more?5then?53?5dimens@ 3160f0f4     ParametricSampler.obj
 0002:0000112c       __real@3d8f5c29            3160f12c     ParametricSampler.obj
 0002:00001130       __real@41a00000            3160f130     ParametricSampler.obj
 0002:00001134       ??_C@_09HJKJEFNK@?$CFs?3?5?$CFf?5?$CFd?$AA@ 3160f134     ParametricSampler.obj
 0002:00001140       __real@41f80000            3160f140     ParametricSampler.obj
 0002:00001144       __real@40400000            3160f144     ParametricSampler.obj
 0002:00001148       ??_C@_0BA@KLKAAMJI@invalid?5sum?3?5?$CFf?$AA@ 3160f148     ParametricSampler.obj
 0002:00001158       ??_C@_0BA@PJAEBMKK@Invalid?5Weights?$AA@ 3160f158     ParametricSampler.obj
 0002:00001168       __real@4f800000            3160f168     ParametricSampler.obj
 0002:0000116c       ??_C@_0CG@CCCLNGHK@CryAnimation?3?5nParaID?5not?5initia@ 3160f16c     ParametricSampler.obj
 0002:00001194       __real@41a80000            3160f194     ParametricSampler.obj
 0002:00001198       ??_C@_07MIGDMPIL@mem?3?5?$CFd?$AA@ 3160f198     ParametricSampler.obj
 0002:000011a0       __real@42c80000            3160f1a0     ParametricSampler.obj
 0002:000011a4       __real@c2c80000            3160f1a4     ParametricSampler.obj
 0002:000011a8       __real@41f00000            3160f1a8     ParametricSampler.obj
 0002:000011ac       __real@3d088889            3160f1ac     ParametricSampler.obj
 0002:000011b0       ??_C@_0BH@KPHNFGHL@CryAnimation?3?5negative?$AA@ 3160f1b0     ParametricSampler.obj
 0002:000011c8       ??_C@_0BI@BNNPNGGM@Sum?5of?5weights?5is?5wrong?$AA@ 3160f1c8     ParametricSampler.obj
 0002:000011e0       __real@40a66666            3160f1e0     ParametricSampler.obj
 0002:000011e4       __real@c0a66666            3160f1e4     ParametricSampler.obj
 0002:000011e8       ??_C@_0BH@KFJNBPEB@CryAnimation?3?5?$CFs?3?5?8?$CFs?8?$AA@ 3160f1e8     ParametricSampler.obj
 0002:00001200       ??_7IPlaceholderCharacter@@6B@ 3160f200     PlaceholderCharacter.obj
 0002:00001200       ??_7IPhonemeLibrary@@6B@   3160f200     LipSync.obj
 0002:00001210       ??_7CPlaceholderCharacter@@6B@ 3160f210     PlaceholderCharacter.obj
 0002:00001224       __real@34000000            3160f224     DirectionalBlender.obj
 0002:00001228       __real@3e70a3d7            3160f228     DirectionalBlender.obj
 0002:0000122c       __real@3ef5c28f            3160f22c     DirectionalBlender.obj
 0002:00001230       __real@39000000            3160f230     DirectionalBlender.obj
 0002:00001234       __real@3fc90fdb            3160f234     DirectionalBlender.obj
 0002:00001238       __real@4022f983            3160f238     DirectionalBlender.obj
 0002:0000123c       __real@3e051eb8            3160f23c     DirectionalBlender.obj
 0002:00001240       __real@3da3d70a            3160f240     DirectionalBlender.obj
 0002:00001244       __real@3fb33333            3160f244     DirectionalBlender.obj
 0002:00001248       __real@bfb33333            3160f248     DirectionalBlender.obj
 0002:0000124c       __real@41d00000            3160f24c     DirectionalBlender.obj
 0002:00001250       __real@c0486c04            3160f250     DirectionalBlender.obj
 0002:00001254       __real@40486c04            3160f254     DirectionalBlender.obj
 0002:00001258       __real@3fcccccd            3160f258     DirectionalBlender.obj
 0002:0000125c       __real@bfc90fdb            3160f25c     DirectionalBlender.obj
 0002:00001260       __real@3feff7ced916872b    3160f260     DirectionalBlender.obj
 0002:00001268       __real@3f8ccccd            3160f268     DirectionalBlender.obj
 0002:0000126c       __real@3fc9309f            3160f26c     DirectionalBlender.obj
 0002:00001270       __real@4049203d            3160f270     DirectionalBlender.obj
 0002:00001274       __real@3ec90fdb            3160f274     DirectionalBlender.obj
 0002:00001278       __real@ba83126f            3160f278     DirectionalBlender.obj
 0002:0000127c       __real@41600000            3160f27c     DirectionalBlender.obj
 0002:00001280       __real@3f99999a            3160f280     DirectionalBlender.obj
 0002:00001284       ??_C@_0BD@GFPCDKCE@fAimPoseWeight?3?5?$CFf?$AA@ 3160f284     DirectionalBlender.obj
 0002:00001298       __real@4019999a            3160f298     DirectionalBlender.obj
 0002:0000129c       ??_C@_0BM@HHDJLNNF@final?5polar?3?5?$CFf?5?$CFf?5?5?5wR?3?5?$CFf?$AA@ 3160f29c     DirectionalBlender.obj
 0002:000012b8       __real@41200000            3160f2b8     DirectionalBlender.obj
 0002:000012bc       ??_7ICryUnknown@@6B@       3160f2bc     OperatorQueue.obj
 0002:000012bc       ??_7IJoystickContext@@6B@  3160f2bc     FaceAnimation.obj
 0002:000012d0       ?iid@?1??IID@ICryUnknown@@CAABUCryGUID@@XZ@4U3@B 3160f2d0     OperatorQueue.obj
 0002:000012e0       ?iid@?1??IID@IAnimationPoseModifier@@CAABUCryGUID@@XZ@4U3@B 3160f2e0     OperatorQueue.obj
 0002:000012f0       ?iid@?1??IID@IAnimationOperatorQueue@@CAABUCryGUID@@XZ@4U3@B 3160f2f0     OperatorQueue.obj
 0002:00001300       ??_7ICryFactory@@6B@       3160f300     OperatorQueue.obj
 0002:00001318       ??_7COperatorQueue@@6B@    3160f318     OperatorQueue.obj
 0002:00001350       ??_7CFactory@COperatorQueue@@6B@ 3160f350     OperatorQueue.obj
 0002:00001368       ??_C@_0CE@INMPALAM@AnimationPoseModifier_OperatorQu@ 3160f368     OperatorQueue.obj
 0002:00001390       ?cid@?1??GetClassID@CFactory@COperatorQueue@@UBEABUCryGUID@@XZ@4U4@B 3160f390     OperatorQueue.obj
 0002:000013a0       ??_7bad_alloc@std@@6B@     3160f3a0     OperatorQueue.obj
 0002:000013a8       ??_C@_0P@GHFPNOJB@bad?5allocation?$AA@ 3160f3a8     OperatorQueue.obj
 0002:000013b8       ??_7sp_counted_base@detail@boost@@6B@ 3160f3b8     OperatorQueue.obj
 0002:000013c8       ??_C@_0BN@FOKPCDPC@Boost?5threw?5an?5exception?3?5?$CFs?$AA@ 3160f3c8     OperatorQueue.obj
 0002:000013e8       ??_7?$sp_counted_impl_p@VCFeetPoseRestore@@@detail@boost@@6B@ 3160f3e8     FeetLock.obj
 0002:000013e8       ??_7?$sp_counted_impl_p@VCRecoil@PoseModifier@@@detail@boost@@6B@ 3160f3e8     Recoil.obj
 0002:000013e8       ??_7?$sp_counted_impl_p@VCPoseBlenderAim@@@detail@boost@@6B@ 3160f3e8     PoseBlenderAim.obj
 0002:000013e8       ??_7?$sp_counted_impl_p@VCFeetPoseStore@@@detail@boost@@6B@ 3160f3e8     FeetLock.obj
 0002:000013e8       ??_7?$sp_counted_impl_p@VCEngineModule_CryAnimation@@@detail@boost@@6B@ 3160f3e8     AnimationBase.obj
 0002:000013e8       ??_7?$sp_counted_impl_p@VCGroundAlignment@@@detail@boost@@6B@ 3160f3e8     GroundAlignment.obj
 0002:000013e8       ??_7?$sp_counted_impl_p@VCPoseBlenderLook@@@detail@boost@@6B@ 3160f3e8     PoseBlenderLook.obj
 0002:000013e8       ??_7?$sp_counted_impl_p@VCPoseAlignerChain@@@detail@boost@@6B@ 3160f3e8     PoseAlignerChain.obj
 0002:000013e8       ??_7?$sp_counted_impl_p@VCPoseMatching@@@detail@boost@@6B@ 3160f3e8     PoseMatching.obj
 0002:000013e8       ??_7?$sp_counted_impl_p@VCLimbIk@@@detail@boost@@6B@ 3160f3e8     LimbIk.obj
 0002:000013e8       ??_7?$sp_counted_impl_p@VCOperatorQueue@@@detail@boost@@6B@ 3160f3e8     OperatorQueue.obj
 0002:00001400       ?iid@?1??IID@IAnimationPoseAlignerChain@@CAABUCryGUID@@XZ@4U3@B 3160f400     PoseAlignerChain.obj
 0002:00001410       __real@322bcc77            3160f410     PoseAlignerChain.obj
 0002:00001414       __real@3f19999a            3160f414     PoseAlignerChain.obj
 0002:00001418       __real@3fd9999a            3160f418     PoseAlignerChain.obj
 0002:0000141c       ??_7CPoseAlignerChain@@6B@ 3160f41c     PoseAlignerChain.obj
 0002:00001444       __real@3e000000            3160f444     PoseAlignerChain.obj
 0002:00001448       __real@c0000000            3160f448     PoseAlignerChain.obj
 0002:0000144c       ??_C@_0BH@ILEOFMKI@a_poseAlignerDebugDraw?$AA@ 3160f44c     PoseAlignerChain.obj
 0002:00001464       ??_7CFactory@CPoseAlignerChain@@6B@ 3160f464     PoseAlignerChain.obj
 0002:0000147c       ??_C@_0CH@JHIPBLIP@AnimationPoseModifier_PoseAligne@ 3160f47c     PoseAlignerChain.obj
 0002:000014a8       ?cid@?1??GetClassID@CFactory@CPoseAlignerChain@@UBEABUCryGUID@@XZ@4U4@B 3160f4a8     PoseAlignerChain.obj
 0002:000014c8       ?iid@?1??IID@IAnimationPoseMatching@@CAABUCryGUID@@XZ@4U3@B 3160f4c8     PoseMatching.obj
 0002:000014d8       ??_7CPoseMatching@@6B@     3160f4d8     PoseMatching.obj
 0002:00001500       __real@501502f9            3160f500     PoseMatching.obj
 0002:00001504       ??_7CFactory@CPoseMatching@@6B@ 3160f504     PoseMatching.obj
 0002:0000151c       ??_C@_0CD@KLIGADKD@AnimationPoseModifier_PoseMatchi@ 3160f51c     PoseMatching.obj
 0002:00001540       ?cid@?1??GetClassID@CFactory@CPoseMatching@@UBEABUCryGUID@@XZ@4U4@B 3160f540     PoseMatching.obj
 0002:00001554       ??_C@_0CC@CNAFILPC@CryAnimation?3?5VEG?9ID?5out?5of?5rang@ 3160f554     SkeletonAnim_Locator.obj
 0002:00001578       ??_C@_0BF@PLHLAKMB@CryAnimation?3?5no?5VEG?$AA@ 3160f578     SkeletonAnim_Locator.obj
 0002:00001590       ??_C@_0CC@CBGNOEAD@No?5Controllers?5found?5in?5Asset?3?5?$CF@ 3160f590     SkeletonAnim_Locator.obj
 0002:000015b4       ??_C@_0DA@KHBKMFJG@CryAnimation?3?5No?5Controllers?5fou@ 3160f5b4     SkeletonAnim_Locator.obj
 0002:000015e8       ??_C@_0EH@DPPJCECM@CryAnimation?3?5reverse?5playback?5o@ 3160f5e8     SkeletonAnim_Locator.obj
 0002:00001630       __real@40133333            3160f630     SkeletonAnim_Locator.obj
 0002:00001634       ??_C@_0DL@MFPHNIBP@fMoveSpeed?3?5?$CFf?5?5fTurnSpeed?3?5?$CFf?5?5@ 3160f634     SkeletonAnim_Locator.obj
 0002:00001670       ?minTexArea@?1???$ComputeTexMappingAreas@U?$Vec3_tpl@M@@USMeshTexCoord@@@CMeshHelpers@@SA_NIPBGIPBU?$Vec3_tpl@M@@IPBUSMeshTexCoord@@IAAM3AAPBD@Z@4MB 3160f670     LoaderCGA.obj
 0002:00001670       __real@33d6bf95            3160f670     SkeletonAnim_Locator.obj
 0002:00001674       __real@80000000            3160f674     SkeletonAnim_Locator.obj
 0002:00001688       ??_7SBatchUpdateValidator@@6B@ 3160f688     SkeletonPhysics.obj
 0002:00001694       __real@d01502f9            3160f694     SkeletonPhysics.obj
 0002:00001698       __real@3e99999a            3160f698     SkeletonPhysics.obj
 0002:0000169c       __real@42100000            3160f69c     SkeletonPhysics.obj
 0002:000016a0       ??_C@_04NHHOEEHI@Calf?$AA@ 3160f6a0     SkeletonPhysics.obj
 0002:000016a8       ??_C@_05NGPCKMLC@Thigh?$AA@ 3160f6a8     SkeletonPhysics.obj
 0002:000016b0       ??_C@_05CBBIAFIL@Spine?$AA@ 3160f6b0     SkeletonPhysics.obj
 0002:000016b8       ??_C@_04BFCCBDOP@Head?$AA@ 3160f6b8     SkeletonPhysics.obj
 0002:000016c0       ??_C@_06EIPNOIEJ@Pelvis?$AA@ 3160f6c0     SkeletonPhysics.obj
 0002:000016c8       ??_C@_07BLFFLKLF@Forearm?$AA@ 3160f6c8     SkeletonPhysics.obj
 0002:000016d0       ??_C@_04IJEANHEE@mass?$AA@ 3160f6d0     SkeletonPhysics.obj
 0002:000016d8       __real@40a00000            3160f6d8     SkeletonPhysics.obj
 0002:000016dc       __real@3eb33333            3160f6dc     SkeletonPhysics.obj
 0002:000016e0       ??_C@_06LMBGEFBP@Spine1?$AA@ 3160f6e0     SkeletonPhysics.obj
 0002:000016e8       ??_C@_04JBBMMDIF@Hand?$AA@ 3160f6e8     SkeletonPhysics.obj
 0002:000016f0       ??_C@_08BOKOBFBJ@UpperArm?$AA@ 3160f6f0     SkeletonPhysics.obj
 0002:000016fc       ??_C@_0CN@BCDMNCJF@CSkeletonPhysics?3?3SynchronizeWit@ 3160f6fc     SkeletonPhysics.obj
 0002:0000172c       ??_C@_0BN@NGOFJCFL@rope_stiffness_controller_?$CFd?$AA@ 3160f72c     SkeletonPhysics.obj
 0002:0000174c       ??_C@_0M@KOHNAGAB@attach_?$CF?4?$CKs?$AA@ 3160f74c     SkeletonPhysics.obj
 0002:00001758       __real@44480000            3160f758     SkeletonPhysics.obj
 0002:0000175c       ??_C@_04GKOOIABA@loop?$AA@ 3160f75c     SkeletonPhysics.obj
 0002:00001764       ??_C@_04JFPBKLKK@rope?$AA@ 3160f764     SkeletonPhysics.obj
 0002:0000176c       __real@c2b40000            3160f76c     SkeletonPhysics.obj
 0002:00001770       __real@43340000            3160f770     SkeletonPhysics.obj
 0002:00001774       ??_C@_0CO@KCAIEJIE@CSkeletonPhysics?3?3Physics_Synchr@ 3160f774     SkeletonPhysics.obj
 0002:000017a4       __real@44610000            3160f7a4     SkeletonPhysics.obj
 0002:000017a8       ??_C@_0CJ@FPNKAHEM@CSkeletonPhysics?3?3SynchronizeWit@ 3160f7a8     SkeletonPhysics.obj
 0002:000017d4       __real@49742400            3160f7d4     SkeletonPhysics.obj
 0002:000017d8       __real@c0c00000            3160f7d8     SkeletonPhysics.obj
 0002:000017f0       ??_C@_0BH@MKEGFDBH@GetStatus?$CI?$CJ?5returned?50?$AA@ 3160f7f0     SkeletonPhysics_SPU.obj
 0002:00001808       ??_C@_0DL@KNAAJKGE@CSkeletonPhysics?3?3SPU_Physics_Sy@ 3160f808     SkeletonPhysics_SPU.obj
 0002:00001844       ??_C@_0DE@DMBPAOJG@CSkeletonPhysics?3?3SPU_Physics_Sy@ 3160f844     SkeletonPhysics_SPU.obj
 0002:00001878       ??_C@_0CO@IEFCAFMK@CSkeletonPhysics?3?3SPU_Physics_Sy@ 3160f878     SkeletonPhysics_SPU.obj
 0002:000018b0       ??_C@_0EL@MHNLDCI@Too?5many?5?$CI?5?$DO?52?5?$CJ?5animations?5in?5t@ 3160f8b0     TransitionQueue.obj
 0002:000018fc       ??_C@_07NBCGADJA@Unknown?$AA@ 3160f8fc     TransitionQueue.obj
 0002:00001904       ??_7CVertexAnimation@@6B@  3160f904     VertexAnimation.obj
 0002:00001914       ??_C@_0DI@LJBCAOEA@CCharInstance?3?3RenderCGA?3?5object@ 3160f914     _Render.obj
 0002:00001950       ??_C@_0EA@HOEPBFKF@CryAnimation?3?5CGA?5should?5not?5hav@ 3160f950     _Render.obj
 0002:00001990       ??_C@_0BP@EKHBKMOH@CCharInstance?3?3GetSkinningData?$AA@ 3160f990     _Render.obj
 0002:000019b0       ??_C@_0M@CCHJNHEL@e_DebugDraw?$AA@ 3160f9b0     _Render.obj
 0002:000019bc       ??_C@_0BO@HOAMFGDG@model?5?8?$CFs?8?5has?5no?5render?5mesh?$AA@ 3160f9bc     _Render.obj
 0002:000019dc       __real@3d6147ae            3160f9dc     _Render.obj
 0002:000019e0       ??_C@_08EALJILLJ@e_LodMin?$AA@ 3160f9e0     _Render.obj
 0002:000019f0       ??_C@_0BO@FHEBEPB@CryAnimation?3?5pMaster?5is?5zero?$AA@ 3160f9f0     _RenderSkins.obj
 0002:00001a10       ??_C@_0CB@BAMEGJJA@CAttachmentSKIN?3?3GetSkinningData@ 3160fa10     _RenderSkins.obj
 0002:00001a38       ??_7IAttachmentObject@@6B@ 3160fa38     AttachmentManager.obj
 0002:00001a78       ??_7CCGFAttachment@@6B@    3160fa78     AttachmentManager.obj
 0002:00001ab8       ??_C@_0BD@NEBKDNEB@CAttachmentManager?$AA@ 3160fab8     AttachmentManager.obj
 0002:00001ad0       ??_7CSKELAttachment@@6B@   3160fad0     AttachmentManager.obj
 0002:00001b10       ??_7CSKINAttachment@@6B@   3160fb10     AttachmentManager.obj
 0002:00001b50       ??_C@_0DC@OPCJEBHN@CAttachmentManager?3?3ProcessAllAt@ 3160fb50     AttachmentManager.obj
 0002:00001b84       ??_C@_0CE@IKGEDBIL@CAttachmentManager?3?3DrawAttachme@ 3160fb84     AttachmentManager.obj
 0002:00001ba8       ??_C@_0DN@LIGJMAJA@CryAnimation?3?5skin?9attachment?5no@ 3160fba8     AttachmentManager.obj
 0002:00001be8       ??_C@_0DL@MILMPAAL@CryAnimation?3?5skin?9attachment?5mu@ 3160fbe8     AttachmentManager.obj
 0002:00001c24       ??_C@_0CH@GBLCFAEO@CryAnimation?3?5no?5character?5creat@ 3160fc24     AttachmentManager.obj
 0002:00001c4c       ??_C@_0DJ@BOJDPIMN@CryAnimation?3?5no?5static?5object?5a@ 3160fc4c     AttachmentManager.obj
 0002:00001c88       ??_C@_0DF@FBPKFMKG@CryAnimation?3?5no?5character?5as?5at@ 3160fc88     AttachmentManager.obj
 0002:00001cc0       ??_C@_03IJBHGJIK@cgf?$AA@  3160fcc0     AttachmentManager.obj
 0002:00001cc4       ??_C@_03MGFGPPEN@cga?$AA@  3160fcc4     AttachmentManager.obj
 0002:00001cc8       ??_C@_03ILFBNHND@cdf?$AA@  3160fcc8     AttachmentManager.obj
 0002:00001cd0       ??_7CAttachmentBONE@@6B@   3160fcd0     AttachmentManager.obj
 0002:00001d60       ??_7CAttachmentFACE@@6B@   3160fd60     AttachmentManager.obj
 0002:00001df0       ??_C@_07HMJPJE@CA_SKIN?$AA@ 3160fdf0     AttachmentManager.obj
 0002:00001df8       ??_C@_07CJKCDLBP@CA_FACE?$AA@ 3160fdf8     AttachmentManager.obj
 0002:00001e00       ??_C@_05BOOEKJH@Flags?$AA@ 3160fe00     AttachmentManager.obj
 0002:00001e08       ??_C@_08EHLKLHMC@lod?$CFd_?$CFs?$AA@ 3160fe08     AttachmentManager.obj
 0002:00001e14       ??_C@_0N@DCGKFBOO@PhysPropType?$AA@ 3160fe14     AttachmentManager.obj
 0002:00001e24       ??_C@_0BC@HKBCGBAC@PA_PendulumOffset?$AA@ 3160fe24     AttachmentManager.obj
 0002:00001e38       ??_C@_0P@BFNFOLOJ@PA_PivotOffset?$AA@ 3160fe38     AttachmentManager.obj
 0002:00001e48       ??_C@_0L@NDCAKFMA@PA_Damping?$AA@ 3160fe48     AttachmentManager.obj
 0002:00001e54       ??_C@_0N@EIIFNMLH@PA_HRotation?$AA@ 3160fe54     AttachmentManager.obj
 0002:00001e64       ??_C@_0M@BGCDNALG@PA_MaxAngle?$AA@ 3160fe64     AttachmentManager.obj
 0002:00001e70       ??_C@_0BA@BKMCDHKE@PA_PendulumType?$AA@ 3160fe70     AttachmentManager.obj
 0002:00001e80       ??_C@_08CPBFELGP@Material?$AA@ 3160fe80     AttachmentManager.obj
 0002:00001e8c       ??_C@_07JPNMPAFE@Binding?$AA@ 3160fe8c     AttachmentManager.obj
 0002:00001e94       ??_C@_08FPDFGKEJ@BoneName?$AA@ 3160fe94     AttachmentManager.obj
 0002:00001ea0       ??_C@_08GCJNLIKG@Position?$AA@ 3160fea0     AttachmentManager.obj
 0002:00001eac       ??_C@_08GFJPCMMD@Rotation?$AA@ 3160feac     AttachmentManager.obj
 0002:00001eb8       ??_C@_05LGOFDGEK@AName?$AA@ 3160feb8     AttachmentManager.obj
 0002:00001ec0       ??_C@_04KOACHJEN@Type?$AA@ 3160fec0     AttachmentManager.obj
 0002:00001ec8       ??_C@_07DECFHJLP@CA_BONE?$AA@ 3160fec8     AttachmentManager.obj
 0002:00001ed0       ??_C@_0L@PHKLKKHI@Attachment?$AA@ 3160fed0     AttachmentManager.obj
 0002:00001edc       ??_C@_0P@NCIHDFGC@AttachmentList?$AA@ 3160fedc     AttachmentManager.obj
 0002:00001ef0       ??_C@_0JE@JIFLDKKB@CryAnimation?3?5Attachment?5CRC32?5f@ 3160fef0     AttachmentManager.obj
 0002:00001f88       ??_C@_0FF@DBCAHCGP@CryAnimation?3?5Attachment?5name?5?8?$CF@ 3160ff88     AttachmentManager.obj
 0002:00001fe0       ??_C@_05GKKHKKE@Cloth?$AA@ 3160ffe0     AttachmentManager.obj
 0002:00001fe8       ??_C@_04FEDAIEKO@Rope?$AA@ 3160ffe8     AttachmentManager.obj
 0002:00001ff4       __real@41000000            3160fff4     CharacterInstance.obj
 0002:00001ff8       ??_7IFacialInstance@@6B@   3160fff8     FacialInstance.obj
 0002:00001ff8       ??_7IAttachmentManager@@6B@ 3160fff8     CharacterInstance.obj
 0002:00002048       ??_7ICharacterInstance@@6B@ 31610048     CharacterInstance.obj
 0002:00002130       ??_C@_0BE@HJMAHGKO@g_useSinglePosition?$AA@ 31610130     CharacterInstance.obj
 0002:00002144       ??_C@_0CI@LCECAICE@CCharInstance?3?3StartAnimationPro@ 31610144     CharacterInstance.obj
 0002:0000216c       ??_C@_0P@KLIDNMJ@fPlaybackScale?$AA@ 3161016c     CharacterInstance.obj
 0002:0000217c       ??_C@_0O@IJLABJDO@CCharInstance?$AA@ 3161017c     CharacterInstance.obj
 0002:0000218c       ??_C@_0CB@GOEOGGKH@Character?5instance?5serialization@ 3161018c     CharacterInstance.obj
 0002:000021b0       ??_C@_0DC@BOFAPKML@CCharInstance?3?3SkinningTransform@ 316101b0     CharacterInstance.obj
 0002:000021e4       ??_C@_0CA@CNAELFJE@CCharInstance?3?3UpdatePhysicsCGA?$AA@ 316101e4     CharacterInstance.obj
 0002:00002204       ??_C@_0CD@IALEGKJH@SkinningTransformationsComputati@ 31610204     CharacterInstance.obj
 0002:00002228       ??_C@_0N@JDNGJMJC@SkeletonPose?$AA@ 31610228     CharacterInstance.obj
 0002:00002238       ??_C@_0N@KPICOJGL@SkeletonAnim?$AA@ 31610238     CharacterInstance.obj
 0002:00002248       ??_C@_0BG@NNIDJJEH@skeletonEffectManager?$AA@ 31610248     CharacterInstance.obj
 0002:00002260       ??_C@_0P@FKGPMGCF@FacialInstance?$AA@ 31610260     CharacterInstance.obj
 0002:00002270       ??_C@_0N@IMBLMJCA@DecalManager?$AA@ 31610270     CharacterInstance.obj
 0002:00002280       ??_7CAttachmentManager@@6B@ 31610280     CharacterInstance.obj
 0002:000022d0       ??_C@_0N@NBFDINLK@Reloading?5?$CFs?$AA@ 316102d0     CharacterInstance.obj
 0002:000022e0       ??_C@_04FPMBEGCJ@?4cga?$AA@ 316102e0     CharacterInstance.obj
 0002:000022e8       ??_C@_04DFHCEAIG@?4chr?$AA@ 316102e8     CharacterInstance.obj
 0002:000022f0       ??_C@_0L@BINJLNLL@?4chrparams?$AA@ 316102f0     CharacterInstance.obj
 0002:000022fc       ??_C@_0P@MPKEIAAE@eye_right_bone?$AA@ 316102fc     CharacterInstance.obj
 0002:0000230c       ??_C@_0O@LEMMFOGJ@eye_left_bone?$AA@ 3161030c     CharacterInstance.obj
 0002:0000231c       ??_C@_0L@GHIHOBPC@Bip01?5Head?$AA@ 3161031c     CharacterInstance.obj
 0002:00002328       ??_C@_0BD@GILDFHIJ@Character?5Instance?$AA@ 31610328     CharacterInstance.obj
 0002:0000233c       ??_C@_0BN@LKLKFLMP@CCharInstance?3?3CCharInstance?$AA@ 3161033c     CharacterInstance.obj
 0002:00002360       ??_7CCharInstance@@6B@     31610360     CharacterInstance.obj
 0002:00002454       ??_C@_0BH@GOPGBEEC@CSkelInstance?3?3Release?$AA@ 31610454     CharacterInstance.obj
 0002:00002478       __real@3fd5555560000000    31610478     SkeletonEffectManager.obj
 0002:00002480       __real@3bb60b61            31610480     SkeletonEffectManager.obj
 0002:00002484       __real@40490fd0            31610484     SkeletonEffectManager.obj
 0002:00002488       ??_C@_0HL@DKCIOAAC@CSkeletonEffectManager?3?3KillAllE@ 31610488     SkeletonEffectManager.obj
 0002:00002504       ??_C@_0O@EDBNCENI@?$DMEFFECT?5NULL?$DO?$AA@ 31610504     SkeletonEffectManager.obj
 0002:00002518       ??_C@_0EJ@CFHONEBF@CSkeletonEffectManager?3?3Update?$CIt@ 31610518     SkeletonEffectManager.obj
 0002:00002564       ??_C@_0BB@EAGAEMEP@effect?5has?5ended?$AA@ 31610564     SkeletonEffectManager.obj
 0002:00002578       ??_C@_0BE@INGNAFEN@animation?5has?5ended?$AA@ 31610578     SkeletonEffectManager.obj
 0002:00002590       ??_C@_0GB@KCJFBAAL@CSkeletonEffectManager?3?3SpawnEff@ 31610590     SkeletonEffectManager.obj
 0002:000025f8       ??_C@_0EC@OODFIMGA@Anim?5events?5cannot?5find?5effect?5?$CC@ 316105f8     SkeletonEffectManager.obj
 0002:0000263c       ??_C@_0BE@GBHJILEN@?$DMMISSING?5ANIM?5NAME?$DO?$AA@ 3161063c     SkeletonEffectManager.obj
 0002:00002650       ??_C@_0GP@PLKJKPDM@CSkeletonEffectManager?3?3SpawnEff@ 31610650     SkeletonEffectManager.obj
 0002:000026c0       ??_C@_0BG@OBHJPKFK@?$DMMISSING?5EFFECT?5NAME?$DO?$AA@ 316106c0     SkeletonEffectManager.obj
 0002:000026e0       ??_7ISkeletonPhysics@@6B@  316106e0     SkeletonPose.obj
 0002:00002740       ?iid@?1??IID@IAnimationPoseBlenderDir@@CAABUCryGUID@@XZ@4U3@B 31610740     SkeletonPose.obj
 0002:00002750       __real@40555555            31610750     SkeletonPose.obj
 0002:00002754       __real@3fd55555            31610754     SkeletonPose.obj
 0002:00002758       ??_7CSkeletonPose@@6B@     31610758     SkeletonPose.obj
 0002:00002814       ??_C@_0BN@FJGLIONO@AnimationPoseModifier_LimbIk?$AA@ 31610814     SkeletonPose.obj
 0002:00002834       ??_C@_0BN@CDBOBPKN@AnimationPoseModifier_Recoil?$AA@ 31610834     SkeletonPose.obj
 0002:00002854       ??_C@_0CF@FNOFOMKI@AnimationPoseModifier_PoseBlende@ 31610854     SkeletonPose.obj
 0002:0000287c       ??_C@_0CG@IACGDDFJ@AnimationPoseModifier_PoseBlende@ 3161087c     SkeletonPose.obj
 0002:000028a8       __real@3be56041            316108a8     SkeletonPose_Debug.obj
 0002:000028ac       __real@3bfc5048            316108ac     SkeletonPose_Debug.obj
 0002:000028b0       ??_C@_0BA@MOHPKELD@ca_filterJoints?$AA@ 316108b0     SkeletonPose_Debug.obj
 0002:000028c8       ??_C@_0FP@NMBIDECH@CryAnimation?3?5Invalid?5BBox?5?$CI?$CF?43f@ 316108c8     SkeletonPose_Process.obj
 0002:00002928       __real@3ecccccd            31610928     SkeletonPose_Process.obj
 0002:00002930       ??_C@_0HG@JKDPDHGB@CryAnimation?3?5Invalid?5BBox?5of?5eA@ 31610930     SkeletonPose_Process.obj
 0002:000029a8       ??_C@_0HI@CDNHHDIC@CryAnimation?3?5Invalid?5BBox?5of?5eA@ 316109a8     SkeletonPose_Process.obj
 0002:00002a20       ??_C@_0GF@BNBINMGD@CryAnimation?3?5Invalid?5BBox?5of?5eA@ 31610a20     SkeletonPose_Process.obj
 0002:00002a88       ??_C@_0HF@DMFLBKPI@CryAnimation?3?5Invalid?5BBox?5of?5eA@ 31610a88     SkeletonPose_Process.obj
 0002:00002b00       __real@464b2000            31610b00     SkeletonPose_Process.obj
 0002:00002b04       __real@c64b2000            31610b04     SkeletonPose_Process.obj
 0002:00002b08       ??_C@_0DC@KCEBGHKH@CryAnimation?3?5Invalid?5BBox?5of?5eA@ 31610b08     SkeletonPose_Process.obj
 0002:00002b3c       ??_C@_0DD@PFPHELGK@CryAnimation?3?5Invalid?5BBox?5of?5eA@ 31610b3c     SkeletonPose_Process.obj
 0002:00002b70       ??_C@_0DB@KGEJIDDH@CryAnimation?3?5Invalid?5BBox?5of?5eA@ 31610b70     SkeletonPose_Process.obj
 0002:00002ba4       ??_C@_01EOFPKCAF@?$EA?$AA@ 31610ba4     SkeletonPose_Process.obj
 0002:00002ba8       ??_C@_0BK@FEFLJLDB@CSkeletonPose?3?3UpdateBBox?$AA@ 31610ba8     SkeletonPose_Process.obj
 0002:00002bc4       ??_C@_0CB@JFODNIDJ@CSkeletonPose?3?3UpdateAttachments@ 31610bc4     SkeletonPose_Process.obj
 0002:00002be8       ??_C@_0CD@NNGGBPBL@CSkeletonPose?3?3SkeletonPostProce@ 31610be8     SkeletonPose_Process.obj
 0002:00002c10       ??_7CSkeletonAnimTask@@6B@ 31610c10     SkeletonAnim.obj
 0002:00002c18       ??_7ISkeletonAnim@@6B@     31610c18     SkeletonAnim.obj
 0002:00002ca8       ??_C@_0EM@NCIMOGPO@Trying?5to?5set?5manual?5mixing?5weig@ 31610ca8     SkeletonAnim.obj
 0002:00002cf8       ??_C@_0HN@OAMMIFAP@Run?5out?5of?5free?5parametric?5slots@ 31610cf8     SkeletonAnim.obj
 0002:00002d78       ??_C@_0BB@JDCEONKJ@nSegmentCounter0?$AA@ 31610d78     SkeletonAnim.obj
 0002:00002d8c       ??_C@_08GICNLBFM@nAnimIDs?$AA@ 31610d8c     SkeletonAnim.obj
 0002:00002d98       ??_C@_02OLOABKKD@ID?$AA@   31610d98     SkeletonAnim.obj
 0002:00002d9c       ??_C@_0O@OBKBEJFL@m_numExamples?$AA@ 31610d9c     SkeletonAnim.obj
 0002:00002dac       ??_C@_0BI@EPLIHMDK@m_MotionParameterFlags3?$AA@ 31610dac     SkeletonAnim.obj
 0002:00002dc4       ??_C@_0BI@FGKDENHL@m_MotionParameterFlags2?$AA@ 31610dc4     SkeletonAnim.obj
 0002:00002ddc       ??_C@_0BI@HNIOBOLI@m_MotionParameterFlags1?$AA@ 31610ddc     SkeletonAnim.obj
 0002:00002df4       ??_C@_0BI@GEJFCPPJ@m_MotionParameterFlags0?$AA@ 31610df4     SkeletonAnim.obj
 0002:00002e0c       ??_C@_0BD@FNMPMFCO@MotionParameterID3?$AA@ 31610e0c     SkeletonAnim.obj
 0002:00002e20       ??_C@_0BD@EENEPEGP@MotionParameterID2?$AA@ 31610e20     SkeletonAnim.obj
 0002:00002e34       ??_C@_0BD@GPPJKHKM@MotionParameterID1?$AA@ 31610e34     SkeletonAnim.obj
 0002:00002e48       ??_C@_0BD@HGOCJGON@MotionParameterID0?$AA@ 31610e48     SkeletonAnim.obj
 0002:00002e5c       ??_C@_0BB@BNGLIPCC@MotionParameter3?$AA@ 31610e5c     SkeletonAnim.obj
 0002:00002e70       ??_C@_0BB@EHALOGD@MotionParameter2?$AA@ 31610e70     SkeletonAnim.obj
 0002:00002e84       ??_C@_0BB@CPFNONKA@MotionParameter1?$AA@ 31610e84     SkeletonAnim.obj
 0002:00002e98       ??_C@_0BB@DGEGNMOB@MotionParameter0?$AA@ 31610e98     SkeletonAnim.obj
 0002:00002eac       ??_C@_0BC@HODPFOO@m_nParametricType?$AA@ 31610eac     SkeletonAnim.obj
 0002:00002ec0       ??_C@_0BA@DGHJNPFJ@m_numDimensions?$AA@ 31610ec0     SkeletonAnim.obj
 0002:00002ed0       ??_C@_0BD@GDFFJPDJ@SParametricSampler?$AA@ 31610ed0     SkeletonAnim.obj
 0002:00002ee4       ??_C@_0BI@KOCPMHMM@CSkeletonAnimTask?3?3Wait?$AA@ 31610ee4     SkeletonAnim.obj
 0002:00002efc       ??_C@_0CG@PKLKOFJC@CSkeletonAnim?3?3ProcessAnimationU@ 31610efc     SkeletonAnim.obj
 0002:00002f24       ??_C@_0BF@LBMBDMEN@CommandBufferExecute?$AA@ 31610f24     SkeletonAnim.obj
 0002:00002f3c       ??_C@_0CL@KIKELEAM@CSkeletonAnim?3?3FinishAnimationCo@ 31610f3c     SkeletonAnim.obj
 0002:00002f68       ??_C@_0M@FBNCIMKH@BlenderLook?$AA@ 31610f68     SkeletonAnim.obj
 0002:00002f74       ??_C@_0L@BCDNODAM@BlenderAim?$AA@ 31610f74     SkeletonAnim.obj
 0002:00002f80       ??_C@_06LNHJHIDK@Recoil?$AA@ 31610f80     SkeletonAnim.obj
 0002:00002f88       ??_C@_06FCIIMNOL@LimbIK?$AA@ 31610f88     SkeletonAnim.obj
 0002:00002f90       ??_C@_0CO@BDOOGFON@Animation?5Task?5started?5while?5alr@ 31610f90     SkeletonAnim.obj
 0002:00002fc0       ??_C@_0CB@KNFFGCC@several?5pre?9updates?3?5FrameID?3?5?$CFx@ 31610fc0     SkeletonAnim.obj
 0002:00002fe8       ??_C@_0EN@CHENBBIP@CSkeletonAnim?3?3ProcessAnimations@ 31610fe8     SkeletonAnim.obj
 0002:00003038       ??_C@_0M@NJMOOCJK@fUserData?$CFi?$AA@ 31611038     SkeletonAnim.obj
 0002:00003044       ??_C@_0L@DGANLLHB@nUserToken?$AA@ 31611044     SkeletonAnim.obj
 0002:00003050       ??_C@_0P@LEFAENAC@fPlaybackSpeed?$AA@ 31611050     SkeletonAnim.obj
 0002:00003060       ??_C@_0L@PHEIIFBJ@fStartTime?$AA@ 31611060     SkeletonAnim.obj
 0002:0000306c       ??_C@_0BA@NAJHGMIJ@fTransitionTime?$AA@ 3161106c     SkeletonAnim.obj
 0002:0000307c       ??_C@_06PGMJADPC@nFlags?$AA@ 3161107c     SkeletonAnim.obj
 0002:00003084       ??_C@_09NIOBDIMK@DynFlags1?$AA@ 31611084     SkeletonAnim.obj
 0002:00003090       ??_C@_09MBPKAJIL@DynFlags0?$AA@ 31611090     SkeletonAnim.obj
 0002:0000309c       ??_C@_0BH@IFGILKFJ@segmentNormalizedTime1?$AA@ 3161109c     SkeletonAnim.obj
 0002:000030b4       ??_C@_0BH@JMHDILBI@segmentNormalizedTime0?$AA@ 316110b4     SkeletonAnim.obj
 0002:000030cc       ??_C@_0BL@JEFJNGNP@segmentNormalizedTimePrev1?$AA@ 316110cc     SkeletonAnim.obj
 0002:000030e8       ??_C@_0BL@INECOHJO@segmentNormalizedTimePrev0?$AA@ 316110e8     SkeletonAnim.obj
 0002:00003104       ??_C@_0BF@ILDLBJEJ@currentSegmentIndex1?$AA@ 31611104     SkeletonAnim.obj
 0002:0000311c       ??_C@_0BF@JCCACIAI@currentSegmentIndex0?$AA@ 3161111c     SkeletonAnim.obj
 0002:00003134       ??_C@_0BN@LADPHNKL@expectedTotalDurationSeconds?$AA@ 31611134     SkeletonAnim.obj
 0002:00003154       ??_C@_0CG@HBMDHLAE@currentSegmentExpectedDurationSe@ 31611154     SkeletonAnim.obj
 0002:0000317c       ??_C@_0BB@NDJBDEPO@transitionWeight?$AA@ 3161117c     SkeletonAnim.obj
 0002:00003190       ??_C@_0BD@HAOBDOND@transitionPriority?$AA@ 31611190     SkeletonAnim.obj
 0002:000031a4       ??_C@_0BL@BKOJBLHA@segmentNormalizedTimeDelta?$AA@ 316111a4     SkeletonAnim.obj
 0002:000031c0       ??_C@_0M@CAHNJPEP@animationId?$AA@ 316111c0     SkeletonAnim.obj
 0002:000031cc       ??_C@_0L@CKOPHJKN@CAnimation?$AA@ 316111cc     SkeletonAnim.obj
 0002:000031d8       ??_7CSkeletonAnim@@6B@     316111d8     SkeletonAnim.obj
 0002:0000326c       ??_C@_0N@NOMPLAGO@nAnimsInFIFO?$AA@ 3161126c     SkeletonAnim.obj
 0002:0000327c       ??_C@_04LIEBAAE@FIFO?$AA@  3161127c     SkeletonAnim.obj
 0002:00003284       ??_C@_0BE@OCLDLCOI@ForceSkeletonUpdate?$AA@ 31611284     SkeletonAnim.obj
 0002:00003298       ??_C@_0BG@IDEPGADK@AnimationDrivenMotion?$AA@ 31611298     SkeletonAnim.obj
 0002:000032b0       ??_C@_0O@EMJFAEAE@CSkeletonAnim?$AA@ 316112b0     SkeletonAnim.obj
 0002:000032c4       ??_C@_0BB@LBPDIKEH@?$CLybVFx3nSIAKTRLM?$AA@ 316112c4     SkeletonAnim_BlendMan.obj
 0002:000032d8       ??_C@_0BF@PAKPFLEL@invalid?5layer?5id?3?5?$CFd?$AA@ 316112d8     SkeletonAnim_BlendMan.obj
 0002:000032f0       ??_C@_0DH@EADFOBJA@SetLayerPlaybackScale?$CI?$CJ?5was?5usin@ 316112f0     SkeletonAnim_BlendMan.obj
 0002:00003328       __real@bf490fdb            31611328     SkeletonAnim_BlendMan.obj
 0002:0000332c       ??_C@_0BK@OFNKCMHP@CryAnimation?3?5weird?5error?$AA@ 3161132c     SkeletonAnim_BlendMan.obj
 0002:00003348       __real@3f50624dd2f1a9fc    31611348     SkeletonAnim_BlendMan.obj
 0002:00003350       __real@3ffffcb9            31611350     SkeletonAnim_BlendMan.obj
 0002:00003354       ??_C@_0BG@DJGEAONA@PM?5class?3?5?$CFs?0?5name?5?$CFs?$AA@ 31611354     SkeletonAnim_BlendMan.obj
 0002:0000336c       ??_C@_0BH@CCCIPAEE@LayerBlendWeight?3?5?$CF?42f?$AA@ 3161136c     SkeletonAnim_BlendMan.obj
 0002:00003384       ??_C@_0BJ@PKAHMHPG@StopLeg?3?5?$CFf?5?5?5locked?3?5?$CFd?$AA@ 31611384     SkeletonAnim_BlendMan.obj
 0002:000033a0       ??_C@_0BK@HCHOIMBG@TurnAngle?3?5?$CFf?5?5locked?3?5?$CFd?$AA@ 316113a0     SkeletonAnim_BlendMan.obj
 0002:000033bc       ??_C@_0BL@PCPKINMJ@TravelDist?3?5?$CFf?5?5locked?3?5?$CFd?$AA@ 316113bc     SkeletonAnim_BlendMan.obj
 0002:000033d8       ??_C@_0BM@MODFLBDB@TravelAngle?3?5?$CFf?5?5locked?3?5?$CFd?$AA@ 316113d8     SkeletonAnim_BlendMan.obj
 0002:000033f4       ??_C@_0BH@GFJBEPIE@Slope?3?5?$CFf?5?5?5locked?3?5?$CFd?$AA@ 316113f4     SkeletonAnim_BlendMan.obj
 0002:0000340c       ??_C@_0BK@JGCNEMDL@TurnSpeed?3?5?$CFf?5?5locked?3?5?$CFd?$AA@ 3161140c     SkeletonAnim_BlendMan.obj
 0002:00003428       ??_C@_0BK@HFGLOKKI@MoveSpeed?3?5?$CFf?5?5locked?3?5?$CFd?$AA@ 31611428     SkeletonAnim_BlendMan.obj
 0002:00003444       ??_C@_0DK@EHGNKBIP@?$CITry?$CJUseAimIK?3?5?$CFd?5?5AimIKBlend?3?5?$CF@ 31611444     SkeletonAnim_BlendMan.obj
 0002:00003480       ??_C@_0HG@KFADONL@AnimInAFIFO?5?$CF02d?3?5t?3?$CFd?5?5?$CFs?5?5ATim@ 31611480     SkeletonAnim_BlendMan.obj
 0002:000034f8       ??_C@_0CJ@JAGHNNHF@CryAnimation?3?5I2M?5without?5Turn?9P@ 316114f8     SkeletonAnim_BlendMan.obj
 0002:00003524       __real@358637bd            31611524     SkeletonAnim_BlendMan.obj
 0002:00003528       ??_C@_0CB@GENKLKFL@CryAnimation?3?5streaming?5file?3?5?$CFs@ 31611528     SkeletonAnim_BlendMan.obj
 0002:0000354c       ??_C@_0BG@BNBLDCEC@Streaming?5Assets?3?5?$CFs?5?$AA@ 3161154c     SkeletonAnim_BlendMan.obj
 0002:00003564       __real@40266666            31611564     SkeletonAnim_BlendMan.obj
 0002:00003568       ??_C@_0DI@BLFGLGHC@CryAnimation?3?5sum?5of?5transition?9@ 31611568     SkeletonAnim_BlendMan.obj
 0002:000035a0       ??_C@_0BM@MAMIHPIG@CSkeletonAnim?3?3BlendManager?$AA@ 316115a0     SkeletonAnim_BlendMan.obj
 0002:000035c0       ??_C@_0CG@ENFHLLOI@CryAnimation?3?5CommandBuffer?5over@ 316115c0     SkeletonAnim_Commands.obj
 0002:000035e8       __real@3ee66666            316115e8     SkeletonAnim_Commands.obj
 0002:000035ec       ??_C@_0DK@MAHKPBIL@CryAnimation?3?5LMG?5asset?5sorting?5@ 316115ec     SkeletonAnim_Commands.obj
 0002:00003628       ??_C@_0EH@KGLPLNGH@CryAnimation?3?5LMG?5weights?5don?8t?5@ 31611628     SkeletonAnim_Commands.obj
 0002:00003670       __real@3db851ec            31611670     SkeletonAnim_Commands.obj
 0002:00003674       ??_C@_0BP@HKBDNLIE@CSkeletonAnim?3?3Commands_Create?$AA@ 31611674     SkeletonAnim_Commands.obj
 0002:0000369c       ??_C@_0DD@LGCDNMMN@animation?9name?5?8?$CFs?8?5not?5in?5CAL?9f@ 3161169c     SkeletonAnim_Queue.obj
 0002:000036d0       ??_C@_04HIBGFPH@NULL?$AA@  316116d0     SkeletonAnim_Queue.obj
 0002:000036d8       ??_C@_04MLLLIHIP@null?$AA@ 316116d8     SkeletonAnim_Queue.obj
 0002:000036e0       ??_C@_0CA@IHMAKIHG@No?5name?5for?5animation?5specified?$AA@ 316116e0     SkeletonAnim_Queue.obj
 0002:00003700       ??_C@_0EP@MOCENKPM@illegal?5layer?5index?5used?5in?5func@ 31611700     SkeletonAnim_Queue.obj
 0002:00003750       ??_C@_0CF@LPDMCJ@Exceeding?5max?5examples?5in?5?$CFs?0?5CR@ 31611750     SkeletonAnim_Queue.obj
 0002:00003778       ??_C@_0BN@CEPHBKBJ@CryAnimation?3?5not?5initalized?$AA@ 31611778     SkeletonAnim_Queue.obj
 0002:00003798       ??_C@_0GB@OIDNMHKB@Animation?9queue?5overflow?4?5More?5t@ 31611798     SkeletonAnim_Queue.obj
 0002:000037fc       ??_C@_0BF@EIDJGIHD@LMG?5is?5invalid?3?5?8?$CFs?8?$AA@ 316117fc     SkeletonAnim_Queue.obj
 0002:00003814       ??_C@_0BM@MJDBPANO@Anim?5asset?5error?3?5?$CFs?5failed?$AA@ 31611814     SkeletonAnim_Queue.obj
 0002:00003830       ??_C@_0BM@JJOGJBAO@rLMG?4IsAssetLMGValid?$CI?$CJ?5?$CB?$DN?50?$AA@ 31611830     SkeletonAnim_Queue.obj
 0002:0000384c       ??_C@_0DL@KFFEMKAN@Asset?5for?5animation?9name?5?8?$CFs?8?5do@ 3161184c     SkeletonAnim_Queue.obj
 0002:00003888       ??_C@_0DI@GLLODHOF@trying?5to?5play?5an?5unloaded?5Look?9@ 31611888     SkeletonAnim_Queue.obj
 0002:000038c0       ??_C@_0DH@PMBKPGAO@trying?5to?5play?5an?5unloaded?5Aim?9P@ 316118c0     SkeletonAnim_Queue.obj
 0002:000038f8       ??_C@_0DK@ECPNMJGD@Asset?5for?5animation?9name?5?8?$CFs?8?5do@ 316118f8     SkeletonAnim_Queue.obj
 0002:00003934       ??_C@_0CC@PLKNFGEP@CSkeletonAnim?3?3StartAnimationByI@ 31611934     SkeletonAnim_Queue.obj
 0002:0000395c       ??_C@_0BF@GGEMLKGC@Eye_right_lower_left?$AA@ 3161195c     EyeMovementFaceAnim.obj
 0002:00003974       ??_C@_0BG@KHLAEODP@Eye_right_middle_left?$AA@ 31611974     EyeMovementFaceAnim.obj
 0002:0000398c       ??_C@_0BF@BDDPHIA@Eye_right_upper_left?$AA@ 3161198c     EyeMovementFaceAnim.obj
 0002:000039a4       ??_C@_0BH@LKHBJMFB@Eye_right_upper_middle?$AA@ 316119a4     EyeMovementFaceAnim.obj
 0002:000039bc       ??_C@_0BG@PHEGLPLO@Eye_right_upper_right?$AA@ 316119bc     EyeMovementFaceAnim.obj
 0002:000039d4       ??_C@_0BH@KMDOJCBK@Eye_right_middle_right?$AA@ 316119d4     EyeMovementFaceAnim.obj
 0002:000039ec       ??_C@_0BG@LJCFEDKH@Eye_right_lower_right?$AA@ 316119ec     EyeMovementFaceAnim.obj
 0002:00003a04       ??_C@_0BH@NOFEFHGN@Eye_right_lower_middle?$AA@ 31611a04     EyeMovementFaceAnim.obj
 0002:00003a1c       ??_C@_0BE@MPOBEKFA@Eye_left_lower_left?$AA@ 31611a1c     EyeMovementFaceAnim.obj
 0002:00003a30       ??_C@_0BF@GPMOLCEP@Eye_left_middle_left?$AA@ 31611a30     EyeMovementFaceAnim.obj
 0002:00003a48       ??_C@_0BE@KIJOAHLC@Eye_left_upper_left?$AA@ 31611a48     EyeMovementFaceAnim.obj
 0002:00003a5c       ??_C@_0BG@OKLMJDJB@Eye_left_upper_middle?$AA@ 31611a5c     EyeMovementFaceAnim.obj
 0002:00003a74       ??_C@_0BF@DPDIEDMO@Eye_left_upper_right?$AA@ 31611a74     EyeMovementFaceAnim.obj
 0002:00003a8c       ??_C@_0BG@PMPDJNNK@Eye_left_middle_right?$AA@ 31611a8c     EyeMovementFaceAnim.obj
 0002:00003aa4       ??_C@_0BF@HBFLLPNH@Eye_left_lower_right?$AA@ 31611aa4     EyeMovementFaceAnim.obj
 0002:00003abc       ??_C@_0BG@IOJJFIKN@Eye_left_lower_middle?$AA@ 31611abc     EyeMovementFaceAnim.obj
 0002:00003ad4       ??_7?$_i_reference_target@H@@6B@ 31611ad4     LoaderSKIN.obj
 0002:00003ad4       ??_7CEyeMovementFaceAnim@@6B@ 31611ad4     EyeMovementFaceAnim.obj
 0002:00003ae0       __real@3ea2f98c            31611ae0     EyeMovementFaceAnim.obj
 0002:00003ae4       __real@3d888889            31611ae4     EyeMovementFaceAnim.obj
 0002:00003ae8       ??_C@_09EDIDEKJE@eye_right?$AA@ 31611ae8     EyeMovementFaceAnim.obj
 0002:00003af4       ??_C@_08MPHIOKHM@eye_left?$AA@ 31611af4     EyeMovementFaceAnim.obj
 0002:00003b00       ??_C@_0BB@LHAAIHLB@?$CF?43f?0?5?$CF?43f?0?5?$CF?43f?$AA@ 31611b00     EyeMovementFaceAnim.obj
 0002:00003b14       __real@3e22f983            31611b14     EyeMovementFaceAnim.obj
 0002:00003b1c       __real@3f800000            31611b1c     Attachment.obj
 0002:00003b20       ??_7JoystickSerializeContext@?4??BindJoystickSetToSequence@CFacialAnimation@@UAEXPAVIJoystickSet@@PAUIFacialAnimSequence@@@Z@6B@ 31611b20     FaceAnimation.obj
 0002:00003b28       ??_C@_09KJHOEFNK@?$CFs?3?$CF?42f?0?5?$AA@ 31611b28     FaceAnimation.obj
 0002:00003b34       ??_C@_0CD@PCKJDCCB@Failed?5to?5load?5facial?5joysticks?5@ 31611b34     FaceAnimation.obj
 0002:00003b58       ??_C@_03DHFGHJCG@joy?$AA@  31611b58     FaceAnimation.obj
 0002:00003b5c       ??_C@_0BI@MKDILCDF@Stop?5Facial?5Sequence?5?$CFs?$AA@ 31611b5c     FaceAnimation.obj
 0002:00003b74       ??_7CFacialAnimSequenceInstance@@6B@ 31611b74     FaceAnimation.obj
 0002:00003b80       ??_7CFacialAnimationContext@@6B@ 31611b80     FaceAnimation.obj
 0002:00003b8c       ??_C@_0BB@KCOAIOFL@?$CFs?5?3?5?$CItime?$DN?$CF?42f?$CJ?$AA@ 31611b8c     FaceAnimation.obj
 0002:00003ba0       ??_C@_0BK@HDFLJAGF@Stop?5All?5Facial?5Sequences?$AA@ 31611ba0     FaceAnimation.obj
 0002:00003bbc       ??_7CFacialAnimation@@6BIJoystickContext@@@ 31611bbc     FaceAnimation.obj
 0002:00003bcc       ??_7CFacialAnimation@@6BIFacialAnimation@@@ 31611bcc     FaceAnimation.obj
 0002:00003c08       ??_C@_0EM@OJIBBPNJ@CFacialAnimationContext?3?3Update?$CI@ 31611c08     FaceAnimation.obj
 0002:00003c54       ??_C@_0CA@JFHDHLDA@CFacialAnimationContext?3?3Update?$AA@ 31611c54     FaceAnimation.obj
 0002:00003c74       ??_C@_0BI@OCHHCIBP@Play?5Facial?5Sequence?5?$CFs?$AA@ 31611c74     FaceAnimation.obj
 0002:00003c8c       ??_C@_0CH@HGMAHIPL@Failed?5to?5allocate?5memory?5for?5se@ 31611c8c     FaceAnimation.obj
 0002:00003cb4       ??_C@_0BP@BPEJPION@Failed?5to?5load?5facial?5sequence?$AA@ 31611cb4     FaceAnimation.obj
 0002:00003cd4       ??_C@_03KAGFBGIC@fsq?$AA@  31611cd4     FaceAnimation.obj
 0002:00003cd8       ??_C@_02MOLJINC@?3?3?$AA@  31611cd8     FaceAnimation.obj
 0002:00003ce0       ??_7IFacialAnimSoundEntry@@6B@ 31611ce0     FaceAnimSequence.obj
 0002:00003cf8       ??_7IFacialAnimSequence@@6B@ 31611cf8     FaceAnimSequence.obj
 0002:00003d80       ??_7ISplineInterpolator@@6B@ 31611d80     FaceAnimSequence.obj
 0002:00003d80       ??_7IFacialAnimChannel@@6B@ 31611d80     FaceAnimSequence.obj
 0002:00003dd8       ??_7IStreamCallback@@6B@   31611dd8     FaceAnimSequence.obj
 0002:00003de8       ??_C@_06DLKDIFGH@Spline?$AA@ 31611de8     FaceAnimSequence.obj
 0002:00003df0       ??_C@_07DMJBFPJJ@Channel?$AA@ 31611df0     FaceAnimSequence.obj
 0002:00003df8       ??_C@_04FABLJDN@Name?$AA@  31611df8     FaceAnimSequence.obj
 0002:00003e00       ??_C@_0FG@JCOJGMCK@CFacialAnimSequence?3?5Getting?5ske@ 31611e00     FaceAnimSequence.obj
 0002:00003e58       __real@3df5c28f            31611e58     FaceAnimSequence.obj
 0002:00003e5c       __real@bdf5c28f            31611e5c     FaceAnimSequence.obj
 0002:00003e60       __real@bdcccccd            31611e60     FaceAnimSequence.obj
 0002:00003e64       ??_7CFacialAnimSoundEntry@@6B@ 31611e64     FaceAnimSequence.obj
 0002:00003e7c       ??_7CFacialAnimSkeletalAnimationEntry@@6B@ 31611e7c     FaceAnimSequence.obj
 0002:00003e98       ??_7CFacialAnimChannel@@6B?$_i_reference_target@H@@@ 31611e98     FaceAnimSequence.obj
 0002:00003ea8       ??_7CFacialAnimChannel@@6BIFacialAnimChannel@@@ 31611ea8     FaceAnimSequence.obj
 0002:00003f00       ??_7?$TSpline@U?$SplineKey@U?$Quat_tpl@M@@@spline@@VHermitBasis@2@@spline@@6B@ 31611f00     FaceAnimSequence.obj
 0002:00003f10       ??_7?$TSpline@U?$TCBSplineKey@U?$Vec3_tpl@M@@@spline@@VHermitBasis@2@@spline@@6B@ 31611f10     FaceAnimSequence.obj
 0002:00003f20       ??_C@_09BLOICCGF@?$CFg?3?$CFg?3?$CFd?0?$AA@ 31611f20     FaceAnimSequence.obj
 0002:00003f2c       ??_C@_08NLFPHCLG@?$CFg?3?$CFg?3?$CFd?$AA@ 31611f2c     FaceAnimSequence.obj
 0002:00003f38       ??_C@_01IHBHIGKO@?0?$AA@   31611f38     FaceAnimSequence.obj
 0002:00003f3c       ??_C@_04EFDEBPGB@Keys?$AA@ 31611f3c     FaceAnimSequence.obj
 0002:00003f44       ??_7?$HermitSplineEx@U?$Quat_tpl@M@@U?$SplineKey@U?$Quat_tpl@M@@@spline@@@spline@@6B@ 31611f44     FaceAnimSequence.obj
 0002:00003f54       ??_7?$HermitSplineEx@MU?$SplineKey@M@spline@@@spline@@6B@ 31611f54     FaceAnimSequence.obj
 0002:00003f64       ??_C@_0BA@KMFEKME@?$CFg?3?$CFg?1?$CFg?1?$CFg?3?$CFd?0?$AA@ 31611f64     FaceAnimSequence.obj
 0002:00003f74       ??_C@_0P@PHDMIPGN@?$CFg?3?$CFg?1?$CFg?1?$CFg?3?$CFd?$AA@ 31611f74     FaceAnimSequence.obj
 0002:00003f84       ??_C@_0BD@MLFCNHLL@?$CFg?3?$CFg?1?$CFg?1?$CFg?1?$CFg?3?$CFd?0?$AA@ 31611f84     FaceAnimSequence.obj
 0002:00003f98       ??_C@_0BC@BLMFLFD@?$CFg?3?$CFg?1?$CFg?1?$CFg?1?$CFg?3?$CFd?$AA@ 31611f98     FaceAnimSequence.obj
 0002:00003fac       ??_7?$TCBSpline@U?$Vec3_tpl@M@@U?$TCBSplineKey@U?$Vec3_tpl@M@@@spline@@@spline@@6B@ 31611fac     FaceAnimSequence.obj
 0002:00003fbc       ??_7?$SSplineBackup@V?$HermitSplineEx@U?$Quat_tpl@M@@U?$SplineKey@U?$Quat_tpl@M@@@spline@@@spline@@@spline@@6B?$HermitSplineEx@U?$Quat_tpl@M@@U?$SplineKey@U?$Quat_tpl@M@@@spline@@@1@@ 31611fbc     FaceAnimSequence.obj
 0002:00003fcc       ??_7?$SSplineBackup@V?$HermitSplineEx@U?$Quat_tpl@M@@U?$SplineKey@U?$Quat_tpl@M@@@spline@@@spline@@@spline@@6BISplineBackup@@@ 31611fcc     FaceAnimSequence.obj
 0002:00003fd8       ??_7?$CBaseSplineInterpolator@MV?$HermitSplineEx@MU?$SplineKey@M@spline@@@spline@@@spline@@6BISplineInterpolator@@@ 31611fd8     FaceAnimSequence.obj
 0002:00004030       ??_7?$SSplineBackup@V?$HermitSplineEx@MU?$SplineKey@M@spline@@@spline@@@spline@@6B?$HermitSplineEx@MU?$SplineKey@M@spline@@@1@@ 31612030     FaceAnimSequence.obj
 0002:00004040       ??_7?$SSplineBackup@V?$HermitSplineEx@MU?$SplineKey@M@spline@@@spline@@@spline@@6BISplineBackup@@@ 31612040     FaceAnimSequence.obj
 0002:00004050       ??_C@_0ED@ECEILDBO@CFacialAnimSequence?3?5Deleting?5no@ 31612050     FaceAnimSequence.obj
 0002:00004098       ??_C@_0FH@FIIKLAIH@CFacialAnimSequence?3?5Deleting?5sk@ 31612098     FaceAnimSequence.obj
 0002:000040f0       ??_7?$SSplineBackup@V?$TCBSpline@U?$Vec3_tpl@M@@U?$TCBSplineKey@U?$Vec3_tpl@M@@@spline@@@spline@@@spline@@6B?$TCBSpline@U?$Vec3_tpl@M@@U?$TCBSplineKey@U?$Vec3_tpl@M@@@spline@@@1@@ 316120f0     FaceAnimSequence.obj
 0002:00004100       ??_7?$SSplineBackup@V?$TCBSpline@U?$Vec3_tpl@M@@U?$TCBSplineKey@U?$Vec3_tpl@M@@@spline@@@spline@@@spline@@6BISplineBackup@@@ 31612100     FaceAnimSequence.obj
 0002:0000410c       ??_7CFacialCameraPathPositionInterpolator@@6B?$TCBSpline@U?$Vec3_tpl@M@@U?$TCBSplineKey@U?$Vec3_tpl@M@@@spline@@@spline@@@ 3161210c     FaceAnimSequence.obj
 0002:00004120       ??_7CFacialCameraPathPositionInterpolator@@6BISplineInterpolator@@@ 31612120     FaceAnimSequence.obj
 0002:00004178       ??_7CFacialCameraPathOrientationInterpolator@@6B?$HermitSplineEx@U?$Quat_tpl@M@@U?$SplineKey@U?$Quat_tpl@M@@@spline@@@spline@@@ 31612178     FaceAnimSequence.obj
 0002:00004188       ??_7CFacialCameraPathOrientationInterpolator@@6BISplineInterpolator@@@ 31612188     FaceAnimSequence.obj
 0002:000041e0       ??_7?$CBaseSplineInterpolator@MV?$HermitSplineEx@MU?$SplineKey@M@spline@@@spline@@@spline@@6B?$HermitSplineEx@MU?$SplineKey@M@spline@@@1@@ 316121e0     FaceAnimSequence.obj
 0002:000041e0       ??_7CFacialAnimChannelInterpolator@@6B?$HermitSplineEx@MU?$SplineKey@M@spline@@@spline@@@ 316121e0     FaceAnimSequence.obj
 0002:000041f0       ??_7CFacialAnimChannelInterpolator@@6BISplineInterpolator@@@ 316121f0     FaceAnimSequence.obj
 0002:00004248       ??_7CFacialAnimSequence@@6BIStreamCallback@@@ 31612248     FaceAnimSequence.obj
 0002:00004258       ??_7CFacialAnimSequence@@6BIFacialAnimSequence@@@ 31612258     FaceAnimSequence.obj
 0002:000042e0       ??_C@_0CG@GNBPJBKH@Failed?5to?5stream?5facial?5sequence@ 316122e0     FaceAnimSequence.obj
 0002:00004308       ??_C@_0CG@HGLPGDO@CFacialAnimSequence?3?3StreamOnCom@ 31612308     FaceAnimSequence.obj
 0002:00004330       ??_C@_0BA@PNDICABG@Neck_left_right?$AA@ 31612330     FaceAnimSequence.obj
 0002:00004340       ??_C@_0N@BKPMEFLO@Neck_up_down?$AA@ 31612340     FaceAnimSequence.obj
 0002:00004350       ??_C@_0BB@LLGBCJAO@Default?5Sequence?$AA@ 31612350     FaceAnimSequence.obj
 0002:00004368       ??_C@_0EL@OGGFCGGC@CFacialAnimSequence?3?5Inserting?5s@ 31612368     FaceAnimSequence.obj
 0002:000043b8       ??_C@_0FI@GCHEDGEC@CFacialAnimSequence?3?5Inserting?5s@ 316123b8     FaceAnimSequence.obj
 0002:00004410       ??_C@_07LDICNKFK@?$CFs?$EA?3?$EA?$CFs?$AA@ 31612410     FaceAnimSequence.obj
 0002:00004418       ??_C@_0DF@PIOFEMFB@Attempting?5to?5merge?5sequence?5wit@ 31612418     FaceAnimSequence.obj
 0002:00004450       ??_C@_0N@NFDKOEAM@BakedLipSync?$AA@ 31612450     FaceAnimSequence.obj
 0002:00004460       ??_C@_0BH@EKOBJLKB@SkeletonAnimationStart?$AA@ 31612460     FaceAnimSequence.obj
 0002:00004478       ??_C@_0BC@LPJKMPGL@SkeletonAnimation?$AA@ 31612478     FaceAnimSequence.obj
 0002:0000448c       ??_C@_0O@IGGNDABF@CameraPathFOV?$AA@ 3161248c     FaceAnimSequence.obj
 0002:0000449c       ??_C@_0BH@HAKIDAOD@CameraPathOrientations?$AA@ 3161249c     FaceAnimSequence.obj
 0002:000044b4       ??_C@_0BE@PILIAEOL@CameraPathPositions?$AA@ 316124b4     FaceAnimSequence.obj
 0002:000044c8       ??_C@_0O@HEOGOAJ@AnimationName?$AA@ 316124c8     FaceAnimSequence.obj
 0002:000044d8       ??_C@_0BH@GHFHCMOE@SkeletonAnimationEntry?$AA@ 316124d8     FaceAnimSequence.obj
 0002:000044f0       ??_C@_05MAHMNMLO@Sound?$AA@ 316124f0     FaceAnimSequence.obj
 0002:000044f8       ??_C@_0L@GBCGONJH@SoundEntry?$AA@ 316124f8     FaceAnimSequence.obj
 0002:00004504       ??_C@_08FJCINCME@Sentence?$AA@ 31612504     FaceAnimSequence.obj
 0002:00004510       ??_C@_09BFDKACGK@Joysticks?$AA@ 31612510     FaceAnimSequence.obj
 0002:0000451c       ??_C@_07GAHEIAPI@EndTime?$AA@ 3161251c     FaceAnimSequence.obj
 0002:00004524       ??_C@_09MHCEAAPI@StartTime?$AA@ 31612524     FaceAnimSequence.obj
 0002:00004534       __real@7f7fffff            31612534     FaceChannelKeyCleanup.obj
 0002:00004540       __real@401921fa00000000    31612540     FaceChannelSmoothing.obj
 0002:00004550       ??_7IFacialEffector@@6B@   31612550     FaceEffector.obj
 0002:000045a4       ??_C@_08EPGFEOCM@Effector?$AA@ 316125a4     FaceEffector.obj
 0002:000045b0       ??_C@_06ODJMJFLN@Weight?$AA@ 316125b0     FaceEffector.obj
 0002:000045b8       ??_C@_09MANMBJC@RotOffset?$AA@ 316125b8     FaceEffector.obj
 0002:000045c4       ??_C@_09CDNBILG@PosOffset?$AA@ 316125c4     FaceEffector.obj
 0002:000045d0       ??_C@_06OCDDEAHI@?$CFg?3?$CFg?0?$AA@ 316125d0     FaceEffector.obj
 0002:000045d8       ??_7?$TSpline@U?$SplineKey@M@spline@@U?$TCoeffBasis@M@2@@spline@@6B@ 316125d8     FaceEffector.obj
 0002:000045d8       ??_7?$TSpline@U?$SplineKey@M@spline@@VHermitBasis@2@@spline@@6B@ 316125d8     FaceAnimSequence.obj
 0002:000045e8       ??_7CFacialEffector@@6BIFacialEffector@@@ 316125e8     FaceEffector.obj
 0002:0000464c       ??_7CFacialEffectorBone@@6B?$_i_reference_target@H@@@ 3161264c     FaceEffectorLibrary.obj
 0002:0000464c       ??_7CFacialEffectorAttachment@@6B?$_i_reference_target@H@@@ 3161264c     FaceEffector.obj
 0002:00004658       ??_7CFacialEffectorAttachment@@6BIFacialEffector@@@ 31612658     FaceEffector.obj
 0002:000046c8       ??_7?$CatmullRomSpline@MU?$SplineKey@M@spline@@$0A@@spline@@6B@ 316126c8     FaceEffector.obj
 0002:000046d8       ??_7?$SSplineBackup@V?$CatmullRomSpline@MU?$SplineKey@M@spline@@$0A@@spline@@@spline@@6B?$CatmullRomSpline@MU?$SplineKey@M@spline@@$0A@@1@@ 316126d8     FaceEffector.obj
 0002:000046e8       ??_7?$SSplineBackup@V?$CatmullRomSpline@MU?$SplineKey@M@spline@@$0A@@spline@@@spline@@6BISplineBackup@@@ 316126e8     FaceEffector.obj
 0002:000046f4       ??_7CFacialEffCtrlSplineInterpolator@@6B?$CatmullRomSpline@MU?$SplineKey@M@spline@@$0A@@spline@@@ 316126f4     FaceEffector.obj
 0002:00004708       ??_7CFacialEffCtrlSplineInterpolator@@6BISplineInterpolator@@@ 31612708     FaceEffector.obj
 0002:00004760       ??_7CFacialEffCtrl@@6B?$_i_reference_target@H@@@ 31612760     FaceEffector.obj
 0002:0000476c       ??_7CFacialEffCtrl@@6BIFacialEffCtrl@@@ 3161276c     FaceEffector.obj
 0002:000047a8       ??_7IJoystick@@6B@         316127a8     FaceJoystick.obj
 0002:000047a8       ??_7IFacialAnimation@@6B@  316127a8     FaceAnimation.obj
 0002:000047a8       ??_7IFacialEffectorsLibrary@@6B@ 316127a8     FaceEffectorLibrary.obj
 0002:000047a8       ??_7IJoystickChannel@@6B@  316127a8     FaceJoystick.obj
 0002:000047e0       ??_C@_07CIFAGBMG@unknown?$AA@ 316127e0     FaceEffectorLibrary.obj
 0002:000047e8       ??_C@_08KNOEMJMM@material?$AA@ 316127e8     FaceEffectorLibrary.obj
 0002:000047f4       ??_C@_0L@HBDHCFKP@attachment?$AA@ 316127f4     FaceEffectorLibrary.obj
 0002:00004800       ??_C@_04ODKJLCFC@bone?$AA@ 31612800     FaceEffectorLibrary.obj
 0002:00004808       ??_C@_05NJNGEDKM@morph?$AA@ 31612808     FaceEffectorLibrary.obj
 0002:00004810       ??_C@_0L@FKCCBALC@expression?$AA@ 31612810     FaceEffectorLibrary.obj
 0002:0000481c       ??_C@_05MGJOOGAJ@group?$AA@ 3161281c     FaceEffectorLibrary.obj
 0002:00004824       ??_C@_07NPCLAIKJ@SubCtrl?$AA@ 31612824     FaceEffectorLibrary.obj
 0002:0000482c       ??_7CFacialEffectorsLibrary@@6B@ 3161282c     FaceEffectorLibrary.obj
 0002:00004868       ??_C@_0EF@BALMIJNF@Attachment?5Effectors?5no?5longer?5s@ 31612868     FaceEffectorLibrary.obj
 0002:000048b0       ??_7CFacialEffectorExpression@@6B?$_i_reference_target@H@@@ 316128b0     FaceEffectorLibrary.obj
 0002:000048b0       ??_7CFacialEffector@@6B?$_i_reference_target@H@@@ 316128b0     FaceEffector.obj
 0002:000048b0       ??_7CFacialMorphTarget@@6B?$_i_reference_target@H@@@ 316128b0     FaceEffectorLibrary.obj
 0002:000048c0       ??_7CFacialMorphTarget@@6BIFacialEffector@@@ 316128c0     FaceEffectorLibrary.obj
 0002:00004924       ??_C@_04BAJDEDPD@Root?$AA@ 31612924     FaceEffectorLibrary.obj
 0002:00004930       ??_7CFacialEffectorExpression@@6BIFacialEffector@@@ 31612930     FaceEffectorLibrary.obj
 0002:00004998       ??_7CFacialEffectorBone@@6BIFacialEffector@@@ 31612998     FaceEffectorLibrary.obj
 0002:00004a08       ??_C@_0DE@HHGOBIHP@Attempting?5to?5merge?5library?5with@ 31612a08     FaceEffectorLibrary.obj
 0002:00004a3c       ??_C@_0M@INHKPGMC@Controllers?$AA@ 31612a3c     FaceEffectorLibrary.obj
 0002:00004a48       ??_C@_0N@MNPGGADE@AllEffectors?$AA@ 31612a48     FaceEffectorLibrary.obj
 0002:00004a58       ??_C@_0CE@HJAMLKEC@Effector?5with?5name?5?$CFs?5already?5ex@ 31612a58     FaceEffectorLibrary.obj
 0002:00004a80       ??_7IFacialEffCtrl@@6B@    31612a80     FaceEffector.obj
 0002:00004a80       ??_7IJoystickSet@@6B@      31612a80     FaceJoystick.obj
 0002:00004ab0       ??_7CFacialJoystickChannel@@6B@ 31612ab0     FaceJoystick.obj
 0002:00004ae8       ??_7CFacialJoystick@@6B@   31612ae8     FaceJoystick.obj
 0002:00004b20       ??_7CFacialJoystickSet@@6B@ 31612b20     FaceJoystick.obj
 0002:00004b50       ??_C@_01EANLCPLP@y?$AA@    31612b50     FaceJoystick.obj
 0002:00004b54       ??_C@_01FJMABOPO@x?$AA@    31612b54     FaceJoystick.obj
 0002:00004b58       ??_C@_0M@LNJPGNEG@VideoOffset?$AA@ 31612b58     FaceJoystick.obj
 0002:00004b64       ??_C@_0L@EDKOHOLB@VideoScale?$AA@ 31612b64     FaceJoystick.obj
 0002:00004b70       ??_C@_07MLKCHEME@Flipped?$AA@ 31612b70     FaceJoystick.obj
 0002:00004b78       ??_C@_08FGBNDLMK@Vertical?$AA@ 31612b78     FaceJoystick.obj
 0002:00004b84       ??_C@_0L@DKFGPADG@Horizontal?$AA@ 31612b84     FaceJoystick.obj
 0002:00004b90       ??_C@_04LBNBCLPC@Axis?$AA@ 31612b90     FaceJoystick.obj
 0002:00004b98       ??_C@_05PDOBBJNA@Color?$AA@ 31612b98     FaceJoystick.obj
 0002:00004ba0       ??_C@_08CJCDADNL@Joystick?$AA@ 31612ba0     FaceJoystick.obj
 0002:00004bac       ??_C@_0L@NDPLFEJ@Dimensions?$AA@ 31612bac     FaceJoystick.obj
 0002:00004bb8       ??_C@_06MCOJAMLH@Centre?$AA@ 31612bb8     FaceJoystick.obj
 0002:00004bc8       ??_C@_0GI@FNHCCAAL@Loading?5facial?5animation?5sequenc@ 31612bc8     FacialInstance.obj
 0002:00004c30       ??_C@_0GD@LMLLHIE@Loading?5facial?5animation?5sequenc@ 31612c30     FacialInstance.obj
 0002:00004c94       ??_C@_0BK@DLLBCJKE@Invalid?5layer?5passed?5?9?5?$CFd?$AA@ 31612c94     FacialInstance.obj
 0002:00004cb0       __real@3b03126f            31612cb0     FacialInstance.obj
 0002:00004cb4       __real@3c9374bc            31612cb4     FacialInstance.obj
 0002:00004cb8       ??_C@_0GF@FLEPIFBF@CFacialInstance?3?3TemporarilyEnab@ 31612cb8     FacialInstance.obj
 0002:00004d20       ??_C@_0FE@MOCEADPK@CFacialInstance?3?3UpdateCurrentSe@ 31612d20     FacialInstance.obj
 0002:00004d78       ??_C@_0EK@LLJKCLIA@CFacialInstance?3?3UpdateCurrentSe@ 31612d78     FacialInstance.obj
 0002:00004dc8       ??_C@_0EK@ELPDFMFO@CFacialInstance?3?3UpdateCurrentSe@ 31612dc8     FacialInstance.obj
 0002:00004e18       ??_C@_0ED@FDFFFADK@CFacialInstance?3?3UpdateCurrentSe@ 31612e18     FacialInstance.obj
 0002:00004e60       ??_C@_0FJ@KLEIDDPM@CFacialInstance?3?3UpdateCurrentSe@ 31612e60     FacialInstance.obj
 0002:00004ebc       ??_C@_0DL@NALGPHFE@CFacialInstance?3?3Update?5?9?5?$CIthis?$DN@ 31612ebc     FacialInstance.obj
 0002:00004ef8       ??_C@_0EA@HHOENHDP@CFacialInstance?3?3PlaySequence?$CIth@ 31612ef8     FacialInstance.obj
 0002:00004f38       ??_C@_0EA@NGPEOLAA@CFacialInstance?3?3StopSequence?$CIth@ 31612f38     FacialInstance.obj
 0002:00004f78       ??_C@_05NCABIDLI@Blink?$AA@ 31612f78     FacialInstance.obj
 0002:00004f80       ??_C@_0CA@IIJMAECO@CFacialInstance?3?3Reset?$CIthis?$DN?$CFp?$CJ?$AA@ 31612f80     FacialInstance.obj
 0002:00004fa0       ??_C@_01KMDKNFGN@?1?$AA@   31612fa0     FacialInstance.obj
 0002:00004fa4       ??_C@_0BA@HMOFIHLL@g_languageAudio?$AA@ 31612fa4     FacialInstance.obj
 0002:00004fb4       __real@3c03126f            31612fb4     FacialInstance.obj
 0002:00004fb8       __real@c0800000            31612fb8     FacialInstance.obj
 0002:00004fbc       ??_7CFacialInstance@@6B?$_i_reference_target@H@@@ 31612fbc     FacialInstance.obj
 0002:00004fc8       ??_7CFacialInstance@@6BIFacialInstance@@@ 31612fc8     FacialInstance.obj
 0002:0000501c       ??_7IFaceState@@6B@        3161301c     FacialModel.obj
 0002:0000501c       ??_7IVertexAnimation@@6B@  3161301c     VertexAnimation.obj
 0002:0000501c       ??_7ISplineBackup@@6B@     3161301c     FaceAnimSequence.obj
 0002:0000501c       ??_7Validator@pe_action_batch_parts_update@@6B@ 3161301c     SkeletonPhysics.obj
 0002:00005028       ??_7CFaceState@@6B?$_i_reference_target@H@@@ 31613028     FacialModel.obj
 0002:00005034       ??_7CFaceState@@6BIFaceState@@@ 31613034     FacialModel.obj
 0002:00005040       ??_C@_0CL@BGMIDNDI@Attachment?5Effectors?5not?5longer?5@ 31613040     FacialModel.obj
 0002:0000506c       ??_C@_0CH@IOKJKNBL@CFacialModel?3?3FillInfoMapFromFac@ 3161306c     FacialModel.obj
 0002:00005094       ??_7CFacialModel@@6B?$_i_reference_target@H@@@ 31613094     FacialModel.obj
 0002:000050a0       ??_7CFacialModel@@6BIFacialModel@@@ 316130a0     FacialModel.obj
 0002:000050bc       ??_C@_08NJFLMLKA@pleasure?$AA@ 316130bc     LipSync.obj
 0002:000050c8       ??_C@_02PEPMCKME@zh?$AA@   316130c8     LipSync.obj
 0002:000050cc       ??_C@_03LMBDLIPK@zap?$AA@  316130cc     LipSync.obj
 0002:000050d0       ??_C@_01GLPGHMHM@z?$AA@    316130d0     LipSync.obj
 0002:000050d4       ??_C@_04BIGBAIKH@yard?$AA@ 316130d4     LipSync.obj
 0002:000050dc       ??_C@_04MKNNKNJH@with?$AA@ 316130dc     LipSync.obj
 0002:000050e4       ??_C@_01NOFIACDB@w?$AA@    316130e4     LipSync.obj
 0002:000050e8       ??_C@_03JCKJMCEG@vat?$AA@  316130e8     LipSync.obj
 0002:000050ec       ??_C@_01MHEDDDHA@v?$AA@    316130ec     LipSync.obj
 0002:000050f0       ??_C@_03JLAIOMFN@too?$AA@  316130f0     LipSync.obj
 0002:000050f4       ??_C@_02DCPKGDGH@uw?$AA@   316130f4     LipSync.obj
 0002:000050f8       ??_C@_04HMOIPFOL@book?$AA@ 316130f8     LipSync.obj
 0002:00005100       ??_C@_02PPKAGNPJ@uh?$AA@   31613100     LipSync.obj
 0002:00005104       ??_C@_04HHGFCHIH@thin?$AA@ 31613104     LipSync.obj
 0002:0000510c       ??_C@_02POGCAHMO@th?$AA@   3161310c     LipSync.obj
 0002:00005110       ??_C@_04HBNBFOKD@talk?$AA@ 31613110     LipSync.obj
 0002:00005118       ??_C@_01PFHFFBPC@t?$AA@    31613118     LipSync.obj
 0002:0000511c       ??_C@_03PJHPCKOL@she?$AA@  3161311c     LipSync.obj
 0002:00005120       ??_C@_02PLCNBBEL@sh?$AA@   31613120     LipSync.obj
 0002:00005124       ??_C@_03KLGEGDMM@sit?$AA@  31613124     LipSync.obj
 0002:00005128       ??_C@_01LKDEMHDF@s?$AA@    31613128     LipSync.obj
 0002:0000512c       ??_C@_03FAAAOPJM@red?$AA@  3161312c     LipSync.obj
 0002:00005130       ??_C@_01KDCPPGHE@r?$AA@    31613130     LipSync.obj
 0002:00005134       ??_C@_03KMONJGDG@put?$AA@  31613134     LipSync.obj
 0002:00005138       ??_C@_01JBBJJEPG@p?$AA@    31613138     LipSync.obj
 0002:0000513c       ??_C@_03IHJAFJIK@toy?$AA@  3161313c     LipSync.obj
 0002:00005140       ??_C@_02LNMIGIEP@oy?$AA@   31613140     LipSync.obj
 0002:00005144       ??_C@_02KPEDIMCA@go?$AA@   31613144     LipSync.obj
 0002:00005148       ??_C@_02CDELEFMB@ow?$AA@   31613148     LipSync.obj
 0002:0000514c       ??_C@_04KJHEDBDO@sing?$AA@ 3161314c     LipSync.obj
 0002:00005154       ??_C@_02GIELDNKH@ng?$AA@   31613154     LipSync.obj
 0002:00005158       ??_C@_02KAJCLHKP@no?$AA@   31613158     LipSync.obj
 0002:0000515c       ??_C@_01EFFIKLCJ@n?$AA@    3161315c     LipSync.obj
 0002:00005160       ??_C@_03BFLBBCNI@mat?$AA@  31613160     LipSync.obj
 0002:00005164       ??_C@_01GOHFPIOK@m?$AA@    31613164     LipSync.obj
 0002:00005168       ??_C@_03OJNMDGFE@lid?$AA@  31613168     LipSync.obj
 0002:0000516c       ??_C@_01HHGOMJKL@l?$AA@    3161316c     LipSync.obj
 0002:00005170       ??_C@_01DICPFPGM@k?$AA@    31613170     LipSync.obj
 0002:00005174       ??_C@_02OINKIJLE@jh?$AA@   31613174     LipSync.obj
 0002:00005178       ??_C@_04KEADKAFO@feel?$AA@ 31613178     LipSync.obj
 0002:00005180       ??_C@_02LJEFBEPN@iy?$AA@   31613180     LipSync.obj
 0002:00005184       ??_C@_04OBAECEGJ@fill?$AA@ 31613184     LipSync.obj
 0002:0000518c       ??_C@_02OKJMDHON@ih?$AA@   3161318c     LipSync.obj
 0002:00005190       ??_C@_04PCJFHION@help?$AA@ 31613190     LipSync.obj
 0002:00005198       ??_C@_01BDACAMKP@h?$AA@    31613198     LipSync.obj
 0002:0000519c       ??_C@_03GBCDPJBA@gut?$AA@  3161319c     LipSync.obj
 0002:000051a0       ??_C@_01JEJKBAGA@g?$AA@    316131a0     LipSync.obj
 0002:000051a4       ??_C@_04JNJGGDAI@fork?$AA@ 316131a4     LipSync.obj
 0002:000051ac       ??_C@_01INIBCBCB@f?$AA@    316131ac     LipSync.obj
 0002:000051b0       ??_C@_03BGFDOPOL@ate?$AA@  316131b0     LipSync.obj
 0002:000051b4       ??_C@_02LAFPONJJ@ey?$AA@   316131b4     LipSync.obj
 0002:000051b8       ??_C@_03IPMFDJPD@fur?$AA@  316131b8     LipSync.obj
 0002:000051bc       ??_C@_02FDKLDEFC@er?$AA@   316131bc     LipSync.obj
 0002:000051c0       ??_C@_03LAMLDFEG@pet?$AA@  316131c0     LipSync.obj
 0002:000051c4       ??_C@_02ODIGMOIJ@eh?$AA@   316131c4     LipSync.obj
 0002:000051c8       ??_C@_04HOHPNOOD@then?$AA@ 316131c8     LipSync.obj
 0002:000051d0       ??_C@_02OCEEKELO@dh?$AA@   316131d0     LipSync.obj
 0002:000051d4       ??_C@_03HEFENHI@dig?$AA@   316131d4     LipSync.obj
 0002:000051d8       ??_C@_01LPLHEDKD@d?$AA@    316131d8     LipSync.obj
 0002:000051dc       ??_C@_04KFKFGMBF@chin?$AA@ 316131dc     LipSync.obj
 0002:000051e4       ??_C@_02OHALLCDL@ch?$AA@   316131e4     LipSync.obj
 0002:000051e8       ??_C@_03CCCOBCKE@big?$AA@  316131e8     LipSync.obj
 0002:000051ec       ??_C@_01OJONOECF@b?$AA@    316131ec     LipSync.obj
 0002:000051f0       ??_C@_04NHHDMLCI@bite?$AA@ 316131f0     LipSync.obj
 0002:000051f8       ??_C@_02LHFGEFEF@ay?$AA@   316131f8     LipSync.obj
 0002:000051fc       ??_C@_03PCNMBKEI@ago?$AA@  316131fc     LipSync.obj
 0002:00005200       ??_C@_02KOENHEAE@ax?$AA@   31613200     LipSync.obj
 0002:00005204       ??_C@_04NHJIODEK@foul?$AA@ 31613204     LipSync.obj
 0002:0000520c       ??_C@_02CJNFGIML@aw?$AA@   3161320c     LipSync.obj
 0002:00005210       ??_C@_03DMIDBMK@dog?$AA@   31613210     LipSync.obj
 0002:00005214       ??_C@_02KLMOPAJC@ao?$AA@   31613214     LipSync.obj
 0002:00005218       ??_C@_03OOEBGOEH@cut?$AA@  31613218     LipSync.obj
 0002:0000521c       ??_C@_02OEIPGGFF@ah?$AA@   3161321c     LipSync.obj
 0002:00005220       ??_C@_03PFGOGFOL@cat?$AA@  31613220     LipSync.obj
 0002:00005224       ??_C@_02FBCBBIBI@ae?$AA@   31613224     LipSync.obj
 0002:00005228       ??_C@_06OIIIAOPN@father?$AA@ 31613228     LipSync.obj
 0002:00005230       ??_C@_02DFENNNBM@aa?$AA@   31613230     LipSync.obj
 0002:00005234       ??_C@_0BF@EPOMEAHF@Silence?5?$CIunderscore?$CJ?$AA@ 31613234     LipSync.obj
 0002:0000524c       ??_C@_01IDAFKMJL@_?$AA@    3161324c     LipSync.obj
 0002:00005250       ??_C@_0CE@DOKFPDIK@Sentence?5terminator?5?$CIquestion?5ma@ 31613250     LipSync.obj
 0002:00005274       ??_C@_01OGPIMHDM@?$DP?$AA@ 31613274     LipSync.obj
 0002:00005278       ??_C@_0BN@EKGECIKE@Sentence?5terminator?5?$CIperiod?$CJ?$AA@ 31613278     LipSync.obj
 0002:00005298       ??_C@_0BM@CMAJFDHL@Sentence?5terminator?5?$CIcomma?$CJ?$AA@ 31613298     LipSync.obj
 0002:000052b4       ??_C@_01HNPIGOCE@?$CG?$AA@ 316132b4     LipSync.obj
 0002:000052b8       ??_C@_0BE@PPDGDKBH@Sentence?5terminator?$AA@ 316132b8     LipSync.obj
 0002:000052cc       ??_C@_01DCLJPIOD@?$CB?$AA@ 316132cc     LipSync.obj
 0002:000052d0       ??_C@_08DMNNLLJJ@syllable?$AA@ 316132d0     LipSync.obj
 0002:000052dc       ??_C@_01JOAMLHOP@?9?$AA@   316132dc     LipSync.obj
 0002:000052e4       ??_7IFacialSentence@@6B@   316132e4     LipSync.obj
 0002:000052e4       ??_7ISkin@@6B@             316132e4     ModelSkin.obj
 0002:00005318       ??_7?$_reference_target@H@@6B@ 31613318     LipSync.obj
 0002:0000531c       __real@447a0000            3161331c     LipSync.obj
 0002:00005320       ??_C@_07OKOCHHP@?$CFs?3?$CF?42f?$AA@ 31613320     LipSync.obj
 0002:00005328       ??_7CFacialSentence@@6B?$_reference_target@H@@@ 31613328     LipSync.obj
 0002:0000532c       ??_7CFacialSentence@@6BIFacialSentence@@@ 3161332c     LipSync.obj
 0002:00005360       ??_7CPhonemesLibrary@@6B@  31613360     LipSync.obj
 0002:00005370       ??_C@_08BHPDILBD@?$CFd?3?$CFd?3?$CFs?$AA@ 31613370     LipSync.obj
 0002:0000537c       ??_C@_03DBKJMAGF@End?$AA@  3161337c     LipSync.obj
 0002:00005380       ??_C@_05FHMJPCKA@Start?$AA@ 31613380     LipSync.obj
 0002:00005388       ??_C@_04IGEPOOPB@Word?$AA@ 31613388     LipSync.obj
 0002:00005390       ??_C@_08PFDKLHBC@Phonemes?$AA@ 31613390     LipSync.obj
 0002:0000539c       ??_C@_05MOCOKHFB@Words?$AA@ 3161339c     LipSync.obj
 0002:000053a4       ??_C@_04OJAHODMC@Text?$AA@ 316133a4     LipSync.obj
 0002:000053b0       ??_7CFeetPoseRestore@@6B@  316133b0     FeetLock.obj
 0002:000053d0       ??_7CFeetPoseStore@@6B@    316133d0     FeetLock.obj
 0002:000053f0       ??_7CFactory@CFeetPoseStore@@6B@ 316133f0     FeetLock.obj
 0002:00005408       ??_C@_0CE@FIJHOGBC@AnimationPoseModifier_FeetPoseSt@ 31613408     FeetLock.obj
 0002:00005430       ?cid@?1??GetClassID@CFactory@CFeetPoseStore@@UBEABUCryGUID@@XZ@4U4@B 31613430     FeetLock.obj
 0002:00005440       ??_7CFactory@CFeetPoseRestore@@6B@ 31613440     FeetLock.obj
 0002:00005458       ??_C@_0CG@OHIIAMBF@AnimationPoseModifier_FeetPoseRe@ 31613458     FeetLock.obj
 0002:00005480       ?cid@?1??GetClassID@CFactory@CFeetPoseRestore@@UBEABUCryGUID@@XZ@4U4@B 31613480     FeetLock.obj
 0002:00005490       ??_C@_08OKNEMAIJ@RgtLeg01?$AA@ 31613490     GroundAlignment.obj
 0002:0000549c       ??_C@_08ECHMFJPE@LftLeg01?$AA@ 3161349c     GroundAlignment.obj
 0002:000054ac       ??_C@_06DCFKOEPA@R?5Heel?$AA@ 316134ac     GroundAlignment.obj
 0002:000054b4       ??_C@_06FLLADGD@L?5Heel?$AA@ 316134b4     GroundAlignment.obj
 0002:000054c0       ?iid@?1??IID@IAnimationGroundAlignment@@CAABUCryGUID@@XZ@4U3@B 316134c0     GroundAlignment.obj
 0002:000054d0       ??_7CGroundAlignment@@6B@  316134d0     GroundAlignment.obj
 0002:000054f4       ??_7CFactory@CGroundAlignment@@6B@ 316134f4     GroundAlignment.obj
 0002:0000550c       ??_C@_0CG@DDGGKLBL@AnimationPoseModifier_GroundAlig@ 3161350c     GroundAlignment.obj
 0002:00005538       ?cid@?1??GetClassID@CFactory@CGroundAlignment@@UBEABUCryGUID@@XZ@4U4@B 31613538     GroundAlignment.obj
 0002:0000554c       ??_7CLimbIk@@6B@           3161354c     LimbIk.obj
 0002:0000556c       ??_7CFactory@CLimbIk@@6B@  3161356c     LimbIk.obj
 0002:00005588       ?cid@?1??GetClassID@CFactory@CLimbIk@@UBEABUCryGUID@@XZ@4U4@B 31613588     LimbIk.obj
 0002:000055a0       ??_7CPoseBlenderAim@@6B@   316135a0     PoseBlenderAim.obj
 0002:000055e4       ??_C@_0DF@INPOJLLI@CryAnimation?3?5No?5weapon?9bone?5spe@ 316135e4     PoseBlenderAim.obj
 0002:0000561c       ??_C@_0CL@CGDELOPI@CryAnimation?3?5No?5AimIK?9Setup?5for@ 3161361c     PoseBlenderAim.obj
 0002:00005648       ??_7CFactory@CPoseBlenderAim@@6B@ 31613648     PoseBlenderAim.obj
 0002:00005660       ?cid@?1??GetClassID@CFactory@CPoseBlenderAim@@UBEABUCryGUID@@XZ@4U4@B 31613660     PoseBlenderAim.obj
 0002:00005674       __real@3f3504f3            31613674     PoseBlenderLook.obj
 0002:00005678       ??_7CPoseBlenderLook@@6B@  31613678     PoseBlenderLook.obj
 0002:000056bc       ??_C@_0DF@EGJAADOE@CryAnimation?3?5Right?5Eyeball?5atta@ 316136bc     PoseBlenderLook.obj
 0002:000056f4       ??_C@_0DE@NBIDDDLC@CryAnimation?3?5Left?5Eyeball?5attac@ 316136f4     PoseBlenderLook.obj
 0002:00005728       ??_C@_0DD@CIEFHBDA@CryAnimation?3?5No?5look?9bone?5speci@ 31613728     PoseBlenderLook.obj
 0002:0000575c       ??_C@_0CM@LFPKMBEO@CryAnimation?3?5No?5LookIK?9Setup?5fo@ 3161375c     PoseBlenderLook.obj
 0002:00005788       ??_C@_0CF@OOHODMO@EyeRight?3?5?$CFf?5?$CFf?5?$CFf?5?$CFf?5?5m_IKBlend@ 31613788     PoseBlenderLook.obj
 0002:000057b0       ??_C@_0CE@DNOEJCJM@EyeLeft?3?5?$CFf?5?$CFf?5?$CFf?5?$CFf?5?5m_IKBlend?3@ 316137b0     PoseBlenderLook.obj
 0002:000057d4       ??_7CFactory@CPoseBlenderLook@@6B@ 316137d4     PoseBlenderLook.obj
 0002:000057f0       ?cid@?1??GetClassID@CFactory@CPoseBlenderLook@@UBEABUCryGUID@@XZ@4U4@B 316137f0     PoseBlenderLook.obj
 0002:00005804       __real@bf7d70a4            31613804     PoseModifierHelper.obj
 0002:00005808       __real@461c4000            31613808     PoseModifierHelper.obj
 0002:0000580c       __real@3fa00000            3161380c     PoseModifierHelper.obj
 0002:00005810       __real@3f7fff58            31613810     PoseModifierHelper.obj
 0002:00005814       __real@2edbe6ff            31613814     PoseModifierHelper.obj
 0002:00005818       __real@bf7ae148            31613818     PoseModifierHelper.obj
 0002:0000581c       __real@3e947ae1            3161381c     PoseModifierHelper.obj
 0002:00005820       __real@bf666666            31613820     PoseModifierHelper.obj
 0002:00005824       __real@3f733333            31613824     PoseModifierHelper.obj
 0002:00005828       __real@3f0ccccd            31613828     PoseModifierHelper.obj
 0002:00005830       ??_7CRecoil@PoseModifier@@6B@ 31613830     Recoil.obj
 0002:00005850       ??_7CFactory@CRecoil@PoseModifier@@6B@ 31613850     Recoil.obj
 0002:00005868       ?cid@?1??GetClassID@CFactory@CRecoil@PoseModifier@@UBEABUCryGUID@@XZ@4U5@B 31613868     Recoil.obj
 0002:0000587c       ??_C@_0DM@PBEMGCIH@CryAnimation?3?5Command?9Buffer?5Inv@ 3161387c     Command_Buffer.obj
 0002:000058b8       ??_C@_0CB@ODGLIDOL@PartPose_FETCH_ADD?3?5w?3?$CFf?5t?3?$CFf?5?$CFs@ 316138b8     Command_Buffer.obj
 0002:000058dc       ??_C@_0CB@BFCOJGGE@BasePose_FETCH_ADD?3?5w?3?$CFf?5t?3?$CFf?5?$CFs@ 316138dc     Command_Buffer.obj
 0002:00005900       ??_C@_0BA@INCLFOHP@State_JOINTMASK?$AA@ 31613900     Command_Buffer.obj
 0002:00005910       ??_C@_0CB@BDNGEMDG@PartAnim_FETCH_ADD?3?5w?3?$CFf?5t?3?$CFf?5?$CFs@ 31613910     Command_Buffer.obj
 0002:00005934       ??_C@_0BB@LGPJFNKO@Proc_POSEMOD?3?5?$CFs?$AA@ 31613934     Command_Buffer.obj
 0002:00005948       ??_C@_0BA@FCLDIGAF@BaseAnim_USCALE?$AA@ 31613948     Command_Buffer.obj
 0002:00005958       ??_C@_0BD@GAMGPJMH@BaseAnim_NORMALIZE?$AA@ 31613958     Command_Buffer.obj
 0002:0000596c       ??_C@_0BC@HPHFEMMB@BaseAnim_COPY_ADD?$AA@ 3161396c     Command_Buffer.obj
 0002:00005980       ??_C@_0CB@OFJDFJLJ@BaseAnim_FETCH_ADD?3?5w?3?$CFf?5t?3?$CFf?5?$CFs@ 31613980     Command_Buffer.obj
 0002:000059a4       ??_C@_0BE@MKAOLHMH@BaseAnim_CLEAR_ROOT?$AA@ 316139a4     Command_Buffer.obj
 0002:000059b8       ??_C@_0BG@BNPBJNAD@BaseAnim_CLEAR_BUFFER?$AA@ 316139b8     Command_Buffer.obj
 0002:000059d0       ??_C@_0CI@DDCDLAMD@m_CommandBufferCounter?5?$CFd?5?5Comma@ 316139d0     Command_Buffer.obj
 0002:000059f8       __real@3c75c28f            316139f8     Command_Buffer.obj
 0002:00005a00       ??_C@_0EI@GABFMADP@LHand_IKTarget?3?5name?3?5?$CFs?5?5rot?3?5?$CI@ 31613a00     Command_Buffer.obj
 0002:00005a48       ??_C@_0BJ@OGGKAMHL@ProcessAnimationDrivenIk?$AA@ 31613a48     Command_Buffer.obj
 0002:00005a64       ??_C@_0BK@OJHNFMAM@Command?3?3CBuffer?3?3Execute?$AA@ 31613a64     Command_Buffer.obj
 0002:00005a84       ??_C@_09NEDHICLM@cryMemcpy?$AA@ 31613a84     Command_Commands.obj
 0002:00005a90       ??_C@_0EF@DIMOALKN@CryAnimation?3?5Asset?5Not?5Loaded?3?5@ 31613a90     Command_Commands.obj
 0002:00005ad8       ??_C@_0DJ@GIJGEOJH@illegal?5index?5in?5RSingleEvaluati@ 31613ad8     Command_Commands.obj
 0002:00005b14       ??_7IAnimationPoseData@@6B@ 31613b14     Skeleton.obj
 0002:00005b3c       ??_7CPoseData@Skeleton@@6B@ 31613b3c     Skeleton.obj
 0002:00005b64       ??_C@_0BE@BNBLBEIO@Character?5Pose?5Data?$AA@ 31613b64     Skeleton.obj
 0002:00005b78       ??_C@_0BL@IJJIPNKE@Character?5Pose?5Data?5Cloned?$AA@ 31613b78     Skeleton.obj
 0002:00005b94       ??_C@_06HOPIODND@effect?$AA@ 31613b94     AnimEventLoader.obj
 0002:00005b9c       ??_C@_04MEMAJGDJ@name?$AA@ 31613b9c     AnimEventLoader.obj
 0002:00005ba4       ??_C@_09KCBFNMAJ@animation?$AA@ 31613ba4     AnimEventLoader.obj
 0002:00005bb0       ??_C@_0L@OBDHBINM@AnimEvents?$AA@ 31613bb0     AnimEventLoader.obj
 0002:00005bbc       ??_C@_06HPGEIPLA@?$DMnull?$DO?$AA@ 31613bbc     CharacterManager.obj
 0002:00005bc4       ??_C@_07KAALEJHI@?$DMlocal?$DO?$AA@ 31613bc4     CharacterManager.obj
 0002:00005bd0       ??_7ICharacterManager@@6B@ 31613bd0     CharacterManager.obj
 0002:00005c88       ??_C@_04PBAHLACE@File?$AA@ 31613c88     CharacterManager.obj
 0002:00005c90       ??_C@_05NFIJOKEG@Model?$AA@ 31613c90     CharacterManager.obj
 0002:00005c98       ??_C@_0DH@OHPBLIHM@CryAnimation?3?5character?9definiti@ 31613c98     CharacterManager.obj
 0002:00005cd0       ??_C@_0BE@OLDKOMJJ@CharacterDefinition?$AA@ 31613cd0     CharacterManager.obj
 0002:00005ce4       ??_C@_0BE@NPEDKBDG@Character?5instances?$AA@ 31613ce4     CharacterManager.obj
 0002:00005cf8       __real@42000000            31613cf8     CharacterManager.obj
 0002:00005cfc       ??_C@_0DG@FKBAHALH@nSkinningPoolSize?3?5?$CFd?5?5?5nTotalSk@ 31613cfc     CharacterManager.obj
 0002:00005d34       ??_C@_0BO@LHHDLBCA@TotalModelMemory?5?$CIMem?3?5?$CF4dKB?$CJ?$AA@ 31613d34     CharacterManager.obj
 0002:00005d58       ??_C@_0EF@KLPBKCHC@nTotalModelSkeletonMemory?3?5?5?$CF4dK@ 31613d58     CharacterManager.obj
 0002:00005da0       ??_C@_0BG@NGMNAJGJ@nAnimationSet?3?5?5?$CF4dKB?$AA@ 31613da0     CharacterManager.obj
 0002:00005db8       ??_C@_0DO@PPBPJBDK@nTotalAttachmentMemory?3?5?5?$CF4dKB?5?5@ 31613db8     CharacterManager.obj
 0002:00005df8       ??_C@_0FK@NEDBHHJB@?9?9?9?9?9?9?9?9?9?9?9?9?9?9?9?9?9?9?9?9?9?9?9?9?9?9?9?9?9?9?9?9@ 31613df8     CharacterManager.obj
 0002:00005e58       ??_C@_0EJ@GCNGJGJK@SKINInstancesCounter?3?$CF3d?5?$CIMem?3?5?$CF@ 31613e58     CharacterManager.obj
 0002:00005ea4       ??_C@_0DI@OOFGLCFP@Model?3?5?$CF3d?5?5Skin?3?5?$CF2d?5imem?3?5?$CF7d?5@ 31613ea4     CharacterManager.obj
 0002:00005ee0       ??_C@_0FC@DGAPPCGC@Model?3?5?$CF3d?5?5?5Skin?3?5?$CF2d?5imem?3?5?$CF7d@ 31613ee0     CharacterManager.obj
 0002:00005f38       ??_C@_0EJ@GJGEHJGL@SKELInstancesCounter?3?$CF3d?5?$CIMem?3?5?$CF@ 31613f38     CharacterManager.obj
 0002:00005f88       ??_C@_0EE@PDECEPPA@Model?3?5?$CF3d?5?5?5Skel?3?5?$CF2d?5?5imem?3?5?$CF7@ 31613f88     CharacterManager.obj
 0002:00005fd0       ??_C@_0ED@JOJCFEF@Model?3?5?$CF3d?5?5?5Skel?3?5?$CF2d?5imem?3?5?$CF7d@ 31613fd0     CharacterManager.obj
 0002:00006014       ??_C@_0BN@PLJJFMHL@CryAnimation?3?5mem?5corruption?$AA@ 31614014     CharacterManager.obj
 0002:00006034       ??_C@_0CP@PHGEPJJL@No?3?$CF04d?5DBA?3?5?$CF08x?5p?3?$CF02x?5q?3?$CF02x?5@ 31614034     CharacterManager.obj
 0002:00006064       ??_C@_02BKFDOEMK@wt?$AA@   31614064     CharacterManager.obj
 0002:00006068       ??_C@_0BH@FONECNPF@No?3?$CF04d?5use?3?$CF05d?5?5?5?$CFs?6?$AA@ 31614068     CharacterManager.obj
 0002:00006080       ??_C@_07OANIALAE@chr?4pak?$AA@ 31614080     CharacterManager.obj
 0002:00006088       ??_C@_0DN@FEBKIFHJ@?$DN?$DN?$DN?$DN?$DN?5Finished?5Preloading?5?$CFd?5Cha@ 31614088     CharacterManager.obj
 0002:000060c8       ??_C@_0CB@FCAIPGCG@?$DN?$DN?$DN?$DN?$DN?5Preloading?5Characters?5?$DN?$DN?$DN?$DN@ 316140c8     CharacterManager.obj
 0002:000060ec       ??_C@_0M@JKINLGFJ@Preload?5CHR?$AA@ 316140ec     CharacterManager.obj
 0002:000060f8       ??_C@_0CD@PDHBIC@CharacterManager?3?3PreloadModelsC@ 316140f8     CharacterManager.obj
 0002:0000611c       ??_C@_0CE@BFGBHKLO@CharacterManager?3?3RegisterModelS@ 3161411c     CharacterManager.obj
 0002:00006140       ??_C@_0CE@COENOBFI@CharacterManager?3?3RegisterModelS@ 31614140     CharacterManager.obj
 0002:00006164       ??_C@_0DA@INOLIAEE@CryAnimation?3?5Reloading?5CHRPARAM@ 31614164     CharacterManager.obj
 0002:00006194       ??_C@_02JDPG@rb?$AA@       31614194     CharacterManager.obj
 0002:00006198       ??_C@_0DH@NAEANFNA@?$DN?$DN?$DN?$DN?$DN?5Finished?5Preloading?5?$CFd?5CGA@ 31614198     CharacterManager.obj
 0002:000061d0       ??_C@_07JDNCALNI@cga?4pak?$AA@ 316141d0     CharacterManager.obj
 0002:000061d8       ??_C@_0M@ECJONIAD@e_StreamCgf?$AA@ 316141d8     CharacterManager.obj
 0002:000061e4       ??_C@_0BL@FJEOOLEB@?$DN?$DN?$DN?$DN?$DN?5Preloading?5CGAs?5?$DN?$DN?$DN?$DN?$AA@ 316141e4     CharacterManager.obj
 0002:00006200       ??_C@_0M@PADOLAPG@Preload?5CGA?$AA@ 31614200     CharacterManager.obj
 0002:0000620c       ??_C@_0CD@GKEAHHCN@CharacterManager?3?3PreloadModelsC@ 3161420c     CharacterManager.obj
 0002:00006230       ??_C@_0BC@MGOEEFL@Animation?5Context?$AA@ 31614230     CharacterManager.obj
 0002:00006244       ??_C@_0BE@KJDJFMJA@STL?5Allocator?5Waste?$AA@ 31614244     CharacterManager.obj
 0002:00006258       ??_C@_0L@HKIBOMFD@Model?5Data?$AA@ 31614258     CharacterManager.obj
 0002:00006264       ??_C@_0BB@KDBPHKIO@Facial?5Animation?$AA@ 31614264     CharacterManager.obj
 0002:00006278       ??_7CharacterDefinition@@6B@ 31614278     CharacterManager.obj
 0002:00006280       ??_C@_0EN@FCGGFBPH@CryAnimation?3?5no?5valid?5character@ 31614280     CharacterManager.obj
 0002:000062d0       ??_C@_0CA@DDELBMIL@CharacterManager?3?3LoadModelSKIN?$AA@ 316142d0     CharacterManager.obj
 0002:000062f0       ??_C@_0L@EMODJLOD@Characters?$AA@ 316142f0     CharacterManager.obj
 0002:000062fc       __real@be800000            316142fc     CharacterManager.obj
 0002:00006300       ??_C@_0BK@GOFBGCI@AnimStats_NotUsed_LMG?4txt?$AA@ 31614300     CharacterManager.obj
 0002:0000631c       ??_C@_0BH@KNBMFCMI@AnimStats_Used_LMG?4txt?$AA@ 3161431c     CharacterManager.obj
 0002:00006334       ??_C@_0BK@NDDJLNFF@AnimStats_NotUsed_CAF?4txt?$AA@ 31614334     CharacterManager.obj
 0002:00006350       ??_C@_0BH@HIMAPJLF@AnimStats_Used_CAF?4txt?$AA@ 31614350     CharacterManager.obj
 0002:00006368       ??_C@_0DD@FOOMPIDA@Anim?3?$CI?$CFd?$CJ?5?5Force?3?$CI?$CFd?$CJ?5?5Visible?3?$CI@ 31614368     CharacterManager.obj
 0002:0000639c       ??_C@_0CL@PHOJHIIJ@Instances?5with?5?8Force?5Skeleton?5U@ 3161439c     CharacterManager.obj
 0002:000063c8       ??_C@_0BE@IOBGFPOI@SkeletonUpdates?3?5?$CFd?$AA@ 316143c8     CharacterManager.obj
 0002:000063dc       ??_C@_0BF@GGOPHLKB@AnimationUpdates?3?5?$CFd?$AA@ 316143dc     CharacterManager.obj
 0002:000063f4       ??_C@_0DE@NJMNECHC@nAnimsPerFrame?3?5?$CF4d?5?5nAnimsMax?3?5@ 316143f4     CharacterManager.obj
 0002:00006428       ??_C@_0BD@GAAEDFAB@arrModelCache?3?5?$CF4d?$AA@ 31614428     CharacterManager.obj
 0002:0000643c       ??_C@_0BM@MAHCAFAA@arrModelCache_CharEdit?3?5?$CF4d?$AA@ 3161443c     CharacterManager.obj
 0002:00006458       ??_C@_0BJ@CDDMONIK@CharacterManager?3?3Update?$AA@ 31614458     CharacterManager.obj
 0002:00006474       ??_7CAnimationManager@@6B@ 31614474     CharacterManager.obj
 0002:00006490       ??_C@_0FF@MKPLPECI@m_arrModelCacheSKEL?5is?5supposed?5@ 31614490     CharacterManager.obj
 0002:000064e8       ??_C@_0BN@NPJPGGNA@m_arrModelCacheSKEL?$FL?$CFi?$FN?5?$DN?5?$CFs?$AA@ 316144e8     CharacterManager.obj
 0002:00006508       ??_C@_0FF@JBCJLFOE@m_arrModelCacheSKIN?5is?5supposed?5@ 31614508     CharacterManager.obj
 0002:00006560       ??_C@_0BN@ICPJJCJA@m_arrModelCacheSKIN?$FL?$CFi?$FN?5?$DN?5?$CFs?$AA@ 31614560     CharacterManager.obj
 0002:00006580       ??_C@_0DM@MHCCPBPK@CharacterManager?3CleanModelCache@ 31614580     CharacterManager.obj
 0002:000065c0       ??_C@_0IA@BDKJANBB@?$CKERROR?$CK?5CharacterManager?3?5?$CFu?5bod@ 316145c0     CharacterManager.obj
 0002:00006640       ??_7CharacterManager@@6B@  31614640     CharacterManager.obj
 0002:000066f8       ??_C@_0EK@FKCNNNGO@CryAnimation?3?5Assets?5has?5no?5cont@ 316146f8     CharacterManager.obj
 0002:00006748       ??_C@_0ED@MKCPEGIJ@CryAnimation?3?5m_arrController?5re@ 31614748     CharacterManager.obj
 0002:00006790       ??_C@_0FA@NJADGAO@CryAnimation?3?5CRC32?5Invalid?$CB?5Mos@ 31614790     CharacterManager.obj
 0002:000067e0       ??_C@_0CP@INOEFHAC@Badly?5exported?5animation?9asset?3?5@ 316147e0     CharacterManager.obj
 0002:00006810       ??_C@_0DO@NPPJMPBB@CryAnimation?3?5the?5list?5with?5Glob@ 31614810     CharacterManager.obj
 0002:00006850       ??_C@_0CM@LCFLJELM@CharacterManager?3?3LoadAnimationI@ 31614850     CharacterManager.obj
 0002:0000687c       ??_C@_0BD@HNEEBJGG@InternalPara1D?4LMG?$AA@ 3161487c     CharacterManager.obj
 0002:00006890       ??_C@_03IGKKBKKP@CDF?$AA@  31614890     CharacterManager.obj
 0002:00006894       ??_C@_0BK@JFFBIKHL@CharacterManager?3?3LoadCDF?$AA@ 31614894     CharacterManager.obj
 0002:000068b0       ??_C@_0DB@BLBFJBND@CryAnimation?3?5character?9definiti@ 316148b0     CharacterManager.obj
 0002:000068e4       __real@3c656042            316148e4     CharacterManager.obj
 0002:000068e8       ??_C@_0DH@NELFFEPE@?$DN?$DN?$DN?$DN?$DN?5Finished?5Preloading?5?$CFd?5CDF@ 316148e8     CharacterManager.obj
 0002:00006920       ??_C@_04BCMGGOLH@?4cdf?$AA@ 31614920     CharacterManager.obj
 0002:00006928       ??_C@_0BL@GKAGNOJN@?$DN?$DN?$DN?$DN?$DN?5Preloading?5CDFs?5?$DN?$DN?$DN?$DN?$AA@ 31614928     CharacterManager.obj
 0002:00006944       ??_C@_0M@LNDJJIGI@Preload?5CDF?$AA@ 31614944     CharacterManager.obj
 0002:00006950       ??_C@_0CD@CHEHFPLD@CharacterManager?3?3PreloadModelsC@ 31614950     CharacterManager.obj
 0002:00006974       ??_C@_0BI@HJHCIGLK@CDF?4?5Finish?4?5Memstat?5?$CFi?$AA@ 31614974     CharacterManager.obj
 0002:0000698c       ??_C@_0CD@BPIDLBGP@Couldn?8t?5create?5base?9character?3?5@ 3161498c     CharacterManager.obj
 0002:000069b0       ??_C@_0EG@MOMOBCLL@CryAnimation?3?5base?9character?5mus@ 316149b0     CharacterManager.obj
 0002:000069f8       ??_C@_0BK@KNHFHPBF@CDF?5?$CFs?4?5Start?4?5Memstat?5?$CFi?$AA@ 316149f8     CharacterManager.obj
 0002:00006a14       ??_C@_0CK@IOKDEHCE@CharacterManager?3?3LoadCharacterD@ 31614a14     CharacterManager.obj
 0002:00006a40       ??_C@_0BD@KHKNKNFF@Preload?5Characters?$AA@ 31614a40     CharacterManager.obj
 0002:00006a54       ??_C@_0CF@NAMGPPIA@CharacterManager?3?3PreloadLevelMo@ 31614a54     CharacterManager.obj
 0002:00006a7c       ??_C@_0CI@JGBNBLAB@Badly?5exported?5aim?9pose?3?5flags?3?5@ 31614a7c     CharacterManager.obj
 0002:00006aa4       ??_C@_0CJ@JOOFGFDA@CharacterManager?3?3LoadAnimationI@ 31614aa4     CharacterManager.obj
 0002:00006ad0       ??_C@_0BK@HHIKGHID@animations?1animations?4img?$AA@ 31614ad0     CharacterManager.obj
 0002:00006aec       ??_C@_0CB@NMEJACKB@animations?1DirectionalBlends?4img@ 31614aec     CharacterManager.obj
 0002:00006b10       ??_C@_0GM@HDENCGKJ@CryAnimation?3FetchPlaceHolderCha@ 31614b10     CharacterManager.obj
 0002:00006b80       ??_C@_0GM@DALBFNHC@CryAnimation?3FetchPlaceHolderCha@ 31614b80     CharacterManager.obj
 0002:00006bf0       ??_C@_0GO@DIGNOCFO@CryAnimation?3FetchPlaceHolderCha@ 31614bf0     CharacterManager.obj
 0002:00006c60       ??_C@_0GM@EHJLEEIM@CryAnimation?3FetchPlaceHolderCha@ 31614c60     CharacterManager.obj
 0002:00006cd0       ??_C@_0GI@BKIDNJII@CryAnimation?3FetchPlaceHolderCha@ 31614cd0     CharacterManager.obj
 0002:00006d38       ??_C@_0BF@COJDDOIE@Instances?5Memstat?5?$CFi?$AA@ 31614d38     CharacterManager.obj
 0002:00006d50       ??_C@_0BP@OLGKDIDE@InitCGAInstance?5?$CFs?4?5Memstat?5?$CFi?$AA@ 31614d50     CharacterManager.obj
 0002:00006d70       ??_C@_0P@DIBCHGHO@Loading?5CGA?5?$CFs?$AA@ 31614d70     CharacterManager.obj
 0002:00006d80       ??_C@_0CE@KMAAOPHC@CharacterManager?3?3CreateCGAInsta@ 31614d80     CharacterManager.obj
 0002:00006da4       ??_C@_09EEDOMAPA@chrparams?$AA@ 31614da4     CharacterManager.obj
 0002:00006db0       ??_C@_0CF@KCPFIJAI@CharacterManager?3?3CreateSKELInst@ 31614db0     CharacterManager.obj
 0002:00006dd8       ??_C@_0CA@IGHIHGN@CharacterManager?3?3LoadModelSKEL?$AA@ 31614dd8     CharacterManager.obj
 0002:00006df8       ??_C@_0DD@LHBEEHJA@CharacterManager?3?3FetchPlaceHold@ 31614df8     CharacterManager.obj
 0002:00006e30       ??_C@_0FI@LOPBNJDN@CPF?5file?5allowed?5for?5use?5only?5in@ 31614e30     CharacterManager.obj
 0002:00006e88       ??_C@_04BHIIPFEC@base?$AA@ 31614e88     CharacterManager.obj
 0002:00006e90       ??_C@_0EB@CIMONDIL@CryAnimation?3?5no?5valid?5character@ 31614e90     CharacterManager.obj
 0002:00006ed4       ??_C@_03JAHONMHP@cpf?$AA@  31614ed4     CharacterManager.obj
 0002:00006ed8       ??_C@_0DM@JCMOKGDP@CryAnimation?3PrefetchCharacterRe@ 31614ed8     CharacterManager.obj
 0002:00006f14       ??_C@_04DOHGOLCD@$lod?$AA@ 31614f14     LoaderCGA.obj
 0002:00006f1c       ??_C@_0CK@PIMHCPOB@Animation?5could?5not?5be?5read?5for?5@ 31614f1c     LoaderCGA.obj
 0002:00006f48       ??_7IController@@6B@       31614f48     LoaderCGA.obj
 0002:00006f84       ??_C@_0CC@LPDMFHBH@indices?5and?1or?5positions?5are?5NUL@ 31614f84     LoaderCGA.obj
 0002:00006fa8       ??_C@_0CO@BKPCLEDN@faces?5are?5too?5small?5or?5have?5stre@ 31614fa8     LoaderCGA.obj
 0002:00006fd8       ??_C@_0BK@MMDPIIJG@bad?5vertex?5index?5detected?$AA@ 31614fd8     LoaderCGA.obj
 0002:00006ff4       ??_C@_0BG@BDLCLLKE@bad?5number?5of?5indices?$AA@ 31614ff4     LoaderCGA.obj
 0002:0000700c       ??_C@_0BN@KFBFLIPO@texture?5coordinates?5are?5NULL?$AA@ 3161500c     LoaderCGA.obj
 0002:0000702c       ??_C@_0BC@HPECBPJJ@vertex?5count?5is?50?$AA@ 3161502c     LoaderCGA.obj
 0002:00007040       ??_C@_0BB@IGNNBDOM@index?5count?5is?50?$AA@ 31615040     LoaderCGA.obj
 0002:00007054       ??_C@_0BB@ELKAEEPN@missing?5vertices?$AA@ 31615054     LoaderCGA.obj
 0002:00007068       ??_C@_0BM@IFOLHLJG@missing?5texture?5coordinates?$AA@ 31615068     LoaderCGA.obj
 0002:00007084       ??_C@_0CB@HMHDCALB@missing?5or?5bad?5indices?5in?5subset@ 31615084     LoaderCGA.obj
 0002:000070a8       ??_C@_0BA@PAFHHGGK@missing?5indices?$AA@ 316150a8     LoaderCGA.obj
 0002:000070b8       ??_C@_0BE@KHFBNAHK@subset?5index?5is?5bad?$AA@ 316150b8     LoaderCGA.obj
 0002:000070cc       ??_C@_0L@CPDIKD@L?5UpperArm?$AA@ 316150cc     LoaderCGA.obj
 0002:000070d8       ??_C@_0L@PMKPNHGO@R?5UpperArm?$AA@ 316150d8     LoaderCGA.obj
 0002:000070e4       ??_C@_07LDJNDMEG@L?5Thigh?$AA@ 316150e4     LoaderCGA.obj
 0002:000070ec       ??_C@_07NKKMBPFP@R?5Thigh?$AA@ 316150ec     LoaderCGA.obj
 0002:000070f4       ??_7?$TSpline@UTCBAngAxisKey@spline@@VHermitBasis@2@@spline@@6B@ 316150f4     LoaderCGA.obj
 0002:00007104       ??_7TCBAngleAxisSpline@spline@@6B@ 31615104     LoaderCGA.obj
 0002:00007118       __real@3f7ff972            31615118     LoaderCGA.obj
 0002:0000711c       __real@40c90fbb            3161511c     LoaderCGA.obj
 0002:00007120       __real@3ea2f983            31615120     LoaderCGA.obj
 0002:00007124       __real@40490fb1            31615124     LoaderCGA.obj
 0002:00007128       ??_7CControllerTCB@@6B@    31615128     LoaderCGA.obj
 0002:00007164       ??_C@_0BE@OMJLCPFJ@Should?5never?5happen?$AA@ 31615164     LoaderCGA.obj
 0002:00007178       ??_C@_0N@HOBCLLKA@CharacterCGA?$AA@ 31615178     LoaderCGA.obj
 0002:00007188       ??_C@_0CG@HICNHCLM@Cannot?5be?5merged?5to?5one?5skin?5ins@ 31615188     LoaderCGA.obj
 0002:000071b0       __real@3bcccccd            316151b0     LoaderCGA.obj
 0002:000071b4       ??_C@_0BM@PFEDBNEJ@Failed?5to?5load?5ANM?9file?3?5?$CFs?$AA@ 316151b4     LoaderCGA.obj
 0002:000071d0       ??_C@_0L@KIBGKOJH@animevents?$AA@ 316151d0     LoaderCGA.obj
 0002:000071dc       ??_C@_04BEANKMFM@?4caf?$AA@ 316151dc     LoaderCGA.obj
 0002:000071e4       ??_C@_04FGKMPKCB@?4anm?$AA@ 316151e4     LoaderCGA.obj
 0002:000071ec       ??_C@_02FNAGIBCP@?4?$CK?$AA@ 316151ec     LoaderCGA.obj
 0002:000071f0       ??_C@_02IDFIDEI@_?$CK?$AA@ 316151f0     LoaderCGA.obj
 0002:000071f4       ??_C@_0BN@DPJAHDFM@CryCGALoader?3?3LoadAnimations?$AA@ 316151f4     LoaderCGA.obj
 0002:00007214       ??_C@_07MCAEODGB@Default?$AA@ 31615214     LoaderCGA.obj
 0002:0000721c       ??_C@_0BK@LLFPEIEJ@Failed?5to?5load?5CGA?9Object?$AA@ 3161521c     LoaderCGA.obj
 0002:00007238       ??_C@_03MLKNDCDB@CGA?$AA@  31615238     LoaderCGA.obj
 0002:00007240       ??_C@_0CC@GEHLENNH@CryCHRLoader?3?3ReuseAnimationFile@ 31615240     LoaderCHR.obj
 0002:00007264       ??_C@_0L@HNGMIHEN@animations?$AA@ 31615264     LoaderCHR.obj
 0002:00007270       ??_C@_0M@HJLLEEH@?1animations?$AA@ 31615270     LoaderCHR.obj
 0002:00007280       ??_C@_0FE@LAHILELP@CryAnimation?3?5Matrix?9Tangents?5ar@ 31615280     LoaderCHR.obj
 0002:000072d4       ??_C@_0DL@PNJAKJAP@Facial?5Effector?5Library?5?$CFs?5not?5f@ 316152d4     LoaderCHR.obj
 0002:00007310       ??_C@_0BK@HAILMHKA@CryCHRLoader?3?3LoadFaceLib?$AA@ 31615310     LoaderCHR.obj
 0002:0000732c       ??_C@_0BP@DMCHIPGL@Physics?3?5No?5material?5in?5lod?5?$CFd?$AA@ 3161532c     LoaderCHR.obj
 0002:0000734c       ??_C@_0CO@KOEOJBCH@Physics?3?5Failed?5to?5create?5phys?5m@ 3161534c     LoaderCHR.obj
 0002:00007380       ??_C@_0EL@JHAFEIHE@Animation?5?$CIcaf?$CJ?5file?5?$CC?$CFs?$CC?5could?5@ 31615380     LoaderCHR.obj
 0002:000073cc       ??_C@_04JDMOLDHM@comb?$AA@ 316153cc     LoaderCHR.obj
 0002:000073d4       ??_C@_06NLFPJIBA@bspace?$AA@ 316153d4     LoaderCHR.obj
 0002:000073dc       ??_C@_03MFPIMNEL@lmg?$AA@  316153dc     LoaderCHR.obj
 0002:000073e0       ??_C@_03INJKBFDI@caf?$AA@  316153e0     LoaderCHR.obj
 0002:000073e4       ??_C@_0CN@IKHFBIPF@The?5GlobalID?5of?5the?5default?5Para@ 316153e4     LoaderCHR.obj
 0002:00007414       ??_C@_0CB@KOBLDDLL@CryCHRLoader?3?3LoadAnimationFiles@ 31615414     LoaderCHR.obj
 0002:00007438       ??_C@_04MKMLCMBL@?4fxl?$AA@ 31615438     LoaderCHR.obj
 0002:00007440       ??_C@_0L@MMMPLAFM@Memstat?5?$CFi?$AA@ 31615440     LoaderCHR.obj
 0002:0000744c       ??_C@_0DA@OMGLPLED@?5?5?$CFd?5animation?9assets?5loaded?5?$CIto@ 3161544c     LoaderCHR.obj
 0002:0000747c       ??_C@_0BN@PKLOMKFG@CryCHRLoader?3?3LoadAnimations?$AA@ 3161547c     LoaderCHR.obj
 0002:000074a0       ??_C@_0GD@BIOBFDCL@Default?9Skeleton?5has?5wrong?5orien@ 316154a0     LoaderCHR.obj
 0002:00007508       __real@3fc1eb8520000000    31615508     LoaderCHR.obj
 0002:00007510       ??_C@_0BO@NBIMBHLL@CryAnimation?3?5assetDefinedLOD?$AA@ 31615510     LoaderCHR.obj
 0002:00007530       ??_C@_0CF@CFMJFCCB@CryAnimation?3?5m_nBaseLOD?5should?5@ 31615530     LoaderCHR.obj
 0002:00007558       ??_C@_0BJ@MBHDKFEE@CryCHRLoader?3?3LoadNewCHR?$AA@ 31615558     LoaderCHR.obj
 0002:00007574       ??_7IControllerRelocatableChain@@6B@ 31615574     LoaderDBA.obj
 0002:00007580       ??_7CControllerOptNonVirtual@@6B@ 31615580     LoaderDBA.obj
 0002:000075ec       ??_7CInternalDatabaseInfo@@6BIControllerRelocatableChain@@@ 316155ec     LoaderDBA.obj
 0002:000075f4       ??_7CInternalDatabaseInfo@@6BIStreamCallback@@@ 316155f4     LoaderDBA.obj
 0002:00007604       ??_C@_0DO@PFPEONFD@Failed?5To?5Load?5Animation?5DBA?5?8?$CFs@ 31615604     LoaderDBA.obj
 0002:00007644       ??_C@_0CO@KBAEHNDD@ERROR?0?5controller?5array?5size?5to?5@ 31615644     LoaderDBA.obj
 0002:00007674       ??_C@_0N@BCCFIHEB@ALL?5DBAs?5?$CFli?$AA@ 31615674     LoaderDBA.obj
 0002:00007684       ??_C@_0BJ@PIMHMAGK@Current?5DBA?4?5Memstat?5?$CFli?$AA@ 31615684     LoaderDBA.obj
 0002:000076a0       ??_C@_0CJ@FLLKFPPC@ReadController903?4?5Finished?4?5Mem@ 316156a0     LoaderDBA.obj
 0002:000076cc       ??_C@_0P@JDIHECOA@Invalid?5GAH?5ID?$AA@ 316156cc     LoaderDBA.obj
 0002:000076dc       ??_C@_0BH@EOMBJNOG@DBA?1CAF?5mismatch?5in?5?$CFs?$AA@ 316156dc     LoaderDBA.obj
 0002:000076f4       ??_C@_0BD@GOOKFDHB@GAH?5does?5not?5exist?$AA@ 316156f4     LoaderDBA.obj
 0002:00007708       ??_C@_0EM@EGJGGEMM@Going?5to?5create?5a?5CAF?5header?5on?5@ 31615708     LoaderDBA.obj
 0002:00007754       ??_C@_0DI@FCIOEJBO@ReadController905?4?5All?5dynamic?5d@ 31615754     LoaderDBA.obj
 0002:0000778c       ??_C@_0BH@MGGDIFFJ@Empty?5controller?5found?$AA@ 3161578c     LoaderDBA.obj
 0002:000077a4       ??_C@_0CN@JCHDIHHA@ReadController905?4?5TracksResize?4@ 316157a4     LoaderDBA.obj
 0002:000077d4       ??_C@_0CF@NHHPDLLA@ReadController905?4?5Init?4?5Memstat@ 316157d4     LoaderDBA.obj
 0002:000077fc       ??_C@_0CD@MLCMJLOB@error?3?5could?5not?5allocate?5?$CFd?5byt@ 316157fc     LoaderDBA.obj
 0002:00007820       ??_C@_0CJ@JICLBEBF@CInternalDatabaseInfo?3?3ReadContr@ 31615820     LoaderDBA.obj
 0002:00007850       ??_C@_0FE@CEPIMKIH@CryAnimation?3?5unknown?5chunk?9vers@ 31615850     LoaderDBA.obj
 0002:000078a8       ??_C@_0FN@ECGHOMFI@CryAnimation?3?5ReadController904?5@ 316158a8     LoaderDBA.obj
 0002:00007908       ??_C@_0FN@CKAOPOAN@CryAnimation?3?5ReadController903?5@ 31615908     LoaderDBA.obj
 0002:00007968       ??_C@_0FN@HKLNJENB@CryAnimation?3?5ReadController902?5@ 31615968     LoaderDBA.obj
 0002:000079c8       ??_C@_0FN@NLNLEBGJ@CryAnimation?3?5ReadController900?5@ 316159c8     LoaderDBA.obj
 0002:00007a28       ??_C@_0BG@GCJJICEA@Failed?5to?5load?5chunks?$AA@ 31615a28     LoaderDBA.obj
 0002:00007a40       ??_C@_0CA@EIBOCEEG@Illegal?5File?5Type?5for?5?4dba?5file?$AA@ 31615a40     LoaderDBA.obj
 0002:00007a60       ??_C@_0BF@EDAFHOON@Bad?5DBA?5file?5version?$AA@ 31615a60     LoaderDBA.obj
 0002:00007a78       ??_C@_0BN@NCKMPNBB@Failed?5to?5stream?5DBA?9file?5?$CFx?$AA@ 31615a78     LoaderDBA.obj
 0002:00007a98       ??_C@_0CN@IKNFBJGB@CInternalDatabaseInfo?3?3StreamAsy@ 31615a98     LoaderDBA.obj
 0002:00007ac8       ??_7CController@@6B@       31615ac8     LoaderTCB.obj
 0002:00007b04       ??_7ITrackInformation@@6B@ 31615b04     LoaderTCB.obj
 0002:00007b0c       ??_7IPositionController@@6B@ 31615b0c     LoaderTCB.obj
 0002:00007b30       ??_7IRotationController@@6B@ 31615b30     LoaderTCB.obj
 0002:00007b58       ??_C@_0ED@CKLAKBPH@Data?5Error?5in?5Win32?5Build?3?5CAF?5f@ 31615b58     LoaderTCB.obj
 0002:00007b9c       ??_C@_0BF@GKLLIPEB@ReadMotionParameters?$AA@ 31615b9c     LoaderTCB.obj
 0002:00007bb4       ??_7?$CAdvancedTrackInformation@U?$Quat_tpl@M@@UQuatLerp@@VIRotationController@@@@6B@ 31615bb4     LoaderTCB.obj
 0002:00007bd8       ??_7?$CAdvancedTrackInformation@U?$Vec3_tpl@M@@UVec3Lerp@@VIPositionController@@@@6B@ 31615bd8     LoaderTCB.obj
 0002:00007bfc       ??_7CHeaderTCB@@6B@        31615bfc     LoaderTCB.obj
 0002:00007c00       ??_C@_0EB@MAFIPHCH@animation?5not?5loaded?3?5found?5unsu@ 31615c00     LoaderTCB.obj
 0002:00007c48       ??_C@_0EB@DGECOHO@animation?5not?5loaded?3?5controller@ 31615c48     LoaderTCB.obj
 0002:00007c90       ??_C@_0EB@CPCKOGLC@animation?5not?5loaded?3?5controller@ 31615c90     LoaderTCB.obj
 0002:00007cd4       ??_C@_0BL@HNEFPEED@CONTROLLER_CHUNK_DESC_0828?$AA@ 31615cd4     LoaderTCB.obj
 0002:00007cf0       ??_C@_0CE@HPJMHPKM@Illegal?5File?5Type?5for?5?4caf?5file?3@ 31615cf0     LoaderTCB.obj
 0002:00007d14       ??_C@_0BJ@BFJPNJCO@Bad?5CAF?5file?5version?3?5?$CFs?$AA@ 31615d14     LoaderTCB.obj
 0002:00007d34       ??_C@_06BNNOMDLO@Handle?$AA@ 31615d34     ParamLoader.obj
 0002:00007d3c       ??_C@_09OBHIPIHP@LIKHandle?$AA@ 31615d3c     ParamLoader.obj
 0002:00007d48       ??_C@_09NIBPEJCE@RIKHandle?$AA@ 31615d48     ParamLoader.obj
 0002:00007d54       ??_C@_08GAHNGDIJ@IKHandle?$AA@ 31615d54     ParamLoader.obj
 0002:00007d60       ??_C@_0BL@DCAKIFLJ@CParamLoader?3?3MemFindFirst?$AA@ 31615d60     ParamLoader.obj
 0002:00007d7c       ??_C@_0BG@PLFGIMMI@Failure?5for?5weight?5?$CFs?$AA@ 31615d7c     ParamLoader.obj
 0002:00007d94       ??_C@_0N@HIPKJGLI@nWeightIdx?$DO0?$AA@ 31615d94     ParamLoader.obj
 0002:00007da4       ??_C@_0BG@NAMCFIGE@Failure?5for?5target?5?$CFs?$AA@ 31615da4     ParamLoader.obj
 0002:00007dbc       ??_C@_0N@PLPGFIAE@nTargetIdx?$DO0?$AA@ 31615dbc     ParamLoader.obj
 0002:00007dcc       ??_C@_06FGANPIPG@Target?$AA@ 31615dcc     ParamLoader.obj
 0002:00007dd4       ??_C@_0L@CGLHJMHG@ADIKTarget?$AA@ 31615dd4     ParamLoader.obj
 0002:00007de0       ??_C@_05ENDOMFAI@Delay?$AA@ 31615de0     ParamLoader.obj
 0002:00007de8       ??_C@_03HKDFLGGP@Arm?$AA@  31615de8     ParamLoader.obj
 0002:00007dec       ??_C@_0M@LDCHAHBG@ImpactJoint?$AA@ 31615dec     ParamLoader.obj
 0002:00007df8       ??_C@_0N@PAHFLIGD@ImpactJoints?$AA@ 31615df8     ParamLoader.obj
 0002:00007e08       ??_C@_0N@FIINBKCH@LWeaponJoint?$AA@ 31615e08     ParamLoader.obj
 0002:00007e18       ??_C@_09KOHFDMLF@JointName?$AA@ 31615e18     ParamLoader.obj
 0002:00007e24       ??_C@_0N@BGGMLAEN@RWeaponJoint?$AA@ 31615e24     ParamLoader.obj
 0002:00007e34       ??_C@_0CI@NKKGJNAP@CryAnimation?5Error?3?5Look?9Poses?5d@ 31615e34     ParamLoader.obj
 0002:00007e60       ??_C@_0EL@DBLACMEL@Look?9Pose?5Error?3?5Reference?5Joint@ 31615e60     ParamLoader.obj
 0002:00007eac       ??_C@_0P@GAPEMHIJ@ReferenceJoint?$AA@ 31615eac     ParamLoader.obj
 0002:00007ec0       ??_C@_0EI@MLODPBJP@Look?9Pose?5Error?3?5?5Start?5JointNam@ 31615ec0     ParamLoader.obj
 0002:00007f08       ??_C@_0L@MNFJAMCB@StartJoint?$AA@ 31615f08     ParamLoader.obj
 0002:00007f18       ??_C@_0EB@NBLLANHO@Look?9Pose?5Error?3?5JointName?5?8?$CFs?8?5@ 31615f18     ParamLoader.obj
 0002:00007f5c       ??_C@_0P@MGJAFNBF@ParameterJoint?$AA@ 31615f5c     ParamLoader.obj
 0002:00007f6c       ??_C@_09JFBKCAJ@AnimToken?$AA@ 31615f6c     ParamLoader.obj
 0002:00007f78       ??_C@_05LEKIHFJL@Joint?$AA@ 31615f78     ParamLoader.obj
 0002:00007f80       ??_C@_0BC@IAPMCPPH@DirectionalBlends?$AA@ 31615f80     ParamLoader.obj
 0002:00007f94       ??_C@_0N@CNHHKGI@PositionList?$AA@ 31615f94     ParamLoader.obj
 0002:00007fa4       ??_C@_08NGDGBBLG@Additive?$AA@ 31615fa4     ParamLoader.obj
 0002:00007fb0       ??_C@_07NAEHBBNL@Primary?$AA@ 31615fb0     ParamLoader.obj
 0002:00007fb8       ??_C@_0DA@BNADLPKC@JointName?5?8?$CFs?8?5for?5Look?9Pose?5not@ 31615fb8     ParamLoader.obj
 0002:00007fe8       ??_C@_0N@FIGHJKFE@RotationList?$AA@ 31615fe8     ParamLoader.obj
 0002:00007ff8       ??_C@_04GIAGJOJD@para?$AA@ 31615ff8     ParamLoader.obj
 0002:00008000       ??_C@_03PHODBHCN@FOV?$AA@  31616000     ParamLoader.obj
 0002:00008004       ??_C@_0P@CFGKLJDI@REyeAttachment?$AA@ 31616004     ParamLoader.obj
 0002:00008014       ??_C@_0P@IMHLDOAC@LEyeAttachment?$AA@ 31616014     ParamLoader.obj
 0002:00008024       ??_C@_0CH@OGOIEFLC@CryAnimation?5Error?3?5Aim?9Poses?5di@ 31616024     ParamLoader.obj
 0002:00008050       ??_C@_0EO@GJJJEFKH@Aim?9Pose?5Error?3?5ProcAdjustment?5J@ 31616050     ParamLoader.obj
 0002:000080a0       ??_C@_0BA@HINOHKMB@ProcAdjustments?$AA@ 316160a0     ParamLoader.obj
 0002:000080b0       ??_C@_0EJ@PPFJJBLB@Aim?9Pose?5Error?3?5Reference?5JointN@ 316160b0     ParamLoader.obj
 0002:00008100       ??_C@_0EE@PGDKGCKI@Aim?9Pose?5Error?3?5StartJointName?5?8@ 31616100     ParamLoader.obj
 0002:00008144       ??_C@_0DP@LDLOABDK@Aim?9Pose?5Error?3?5JointName?5?8?$CFs?8?5f@ 31616144     ParamLoader.obj
 0002:00008184       ??_C@_03EMIMMIHL@?$CK?4?$CK?$AA@ 31616184     ParamLoader.obj
 0002:00008188       ??_C@_0BC@KHIBCMBD@Failure?5for?5J4?5?$CFs?$AA@ 31616188     ParamLoader.obj
 0002:0000819c       ??_C@_08HCPLBCDA@nJ4Idx?$DO0?$AA@ 3161619c     ParamLoader.obj
 0002:000081a8       ??_C@_02MGJJNNAM@J4?$AA@   316161a8     ParamLoader.obj
 0002:000081ac       ??_C@_0BC@BFKBPAAD@Failure?5for?5J3?5?$CFs?$AA@ 316161ac     ParamLoader.obj
 0002:000081c0       ??_C@_08LHFMCMLO@nJ3Idx?$DO0?$AA@ 316161c0     ParamLoader.obj
 0002:000081cc       ??_C@_02IJNIELML@J3?$AA@   316161cc     ParamLoader.obj
 0002:000081d0       ??_C@_09MCEHMCIG@For?5J2?5?$CFs?$AA@ 316161d0     ParamLoader.obj
 0002:000081dc       ??_C@_08BBCLCHAK@nJ2Idx?$DO0?$AA@ 316161dc     ParamLoader.obj
 0002:000081e8       ??_C@_02JAMDHKIK@J2?$AA@   316161e8     ParamLoader.obj
 0002:000081ec       ??_C@_09IFOHLIFG@For?5J1?5?$CFs?$AA@ 316161ec     ParamLoader.obj
 0002:000081f8       ??_C@_08CAMDDNJH@nJ1Idx?$DO0?$AA@ 316161f8     ParamLoader.obj
 0002:00008204       ??_C@_02LLOOCJEJ@J1?$AA@   31616204     ParamLoader.obj
 0002:00008208       ??_C@_09LIIHJBOG@For?5J0?5?$CFs?$AA@ 31616208     ParamLoader.obj
 0002:00008214       ??_C@_08IGLEDGCD@nJ0Idx?$DO0?$AA@ 31616214     ParamLoader.obj
 0002:00008220       ??_C@_02KCPFBIAI@J0?$AA@   31616220     ParamLoader.obj
 0002:00008224       ??_C@_0P@JNLINEBF@nMaxInteration?$AA@ 31616224     ParamLoader.obj
 0002:00008234       ??_C@_0L@ELELNKBI@fThreshold?$AA@ 31616234     ParamLoader.obj
 0002:00008240       ??_C@_09JJEBABC@fStepSize?$AA@ 31616240     ParamLoader.obj
 0002:0000824c       ??_C@_0M@KANHEFDJ@EndEffector?$AA@ 3161624c     ParamLoader.obj
 0002:00008258       ??_C@_06MIIPBJJH@Solver?$AA@ 31616258     ParamLoader.obj
 0002:00008260       ??_C@_02GMHIAGGM@IK?$AA@   31616260     ParamLoader.obj
 0002:00008264       ??_C@_0BO@JNONGKEO@CParamLoader?3?3ExpandWildcards?$AA@ 31616264     ParamLoader.obj
 0002:00008284       ??_C@_05KJNJLLGA@level?$AA@ 31616284     ParamLoader.obj
 0002:0000828c       ??_C@_09FEGAOKFA@JointList?$AA@ 3161628c     ParamLoader.obj
 0002:00008298       ??_C@_0BB@PKMHEMPI@AimIK_Definition?$AA@ 31616298     ParamLoader.obj
 0002:000082ac       ??_C@_0BC@OMKLAMBI@LookIK_Definition?$AA@ 316162ac     ParamLoader.obj
 0002:000082c0       ??_C@_0BC@MHDOBOAO@Recoil_Definition?$AA@ 316162c0     ParamLoader.obj
 0002:000082d4       ??_C@_0BE@HPIABMHN@FeetLock_Definition?$AA@ 316162d4     ParamLoader.obj
 0002:000082e8       ??_C@_0BM@JLBGLKEH@Animation_Driven_IK_Targets?$AA@ 316162e8     ParamLoader.obj
 0002:00008304       ??_C@_0BC@LKENIJBM@LimbIK_Definition?$AA@ 31616304     ParamLoader.obj
 0002:00008318       ??_C@_0O@GCHJNOID@IK_Definition?$AA@ 31616318     ParamLoader.obj
 0002:00008328       ??_C@_07DHMEHIPB@?5?7?6?$AN?0?$CI?$CJ?$AA@ 31616328     ParamLoader.obj
 0002:00008330       ??_C@_06EDBFFAMA@?5?7?6?$AN?$DN?$CI?$AA@ 31616330     ParamLoader.obj
 0002:00008338       ??_C@_0FB@CKLBBPDE@Failed?5to?5create?5animation?5alias@ 31616338     ParamLoader.obj
 0002:0000838c       ??_C@_05GFOLEBJA@?$CFs?1?$CFs?$AA@ 3161638c     ParamLoader.obj
 0002:00008394       ??_C@_0BK@FGLKMAKN@Deprecated?5directive?5?$CC?$CFs?$CC?$AA@ 31616394     ParamLoader.obj
 0002:000083b0       ??_C@_0BK@PIIOJFFC@Unknown?5directive?5in?5?8?$CFs?8?$AA@ 316163b0     ParamLoader.obj
 0002:000083cc       ??_C@_0DN@FAJPOACF@Failed?5to?5set?5face?5lib?5?$CC?$CFs?$CC?4?5Fac@ 316163cc     ParamLoader.obj
 0002:0000840c       ??_C@_08BKGFCPAD@$FaceLib?$AA@ 3161640c     ParamLoader.obj
 0002:00008418       ??_C@_0O@PNFLLIOM@AnimationList?$AA@ 31616418     ParamLoader.obj
 0002:00008428       ??_C@_06MGHLEEEG@Params?$AA@ 31616428     ParamLoader.obj
 0002:00008430       ??_C@_08PCKHJNII@$Include?$AA@ 31616430     ParamLoader.obj
 0002:0000843c       ??_C@_0L@DLDGMDEL@persistent?$AA@ 3161643c     ParamLoader.obj
 0002:00008448       ??_C@_05GECEPKB@flags?$AA@ 31616448     ParamLoader.obj
 0002:00008450       ??_C@_0CO@HDNFLOKE@Duplicate?5model?5tracks?5database?5@ 31616450     ParamLoader.obj
 0002:00008480       ??_C@_0BA@FHGJMAGE@$TracksDatabase?$AA@ 31616480     ParamLoader.obj
 0002:00008490       ??_C@_0BD@CPBAAOIB@$AnimEventDatabase?$AA@ 31616490     ParamLoader.obj
 0002:000084a4       ??_C@_0P@DEBICNIP@$AnimDirectory?$AA@ 316164a4     ParamLoader.obj
 0002:000084b4       ??_C@_0BE@CDPOIOIF@$AnimationDirectory?$AA@ 316164b4     ParamLoader.obj
 0002:000084c8       ??_C@_08PIHFAEOK@$AnimDir?$AA@ 316164c8     ParamLoader.obj
 0002:000084d4       ??_C@_0O@LIIBPCBH@$AnimationDir?$AA@ 316164d4     ParamLoader.obj
 0002:000084e4       ??_C@_04LOAJBDKD@true?$AA@ 316164e4     ParamLoader.obj
 0002:000084ec       ??_C@_0BB@JJMFGJMC@?$CDParseSubFolders?$AA@ 316164ec     ParamLoader.obj
 0002:00008500       ??_C@_09MIHJIFBG@?$CDfilepath?$AA@ 31616500     ParamLoader.obj
 0002:0000850c       ??_C@_05EJAMACJC@?5?7?6?$AN?$DN?$AA@ 3161650c     ParamLoader.obj
 0002:00008514       ??_C@_04LNEJFJGI@path?$AA@ 31616514     ParamLoader.obj
 0002:0000851c       ??_C@_09ONEINPNJ@Animation?$AA@ 3161651c     ParamLoader.obj
 0002:00008528       ??_C@_05GPNABNFL@null?1?$AA@ 31616528     ParamLoader.obj
 0002:00008530       ??_C@_0BL@PPLFDBBD@CParamLoader?3?3LoadAnimList?$AA@ 31616530     ParamLoader.obj
 0002:0000854c       ??_C@_0BO@DIJIECID@Failed?5to?5load?5animations?3?5?$CFs?$AA@ 3161654c     ParamLoader.obj
 0002:0000856c       ??_C@_03ENGDOFNI@Lod?$AA@  3161656c     ParamLoader.obj
 0002:00008570       ??_C@_0BG@CANMHDPD@CParamLoader?3?3LoadXML?$AA@ 31616570     ParamLoader.obj
 0002:0000858c       ??_C@_0M@FAGLBHGK@mat_default?$AA@ 3161658c     Model.obj
 0002:00008598       ??_7ICharacterModel@@6B@   31616598     Model.obj
 0002:000085ec       ??_7IFacialModel@@6B@      316165ec     FacialModel.obj
 0002:000085ec       ??_7IAnimEventList@@6B@    316165ec     AnimEventList.obj
 0002:000085ec       ??_7IAnimEvents@@6B@       316165ec     CharacterManager.obj
 0002:000085ec       ??_7IFacialAnimSkeletonAnimationEntry@@6B@ 316165ec     FaceAnimSequence.obj
 0002:000085ec       ??_7ICharacterModelSkeleton@@6B@ 316165ec     Model.obj
 0002:00008608       ??_C@_06FOHEPPJH@sphere?$AA@ 31616608     Model.obj
 0002:00008610       ??_C@_07FJIOKKEJ@capsule?$AA@ 31616610     Model.obj
 0002:00008618       ??_C@_08GNLJBPEP@cylinder?$AA@ 31616618     Model.obj
 0002:00008624       ??_C@_03OLPJGAII@box?$AA@  31616624     Model.obj
 0002:00008628       ??_C@_0M@NKEMBHLE@DampingAnim?$AA@ 31616628     Model.obj
 0002:00008634       ??_C@_0BD@JFPAJNFL@StiffnessDecayAnim?$AA@ 31616634     Model.obj
 0002:00008648       ??_C@_0O@KLKDFFAF@StiffnessAnim?$AA@ 31616648     Model.obj
 0002:00008658       ??_C@_0O@MCPAABAE@AirResistance?$AA@ 31616658     Model.obj
 0002:00008668       ??_C@_0O@KEGAKDKO@StiffnessTang?$AA@ 31616668     Model.obj
 0002:00008678       ??_C@_0O@IBDMOJCA@StiffnessNorm?$AA@ 31616678     Model.obj
 0002:00008688       ??_C@_0L@CLKEODIP@MaxStretch?$AA@ 31616688     Model.obj
 0002:00008694       ??_C@_0BF@JLJEJDNJ@StiffnessControlBone?$AA@ 31616694     Model.obj
 0002:000086ac       ??_C@_09CEKHLCFH@Thickness?$AA@ 316166ac     Model.obj
 0002:000086b8       ??_C@_04EIIBPIEA@Mass?$AA@ 316166b8     Model.obj
 0002:000086c0       ??_C@_0P@JHEAKJPO@BodyCollisions?$AA@ 316166c0     Model.obj
 0002:000086d0       ??_C@_0O@KEMNECCG@EnvCollisions?$AA@ 316166d0     Model.obj
 0002:000086e0       ??_C@_0P@ELOPBDHG@SimpleBlending?$AA@ 316166e0     Model.obj
 0002:000086f0       ??_C@_08DIMMEHEB@Friction?$AA@ 316166f0     Model.obj
 0002:000086fc       ??_C@_07HJKIPEFI@Damping?$AA@ 316166fc     Model.obj
 0002:00008704       ??_C@_0P@MPIGCMMH@StiffnessDecay?$AA@ 31616704     Model.obj
 0002:00008714       ??_C@_09GCCJCEDC@Stiffness?$AA@ 31616714     Model.obj
 0002:00008720       ??_C@_0M@DHGMMGNF@MaxTimestep?$AA@ 31616720     Model.obj
 0002:0000872c       ??_C@_0BD@NEJDDAMA@JointLimitIncrease?$AA@ 3161672c     Model.obj
 0002:00008740       ??_C@_0L@IEFEJNGD@JointLimit?$AA@ 31616740     Model.obj
 0002:0000874c       ??_C@_07JMGDFJEK@Gravity?$AA@ 3161674c     Model.obj
 0002:00008754       ??_C@_0M@JFHCMOIP@cloth_proxy?$AA@ 31616754     Model.obj
 0002:00008760       ??_C@_0O@JNEDNOB@CollisionInfo?$AA@ 31616760     Model.obj
 0002:00008770       ??_C@_0M@MLNNNIFK@FacialModel?$AA@ 31616770     Model.obj
 0002:0000877c       ??_C@_0O@BPDDIHEF@AnimationSets?$AA@ 3161677c     Model.obj
 0002:0000878c       ??_C@_0O@FNBEOPPF@ModelSkeleton?$AA@ 3161678c     Model.obj
 0002:0000879c       ??_7CModelSkeleton@@6B?$_reference_target@H@@@ 3161679c     Model.obj
 0002:000087a0       ??_7CModelSkeleton@@6BICharacterModelSkeleton@@@ 316167a0     Model.obj
 0002:000087c0       ??_7CSkel@@6B@             316167c0     Model.obj
 0002:00008818       ??_C@_0BC@BCDELJLP@CSkel?5Release?3?5?$CFs?$AA@ 31616818     Model.obj
 0002:00008830       ??_C@_0FH@BFCNOANF@The?5model?5?8?$CFs?8?5still?5has?5?$CFd?5skel@ 31616830     Model.obj
 0002:00008888       ??_7IAnimationSet@@6B@     31616888     ModelAnimationSet.obj
 0002:0000891c       ??_C@_0CH@KKJIOKKC@Invalid?5Animation?5ID?3?5?$CFd?5for?5Mod@ 3161691c     ModelAnimationSet.obj
 0002:00008944       ??_C@_0CH@GBJHKOKG@CAnimationSet?3?3GetModelAnimation@ 31616944     ModelAnimationSet.obj
 0002:0000896c       ??_C@_0BI@FLFIHPFJ@?$CBNEGATIVE?5ANIMATION?5ID?$CB?$AA@ 3161696c     ModelAnimationSet.obj
 0002:00008984       ??_C@_0BM@ICDIPNOO@?$CBANIMATION?5ID?5OUT?5OF?5RANGE?$CB?$AA@ 31616984     ModelAnimationSet.obj
 0002:000089a0       ??_C@_0CL@CAADJKCO@illegal?5animation?5index?5?8?$CFd?8?5for@ 316169a0     ModelAnimationSet.obj
 0002:000089d0       ??_C@_0EL@IGFMDGNC@illegal?5animation?5index?5used?5in?5@ 316169d0     ModelAnimationSet.obj
 0002:00008a20       ??_C@_0EO@LPMHKCIG@illegal?5animation?5index?5used?5in?5@ 31616a20     ModelAnimationSet.obj
 0002:00008a70       ??_C@_0EG@LPAFCHLM@illegal?5animation?5index?5used?5in?5@ 31616a70     ModelAnimationSet.obj
 0002:00008ab8       ??_C@_0DB@IBBOCMGJ@animation?9name?5not?5in?5cal?9file?3?5@ 31616ab8     ModelAnimationSet.obj
 0002:00008aec       ??_C@_0BL@HBHKFCBB@?$CBNEGATIVE?5MORPH?5TARGET?5ID?$CB?$AA@ 31616aec     ModelAnimationSet.obj
 0002:00008b08       ??_C@_0EE@HMPGHNOG@CAnimationSet?3?3GetAnimationDCCWo@ 31616b08     ModelAnimationSet.obj
 0002:00008b50       ??_C@_0EA@LJNOOANO@CAnimationSet?3?3GetAnimationDCCWo@ 31616b50     ModelAnimationSet.obj
 0002:00008b90       ??_C@_0CG@ECBPIFCO@illegal?5joint?5index?3?5?$CFd?5for?5Mode@ 31616b90     ModelAnimationSet.obj
 0002:00008bb8       ??_C@_0DC@BICBPBBO@animation?9name?5?8?$CFs?8?5not?5in?5CAL?9f@ 31616bb8     ModelAnimationSet.obj
 0002:00008bf0       ??_C@_0EG@GLAOHHAM@?$CL?$CL?$CL?$CL?5Trying?5to?5get?5StartLocation@ 31616bf0     ModelAnimationSet.obj
 0002:00008c38       ??_C@_0CE@KIHHODMM@CryAnimation?3?5CAL?9file?5loaded?5tw@ 31616c38     ModelAnimationSet.obj
 0002:00008c60       ??_7CAnimationSet@@6B@     31616c60     ModelAnimationSet.obj
 0002:00008cf8       ??_C@_0EH@FLFJJNIB@Unnecessary?5Loading?5of?5CAF?9files@ 31616cf8     ModelAnimationSet.obj
 0002:00008d40       ??_C@_0EH@OEMEILP@Unnecessary?5Loading?5of?5CAF?9files@ 31616d40     ModelAnimationSet.obj
 0002:00008d88       ??_C@_0MB@DLLCPOOG@CryAnimation?3?3?5Trying?5to?5load?5an@ 31616d88     ModelAnimationSet.obj
 0002:00008e4c       ??_C@_0CC@DGFFKLPE@Failed?5to?5load?5animation?5CAF?5fil@ 31616e4c     ModelAnimationSet.obj
 0002:00008e70       ??_C@_0CI@MFGAAJDC@CryAnimation?3?3?5weird?5access?5of?5A@ 31616e70     ModelAnimationSet.obj
 0002:00008e98       ??_C@_0CI@DKHEGOPL@CryAnimation?3?3?5weird?5access?5of?5C@ 31616e98     ModelAnimationSet.obj
 0002:00008ec4       __real@3e2aaaab            31616ec4     ModelMesh.obj
 0002:00008ec8       ??_C@_0BJ@DPHJOGLI@FindClosestPointOnMesh?3?5?$AA@ 31616ec8     ModelMesh.obj
 0002:00008ee4       __real@4cbebc20            31616ee4     ModelMesh.obj
 0002:00008ee8       ??_C@_0N@ECCGOBMG@Bip01?5R?5Toe0?$AA@ 31616ee8     ModelSkeleton.obj
 0002:00008ef8       ??_C@_0N@JOIFGJHJ@Bip01?5R?5Heel?$AA@ 31616ef8     ModelSkeleton.obj
 0002:00008f08       ??_C@_0N@MBIECKPD@Bip01?5R?5Foot?$AA@ 31616f08     ModelSkeleton.obj
 0002:00008f18       ??_C@_0N@JDAJBMDK@Bip01?5R?5Calf?$AA@ 31616f18     ModelSkeleton.obj
 0002:00008f28       ??_C@_0N@HFMHAGFF@Bip01?5L?5Toe0?$AA@ 31616f28     ModelSkeleton.obj
 0002:00008f38       ??_C@_0N@KJGEIOOK@Bip01?5L?5Heel?$AA@ 31616f38     ModelSkeleton.obj
 0002:00008f48       ??_C@_0N@PGGFMNGA@Bip01?5L?5Foot?$AA@ 31616f48     ModelSkeleton.obj
 0002:00008f58       ??_C@_0N@KEOIPLKJ@Bip01?5L?5Calf?$AA@ 31616f58     ModelSkeleton.obj
 0002:00008f68       ??_C@_0BI@IDONHEOJ@todo?3?5delete?5bones?5phys?$AA@ 31616f68     ModelSkeleton.obj
 0002:00008f80       ??_C@_0M@OHJCPMGN@active_phys?$AA@ 31616f80     ModelSkeleton.obj
 0002:00008f8c       ??_C@_07GFBFDLBM@gravity?$AA@ 31616f8c     ModelSkeleton.obj
 0002:00008f94       __real@c61c3c00            31616f94     AnimationManager.obj
 0002:00008f98       ??_C@_05NCCFOPHA@model?$AA@ 31616f98     AnimationManager.obj
 0002:00008fa0       ??_C@_03DAPAKLGM@dir?$AA@  31616fa0     AnimationManager.obj
 0002:00008fa4       ??_C@_06KLHHMIGM@offset?$AA@ 31616fa4     AnimationManager.obj
 0002:00008fac       ??_C@_09DAGAJHIH@parameter?$AA@ 31616fac     AnimationManager.obj
 0002:00008fb8       ??_C@_07JJACOCKO@endTime?$AA@ 31616fb8     AnimationManager.obj
 0002:00008fc0       ??_C@_04CLCEDBPF@time?$AA@ 31616fc0     AnimationManager.obj
 0002:00008fc8       ??_C@_05GFHEIIDD@event?$AA@ 31616fc8     AnimationManager.obj
 0002:00008fd0       ??_C@_0BJ@FBLMMOEB@CAF?5Reloading?5failed?3?5?$CFs?$AA@ 31616fd0     AnimationManager.obj
 0002:00008fec       ??_C@_0CC@IBDFJLNA@Hot?5loaded?5animation?5CAF?9file?3?5?$CF@ 31616fec     AnimationManager.obj
 0002:00009010       ??_C@_0FH@GLDCLENN@Could?5not?5process?5aim?5poses?5from@ 31617010     AnimationManager.obj
 0002:00009068       ??_C@_0BL@PEJBPCKA@Re?9Processed?5Look?9Pose?3?5?$CFs?$AA@ 31617068     AnimationManager.obj
 0002:00009084       ??_C@_0BK@KIKPHPJP@Re?9Processed?5Aim?9Pose?3?5?$CFs?$AA@ 31617084     AnimationManager.obj
 0002:000090a0       ??_C@_0DK@CLFMPEFJ@Hot?5loaded?5animation?5CAF?9file?5fo@ 316170a0     AnimationManager.obj
 0002:000090dc       ??_C@_0DK@BABPPFII@CAF?5Reloading?5failed?0?5asset?5wasn@ 316170dc     AnimationManager.obj
 0002:00009118       ??_C@_0CC@GCMBNMKE@Hot?5loaded?5animation?5LMG?9file?3?5?$CF@ 31617118     AnimationManager.obj
 0002:0000913c       ??_C@_0BJ@JDJPOJGL@LMG?5Reloading?5failed?3?5?$CFs?$AA@ 3161713c     AnimationManager.obj
 0002:00009158       ??_C@_0M@EGNNJIMG@__unnamed__?$AA@ 31617158     AnimationManager.obj
 0002:00009164       ??_C@_08NAFBJPAH@segment4?$AA@ 31617164     AnimationManager.obj
 0002:00009170       ??_C@_08JPBAAJMA@segment3?$AA@ 31617170     AnimationManager.obj
 0002:0000917c       ??_C@_08IGALDIIB@segment2?$AA@ 3161717c     AnimationManager.obj
 0002:00009188       ??_C@_08KNCGGLEC@segment1?$AA@ 31617188     AnimationManager.obj
 0002:00009194       ??_C@_0N@HLEDPIHE@Total?3?5?$CF4dKB?$AA@ 31617194     AnimationManager.obj
 0002:000091a8       ??_C@_0FH@MOAGBIJJ@CharInstances?3?$CF3d?5?$CIMem?3?5?$CF4dKB?$CJ?5S@ 316171a8     AnimationManager.obj
 0002:00009200       __real@41c80000            31617200     AnimationManager.obj
 0002:00009204       __real@400ccccd            31617204     AnimationManager.obj
 0002:00009208       ??_C@_0DC@DAFNBAKF@Defrag?5heap?3?5?$CFiKB?5moveable?5?$CFiKB?5@ 31617208     AnimationManager.obj
 0002:0000923c       ??_C@_0DN@HMBLBPBC@LMG?3?5?$CF04d?5?5?5?5Loaded?3?5?$CF04d?5?5?5?5Use@ 3161723c     AnimationManager.obj
 0002:0000927c       ??_C@_0DO@OFMPJGHE@AIM?3?5?$CF04d?5?5?5?5Loaded?3?5?$CF04d?5?5?5?5Use@ 3161727c     AnimationManager.obj
 0002:000092c0       ??_C@_0EF@DIODCEKM@CAF?3?5?$CF04d?5?5?5?5Loaded?3?5?$CF04d?5?5?5?5Use@ 316172c0     AnimationManager.obj
 0002:00009308       ??_C@_0BI@DFAHFJLE@nSizeOfLoadedKeys?3?5?$CF07d?$AA@ 31617308     AnimationManager.obj
 0002:00009320       ??_C@_0BP@JGLJADPL@CafInMemory?3?5?$CF07d?5FilePath?3?5?$CFs?$AA@ 31617320     AnimationManager.obj
 0002:00009340       ??_C@_0CH@CJCBCHLJ@CafInMemory?3?5?$CF7d?5ref?3?5?$CF5d?5FilePa@ 31617340     AnimationManager.obj
 0002:00009368       ??_C@_0DE@FGOCMMFD@DBA?3?5?$CFd?5KBytes?5?5?5Clients?3?5?$CFd?5KBy@ 31617368     AnimationManager.obj
 0002:0000939c       ??_C@_0DJ@IAMGMGNJ@size?5of?5path?5names?3?5?$CFd?5bytes?5?5?5?5@ 3161739c     AnimationManager.obj
 0002:000093d8       __real@41300000            316173d8     AnimationManager.obj
 0002:000093dc       ??_C@_0DL@HJBFHPHA@UsedAssets?3?5?$CF04d?5?5nTCount?3?5?$CFu?5?5S@ 316173dc     AnimationManager.obj
 0002:00009418       ??_C@_0CC@DMIIEABE@CAnimationManager?3?3DebugAnimUsag@ 31617418     AnimationManager.obj
 0002:0000943c       ??_C@_0O@EHHLMIFF@AnimationKeys?$AA@ 3161743c     AnimationManager.obj
 0002:0000944c       ??_C@_0CE@CGKHFNED@CAnimationManager?3?3LoadAnimation@ 3161744c     AnimationManager.obj
 0002:00009470       ?m_byteTable@ControllerHelper@@3QBEB 31617470     ControllerPQ.obj
 0002:00009570       ?m_byteLowBit@ControllerHelper@@3QBEB 31617570     ControllerPQ.obj
 0002:00009670       ?m_byteHighBit@ControllerHelper@@3QBEB 31617670     ControllerPQ.obj
 0002:00009770       __real@383505e6            31617770     ControllerPQ.obj
 0002:00009774       __real@493504e0            31617774     ControllerPQ.obj
 0002:00009778       __real@49b504e8            31617778     ControllerPQ.obj
 0002:0000977c       ??_7?$CTrackDataStorageInt@U?$Vec3_tpl@M@@UNoCompressVec3@@VITrackPositionStorage@@@@6B@ 3161777c     ControllerPQ.obj
 0002:000097a4       ??_7?$CTrackDataStorageInt@U?$Quat_tpl@M@@UNoCompressQuat@@VITrackRotationStorage@@@@6B@ 316177a4     ControllerPQ.obj
 0002:000097c8       ??_7?$CTrackDataStorageInt@U?$Quat_tpl@M@@USmallTree48BitQuat@@VITrackRotationStorage@@@@6B@ 316177c8     ControllerPQ.obj
 0002:000097ec       ??_7?$CTrackDataStorageInt@U?$Quat_tpl@M@@USmallTree64BitQuat@@VITrackRotationStorage@@@@6B@ 316177ec     ControllerPQ.obj
 0002:00009810       ??_7?$CTrackDataStorageInt@U?$Quat_tpl@M@@USmallTree64BitExtQuat@@VITrackRotationStorage@@@@6B@ 31617810     ControllerPQ.obj
 0002:00009834       ??_7CKeyTimesInformationBitSet@@6B@ 31617834     ControllerPQ.obj
 0002:0000985c       ??_C@_0CI@NIMGLEEI@Unknown?5Rotation?5Compression?5for@ 3161785c     ControllerPQ.obj
 0002:00009884       ??_7?$CTrackDataStorage@U?$Vec3_tpl@M@@UNoCompressVec3@@VITrackPositionStorage@@@@6B@ 31617884     ControllerPQ.obj
 0002:000098b4       ??_7?$CTrackDataStorage@U?$Quat_tpl@M@@UNoCompressQuat@@VITrackRotationStorage@@@@6B@ 316178b4     ControllerPQ.obj
 0002:000098e4       ??_7?$CTrackDataStorage@U?$Quat_tpl@M@@USmallTree48BitQuat@@VITrackRotationStorage@@@@6B@ 316178e4     ControllerPQ.obj
 0002:00009914       ??_7?$CTrackDataStorage@U?$Quat_tpl@M@@USmallTree64BitQuat@@VITrackRotationStorage@@@@6B@ 31617914     ControllerPQ.obj
 0002:00009944       ??_7?$CTrackDataStorage@U?$Quat_tpl@M@@USmallTree64BitExtQuat@@VITrackRotationStorage@@@@6B@ 31617944     ControllerPQ.obj
 0002:00009974       ??_7?$CKeyTimesInformation@MUF32Encoder@@@@6BIControllerRelocatableChain@@@ 31617974     ControllerPQ.obj
 0002:0000997c       ??_7?$CKeyTimesInformation@MUF32Encoder@@@@6BIKeyTimesInformation@@@ 3161797c     ControllerPQ.obj
 0002:000099a4       ??_7?$CKeyTimesInformation@GUUINT16Encoder@@@@6BIControllerRelocatableChain@@@ 316179a4     ControllerPQ.obj
 0002:000099ac       ??_7?$CKeyTimesInformation@GUUINT16Encoder@@@@6BIKeyTimesInformation@@@ 316179ac     ControllerPQ.obj
 0002:000099d4       ??_7?$CKeyTimesInformation@EUByteEncoder@@@@6BIControllerRelocatableChain@@@ 316179d4     ControllerPQ.obj
 0002:000099dc       ??_7?$CKeyTimesInformation@EUByteEncoder@@@@6BIKeyTimesInformation@@@ 316179dc     ControllerPQ.obj
 0002:00009a04       ??_7?$CKeyTimesInformationStartStop@MUF32StartStopEncoder@@@@6B@ 31617a04     ControllerPQ.obj
 0002:00009a2c       ??_7?$CKeyTimesInformationStartStop@GUUINT16StartStopEncoder@@@@6B@ 31617a2c     ControllerPQ.obj
 0002:00009a54       ??_7?$CKeyTimesInformationStartStop@EUByteStartStopEncoder@@@@6B@ 31617a54     ControllerPQ.obj
 0002:00009a80       __real@3eb0c6f7a0000000    31617a80     ControllerPQLog.obj
 0002:00009a88       __real@400921fb54442d18    31617a88     ControllerPQLog.obj
 0002:00009a90       __real@3ff921fb54442d18    31617a90     ControllerPQLog.obj
 0002:00009a98       ??_7CControllerPQLog@@6B@  31617a98     ControllerPQLog.obj
 0002:00009ad4       __real@ff7fffff            31617ad4     ControllerPQLog.obj
 0002:00009ae0       __real@bff0000000000000    31617ae0     GlobalAnimationHeaderAIM.obj
 0002:00009ae8       __real@0010000000000000    31617ae8     GlobalAnimationHeaderAIM.obj
 0002:00009af0       __real@bf333334            31617af0     GlobalAnimationHeaderAIM.obj
 0002:00009af4       __real@3ff33333            31617af4     GlobalAnimationHeaderAIM.obj
 0002:00009af8       __real@be4cccd0            31617af8     GlobalAnimationHeaderAIM.obj
 0002:00009afc       __real@bf19999a            31617afc     GlobalAnimationHeaderAIM.obj
 0002:00009b00       __real@3ddb7cdfd9d7bdbb    31617b00     GlobalAnimationHeaderAIM.obj
 0002:00009b08       __real@4024000000000000    31617b08     GlobalAnimationHeaderAIM.obj
 0002:00009b10       __real@3f847ae140000000    31617b10     GlobalAnimationHeaderAIM.obj
 0002:00009b18       __real@4008000000000000    31617b18     GlobalAnimationHeaderAIM.obj
 0002:00009b20       __real@3fd0000000000000    31617b20     GlobalAnimationHeaderAIM.obj
 0002:00009b28       __real@403e000000000000    31617b28     GlobalAnimationHeaderAIM.obj
 0002:00009b30       __real@3f847ae147ae147b    31617b30     GlobalAnimationHeaderAIM.obj
 0002:00009b38       __real@3f80a3d7            31617b38     GlobalAnimationHeaderAIM.obj
 0002:00009b3c       ??_C@_0BL@ODMGNJMN@CONTROLLER_CHUNK_DESC_0826?$AA@ 31617b3c     GlobalAnimationHeaderAIM.obj
 0002:00009b58       ??_C@_0CG@HDJMEILE@Animation?5file?5has?5no?5compressed@ 31617b58     GlobalAnimationHeaderAIM.obj
 0002:00009b80       ??_C@_0CF@OGCHLH@Animation?5file?5has?5uncompressed?5@ 31617b80     GlobalAnimationHeaderAIM.obj
 0002:00009ba8       ??_C@_0BB@HBALHEOC@weird?5controller?$AA@ 31617ba8     GlobalAnimationHeaderAIM.obj
 0002:00009bbc       ??_C@_0BL@KNEFCFDN@CONTROLLER_CHUNK_DESC_0831?$AA@ 31617bbc     GlobalAnimationHeaderAIM.obj
 0002:00009bd8       ??_C@_0BL@LEFOBEHM@CONTROLLER_CHUNK_DESC_0830?$AA@ 31617bd8     GlobalAnimationHeaderAIM.obj
 0002:00009bf4       ??_C@_0L@NECCCPPF@TCB?5chunks?$AA@ 31617bf4     GlobalAnimationHeaderAIM.obj
 0002:00009c00       ??_C@_0CE@FCEPGAHG@Illegal?5File?5Type?5for?5?4CAF?5file?3@ 31617c00     GlobalAnimationHeaderAIM.obj
 0002:00009c28       __real@40c0000000000000    31617c28     GlobalAnimationHeaderAIM.obj
 0002:00009c30       __real@3ff00068db8bac71    31617c30     GlobalAnimationHeaderAIM.obj
 0002:00009c38       __real@3ff004189374bc6a    31617c38     GlobalAnimationHeaderAIM.obj
 0002:00009c40       __real@3fa999999999999a    31617c40     GlobalAnimationHeaderAIM.obj
 0002:00009c48       __real@3fd921fb54442d18    31617c48     GlobalAnimationHeaderAIM.obj
 0002:00009c50       __real@40c3878000000000    31617c50     GlobalAnimationHeaderAIM.obj
 0002:00009c58       __real@4058c00000000000    31617c58     GlobalAnimationHeaderAIM.obj
 0002:00009c60       ??_C@_0EM@OIFELHKN@CryAnimation?3?5Aimpose?5?8?$CFs?8?5disab@ 31617c60     GlobalAnimationHeaderAIM.obj
 0002:00009cb0       ??_C@_0ED@KBHGCNDO@CryAnimation?3?5Parameter?5joint?5?8?$CF@ 31617cb0     GlobalAnimationHeaderAIM.obj
 0002:00009cf4       ??_C@_0DN@PJFOJMDA@CryAnimation?3?5Parameter?5joint?5?8?$CF@ 31617cf4     GlobalAnimationHeaderAIM.obj
 0002:00009d34       ??_C@_0CD@LDOKNDOJ@CryAnimation?3?5process?5Aimpose?5?8?$CF@ 31617d34     GlobalAnimationHeaderAIM.obj
 0002:00009d58       ??_C@_01LOCGONAA@?$AA?$AA@ 31617d58     GlobalAnimationHeaderAIM.obj
 0002:00009d68       ??_C@_0CH@FGLCCHPF@GlobalAnimationHeaderCAF?3?3DoesEx@ 31617d68     GlobalAnimationHeaderCAF.obj
 0002:00009d90       ??_C@_0O@HEFJBIFC@Animation?5DBA?$AA@ 31617d90     GlobalAnimationHeaderCAF.obj
 0002:00009da0       ??_C@_0CK@PCKLFE@SPEED_CHUNK_DESC_1?5not?5supported@ 31617da0     GlobalAnimationHeaderCAF.obj
 0002:00009dcc       ??_C@_0CI@CHBFAPGJ@SPEED_CHUNK_DESC?5not?5supported?5a@ 31617dcc     GlobalAnimationHeaderCAF.obj
 0002:00009df4       ??_7GlobalAnimationHeaderCAFStreamContent@@6B@ 31617df4     GlobalAnimationHeaderCAF.obj
 0002:00009e04       ??_C@_0BJ@CLIKGAMM@?$CFd?5?$CFf?5?$CFf?5?$CFf?5?$CFf?5?$CFf?5?$CFf?5?$CFf?6?$AA@ 31617e04     GlobalAnimationHeaderCAF.obj
 0002:00009e20       ??_C@_05MGFEFMAH@?$FL?$CFs?$FN?6?$AA@ 31617e20     GlobalAnimationHeaderCAF.obj
 0002:00009e28       ??_C@_0BK@GMCOOBCN@?$CDFr?7Tx?7Ty?7Tz?7Rx?7Ry?7Rz?7SF?6?$AA@ 31617e28     GlobalAnimationHeaderCAF.obj
 0002:00009e44       ??_C@_0CH@HOGCBNHO@?$CDBeginning?5of?5Data?4?5Separated?5by@ 31617e44     GlobalAnimationHeaderCAF.obj
 0002:00009e6c       ??_C@_0BK@MLILPEIB@?$CFs?5?$CFf?5?$CFf?5?$CFf?5?$CFf?5?$CFf?5?$CFf?5?$CFf?5?6?$AA@ 31617e6c     GlobalAnimationHeaderCAF.obj
 0002:00009e88       ??_C@_0DB@GOIDDDLG@?$CDSegmentName?5Tx?0?5Ty?0?5Tz?0?5Rx?0?5Ry?0@ 31617e88     GlobalAnimationHeaderCAF.obj
 0002:00009ebc       ??_C@_0BA@HCLCKBKE@?$FLBasePosition?$FN?6?$AA@ 31617ebc     GlobalAnimationHeaderCAF.obj
 0002:00009ecc       ??_C@_06IINFAHFO@?$CFs?5?$CFs?6?$AA@ 31617ecc     GlobalAnimationHeaderCAF.obj
 0002:00009ed4       ??_C@_06FNIPBJLB@GLOBAL?$AA@ 31617ed4     GlobalAnimationHeaderCAF.obj
 0002:00009edc       ??_C@_07DNODLGKM@INVALID?$AA@ 31617edc     GlobalAnimationHeaderCAF.obj
 0002:00009ee4       ??_C@_0P@KNDGJNPN@?$CDCHILD?7PARENT?6?$AA@ 31617ee4     GlobalAnimationHeaderCAF.obj
 0002:00009ef4       ??_C@_0BK@FIEHECJB@?$FLSegmentNames?$CGHierarchy?$FN?6?$AA@ 31617ef4     GlobalAnimationHeaderCAF.obj
 0002:00009f10       ??_C@_0BC@PLMODGGP@ScaleFactor?51?400?6?$AA@ 31617f10     GlobalAnimationHeaderCAF.obj
 0002:00009f24       ??_C@_0BC@LACMDAJF@BoneLengthAxis?5Y?6?$AA@ 31617f24     GlobalAnimationHeaderCAF.obj
 0002:00009f38       ??_C@_0BH@IBIJNGBE@GlobalAxisofGravity?5Y?6?$AA@ 31617f38     GlobalAnimationHeaderCAF.obj
 0002:00009f50       ??_C@_0BH@DGLENGCE@RotationUnits?5Degrees?6?$AA@ 31617f50     GlobalAnimationHeaderCAF.obj
 0002:00009f68       ??_C@_0BF@OKDFJOBC@CalibrationUnits?5mm?6?$AA@ 31617f68     GlobalAnimationHeaderCAF.obj
 0002:00009f80       ??_C@_0BI@LACHBPJI@EulerRotationOrder?5ZYX?6?$AA@ 31617f80     GlobalAnimationHeaderCAF.obj
 0002:00009f98       ??_C@_0DK@GLCCHHDF@DataFrameRate?5?$CFd?7?7?$CDinteger?0?5data@ 31617f98     GlobalAnimationHeaderCAF.obj
 0002:00009fd4       ??_C@_0BI@FJIJOOIN@NumFrames?5?$CFd?7?7?$CDinteger?6?$AA@ 31617fd4     GlobalAnimationHeaderCAF.obj
 0002:00009fec       ??_C@_0BK@BFNNFED@NumSegments?5?$CFd?7?7?$CDinteger?6?$AA@ 31617fec     GlobalAnimationHeaderCAF.obj
 0002:0000a008       ??_C@_0BJ@IBCLPNKG@FileVersion?51?7?7?$CDinteger?6?$AA@ 31618008     GlobalAnimationHeaderCAF.obj
 0002:0000a028       ??_C@_0EB@PEACHJMM@DataType?5HTRS?7?7?$CDTranslation?5foll@ 31618028     GlobalAnimationHeaderCAF.obj
 0002:0000a06c       ??_C@_0CD@PNOAEFKH@FileType?5HTR?7?7?$CDSingle?5word?5strin@ 3161806c     GlobalAnimationHeaderCAF.obj
 0002:0000a090       ??_C@_0DC@IACPGBAE@?$CDHeader?5keywords?5are?5followed?5by@ 31618090     GlobalAnimationHeaderCAF.obj
 0002:0000a0c4       ??_C@_0L@CALEHGCD@?$FLHeader?$FN?7?6?$AA@ 316180c4     GlobalAnimationHeaderCAF.obj
 0002:0000a0d0       ??_C@_0DF@OKGHBAIO@?$CDHierarchical?5Translation?5and?5Ro@ 316180d0     GlobalAnimationHeaderCAF.obj
 0002:0000a108       ??_C@_0DG@DKOOKMLC@?$CDComment?5line?5ignore?5any?5data?5fo@ 31618108     GlobalAnimationHeaderCAF.obj
 0002:0000a140       ??_C@_04PHEPJNJD@?4htr?$AA@ 31618140     GlobalAnimationHeaderCAF.obj
 0002:0000a148       ??_C@_0CA@GHFHHAOC@Illegal?5File?5Type?5for?5?4caf?5file?$AA@ 31618148     GlobalAnimationHeaderCAF.obj
 0002:0000a168       ??_C@_0BF@NBFOLJEO@Bad?5CAF?5file?5version?$AA@ 31618168     GlobalAnimationHeaderCAF.obj
 0002:0000a180       ??_C@_0HL@BICADCBF@GlobalAnimationHeaderCAF?5is?5not?5@ 31618180     GlobalAnimationHeaderCAF.obj
 0002:0000a200       ??_C@_0EO@DNGKKJGM@CryAnimation?5CAF?3?5Assets?5has?5no?5@ 31618200     GlobalAnimationHeaderCAF.obj
 0002:0000a250       ??_C@_0BH@KADPCBAF@CAF?9File?5Not?5Found?3?5?$CFs?$AA@ 31618250     GlobalAnimationHeaderCAF.obj
 0002:0000a268       ??_C@_0BB@LGNCGFD@CAF?5Animation?5?$CFs?$AA@ 31618268     GlobalAnimationHeaderCAF.obj
 0002:0000a27c       ??_C@_0CI@CEIBOAIJ@Animation?9asset?5not?5in?5Animation@ 3161827c     GlobalAnimationHeaderCAF.obj
 0002:0000a2a4       ??_C@_0CC@OFOPDEKN@GlobalAnimationHeaderCAF?3?3LoadCA@ 316182a4     GlobalAnimationHeaderCAF.obj
 0002:0000a2c8       ??_C@_0BM@JEBLFMNF@Failed?5to?5parse?5CAF?9file?5?$CFx?$AA@ 316182c8     GlobalAnimationHeaderCAF.obj
 0002:0000a2e4       ??_C@_0DI@GIACGBCH@GlobalAnimationHeaderCAFStreamCo@ 316182e4     GlobalAnimationHeaderCAF.obj
 0002:0000a320       ??_C@_09JDIBPAEJ@?$DM?1VGrid?$DO?6?$AA@ 31618320     GlobalAnimationHeaderLMG.obj
 0002:0000a330       ??_C@_0LJ@NKMLEKDJ@?7?$DMVExample?5i0?$DN?$CC?$CF2d?$CC?5i1?$DN?$CC?$CF2d?$CC?5i2?$DN@ 31618330     GlobalAnimationHeaderLMG.obj
 0002:0000a3ec       ??_C@_08HBIAJAJD@?$DMVGrid?$DO?6?$AA@ 316183ec     GlobalAnimationHeaderLMG.obj
 0002:0000a3f8       ??_C@_0DP@CFNOMPCL@CryAnimation?3?5asset?5for?5paramete@ 316183f8     GlobalAnimationHeaderLMG.obj
 0002:0000a438       ??_C@_0CL@EDKCNNKH@Error?3?5ParaGroup?5has?5no?5examples@ 31618438     GlobalAnimationHeaderLMG.obj
 0002:0000a464       ??_C@_0BA@IJGNAHAN@?8?5was?5not?5found?$AA@ 31618464     GlobalAnimationHeaderLMG.obj
 0002:0000a474       ??_C@_0BL@JDPLPDDI@Error?3?5The?5included?5file?5?8?$AA@ 31618474     GlobalAnimationHeaderLMG.obj
 0002:0000a490       ??_C@_0P@EPLPMDPH@?8?5is?5not?5valid?$AA@ 31618490     GlobalAnimationHeaderLMG.obj
 0002:0000a4a0       ??_C@_0CC@BNBCGHJD@Error?3?5The?5included?5blend?9space?5@ 316184a0     GlobalAnimationHeaderLMG.obj
 0002:0000a4c4       ??_C@_0DO@GDICJIMA@Error?3?5More?5then?54?5dimensions?5pe@ 316184c4     GlobalAnimationHeaderLMG.obj
 0002:0000a504       ??_C@_05HAIIBMHI@aname?$AA@ 31618504     GlobalAnimationHeaderLMG.obj
 0002:0000a50c       ??_C@_0L@NPKCPEDM@BlendSpace?$AA@ 3161850c     GlobalAnimationHeaderLMG.obj
 0002:0000a518       ??_C@_0M@CLKCPEEG@BlendSpaces?$AA@ 31618518     GlobalAnimationHeaderLMG.obj
 0002:0000a524       ??_C@_0BB@ECHECOCG@ChooseBlendSpace?$AA@ 31618524     GlobalAnimationHeaderLMG.obj
 0002:0000a538       ??_C@_09KDJIBPJO@ParaScale?$AA@ 31618538     GlobalAnimationHeaderLMG.obj
 0002:0000a544       ??_C@_0CN@LMDFKGDA@Error?3?5ParaGroup?5has?5no?5dimensio@ 31618544     GlobalAnimationHeaderLMG.obj
 0002:0000a574       ??_C@_0BF@JMFFNCEF@Error?3?5The?5XML?9Tag?5?8?$AA@ 31618574     GlobalAnimationHeaderLMG.obj
 0002:0000a590       ??_C@_0FK@KEJALHHG@The?5ParaGroup?5?8?$CFs?8?5is?5invalid?$CB?5T@ 31618590     GlobalAnimationHeaderLMG.obj
 0002:0000a5ec       ??_C@_0CF@JNIHMDHP@Error?3?5The?5asset?5for?5the?5animati@ 316185ec     GlobalAnimationHeaderLMG.obj
 0002:0000a614       ??_C@_0BB@JKIDKOJK@?8?5does?5not?5exist?$AA@ 31618614     GlobalAnimationHeaderLMG.obj
 0002:0000a628       ??_C@_0FE@DOPPMCAJ@The?5ParaGroup?5?8?$CFs?8?5is?5invalid?$CB?5T@ 31618628     GlobalAnimationHeaderLMG.obj
 0002:0000a67c       ??_C@_0BH@BIDNBJJH@Error?3?5The?5animation?5?8?$AA@ 3161867c     GlobalAnimationHeaderLMG.obj
 0002:0000a694       ??_C@_0BJ@DCBDEEAK@?8?5is?5not?5in?5the?5CAL?9file?$AA@ 31618694     GlobalAnimationHeaderLMG.obj
 0002:0000a6b0       ??_C@_0CC@BLKFDNDD@?8?4?5It?5is?5expected?5to?5be?5?8Example@ 316186b0     GlobalAnimationHeaderLMG.obj
 0002:0000a6d4       ??_C@_0CK@FPFCGPOG@Error?3?5The?5ExampleTAG?5for?5an?5exa@ 316186d4     GlobalAnimationHeaderLMG.obj
 0002:0000a700       ??_C@_0EG@HMKJJPIC@Error?3?5More?5then?54?5additional?5ex@ 31618700     GlobalAnimationHeaderLMG.obj
 0002:0000a748       ??_C@_0BN@EPHGHLEL@?8?5is?5currently?5not?5supported?$AA@ 31618748     GlobalAnimationHeaderLMG.obj
 0002:0000a768       ??_C@_0BH@FMDDKGDP@Error?3?5The?5parameter?5?8?$AA@ 31618768     GlobalAnimationHeaderLMG.obj
 0002:0000a780       ??_C@_0EA@NACDAFHJ@Error?3?5More?5then?53?5dimensions?5pe@ 31618780     GlobalAnimationHeaderLMG.obj
 0002:0000a7c0       ??_C@_05IHAFCALK@Style?$AA@ 316187c0     GlobalAnimationHeaderLMG.obj
 0002:0000a7c8       ??_C@_08HHFKANFI@NewStyle?$AA@ 316187c8     GlobalAnimationHeaderLMG.obj
 0002:0000a7d4       ??_C@_0BC@ICLDOOLI@MotionCombination?$AA@ 316187d4     GlobalAnimationHeaderLMG.obj
 0002:0000a7e8       ??_C@_02MBAHPIAM@w7?$AA@   316187e8     GlobalAnimationHeaderLMG.obj
 0002:0000a7ec       ??_C@_02NIBMMJEN@w6?$AA@   316187ec     GlobalAnimationHeaderLMG.obj
 0002:0000a7f0       ??_C@_02PDDBJKIO@w5?$AA@   316187f0     GlobalAnimationHeaderLMG.obj
 0002:0000a7f4       ??_C@_02OKCKKLMP@w4?$AA@   316187f4     GlobalAnimationHeaderLMG.obj
 0002:0000a7f8       ??_C@_02KFGLDNAI@w3?$AA@   316187f8     GlobalAnimationHeaderLMG.obj
 0002:0000a7fc       ??_C@_02LMHAAMEJ@w2?$AA@   316187fc     GlobalAnimationHeaderLMG.obj
 0002:0000a800       ??_C@_02NHLPHGHG@i7?$AA@   31618800     GlobalAnimationHeaderLMG.obj
 0002:0000a804       ??_C@_02MOKEEHDH@i6?$AA@   31618804     GlobalAnimationHeaderLMG.obj
 0002:0000a808       ??_C@_02OFIJBEPE@i5?$AA@   31618808     GlobalAnimationHeaderLMG.obj
 0002:0000a80c       ??_C@_02PMJCCFLF@i4?$AA@   3161880c     GlobalAnimationHeaderLMG.obj
 0002:0000a810       ??_C@_02LDNDLDHC@i3?$AA@   31618810     GlobalAnimationHeaderLMG.obj
 0002:0000a814       ??_C@_02KKMIICDD@i2?$AA@   31618814     GlobalAnimationHeaderLMG.obj
 0002:0000a818       ??_C@_02IBOFNBPA@i1?$AA@   31618818     GlobalAnimationHeaderLMG.obj
 0002:0000a81c       ??_C@_02JIPOOALB@i0?$AA@   3161881c     GlobalAnimationHeaderLMG.obj
 0002:0000a820       ??_C@_08DGDGODFB@VExample?$AA@ 31618820     GlobalAnimationHeaderLMG.obj
 0002:0000a82c       ??_C@_05PJJIAHPE@VGrid?$AA@ 3161882c     GlobalAnimationHeaderLMG.obj
 0002:0000a834       ??_C@_02MEEIOOIJ@p7?$AA@   31618834     GlobalAnimationHeaderLMG.obj
 0002:0000a838       ??_C@_02NNFDNPMI@p6?$AA@   31618838     GlobalAnimationHeaderLMG.obj
 0002:0000a83c       ??_C@_02PGHOIMAL@p5?$AA@   3161883c     GlobalAnimationHeaderLMG.obj
 0002:0000a840       ??_C@_02OPGFLNEK@p4?$AA@   31618840     GlobalAnimationHeaderLMG.obj
 0002:0000a844       ??_C@_02KACECLIN@p3?$AA@   31618844     GlobalAnimationHeaderLMG.obj
 0002:0000a848       ??_C@_02LJDPBKMM@p2?$AA@   31618848     GlobalAnimationHeaderLMG.obj
 0002:0000a84c       ??_C@_04DPOPNPPG@Face?$AA@ 3161884c     GlobalAnimationHeaderLMG.obj
 0002:0000a854       ??_C@_09IALACKFM@Blendable?$AA@ 31618854     GlobalAnimationHeaderLMG.obj
 0002:0000a860       ??_C@_02JHFNFPIK@w1?$AA@   31618860     GlobalAnimationHeaderLMG.obj
 0002:0000a864       ??_C@_02IOEGGOML@w0?$AA@   31618864     GlobalAnimationHeaderLMG.obj
 0002:0000a868       ??_C@_02JCBCEJAP@p1?$AA@   31618868     GlobalAnimationHeaderLMG.obj
 0002:0000a86c       ??_C@_02ILAJHIEO@p0?$AA@   3161886c     GlobalAnimationHeaderLMG.obj
 0002:0000a870       ??_C@_06GMHIAKFO@Pseudo?$AA@ 31618870     GlobalAnimationHeaderLMG.obj
 0002:0000a878       ??_C@_0BL@BKKBLDIH@UseDirectlyForDeltaMotion3?$AA@ 31618878     GlobalAnimationHeaderLMG.obj
 0002:0000a894       ??_C@_0BL@DLKICMG@UseDirectlyForDeltaMotion2?$AA@ 31618894     GlobalAnimationHeaderLMG.obj
 0002:0000a8b0       ??_C@_0BL@CIJHNBAF@UseDirectlyForDeltaMotion1?$AA@ 316188b0     GlobalAnimationHeaderLMG.obj
 0002:0000a8cc       ??_C@_0BL@DBIMOAEE@UseDirectlyForDeltaMotion0?$AA@ 316188cc     GlobalAnimationHeaderLMG.obj
 0002:0000a8e8       ??_C@_08GJBDGDP@SetPara3?$AA@ 316188e8     GlobalAnimationHeaderLMG.obj
 0002:0000a8f4       ??_C@_08BPIKAHHO@SetPara2?$AA@ 316188f4     GlobalAnimationHeaderLMG.obj
 0002:0000a900       ??_C@_08DEKHFELN@SetPara1?$AA@ 31618900     GlobalAnimationHeaderLMG.obj
 0002:0000a90c       ??_C@_08CNLMGFPM@SetPara0?$AA@ 3161890c     GlobalAnimationHeaderLMG.obj
 0002:0000a918       ??_C@_0O@GMBENGPI@PlaybackScale?$AA@ 31618918     GlobalAnimationHeaderLMG.obj
 0002:0000a928       ??_C@_07LEFFBAGK@Example?$AA@ 31618928     GlobalAnimationHeaderLMG.obj
 0002:0000a930       ??_C@_0BF@CFNNMGLO@AdditionalExtraction?$AA@ 31618930     GlobalAnimationHeaderLMG.obj
 0002:0000a948       ??_C@_06KKBPGBGI@locked?$AA@ 31618948     GlobalAnimationHeaderLMG.obj
 0002:0000a950       ??_C@_04DEMJELKJ@ekey?$AA@ 31618950     GlobalAnimationHeaderLMG.obj
 0002:0000a958       ??_C@_04NLGJCJIL@skey?$AA@ 31618958     GlobalAnimationHeaderLMG.obj
 0002:0000a960       ??_C@_05MHMEBBGO@scale?$AA@ 31618960     GlobalAnimationHeaderLMG.obj
 0002:0000a968       ??_C@_05KFKAILFP@cells?$AA@ 31618968     GlobalAnimationHeaderLMG.obj
 0002:0000a970       ??_C@_03LJAEFNNE@max?$AA@  31618970     GlobalAnimationHeaderLMG.obj
 0002:0000a974       ??_C@_03KLIPLJLL@min?$AA@  31618974     GlobalAnimationHeaderLMG.obj
 0002:0000a978       ??_C@_07OMEBGOOF@StopLeg?$AA@ 31618978     GlobalAnimationHeaderLMG.obj
 0002:0000a980       ??_C@_0M@HEHNJKHP@BlendWeight?$AA@ 31618980     GlobalAnimationHeaderLMG.obj
 0002:0000a98c       ??_C@_09DOPCOEIN@TurnAngle?$AA@ 3161898c     GlobalAnimationHeaderLMG.obj
 0002:0000a998       ??_C@_0L@NPIFDIHI@TravelDist?$AA@ 31618998     GlobalAnimationHeaderLMG.obj
 0002:0000a9a4       ??_C@_0M@GJCIJMHH@TravelAngle?$AA@ 316189a4     GlobalAnimationHeaderLMG.obj
 0002:0000a9b0       ??_C@_0M@INHOBOHM@TravelSlope?$AA@ 316189b0     GlobalAnimationHeaderLMG.obj
 0002:0000a9bc       ??_C@_09BDPPKMLL@TurnSpeed?$AA@ 316189bc     GlobalAnimationHeaderLMG.obj
 0002:0000a9c8       ??_C@_09HHOHJEHG@MoveSpeed?$AA@ 316189c8     GlobalAnimationHeaderLMG.obj
 0002:0000a9d4       ??_C@_05LOJBNELM@Param?$AA@ 316189d4     GlobalAnimationHeaderLMG.obj
 0002:0000a9dc       ??_C@_09ODPNOLPG@Idle2Move?$AA@ 316189dc     GlobalAnimationHeaderLMG.obj
 0002:0000a9e8       ??_C@_09HAFMGPLD@VEGPARAMS?$AA@ 316189e8     GlobalAnimationHeaderLMG.obj
 0002:0000a9f4       ??_C@_02IGJGHHBN@tz?$AA@   316189f4     GlobalAnimationHeaderLMG.obj
 0002:0000a9f8       ??_C@_0EL@GBNGEHGE@Error?3?5too?5many?5examples?5in?5one?5@ 316189f8     GlobalAnimationHeaderLMG.obj
 0002:0000aa44       ??_C@_0CG@DOEGIGK@Error?3?5no?5examples?5in?5this?5ParaG@ 31618a44     GlobalAnimationHeaderLMG.obj
 0002:0000aa6c       ??_C@_09EILGBNO@THRESHOLD?$AA@ 31618a6c     GlobalAnimationHeaderLMG.obj
 0002:0000aa78       ??_C@_0O@PJOADIDN@ExamplePseudo?$AA@ 31618a78     GlobalAnimationHeaderLMG.obj
 0002:0000aa88       ??_C@_0M@IFLEANKJ@ExampleList?$AA@ 31618a88     GlobalAnimationHeaderLMG.obj
 0002:0000aa94       ??_C@_0BH@MALMLOBG@Error?3?5The?5XMLTAG?5is?5?8?$AA@ 31618a94     GlobalAnimationHeaderLMG.obj
 0002:0000aaac       ??_C@_0DM@GGNNFPCH@?8?4?5It?5is?5expected?5to?5be?5?8ParaGro@ 31618aac     GlobalAnimationHeaderLMG.obj
 0002:0000aae8       ??_C@_0BD@FPPGAOB@CombinedBlendSpace?$AA@ 31618ae8     GlobalAnimationHeaderLMG.obj
 0002:0000aafc       ??_C@_09KCMCOIPJ@ParaGroup?$AA@ 31618afc     GlobalAnimationHeaderLMG.obj
 0002:0000ab08       ??_C@_0CC@GGJPBFGD@Error?3?5Parametric?9Group?5not?5foun@ 31618b08     GlobalAnimationHeaderLMG.obj
 0002:0000ab2c       ??_C@_0BE@GIKNGEKK@CryAnimation?5?$CFs?3?5?$CFs?$AA@ 31618b2c     GlobalAnimationHeaderLMG.obj
 0002:0000ab40       ??_C@_0EI@PNPGPCFE@Error?3?5Parametric?9Group?5loaded?5f@ 31618b40     GlobalAnimationHeaderLMG.obj
 0002:0000ab88       ??_C@_0EJ@PGHDDIJ@Error?3?5Parametric?9Group?5loaded?5f@ 31618b88     GlobalAnimationHeaderLMG.obj
 0002:0000abd8       ??_C@_0GA@FLLAOKLL@CryAnimation?3?5?5LMGs?5not?5supporte@ 31618bd8     GlobalAnimationHeaderLMG.obj
 0002:0000ac38       ??_C@_0BM@CDIMEJKN@CryAnimation?3?5data?5mismatch?$AA@ 31618c38     GlobalAnimationHeaderLMG.obj
 0002:0000ac54       __real@bf99999a            31618c54     GlobalAnimationHeaderLMG.obj
 0002:0000ac5c       ??_C@_01GBGANLPD@0?$AA@    31618c5c     AnimationBase.obj
 0002:0000ac60       __real@2f800000            31618c60     AnimationBase.obj
 0002:0000ac64       ??_C@_0DJ@DLJMMMP@Could?5not?5access?5CrySystem?4dll?5?$CI@ 31618c64     AnimationBase.obj
 0002:0000aca0       ??_C@_0P@NHEMOHAI@Memory?5Manager?$AA@ 31618ca0     AnimationBase.obj
 0002:0000acb0       ??_C@_0O@FFDHMLKN@CrySystem?4dll?$AA@ 31618cb0     AnimationBase.obj
 0002:0000acc0       ??_C@_0BO@JDKBDPNB@CryGetIMemoryManagerInterface?$AA@ 31618cc0     AnimationBase.obj
 0002:0000ace0       ??_C@_0BB@PNKHDABP@CrySystemCrtFree?$AA@ 31618ce0     AnimationBase.obj
 0002:0000acf4       ??_C@_0BB@MFMFBMDO@CrySystemCrtSize?$AA@ 31618cf4     AnimationBase.obj
 0002:0000ad08       ??_C@_0BD@BBIFHONI@CrySystemCrtMalloc?$AA@ 31618d08     AnimationBase.obj
 0002:0000ad1c       ??_C@_0O@LCCIKADF@CryGetMemSize?$AA@ 31618d1c     AnimationBase.obj
 0002:0000ad2c       ??_C@_07CKAGCLEE@CryFree?$AA@ 31618d2c     AnimationBase.obj
 0002:0000ad34       ??_C@_0L@FICCDMFO@CryRealloc?$AA@ 31618d34     AnimationBase.obj
 0002:0000ad40       ??_C@_09MCKPOEAK@CryMalloc?$AA@ 31618d40     AnimationBase.obj
 0002:0000ad50       ?iid@?1??IID@IEngineModule@@CAABUCryGUID@@XZ@4U3@B 31618d50     AnimationBase.obj
 0002:0000ad60       ??_7IFacialJoystickSerializeContext@@6B@ 31618d60     FaceAnimation.obj
 0002:0000ad60       ??_7ISystemEventListener@@6B@ 31618d60     AnimationBase.obj
 0002:0000ad68       __real@40c00000            31618d68     AnimationBase.obj
 0002:0000ad6c       ??_C@_0BD@PJOKHJBB@Pure?5function?5call?$AA@ 31618d6c     AnimationBase.obj
 0002:0000ad80       ??_C@_0CL@LKHBOBAH@Invalid?5parameter?5detected?5in?5CR@ 31618d80     AnimationBase.obj
 0002:0000adac       ??_C@_0BO@HAMEIFMK@Critical?5Section?5hanging?5lock?$AA@ 31618dac     AnimationBase.obj
 0002:0000adcc       ??_7CSystemEventListner_Animation@@6B@ 31618dcc     AnimationBase.obj
 0002:0000add4       ??_7CEngineModule_CryAnimation@@6B@ 31618dd4     AnimationBase.obj
 0002:0000adf0       ??_C@_0N@EMOPHPFF@CryAnimation?$AA@ 31618df0     AnimationBase.obj
 0002:0000ae00       ??_C@_09BHIABECK@CryEngine?$AA@ 31618e00     AnimationBase.obj
 0002:0000ae0c       ??_7CFactory@CEngineModule_CryAnimation@@6B@ 31618e0c     AnimationBase.obj
 0002:0000ae24       ??_C@_0BK@PCOPBKHN@EngineModule_CryAnimation?$AA@ 31618e24     AnimationBase.obj
 0002:0000ae40       ?cid@?1??GetClassID@CFactory@CEngineModule_CryAnimation@@UBEABUCryGUID@@XZ@4U4@B 31618e40     AnimationBase.obj
 0002:0000ae50       ??_7CAnimationThreadTask@@6B@ 31618e50     AnimationThreadTask.obj
 0002:0000ae58       ??_C@_0M@EBCFMMOO@ca_DrawPose?$AA@ 31618e58     cvars.obj
 0002:0000ae64       ??_C@_0BE@JOJOEEHJ@Character?5LOD?5ratio?$AA@ 31618e64     cvars.obj
 0002:0000ae78       ??_C@_0N@HBLINJMH@ca_lod_ratio?$AA@ 31618e78     cvars.obj
 0002:0000ae88       ??_C@_0BJ@EFBPDBDN@ca_FacialAnimationRadius?$AA@ 31618e88     cvars.obj
 0002:0000aea8       ??_C@_0FE@PMLLDBLE@Maximum?5distance?5at?5which?5facial@ 31618ea8     cvars.obj
 0002:0000aefc       ??_C@_0BI@JIEFPKKN@ca_cloth_air_resistance?$AA@ 31618efc     cvars.obj
 0002:0000af14       ??_C@_0CN@OHMALND@?$CCadvanced?$CC?5?$CImore?5correct?$CJ?5versio@ 31618f14     cvars.obj
 0002:0000af44       ??_C@_0BB@FOEHFOJF@ca_cloth_damping?$AA@ 31618f44     cvars.obj
 0002:0000af58       ??_C@_0BI@MCPNLIO@ca_cloth_stiffness_tang?$AA@ 31618f58     cvars.obj
 0002:0000af70       ??_C@_0DB@ONEEGFBO@stiffness?5for?5shape?5preservation@ 31618f70     cvars.obj
 0002:0000afa4       ??_C@_0BI@CJHDJBAA@ca_cloth_stiffness_norm?$AA@ 31618fa4     cvars.obj
 0002:0000afc0       ??_C@_0EK@DDGLJPG@stiffness?5for?5shape?5preservation@ 31618fc0     cvars.obj
 0002:0000b00c       ??_C@_0BC@NNDOBGOG@ca_cloth_friction?$AA@ 3161900c     cvars.obj
 0002:0000b020       ??_C@_0BD@GMPAHGEN@ca_cloth_thickness?$AA@ 31619020     cvars.obj
 0002:0000b034       ??_C@_0BP@NJANAPLJ@thickness?5for?5collision?5checks?$AA@ 31619034     cvars.obj
 0002:0000b054       ??_C@_0BD@CKHOOACI@ca_cloth_stiffness?$AA@ 31619054     cvars.obj
 0002:0000b068       ??_C@_0BJ@FAIMJLEO@stiffness?5for?5stretching?$AA@ 31619068     cvars.obj
 0002:0000b084       ??_C@_0BH@LJCFFBDO@ca_cloth_max_safe_step?$AA@ 31619084     cvars.obj
 0002:0000b0a0       ??_C@_0FG@KEFONKLH@if?5a?5segment?5stretches?5more?5than@ 316190a0     cvars.obj
 0002:0000b0f8       ??_C@_0BG@BFLELBCD@ca_cloth_max_timestep?$AA@ 316190f8     cvars.obj
 0002:0000b110       ??_C@_0BL@OAGPEHCI@ca_AttachmentCullingRation?$AA@ 31619110     cvars.obj
 0002:0000b12c       ??_C@_0DJ@OHMCHNBH@ration?5between?5size?5of?5attachmen@ 3161912c     cvars.obj
 0002:0000b168       __real@43480000            31619168     cvars.obj
 0002:0000b16c       ??_C@_0BM@DHENNHLO@ca_lipsync_phoneme_strength?$AA@ 3161916c     cvars.obj
 0002:0000b188       ??_C@_0BJ@JEKMPDAK@LipSync?5phoneme?5strength?$AA@ 31619188     cvars.obj
 0002:0000b1a4       ??_C@_0BH@FPKPCHNI@ca_lipsync_vertex_drag?$AA@ 316191a4     cvars.obj
 0002:0000b1bc       ??_C@_0DE@MGCDNDAD@Vertex?5drag?5coefficient?5when?5ble@ 316191bc     cvars.obj
 0002:0000b1f0       ??_C@_0BC@FCFJEAPB@ca_DeathBlendTime?$AA@ 316191f0     cvars.obj
 0002:0000b208       ??_C@_0FH@NFBJKPON@Specifies?5the?5blending?5time?5betw@ 31619208     cvars.obj
 0002:0000b260       ??_C@_0BP@IMGGOJJB@ca_MotionBlurMovementThreshold?$AA@ 31619260     cvars.obj
 0002:0000b280       ??_C@_0EM@LCCEBGGB@?$CCadvanced?$CC?5Set?5motion?5blur?5movem@ 31619280     cvars.obj
 0002:0000b2cc       ??_C@_0BG@BMEEJOGJ@ca_ParametricPoolSize?$AA@ 316192cc     cvars.obj
 0002:0000b2e4       ??_C@_0BM@IDPDBJFB@Size?5of?5the?5parametric?5pool?$AA@ 316192e4     cvars.obj
 0002:0000b300       ??_C@_0BH@INCACHFD@ca_MemoryDefragEnabled?$AA@ 31619300     cvars.obj
 0002:0000b318       ??_C@_0CF@IHFPNJPB@Enables?5defragmentation?5of?5anim?5@ 31619318     cvars.obj
 0002:0000b340       ??_C@_0BI@NFLCLMJD@ca_MemoryDefragPoolSize?$AA@ 31619340     cvars.obj
 0002:0000b358       ??_C@_0CN@LMOEMFHO@Sets?5the?5upper?5limit?5on?5the?5defr@ 31619358     cvars.obj
 0002:0000b388       ??_C@_0BC@GNNEHGKD@ca_MemoryUsageLog?$AA@ 31619388     cvars.obj
 0002:0000b39c       ??_C@_0BL@HFBKIPEK@enables?5a?5memory?5usage?5log?$AA@ 3161939c     cvars.obj
 0002:0000b3b8       ??_C@_0BI@FJMAFHBD@ca_physicsProcessImpact?$AA@ 316193b8     cvars.obj
 0002:0000b3d0       ??_C@_0BP@BOCAJCHI@Process?5physics?5impact?5pulses?4?$AA@ 316193d0     cvars.obj
 0002:0000b3f0       ??_C@_0BH@FNDDEFNL@ca_DecalSizeMultiplier?$AA@ 316193f0     cvars.obj
 0002:0000b408       ??_C@_0CD@HKOANJDA@The?5multiplier?5for?5the?5decal?5siz@ 31619408     cvars.obj
 0002:0000b42c       ??_C@_0P@MMIJBJMP@ca_DrawVEGInfo?$AA@ 3161942c     cvars.obj
 0002:0000b43c       ??_C@_0CJ@JONDKHCD@if?5set?5to?51?0?5the?5VEG?5debug?5info?5@ 3161943c     cvars.obj
 0002:0000b468       ??_C@_0BN@FLHDGLEO@ca_DisableAnimationUnloading?$AA@ 31619468     cvars.obj
 0002:0000b488       ??_C@_0BN@PCALLINP@Disable?5Animation?5Unloading?4?$AA@ 31619488     cvars.obj
 0002:0000b4a8       ??_C@_0BJ@ECNHADFF@ca_PrecacheAnimationSets?$AA@ 316194a8     cvars.obj
 0002:0000b4c4       ??_C@_0DD@JJEHANKB@Enable?5Precaching?5of?5Animation?5S@ 316194c4     cvars.obj
 0002:0000b4f8       ??_C@_0BH@HIIBGPEN@ca_DBAUnloadRemoveTime?$AA@ 316194f8     cvars.obj
 0002:0000b510       ??_C@_0CE@LLCCBPLI@DBA?5Unload?5Timing?3?5DBA?5Remove?5Ti@ 31619510     cvars.obj
 0002:0000b534       ??_C@_0BL@HBKEKJMC@ca_DBAUnloadUnregisterTime?$AA@ 31619534     cvars.obj
 0002:0000b550       ??_C@_0CI@CFJDCLLO@DBA?5Unload?5Timing?3?5CAF?5Unregiste@ 31619550     cvars.obj
 0002:0000b578       ??_C@_0BD@PGAODFMP@ca_thread1Affinity?$AA@ 31619578     cvars.obj
 0002:0000b58c       ??_C@_0CF@HFPHNJC@Affinity?5of?5second?5Animation?5Thr@ 3161958c     cvars.obj
 0002:0000b5b4       ??_C@_0BD@BJMMFOPB@ca_thread0Affinity?$AA@ 316195b4     cvars.obj
 0002:0000b5c8       ??_C@_0CE@ILFKAAMM@Affinity?5of?5first?5Animation?5Thre@ 316195c8     cvars.obj
 0002:0000b5ec       ??_C@_09NKFFJOFC@ca_thread?$AA@ 316195ec     cvars.obj
 0002:0000b5f8       ??_C@_0CJ@ILBOOLCK@If?5?$DO0?5enables?5Animation?5Multi?9Th@ 316195f8     cvars.obj
 0002:0000b624       ??_C@_0BC@BLCGFKPE@ca_disable_thread?$AA@ 31619624     cvars.obj
 0002:0000b638       ??_C@_0BP@HOGKGLKJ@TEMP?5Disable?5Animation?5Thread?4?$AA@ 31619638     cvars.obj
 0002:0000b658       ??_C@_0BD@ICEENPMF@ca_UseJointMasking?$AA@ 31619658     cvars.obj
 0002:0000b66c       ??_C@_0CP@JFBGPMJI@Use?5Joint?5Masking?5to?5speed?5up?5mo@ 3161966c     cvars.obj
 0002:0000b69c       ??_C@_0M@NIBNONAK@ca_Validate?$AA@ 3161969c     cvars.obj
 0002:0000b6a8       ??_C@_0DD@OGEBBLJF@if?5set?5to?51?0?5will?5run?5validation@ 316196a8     cvars.obj
 0002:0000b6e0       ??_C@_0GL@CKPBEHGA@Lowers?5render?5LODs?5for?5character@ 316196e0     cvars.obj
 0002:0000b74c       ??_C@_0CC@ELAFCBEH@ca_AllowMultipleEffectsOfSameNam@ 3161974c     cvars.obj
 0002:0000b770       ??_C@_0HB@BPKNANN@Allow?5a?5skeleton?5animation?5to?5sp@ 31619770     cvars.obj
 0002:0000b7e4       ??_C@_0BM@JGBPONLD@ca_FacialAnimationFramerate?$AA@ 316197e4     cvars.obj
 0002:0000b800       ??_C@_0GP@JJBJNLJN@Update?5facial?5system?5at?5a?5maximu@ 31619800     cvars.obj
 0002:0000b870       ??_C@_0BJ@DLDLGCNK@ca_SerializeSkeletonAnim?$AA@ 31619870     cvars.obj
 0002:0000b88c       ??_C@_0CF@IPALCDKO@Turn?5on?5CSkeletonAnim?5Serializat@ 3161988c     cvars.obj
 0002:0000b8b4       ??_C@_0BE@IFJGJCEG@ca_cloth_vars_reset?$AA@ 316198b4     cvars.obj
 0002:0000b8c8       ??_C@_0EI@LIDOPPLP@1?5?9?5load?5the?5values?5from?5the?5nex@ 316198c8     cvars.obj
 0002:0000b910       ??_C@_0BL@JPIFKACH@ca_MinInPlaceCAFStreamSize?$AA@ 31619910     cvars.obj
 0002:0000b92c       ??_C@_0DA@KAGFHHNF@min?5size?5a?5caf?5should?5be?5for?5in?9@ 3161992c     cvars.obj
 0002:0000b95c       ??_C@_0BG@FKJHEGLJ@ca_UnloadAnimationDBA?$AA@ 3161995c     cvars.obj
 0002:0000b974       ??_C@_0CC@GHFLMPAJ@if?51?0?5then?5unload?5DBA?5if?5not?5use@ 31619974     cvars.obj
 0002:0000b998       ??_C@_0BG@IKEHFGJO@ca_UnloadAnimationCAF?$AA@ 31619998     cvars.obj
 0002:0000b9b0       ??_C@_0DF@NHCELDFK@unloading?5streamed?5CAFs?5as?5soon?5@ 316199b0     cvars.obj
 0002:0000b9e8       ??_C@_0O@ODDFHGJE@ca_UseIMG_AIM?$AA@ 316199e8     cvars.obj
 0002:0000b9f8       ??_C@_0O@KENLDGGM@ca_UseIMG_CAF?$AA@ 316199f8     cvars.obj
 0002:0000ba08       ??_C@_0EM@LEHOJILF@if?51?0?5then?5we?5use?5the?5IMG?5file?4?5@ 31619a08     cvars.obj
 0002:0000ba54       ??_C@_0BH@ICIDFFCH@ca_DebugCriticalErrors?$AA@ 31619a54     cvars.obj
 0002:0000ba70       ??_C@_0ED@IHNECKBD@if?51?0?5then?5we?5stop?5with?5a?5Fatal?9@ 31619a70     cvars.obj
 0002:0000bab4       ??_C@_0M@HFNGIPLD@ca_SaveAABB?$AA@ 31619ab4     cvars.obj
 0002:0000bac0       ??_C@_0DH@LDGHIGLM@if?5the?5AABB?5is?5invalid?0?5replace?5@ 31619ac0     cvars.obj
 0002:0000baf8       ??_C@_0BE@NGCNMBH@ca_DebugADIKTargets?$AA@ 31619af8     cvars.obj
 0002:0000bb10       ??_C@_0FB@HHNKIAKE@If?51?0?5then?5it?5will?5show?5if?5there@ 31619b10     cvars.obj
 0002:0000bb64       ??_C@_0BC@KOCIPNFH@ca_useADIKTargets?$AA@ 31619b64     cvars.obj
 0002:0000bb78       ??_C@_0CB@JPJDCCLB@Use?5Animation?5Driven?5Ik?5Targets?4@ 31619b78     cvars.obj
 0002:0000bb9c       ??_C@_0BD@JJBPFNOD@ca_SkipLoadThinFat?$AA@ 31619b9c     cvars.obj
 0002:0000bbb0       ??_C@_0CG@KNEIJJLF@Skip?5loading?5fat?7hin?5stuff?5if?5en@ 31619bb0     cvars.obj
 0002:0000bbd8       ??_C@_0BD@EADKPCNL@ca_DebugFacialEyes?$AA@ 31619bd8     cvars.obj
 0002:0000bbec       ??_C@_0BH@BMFMOOJN@Debug?5facial?5eyes?5info?$AA@ 31619bec     cvars.obj
 0002:0000bc04       ??_C@_0P@BPDLLOAN@ca_DebugFacial?$AA@ 31619c04     cvars.obj
 0002:0000bc14       ??_C@_0BL@IAGGECCM@Debug?5facial?5playback?5info?$AA@ 31619c14     cvars.obj
 0002:0000bc30       ??_C@_0BB@JIJFFIF@ca_lipsync_debug?$AA@ 31619c30     cvars.obj
 0002:0000bc44       ??_C@_0CE@HJKBKFCI@Enables?5facial?5animation?5debug?5d@ 31619c44     cvars.obj
 0002:0000bc68       ??_C@_0BD@PACKHAKI@ca_eyes_procedural?$AA@ 31619c68     cvars.obj
 0002:0000bc7c       ??_C@_0CL@JEGBKNKL@Enables?1Disables?5procedural?5eyes@ 31619c7c     cvars.obj
 0002:0000bca8       ??_C@_0BN@GPJFFPOO@ca_lipsync_phoneme_crossfade?$AA@ 31619ca8     cvars.obj
 0002:0000bcc8       ??_C@_0DB@CMGMAGFM@Cross?5fade?5time?5between?5phonemes@ 31619cc8     cvars.obj
 0002:0000bcfc       ??_C@_0BK@GHKEBONN@ca_lipsync_phoneme_offset?$AA@ 31619cfc     cvars.obj
 0002:0000bd18       ??_C@_0DI@KHLBKNAK@Offset?5phoneme?5start?5time?5by?5thi@ 31619d18     cvars.obj
 0002:0000bd50       ??_C@_0BI@KPCIAMFN@ca_DebugSkeletonEffects?$AA@ 31619d50     cvars.obj
 0002:0000bd68       ??_C@_0DO@JINKPBJJ@If?5true?0?5dump?5log?5messages?5when?5@ 31619d68     cvars.obj
 0002:0000bda8       ??_C@_0O@MCJKIJHD@ca_KeepModels?$AA@ 31619da8     cvars.obj
 0002:0000bdb8       ??_C@_0GP@BADIOIKE@If?5set?5to?51?0?5will?5prevent?5models@ 31619db8     cvars.obj
 0002:0000be28       ??_C@_0BE@FHGGOKBM@ca_AnimWarningLevel?$AA@ 31619e28     cvars.obj
 0002:0000be40       ??_C@_0FF@LOGLEDBK@if?5you?5set?5this?5to?50?0?5there?5won?8@ 31619e40     cvars.obj
 0002:0000be98       ??_C@_0BB@HNJCBPAG@ca_DumpUsedAnims?$AA@ 31619e98     cvars.obj
 0002:0000beac       ??_C@_0CO@IKBCLPFN@writes?5animation?5asset?5statistic@ 31619eac     cvars.obj
 0002:0000bedc       ??_C@_0BI@PDMPAFEP@ca_StoreAnimNamesOnLoad?$AA@ 31619edc     cvars.obj
 0002:0000bef8       ??_C@_0EO@EOFGBPOE@stores?5the?5names?5of?5animations?5d@ 31619ef8     cvars.obj
 0002:0000bf48       ??_C@_0BO@HPFFLABM@ca_DebugAnimUsageOnFileAccess?$AA@ 31619f48     cvars.obj
 0002:0000bf68       ??_C@_0FG@NHLJNPAJ@shows?5what?5animation?5assets?5are?5@ 31619f68     cvars.obj
 0002:0000bfc0       ??_C@_0BC@DAKMICOE@ca_DebugAnimUsage?$AA@ 31619fc0     cvars.obj
 0002:0000bfd4       ??_C@_0DC@KNJOJOPG@shows?5what?5animation?5assets?5are?5@ 31619fd4     cvars.obj
 0002:0000c008       ??_C@_0BE@HFGKIJMC@ca_DebugAnimUpdates?$AA@ 3161a008     cvars.obj
 0002:0000c01c       ??_C@_0CF@EKFABEPM@shows?5the?5amount?5of?5skeleton?9upd@ 3161a01c     cvars.obj
 0002:0000c044       ??_C@_0BG@BADHPGJH@ca_ReloadAllCHRPARAMS?$AA@ 3161a044     cvars.obj
 0002:0000c05c       ??_C@_0BF@KHBHJIJP@realod?5all?5CHRPARAMS?$AA@ 3161a05c     cvars.obj
 0002:0000c074       ??_C@_0BI@EMMOJMOM@ca_TrackSkinTransMemory?$AA@ 3161a074     cvars.obj
 0002:0000c08c       ??_C@_0DI@IMICCPNO@shows?5how?5much?5memory?5the?5Skinni@ 3161a08c     cvars.obj
 0002:0000c0c4       ??_C@_0BD@MGJEPDDC@ca_DebugModelCache?$AA@ 3161a0c4     cvars.obj
 0002:0000c0d8       ??_C@_0EF@DJBHIAFJ@shows?5what?5models?5are?5currently?5@ 3161a0d8     cvars.obj
 0002:0000c120       ??_C@_0N@OFLBFAKC@ca_UseDecals?$AA@ 3161a120     cvars.obj
 0002:0000c130       ??_C@_0HN@KMILDOJK@if?5set?5to?50?0?5effectively?5disable@ 3161a130     cvars.obj
 0002:0000c1b0       ??_C@_0BM@HPCOFAEL@ca_ApplyJointVelocitiesMode?$AA@ 3161a1b0     cvars.obj
 0002:0000c1d0       ??_C@_0FI@MPAFKAPI@Joint?5velocity?5preservation?5code@ 3161a1d0     cvars.obj
 0002:0000c228       ??_C@_0BI@PFJEMCOI@ca_ForceUpdateSkeletons?$AA@ 3161a228     cvars.obj
 0002:0000c240       ??_C@_0DC@NELAHNFF@Always?5update?5all?5skeletons?0?5eve@ 3161a240     cvars.obj
 0002:0000c274       ??_C@_0BC@PILFPGJD@ca_LockFeetWithIK?$AA@ 3161a274     cvars.obj
 0002:0000c288       ??_C@_0GA@GOGDMLA@If?5this?5is?5set?5to?51?0?5then?5we?5loc@ 3161a288     cvars.obj
 0002:0000c2e8       ??_C@_0BG@FKLMHNFH@ca_UseFacialAnimation?$AA@ 3161a2e8     cvars.obj
 0002:0000c300       ??_C@_0DD@CHNCAAIJ@If?5this?5is?5set?5to?51?0?5we?5can?5play@ 3161a300     cvars.obj
 0002:0000c334       ??_C@_0BD@DLIDBMDO@ca_DrawAimIKVEGrid?$AA@ 3161a334     cvars.obj
 0002:0000c348       ??_C@_0DM@IAKBDCDE@if?5set?5to?51?0?5we?5will?5the?5the?5gri@ 3161a348     cvars.obj
 0002:0000c384       ??_C@_0M@DEJLCBPH@ca_UseAimIK?$AA@ 3161a384     cvars.obj
 0002:0000c390       ??_C@_0N@PEJBAIDG@ca_UseLookIK?$AA@ 3161a390     cvars.obj
 0002:0000c3a0       ??_C@_0EM@MHHKLIJM@If?5this?5is?5set?5to?51?0?5then?5we?5are@ 3161a3a0     cvars.obj
 0002:0000c3ec       ??_C@_0O@DGJMLBON@ca_UsePhysics?$AA@ 3161a3ec     cvars.obj
 0002:0000c3fc       ??_C@_0DA@COLJGECI@the?5physics?5is?5not?5applied?5?$CIeffe@ 3161a3fc     cvars.obj
 0002:0000c42c       ??_C@_09CFBCPLFA@ca_NoAnim?$AA@ 3161a42c     cvars.obj
 0002:0000c438       ??_C@_0EF@HCMHNOKH@the?5animation?5isn?8t?5updated?5?$CIthe@ 3161a438     cvars.obj
 0002:0000c480       ??_C@_0M@FBHAPKJL@ca_UseMorph?$AA@ 3161a480     cvars.obj
 0002:0000c490       ??_C@_0FE@IAIFCBEP@the?5morph?5skinning?5step?5is?5skipp@ 3161a490     cvars.obj
 0002:0000c4e4       ??_C@_0BK@MPBPEBJP@ca_LoadUncompressedChunks?$AA@ 3161a4e4     cvars.obj
 0002:0000c500       ??_C@_0EE@NHPHCLII@If?5this?51?0?5then?5uncompressed?5chu@ 3161a500     cvars.obj
 0002:0000c544       ??_C@_0BL@OKMLDGKP@ca_DebugAnimationStreaming?$AA@ 3161a544     cvars.obj
 0002:0000c560       ??_C@_0DM@DAIEEMPF@if?5this?5is?51?0?5then?5it?5shows?5what@ 3161a560     cvars.obj
 0002:0000c59c       ??_C@_0BG@BBDHFJLC@ca_DebugCommandBuffer?$AA@ 3161a59c     cvars.obj
 0002:0000c5b8       ??_C@_0EI@OMBFEIBM@if?5this?5is?51?0?5it?5will?5print?5the?5@ 3161a5b8     cvars.obj
 0002:0000c600       ??_C@_0N@HDBDOJNB@ca_DebugText?$AA@ 3161a600     cvars.obj
 0002:0000c610       ??_C@_0JG@OKJGDI@if?5this?5is?51?0?5it?5will?5print?5some@ 3161a610     cvars.obj
 0002:0000c6a8       ??_C@_0BI@DBBEJHFA@ca_DebugAnimMemTracking?$AA@ 3161a6a8     cvars.obj
 0002:0000c6c0       ??_C@_0DG@JDKMHCEB@if?5this?5is?51?0?5then?5its?5shows?5the@ 3161a6c0     cvars.obj
 0002:0000c6f8       ??_C@_0BD@CMLGDBNA@ca_DebugSWSkinning?$AA@ 3161a6f8     cvars.obj
 0002:0000c710       ??_C@_0FD@KLENFGMF@if?5this?5is?51?0?5then?5we?5will?5see?5a@ 3161a710     cvars.obj
 0002:0000c764       ??_C@_0BB@NHGLINGA@ca_DrawCGAAsSkin?$AA@ 3161a764     cvars.obj
 0002:0000c778       ??_C@_0EL@HPAKLPED@if?5this?5is?51?0?5will?5draw?5the?5CGA?5@ 3161a778     cvars.obj
 0002:0000c7c4       ??_C@_09OMCHEIFA@ca_DrawCC?$AA@ 3161a7c4     cvars.obj
 0002:0000c7d0       ??_C@_0CO@CCJDMHEB@if?5this?5is?50?0?5will?5not?5draw?5the?5@ 3161a7d0     cvars.obj
 0002:0000c800       ??_C@_0L@OPFPKGIL@ca_DrawCHR?$AA@ 3161a800     cvars.obj
 0002:0000c80c       ??_C@_0CP@HHALCDAN@if?5this?5is?50?0?5will?5not?5draw?5the?5@ 3161a80c     cvars.obj
 0002:0000c83c       ??_C@_0L@IFOMKACE@ca_DrawCGA?$AA@ 3161a83c     cvars.obj
 0002:0000c848       ??_C@_0CP@CIFCFNOP@if?5this?5is?50?0?5will?5not?5draw?5the?5@ 3161a848     cvars.obj
 0002:0000c878       ??_C@_0P@OIKKJBHD@ca_DrawLocator?$AA@ 3161a878     cvars.obj
 0002:0000c888       ??_C@_0HA@LKFLMFEA@if?5this?5is?51?0?5we?5will?5draw?5the?5b@ 3161a888     cvars.obj
 0002:0000c8f8       ??_C@_0BA@IHIJCMGE@ca_DrawBaseMesh?$AA@ 3161a8f8     cvars.obj
 0002:0000c908       ??_C@_0CL@LLDIBBLG@if?5this?5is?50?0?5will?5not?5draw?5the?5@ 3161a908     cvars.obj
 0002:0000c934       ??_C@_0BF@OJMPMHBN@ca_DrawAttachmentOBB?$AA@ 3161a934     cvars.obj
 0002:0000c94c       ??_C@_0BD@DFPABPCK@ca_DrawAttachments?$AA@ 3161a94c     cvars.obj
 0002:0000c960       ??_C@_0DE@GKAJOCDP@if?5this?5is?50?0?5will?5not?5draw?5the?5@ 3161a960     cvars.obj
 0002:0000c994       ??_C@_0P@NLGPICIE@ca_DrawNormals?$AA@ 3161a994     cvars.obj
 0002:0000c9a4       ??_C@_0CM@PHOOPKHH@draws?5the?5normals?5of?5the?5rendere@ 3161a9a4     cvars.obj
 0002:0000c9d0       ??_C@_0BB@IOBJBGIF@ca_DrawBinormals?$AA@ 3161a9d0     cvars.obj
 0002:0000c9e4       ??_C@_0CO@DAEPAFP@draws?5the?5binormals?5of?5the?5rende@ 3161a9e4     cvars.obj
 0002:0000ca14       ??_C@_0BA@JJFLHFEB@ca_DrawTangents?$AA@ 3161aa14     cvars.obj
 0002:0000ca24       ??_C@_0CN@OIDHNMMA@draws?5the?5tangents?5of?5the?5render@ 3161aa24     cvars.obj
 0002:0000ca54       ??_C@_0O@NLFIMKFH@ca_DrawLookIK?$AA@ 3161aa54     cvars.obj
 0002:0000ca64       ??_C@_0CB@BMHNHPOO@draws?5a?5visualization?5of?5look?5ik@ 3161aa64     cvars.obj
 0002:0000ca88       ??_C@_0BA@HBFJBKOG@ca_DrawAimPoses?$AA@ 3161aa88     cvars.obj
 0002:0000ca98       ??_C@_0CF@GBEFKEKH@draws?5the?5wireframe?5of?5the?5aim?5p@ 3161aa98     cvars.obj
 0002:0000cac0       ??_C@_0BB@KHFHLIDN@ca_DrawWireframe?$AA@ 3161aac0     cvars.obj
 0002:0000cad4       ??_C@_0DD@NFCANLL@draws?5a?5wireframe?5on?5top?5of?5the?5@ 3161aad4     cvars.obj
 0002:0000cb08       ??_C@_0BI@HGFGBAN@ca_DrawEmptyAttachments?$AA@ 3161ab08     cvars.obj
 0002:0000cb20       ??_C@_0EF@ONPLPOJD@draws?5a?5wireframe?5cube?5if?5there?5@ 3161ab20     cvars.obj
 0002:0000cb68       ??_C@_0BE@NOHAPOFE@ca_DrawPositionPost?$AA@ 3161ab68     cvars.obj
 0002:0000cb7c       ??_C@_0DJ@EDKKDGKP@draws?5the?5world?5position?5of?5the?5@ 3161ab7c     cvars.obj
 0002:0000cbb8       ??_C@_0BE@GAOKAHKJ@ca_DrawDecalsBBoxes?$AA@ 3161abb8     cvars.obj
 0002:0000cbcc       ??_C@_0CJ@CMAGMJDF@if?5set?5to?51?0?5the?5decals?5bboxes?5a@ 3161abcc     cvars.obj
 0002:0000cbf8       ??_C@_0BA@NEIBDHAP@ca_DrawSkeleton?$AA@ 3161abf8     cvars.obj
 0002:0000cc08       ??_C@_0CD@BAIOFGGC@if?5set?5to?51?0?5the?5skeleton?5is?5dra@ 3161ac08     cvars.obj
 0002:0000cc2c       ??_C@_0M@ODANEJOH@ca_DrawBBox?$AA@ 3161ac2c     cvars.obj
 0002:0000cc38       ??_C@_0DM@HALBLLMA@if?5set?5to?51?0?5the?5own?5bounding?5bo@ 3161ac38     cvars.obj
 0002:0000cc74       ??_C@_0BB@FGCINMPC@ca_usePhysicsLOD?$AA@ 3161ac74     cvars.obj
 0002:0000cc88       ??_C@_0DP@OALMMENO@If?5set?5to?50?5it?5loads?5only?5LOD0?4?5@ 3161ac88     cvars.obj
 0002:0000ccc8       ??_C@_0BA@HNABOPEG@ca_FilterJoints?$AA@ 3161acc8     cvars.obj
 0002:0000ccd8       ??_C@_0BB@BCONMOMD@ca_CharEditModel?$AA@ 3161acd8     cvars.obj
 0002:0000ccec       ??_C@_0DI@MGGBHHJD@objects?1characters?1human?1us?1nano@ 3161acec     cvars.obj
 0002:0000cd30       ??_7CPool@Memory@@6B@      3161ad30     Pool.obj
 0002:0000cd44       ??_C@_05FHGOFLKH@Fatal?$AA@ 3161ad44     Pool.obj
 0002:0000cd4c       ??_7CPoolFrameLocal@Memory@@6B@ 3161ad4c     Pool.obj
 0002:0000cd60       ??_C@_0BH@MCAFGJEB@SkinAttachmentTangents?$AA@ 3161ad60     _RenderSkinsSW.obj
 0002:0000cd78       __pDefaultRawDllMain       3161ad78     MSVCRT:crtdll.obj
 0002:0000cd78       __pRawDllMain              3161ad78     MSVCRT:crtdll.obj
 0002:0000cd88       __load_config_used         3161ad88     MSVCRT:loadcfg.obj
 0002:0000ce30       ___safe_se_handler_table   3161ae30     <linker-defined>
 0002:0000ce34       ___rtc_iaa                 3161ae34     MSVCRT:_initsect_.obj
 0002:0000ce38       ___rtc_izz                 3161ae38     MSVCRT:_initsect_.obj
 0002:0000ce3c       ___rtc_taa                 3161ae3c     MSVCRT:_initsect_.obj
 0002:0000ce40       ___rtc_tzz                 3161ae40     MSVCRT:_initsect_.obj
 0002:0000ceac       __IMPORT_DESCRIPTOR_KERNEL32 3161aeac     kernel32:KERNEL32.dll
 0002:0000cec0       __IMPORT_DESCRIPTOR_USER32 3161aec0     user32:USER32.dll
 0002:0000ced4       __IMPORT_DESCRIPTOR_MSVCR100 3161aed4     MSVCRT:MSVCR100.dll
 0002:0000cee8       __NULL_IMPORT_DESCRIPTOR   3161aee8     kernel32:KERNEL32.dll
 0003:00000000       ?sEmptyStringBuffer@?1??_emptyHeader@?$CryStringT@D@@KAPAUStrHeader@2@XZ@4PAU32@A 3161c000     AnimEventList.obj
 0003:00000018       ?s_factory@CFactory@COperatorQueue@@0V12@A 3161c018     OperatorQueue.obj
 0003:0000002c       ?s_factory@CFactory@CPoseAlignerChain@@0V12@A 3161c02c     PoseAlignerChain.obj
 0003:00000040       ?s_factory@CFactory@CPoseMatching@@0V12@A 3161c040     PoseMatching.obj
 0003:00000054       ?g_firstValidator@SBatchUpdateValidator@@2U1@A 3161c054     SkeletonPhysics.obj
 0003:0000006c       ?szEyeBoneNames@CEyeMovementFaceAnim@@0PAPBDA 3161c06c     EyeMovementFaceAnim.obj
 0003:000002ac       ?g_leftLeg@@3PBDB          3161c2ac     GroundAlignment.obj
 0003:000002b0       ?g_rightLeg@@3PBDB         3161c2b0     GroundAlignment.obj
 0003:000002b4       ?s_factory@CFactory@CGroundAlignment@@0V12@A 3161c2b4     GroundAlignment.obj
 0003:000002c8       ?fVec3_OneZ@?$Vec3Constants@M@@2U?$Vec3_tpl@M@@B 3161c2c8     GroundAlignment.obj
 0003:000002d4       ?s_factory@CFactory@CPoseBlenderAim@@0V12@A 3161c2d4     PoseBlenderAim.obj
 0003:000002e8       ?s_factory@CFactory@CPoseBlenderLook@@0V12@A 3161c2e8     PoseBlenderLook.obj
 0003:00000308       ?g_arrLimbNames@?1??SetJointName@CModelJoint@@QAEXPBD@Z@4PAPBDA 3161c308     LoaderCGA.obj
 0003:00002118       ?strEmpty@@3PBDB           3161e118     ModelAnimationSet.obj
 0003:00002120       ?m_seed@CLCGRndGen@@0_KA   3161e120     AnimationBase.obj
 0003:00002148       ?g_DefaultAnim@@3VCAnimation@@A 3161e148     AnimationBase.obj
 0003:000021b0       ?g_IdentityQuatT@@3U?$QuatT_tpl@M@@A 3161e1b0     AnimationBase.obj
 0003:000021d0       ?g_Consoleself@@3UConsole@@A 3161e1d0     cvars.obj
 0003:00002390       ?fVec3_Zero@?$Vec3Constants@M@@2U?$Vec3_tpl@M@@B 3161e390     stdafx.obj
 0003:0000239c       ?fVec3_One@?$Vec3Constants@M@@2U?$Vec3_tpl@M@@B 3161e39c     stdafx.obj
 0003:000023a8       ?fVec2_Zero@?$Vec2Constants@M@@2U?$Vec2_tpl@M@@A 3161e3a8     stdafx.obj
 0003:000023b0       ?fVec2_OneX@?$Vec2Constants@M@@2U?$Vec2_tpl@M@@A 3161e3b0     stdafx.obj
 0003:000023b8       ?fVec2_OneY@?$Vec2Constants@M@@2U?$Vec2_tpl@M@@A 3161e3b8     stdafx.obj
 0003:000023c0       ?fVec2_One@?$Vec2Constants@M@@2U?$Vec2_tpl@M@@A 3161e3c0     stdafx.obj
 0003:000023d0       ___native_dllmain_reason   3161e3d0     MSVCRT:natstart.obj
 0003:000023d4       ___native_vcclrit_reason   3161e3d4     MSVCRT:natstart.obj
 0003:000023d8       ___security_cookie         3161e3d8     MSVCRT:gs_cookie.obj
 0003:000023dc       ___security_cookie_complement 3161e3dc     MSVCRT:gs_cookie.obj
 0003:000023e0       ?s_used_memory@?1??_usedMemory@?$CryStringT@D@@SAIH@Z@4IA 3161e3e0     AnimEventList.obj
 0003:000023e4       ?s_EmptyElems@?1??set_null@?$SmallDynStorage@VCAnimEventData@@HUStandardAlloc@NAlloc@@@NArray@@IAEXXZ@4PAVCAnimEventData@@A 3161e3e4     AnimEventList.obj
 0003:000023e8       ?s_EmptyHeader@?1??set_null@?$SmallDynStorage@VCAnimEventData@@HUStandardAlloc@NAlloc@@@NArray@@IAEXXZ@4UEmptyHeader@23@A 3161e3e8     AnimEventList.obj
 0003:000023f0       ??_B?1??set_null@?$SmallDynStorage@VCAnimEventData@@HUStandardAlloc@NAlloc@@@NArray@@IAEXXZ@51 3161e3f0     AnimEventList.obj
 0003:000023f4       ?s_pMemReplay@?1??CryGetIMemReplay@@YAPAUIMemReplay@@XZ@4PAU2@A 3161e3f4     AnimEventList.obj
 0003:000023f8       ?s_dummyMemReplay@?1??CryGetIMemReplay@@YAPAUIMemReplay@@XZ@4UCDummyMemReplay@@A 3161e3f8     AnimEventList.obj
 0003:000023fc       ??_B?1??CryGetIMemReplay@@YAPAUIMemReplay@@XZ@51 3161e3fc     AnimEventList.obj
 0003:00002400       ?s_EmptyElems@?1??set_null@?$SmallDynStorage@EHUStandardAlloc@NAlloc@@@NArray@@IAEXXZ@4PAEA 3161e400     Attachment.obj
 0003:00002404       ?s_EmptyHeader@?1??set_null@?$SmallDynStorage@EHUStandardAlloc@NAlloc@@@NArray@@IAEXXZ@4UEmptyHeader@23@A 3161e404     Attachment.obj
 0003:0000240c       ??_B?1??set_null@?$SmallDynStorage@EHUStandardAlloc@NAlloc@@@NArray@@IAEXXZ@51 3161e40c     Attachment.obj
 0003:000027f4       ?s_used_memory@?1??_usedMemory@?$CryStackStringT@D$0CAA@@@SAII@Z@4IA 3161e7f4     LoaderSKIN.obj
 0003:000027f8       ?s_EmptyElems@?1??set_null@?$SmallDynStorage@UMorphTargetVertex@@HUStandardAlloc@NAlloc@@@NArray@@IAEXXZ@4PAUMorphTargetVertex@@A 3161e7f8     LoaderSKIN.obj
 0003:000027fc       ?s_EmptyHeader@?1??set_null@?$SmallDynStorage@UMorphTargetVertex@@HUStandardAlloc@NAlloc@@@NArray@@IAEXXZ@4UEmptyHeader@23@A 3161e7fc     LoaderSKIN.obj
 0003:00002804       ??_B?1??set_null@?$SmallDynStorage@UMorphTargetVertex@@HUStandardAlloc@NAlloc@@@NArray@@IAEXXZ@51 3161e804     LoaderSKIN.obj
 0003:00002808       ?s_EmptyElems@?1??set_null@?$SmallDynStorage@UExtSkinVertex@@HUStandardAlloc@NAlloc@@@NArray@@IAEXXZ@4PAUExtSkinVertex@@A 3161e808     LoaderSKIN.obj
 0003:0000280c       ?s_EmptyHeader@?1??set_null@?$SmallDynStorage@UExtSkinVertex@@HUStandardAlloc@NAlloc@@@NArray@@IAEXXZ@4UEmptyHeader@23@A 3161e80c     LoaderSKIN.obj
 0003:00002814       ??_B?1??set_null@?$SmallDynStorage@UExtSkinVertex@@HUStandardAlloc@NAlloc@@@NArray@@IAEXXZ@51 3161e814     LoaderSKIN.obj
 0003:00002818       ?s_EmptyElems@?1??set_null@?$SmallDynStorage@VCModelMesh@@HUStandardAlloc@NAlloc@@@NArray@@IAEXXZ@4PAVCModelMesh@@A 3161e818     LoaderSKIN.obj
 0003:0000281c       ?s_EmptyHeader@?1??set_null@?$SmallDynStorage@VCModelMesh@@HUStandardAlloc@NAlloc@@@NArray@@IAEXXZ@4UEmptyHeader@23@A 3161e81c     LoaderSKIN.obj
 0003:00002824       ??_B?1??set_null@?$SmallDynStorage@VCModelMesh@@HUStandardAlloc@NAlloc@@@NArray@@IAEXXZ@51 3161e824     LoaderSKIN.obj
 0003:00002828       ?s_EmptyElems@?1??set_null@?$SmallDynStorage@USJointInfo@CSkin@@HUStandardAlloc@NAlloc@@@NArray@@IAEXXZ@4PAUSJointInfo@CSkin@@A 3161e828     LoaderSKIN.obj
 0003:0000282c       ?s_EmptyHeader@?1??set_null@?$SmallDynStorage@USJointInfo@CSkin@@HUStandardAlloc@NAlloc@@@NArray@@IAEXXZ@4UEmptyHeader@23@A 3161e82c     LoaderSKIN.obj
 0003:00002834       ??_B?1??set_null@?$SmallDynStorage@USJointInfo@CSkin@@HUStandardAlloc@NAlloc@@@NArray@@IAEXXZ@51 3161e834     LoaderSKIN.obj
 0003:00002838       ?s_EmptyElems@?1??set_null@?$SmallDynStorage@U?$Vec3_tpl@M@@HUStandardAlloc@NAlloc@@@NArray@@IAEXXZ@4PAU?$Vec3_tpl@M@@A 3161e838     LoaderSKIN.obj
 0003:0000283c       ?s_EmptyHeader@?1??set_null@?$SmallDynStorage@U?$Vec3_tpl@M@@HUStandardAlloc@NAlloc@@@NArray@@IAEXXZ@4UEmptyHeader@23@A 3161e83c     LoaderSKIN.obj
 0003:00002844       ??_B?1??set_null@?$SmallDynStorage@U?$Vec3_tpl@M@@HUStandardAlloc@NAlloc@@@NArray@@IAEXXZ@51 3161e844     LoaderSKIN.obj
 0003:00002848       ?s_EmptyElems@?1??set_null@?$SmallDynStorage@U?$Quat_tpl@M@@HUStandardAlloc@NAlloc@@@NArray@@IAEXXZ@4PAU?$Quat_tpl@M@@A 3161e848     LoaderSKIN.obj
 0003:0000284c       ?s_EmptyHeader@?1??set_null@?$SmallDynStorage@U?$Quat_tpl@M@@HUStandardAlloc@NAlloc@@@NArray@@IAEXXZ@4UEmptyHeader@23@A 3161e84c     LoaderSKIN.obj
 0003:00002854       ??_B?1??set_null@?$SmallDynStorage@U?$Quat_tpl@M@@HUStandardAlloc@NAlloc@@@NArray@@IAEXXZ@51 3161e854     LoaderSKIN.obj
 0003:00002858       ?s_EmptyElems@?1??set_null@?$SmallDynStorage@URChunk@@HUStandardAlloc@NAlloc@@@NArray@@IAEXXZ@4PAURChunk@@A 3161e858     LoaderSKIN.obj
 0003:0000285c       ?s_EmptyHeader@?1??set_null@?$SmallDynStorage@URChunk@@HUStandardAlloc@NAlloc@@@NArray@@IAEXXZ@4UEmptyHeader@23@A 3161e85c     LoaderSKIN.obj
 0003:00002864       ??_B?1??set_null@?$SmallDynStorage@URChunk@@HUStandardAlloc@NAlloc@@@NArray@@IAEXXZ@51 3161e864     LoaderSKIN.obj
 0003:00002868       ?s_EmptyElems@?1??set_null@?$SmallDynStorage@UBoneIndices8@@HUStandardAlloc@NAlloc@@@NArray@@IAEXXZ@4PAUBoneIndices8@@A 3161e868     LoaderSKIN.obj
 0003:0000286c       ?s_EmptyHeader@?1??set_null@?$SmallDynStorage@UBoneIndices8@@HUStandardAlloc@NAlloc@@@NArray@@IAEXXZ@4UEmptyHeader@23@A 3161e86c     LoaderSKIN.obj
 0003:00002874       ??_B?1??set_null@?$SmallDynStorage@UBoneIndices8@@HUStandardAlloc@NAlloc@@@NArray@@IAEXXZ@51 3161e874     LoaderSKIN.obj
 0003:00002878       ?s_EmptyElems@?1??set_null@?$SmallDynStorage@UBoneWeights8@@HUStandardAlloc@NAlloc@@@NArray@@IAEXXZ@4PAUBoneWeights8@@A 3161e878     LoaderSKIN.obj
 0003:0000287c       ?s_EmptyHeader@?1??set_null@?$SmallDynStorage@UBoneWeights8@@HUStandardAlloc@NAlloc@@@NArray@@IAEXXZ@4UEmptyHeader@23@A 3161e87c     LoaderSKIN.obj
 0003:00002884       ??_B?1??set_null@?$SmallDynStorage@UBoneWeights8@@HUStandardAlloc@NAlloc@@@NArray@@IAEXXZ@51 3161e884     LoaderSKIN.obj
 0003:00002888       ?s_EmptyElems@?1??set_null@?$SmallDynStorage@V?$_smart_ptr@UCMorphTarget@@@@HUStandardAlloc@NAlloc@@@NArray@@IAEXXZ@4PAV?$_smart_ptr@UCMorphTarget@@@@A 3161e888     LoaderSKIN.obj
 0003:0000288c       ?s_EmptyHeader@?1??set_null@?$SmallDynStorage@V?$_smart_ptr@UCMorphTarget@@@@HUStandardAlloc@NAlloc@@@NArray@@IAEXXZ@4UEmptyHeader@23@A 3161e88c     LoaderSKIN.obj
 0003:00002894       ??_B?1??set_null@?$SmallDynStorage@V?$_smart_ptr@UCMorphTarget@@@@HUStandardAlloc@NAlloc@@@NArray@@IAEXXZ@51 3161e894     LoaderSKIN.obj
 0003:00002898       ?BIAS_SCALE_16BIT@?6??FromFrameReflection@QTangent@@YA?AU?$Quat_tpl@M@@U3@M@Z@4MB 3161e898     LoaderSKIN.obj
 0003:0000289c       ??_B?6??FromFrameReflection@QTangent@@YA?AU?$Quat_tpl@M@@U2@M@Z@56 3161e89c     LoaderSKIN.obj
 0003:00002c84       ?s_EmptyElems@?1??set_null@?$SmallDynStorage@PAVCAttachmentSKIN@@HUStandardAlloc@NAlloc@@@NArray@@IAEXXZ@4PAPAVCAttachmentSKIN@@A 3161ec84     ModelSkin.obj
 0003:00002c88       ?s_EmptyHeader@?1??set_null@?$SmallDynStorage@PAVCAttachmentSKIN@@HUStandardAlloc@NAlloc@@@NArray@@IAEXXZ@4UEmptyHeader@23@A 3161ec88     ModelSkin.obj
 0003:00002c90       ??_B?1??set_null@?$SmallDynStorage@PAVCAttachmentSKIN@@HUStandardAlloc@NAlloc@@@NArray@@IAEXXZ@51 3161ec90     ModelSkin.obj
 0003:00002c94       ?pClouds@?1??InitRenderingFlags@SRenderingPassInfo@@AAEXI@Z@4PAUICVar@@A 3161ec94     ParametricSampler.obj
 0003:00002c98       ?pRoads@?1??InitRenderingFlags@SRenderingPassInfo@@AAEXI@Z@4PAUICVar@@A 3161ec98     ParametricSampler.obj
 0003:00002c9c       ?pWaterVolumes@?1??InitRenderingFlags@SRenderingPassInfo@@AAEXI@Z@4PAUICVar@@A 3161ec9c     ParametricSampler.obj
 0003:00002ca0       ?pWaterWaves@?1??InitRenderingFlags@SRenderingPassInfo@@AAEXI@Z@4PAUICVar@@A 3161eca0     ParametricSampler.obj
 0003:00002ca4       ?pDecals@?1??InitRenderingFlags@SRenderingPassInfo@@AAEXI@Z@4PAUICVar@@A 3161eca4     ParametricSampler.obj
 0003:00002ca8       ?pParticles@?1??InitRenderingFlags@SRenderingPassInfo@@AAEXI@Z@4PAUICVar@@A 3161eca8     ParametricSampler.obj
 0003:00002cac       ?pWaterOcean@?1??InitRenderingFlags@SRenderingPassInfo@@AAEXI@Z@4PAUICVar@@A 3161ecac     ParametricSampler.obj
 0003:00002cb0       ?pTerrain@?1??InitRenderingFlags@SRenderingPassInfo@@AAEXI@Z@4PAUICVar@@A 3161ecb0     ParametricSampler.obj
 0003:00002cb4       ?pEntities@?1??InitRenderingFlags@SRenderingPassInfo@@AAEXI@Z@4PAUICVar@@A 3161ecb4     ParametricSampler.obj
 0003:00002cb8       ?pVegetation@?1??InitRenderingFlags@SRenderingPassInfo@@AAEXI@Z@4PAUICVar@@A 3161ecb8     ParametricSampler.obj
 0003:00002cbc       ?pBrushes@?1??InitRenderingFlags@SRenderingPassInfo@@AAEXI@Z@4PAUICVar@@A 3161ecbc     ParametricSampler.obj
 0003:00002cc0       ?pShadows@?1??InitRenderingFlags@SRenderingPassInfo@@AAEXI@Z@4PAUICVar@@A 3161ecc0     ParametricSampler.obj
 0003:00002cc4       ?pVoxTer@?1??InitRenderingFlags@SRenderingPassInfo@@AAEXI@Z@4PAUICVar@@A 3161ecc4     ParametricSampler.obj
 0003:00002cc8       ?pVoxel@?1??InitRenderingFlags@SRenderingPassInfo@@AAEXI@Z@4PAUICVar@@A 3161ecc8     ParametricSampler.obj
 0003:00002ccc       ?pDefaultMaterial@?1??InitRenderingFlags@SRenderingPassInfo@@AAEXI@Z@4PAUICVar@@A 3161eccc     ParametricSampler.obj
 0003:00002cd0       ??_B?1??InitRenderingFlags@SRenderingPassInfo@@AAEXI@Z@51 3161ecd0     ParametricSampler.obj
 0003:00002cd4       ?pCameraFreeze@?1??CreateGeneralPassRenderingInfo@SRenderingPassInfo@@SA?AU2@ABVCCamera@@I@Z@4PAUICVar@@A 3161ecd4     ParametricSampler.obj
 0003:00002cd8       ??_B?1??CreateGeneralPassRenderingInfo@SRenderingPassInfo@@SA?AU1@ABVCCamera@@I@Z@51 3161ecd8     ParametricSampler.obj
 0003:00002cdc       ?s_EmptyElems@?1??set_null@?$SmallDynStorage@UVirtualExample1D@@HUStandardAlloc@NAlloc@@@NArray@@IAEXXZ@4PAUVirtualExample1D@@A 3161ecdc     ParametricSampler.obj
 0003:00002ce0       ?s_EmptyHeader@?1??set_null@?$SmallDynStorage@UVirtualExample1D@@HUStandardAlloc@NAlloc@@@NArray@@IAEXXZ@4UEmptyHeader@23@A 3161ece0     ParametricSampler.obj
 0003:00002ce8       ??_B?1??set_null@?$SmallDynStorage@UVirtualExample1D@@HUStandardAlloc@NAlloc@@@NArray@@IAEXXZ@51 3161ece8     ParametricSampler.obj
 0003:00002cec       ?s_EmptyElems@?1??set_null@?$SmallDynStorage@UVirtualExample2D@@HUStandardAlloc@NAlloc@@@NArray@@IAEXXZ@4PAUVirtualExample2D@@A 3161ecec     ParametricSampler.obj
 0003:00002cf0       ?s_EmptyHeader@?1??set_null@?$SmallDynStorage@UVirtualExample2D@@HUStandardAlloc@NAlloc@@@NArray@@IAEXXZ@4UEmptyHeader@23@A 3161ecf0     ParametricSampler.obj
 0003:00002cf8       ??_B?1??set_null@?$SmallDynStorage@UVirtualExample2D@@HUStandardAlloc@NAlloc@@@NArray@@IAEXXZ@51 3161ecf8     ParametricSampler.obj
 0003:00002cfc       ?s_EmptyElems@?1??set_null@?$SmallDynStorage@UVirtualExample3D@@HUStandardAlloc@NAlloc@@@NArray@@IAEXXZ@4PAUVirtualExample3D@@A 3161ecfc     ParametricSampler.obj
 0003:00002d00       ?s_EmptyHeader@?1??set_null@?$SmallDynStorage@UVirtualExample3D@@HUStandardAlloc@NAlloc@@@NArray@@IAEXXZ@4UEmptyHeader@23@A 3161ed00     ParametricSampler.obj
 0003:00002d08       ??_B?1??set_null@?$SmallDynStorage@UVirtualExample3D@@HUStandardAlloc@NAlloc@@@NArray@@IAEXXZ@51 3161ed08     ParametricSampler.obj
 0003:00002d58       ?s_globalObjectCount@CPlaceholderCharacter@@0HA 3161ed58     PlaceholderCharacter.obj
 0003:00002d5c       ?s_EmptyElems@?1??set_null@?$SmallDynStorage@V?$_smart_ptr@VIController@@@@HUStandardAlloc@NAlloc@@@NArray@@IAEXXZ@4PAV?$_smart_ptr@VIController@@@@A 3161ed5c     DirectionalBlender.obj
 0003:00002d60       ?s_EmptyHeader@?1??set_null@?$SmallDynStorage@V?$_smart_ptr@VIController@@@@HUStandardAlloc@NAlloc@@@NArray@@IAEXXZ@4UEmptyHeader@23@A 3161ed60     DirectionalBlender.obj
 0003:00002d68       ??_B?1??set_null@?$SmallDynStorage@V?$_smart_ptr@VIController@@@@HUStandardAlloc@NAlloc@@@NArray@@IAEXXZ@51 3161ed68     DirectionalBlender.obj
 0003:00002d6c       ?s_EmptyElems@?1??set_null@?$SmallDynStorage@UAimIKPose@@HUStandardAlloc@NAlloc@@@NArray@@IAEXXZ@4PAUAimIKPose@@A 3161ed6c     DirectionalBlender.obj
 0003:00002d70       ?s_EmptyHeader@?1??set_null@?$SmallDynStorage@UAimIKPose@@HUStandardAlloc@NAlloc@@@NArray@@IAEXXZ@4UEmptyHeader@23@A 3161ed70     DirectionalBlender.obj
 0003:00002d78       ??_B?1??set_null@?$SmallDynStorage@UAimIKPose@@HUStandardAlloc@NAlloc@@@NArray@@IAEXXZ@51 3161ed78     DirectionalBlender.obj
 0003:00002d7c       ?s_EmptyElems@?1??set_null@?$SmallDynStorage@UVirtualExampleInit2@CHUNK_GAHAIM_INFO@@HUStandardAlloc@NAlloc@@@NArray@@IAEXXZ@4PAUVirtualExampleInit2@CHUNK_GAHAIM_INFO@@A 3161ed7c     DirectionalBlender.obj
 0003:00002d80       ?s_EmptyHeader@?1??set_null@?$SmallDynStorage@UVirtualExampleInit2@CHUNK_GAHAIM_INFO@@HUStandardAlloc@NAlloc@@@NArray@@IAEXXZ@4UEmptyHeader@23@A 3161ed80     DirectionalBlender.obj
 0003:00002d88       ??_B?1??set_null@?$SmallDynStorage@UVirtualExampleInit2@CHUNK_GAHAIM_INFO@@HUStandardAlloc@NAlloc@@@NArray@@IAEXXZ@51 3161ed88     DirectionalBlender.obj
 0003:00002db8       ?supportedIIDs@?1???0CFactory@COperatorQueue@@AAE@XZ@4PAUCryGUID@@A 3161edb8     OperatorQueue.obj
 0003:00002df0       ?supportedIIDs@?1???0CFactory@CPoseAlignerChain@@AAE@XZ@4PAUCryGUID@@A 3161edf0     PoseAlignerChain.obj
 0003:00002e20       ?supportedIIDs@?1???0CFactory@CPoseMatching@@AAE@XZ@4PAUCryGUID@@A 3161ee20     PoseMatching.obj
 0003:00002e50       ?g_lockList@SBatchUpdateValidator@@2HC 3161ee50     SkeletonPhysics.obj
 0003:00002e54       ?s_EmptyElems@?1??set_null@?$SmallDynStorage@U?$QuatT_tpl@M@@HUStandardAlloc@NAlloc@@@NArray@@IAEXXZ@4PAU?$QuatT_tpl@M@@A 3161ee54     SkeletonPhysics.obj
 0003:00002e58       ?s_EmptyHeader@?1??set_null@?$SmallDynStorage@U?$QuatT_tpl@M@@HUStandardAlloc@NAlloc@@@NArray@@IAEXXZ@4UEmptyHeader@23@A 3161ee58     SkeletonPhysics.obj
 0003:00002e60       ??_B?1??set_null@?$SmallDynStorage@U?$QuatT_tpl@M@@HUStandardAlloc@NAlloc@@@NArray@@IAEXXZ@51 3161ee60     SkeletonPhysics.obj
 0003:00002e64       ?s_EmptyElems@?1??set_null@?$SmallDynStorage@HHUStandardAlloc@NAlloc@@@NArray@@IAEXXZ@4PAHA 3161ee64     SkeletonPhysics.obj
 0003:00002e68       ?s_EmptyHeader@?1??set_null@?$SmallDynStorage@HHUStandardAlloc@NAlloc@@@NArray@@IAEXXZ@4UEmptyHeader@23@A 3161ee68     SkeletonPhysics.obj
 0003:00002e70       ??_B?1??set_null@?$SmallDynStorage@HHUStandardAlloc@NAlloc@@@NArray@@IAEXXZ@51 3161ee70     SkeletonPhysics.obj
 0003:000031ec       ?s_EmptyElems@?1??set_null@?$SmallDynStorage@UCPhysicsJoint@@HUStandardAlloc@NAlloc@@@NArray@@IAEXXZ@4PAUCPhysicsJoint@@A 3161f1ec     SkeletonPhysics.obj
 0003:000031f0       ?s_EmptyHeader@?1??set_null@?$SmallDynStorage@UCPhysicsJoint@@HUStandardAlloc@NAlloc@@@NArray@@IAEXXZ@4UEmptyHeader@23@A 3161f1f0     SkeletonPhysics.obj
 0003:000031f8       ??_B?1??set_null@?$SmallDynStorage@UCPhysicsJoint@@HUStandardAlloc@NAlloc@@@NArray@@IAEXXZ@51 3161f1f8     SkeletonPhysics.obj
 0003:00004354       ?s_EmptyElems@?1??set_null@?$SmallDynStorage@USEntry@CPoseModifierQueue@@HUStandardAlloc@NAlloc@@@NArray@@IAEXXZ@4PAUSEntry@CPoseModifierQueue@@A 31620354     TransitionQueue.obj
 0003:00004358       ?s_EmptyHeader@?1??set_null@?$SmallDynStorage@USEntry@CPoseModifierQueue@@HUStandardAlloc@NAlloc@@@NArray@@IAEXXZ@4UEmptyHeader@23@A 31620358     TransitionQueue.obj
 0003:00004360       ??_B?1??set_null@?$SmallDynStorage@USEntry@CPoseModifierQueue@@HUStandardAlloc@NAlloc@@@NArray@@IAEXXZ@51 31620360     TransitionQueue.obj
 0003:00004364       ?s_EmptyElems@?1??set_null@?$SmallDynStorage@VCAnimation@@HUStandardAlloc@NAlloc@@@NArray@@IAEXXZ@4PAVCAnimation@@A 31620364     TransitionQueue.obj
 0003:00004368       ?s_EmptyHeader@?1??set_null@?$SmallDynStorage@VCAnimation@@HUStandardAlloc@NAlloc@@@NArray@@IAEXXZ@4UEmptyHeader@23@A 31620368     TransitionQueue.obj
 0003:00004370       ??_B?1??set_null@?$SmallDynStorage@VCAnimation@@HUStandardAlloc@NAlloc@@@NArray@@IAEXXZ@51 31620370     TransitionQueue.obj
 0003:00004374       ?s_EmptyElems@?1??set_null@?$SmallDynStorage@USVertexFrameState@@HUStandardAlloc@NAlloc@@@NArray@@IAEXXZ@4PAUSVertexFrameState@@A 31620374     VertexAnimation.obj
 0003:00004378       ?s_EmptyHeader@?1??set_null@?$SmallDynStorage@USVertexFrameState@@HUStandardAlloc@NAlloc@@@NArray@@IAEXXZ@4UEmptyHeader@23@A 31620378     VertexAnimation.obj
 0003:00004380       ??_B?1??set_null@?$SmallDynStorage@USVertexFrameState@@HUStandardAlloc@NAlloc@@@NArray@@IAEXXZ@51 31620380     VertexAnimation.obj
 0003:00004384       ?s_EmptyElems@?1??set_null@?$SmallDynStorage@USVF_P3F@@HUStandardAlloc@NAlloc@@@NArray@@IAEXXZ@4PAUSVF_P3F@@A 31620384     VertexData.obj
 0003:00004388       ?s_EmptyHeader@?1??set_null@?$SmallDynStorage@USVF_P3F@@HUStandardAlloc@NAlloc@@@NArray@@IAEXXZ@4UEmptyHeader@23@A 31620388     VertexData.obj
 0003:00004390       ??_B?1??set_null@?$SmallDynStorage@USVF_P3F@@HUStandardAlloc@NAlloc@@@NArray@@IAEXXZ@51 31620390     VertexData.obj
 0003:00004ad0       ?s_EmptyElems@?1??set_null@?$SmallDynStorage@V?$_smart_ptr@UIAttachment@@@@HUStandardAlloc@NAlloc@@@NArray@@IAEXXZ@4PAV?$_smart_ptr@UIAttachment@@@@A 31620ad0     AttachmentManager.obj
 0003:00004ad4       ?s_EmptyHeader@?1??set_null@?$SmallDynStorage@V?$_smart_ptr@UIAttachment@@@@HUStandardAlloc@NAlloc@@@NArray@@IAEXXZ@4UEmptyHeader@23@A 31620ad4     AttachmentManager.obj
 0003:00004adc       ??_B?1??set_null@?$SmallDynStorage@V?$_smart_ptr@UIAttachment@@@@HUStandardAlloc@NAlloc@@@NArray@@IAEXXZ@51 31620adc     AttachmentManager.obj
 0003:00004ae0       ?s_EmptyElems@?1??set_null@?$SmallDynStorage@UCharacterAttachment@@HUStandardAlloc@NAlloc@@@NArray@@IAEXXZ@4PAUCharacterAttachment@@A 31620ae0     AttachmentManager.obj
 0003:00004ae4       ?s_EmptyHeader@?1??set_null@?$SmallDynStorage@UCharacterAttachment@@HUStandardAlloc@NAlloc@@@NArray@@IAEXXZ@4UEmptyHeader@23@A 31620ae4     AttachmentManager.obj
 0003:00004aec       ??_B?1??set_null@?$SmallDynStorage@UCharacterAttachment@@HUStandardAlloc@NAlloc@@@NArray@@IAEXXZ@51 31620aec     AttachmentManager.obj
 0003:000051dc       ?gJobHandleTSkinningTransformationsComputation@Detail@JobManager@@3PAUSJobStringHandle@2@A 316211dc     CharacterInstance.obj
 0003:000051e0       ?s_EmptyElems@?1??set_null@?$SmallDynStorage@MHUStandardAlloc@NAlloc@@@NArray@@IAEXXZ@4PAMA 316211e0     CharacterInstance.obj
 0003:000051e4       ?s_EmptyHeader@?1??set_null@?$SmallDynStorage@MHUStandardAlloc@NAlloc@@@NArray@@IAEXXZ@4UEmptyHeader@23@A 316211e4     CharacterInstance.obj
 0003:000051ec       ??_B?1??set_null@?$SmallDynStorage@MHUStandardAlloc@NAlloc@@@NArray@@IAEXXZ@51 316211ec     CharacterInstance.obj
 0003:000051f0       ?s_EmptyElems@?1??set_null@?$SmallDynStorage@UGeomQuery@@HUStandardAlloc@NAlloc@@@NArray@@IAEXXZ@4PAUGeomQuery@@A 316211f0     CharacterInstance.obj
 0003:000051f4       ?s_EmptyHeader@?1??set_null@?$SmallDynStorage@UGeomQuery@@HUStandardAlloc@NAlloc@@@NArray@@IAEXXZ@4UEmptyHeader@23@A 316211f4     CharacterInstance.obj
 0003:000051fc       ??_B?1??set_null@?$SmallDynStorage@UGeomQuery@@HUStandardAlloc@NAlloc@@@NArray@@IAEXXZ@51 316211fc     CharacterInstance.obj
 0003:00005200       ?s_EmptyElems@?1??set_null@?$SmallDynStorage@_NHUStandardAlloc@NAlloc@@@NArray@@IAEXXZ@4PA_NA 31621200     CharacterInstance.obj
 0003:00005204       ?s_EmptyHeader@?1??set_null@?$SmallDynStorage@_NHUStandardAlloc@NAlloc@@@NArray@@IAEXXZ@4UEmptyHeader@23@A 31621204     CharacterInstance.obj
 0003:0000520c       ??_B?1??set_null@?$SmallDynStorage@_NHUStandardAlloc@NAlloc@@@NArray@@IAEXXZ@51 3162120c     CharacterInstance.obj
 0003:00005210       ?s_EmptyElems@?1??set_null@?$SmallDynStorage@IHUStandardAlloc@NAlloc@@@NArray@@IAEXXZ@4PAIA 31621210     CharacterInstance.obj
 0003:00005214       ?s_EmptyHeader@?1??set_null@?$SmallDynStorage@IHUStandardAlloc@NAlloc@@@NArray@@IAEXXZ@4UEmptyHeader@23@A 31621214     CharacterInstance.obj
 0003:0000521c       ??_B?1??set_null@?$SmallDynStorage@IHUStandardAlloc@NAlloc@@@NArray@@IAEXXZ@51 3162121c     CharacterInstance.obj
 0003:00005220       ?s_EmptyElems@?1??set_null@?$SmallDynStorage@V?$CryStringT@D@@HUStandardAlloc@NAlloc@@@NArray@@IAEXXZ@4PAV?$CryStringT@D@@A 31621220     CharacterInstance.obj
 0003:00005224       ?s_EmptyHeader@?1??set_null@?$SmallDynStorage@V?$CryStringT@D@@HUStandardAlloc@NAlloc@@@NArray@@IAEXXZ@4UEmptyHeader@23@A 31621224     CharacterInstance.obj
 0003:0000522c       ??_B?1??set_null@?$SmallDynStorage@V?$CryStringT@D@@HUStandardAlloc@NAlloc@@@NArray@@IAEXXZ@51 3162122c     CharacterInstance.obj
 0003:00005c9c       ?g_arrVerticesBS@@3V?$vector@U?$Vec3_tpl@M@@V?$allocator@U?$Vec3_tpl@M@@@stlpmtx_std@@@stlpmtx_std@@A 31621c9c     DecalManager.obj
 0003:00005ca8       ?g_arrDecalVertexMapping@@3V?$vector@HV?$allocator@H@stlpmtx_std@@@stlpmtx_std@@A 31621ca8     DecalManager.obj
 0003:00005cb4       ?g_arrDecalFaceMapping@@3V?$vector@HV?$allocator@H@stlpmtx_std@@@stlpmtx_std@@A 31621cb4     DecalManager.obj
 0003:00005cc0       ?s_EmptyElems@?1??set_null@?$SmallDynStorage@UEffectEntry@CSkeletonEffectManager@@HUStandardAlloc@NAlloc@@@NArray@@IAEXXZ@4PAUEffectEntry@CSkeletonEffectManager@@A 31621cc0     SkeletonEffectManager.obj
 0003:00005cc4       ?s_EmptyHeader@?1??set_null@?$SmallDynStorage@UEffectEntry@CSkeletonEffectManager@@HUStandardAlloc@NAlloc@@@NArray@@IAEXXZ@4UEmptyHeader@23@A 31621cc4     SkeletonEffectManager.obj
 0003:00005ccc       ??_B?1??set_null@?$SmallDynStorage@UEffectEntry@CSkeletonEffectManager@@HUStandardAlloc@NAlloc@@@NArray@@IAEXXZ@51 31621ccc     SkeletonEffectManager.obj
 0003:00005cd0       ?s_EmptyElems@?1??set_null@?$SmallDynStorage@UCCGAJoint@@HUStandardAlloc@NAlloc@@@NArray@@IAEXXZ@4PAUCCGAJoint@@A 31621cd0     SkeletonPose.obj
 0003:00005cd4       ?s_EmptyHeader@?1??set_null@?$SmallDynStorage@UCCGAJoint@@HUStandardAlloc@NAlloc@@@NArray@@IAEXXZ@4UEmptyHeader@23@A 31621cd4     SkeletonPose.obj
 0003:00005cdc       ??_B?1??set_null@?$SmallDynStorage@UCCGAJoint@@HUStandardAlloc@NAlloc@@@NArray@@IAEXXZ@51 31621cdc     SkeletonPose.obj
 0003:00005ce0       ?s_EmptyElems@?1??set_null@?$SmallDynStorage@USPostProcess@@HUStandardAlloc@NAlloc@@@NArray@@IAEXXZ@4PAUSPostProcess@@A 31621ce0     SkeletonPose.obj
 0003:00005ce4       ?s_EmptyHeader@?1??set_null@?$SmallDynStorage@USPostProcess@@HUStandardAlloc@NAlloc@@@NArray@@IAEXXZ@4UEmptyHeader@23@A 31621ce4     SkeletonPose.obj
 0003:00005cec       ??_B?1??set_null@?$SmallDynStorage@USPostProcess@@HUStandardAlloc@NAlloc@@@NArray@@IAEXXZ@51 31621cec     SkeletonPose.obj
 0003:00006780       ?gJobHandleTCommandBufferExecuteJob@Detail@JobManager@@3PAUSJobStringHandle@2@A 31622780     SkeletonAnim.obj
 0003:00006784       ?s_pMemoryPool@CSkeletonAnimTask@@0PAVCPoolFrameLocal@Memory@@A 31622784     SkeletonAnim.obj
 0003:00006788       ?GUID_AnimationPoseModifier_TransformationPin@@3UCryGUID@@A 31622788     SkeletonAnim.obj
 0003:00006798       ?instance@?1??Instance@CAnimationContext@@SAAAV2@XZ@4V2@A 31622798     SkeletonAnim.obj
 0003:0000679c       ??_B?1??Instance@CAnimationContext@@SAAAV1@XZ@51 3162279c     SkeletonAnim.obj
 0003:0000808c       ?s_EmptyElems@?1??set_null@?$SmallDynStorage@U?$SplineKey@M@spline@@HUStandardAlloc@NAlloc@@@NArray@@IAEXXZ@4PAU?$SplineKey@M@spline@@A 3162408c     FaceAnimSequence.obj
 0003:00008090       ?s_EmptyHeader@?1??set_null@?$SmallDynStorage@U?$SplineKey@M@spline@@HUStandardAlloc@NAlloc@@@NArray@@IAEXXZ@4UEmptyHeader@23@A 31624090     FaceAnimSequence.obj
 0003:00008098       ??_B?1??set_null@?$SmallDynStorage@U?$SplineKey@M@spline@@HUStandardAlloc@NAlloc@@@NArray@@IAEXXZ@51 31624098     FaceAnimSequence.obj
 0003:0000809c       ?s_EmptyElems@?1??set_null@?$SmallDynStorage@U?$SplineKey@U?$Quat_tpl@M@@@spline@@HUStandardAlloc@NAlloc@@@NArray@@IAEXXZ@4PAU?$SplineKey@U?$Quat_tpl@M@@@spline@@A 3162409c     FaceAnimSequence.obj
 0003:000080a0       ?s_EmptyHeader@?1??set_null@?$SmallDynStorage@U?$SplineKey@U?$Quat_tpl@M@@@spline@@HUStandardAlloc@NAlloc@@@NArray@@IAEXXZ@4UEmptyHeader@23@A 316240a0     FaceAnimSequence.obj
 0003:000080a8       ??_B?1??set_null@?$SmallDynStorage@U?$SplineKey@U?$Quat_tpl@M@@@spline@@HUStandardAlloc@NAlloc@@@NArray@@IAEXXZ@51 316240a8     FaceAnimSequence.obj
 0003:000080ac       ?s_EmptyElems@?1??set_null@?$SmallDynStorage@U?$TCBSplineKey@U?$Vec3_tpl@M@@@spline@@HUStandardAlloc@NAlloc@@@NArray@@IAEXXZ@4PAU?$TCBSplineKey@U?$Vec3_tpl@M@@@spline@@A 316240ac     FaceAnimSequence.obj
 0003:000080b0       ?s_EmptyHeader@?1??set_null@?$SmallDynStorage@U?$TCBSplineKey@U?$Vec3_tpl@M@@@spline@@HUStandardAlloc@NAlloc@@@NArray@@IAEXXZ@4UEmptyHeader@23@A 316240b0     FaceAnimSequence.obj
 0003:000080b8       ??_B?1??set_null@?$SmallDynStorage@U?$TCBSplineKey@U?$Vec3_tpl@M@@@spline@@HUStandardAlloc@NAlloc@@@NArray@@IAEXXZ@51 316240b8     FaceAnimSequence.obj
 0003:0000843c       ?s_EmptyElems@?1??set_null@?$SmallDynStorage@VCFacialAnimForcedRotationEntry@@HUStandardAlloc@NAlloc@@@NArray@@IAEXXZ@4PAVCFacialAnimForcedRotationEntry@@A 3162443c     FacialInstance.obj
 0003:00008440       ?s_EmptyHeader@?1??set_null@?$SmallDynStorage@VCFacialAnimForcedRotationEntry@@HUStandardAlloc@NAlloc@@@NArray@@IAEXXZ@4UEmptyHeader@23@A 31624440     FacialInstance.obj
 0003:00008448       ??_B?1??set_null@?$SmallDynStorage@VCFacialAnimForcedRotationEntry@@HUStandardAlloc@NAlloc@@@NArray@@IAEXXZ@51 31624448     FacialInstance.obj
 0003:000087d0       ?supportedIIDs@?1???0CFactory@CFeetPoseStore@@AAE@XZ@4PAUCryGUID@@A 316247d0     FeetLock.obj
 0003:000087f0       ?supportedIIDs@?1???0CFactory@CFeetPoseRestore@@AAE@XZ@4PAUCryGUID@@A 316247f0     FeetLock.obj
 0003:00008810       ?s_factory@CFactory@CFeetPoseStore@@0V12@A 31624810     FeetLock.obj
 0003:00008824       ?s_factory@CFactory@CFeetPoseRestore@@0V12@A 31624824     FeetLock.obj
 0003:00008838       ?supportedIIDs@?1???0CFactory@CGroundAlignment@@AAE@XZ@4PAUCryGUID@@A 31624838     GroundAlignment.obj
 0003:00008868       ?supportedIIDs@?1???0CFactory@CLimbIk@@AAE@XZ@4PAUCryGUID@@A 31624868     LimbIk.obj
 0003:00008888       ?s_factory@CFactory@CLimbIk@@0V12@A 31624888     LimbIk.obj
 0003:000088b0       ?supportedIIDs@?1???0CFactory@CPoseBlenderAim@@AAE@XZ@4PAUCryGUID@@A 316248b0     PoseBlenderAim.obj
 0003:000088f0       ?supportedIIDs@?1???0CFactory@CPoseBlenderLook@@AAE@XZ@4PAUCryGUID@@A 316248f0     PoseBlenderLook.obj
 0003:00008920       ?supportedIIDs@?1???0CFactory@CRecoil@PoseModifier@@AAE@XZ@4PAUCryGUID@@A 31624920     Recoil.obj
 0003:00008940       ?s_factory@CFactory@CRecoil@PoseModifier@@0V123@A 31624940     Recoil.obj
 0003:000093c4       ?g_result@Skeleton@@3IA    316253c4     Skeleton.obj
 0003:000093d0       ?g_YLine@@3MA              316253d0     CharacterManager.obj
 0003:000093d4       ?s_bPaused@CharacterManager@@2_NA 316253d4     CharacterManager.obj
 0003:000093d8       ?s_renderFrameIdLocal@CharacterManager@@2IA 316253d8     CharacterManager.obj
 0003:000093f8       ?s_EmptyElems@?1??set_null@?$SmallDynStorage@UDebugInstances@@HUStandardAlloc@NAlloc@@@NArray@@IAEXXZ@4PAUDebugInstances@@A 316253f8     CharacterManager.obj
 0003:000093fc       ?s_EmptyHeader@?1??set_null@?$SmallDynStorage@UDebugInstances@@HUStandardAlloc@NAlloc@@@NArray@@IAEXXZ@4UEmptyHeader@23@A 316253fc     CharacterManager.obj
 0003:00009404       ??_B?1??set_null@?$SmallDynStorage@UDebugInstances@@HUStandardAlloc@NAlloc@@@NArray@@IAEXXZ@51 31625404     CharacterManager.obj
 0003:00009408       ?s_EmptyElems@?1??set_null@?$SmallDynStorage@V?$TCBSpline@U?$Vec3_tpl@M@@U?$TCBSplineKey@U?$Vec3_tpl@M@@@spline@@@spline@@HUStandardAlloc@NAlloc@@@NArray@@IAEXXZ@4PAV?$TCBSpline@U?$Vec3_tpl@M@@U?$TCBSplineKey@U?$Vec3_tpl@M@@@spline@@@spline@@A 31625408     CharacterManager.obj
 0003:0000940c       ?s_EmptyHeader@?1??set_null@?$SmallDynStorage@V?$TCBSpline@U?$Vec3_tpl@M@@U?$TCBSplineKey@U?$Vec3_tpl@M@@@spline@@@spline@@HUStandardAlloc@NAlloc@@@NArray@@IAEXXZ@4UEmptyHeader@23@A 3162540c     CharacterManager.obj
 0003:00009414       ??_B?1??set_null@?$SmallDynStorage@V?$TCBSpline@U?$Vec3_tpl@M@@U?$TCBSplineKey@U?$Vec3_tpl@M@@@spline@@@spline@@HUStandardAlloc@NAlloc@@@NArray@@IAEXXZ@51 31625414     CharacterManager.obj
 0003:00009418       ?s_EmptyElems@?1??set_null@?$SmallDynStorage@VTCBAngleAxisSpline@spline@@HUStandardAlloc@NAlloc@@@NArray@@IAEXXZ@4PAVTCBAngleAxisSpline@spline@@A 31625418     CharacterManager.obj
 0003:0000941c       ?s_EmptyHeader@?1??set_null@?$SmallDynStorage@VTCBAngleAxisSpline@spline@@HUStandardAlloc@NAlloc@@@NArray@@IAEXXZ@4UEmptyHeader@23@A 3162541c     CharacterManager.obj
 0003:00009424       ??_B?1??set_null@?$SmallDynStorage@VTCBAngleAxisSpline@spline@@HUStandardAlloc@NAlloc@@@NArray@@IAEXXZ@51 31625424     CharacterManager.obj
 0003:00009428       ?s_EmptyElems@?1??set_null@?$SmallDynStorage@UCControllerType@@HUStandardAlloc@NAlloc@@@NArray@@IAEXXZ@4PAUCControllerType@@A 31625428     CharacterManager.obj
 0003:0000942c       ?s_EmptyHeader@?1??set_null@?$SmallDynStorage@UCControllerType@@HUStandardAlloc@NAlloc@@@NArray@@IAEXXZ@4UEmptyHeader@23@A 3162542c     CharacterManager.obj
 0003:00009434       ??_B?1??set_null@?$SmallDynStorage@UCControllerType@@HUStandardAlloc@NAlloc@@@NArray@@IAEXXZ@51 31625434     CharacterManager.obj
 0003:00009438       ?s_EmptyElems@?1??set_null@?$SmallDynStorage@UNodeDesc@@HUStandardAlloc@NAlloc@@@NArray@@IAEXXZ@4PAUNodeDesc@@A 31625438     CharacterManager.obj
 0003:0000943c       ?s_EmptyHeader@?1??set_null@?$SmallDynStorage@UNodeDesc@@HUStandardAlloc@NAlloc@@@NArray@@IAEXXZ@4UEmptyHeader@23@A 3162543c     CharacterManager.obj
 0003:00009444       ??_B?1??set_null@?$SmallDynStorage@UNodeDesc@@HUStandardAlloc@NAlloc@@@NArray@@IAEXXZ@51 31625444     CharacterManager.obj
 0003:00009448       ?s_EmptyElems@?1??set_null@?$SmallDynStorage@UCControllerTCB@@HUStandardAlloc@NAlloc@@@NArray@@IAEXXZ@4PAUCControllerTCB@@A 31625448     CharacterManager.obj
 0003:0000944c       ?s_EmptyHeader@?1??set_null@?$SmallDynStorage@UCControllerTCB@@HUStandardAlloc@NAlloc@@@NArray@@IAEXXZ@4UEmptyHeader@23@A 3162544c     CharacterManager.obj
 0003:00009454       ??_B?1??set_null@?$SmallDynStorage@UCControllerTCB@@HUStandardAlloc@NAlloc@@@NArray@@IAEXXZ@51 31625454     CharacterManager.obj
 0003:00009458       ?s_EmptyElems@?1??set_null@?$SmallDynStorage@UCGlobalHeaderDBA@@HUStandardAlloc@NAlloc@@@NArray@@IAEXXZ@4PAUCGlobalHeaderDBA@@A 31625458     CharacterManager.obj
 0003:0000945c       ?s_EmptyHeader@?1??set_null@?$SmallDynStorage@UCGlobalHeaderDBA@@HUStandardAlloc@NAlloc@@@NArray@@IAEXXZ@4UEmptyHeader@23@A 3162545c     CharacterManager.obj
 0003:00009464       ??_B?1??set_null@?$SmallDynStorage@UCGlobalHeaderDBA@@HUStandardAlloc@NAlloc@@@NArray@@IAEXXZ@51 31625464     CharacterManager.obj
 0003:00009468       ?s_EmptyElems@?1??set_null@?$SmallDynStorage@UGlobalAnimationHeaderCAF@@HUStandardAlloc@NAlloc@@@NArray@@IAEXXZ@4PAUGlobalAnimationHeaderCAF@@A 31625468     CharacterManager.obj
 0003:0000946c       ?s_EmptyHeader@?1??set_null@?$SmallDynStorage@UGlobalAnimationHeaderCAF@@HUStandardAlloc@NAlloc@@@NArray@@IAEXXZ@4UEmptyHeader@23@A 3162546c     CharacterManager.obj
 0003:00009474       ??_B?1??set_null@?$SmallDynStorage@UGlobalAnimationHeaderCAF@@HUStandardAlloc@NAlloc@@@NArray@@IAEXXZ@51 31625474     CharacterManager.obj
 0003:00009478       ?s_EmptyElems@?1??set_null@?$SmallDynStorage@UGlobalAnimationHeaderAIM@@HUStandardAlloc@NAlloc@@@NArray@@IAEXXZ@4PAUGlobalAnimationHeaderAIM@@A 31625478     CharacterManager.obj
 0003:0000947c       ?s_EmptyHeader@?1??set_null@?$SmallDynStorage@UGlobalAnimationHeaderAIM@@HUStandardAlloc@NAlloc@@@NArray@@IAEXXZ@4UEmptyHeader@23@A 3162547c     CharacterManager.obj
 0003:00009488       ??_B?1??set_null@?$SmallDynStorage@UGlobalAnimationHeaderAIM@@HUStandardAlloc@NAlloc@@@NArray@@IAEXXZ@51 31625488     CharacterManager.obj
 0003:0000948c       ?s_EmptyElems@?1??set_null@?$SmallDynStorage@UGlobalAnimationHeaderLMG@@HUStandardAlloc@NAlloc@@@NArray@@IAEXXZ@4PAUGlobalAnimationHeaderLMG@@A 3162548c     CharacterManager.obj
 0003:00009490       ?s_EmptyHeader@?1??set_null@?$SmallDynStorage@UGlobalAnimationHeaderLMG@@HUStandardAlloc@NAlloc@@@NArray@@IAEXXZ@4UEmptyHeader@23@A 31625490     CharacterManager.obj
 0003:00009498       ??_B?1??set_null@?$SmallDynStorage@UGlobalAnimationHeaderLMG@@HUStandardAlloc@NAlloc@@@NArray@@IAEXXZ@51 31625498     CharacterManager.obj
 0003:0000949c       ?s_EmptyElems@?1??set_null@?$SmallDynStorage@UBSParameter@@HUStandardAlloc@NAlloc@@@NArray@@IAEXXZ@4PAUBSParameter@@A 3162549c     CharacterManager.obj
 0003:000094a0       ?s_EmptyHeader@?1??set_null@?$SmallDynStorage@UBSParameter@@HUStandardAlloc@NAlloc@@@NArray@@IAEXXZ@4UEmptyHeader@23@A 316254a0     CharacterManager.obj
 0003:000094a8       ??_B?1??set_null@?$SmallDynStorage@UBSParameter@@HUStandardAlloc@NAlloc@@@NArray@@IAEXXZ@51 316254a8     CharacterManager.obj
 0003:000094ac       ?s_EmptyElems@?1??set_null@?$SmallDynStorage@UBSBlendable@@HUStandardAlloc@NAlloc@@@NArray@@IAEXXZ@4PAUBSBlendable@@A 316254ac     CharacterManager.obj
 0003:000094b0       ?s_EmptyHeader@?1??set_null@?$SmallDynStorage@UBSBlendable@@HUStandardAlloc@NAlloc@@@NArray@@IAEXXZ@4UEmptyHeader@23@A 316254b0     CharacterManager.obj
 0003:000094b8       ??_B?1??set_null@?$SmallDynStorage@UBSBlendable@@HUStandardAlloc@NAlloc@@@NArray@@IAEXXZ@51 316254b8     CharacterManager.obj
 0003:000094bc       ?s_EmptyElems@?1??set_null@?$SmallDynStorage@UBlendSpaceInfo@@HUStandardAlloc@NAlloc@@@NArray@@IAEXXZ@4PAUBlendSpaceInfo@@A 316254bc     CharacterManager.obj
 0003:000094c0       ?s_EmptyHeader@?1??set_null@?$SmallDynStorage@UBlendSpaceInfo@@HUStandardAlloc@NAlloc@@@NArray@@IAEXXZ@4UEmptyHeader@23@A 316254c0     CharacterManager.obj
 0003:000094c8       ??_B?1??set_null@?$SmallDynStorage@UBlendSpaceInfo@@HUStandardAlloc@NAlloc@@@NArray@@IAEXXZ@51 316254c8     CharacterManager.obj
 0003:000094cc       ?s_EmptyElems@?1??set_null@?$SmallDynStorage@USCRCName@@HUStandardAlloc@NAlloc@@@NArray@@IAEXXZ@4PAUSCRCName@@A 316254cc     CharacterManager.obj
 0003:000094d0       ?s_EmptyHeader@?1??set_null@?$SmallDynStorage@USCRCName@@HUStandardAlloc@NAlloc@@@NArray@@IAEXXZ@4UEmptyHeader@23@A 316254d0     CharacterManager.obj
 0003:000094d8       ??_B?1??set_null@?$SmallDynStorage@USCRCName@@HUStandardAlloc@NAlloc@@@NArray@@IAEXXZ@51 316254d8     CharacterManager.obj
 0003:000094dc       ?s_EmptyElems@?1??set_null@?$SmallDynStorage@PAVCAnimationSet@@HUStandardAlloc@NAlloc@@@NArray@@IAEXXZ@4PAPAVCAnimationSet@@A 316254dc     CharacterManager.obj
 0003:000094e0       ?s_EmptyHeader@?1??set_null@?$SmallDynStorage@PAVCAnimationSet@@HUStandardAlloc@NAlloc@@@NArray@@IAEXXZ@4UEmptyHeader@23@A 316254e0     CharacterManager.obj
 0003:000094e8       ??_B?1??set_null@?$SmallDynStorage@PAVCAnimationSet@@HUStandardAlloc@NAlloc@@@NArray@@IAEXXZ@51 316254e8     CharacterManager.obj
 0003:00009874       ?s_EmptyElems@?1??set_null@?$SmallDynStorage@USMeshSubset@@HUStandardAlloc@NAlloc@@@NArray@@IAEXXZ@4PAUSMeshSubset@@A 31625874     LoaderCGA.obj
 0003:00009878       ?s_EmptyHeader@?1??set_null@?$SmallDynStorage@USMeshSubset@@HUStandardAlloc@NAlloc@@@NArray@@IAEXXZ@4UEmptyHeader@23@A 31625878     LoaderCGA.obj
 0003:00009880       ??_B?1??set_null@?$SmallDynStorage@USMeshSubset@@HUStandardAlloc@NAlloc@@@NArray@@IAEXXZ@51 31625880     LoaderCGA.obj
 0003:00009884       ?s_EmptyElems@?1??set_null@?$SmallDynStorage@VCModelJoint@@HUStandardAlloc@NAlloc@@@NArray@@IAEXXZ@4PAVCModelJoint@@A 31625884     LoaderCGA.obj
 0003:00009888       ?s_EmptyHeader@?1??set_null@?$SmallDynStorage@VCModelJoint@@HUStandardAlloc@NAlloc@@@NArray@@IAEXXZ@4UEmptyHeader@23@A 31625888     LoaderCGA.obj
 0003:00009890       ??_B?1??set_null@?$SmallDynStorage@VCModelJoint@@HUStandardAlloc@NAlloc@@@NArray@@IAEXXZ@51 31625890     LoaderCGA.obj
 0003:00009894       ?s_EmptyElems@?1??set_null@?$SmallDynStorage@UTCBAngAxisKey@spline@@HUStandardAlloc@NAlloc@@@NArray@@IAEXXZ@4PAUTCBAngAxisKey@spline@@A 31625894     LoaderCGA.obj
 0003:00009898       ?s_EmptyHeader@?1??set_null@?$SmallDynStorage@UTCBAngAxisKey@spline@@HUStandardAlloc@NAlloc@@@NArray@@IAEXXZ@4UEmptyHeader@23@A 31625898     LoaderCGA.obj
 0003:000098a0       ??_B?1??set_null@?$SmallDynStorage@UTCBAngAxisKey@spline@@HUStandardAlloc@NAlloc@@@NArray@@IAEXXZ@51 316258a0     LoaderCGA.obj
 0003:000098a4       ?s_used_memory@?1??_usedMemory@?$CryStackStringT@D$0BAA@@@SAII@Z@4IA 316258a4     LoaderCHR.obj
 0003:000098a8       ?s_EmptyElems@?1??set_null@?$SmallDynStorage@UModelAnimationHeader@@HUStandardAlloc@NAlloc@@@NArray@@IAEXXZ@4PAUModelAnimationHeader@@A 316258a8     LoaderCHR.obj
 0003:000098ac       ?s_EmptyHeader@?1??set_null@?$SmallDynStorage@UModelAnimationHeader@@HUStandardAlloc@NAlloc@@@NArray@@IAEXXZ@4UEmptyHeader@23@A 316258ac     LoaderCHR.obj
 0003:000098b4       ??_B?1??set_null@?$SmallDynStorage@UModelAnimationHeader@@HUStandardAlloc@NAlloc@@@NArray@@IAEXXZ@51 316258b4     LoaderCHR.obj
 0003:000098b8       ?s_EmptyElems@?1??set_null@?$SmallDynStorage@USAnimFile@@HUStandardAlloc@NAlloc@@@NArray@@IAEXXZ@4PAUSAnimFile@@A 316258b8     LoaderCHR.obj
 0003:000098bc       ?s_EmptyHeader@?1??set_null@?$SmallDynStorage@USAnimFile@@HUStandardAlloc@NAlloc@@@NArray@@IAEXXZ@4UEmptyHeader@23@A 316258bc     LoaderCHR.obj
 0003:000098c4       ??_B?1??set_null@?$SmallDynStorage@USAnimFile@@HUStandardAlloc@NAlloc@@@NArray@@IAEXXZ@51 316258c4     LoaderCHR.obj
 0003:000098c8       ?s_EmptyElems@?1??set_null@?$SmallDynStorage@DHUStandardAlloc@NAlloc@@@NArray@@IAEXXZ@4PADA 316258c8     LoaderCHR.obj
 0003:000098cc       ?s_EmptyHeader@?1??set_null@?$SmallDynStorage@DHUStandardAlloc@NAlloc@@@NArray@@IAEXXZ@4UEmptyHeader@23@A 316258cc     LoaderCHR.obj
 0003:000098d4       ??_B?1??set_null@?$SmallDynStorage@DHUStandardAlloc@NAlloc@@@NArray@@IAEXXZ@51 316258d4     LoaderCHR.obj
 0003:000098d8       ?s_EmptyElems@?1??set_null@?$SmallDynStorage@GHUStandardAlloc@NAlloc@@@NArray@@IAEXXZ@4PAGA 316258d8     LoaderCHR.obj
 0003:000098dc       ?s_EmptyHeader@?1??set_null@?$SmallDynStorage@GHUStandardAlloc@NAlloc@@@NArray@@IAEXXZ@4UEmptyHeader@23@A 316258dc     LoaderCHR.obj
 0003:000098e4       ??_B?1??set_null@?$SmallDynStorage@GHUStandardAlloc@NAlloc@@@NArray@@IAEXXZ@51 316258e4     LoaderCHR.obj
 0003:00009fd4       ?s_EmptyElems@?1??set_null@?$SmallDynStorage@PAU?$DynArray@UCryTCB3Key@@HU?$SmallDynStorage@UCryTCB3Key@@HUStandardAlloc@NAlloc@@@NArray@@@@HUStandardAlloc@NAlloc@@@NArray@@IAEXXZ@4PAPAU?$DynArray@UCryTCB3Key@@HU?$SmallDynStorage@UCryTCB3Key@@HUStandardAlloc@NAlloc@@@NArray@@@@A 31625fd4     LoaderTCB.obj
 0003:00009fd8       ?s_EmptyHeader@?1??set_null@?$SmallDynStorage@PAU?$DynArray@UCryTCB3Key@@HU?$SmallDynStorage@UCryTCB3Key@@HUStandardAlloc@NAlloc@@@NArray@@@@HUStandardAlloc@NAlloc@@@NArray@@IAEXXZ@4UEmptyHeader@23@A 31625fd8     LoaderTCB.obj
 0003:00009fe0       ??_B?1??set_null@?$SmallDynStorage@PAU?$DynArray@UCryTCB3Key@@HU?$SmallDynStorage@UCryTCB3Key@@HUStandardAlloc@NAlloc@@@NArray@@@@HUStandardAlloc@NAlloc@@@NArray@@IAEXXZ@51 31625fe0     LoaderTCB.obj
 0003:00009fe4       ?s_EmptyElems@?1??set_null@?$SmallDynStorage@PAU?$DynArray@UCryTCBQKey@@HU?$SmallDynStorage@UCryTCBQKey@@HUStandardAlloc@NAlloc@@@NArray@@@@HUStandardAlloc@NAlloc@@@NArray@@IAEXXZ@4PAPAU?$DynArray@UCryTCBQKey@@HU?$SmallDynStorage@UCryTCBQKey@@HUStandardAlloc@NAlloc@@@NArray@@@@A 31625fe4     LoaderTCB.obj
 0003:00009fe8       ?s_EmptyHeader@?1??set_null@?$SmallDynStorage@PAU?$DynArray@UCryTCBQKey@@HU?$SmallDynStorage@UCryTCBQKey@@HUStandardAlloc@NAlloc@@@NArray@@@@HUStandardAlloc@NAlloc@@@NArray@@IAEXXZ@4UEmptyHeader@23@A 31625fe8     LoaderTCB.obj
 0003:00009ff0       ??_B?1??set_null@?$SmallDynStorage@PAU?$DynArray@UCryTCBQKey@@HU?$SmallDynStorage@UCryTCBQKey@@HUStandardAlloc@NAlloc@@@NArray@@@@HUStandardAlloc@NAlloc@@@NArray@@IAEXXZ@51 31625ff0     LoaderTCB.obj
 0003:00009ff4       ?s_EmptyElems@?1??set_null@?$SmallDynStorage@UTCBFlags@@HUStandardAlloc@NAlloc@@@NArray@@IAEXXZ@4PAUTCBFlags@@A 31625ff4     LoaderTCB.obj
 0003:00009ff8       ?s_EmptyHeader@?1??set_null@?$SmallDynStorage@UTCBFlags@@HUStandardAlloc@NAlloc@@@NArray@@IAEXXZ@4UEmptyHeader@23@A 31625ff8     LoaderTCB.obj
 0003:0000a000       ??_B?1??set_null@?$SmallDynStorage@UTCBFlags@@HUStandardAlloc@NAlloc@@@NArray@@IAEXXZ@51 31626000     LoaderTCB.obj
 0003:0000a004       ?s_EmptyElems@?1??set_null@?$SmallDynStorage@UCryTCB3Key@@HUStandardAlloc@NAlloc@@@NArray@@IAEXXZ@4PAUCryTCB3Key@@A 31626004     LoaderTCB.obj
 0003:0000a008       ?s_EmptyHeader@?1??set_null@?$SmallDynStorage@UCryTCB3Key@@HUStandardAlloc@NAlloc@@@NArray@@IAEXXZ@4UEmptyHeader@23@A 31626008     LoaderTCB.obj
 0003:0000a010       ??_B?1??set_null@?$SmallDynStorage@UCryTCB3Key@@HUStandardAlloc@NAlloc@@@NArray@@IAEXXZ@51 31626010     LoaderTCB.obj
 0003:0000a014       ?s_EmptyElems@?1??set_null@?$SmallDynStorage@UCryTCBQKey@@HUStandardAlloc@NAlloc@@@NArray@@IAEXXZ@4PAUCryTCBQKey@@A 31626014     LoaderTCB.obj
 0003:0000a018       ?s_EmptyHeader@?1??set_null@?$SmallDynStorage@UCryTCBQKey@@HUStandardAlloc@NAlloc@@@NArray@@IAEXXZ@4UEmptyHeader@23@A 31626018     LoaderTCB.obj
 0003:0000a020       ??_B?1??set_null@?$SmallDynStorage@UCryTCBQKey@@HUStandardAlloc@NAlloc@@@NArray@@IAEXXZ@51 31626020     LoaderTCB.obj
 0003:0000a024       ?s_EmptyElems@?1??set_null@?$SmallDynStorage@UPQLog@@HUStandardAlloc@NAlloc@@@NArray@@IAEXXZ@4PAUPQLog@@A 31626024     LoaderTCB.obj
 0003:0000a028       ?s_EmptyHeader@?1??set_null@?$SmallDynStorage@UPQLog@@HUStandardAlloc@NAlloc@@@NArray@@IAEXXZ@4UEmptyHeader@23@A 31626028     LoaderTCB.obj
 0003:0000a030       ??_B?1??set_null@?$SmallDynStorage@UPQLog@@HUStandardAlloc@NAlloc@@@NArray@@IAEXXZ@51 31626030     LoaderTCB.obj
 0003:0000a034       ?s_EmptyElems@?1??set_null@?$SmallDynStorage@USAnimListInfo@@HUStandardAlloc@NAlloc@@@NArray@@IAEXXZ@4PAUSAnimListInfo@@A 31626034     ParamLoader.obj
 0003:0000a038       ?s_EmptyHeader@?1??set_null@?$SmallDynStorage@USAnimListInfo@@HUStandardAlloc@NAlloc@@@NArray@@IAEXXZ@4UEmptyHeader@23@A 31626038     ParamLoader.obj
 0003:0000a040       ??_B?1??set_null@?$SmallDynStorage@USAnimListInfo@@HUStandardAlloc@NAlloc@@@NArray@@IAEXXZ@51 31626040     ParamLoader.obj
 0003:0000a044       ?s_EmptyElems@?1??set_null@?$SmallDynStorage@U?$DynArray@IHU?$SmallDynStorage@IHUStandardAlloc@NAlloc@@@NArray@@@@HUStandardAlloc@NAlloc@@@NArray@@IAEXXZ@4PAU?$DynArray@IHU?$SmallDynStorage@IHUStandardAlloc@NAlloc@@@NArray@@@@A 31626044     ParamLoader.obj
 0003:0000a048       ?s_EmptyHeader@?1??set_null@?$SmallDynStorage@U?$DynArray@IHU?$SmallDynStorage@IHUStandardAlloc@NAlloc@@@NArray@@@@HUStandardAlloc@NAlloc@@@NArray@@IAEXXZ@4UEmptyHeader@23@A 31626048     ParamLoader.obj
 0003:0000a050       ??_B?1??set_null@?$SmallDynStorage@U?$DynArray@IHU?$SmallDynStorage@IHUStandardAlloc@NAlloc@@@NArray@@@@HUStandardAlloc@NAlloc@@@NArray@@IAEXXZ@51 31626050     ParamLoader.obj
 0003:0000a054       ?s_EmptyElems@?1??set_null@?$SmallDynStorage@FHUStandardAlloc@NAlloc@@@NArray@@IAEXXZ@4PAFA 31626054     ParamLoader.obj
 0003:0000a058       ?s_EmptyHeader@?1??set_null@?$SmallDynStorage@FHUStandardAlloc@NAlloc@@@NArray@@IAEXXZ@4UEmptyHeader@23@A 31626058     ParamLoader.obj
 0003:0000a060       ??_B?1??set_null@?$SmallDynStorage@FHUStandardAlloc@NAlloc@@@NArray@@IAEXXZ@51 31626060     ParamLoader.obj
 0003:0000a064       ?s_EmptyElems@?1??set_null@?$SmallDynStorage@USJointsAimIK_Rot@@HUStandardAlloc@NAlloc@@@NArray@@IAEXXZ@4PAUSJointsAimIK_Rot@@A 31626064     ParamLoader.obj
 0003:0000a068       ?s_EmptyHeader@?1??set_null@?$SmallDynStorage@USJointsAimIK_Rot@@HUStandardAlloc@NAlloc@@@NArray@@IAEXXZ@4UEmptyHeader@23@A 31626068     ParamLoader.obj
 0003:0000a070       ??_B?1??set_null@?$SmallDynStorage@USJointsAimIK_Rot@@HUStandardAlloc@NAlloc@@@NArray@@IAEXXZ@51 31626070     ParamLoader.obj
 0003:0000a074       ?s_EmptyElems@?1??set_null@?$SmallDynStorage@USJointsAimIK_Pos@@HUStandardAlloc@NAlloc@@@NArray@@IAEXXZ@4PAUSJointsAimIK_Pos@@A 31626074     ParamLoader.obj
 0003:0000a078       ?s_EmptyHeader@?1??set_null@?$SmallDynStorage@USJointsAimIK_Pos@@HUStandardAlloc@NAlloc@@@NArray@@IAEXXZ@4UEmptyHeader@23@A 31626078     ParamLoader.obj
 0003:0000a080       ??_B?1??set_null@?$SmallDynStorage@USJointsAimIK_Pos@@HUStandardAlloc@NAlloc@@@NArray@@IAEXXZ@51 31626080     ParamLoader.obj
 0003:0000a084       ?s_EmptyElems@?1??set_null@?$SmallDynStorage@UDirectionalBlends@@HUStandardAlloc@NAlloc@@@NArray@@IAEXXZ@4PAUDirectionalBlends@@A 31626084     ParamLoader.obj
 0003:0000a088       ?s_EmptyHeader@?1??set_null@?$SmallDynStorage@UDirectionalBlends@@HUStandardAlloc@NAlloc@@@NArray@@IAEXXZ@4UEmptyHeader@23@A 31626088     ParamLoader.obj
 0003:0000a090       ??_B?1??set_null@?$SmallDynStorage@UDirectionalBlends@@HUStandardAlloc@NAlloc@@@NArray@@IAEXXZ@51 31626090     ParamLoader.obj
 0003:0000a094       ?s_EmptyElems@?1??set_null@?$SmallDynStorage@UIdxAndName@@HUStandardAlloc@NAlloc@@@NArray@@IAEXXZ@4PAUIdxAndName@@A 31626094     ParamLoader.obj
 0003:0000a098       ?s_EmptyHeader@?1??set_null@?$SmallDynStorage@UIdxAndName@@HUStandardAlloc@NAlloc@@@NArray@@IAEXXZ@4UEmptyHeader@23@A 31626098     ParamLoader.obj
 0003:0000a0a0       ??_B?1??set_null@?$SmallDynStorage@UIdxAndName@@HUStandardAlloc@NAlloc@@@NArray@@IAEXXZ@51 316260a0     ParamLoader.obj
 0003:0000a0a4       ?s_EmptyElems@?1??set_null@?$SmallDynStorage@USRecoilJoints@@HUStandardAlloc@NAlloc@@@NArray@@IAEXXZ@4PAUSRecoilJoints@@A 316260a4     ParamLoader.obj
 0003:0000a0a8       ?s_EmptyHeader@?1??set_null@?$SmallDynStorage@USRecoilJoints@@HUStandardAlloc@NAlloc@@@NArray@@IAEXXZ@4UEmptyHeader@23@A 316260a8     ParamLoader.obj
 0003:0000a0b0       ??_B?1??set_null@?$SmallDynStorage@USRecoilJoints@@HUStandardAlloc@NAlloc@@@NArray@@IAEXXZ@51 316260b0     ParamLoader.obj
 0003:0000a0b4       ?s_EmptyElems@?1??set_null@?$SmallDynStorage@UProcAdjust@@HUStandardAlloc@NAlloc@@@NArray@@IAEXXZ@4PAUProcAdjust@@A 316260b4     ParamLoader.obj
 0003:0000a0b8       ?s_EmptyHeader@?1??set_null@?$SmallDynStorage@UProcAdjust@@HUStandardAlloc@NAlloc@@@NArray@@IAEXXZ@4UEmptyHeader@23@A 316260b8     ParamLoader.obj
 0003:0000a0c0       ??_B?1??set_null@?$SmallDynStorage@UProcAdjust@@HUStandardAlloc@NAlloc@@@NArray@@IAEXXZ@51 316260c0     ParamLoader.obj
 0003:0000a0c4       ?s_EmptyElems@?1??set_null@?$SmallDynStorage@UIKLimbType@@HUStandardAlloc@NAlloc@@@NArray@@IAEXXZ@4PAUIKLimbType@@A 316260c4     ParamLoader.obj
 0003:0000a0c8       ?s_EmptyHeader@?1??set_null@?$SmallDynStorage@UIKLimbType@@HUStandardAlloc@NAlloc@@@NArray@@IAEXXZ@4UEmptyHeader@23@A 316260c8     ParamLoader.obj
 0003:0000a0d4       ??_B?1??set_null@?$SmallDynStorage@UIKLimbType@@HUStandardAlloc@NAlloc@@@NArray@@IAEXXZ@51 316260d4     ParamLoader.obj
 0003:0000a0d8       ?s_EmptyElems@?1??set_null@?$SmallDynStorage@UADIKTarget@@HUStandardAlloc@NAlloc@@@NArray@@IAEXXZ@4PAUADIKTarget@@A 316260d8     ParamLoader.obj
 0003:0000a0dc       ?s_EmptyHeader@?1??set_null@?$SmallDynStorage@UADIKTarget@@HUStandardAlloc@NAlloc@@@NArray@@IAEXXZ@4UEmptyHeader@23@A 316260dc     ParamLoader.obj
 0003:0000a0e8       ??_B?1??set_null@?$SmallDynStorage@UADIKTarget@@HUStandardAlloc@NAlloc@@@NArray@@IAEXXZ@51 316260e8     ParamLoader.obj
 0003:0000a0ec       ?s_EmptyElems@?1??set_null@?$SmallDynStorage@PAVCCharInstance@@HUStandardAlloc@NAlloc@@@NArray@@IAEXXZ@4PAPAVCCharInstance@@A 316260ec     Model.obj
 0003:0000a0f0       ?s_EmptyHeader@?1??set_null@?$SmallDynStorage@PAVCCharInstance@@HUStandardAlloc@NAlloc@@@NArray@@IAEXXZ@4UEmptyHeader@23@A 316260f0     Model.obj
 0003:0000a0f8       ??_B?1??set_null@?$SmallDynStorage@PAVCCharInstance@@HUStandardAlloc@NAlloc@@@NArray@@IAEXXZ@51 316260f8     Model.obj
 0003:0000a0fc       ?s_EmptyElems@?1??set_null@?$SmallDynStorage@USJointProperty@@HUStandardAlloc@NAlloc@@@NArray@@IAEXXZ@4PAUSJointProperty@@A 316260fc     Model.obj
 0003:0000a100       ?s_EmptyHeader@?1??set_null@?$SmallDynStorage@USJointProperty@@HUStandardAlloc@NAlloc@@@NArray@@IAEXXZ@4UEmptyHeader@23@A 31626100     Model.obj
 0003:0000a108       ??_B?1??set_null@?$SmallDynStorage@USJointProperty@@HUStandardAlloc@NAlloc@@@NArray@@IAEXXZ@51 31626108     Model.obj
 0003:0000a10c       ?s_EmptyElems@?1??set_null@?$SmallDynStorage@UMeshCollisionInfo@@HUStandardAlloc@NAlloc@@@NArray@@IAEXXZ@4PAUMeshCollisionInfo@@A 3162610c     Model.obj
 0003:0000a110       ?s_EmptyHeader@?1??set_null@?$SmallDynStorage@UMeshCollisionInfo@@HUStandardAlloc@NAlloc@@@NArray@@IAEXXZ@4UEmptyHeader@23@A 31626110     Model.obj
 0003:0000a118       ??_B?1??set_null@?$SmallDynStorage@UMeshCollisionInfo@@HUStandardAlloc@NAlloc@@@NArray@@IAEXXZ@51 31626118     Model.obj
 0003:0000a830       ?div@SmallTree48BitQuat@@2T__m128@@A 31626830     ControllerPQ.obj
 0003:0000a840       ?ran@SmallTree48BitQuat@@2T__m128@@A 31626840     ControllerPQ.obj
 0003:0000a850       ?Init48b@@3HA              31626850     ControllerPQ.obj
 0003:0000abd0       ?g_pCharacterManager@@3PAVCharacterManager@@A 31626bd0     AnimationBase.obj
 0003:0000abd4       ?numAllocations@_CryMemoryManagerPoolHelper@@2HC 31626bd4     AnimationBase.obj
 0003:0000abd8       ?requestedMemory@_CryMemoryManagerPoolHelper@@2JC 31626bd8     AnimationBase.obj
 0003:0000abdc       ?freedMemory@_CryMemoryManagerPoolHelper@@2JC 31626bdc     AnimationBase.obj
 0003:0000abe0       ?allocatedMemory@_CryMemoryManagerPoolHelper@@2JC 31626be0     AnimationBase.obj
 0003:0000abe4       ?gEnv@@3PAUSSystemGlobalEnvironment@@A 31626be4     AnimationBase.obj
 0003:0000abe8       ?m_pFirst@Test@CryUnitTest@@2PAU12@A 31626be8     AnimationBase.obj
 0003:0000abec       ?m_pLast@Test@CryUnitTest@@2PAU12@A 31626bec     AnimationBase.obj
 0003:0000abf0       ?g_pHeadToRegFactories@@3PAUSRegFactoryNode@@A 31626bf0     AnimationBase.obj
 0003:0000abf4       ?g_bProfilerEnabled@@3_NA  31626bf4     AnimationBase.obj
 0003:0000abf5       ?g_bForceLOD@@3_NA         31626bf5     AnimationBase.obj
 0003:0000abf6       ?g_bProfilerOn@@3_NA       31626bf6     AnimationBase.obj
 0003:0000abf8       ?g_iTraceAllocations@@3HA  31626bf8     AnimationBase.obj
 0003:0000abfc       ?_CryMalloc@_CryMemoryManagerPoolHelper@@2P6APAXIAAII@ZA 31626bfc     AnimationBase.obj
 0003:0000ac00       ?_CryGetMemSize@_CryMemoryManagerPoolHelper@@2P6AIPAXI@ZA 31626c00     AnimationBase.obj
 0003:0000ac04       ?_CryRealloc@_CryMemoryManagerPoolHelper@@2P6APAXPAXIAAI1I@ZA 31626c04     AnimationBase.obj
 0003:0000ac08       ?_CryFree@_CryMemoryManagerPoolHelper@@2P6AIPAXI@ZA 31626c08     AnimationBase.obj
 0003:0000ac0c       ?_CryCrtMalloc@_CryMemoryManagerPoolHelper@@2P6APAXI@ZA 31626c0c     AnimationBase.obj
 0003:0000ac10       ?_CryCrtRealloc@_CryMemoryManagerPoolHelper@@2P6APAXPAXI@ZA 31626c10     AnimationBase.obj
 0003:0000ac14       ?_CryCrtFree@_CryMemoryManagerPoolHelper@@2P6AIPAX@ZA 31626c14     AnimationBase.obj
 0003:0000ac18       ?_CryCrtSize@_CryMemoryManagerPoolHelper@@2P6AIPAX@ZA 31626c18     AnimationBase.obj
 0003:0000ac1c       ?_CryGetIMemoryManagerInterface@_CryMemoryManagerPoolHelper@@2P6AXPAPAX@ZA 31626c1c     AnimationBase.obj
 0003:0000ac20       ?m_bInitialized@_CryMemoryManagerPoolHelper@@2HA 31626c20     AnimationBase.obj
 0003:0000ac24       ?g_pISystem@@3PAUISystem@@A 31626c24     AnimationBase.obj
 0003:0000ac28       ?g_pITimer@@3PAUITimer@@A  31626c28     AnimationBase.obj
 0003:0000ac2c       ?g_pILog@@3PAUILog@@A      31626c2c     AnimationBase.obj
 0003:0000ac30       ?g_pIConsole@@3PAUIConsole@@A 31626c30     AnimationBase.obj
 0003:0000ac34       ?g_pIPak@@3PAUICryPak@@A   31626c34     AnimationBase.obj
 0003:0000ac38       ?g_pIStreamEngine@@3PAUIStreamEngine@@A 31626c38     AnimationBase.obj
 0003:0000ac3c       ?g_pCrc32Gen@@3PAVCrc32Gen@@A 31626c3c     AnimationBase.obj
 0003:0000ac40       ?g_pIRenderer@@3PAUIRenderer@@A 31626c40     AnimationBase.obj
 0003:0000ac44       ?g_pAuxGeom@@3PAUIRenderAuxGeom@@A 31626c44     AnimationBase.obj
 0003:0000ac48       ?g_pIPhysicalWorld@@3PAUIPhysicalWorld@@A 31626c48     AnimationBase.obj
 0003:0000ac4c       ?g_pI3DEngine@@3PAUI3DEngine@@A 31626c4c     AnimationBase.obj
 0003:0000ac50       ?g_AverageFrameTime@@3MA   31626c50     AnimationBase.obj
 0003:0000ac54       ?g_nRenderThreadUpdateID@@3HA 31626c54     AnimationBase.obj
 0003:0000ac58       ?g_parametricPool@@3PAUSParametricSamplerInternal@@A 31626c58     AnimationBase.obj
 0003:0000ac5c       ?g_usedParametrics@@3PA_NA 31626c5c     AnimationBase.obj
 0003:0000ac60       ?g_totalParametrics@@3HA   31626c60     AnimationBase.obj
 0003:0000ac64       ?g_ForcedLODNum@@3HA       31626c64     AnimationBase.obj
 0003:0000ac68       ?g_fCurrTime@@3MA          31626c68     AnimationBase.obj
 0003:0000ac6c       ?g_CpuFlags@@3HA           31626c6c     AnimationBase.obj
 0003:0000ac70       ?g_random_generator@@3VCLCGRndGen@@A 31626c70     AnimationBase.obj
 0003:0000ac74       ?s_factory@CFactory@CEngineModule_CryAnimation@@0V12@A 31626c74     AnimationBase.obj
 0003:0000aca0       ?g_DataMismatch@@3U?$DynArray@V?$CryStringT@D@@HU?$SmallDynStorage@V?$CryStringT@D@@HUStandardAlloc@NAlloc@@@NArray@@@@A 31626ca0     AnimationBase.obj
 0003:0000aca4       ?g_IdentityAABB@@3UAABB@@A 31626ca4     AnimationBase.obj
 0003:0000acc0       ?g_controllerHeap@@3VCControllerDefragHeap@@A 31626cc0     AnimationBase.obj
 0003:0000b230       ?g_AnimStatisticsInfo@@3UAnimStatisticsInfo@@A 31627230     AnimationBase.obj
 0003:0000b254       ?s_used_memory@?1??_usedMemory@?$CryStringT@_W@@SAIH@Z@4IA 31627254     AnimationBase.obj
 0003:0000b258       ?supportedIIDs@?1???0CFactory@CEngineModule_CryAnimation@@AAE@XZ@4PAUCryGUID@@A 31627258     AnimationBase.obj
 0003:0000b278       ?p@?1??CreateClassInstance@CFactory@CEngineModule_CryAnimation@@UBE?AV?$shared_ptr@UICryUnknown@@@boost@@XZ@4V?$shared_ptr@VCEngineModule_CryAnimation@@@5@A 31627278     AnimationBase.obj
 0003:0000b280       ??_B?1??CreateClassInstance@CFactory@CEngineModule_CryAnimation@@UBE?AV?$shared_ptr@UICryUnknown@@@boost@@XZ@51 31627280     AnimationBase.obj
 0003:0000b284       ?g_ConsoleInstanceCount@?A0xe26663e7@@3HA 31627284     cvars.obj
 0003:0000b298       ?g_globalSections@?$Node_Alloc_Lock@$00$00@@2PAUInternalCriticalSectionDummy@@A 31627298     stdafx.obj
 0003:0000d318       ?m_bInitialized@?$Node_Alloc_Lock@$00$00@@2_NA 31629318     stdafx.obj
 0003:0000d31c       ?gJobHandleTSkinAttachmentTangents@Detail@JobManager@@3PAUSJobStringHandle@2@A 3162931c     _RenderSkinsSW.obj
 0003:0000d320       ?gJobHandleTSkinAttachmentQtangents@Detail@JobManager@@3PAUSJobStringHandle@2@A 31629320     _RenderSkinsSW.obj
 0003:0000d328       ?__type_info_root_node@@3U__type_info_node@@A 31629328     MSVCRT:tncleanup.obj
 0003:0000d654       ___native_startup_state    31629654     <common>
 0003:0000d658       ___native_startup_lock     31629658     <common>
 0003:0000d65c       ___sse2_available          3162965c     <common>
 0003:0000d660       ___dyn_tls_init_callback   31629660     <common>
 0003:0000d664       ___onexitend               31629664     <common>
 0003:0000d668       ___onexitbegin             31629668     <common>
 0004:00000000       ?m_Self@CrySimpleThreadSelf@@1PAV1@A 3162a000     AnimationBase.obj

 entry point at        0001:0010ba9d

 Static symbols

 0001:00013730       ?GetLODName@CryCHRLoader_LoadNewSKIN_Helpers@@YA?AV?$CryStringT@D@@ABV2@PBDI@Z 31514730 f   LoaderSKIN.obj
 0001:000139e0       ?release@ContentCgfs@?6??LoadNewSKIN@CryCHRLoader@@QAEPAVCSkin@@PBDI@Z@QAEXXZ 315149e0 f   LoaderSKIN.obj
 0001:000139e0       ?release@ContentCgfs@?4??LoadNewCHR@CryCHRLoader@@QAEPAVCSkel@@PBDI@Z@QAEXXZ 315149e0 f   LoaderSKIN.obj
 0001:00013b30       ??1ContentCgfs@?4??LoadNewCHR@CryCHRLoader@@QAEPAVCSkel@@PBDI@Z@QAE@XZ 31514b30 f   LoaderSKIN.obj
 0001:00013b30       ??1ContentCgfs@?6??LoadNewSKIN@CryCHRLoader@@QAEPAVCSkin@@PBDI@Z@QAE@XZ 31514b30 f   LoaderSKIN.obj
 0001:00014330       ?ExtractExternalVertices@CryCHRLoader_LoadNewSKIN_Helpers@@YA_NAAU?$DynArray@UExtSkinVertex@@HU?$SmallDynStorage@UExtSkinVertex@@HUStandardAlloc@NAlloc@@@NArray@@@@PBVCModelMesh@@IPBVCMesh@@PBDH@Z 31515330 f   LoaderSKIN.obj
 0001:000157c0       ?CopyMorphTargets@CryCHRLoader_LoadNewCHR_Helpers@@YA_NPAVCModelMesh@@IPAUCSkinningInfo@@ABU?$DynArray@UExtSkinVertex@@HU?$SmallDynStorage@UExtSkinVertex@@HUStandardAlloc@NAlloc@@@NArray@@@@ABV?$VectorMap@V?$CryStringT@D@@HU?$less@V?$CryStringT@D@@@stlpmtx_std@@V?$allocator@U?$pair@V?$CryStringT@D@@H@stlpmtx_std@@@3@@@PBDH@Z 315167c0 f   LoaderSKIN.obj
 0001:000157c0       ?CopyMorphTargets@CryCHRLoader_LoadNewSKIN_Helpers@@YA_NPAVCModelMesh@@IPAUCSkinningInfo@@ABU?$DynArray@UExtSkinVertex@@HU?$SmallDynStorage@UExtSkinVertex@@HUStandardAlloc@NAlloc@@@NArray@@@@ABV?$VectorMap@V?$CryStringT@D@@HU?$less@V?$CryStringT@D@@@stlpmtx_std@@V?$allocator@U?$pair@V?$CryStringT@D@@H@stlpmtx_std@@@3@@@PBDH@Z 315167c0 f   LoaderSKIN.obj
 0001:00016800       ?InitializeBones@CryCHRLoader_LoadNewSKIN_Helpers@@YA_NPAVCSkin@@PAUCSkinningInfo@@PBD@Z 31517800 f   LoaderSKIN.obj
 0001:00016d70       ?CreateMorphNameToIndexMap@CryCHRLoader_LoadNewSKIN_Helpers@@YA_NAAV?$VectorMap@V?$CryStringT@D@@HU?$less@V?$CryStringT@D@@@stlpmtx_std@@V?$allocator@U?$pair@V?$CryStringT@D@@H@stlpmtx_std@@@3@@@PAPAVCContentCGF@@HPBD@Z 31517d70 f   LoaderSKIN.obj
 0001:00016d70       ?CreateMorphNameToIndexMap@CryCHRLoader_LoadNewCHR_Helpers@@YA_NAAV?$VectorMap@V?$CryStringT@D@@HU?$less@V?$CryStringT@D@@@stlpmtx_std@@V?$allocator@U?$pair@V?$CryStringT@D@@H@stlpmtx_std@@@3@@@PAPAVCContentCGF@@HPBD@Z 31517d70 f   LoaderSKIN.obj
 0001:00063cc0       ?strstri@@YAPBDPBD0@Z      31564cc0 f   SkeletonPose_Debug.obj
 0001:0006ff50       ?FindChannel@JoystickSerializeContext@?4??BindJoystickSetToSequence@CFacialAnimation@@UAEXPAVIJoystickSet@@PAUIFacialAnimSequence@@@Z@UAEPAUIFacialAnimChannel@@PBD@Z 31570f50 f   FaceAnimation.obj
 0001:00078b30       ??RRecurser@?CL@??BindChannels@CFacialAnimSequenceInstance@@QAEXPAVCFacialAnimationContext@@PAVCFacialAnimSequence@@@Z@QAEXPAUIFacialEffector@@@Z 31579b30 f   FaceAnimSequence.obj
 0001:00088330       ?Recurse@Recurser@?M@??RemoveEffector@CFacialEffectorsLibrary@@UAEXPAUIFacialEffector@@@Z@AAEX0@Z 31589330 f   FaceEffectorLibrary.obj
 0001:000883a0       ?CopyController@Recurser@?4??MergeLibrary@CFacialEffectorsLibrary@@UAEXPAUIFacialEffectorsLibrary@@ABV?$Functor1wRet@PBDW4MergeCollisionAction@@@@@Z@AAEXPAUIFacialEffCtrl@@2@Z 315893a0 f   FaceEffectorLibrary.obj
 0001:00088640       ?Recurse@Recurser@?M@??ReplaceEffector@CFacialEffectorsLibrary@@AAEXPAVCFacialEffector@@0@Z@AAEXPAUIFacialEffector@@@Z 31589640 f   FaceEffectorLibrary.obj
 0001:00089820       ?Recurse@Recurser@?4??MergeLibrary@CFacialEffectorsLibrary@@UAEXPAUIFacialEffectorsLibrary@@ABV?$Functor1wRet@PBDW4MergeCollisionAction@@@@@Z@AAEXPAUIFacialEffector@@2@Z 3158a820 f   FaceEffectorLibrary.obj
 0001:000b9540       ?GetLodIndex@CryCGALoaderHelper@@YAHQBD@Z 315ba540 f   LoaderCGA.obj
 0001:000c5290       ?ValidateLodSkeleton@CryCHRLoader_LoadNewSKIN_Helpers@@YA_NPAUCSkinningInfo@@0HPBD@Z 315c6290 f   LoaderCHR.obj
 0001:000c5290       ?ValidateLodSkeleton@CryCHRLoader_LoadNewCHR_Helpers@@YA_NPAUCSkinningInfo@@0HPBD@Z 315c6290 f   LoaderCHR.obj
 0001:000c6e70       ?GetLODName@CryCHRLoader_LoadNewCHR_Helpers@@YA?AV?$CryStringT@D@@ABV2@PBDI@Z 315c7e70 f   LoaderCHR.obj
 0001:000c7160       ?FindFirstMeshAndMaterial@CryCHRLoader_LoadNewCHR_Helpers@@YA_NAAPAVCMesh@@AAPAUCNodeCGF@@AAV?$_smart_ptr@UIMaterial@@@@PAVCContentCGF@@PBDH@Z 315c8160 f   LoaderCHR.obj
 0001:000c7160       ?FindFirstMeshAndMaterial@CryCHRLoader_LoadNewSKIN_Helpers@@YA_NAAPAVCMesh@@AAPAUCNodeCGF@@AAV?$_smart_ptr@UIMaterial@@@@PAVCContentCGF@@PBDH@Z 315c8160 f   LoaderCHR.obj
 0001:000c7790       ?ExtractExternalVertices@CryCHRLoader_LoadNewCHR_Helpers@@YA_NAAU?$DynArray@UExtSkinVertex@@HU?$SmallDynStorage@UExtSkinVertex@@HUStandardAlloc@NAlloc@@@NArray@@@@PBVCModelMesh@@IPBVCMesh@@PBDH@Z 315c8790 f   LoaderCHR.obj
 0001:000c7e10       ?SetupPhysicalProxies@CryCHRLoader_LoadNewCHR_Helpers@@YA_NPAUIGeomManager@@PAVCSkel@@PAUIMaterial@@PBUCSkinningInfo@@PBDH@Z 315c8e10 f   LoaderCHR.obj
 0001:000c8c80       ?InitializeBones@CryCHRLoader_LoadNewCHR_Helpers@@YA_NPAVCModelSkeleton@@PAUCSkinningInfo@@PBD@Z 315c9c80 f   LoaderCHR.obj
 0001:00108b90       ?CADebugText@@YAXPAUIConsoleCmdArgs@@@Z 31609b90 f   cvars.obj
 0001:0010b72f       _pre_c_init                3160c72f f   MSVCRT:crtdll.obj
 0001:0010b987       ___DllMainCRTStartup       3160c987 f   MSVCRT:crtdll.obj
 0001:0010bf20       ??__E?s_factory@CFactory@COperatorQueue@@0V12@A@@YAXXZ 3160cf20 f   OperatorQueue.obj
 0001:0010bf70       ??__E?s_factory@CFactory@CPoseAlignerChain@@0V12@A@@YAXXZ 3160cf70 f   PoseAlignerChain.obj
 0001:0010bfc0       ??__E?s_factory@CFactory@CPoseMatching@@0V12@A@@YAXXZ 3160cfc0 f   PoseMatching.obj
 0001:0010c010       ??__E?g_firstValidator@SBatchUpdateValidator@@2U1@A@@YAXXZ 3160d010 f   SkeletonPhysics.obj
 0001:0010c080       ??__Eg_arrVerticesBS@@YAXXZ 3160d080 f   DecalManager.obj
 0001:0010c0b0       ??__Eg_arrDecalVertexMapping@@YAXXZ 3160d0b0 f   DecalManager.obj
 0001:0010c0e0       ??__Eg_arrDecalFaceMapping@@YAXXZ 3160d0e0 f   DecalManager.obj
 0001:0010c110       ??__EGUID_AnimationPoseModifier_TransformationPin@@YAXXZ 3160d110 f   SkeletonAnim.obj
 0001:0010c140       ??__E?s_factory@CFactory@CFeetPoseStore@@0V12@A@@YAXXZ 3160d140 f   FeetLock.obj
 0001:0010c160       ??__E?s_factory@CFactory@CFeetPoseRestore@@0V12@A@@YAXXZ 3160d160 f   FeetLock.obj
 0001:0010c180       ??__E?s_factory@CFactory@CGroundAlignment@@0V12@A@@YAXXZ 3160d180 f   GroundAlignment.obj
 0001:0010c1d0       ??__E?s_factory@CFactory@CLimbIk@@0V12@A@@YAXXZ 3160d1d0 f   LimbIk.obj
 0001:0010c1f0       ??__E?s_factory@CFactory@CPoseBlenderAim@@0V12@A@@YAXXZ 3160d1f0 f   PoseBlenderAim.obj
 0001:0010c240       ??__E?s_factory@CFactory@CPoseBlenderLook@@0V12@A@@YAXXZ 3160d240 f   PoseBlenderLook.obj
 0001:0010c290       ??__E?s_factory@CFactory@CRecoil@PoseModifier@@0V123@A@@YAXXZ 3160d290 f   Recoil.obj
 0001:0010c2b0       ??__ECryUserInvalidID@@YAXXZ 3160d2b0 f   CharacterManager.obj
 0001:0010c2c0       ??__ECrySessionInvalidID@@YAXXZ 3160d2c0 f   CharacterManager.obj
 0001:0010c2d0       ??__EInit48b@@YAXXZ        3160d2d0 f   ControllerPQ.obj
 0001:0010c310       ??__Eg_random_generator@@YAXXZ 3160d310 f   AnimationBase.obj
 0001:0010c330       ??__Eg_system_event_listener_anim@@YAXXZ 3160d330 f   AnimationBase.obj
 0001:0010c340       ??__E?s_factory@CFactory@CEngineModule_CryAnimation@@0V12@A@@YAXXZ 3160d340 f   AnimationBase.obj
 0001:0010c360       ??__Eg_DefaultAnim@@YAXXZ  3160d360 f   AnimationBase.obj
 0001:0010c370       ??__Eg_DataMismatch@@YAXXZ 3160d370 f   AnimationBase.obj
 0001:0010c3c0       ??__Eg_IdentityAABB@@YAXXZ 3160d3c0 f   AnimationBase.obj
 0001:0010c420       ??__Eg_controllerHeap@@YAXXZ 3160d420 f   AnimationBase.obj
 0001:0010c440       ??__Eg_Consoleself@@YAXXZ  3160d440 f   cvars.obj
 0001:0010c470       ??__EautoInitializer@@YAXXZ 3160d470 f   stdafx.obj
 0001:0010c4c0       ??__FarrExtSkinnedStream@?1??DrawWireframeStatic@CModelMesh@@QAEXABU?$Matrix34_tpl@M@@PAUIRenderMesh@@I@Z@YAXXZ 3160d4c0 f   ModelMesh_DebugPC.obj
 0001:0010c4f0       ??__FarrExtSkinnedStream@?EI@??SoftwareSkinningDQ@CModelMesh@@QAEXPAUIRenderMesh@@PAVCCharInstance@@PAVCAttachmentSKIN@@U?$Matrix34_tpl@M@@EEEEPAU?$DualQuat_tpl@M@@@Z@YAXXZ 3160d4f0 f   ModelMesh_DebugPC.obj
 0001:0010c520       ??__FarrExtVColors@?EE@??SoftwareSkinningDQ@CModelMesh@@QAEXPAUIRenderMesh@@PAVCCharInstance@@PAVCAttachmentSKIN@@U?$Matrix34_tpl@M@@EEEEPAU?$DualQuat_tpl@M@@@Z@YAXXZ 3160d520 f   ModelMesh_DebugPC.obj
 0001:0010c550       ??__FarrExtSkinnedStream@?DN@??SoftwareSkinningDQ@CModelMesh@@QAEXPAUIRenderMesh@@PAVCCharInstance@@PAVCAttachmentSKIN@@U?$Matrix34_tpl@M@@EEEEPAU?$DualQuat_tpl@M@@@Z@YAXXZ 3160d550 f   ModelMesh_DebugPC.obj
 0001:0010c580       ??__FarrExtVColors@?DJ@??SoftwareSkinningDQ@CModelMesh@@QAEXPAUIRenderMesh@@PAVCCharInstance@@PAVCAttachmentSKIN@@U?$Matrix34_tpl@M@@EEEEPAU?$DualQuat_tpl@M@@@Z@YAXXZ 3160d580 f   ModelMesh_DebugPC.obj
 0001:0010c5b0       ??__FarrExtSkinnedStream@?DC@??SoftwareSkinningDQ@CModelMesh@@QAEXPAUIRenderMesh@@PAVCCharInstance@@PAVCAttachmentSKIN@@U?$Matrix34_tpl@M@@EEEEPAU?$DualQuat_tpl@M@@@Z@YAXXZ 3160d5b0 f   ModelMesh_DebugPC.obj
 0001:0010c5e0       ??__FarrExtVColors@?CO@??SoftwareSkinningDQ@CModelMesh@@QAEXPAUIRenderMesh@@PAVCCharInstance@@PAVCAttachmentSKIN@@U?$Matrix34_tpl@M@@EEEEPAU?$DualQuat_tpl@M@@@Z@YAXXZ 3160d5e0 f   ModelMesh_DebugPC.obj
 0001:0010c610       ??__Fg_arrQTangents@?1??SoftwareSkinningDQ@CModelMesh@@QAEXPAUIRenderMesh@@PAVCCharInstance@@PAVCAttachmentSKIN@@U?$Matrix34_tpl@M@@EEEEPAU?$DualQuat_tpl@M@@@Z@YAXXZ 3160d610 f   ModelMesh_DebugPC.obj
 0001:0010c640       ??__Fg_arrExtSkinnedStream@?1??SoftwareSkinningDQ@CModelMesh@@QAEXPAUIRenderMesh@@PAVCCharInstance@@PAVCAttachmentSKIN@@U?$Matrix34_tpl@M@@EEEEPAU?$DualQuat_tpl@M@@@Z@YAXXZ 3160d640 f   ModelMesh_DebugPC.obj
 0001:0010c670       ??__F?s_factory@CFactory@COperatorQueue@@0V12@A@@YAXXZ 3160d670 f   OperatorQueue.obj
 0001:0010c680       ??__F?s_factory@CFactory@CPoseAlignerChain@@0V12@A@@YAXXZ 3160d680 f   PoseAlignerChain.obj
 0001:0010c690       ??__F?s_factory@CFactory@CPoseMatching@@0V12@A@@YAXXZ 3160d690 f   PoseMatching.obj
 0001:0010c6a0       ??__F?g_firstValidator@SBatchUpdateValidator@@2U1@A@@YAXXZ 3160d6a0 f   SkeletonPhysics.obj
 0001:0010c710       ??__FarrExtSkinnedStream@?GA@??DrawAttachment@CAttachmentSKIN@@UAEXAAUSRendParams@@ABUSRenderingPassInfo@@ABU?$Matrix34_tpl@M@@M@Z@YAXXZ 3160d710 f   _RenderSkins.obj
 0001:0010c740       ??__FarrExtVColors@?FM@??DrawAttachment@CAttachmentSKIN@@UAEXAAUSRendParams@@ABUSRenderingPassInfo@@ABU?$Matrix34_tpl@M@@M@Z@YAXXZ 3160d740 f   _RenderSkins.obj
 0001:0010c770       ??__FarrDstPositions@?FD@??DrawAttachment@CAttachmentSKIN@@UAEXAAUSRendParams@@ABUSRenderingPassInfo@@ABU?$Matrix34_tpl@M@@M@Z@YAXXZ 3160d770 f   _RenderSkins.obj
 0001:0010c7a0       ??__Fg_arrDecalFaceMapping@@YAXXZ 3160d7a0 f   DecalManager.obj
 0001:0010c7d0       ??__Fg_arrVerticesBS@@YAXXZ 3160d7d0 f   DecalManager.obj
 0001:0010c800       ??__Fg_arrDecalVertexMapping@@YAXXZ 3160d800 f   DecalManager.obj
 0001:0010c830       ??__F?s_factory@CFactory@CFeetPoseStore@@0V12@A@@YAXXZ 3160d830 f   FeetLock.obj
 0001:0010c840       ??__F?s_factory@CFactory@CFeetPoseRestore@@0V12@A@@YAXXZ 3160d840 f   FeetLock.obj
 0001:0010c850       ??__F?s_factory@CFactory@CGroundAlignment@@0V12@A@@YAXXZ 3160d850 f   GroundAlignment.obj
 0001:0010c860       ??__F?s_factory@CFactory@CLimbIk@@0V12@A@@YAXXZ 3160d860 f   LimbIk.obj
 0001:0010c870       ??__F?s_factory@CFactory@CPoseBlenderAim@@0V12@A@@YAXXZ 3160d870 f   PoseBlenderAim.obj
 0001:0010c880       ??__F?s_factory@CFactory@CPoseBlenderLook@@0V12@A@@YAXXZ 3160d880 f   PoseBlenderLook.obj
 0001:0010c890       ??__F?s_factory@CFactory@CRecoil@PoseModifier@@0V123@A@@YAXXZ 3160d890 f   Recoil.obj
 0001:0010c8a0       ??__FCrySessionInvalidID@@YAXXZ 3160d8a0 f   CharacterManager.obj
 0001:0010c8e0       ??__FCryUserInvalidID@@YAXXZ 3160d8e0 f   CharacterManager.obj
 0001:0010c920       ??__Fg_controllerHeap@@YAXXZ 3160d920 f   AnimationBase.obj
 0001:0010c930       ??__F?s_factory@CFactory@CEngineModule_CryAnimation@@0V12@A@@YAXXZ 3160d930 f   AnimationBase.obj
 0001:0010c950       ??__Fg_DefaultAnim@@YAXXZ  3160d950 f   AnimationBase.obj
 0001:0010c960       ??__Fg_system_event_listener_anim@@YAXXZ 3160d960 f   AnimationBase.obj
 0001:0010c9b0       ??__Fg_DataMismatch@@YAXXZ 3160d9b0 f   AnimationBase.obj
 0001:0010ca00       ??__Fg_Consoleself@@YAXXZ  3160da00 f   cvars.obj
 0001:0010ca30       ??__FautoInitializer@@YAXXZ 3160da30 f   stdafx.obj
